 mysqlmanager

 Timestamp is 4f50de9c (Fri Mar 02 15:52:12 2012)

 Preferred load address is 0000000140000000

 Start         Length     Name                   Class
 0001:00000000 000e42b3H .text                   CODE
 0001:000e42c0 00001026H .text$0                 CODE
 0001:000e52f0 000010a0H .text$00                CODE
 0001:000e6390 00001020H .text$yd                CODE
 0002:00000000 00000109H .CRT$XCA                DATA
 0002:00000110 00000109H .CRT$XCZ                DATA
 0002:00000220 00000109H .CRT$XIA                DATA
 0002:00000330 0000011cH .CRT$XIC                DATA
 0002:00000450 00000109H .CRT$XIY                DATA
 0002:00000560 00000109H .CRT$XIZ                DATA
 0002:00000670 00000008H .CRT$XLA                DATA
 0002:00000678 00000008H .CRT$XLZ                DATA
 0002:00000680 00000109H .CRT$XPA                DATA
 0002:00000790 00000109H .CRT$XPX                DATA
 0002:000008a0 00000109H .CRT$XPXA               DATA
 0002:000009b0 00000109H .CRT$XPZ                DATA
 0002:00000ac0 00000109H .CRT$XTA                DATA
 0002:00000bd0 00000109H .CRT$XTZ                DATA
 0002:00000ce0 0001732aH .rdata                  DATA
 0002:00018010 00000130H .rdata$T                DATA
 0002:00018140 000001abH .rdata$debug            DATA
 0002:000182f0 00003b15H .rdata$r                DATA
 0002:0001be08 00000109H .rtc$IAA                DATA
 0002:0001bf18 00000109H .rtc$IZZ                DATA
 0002:0001c028 00000109H .rtc$TAA                DATA
 0002:0001c138 00000109H .rtc$TZZ                DATA
 0002:0001c248 00010ba9H .xdata                  DATA
 0002:0002cdf8 0000019eH .xdata$x                DATA
 0002:0002cf96 00000000H .edata                  DATA
 0003:00000000 00136481H .data                   DATA
 0003:001364a0 00005364H .bss                    DATA
 0004:00000000 0000af80H .pdata                  DATA
 0005:00000000 00000050H .idata$2                DATA
 0005:00000050 00000014H .idata$3                DATA
 0005:00000068 000007e0H .idata$4                DATA
 0005:00000848 000007e0H .idata$5                DATA
 0005:00001028 00000d4eH .idata$6                DATA
 0006:00000000 00000101H .tls                    DATA
 0006:00000110 000001e6H .tls$                   DATA
 0006:000002f6 00000101H .tls$ZZZ                DATA

  Address         Publics by Value              Rva+Base               Lib:Object

 0000:00000000       ___safe_se_handler_table   0000000000000000     <absolute>
 0000:00000000       ___safe_se_handler_count   0000000000000000     <absolute>
 0000:00000000       __ImageBase                0000000140000000     <linker-defined>
 0001:00000b80       ?reserve@Buffer@@QEAAHII@Z 0000000140001b80 f   buffer.obj
 0001:00000c60       ?get_size@Buffer@@QEAAHXZ  0000000140001c60 f   buffer.obj
 0001:00000c70       ?is_error@Buffer@@QEAAHXZ  0000000140001c70 f   buffer.obj
 0001:00000c80       ?append@Buffer@@QEAAHIPEBDI@Z 0000000140001c80 f   buffer.obj
 0001:00000d00       ??0Command@@QEAA@PEAVInstance_map@@@Z 0000000140001d00 f   command.obj
 0001:00000d20       ??1Command@@UEAA@XZ        0000000140001d20 f   command.obj
 0001:00000d30       ??_ECommand@@UEAAPEAXI@Z   0000000140001d30 f i command.obj
 0001:00000d30       ??_GCommand@@UEAAPEAXI@Z   0000000140001d30 f i command.obj
 0001:00000d60       ?strchr@@YAPEADPEADH@Z     0000000140001d60 f i commands.obj
 0001:00000d70       ??0Buffer@@QEAA@_K@Z       0000000140001d70 f i commands.obj
 0001:00000dc0       ??1Buffer@@QEAA@XZ         0000000140001dc0 f i commands.obj
 0001:00000dd0       ??0Iterator@Instance_map@@QEAA@PEAV1@@Z 0000000140001dd0 f i commands.obj
 0001:00000e00       ?execute@Show_instances@@UEAAHPEAUst_net@@K@Z 0000000140001e00 f   commands.obj
 0001:00001020       ?execute@Flush_instances@@UEAAHPEAUst_net@@K@Z 0000000140002020 f   commands.obj
 0001:00001080       ??0Show_instance_status@@QEAA@PEAVInstance_map@@PEBDI@Z 0000000140002080 f   commands.obj
 0001:00001120       ??1Show_instance_status@@UEAA@XZ 0000000140002120 f i commands.obj
 0001:00001130       ?execute@Show_instance_status@@UEAAHPEAUst_net@@K@Z 0000000140002130 f   commands.obj
 0001:000013b0       ??0Show_instance_options@@QEAA@PEAVInstance_map@@PEBDI@Z 00000001400023b0 f   commands.obj
 0001:00001450       ??1Show_instance_options@@UEAA@XZ 0000000140002450 f i commands.obj
 0001:00001460       ?execute@Show_instance_options@@UEAAHPEAUst_net@@K@Z 0000000140002460 f   commands.obj
 0001:000018d0       ??0Start_instance@@QEAA@PEAVInstance_map@@PEBDI@Z 00000001400028d0 f   commands.obj
 0001:00001950       ??1Start_instance@@UEAA@XZ 0000000140002950 f i commands.obj
 0001:00001960       ?execute@Start_instance@@UEAAHPEAUst_net@@K@Z 0000000140002960 f   commands.obj
 0001:00001a00       ??0Show_instance_log@@QEAA@PEAVInstance_map@@PEBDIW4Log_type@@11@Z 0000000140002a00 f   commands.obj
 0001:00001ad0       ??1Show_instance_log@@UEAA@XZ 0000000140002ad0 f i commands.obj
 0001:00001ae0       ?execute@Show_instance_log@@UEAAHPEAUst_net@@K@Z 0000000140002ae0 f   commands.obj
 0001:00001e40       ??0Show_instance_log_files@@QEAA@PEAVInstance_map@@PEBDI@Z 0000000140002e40 f   commands.obj
 0001:00001ee0       ??1Show_instance_log_files@@UEAA@XZ 0000000140002ee0 f i commands.obj
 0001:00001ef0       ?execute@Show_instance_log_files@@UEAAHPEAUst_net@@K@Z 0000000140002ef0 f   commands.obj
 0001:00002280       ??0Set_option@@QEAA@PEAVInstance_map@@PEBDI1I1I@Z 0000000140003280 f   commands.obj
 0001:00002390       ??1Set_option@@UEAA@XZ     0000000140003390 f i commands.obj
 0001:000023a0       ??_ESet_option@@UEAAPEAXI@Z 00000001400033a0 f i commands.obj
 0001:000023a0       ??_GSet_option@@UEAAPEAXI@Z 00000001400033a0 f i commands.obj
 0001:000023e0       ?correct_file@Set_option@@IEAAHH@Z 00000001400033e0 f   commands.obj
 0001:00002430       ?do_command@Set_option@@UEAAHPEAUst_net@@@Z 0000000140003430 f   commands.obj
 0001:00002480       ?execute@Set_option@@UEAAHPEAUst_net@@K@Z 0000000140003480 f   commands.obj
 0001:000024f0       ?do_command@Unset_option@@UEAAHPEAUst_net@@@Z 00000001400034f0 f   commands.obj
 0001:00002500       ??0Stop_instance@@QEAA@PEAVInstance_map@@PEBDI@Z 0000000140003500 f   commands.obj
 0001:00002580       ??1Stop_instance@@UEAA@XZ  0000000140003580 f i commands.obj
 0001:00002590       ?execute@Stop_instance@@UEAAHPEAUst_net@@K@Z 0000000140003590 f   commands.obj
 0001:00002630       ?execute@Syntax_error@@UEAAHPEAUst_net@@K@Z 0000000140003630 f   commands.obj
 0001:00002640       ??_EShow_instance_status@@UEAAPEAXI@Z 0000000140003640 f i commands.obj
 0001:00002640       ??_GShow_instance_status@@UEAAPEAXI@Z 0000000140003640 f i commands.obj
 0001:00002680       ??_EShow_instance_options@@UEAAPEAXI@Z 0000000140003680 f i commands.obj
 0001:00002680       ??_GShow_instance_options@@UEAAPEAXI@Z 0000000140003680 f i commands.obj
 0001:000026c0       ??_EStart_instance@@UEAAPEAXI@Z 00000001400036c0 f i commands.obj
 0001:000026c0       ??_GStart_instance@@UEAAPEAXI@Z 00000001400036c0 f i commands.obj
 0001:00002700       ??_GShow_instance_log@@UEAAPEAXI@Z 0000000140003700 f i commands.obj
 0001:00002700       ??_EShow_instance_log@@UEAAPEAXI@Z 0000000140003700 f i commands.obj
 0001:00002740       ??_GShow_instance_log_files@@UEAAPEAXI@Z 0000000140003740 f i commands.obj
 0001:00002740       ??_EShow_instance_log_files@@UEAAPEAXI@Z 0000000140003740 f i commands.obj
 0001:00002780       ??_GStop_instance@@UEAAPEAXI@Z 0000000140003780 f i commands.obj
 0001:00002780       ??_EStop_instance@@UEAAPEAXI@Z 0000000140003780 f i commands.obj
 0001:000027d0       ??0Guardian_thread_args@@QEAA@AEAVThread_registry@@PEAVInstance_map@@I@Z 00000001400037d0 f i guardian.obj
 0001:000027f0       ??0Guardian_thread@@QEAA@AEAVThread_registry@@PEAVInstance_map@@I@Z 00000001400037f0 f   guardian.obj
 0001:00002890       ??1Guardian_thread@@QEAA@XZ 0000000140003890 f   guardian.obj
 0001:000028f0       ?process_instance@Guardian_thread@@AEAAXPEAVInstance@@PEAUGUARD_NODE@1@PEAPEAUst_list@@PEAU4@@Z 00000001400038f0 f   guardian.obj
 0001:00002b60       ?run@Guardian_thread@@QEAAXXZ 0000000140003b60 f   guardian.obj
 0001:00002d00       ?is_stopped@Guardian_thread@@QEAAHXZ 0000000140003d00 f   guardian.obj
 0001:00002d40       ?guard@Guardian_thread@@QEAAHPEAVInstance@@_N@Z 0000000140003d40 f   guardian.obj
 0001:00002e50       ?stop_guard@Guardian_thread@@QEAAHPEAVInstance@@@Z 0000000140003e50 f   guardian.obj
 0001:00002ee0       ?stop_instances@Guardian_thread@@AEAAHXZ 0000000140003ee0 f   guardian.obj
 0001:00002f90       ?lock@Guardian_thread@@QEAAXXZ 0000000140003f90 f   guardian.obj
 0001:00002fa0       ?unlock@Guardian_thread@@QEAAXXZ 0000000140003fa0 f   guardian.obj
 0001:00002fb0       guardian                   0000000140003fb0 f   guardian.obj
 0001:00002fd0       ?request_shutdown@Guardian_thread@@QEAAXXZ 0000000140003fd0 f   guardian.obj
 0001:00003020       ?init@Guardian_thread@@QEAAHXZ 0000000140004020 f   guardian.obj
 0001:00003100       ??0Instance_options@@QEAA@XZ 0000000140004100 f i instance.obj
 0001:000033f0       ?get_map@Instance@@QEAAPEAVInstance_map@@XZ 00000001400043f0 f   instance.obj
 0001:00003400       ?remove_pid@Instance@@AEAAXXZ 0000000140004400 f   instance.obj
 0001:00003450       ?set_crash_flag_n_wake_all@Instance@@QEAAXXZ 0000000140004450 f   instance.obj
 0001:000034d0       ??0Instance@@QEAA@XZ       00000001400044d0 f   instance.obj
 0001:00003580       ??1Instance@@QEAA@XZ       0000000140004580 f   instance.obj
 0001:000035c0       ?is_crashed@Instance@@QEAAHXZ 00000001400045c0 f   instance.obj
 0001:00003610       ?is_running@Instance@@QEAA_NXZ 0000000140004610 f   instance.obj
 0001:000037b0       ?SafeTerminateProcess@@YAHPEAXI@Z 00000001400047b0 f   instance.obj
 0001:00003950       ?kill@@YAHHH@Z             0000000140004950 f   instance.obj
 0001:000039a0       ?kill_instance@Instance@@QEAAXH@Z 00000001400049a0 f   instance.obj
 0001:00003a10       ?init@Instance@@QEAAHPEBD@Z 0000000140004a10 f   instance.obj
 0001:00003a20       ?complete_initialization@Instance@@QEAAHPEAVInstance_map@@PEBDI@Z 0000000140004a20 f   instance.obj
 0001:00003b40       ?stop@Instance@@QEAAHXZ    0000000140004b40 f   instance.obj
 0001:00003c60       proxy                      0000000140004c60 f   instance.obj
 0001:00003c80       ?start@Instance@@QEAAHXZ   0000000140004c80 f   instance.obj
 0001:00003d90       ??_GInstance@@QEAAPEAXI@Z  0000000140004d90 f i instance_map.obj
 0001:00003dd0       ?process_one_option@Instance_map@@QEAAHPEBD0@Z 0000000140004dd0 f   instance_map.obj
 0001:00003f10       ??0Instance_map@@QEAA@PEBD@Z 0000000140004f10 f   instance_map.obj
 0001:00003f40       ??1Instance_map@@QEAA@XZ   0000000140004f40 f   instance_map.obj
 0001:00003f90       ?lock@Instance_map@@QEAAXXZ 0000000140004f90 f   instance_map.obj
 0001:00003fa0       ?unlock@Instance_map@@QEAAXXZ 0000000140004fa0 f   instance_map.obj
 0001:00003fb0       ?find@Instance_map@@QEAAPEAVInstance@@PEBDI@Z 0000000140004fb0 f   instance_map.obj
 0001:00004030       ?complete_initialization@Instance_map@@AEAAHXZ 0000000140005030 f   instance_map.obj
 0001:00004160       ?go_to_first@Iterator@Instance_map@@QEAAXXZ 0000000140005160 f   instance_map.obj
 0001:00004170       ?next@Iterator@Instance_map@@QEAAPEAVInstance@@XZ 0000000140005170 f   instance_map.obj
 0001:000041e0       ?init@Instance_map@@QEAAHXZ 00000001400051e0 f   instance_map.obj
 0001:00004240       ?load@Instance_map@@AEAAHXZ 0000000140005240 f   instance_map.obj
 0001:00004380       ?flush_instances@Instance_map@@QEAAHXZ 0000000140005380 f   instance_map.obj
 0001:00004450       ?strstr@@YAPEADPEADPEBD@Z  0000000140005450 f i instance_options.obj
 0001:00004530       ?get_default_option@Instance_options@@AEAAHPEAD_KPEBD@Z 0000000140005530 f   instance_options.obj
 0001:000046e0       ?fill_instance_version@Instance_options@@AEAAHXZ 00000001400056e0 f   instance_options.obj
 0001:00004930       ?fill_mysqld_real_path@Instance_options@@AEAAHXZ 0000000140005930 f   instance_options.obj
 0001:00004b70       ?fill_log_options@Instance_options@@AEAAHXZ 0000000140005b70 f   instance_options.obj
 0001:00004fa0       ?get_pid_filename@Instance_options@@QEAAHPEAD@Z 0000000140005fa0 f   instance_options.obj
 0001:000050a0       ?unlink_pidfile@Instance_options@@QEAAHXZ 00000001400060a0 f   instance_options.obj
 0001:000050b0       ?get_pid@Instance_options@@QEAAHXZ 00000001400060b0 f   instance_options.obj
 0001:00005130       ?add_option@Instance_options@@QEAAHPEBD@Z 0000000140006130 f   instance_options.obj
 0001:00005450       ?add_to_argv@Instance_options@@AEAAHPEBD@Z 0000000140006450 f   instance_options.obj
 0001:00005480       ?print_argv@Instance_options@@QEAAXXZ 0000000140006480 f   instance_options.obj
 0001:00005500       ?init@Instance_options@@QEAAHPEBD@Z 0000000140006500 f   instance_options.obj
 0001:000055d0       ??1Instance_options@@QEAA@XZ 00000001400065d0 f   instance_options.obj
 0001:00005610       ?complete_initialization@Instance_options@@QEAAHPEBDI@Z 0000000140006610 f   instance_options.obj
 0001:00005960       ??0Listener_thread_args@@QEAA@AEAVThread_registry@@AEBUOptions@@AEBVUser_map@@AEAVInstance_map@@@Z 0000000140006960 f i listener.obj
 0001:00005980       ?is_shutdown@Thread_registry@@QEAA_NXZ 0000000140006980 f i listener.obj
 0001:00005a10       ??0Listener_thread@@QEAA@AEBUListener_thread_args@@@Z 0000000140006a10 f   listener.obj
 0001:00005a80       ??1Listener_thread@@QEAA@XZ 0000000140006a80 f   listener.obj
 0001:00005a90       ?create_tcp_socket@Listener_thread@@AEAAHXZ 0000000140006a90 f   listener.obj
 0001:00005c90       ?handle_new_mysql_connection@Listener_thread@@AEAAXPEAUst_vio@@@Z 0000000140006c90 f   listener.obj
 0001:00005d90       ?run@Listener_thread@@QEAAXXZ 0000000140006d90 f   listener.obj
 0001:000060a0       listener                   00000001400070a0 f   listener.obj
 0001:00006370       ?log_error@@YAXPEBDZZ      0000000140007370 f   log.obj
 0001:000063c0       ?log_info@@YAXPEBDZZ       00000001400073c0 f   log.obj
 0001:00006410       ?print_info@@YAXPEBDZZ     0000000140007410 f   log.obj
 0001:00006460       ?print_error@@YAXPEBDZZ    0000000140007460 f   log.obj
 0001:000064b0       ?log_init@@YAXXZ           00000001400074b0 f   log.obj
 0001:000064d0       ?die@@YAXPEBDZZ            00000001400074d0 f   log.obj
 0001:00006560       ??0User_map@@QEAA@XZ       0000000140007560 f i manager.obj
 0001:00006570       ?create_pid_file@@YAHPEBDH@Z 0000000140007570 f   manager.obj
 0001:00006630       ?onsignal@@YAXH@Z          0000000140007630 f   manager.obj
 0001:00006640       ?set_signals@@YAXPEAH@Z    0000000140007640 f   manager.obj
 0001:00006680       ?my_sigwait@@YAHPEBHPEAH@Z 0000000140007680 f   manager.obj
 0001:000066c0       ?stop_all@@YAXPEAVGuardian_thread@@PEAVThread_registry@@@Z 00000001400076c0 f   manager.obj
 0001:00006710       ?manager@@YAHAEBUOptions@@@Z 0000000140007710 f   manager.obj
 0001:00006d30       ?message@@YAPEBDI@Z        0000000140007d30 f   messages.obj
 0001:00006d40       ?errno_to_sqlstate@@YAPEBDI@Z 0000000140007d40 f   messages.obj
 0001:00006d60       ??0Mysql_connection_thread_args@@QEAA@PEAUst_vio@@AEAVThread_registry@@AEBVUser_map@@KAEAVInstance_map@@@Z 0000000140007d60 f   mysql_connection.obj
 0001:00006d90       ??0Mysql_connection_thread@@QEAA@AEBUMysql_connection_thread_args@@@Z 0000000140007d90 f   mysql_connection.obj
 0001:00006e10       my_net_local_init          0000000140007e10 f   mysql_connection.obj
 0001:00006e70       slave_io_thread_detach_vio 0000000140007e70 f   mysql_connection.obj
 0001:00006e80       ?init@Mysql_connection_thread@@QEAAHXZ 0000000140007e80 f   mysql_connection.obj
 0001:00006f50       ?cleanup@Mysql_connection_thread@@QEAAXXZ 0000000140007f50 f   mysql_connection.obj
 0001:00006f60       ??1Mysql_connection_thread@@QEAA@XZ 0000000140007f60 f   mysql_connection.obj
 0001:00006f90       ?check_connection@Mysql_connection_thread@@AEAAHXZ 0000000140007f90 f   mysql_connection.obj
 0001:00007230       ?dispatch_command@Mysql_connection_thread@@AEAAHW4enum_server_command@@PEBDI@Z 0000000140008230 f   mysql_connection.obj
 0001:000073c0       ?do_command@Mysql_connection_thread@@AEAAHXZ 00000001400083c0 f   mysql_connection.obj
 0001:000074f0       ?run@Mysql_connection_thread@@QEAAXXZ 00000001400084f0 f   mysql_connection.obj
 0001:000075d0       mysql_connection           00000001400085d0 f   mysql_connection.obj
 0001:00007690       ??0Options@@QEAA@XZ        0000000140008690 f i mysqlmanager.obj
 0001:000076e0       main                       00000001400086e0 f   mysqlmanager.obj
 0001:00007780       ?strrchr@@YAPEADPEADH@Z    0000000140008780 f i options.obj
 0001:00007ac0       ?cleanup@Options@@QEAAXXZ  0000000140008ac0 f   options.obj
 0001:00007ae0       ?setup_windows_defaults@Options@@QEAAHXZ 0000000140008ae0 f   options.obj
 0001:00007be0       ?load@Options@@QEAAHHPEAPEAD@Z 0000000140008be0 f   options.obj
 0001:00007d20       ?get_word@@YAXPEAPEBDPEAIH@Z 0000000140008d20 f i parse.obj
 0001:00007e00       ??0Show_instances@@QEAA@PEAVInstance_map@@@Z 0000000140008e00 f i parse.obj
 0001:00007e30       ??1Show_instances@@UEAA@XZ 0000000140008e30 f i parse.obj
 0001:00007e40       ??0Flush_instances@@QEAA@PEAVInstance_map@@@Z 0000000140008e40 f i parse.obj
 0001:00007e70       ??1Flush_instances@@UEAA@XZ 0000000140008e70 f i parse.obj
 0001:00007e80       ??0Syntax_error@@QEAA@XZ   0000000140008e80 f i parse.obj
 0001:00007eb0       ??1Syntax_error@@UEAA@XZ   0000000140008eb0 f i parse.obj
 0001:00007ec0       ?find_token@@YA?AW4Token@@PEBDI@Z 0000000140008ec0 f i parse.obj
 0001:00007f70       ?get_token@@YA?AW4Token@@PEAPEBDPEAI@Z 0000000140008f70 f   parse.obj
 0001:000080b0       ?shift_token@@YA?AW4Token@@PEAPEBDPEAI@Z 00000001400090b0 f   parse.obj
 0001:000080e0       ?get_text_id@@YAHPEAPEBDPEAI0@Z 00000001400090e0 f   parse.obj
 0001:000081a0       ??_EShow_instances@@UEAAPEAXI@Z 00000001400091a0 f i parse.obj
 0001:000081a0       ??_GShow_instances@@UEAAPEAXI@Z 00000001400091a0 f i parse.obj
 0001:000081e0       ??_EFlush_instances@@UEAAPEAXI@Z 00000001400091e0 f i parse.obj
 0001:000081e0       ??_GFlush_instances@@UEAAPEAXI@Z 00000001400091e0 f i parse.obj
 0001:00008220       ??_ESyntax_error@@UEAAPEAXI@Z 0000000140009220 f i parse.obj
 0001:00008220       ??_GSyntax_error@@UEAAPEAXI@Z 0000000140009220 f i parse.obj
 0001:00008260       ??0Unset_option@@QEAA@PEAVInstance_map@@PEBDI1I1I@Z 0000000140009260 f i parse.obj
 0001:000082c0       ??1Unset_option@@UEAA@XZ   00000001400092c0 f i parse.obj
 0001:000082d0       ??_EUnset_option@@UEAAPEAXI@Z 00000001400092d0 f i parse.obj
 0001:000082d0       ??_GUnset_option@@UEAAPEAXI@Z 00000001400092d0 f i parse.obj
 0001:00008310       ?parse_command@@YAPEAVCommand@@PEAVInstance_map@@PEBD@Z 0000000140009310 f   parse.obj
 0001:00008f90       ?trim_space@@YAXPEAPEBDPEAI@Z 0000000140009f90 f   parse_output.obj
 0001:00009010       ?parse_output_and_get_value@@YAHPEBD0PEAD_KI@Z 000000014000a010 f   parse_output.obj
 0001:00009190       ?set_stacksize_n_create_thread@@YAHPEAPEAXPEAUthread_attr@@P6APEAXPEAX@Z2@Z 000000014000a190 f   priv.obj
 0001:000091a0       ?net_send_error@@YAHPEAUst_net@@I@Z 000000014000a1a0 f   protocol.obj
 0001:000092a0       ?net_send_error_323@@YAHPEAUst_net@@I@Z 000000014000a2a0 f   protocol.obj
 0001:00009370       ?net_store_length@@YAPEADPEADI@Z 000000014000a370 f   protocol.obj
 0001:000093a0       ?store_to_protocol_packet@@YAHPEAVBuffer@@PEBDPEAII@Z 000000014000a3a0 f   protocol.obj
 0001:00009450       ?store_to_protocol_packet@@YAHPEAVBuffer@@PEBDPEAI@Z 000000014000a450 f   protocol.obj
 0001:00009490       ?send_eof@@YAHPEAUst_net@@@Z 000000014000a490 f   protocol.obj
 0001:000094f0       ?send_fields@@YAHPEAUst_net@@PEAUst_list@@@Z 000000014000a4f0 f   protocol.obj
 0001:00009770       ?net_send_ok@@YAHPEAUst_net@@KPEBD@Z 000000014000a770 f   protocol.obj
 0001:000098d0       ??0Thread_info@@QEAA@XZ    000000014000a8d0 f   thread_registry.obj
 0001:000098e0       ??0Thread_info@@QEAA@PEAX@Z 000000014000a8e0 f   thread_registry.obj
 0001:000098f0       ??0Thread_registry@@QEAA@XZ 000000014000a8f0 f   thread_registry.obj
 0001:00009950       ??1Thread_registry@@QEAA@XZ 000000014000a950 f   thread_registry.obj
 0001:000099a0       ?register_thread@Thread_registry@@QEAAXPEAVThread_info@@@Z 000000014000a9a0 f   thread_registry.obj
 0001:00009a10       ?unregister_thread@Thread_registry@@QEAAXPEAVThread_info@@@Z 000000014000aa10 f   thread_registry.obj
 0001:00009a90       ?cond_wait@Thread_registry@@QEAAHPEAVThread_info@@PEAUpthread_cond_t@@PEAU_RTL_CRITICAL_SECTION@@@Z 000000014000aa90 f   thread_registry.obj
 0001:00009b50       ?cond_timedwait@Thread_registry@@QEAAHPEAVThread_info@@PEAUpthread_cond_t@@PEAU_RTL_CRITICAL_SECTION@@PEAUtimespec@@@Z 000000014000ab50 f   thread_registry.obj
 0001:00009c20       ?deliver_shutdown@Thread_registry@@QEAAXXZ 000000014000ac20 f   thread_registry.obj
 0001:00009d60       ?request_shutdown@Thread_registry@@QEAAXXZ 000000014000ad60 f   thread_registry.obj
 0001:00009d80       ?get_error_status@Thread_registry@@QEAAHXZ 000000014000ad80 f   thread_registry.obj
 0001:00009dd0       ?set_error_status@Thread_registry@@QEAAXXZ 000000014000add0 f   thread_registry.obj
 0001:00009e10       ??0User@@QEAA@XZ           000000014000ae10 f i user_map.obj
 0001:00009e20       ?init@User@@QEAAHPEBD@Z    000000014000ae20 f   user_map.obj
 0001:00009fa0       ?init@User_map@@QEAAHXZ    000000014000afa0 f   user_map.obj
 0001:0000a000       ??1User_map@@QEAA@XZ       000000014000b000 f   user_map.obj
 0001:0000a010       ?load@User_map@@QEAAHPEBD@Z 000000014000b010 f   user_map.obj
 0001:0000a1a0       ?authenticate@User_map@@QEBAHPEBDI00@Z 000000014000b1a0 f   user_map.obj
 0001:0000a1f0       ??0IMService@@QEAA@XZ      000000014000b1f0 f   IMService.obj
 0001:0000a250       ?Shutdown@WindowsService@@MEAAXXZ 000000014000b250 f i IMService.obj
 0001:0000a260       ?Pause@WindowsService@@MEAAXXZ 000000014000b260 f i IMService.obj
 0001:0000a270       ?Continue@WindowsService@@MEAAXXZ 000000014000b270 f i IMService.obj
 0001:0000a280       ??1IMService@@QEAA@XZ      000000014000b280 f   IMService.obj
 0001:0000a2a0       ?Stop@IMService@@MEAAXXZ   000000014000b2a0 f   IMService.obj
 0001:0000a2d0       ?Run@IMService@@MEAAXKPEAPEAD@Z 000000014000b2d0 f   IMService.obj
 0001:0000a360       ?Log@IMService@@MEAAXPEBD@Z 000000014000b360 f   IMService.obj
 0001:0000a370       ?HandleServiceOptions@@YAHUOptions@@@Z 000000014000b370 f   IMService.obj
 0001:0000a480       ??0WindowsService@@QEAA@XZ 000000014000b480 f   WindowsService.obj
 0001:0000a4d0       ?Stop@WindowsService@@MEAAXXZ 000000014000b4d0 f i WindowsService.obj
 0001:0000a4e0       ?Log@WindowsService@@MEAAXPEBD@Z 000000014000b4e0 f i WindowsService.obj
 0001:0000a4f0       ??1WindowsService@@QEAA@XZ 000000014000b4f0 f   WindowsService.obj
 0001:0000a500       ?IsInstalled@WindowsService@@QEAAHXZ 000000014000b500 f   WindowsService.obj
 0001:0000a570       ?SetAcceptedControls@WindowsService@@QEAAXK@Z 000000014000b570 f   WindowsService.obj
 0001:0000a580       ?ReportStatus@WindowsService@@IEAAHKKK@Z 000000014000b580 f   WindowsService.obj
 0001:0000a650       ?HandleControlCode@WindowsService@@IEAAXK@Z 000000014000b650 f   WindowsService.obj
 0001:0000a6e0       ?ControlHandler@WindowsService@@SAXK@Z 000000014000b6e0 f   WindowsService.obj
 0001:0000a700       ?Install@WindowsService@@QEAAHXZ 000000014000b700 f   WindowsService.obj
 0001:0000a850       ?Remove@WindowsService@@QEAAHXZ 000000014000b850 f   WindowsService.obj
 0001:0000a930       ?RegisterAndRun@WindowsService@@IEAAXKPEAPEAD@Z 000000014000b930 f   WindowsService.obj
 0001:0000a9d0       ?ServiceMain@WindowsService@@SAXKPEAPEAD@Z 000000014000b9d0 f   WindowsService.obj
 0001:0000a9f0       ?Init@WindowsService@@QEAAHXZ 000000014000b9f0 f   WindowsService.obj
 0001:0000aa50       my_net_init                000000014000ba50 f   net_serv.obj
 0001:0000ab50       net_end                    000000014000bb50 f   net_serv.obj
 0001:0000ab80       net_realloc                000000014000bb80 f   net_serv.obj
 0001:0000ad00       net_clear                  000000014000bd00 f   net_serv.obj
 0001:0000ad80       net_real_write             000000014000bd80 f   net_serv.obj
 0001:0000b290       my_net_read                000000014000c290 f   net_serv.obj
 0001:0000b520       my_net_set_read_timeout    000000014000c520 f   net_serv.obj
 0001:0000b550       my_net_set_write_timeout   000000014000c550 f   net_serv.obj
 0001:0000b580       net_flush                  000000014000c580 f   net_serv.obj
 0001:0000b730       my_net_write               000000014000c730 f   net_serv.obj
 0001:0000b890       net_write_command          000000014000c890 f   net_serv.obj
 0001:0000ba60       net_field_length           000000014000ca60 f   pack.obj
 0001:0000bad0       net_field_length_ll        000000014000cad0 f   pack.obj
 0001:0000bb50       net_store_length           000000014000cb50 f   pack.obj
 0001:0000bbc0       randominit                 000000014000cbc0 f   password.obj
 0001:0000bc40       my_rnd                     000000014000cc40 f   password.obj
 0001:0000bc80       hash_password              000000014000cc80 f   password.obj
 0001:0000bd30       my_make_scrambled_password_323 000000014000cd30 f   password.obj
 0001:0000bd70       make_scrambled_password_323 000000014000cd70 f   password.obj
 0001:0000bdb0       scramble_323               000000014000cdb0 f   password.obj
 0001:0000bf50       check_scramble_323         000000014000cf50 f   password.obj
 0001:0000c100       get_salt_from_password_323 000000014000d100 f   password.obj
 0001:0000c1a0       make_password_from_salt_323 000000014000d1a0 f   password.obj
 0001:0000c1c0       create_random_string       000000014000d1c0 f   password.obj
 0001:0000c250       octet2hex                  000000014000d250 f   password.obj
 0001:0000c3a0       my_make_scrambled_password 000000014000d3a0 f   password.obj
 0001:0000c480       make_scrambled_password    000000014000d480 f   password.obj
 0001:0000c4c0       scramble                   000000014000d4c0 f   password.obj
 0001:0000c620       check_scramble             000000014000d620 f   password.obj
 0001:0000c750       get_salt_from_password     000000014000d750 f   password.obj
 0001:0000c770       make_password_from_salt    000000014000d770 f   password.obj
 0001:0000c790       mysql_errno_to_sqlstate    000000014000d790 f   sql_state.obj
 0001:0000c7f0       my_connect                 000000014000d7f0 f   client.obj
 0001:0000c800       create_named_pipe          000000014000d800 f   client.obj
 0001:0000ca60       free_rows                  000000014000da60 f   client.obj
 0001:0000caa0       free_old_query             000000014000daa0 f   client.obj
 0001:0000cb10       set_mysql_error            000000014000db10 f   client.obj
 0001:0000cc70       end_server                 000000014000dc70 f   client.obj
 0001:0000cce0       mysql_free_result          000000014000dce0 f   client.obj
 0001:0000ce70       mysql_read_default_options 000000014000de70 f   client.obj
 0001:0000d4b0       unpack_fields              000000014000e4b0 f   client.obj
 0001:0000d9a0       mysql_init                 000000014000e9a0 f   client.obj
 0001:0000da90       mysql_ssl_set              000000014000ea90 f   client.obj
 0001:0000dc80       mysql_get_ssl_cipher       000000014000ec80 f   client.obj
 0001:0000dde0       mysql_init_character_set   000000014000ede0 f   client.obj
 0001:0000e100       mysql_select_db            000000014000f100 f   client.obj
 0001:0000e380       mysql_detach_stmt_list     000000014000f380 f   client.obj
 0001:0000e390       mysql_close                000000014000f390 f   client.obj
 0001:0000e4a0       mysql_send_query           000000014000f4a0 f   client.obj
 0001:0000e4f0       mysql_real_query           000000014000f4f0 f   client.obj
 0001:0000e530       mysql_store_result         000000014000f530 f   client.obj
 0001:0000e8a0       mysql_fetch_lengths        000000014000f8a0 f   client.obj
 0001:0000e8f0       mysql_options              000000014000f8f0 f   client.obj
 0001:0000ec90       mysql_num_rows             000000014000fc90 f   client.obj
 0001:0000eca0       mysql_num_fields           000000014000fca0 f   client.obj
 0001:0000ecb0       mysql_errno                000000014000fcb0 f   client.obj
 0001:0000ecd0       mysql_error                000000014000fcd0 f   client.obj
 0001:0000ecf0       mysql_get_server_version   000000014000fcf0 f   client.obj
 0001:0000ed80       mysql_set_character_set    000000014000fd80 f   client.obj
 0001:0000ef50       cli_safe_read              000000014000ff50 f   client.obj
 0001:0000f130       cli_read_rows              0000000140010130 f   client.obj
 0001:0000f630       mysql_real_connect         0000000140010630 f   client.obj
 0001:00010870       mysql_reconnect            0000000140011870 f   client.obj
 0001:00010e10       mysql_fetch_row            0000000140011e10 f   client.obj
 0001:00010f20       cli_advanced_command       0000000140011f20 f   client.obj
 0001:000111d0       get_tty_password           00000001400121d0 f   get_password.obj
 0001:00011320       init_client_errs           0000000140012320 f   errmsg.obj
 0001:00011340       finish_client_errs         0000000140012340 f   errmsg.obj
 0001:00011350       InitializeCriticalSection  0000000140012350 f   kernel32:KERNEL32.dll
 0001:00011356       DeleteCriticalSection      0000000140012356 f   kernel32:KERNEL32.dll
 0001:0001135c       LeaveCriticalSection       000000014001235c f   kernel32:KERNEL32.dll
 0001:00011362       EnterCriticalSection       0000000140012362 f   kernel32:KERNEL32.dll
 0001:00011368       GetSystemTimeAsFileTime    0000000140012368 f   kernel32:KERNEL32.dll
 0001:0001136e       CloseHandle                000000014001236e f   kernel32:KERNEL32.dll
 0001:00011374       GetExitCodeProcess         0000000140012374 f   kernel32:KERNEL32.dll
 0001:0001137a       WaitForSingleObject        000000014001237a f   kernel32:KERNEL32.dll
 0001:00011380       CreateProcessA             0000000140012380 f   kernel32:KERNEL32.dll
 0001:00011386       SetLastError               0000000140012386 f   kernel32:KERNEL32.dll
 0001:0001138c       GetLastError               000000014001238c f   kernel32:KERNEL32.dll
 0001:00011392       CreateRemoteThread         0000000140012392 f   kernel32:KERNEL32.dll
 0001:00011398       GetProcAddress             0000000140012398 f   kernel32:KERNEL32.dll
 0001:0001139e       DuplicateHandle            000000014001239e f   kernel32:KERNEL32.dll
 0001:000113a4       GetCurrentProcess          00000001400123a4 f   kernel32:KERNEL32.dll
 0001:000113aa       GetModuleHandleA           00000001400123aa f   kernel32:KERNEL32.dll
 0001:000113b0       TerminateProcess           00000001400123b0 f   kernel32:KERNEL32.dll
 0001:000113b6       OpenProcess                00000001400123b6 f   kernel32:KERNEL32.dll
 0001:000113bc       Sleep                      00000001400123bc f   kernel32:KERNEL32.dll
 0001:000113c2       GetCurrentThreadId         00000001400123c2 f   kernel32:KERNEL32.dll
 0001:000113c8       GetModuleFileNameA         00000001400123c8 f   kernel32:KERNEL32.dll
 0001:000113ce       SetNamedPipeHandleState    00000001400123ce f   kernel32:KERNEL32.dll
 0001:000113d4       WaitNamedPipeA             00000001400123d4 f   kernel32:KERNEL32.dll
 0001:000113da       CreateFileA                00000001400123da f   kernel32:KERNEL32.dll
 0001:000113e0       CloseServiceHandle         00000001400123e0 f   advapi32:ADVAPI32.dll
 0001:000113e6       OpenServiceA               00000001400123e6 f   advapi32:ADVAPI32.dll
 0001:000113ec       OpenSCManagerA             00000001400123ec f   advapi32:ADVAPI32.dll
 0001:000113f2       SetServiceStatus           00000001400123f2 f   advapi32:ADVAPI32.dll
 0001:000113f8       CreateServiceA             00000001400123f8 f   advapi32:ADVAPI32.dll
 0001:000113fe       DeleteService              00000001400123fe f   advapi32:ADVAPI32.dll
 0001:00011404       RegisterServiceCtrlHandlerA 0000000140012404 f   advapi32:ADVAPI32.dll
 0001:0001140a       StartServiceCtrlDispatcherA 000000014001240a f   advapi32:ADVAPI32.dll
 0001:00011410       my_realloc                 0000000140012410 f   mysys:my_realloc.obj
 0001:000114c0       my_malloc                  00000001400124c0 f   mysys:my_malloc.obj
 0001:00011580       my_no_flags_free           0000000140012580 f   mysys:my_malloc.obj
 0001:000115a0       my_memdup                  00000001400125a0 f   mysys:my_malloc.obj
 0001:000115f0       my_strdup                  00000001400125f0 f   mysys:my_malloc.obj
 0001:00011650       my_strdup_with_length      0000000140012650 f   mysys:my_malloc.obj
 0001:000116a0       list_add                   00000001400126a0 f   mysys:list.obj
 0001:000116e0       list_delete                00000001400126e0 f   mysys:list.obj
 0001:00011710       list_free                  0000000140012710 f   mysys:list.obj
 0001:00011770       list_cons                  0000000140012770 f   mysys:list.obj
 0001:000117c0       list_reverse               00000001400127c0 f   mysys:list.obj
 0001:000117f0       list_length                00000001400127f0 f   mysys:list.obj
 0001:00011810       list_walk                  0000000140012810 f   mysys:list.obj
 0001:00011860       init_dynamic_array         0000000140012860 f   mysys:array.obj
 0001:000118e0       alloc_dynamic              00000001400128e0 f   mysys:array.obj
 0001:00011940       pop_dynamic                0000000140012940 f   mysys:array.obj
 0001:00011960       set_dynamic                0000000140012960 f   mysys:array.obj
 0001:00011a20       get_dynamic                0000000140012a20 f   mysys:array.obj
 0001:00011a60       delete_dynamic             0000000140012a60 f   mysys:array.obj
 0001:00011a90       delete_dynamic_element     0000000140012a90 f   mysys:array.obj
 0001:00011ac0       freeze_size                0000000140012ac0 f   mysys:array.obj
 0001:00011b10       insert_dynamic             0000000140012b10 f   mysys:array.obj
 0001:00011b70       my_read                    0000000140012b70 f   mysys:my_read.obj
 0001:00011cd0       my_seek                    0000000140012cd0 f   mysys:my_seek.obj
 0001:00011d80       my_tell                    0000000140012d80 f   mysys:my_seek.obj
 0001:00011de0       my_dirend                  0000000140012de0 f   mysys:my_lib.obj
 0001:00011e50       my_dir                     0000000140012e50 f   mysys:my_lib.obj
 0001:00012120       my_fstat                   0000000140013120 f   mysys:my_lib.obj
 0001:00012130       my_stat                    0000000140013130 f   mysys:my_lib.obj
 0001:000121f0       my_close                   00000001400131f0 f   mysys:my_open.obj
 0001:000122e0       my_register_filename       00000001400132e0 f   mysys:my_open.obj
 0001:00012430       my_sopen                   0000000140013430 f   mysys:my_open.obj
 0001:000126b0       my_open                    00000001400136b0 f   mysys:my_open.obj
 0001:00012780       modify_defaults_file       0000000140013780 f   mysys:default_modify.obj
 0001:00012c10       init_alloc_root            0000000140013c10 f   mysys:my_alloc.obj
 0001:00012c90       reset_root_defaults        0000000140013c90 f   mysys:my_alloc.obj
 0001:00012d60       alloc_root                 0000000140013d60 f   mysys:my_alloc.obj
 0001:00012e70       multi_alloc_root           0000000140013e70 f   mysys:my_alloc.obj
 0001:00012f60       free_root                  0000000140013f60 f   mysys:my_alloc.obj
 0001:00013070       set_prealloc_root          0000000140014070 f   mysys:my_alloc.obj
 0001:000130c0       strmake_root               00000001400140c0 f   mysys:my_alloc.obj
 0001:00013110       memdup_root                0000000140014110 f   mysys:my_alloc.obj
 0001:00013160       strdup_root                0000000140014160 f   mysys:my_alloc.obj
 0001:000131a0       pthread_cond_init          00000001400141a0 f   mysys:my_wincond.obj
 0001:00013220       pthread_cond_destroy       0000000140014220 f   mysys:my_wincond.obj
 0001:00013270       pthread_cond_timedwait     0000000140014270 f   mysys:my_wincond.obj
 0001:00013380       pthread_cond_signal        0000000140014380 f   mysys:my_wincond.obj
 0001:000133c0       pthread_cond_broadcast     00000001400143c0 f   mysys:my_wincond.obj
 0001:00013410       pthread_attr_init          0000000140014410 f   mysys:my_wincond.obj
 0001:00013420       pthread_attr_setstacksize  0000000140014420 f   mysys:my_wincond.obj
 0001:00013430       pthread_attr_setprio       0000000140014430 f   mysys:my_wincond.obj
 0001:00013440       pthread_attr_destroy       0000000140014440 f   mysys:my_wincond.obj
 0001:00013450       localtime_r                0000000140014450 f   mysys:my_wincond.obj
 0001:00013500       pthread_cond_wait          0000000140014500 f   mysys:my_wincond.obj
 0001:00013510       my_thread_global_end       0000000140014510 f   mysys:my_thr_init.obj
 0001:00013660       my_thread_init             0000000140014660 f   mysys:my_thr_init.obj
 0001:00013700       my_thread_end              0000000140014700 f   mysys:my_thr_init.obj
 0001:00013780       _my_thread_var             0000000140014780 f   mysys:my_thr_init.obj
 0001:000137a0       my_thread_id               00000001400147a0 f   mysys:my_thr_init.obj
 0001:000137c0       my_thread_name             00000001400147c0 f   mysys:my_thr_init.obj
 0001:000137e0       my_thread_global_init      00000001400147e0 f   mysys:my_thr_init.obj
 0001:000138f0       win_pthread_init           00000001400148f0 f   mysys:my_winthread.obj
 0001:00013900       win_pthread_mutex_trylock  0000000140014900 f   mysys:my_winthread.obj
 0001:00013940       pthread_exit               0000000140014940 f   mysys:my_winthread.obj
 0001:00013950       win_pthread_setspecific    0000000140014950 f   mysys:my_winthread.obj
 0001:00013970       pthread_start              0000000140014970 f   mysys:my_winthread.obj
 0001:000139e0       pthread_create             00000001400149e0 f   mysys:my_winthread.obj
 0001:00013ac0       gmtime_r                   0000000140014ac0 f   mysys:my_pthread.obj
 0001:00013b40       pthread_no_free            0000000140014b40 f   mysys:my_pthread.obj
 0001:00013b50       pthread_dummy              0000000140014b50 f   mysys:my_pthread.obj
 0001:00013ba0       _hash_init                 0000000140014ba0 f   mysys:hash.obj
 0001:00013c70       hash_free                  0000000140014c70 f   mysys:hash.obj
 0001:00013ce0       my_hash_reset              0000000140014ce0 f   mysys:hash.obj
 0001:00013f30       my_hash_insert             0000000140014f30 f   mysys:hash.obj
 0001:00014210       hash_delete                0000000140015210 f   mysys:hash.obj
 0001:00014520       hash_update                0000000140015520 f   mysys:hash.obj
 0001:00014710       hash_element               0000000140015710 f   mysys:hash.obj
 0001:00014730       hash_replace               0000000140015730 f   mysys:hash.obj
 0001:00014750       hash_first                 0000000140015750 f   mysys:hash.obj
 0001:00014830       hash_next                  0000000140015830 f   mysys:hash.obj
 0001:000148e0       hash_search                00000001400158e0 f   mysys:hash.obj
 0001:00014900       my_charset_same            0000000140015900 f   mysys:charset.obj
 0001:000150e0       get_charsets_dir           00000001400160e0 f   mysys:charset.obj
 0001:000151a0       add_compiled_collation     00000001400161a0 f   mysys:charset.obj
 0001:000152f0       free_charsets              00000001400162f0 f   mysys:charset.obj
 0001:00015300       get_collation_number       0000000140016300 f   mysys:charset.obj
 0001:00015320       get_charset_number         0000000140016320 f   mysys:charset.obj
 0001:000153b0       get_charset_name           00000001400163b0 f   mysys:charset.obj
 0001:00015500       get_charset                0000000140016500 f   mysys:charset.obj
 0001:000155e0       get_charset_by_name        00000001400165e0 f   mysys:charset.obj
 0001:00015690       get_charset_by_csname      0000000140016690 f   mysys:charset.obj
 0001:00015740       escape_string_for_mysql    0000000140016740 f   mysys:charset.obj
 0001:00015950       fs_character_set           0000000140016950 f   mysys:charset.obj
 0001:00015a20       escape_quotes_for_mysql    0000000140016a20 f   mysys:charset.obj
 0001:00015b40       get_compatible_charset_with_ctype 0000000140016b40 f   mysys:charset.obj
 0001:00015c70       get_defaults_options       0000000140016c70 f   mysys:default.obj
 0001:00015d70       free_defaults              0000000140016d70 f   mysys:default.obj
 0001:00016990       my_print_default_files     0000000140017990 f   mysys:default.obj
 0001:00016b50       print_defaults             0000000140017b50 f   mysys:default.obj
 0001:00016cd0       my_search_option_files     0000000140017cd0 f   mysys:default.obj
 0001:00017010       load_defaults              0000000140018010 f   mysys:default.obj
 0001:00017390       strlength                  0000000140018390 f   mysys:mf_format.obj
 0001:000173f0       fn_format                  00000001400183f0 f   mysys:mf_format.obj
 0001:00017630       my_load_path               0000000140018630 f   mysys:mf_loadpath.obj
 0001:00017770       my_fclose                  0000000140018770 f   mysys:my_fopen.obj
 0001:000178c0       my_fopen                   00000001400188c0 f   mysys:my_fopen.obj
 0001:00017a40       my_fdopen                  0000000140018a40 f   mysys:my_fopen.obj
 0001:00017b40       dirname_length             0000000140018b40 f   mysys:mf_dirname.obj
 0001:00017ba0       convert_dirname            0000000140018ba0 f   mysys:mf_dirname.obj
 0001:00017cb0       dirname_part               0000000140018cb0 f   mysys:mf_dirname.obj
 0001:00017d00       my_delete                  0000000140018d00 f   mysys:my_delete.obj
 0001:00017d80       nt_share_delete            0000000140018d80 f   mysys:my_delete.obj
 0001:00017ee0       my_end                     0000000140018ee0 f   mysys:my_init.obj
 0001:00017f90       setEnvString               0000000140018f90 f   mysys:my_init.obj
 0001:00017fc0       my_parameter_handler       0000000140018fc0 f   mysys:my_init.obj
 0001:00018290       my_init                    0000000140019290 f   mysys:my_init.obj
 0001:00018400       my_getopt_register_get_addr 0000000140019400 f   mysys:my_getopt.obj
 0001:000184a0       getopt_compare_strings     00000001400194a0 f   mysys:my_getopt.obj
 0001:000186d0       getopt_ull_limit_value     00000001400196d0 f   mysys:my_getopt.obj
 0001:00018940       my_print_help              0000000140019940 f   mysys:my_getopt.obj
 0001:00018be0       my_print_variables         0000000140019be0 f   mysys:my_getopt.obj
 0001:000190b0       handle_options             000000014001a0b0 f   mysys:my_getopt.obj
 0001:00019b10       my_compress_alloc          000000014001ab10 f   mysys:my_compress.obj
 0001:00019bb0       my_uncompress              000000014001abb0 f   mysys:my_compress.obj
 0001:00019c40       my_compress                000000014001ac40 f   mysys:my_compress.obj
 0001:00019cb0       mysql_sha1_reset           000000014001acb0 f   mysys:sha1.obj
 0001:0001a350       mysql_sha1_result          000000014001b350 f   mysys:sha1.obj
 0001:0001a3f0       mysql_sha1_input           000000014001b3f0 f   mysys:sha1.obj
 0001:0001a460       find_type                  000000014001b460 f   mysys:typelib.obj
 0001:0001a5d0       get_type                   000000014001b5d0 f   mysys:typelib.obj
 0001:0001a5f0       copy_typelib               000000014001b5f0 f   mysys:typelib.obj
 0001:0001a730       make_type                  000000014001b730 f   mysys:typelib.obj
 0001:0001a760       my_error                   000000014001b760 f   mysys:my_error.obj
 0001:0001a830       my_printf_error            000000014001b830 f   mysys:my_error.obj
 0001:0001a8a0       my_message                 000000014001b8a0 f   mysys:my_error.obj
 0001:0001a8b0       my_error_register          000000014001b8b0 f   mysys:my_error.obj
 0001:0001a960       my_error_unregister        000000014001b960 f   mysys:my_error.obj
 0001:0001a9c0       my_multi_malloc            000000014001b9c0 f   mysys:mulalloc.obj
 0001:0001aa70       my_inet_ntoa               000000014001ba70 f   mysys:my_net.obj
 0001:0001aac0       my_gethostbyname_r         000000014001bac0 f   mysys:my_net.obj
 0001:0001ab00       my_gethostbyname_r_free    000000014001bb00 f   mysys:my_net.obj
 0001:0001ab10       thr_alarm_kill             000000014001bb10 f   mysys:thr_alarm.obj
 0001:0001ab20       process_alarm              000000014001bb20 f   mysys:thr_alarm.obj
 0001:0001ab30       thr_alarm                  000000014001bb30 f   mysys:thr_alarm.obj
 0001:0001ab80       thr_got_alarm              000000014001bb80 f   mysys:thr_alarm.obj
 0001:0001abf0       thr_end_alarm              000000014001bbf0 f   mysys:thr_alarm.obj
 0001:0001ac20       end_thr_alarm              000000014001bc20 f   mysys:thr_alarm.obj
 0001:0001ac30       init_thr_alarm             000000014001bc30 f   mysys:thr_alarm.obj
 0001:0001ac40       thr_alarm_info             000000014001bc40 f   mysys:thr_alarm.obj
 0001:0001ac50       resize_thr_alarm           000000014001bc50 f   mysys:thr_alarm.obj
 0001:0001ac60       my_filename                000000014001bc60 f   mysys:my_div.obj
 0001:0001aca0       my_qsort                   000000014001bca0 f   mysys:mf_qsort.obj
 0001:0001b500       my_access                  000000014001c500 f   mysys:my_access.obj
 0001:0001b550       check_if_legal_filename    000000014001c550 f   mysys:my_access.obj
 0001:0001b600       my_fread                   000000014001c600 f   mysys:my_fstream.obj
 0001:0001b700       my_fseek                   000000014001c700 f   mysys:my_fstream.obj
 0001:0001b730       my_ftell                   000000014001c730 f   mysys:my_fstream.obj
 0001:0001b740       my_fwrite                  000000014001c740 f   mysys:my_fstream.obj
 0001:0001b860       my_chsize                  000000014001c860 f   mysys:my_chsize.obj
 0001:0001b9d0       my_once_alloc              000000014001c9d0 f   mysys:my_once.obj
 0001:0001bab0       my_once_strdup             000000014001cab0 f   mysys:my_once.obj
 0001:0001bb00       my_once_memdup             000000014001cb00 f   mysys:my_once.obj
 0001:0001bb50       my_once_free               000000014001cb50 f   mysys:my_once.obj
 0001:0001bb90       my_getwd                   000000014001cb90 f   mysys:my_getwd.obj
 0001:0001bc50       test_if_hard_path          000000014001cc50 f   mysys:my_getwd.obj
 0001:0001bcc0       has_path                   000000014001ccc0 f   mysys:my_getwd.obj
 0001:0001bd10       my_setwd                   000000014001cd10 f   mysys:my_getwd.obj
 0001:0001bde0       init_compiled_charsets     000000014001cde0 f   mysys:charset-def.obj
 0001:0001c130       array_append_string_unique 000000014001d130 f   mysys:mf_arr_appstr.obj
 0001:0001c1c0       cleanup_dirname            000000014001d1c0 f   mysys:mf_pack.obj
 0001:0001c4d0       symdirget                  000000014001d4d0 f   mysys:mf_pack.obj
 0001:0001c650       system_filename            000000014001d650 f   mysys:mf_pack.obj
 0001:0001c670       intern_filename            000000014001d670 f   mysys:mf_pack.obj
 0001:0001c710       pack_dirname               000000014001d710 f   mysys:mf_pack.obj
 0001:0001c920       normalize_dirname          000000014001d920 f   mysys:mf_pack.obj
 0001:0001c9d0       unpack_dirname             000000014001d9d0 f   mysys:mf_pack.obj
 0001:0001cb00       unpack_filename            000000014001db00 f   mysys:mf_pack.obj
 0001:0001cbb0       fn_ext                     000000014001dbb0 f   mysys:mf_fn_ext.obj
 0001:0001cc20       my_readlink                000000014001dc20 f   mysys:my_symlink.obj
 0001:0001cc40       my_symlink                 000000014001dc40 f   mysys:my_symlink.obj
 0001:0001cc50       my_is_symlink              000000014001dc50 f   mysys:my_symlink.obj
 0001:0001cc80       my_realpath                000000014001dc80 f   mysys:my_symlink.obj
 0001:0001cd20       my_message_no_curses       000000014001dd20 f   mysys:my_messnc.obj
 0001:0001cdd0       init_glob_errs             000000014001ddd0 f   mysys:errors.obj
 0001:0001cde0       wait_for_free_space        000000014001dde0 f   mysys:errors.obj
 0001:0001ce70       my_write                   000000014001de70 f   mysys:my_write.obj
 0001:0001cfe0       strnmov                    000000014001dfe0 f   strings:strnmov.obj
 0001:0001d020       int2str                    000000014001e020 f   strings:int2str.obj
 0001:0001d120       int10_to_str               000000014001e120 f   strings:int2str.obj
 0001:0001d200       strmake                    000000014001e200 f   strings:strmake.obj
 0001:0001d240       strmov                     000000014001e240 f   strings:strmov.obj
 0001:0001d270       strxnmov                   000000014001e270 f   strings:strxnmov.obj
 0001:0001d2d0       strend                     000000014001e2d0 f   strings:strend.obj
 0001:0001d2f0       is_prefix                  000000014001e2f0 f   strings:is_prefix.obj
 0001:0001d620       my_hash_sort_latin1_de     000000014001e620 f   strings:ctype-latin1.obj
 0001:0001d6e0       my_vsnprintf               000000014001e6e0 f   strings:my_vsnprintf.obj
 0001:0001da40       my_snprintf                000000014001ea40 f   strings:my_vsnprintf.obj
 0001:0001da60       strcend                    000000014001ea60 f   strings:strcend.obj
 0001:0001da80       my_strnxfrmlen_simple      000000014001ea80 f   strings:ctype-simple.obj
 0001:0001daa0       my_strnxfrm_simple         000000014001eaa0 f   strings:ctype-simple.obj
 0001:0001db40       my_strnncoll_simple        000000014001eb40 f   strings:ctype-simple.obj
 0001:0001dbe0       my_strnncollsp_simple      000000014001ebe0 f   strings:ctype-simple.obj
 0001:0001dcc0       my_caseup_str_8bit         000000014001ecc0 f   strings:ctype-simple.obj
 0001:0001dd00       my_casedn_str_8bit         000000014001ed00 f   strings:ctype-simple.obj
 0001:0001dd40       my_caseup_8bit             000000014001ed40 f   strings:ctype-simple.obj
 0001:0001dd70       my_casedn_8bit             000000014001ed70 f   strings:ctype-simple.obj
 0001:0001dda0       my_strcasecmp_8bit         000000014001eda0 f   strings:ctype-simple.obj
 0001:0001de00       my_mb_wc_8bit              000000014001ee00 f   strings:ctype-simple.obj
 0001:0001de40       my_wc_mb_8bit              000000014001ee40 f   strings:ctype-simple.obj
 0001:0001dea0       my_snprintf_8bit           000000014001eea0 f   strings:ctype-simple.obj
 0001:0001ded0       my_hash_sort_simple        000000014001eed0 f   strings:ctype-simple.obj
 0001:0001df60       my_strntol_8bit            000000014001ef60 f   strings:ctype-simple.obj
 0001:0001e0e0       my_strntoul_8bit           000000014001f0e0 f   strings:ctype-simple.obj
 0001:0001e240       my_strntoll_8bit           000000014001f240 f   strings:ctype-simple.obj
 0001:0001e3d0       my_strntoull_8bit          000000014001f3d0 f   strings:ctype-simple.obj
 0001:0001e540       my_strntod_8bit            000000014001f540 f   strings:ctype-simple.obj
 0001:0001e570       my_long10_to_str_8bit      000000014001f570 f   strings:ctype-simple.obj
 0001:0001e680       my_longlong10_to_str_8bit  000000014001f680 f   strings:ctype-simple.obj
 0001:0001e7c0       my_wildcmp_8bit            000000014001f7c0 f   strings:ctype-simple.obj
 0001:0001e9e0       my_like_range_simple       000000014001f9e0 f   strings:ctype-simple.obj
 0001:0001eb40       my_scan_8bit               000000014001fb40 f   strings:ctype-simple.obj
 0001:0001eba0       my_fill_8bit               000000014001fba0 f   strings:ctype-simple.obj
 0001:0001ebb0       my_numchars_8bit           000000014001fbb0 f   strings:ctype-simple.obj
 0001:0001ebc0       my_numcells_8bit           000000014001fbc0 f   strings:ctype-simple.obj
 0001:0001ebd0       my_charpos_8bit            000000014001fbd0 f   strings:ctype-simple.obj
 0001:0001ebe0       my_well_formed_len_8bit    000000014001fbe0 f   strings:ctype-simple.obj
 0001:0001ec00       my_lengthsp_8bit           000000014001fc00 f   strings:ctype-simple.obj
 0001:0001ec30       my_instr_simple            000000014001fc30 f   strings:ctype-simple.obj
 0001:0001f030       my_strtoll10_8bit          0000000140020030 f   strings:ctype-simple.obj
 0001:0001f050       my_strntoull10rnd_8bit     0000000140020050 f   strings:ctype-simple.obj
 0001:0001f480       my_propagate_simple        0000000140020480 f   strings:ctype-simple.obj
 0001:0001f490       my_propagate_complex       0000000140020490 f   strings:ctype-simple.obj
 0001:0001f500       my_lengthsp_binary         0000000140020500 f   strings:ctype-bin.obj
 0001:0001f660       my_mbcharlen_8bit          0000000140020660 f   strings:ctype-bin.obj
 0001:0001f6b0       my_hash_sort_8bit_bin      00000001400206b0 f   strings:ctype-bin.obj
 0001:0001f710       my_hash_sort_bin           0000000140020710 f   strings:ctype-bin.obj
 0001:0001f770       my_wildcmp_bin             0000000140020770 f   strings:ctype-bin.obj
 0001:000201b0       my_parse_charset_xml       00000001400211b0 f   strings:ctype.obj
 0001:00020270       my_string_repertoire       0000000140021270 f   strings:ctype.obj
 0001:00020320       my_charset_repertoire      0000000140021320 f   strings:ctype.obj
 0001:00020330       my_charset_is_ascii_based  0000000140021330 f   strings:ctype.obj
 0001:00020370       my_charset_is_8bit_pure_ascii 0000000140021370 f   strings:ctype.obj
 0001:00021a30       strxmov                    0000000140022a30 f   strings:strxmov.obj
 0001:000223a0       str2int                    00000001400233a0 f   strings:str2int.obj
 0001:00022580       strtoll                    0000000140023580 f   strings:strtoll.obj
 0001:00022790       llstr                      0000000140023790 f   strings:llstr.obj
 0001:000227b0       ullstr                     00000001400237b0 f   strings:llstr.obj
 0001:000227d0       longlong2str               00000001400237d0 f   strings:longlong2str.obj
 0001:00022910       longlong10_to_str          0000000140023910 f   strings:longlong2str.obj
 0001:00022a30       my_wildcmp_unicode         0000000140023a30 f   strings:ctype-utf8.obj
 0001:000267e0       my_strntol_ucs2            00000001400277e0 f   strings:ctype-ucs2.obj
 0001:00026a10       my_strntoul_ucs2           0000000140027a10 f   strings:ctype-ucs2.obj
 0001:00026c10       my_strntoll_ucs2           0000000140027c10 f   strings:ctype-ucs2.obj
 0001:00026e90       my_strntoull_ucs2          0000000140027e90 f   strings:ctype-ucs2.obj
 0001:000270a0       my_strntod_ucs2            00000001400280a0 f   strings:ctype-ucs2.obj
 0001:000271a0       my_strntoull10rnd_ucs2     00000001400281a0 f   strings:ctype-ucs2.obj
 0001:000272b0       my_l10tostr_ucs2           00000001400282b0 f   strings:ctype-ucs2.obj
 0001:000273e0       my_ll10tostr_ucs2          00000001400283e0 f   strings:ctype-ucs2.obj
 0001:00027530       my_strtoll10_ucs2          0000000140028530 f   strings:ctype-ucs2.obj
 0001:00027ca0       my_like_range_ucs2         0000000140028ca0 f   strings:ctype-ucs2.obj
 0001:00028000       my_scan_ucs2               0000000140029000 f   strings:ctype-ucs2.obj
 0001:00028d50       my_strnncoll_gbk_internal  0000000140029d50 f   strings:ctype-gbk.obj
 0001:00028e90       my_strnncoll_gbk           0000000140029e90 f   strings:ctype-gbk.obj
 0001:0002db90       bchange                    000000014002eb90 f   strings:bchange.obj
 0001:0002dc00       bmove_upp                  000000014002ec00 f   strings:bmove_upp.obj
 0001:0002dc30       my_strtod                  000000014002ec30 f   strings:strtod.obj
 0001:0002dfb0       my_atof                    000000014002efb0 f   strings:strtod.obj
 0001:0002dfe0       my_strtoll10               000000014002efe0 f   strings:my_strtoll10.obj
 0001:0002e8c0       my_xml_parse               000000014002f8c0 f   strings:xml.obj
 0001:0002ec80       my_xml_parser_create       000000014002fc80 f   strings:xml.obj
 0001:0002ec90       my_xml_parser_free         000000014002fc90 f   strings:xml.obj
 0001:0002eca0       my_xml_set_value_handler   000000014002fca0 f   strings:xml.obj
 0001:0002ecb0       my_xml_set_enter_handler   000000014002fcb0 f   strings:xml.obj
 0001:0002ecc0       my_xml_set_leave_handler   000000014002fcc0 f   strings:xml.obj
 0001:0002ecd0       my_xml_set_user_data       000000014002fcd0 f   strings:xml.obj
 0001:0002ece0       my_xml_error_string        000000014002fce0 f   strings:xml.obj
 0001:0002ecf0       my_xml_error_pos           000000014002fcf0 f   strings:xml.obj
 0001:0002ed30       my_xml_error_lineno        000000014002fd30 f   strings:xml.obj
 0001:0002ed60       my_caseup_str_mb           000000014002fd60 f   strings:ctype-mb.obj
 0001:0002edf0       my_casedn_str_mb           000000014002fdf0 f   strings:ctype-mb.obj
 0001:0002ee80       my_caseup_mb               000000014002fe80 f   strings:ctype-mb.obj
 0001:0002ef00       my_casedn_mb               000000014002ff00 f   strings:ctype-mb.obj
 0001:0002ef80       my_strcasecmp_mb           000000014002ff80 f   strings:ctype-mb.obj
 0001:0002f050       my_wildcmp_mb              0000000140030050 f   strings:ctype-mb.obj
 0001:0002f470       my_numchars_mb             0000000140030470 f   strings:ctype-mb.obj
 0001:0002f4e0       my_charpos_mb              00000001400304e0 f   strings:ctype-mb.obj
 0001:0002f570       my_well_formed_len_mb      0000000140030570 f   strings:ctype-mb.obj
 0001:0002f600       my_instr_mb                0000000140030600 f   strings:ctype-mb.obj
 0001:0002f9b0       my_like_range_mb           00000001400309b0 f   strings:ctype-mb.obj
 0001:00030040       my_numcells_mb             0000000140031040 f   strings:ctype-mb.obj
 0001:00030110       vio_delete                 0000000140031110 f   vio:vio.obj
 0001:00030150       vio_end                    0000000140031150 f   vio:vio.obj
 0001:000304a0       vio_reset                  00000001400314a0 f   vio:vio.obj
 0001:00030500       vio_new                    0000000140031500 f   vio:vio.obj
 0001:000305a0       vio_new_win32pipe          00000001400315a0 f   vio:vio.obj
 0001:00030600       vio_new_win32shared_memory 0000000140031600 f   vio:vio.obj
 0001:000306f0       vio_errno                  00000001400316f0 f   vio:viosocket.obj
 0001:00030700       vio_read                   0000000140031700 f   vio:viosocket.obj
 0001:00030710       vio_read_buff              0000000140031710 f   vio:viosocket.obj
 0001:000307d0       vio_write                  00000001400317d0 f   vio:viosocket.obj
 0001:000307e0       vio_blocking               00000001400317e0 f   vio:viosocket.obj
 0001:00030860       vio_is_blocking            0000000140031860 f   vio:viosocket.obj
 0001:00030870       vio_fastsend               0000000140031870 f   vio:viosocket.obj
 0001:000308b0       vio_keepalive              00000001400318b0 f   vio:viosocket.obj
 0001:00030900       vio_should_retry           0000000140031900 f   vio:viosocket.obj
 0001:00030930       vio_was_interrupted        0000000140031930 f   vio:viosocket.obj
 0001:00030970       vio_close                  0000000140031970 f   vio:viosocket.obj
 0001:000309e0       vio_description            00000001400319e0 f   vio:viosocket.obj
 0001:000309f0       vio_type                   00000001400319f0 f   vio:viosocket.obj
 0001:00030a00       vio_fd                     0000000140031a00 f   vio:viosocket.obj
 0001:00030a10       vio_peer_addr              0000000140031a10 f   vio:viosocket.obj
 0001:00030ab0       vio_in_addr                0000000140031ab0 f   vio:viosocket.obj
 0001:00030ad0       vio_poll_read              0000000140031ad0 f   vio:viosocket.obj
 0001:00030ae0       vio_timeout                0000000140031ae0 f   vio:viosocket.obj
 0001:00030b20       vio_read_pipe              0000000140031b20 f   vio:viosocket.obj
 0001:00030b50       vio_write_pipe             0000000140031b50 f   vio:viosocket.obj
 0001:00030b80       vio_close_pipe             0000000140031b80 f   vio:viosocket.obj
 0001:00030bb0       vio_ignore_timeout         0000000140031bb0 f   vio:viosocket.obj
 0001:00030bc0       vio_read_shared_memory     0000000140031bc0 f   vio:viosocket.obj
 0001:00030ce0       vio_write_shared_memory    0000000140031ce0 f   vio:viosocket.obj
 0001:00030dd0       vio_close_shared_memory    0000000140031dd0 f   vio:viosocket.obj
 0001:00030ee0       vio_ssl_read               0000000140031ee0 f   vio:viossl.obj
 0001:00030ef0       vio_ssl_write              0000000140031ef0 f   vio:viossl.obj
 0001:00030f00       vio_ssl_close              0000000140031f00 f   vio:viossl.obj
 0001:00030f40       vio_ssl_delete             0000000140031f40 f   vio:viossl.obj
 0001:00031090       sslaccept                  0000000140032090 f   vio:viossl.obj
 0001:000310a0       sslconnect                 00000001400320a0 f   vio:viossl.obj
 0001:000310b0       vio_ssl_blocking           00000001400320b0 f   vio:viossl.obj
 0001:00031170       sslGetErrString            0000000140032170 f   vio:viosslfactories.obj
 0001:00031400       new_VioSSLConnectorFd      0000000140032400 f   vio:viosslfactories.obj
 0001:00031490       new_VioSSLAcceptorFd       0000000140032490 f   vio:viosslfactories.obj
 0001:00031530       ??2@YAPEAX_KPEAUDummy@@@Z  0000000140032530 f i yassl:ssl.obj
 0001:00031540       ??1Message@yaSSL@@UEAA@XZ  0000000140032540 f i yassl:ssl.obj
 0001:00031550       ??_GMessage@yaSSL@@UEAAPEAXI@Z 0000000140032550 f i yassl:ssl.obj
 0001:00031550       ??_EMessage@yaSSL@@UEAAPEAXI@Z 0000000140032550 f i yassl:ssl.obj
 0001:00031580       ??1Alert@yaSSL@@UEAA@XZ    0000000140032580 f i yassl:ssl.obj
 0001:00031590       ??1HandShakeBase@yaSSL@@UEAA@XZ 0000000140032590 f i yassl:ssl.obj
 0001:000315a0       ??_EHandShakeBase@yaSSL@@UEAAPEAXI@Z 00000001400325a0 f i yassl:ssl.obj
 0001:000315a0       ??_GHandShakeBase@yaSSL@@UEAAPEAXI@Z 00000001400325a0 f i yassl:ssl.obj
 0001:000315d0       ??0EncryptedInfo@yaSSL@@QEAA@XZ 00000001400325d0 f i yassl:ssl.obj
 0001:000315e0       ??0Error@TaoCrypt@@QEAA@W4ErrorNumber@1@@Z 00000001400325e0 f i yassl:ssl.obj
 0001:000315f0       ?assign@BIGNUM@yaSSL@@QEAAXPEBEI@Z 00000001400325f0 f i yassl:ssl.obj
 0001:00031600       ??1Finished@yaSSL@@UEAA@XZ 0000000140032600 f i yassl:ssl.obj
 0001:00031610       ??1HASH@TaoCrypt@@UEAA@XZ  0000000140032610 f i yassl:ssl.obj
 0001:00031620       ??_GHASH@TaoCrypt@@UEAAPEAXI@Z 0000000140032620 f i yassl:ssl.obj
 0001:00031620       ??_EHASH@TaoCrypt@@UEAAPEAXI@Z 0000000140032620 f i yassl:ssl.obj
 0001:00031650       ??1HASHwithTransform@TaoCrypt@@UEAA@XZ 0000000140032650 f i yassl:ssl.obj
 0001:00031660       ??0MD5@TaoCrypt@@QEAA@XZ   0000000140032660 f i yassl:ssl.obj
 0001:000316a0       ?getByteOrder@MD5@TaoCrypt@@UEBA?AW4ByteOrder@2@XZ 00000001400326a0 f i yassl:ssl.obj
 0001:000316b0       ?getBlockSize@MD5@TaoCrypt@@UEBAIXZ 00000001400326b0 f i yassl:ssl.obj
 0001:000316c0       ?getDigestSize@MD5@TaoCrypt@@UEBAIXZ 00000001400326c0 f i yassl:ssl.obj
 0001:000316d0       ?getPadSize@MD5@TaoCrypt@@UEBAIXZ 00000001400326d0 f i yassl:ssl.obj
 0001:000316e0       ??1MD5@TaoCrypt@@UEAA@XZ   00000001400326e0 f i yassl:ssl.obj
 0001:000316f0       ??0MD4@TaoCrypt@@QEAA@XZ   00000001400326f0 f i yassl:ssl.obj
 0001:00031730       ?getByteOrder@MD4@TaoCrypt@@UEBA?AW4ByteOrder@2@XZ 0000000140032730 f i yassl:ssl.obj
 0001:00031740       ?getBlockSize@MD4@TaoCrypt@@UEBAIXZ 0000000140032740 f i yassl:ssl.obj
 0001:00031750       ?getDigestSize@MD4@TaoCrypt@@UEBAIXZ 0000000140032750 f i yassl:ssl.obj
 0001:00031760       ?getPadSize@MD4@TaoCrypt@@UEBAIXZ 0000000140032760 f i yassl:ssl.obj
 0001:00031770       ??1MD4@TaoCrypt@@UEAA@XZ   0000000140032770 f i yassl:ssl.obj
 0001:00031780       yaSSLv3_server_method      0000000140032780 f   yassl:ssl.obj
 0001:000317d0       yaSSLv3_client_method      00000001400327d0 f   yassl:ssl.obj
 0001:00031820       yaTLSv1_server_method      0000000140032820 f   yassl:ssl.obj
 0001:00031870       yaTLSv1_client_method      0000000140032870 f   yassl:ssl.obj
 0001:000318c0       yaTLSv1_1_server_method    00000001400328c0 f   yassl:ssl.obj
 0001:00031910       yaTLSv1_1_client_method    0000000140032910 f   yassl:ssl.obj
 0001:00031960       yaSSLv23_server_method     0000000140032960 f   yassl:ssl.obj
 0001:000319b0       yaSSLv23_client_method     00000001400329b0 f   yassl:ssl.obj
 0001:00031a00       yaSSL_CTX_new              0000000140032a00 f   yassl:ssl.obj
 0001:00031a30       yaSSL_new                  0000000140032a30 f   yassl:ssl.obj
 0001:00031a60       yaSSL_set_fd               0000000140032a60 f   yassl:ssl.obj
 0001:00031a90       yaSSL_get_fd               0000000140032a90 f   yassl:ssl.obj
 0001:00031ab0       yaSSL_connect              0000000140032ab0 f   yassl:ssl.obj
 0001:00031de0       yaSSL_write                0000000140032de0 f   yassl:ssl.obj
 0001:00031df0       ??1Data@yaSSL@@UEAA@XZ     0000000140032df0 f i yassl:ssl.obj
 0001:00031e00       yaSSL_accept               0000000140032e00 f   yassl:ssl.obj
 0001:00032130       yaSSL_do_handshake         0000000140033130 f   yassl:ssl.obj
 0001:00032170       yaSSL_clear                0000000140033170 f   yassl:ssl.obj
 0001:00032190       yaSSL_shutdown             0000000140033190 f   yassl:ssl.obj
 0001:00032210       yaSSL_set_quiet_shutdown   0000000140033210 f   yassl:ssl.obj
 0001:00032220       yaSSL_get_quiet_shutdown   0000000140033220 f   yassl:ssl.obj
 0001:00032240       yaSSL_CTX_set_session_cache_mode 0000000140033240 f   yassl:ssl.obj
 0001:00032270       yaSSL_get_session          0000000140033270 f   yassl:ssl.obj
 0001:000322d0       yaSSL_set_session          00000001400332d0 f   yassl:ssl.obj
 0001:00032330       yaSSL_session_reused       0000000140033330 f   yassl:ssl.obj
 0001:00032350       yaSSL_SESSION_set_timeout  0000000140033350 f   yassl:ssl.obj
 0001:00032370       yaSSL_get_default_timeout  0000000140033370 f   yassl:ssl.obj
 0001:00032380       yaSSL_flush_sessions       0000000140033380 f   yassl:ssl.obj
 0001:000323a0       yaSSL_get_cipher           00000001400333a0 f   yassl:ssl.obj
 0001:000323c0       yaSSL_get_shared_ciphers   00000001400333c0 f   yassl:ssl.obj
 0001:000323e0       yaSSL_get_cipher_list      00000001400333e0 f   yassl:ssl.obj
 0001:00032450       yaSSL_CTX_set_cipher_list  0000000140033450 f   yassl:ssl.obj
 0001:00032470       yaSSL_get_version          0000000140033470 f   yassl:ssl.obj
 0001:000324a0       yaSSLeay_version           00000001400334a0 f   yassl:ssl.obj
 0001:000324b0       yaSSL_get_error            00000001400334b0 f   yassl:ssl.obj
 0001:000324d0       yaSSL_set_compression      00000001400334d0 f   yassl:ssl.obj
 0001:000324e0       yaSSL_get_peer_certificate 00000001400334e0 f   yassl:ssl.obj
 0001:00032500       yaX509_free                0000000140033500 f   yassl:ssl.obj
 0001:00032510       yaX509_STORE_CTX_get_current_cert 0000000140033510 f   yassl:ssl.obj
 0001:00032520       yaX509_STORE_CTX_get_error 0000000140033520 f   yassl:ssl.obj
 0001:00032530       yaX509_STORE_CTX_get_error_depth 0000000140033530 f   yassl:ssl.obj
 0001:00032540       yaX509_NAME_oneline        0000000140033540 f   yassl:ssl.obj
 0001:000325f0       yaX509_get_issuer_name     00000001400335f0 f   yassl:ssl.obj
 0001:00032600       yaX509_get_subject_name    0000000140033600 f   yassl:ssl.obj
 0001:00032610       yaSSL_load_error_strings   0000000140033610 f   yassl:ssl.obj
 0001:00032620       yaSSL_set_connect_state    0000000140033620 f   yassl:ssl.obj
 0001:00032630       yaSSL_set_accept_state     0000000140033630 f   yassl:ssl.obj
 0001:00032650       yaSSL_get_verify_result    0000000140033650 f   yassl:ssl.obj
 0001:00032660       yaSSL_CTX_sess_set_cache_size 0000000140033660 f   yassl:ssl.obj
 0001:00032670       yaSSL_CTX_get_session_cache_mode 0000000140033670 f   yassl:ssl.obj
 0001:00032680       yaSSL_CTX_set_tmp_dh       0000000140033680 f   yassl:ssl.obj
 0001:000326a0       yaSSL_CTX_set_verify       00000001400336a0 f   yassl:ssl.obj
 0001:00032700       yaSSL_CTX_set_default_verify_paths 0000000140033700 f   yassl:ssl.obj
 0001:00032710       yaSSL_CTX_set_session_id_context 0000000140033710 f   yassl:ssl.obj
 0001:00032720       yaSSL_CTX_check_private_key 0000000140033720 f   yassl:ssl.obj
 0001:00032730       yaSSL_CTX_sess_accept      0000000140033730 f   yassl:ssl.obj
 0001:00032740       yaSSL_CTX_sess_connect     0000000140033740 f   yassl:ssl.obj
 0001:00032760       yaSSL_CTX_sess_accept_good 0000000140033760 f   yassl:ssl.obj
 0001:00032780       yaSSL_CTX_sess_connect_good 0000000140033780 f   yassl:ssl.obj
 0001:000327a0       yaSSL_CTX_sess_accept_renegotiate 00000001400337a0 f   yassl:ssl.obj
 0001:000327c0       yaSSL_CTX_sess_connect_renegotiate 00000001400337c0 f   yassl:ssl.obj
 0001:000327e0       yaSSL_CTX_sess_hits        00000001400337e0 f   yassl:ssl.obj
 0001:00032800       yaSSL_CTX_sess_cb_hits     0000000140033800 f   yassl:ssl.obj
 0001:00032820       yaSSL_CTX_sess_cache_full  0000000140033820 f   yassl:ssl.obj
 0001:00032840       yaSSL_CTX_sess_misses      0000000140033840 f   yassl:ssl.obj
 0001:00032860       yaSSL_CTX_sess_timeouts    0000000140033860 f   yassl:ssl.obj
 0001:00032880       yaSSL_CTX_sess_number      0000000140033880 f   yassl:ssl.obj
 0001:000328a0       yaSSL_CTX_sess_get_cache_size 00000001400338a0 f   yassl:ssl.obj
 0001:000328c0       yaSSL_CTX_get_verify_mode  00000001400338c0 f   yassl:ssl.obj
 0001:000328e0       yaSSL_get_verify_mode      00000001400338e0 f   yassl:ssl.obj
 0001:00032910       yaSSL_CTX_get_verify_depth 0000000140033910 f   yassl:ssl.obj
 0001:00032930       yaSSL_get_verify_depth     0000000140033930 f   yassl:ssl.obj
 0001:00032960       yaSSL_CTX_set_options      0000000140033960 f   yassl:ssl.obj
 0001:00032970       yaSSL_CTX_set_info_callback 0000000140033970 f   yassl:ssl.obj
 0001:00032980       yaOpenSSL_add_all_algorithms 0000000140033980 f   yassl:ssl.obj
 0001:00032990       yaSSL_library_init         0000000140033990 f   yassl:ssl.obj
 0001:000329a0       yaDH_new                   00000001400339a0 f   yassl:ssl.obj
 0001:000329d0       ??0BIGNUM@yaSSL@@QEAA@XZ   00000001400339d0 f i yassl:ssl.obj
 0001:000329f0       yaERR_get_error_line_data  00000001400339f0 f   yassl:ssl.obj
 0001:00032a00       yaERR_print_errors_fp      0000000140033a00 f   yassl:ssl.obj
 0001:00032a10       yaERR_error_string         0000000140033a10 f   yassl:ssl.obj
 0001:00032a40       yaX509_verify_cert_error_string 0000000140033a40 f   yassl:ssl.obj
 0001:00032a50       yaEVP_md5                  0000000140033a50 f   yassl:ssl.obj
 0001:00032a60       yaEVP_des_ede3_cbc         0000000140033a60 f   yassl:ssl.obj
 0001:00032a70       yaEVP_BytesToKey           0000000140033a70 f   yassl:ssl.obj
 0001:00032d70       yaDES_set_key_unchecked    0000000140033d70 f   yassl:ssl.obj
 0001:00032d80       yaDES_ede3_cbc_encrypt     0000000140033d80 f   yassl:ssl.obj
 0001:00032e60       yaRAND_status              0000000140033e60 f   yassl:ssl.obj
 0001:00032e70       yaDES_set_key              0000000140033e70 f   yassl:ssl.obj
 0001:00032e80       yaDES_set_odd_parity       0000000140033e80 f   yassl:ssl.obj
 0001:00032e90       yaDES_ecb_encrypt          0000000140033e90 f   yassl:ssl.obj
 0001:00032f20       yaSSL_CTX_set_default_passwd_cb_userdata 0000000140033f20 f   yassl:ssl.obj
 0001:00032f30       yaSSL_get_certificate      0000000140033f30 f   yassl:ssl.obj
 0001:00032f40       yaSSL_get_privatekey       0000000140033f40 f   yassl:ssl.obj
 0001:00032f50       yaSSL_SESSION_free         0000000140033f50 f   yassl:ssl.obj
 0001:00032f60       yaX509_get_pubkey          0000000140033f60 f   yassl:ssl.obj
 0001:00032f70       yaEVP_PKEY_copy_parameters 0000000140033f70 f   yassl:ssl.obj
 0001:00032f80       yaEVP_PKEY_free            0000000140033f80 f   yassl:ssl.obj
 0001:00032f90       yaERR_error_string_n       0000000140033f90 f   yassl:ssl.obj
 0001:00032fb0       yaERR_free_strings         0000000140033fb0 f   yassl:ssl.obj
 0001:00032fc0       yaEVP_cleanup              0000000140033fc0 f   yassl:ssl.obj
 0001:00032fd0       yaX509_get_notBefore       0000000140033fd0 f   yassl:ssl.obj
 0001:00032fe0       yaX509_get_notAfter        0000000140033fe0 f   yassl:ssl.obj
 0001:00032ff0       yaSSLv2_client_method      0000000140033ff0 f   yassl:ssl.obj
 0001:00033000       yaSSL_get1_session         0000000140034000 f   yassl:ssl.obj
 0001:00033010       yaGENERAL_NAMES_free       0000000140034010 f   yassl:ssl.obj
 0001:00033020       yask_GENERAL_NAME_num      0000000140034020 f   yassl:ssl.obj
 0001:00033030       yask_GENERAL_NAME_value    0000000140034030 f   yassl:ssl.obj
 0001:00033040       yaASN1_STRING_data         0000000140034040 f   yassl:ssl.obj
 0001:00033050       yaASN1_STRING_length       0000000140034050 f   yassl:ssl.obj
 0001:00033060       yaASN1_STRING_type         0000000140034060 f   yassl:ssl.obj
 0001:00033070       yaX509_NAME_get_index_by_NID 0000000140034070 f   yassl:ssl.obj
 0001:000330e0       yaX509_NAME_ENTRY_get_data 00000001400340e0 f   yassl:ssl.obj
 0001:000330f0       yaX509_NAME_get_entry      00000001400340f0 f   yassl:ssl.obj
 0001:00033100       yaASN1_STRING_to_UTF8      0000000140034100 f   yassl:ssl.obj
 0001:00033170       yaX509_get_ext_d2i         0000000140034170 f   yassl:ssl.obj
 0001:00033180       yaMD4_Init                 0000000140034180 f   yassl:ssl.obj
 0001:000331c0       yaMD4_Update               00000001400341c0 f   yassl:ssl.obj
 0001:000331d0       yaMD4_Final                00000001400341d0 f   yassl:ssl.obj
 0001:000331e0       yaMD5_Init                 00000001400341e0 f   yassl:ssl.obj
 0001:00033220       yaMD5_Update               0000000140034220 f   yassl:ssl.obj
 0001:00033230       yaMD5_Final                0000000140034230 f   yassl:ssl.obj
 0001:00033240       yaRAND_bytes               0000000140034240 f   yassl:ssl.obj
 0001:000332b0       yaSSL_peek                 00000001400342b0 f   yassl:ssl.obj
 0001:000332f0       yaSSL_pending              00000001400342f0 f   yassl:ssl.obj
 0001:00033320       yaSSL_CTX_set_default_passwd_cb 0000000140034320 f   yassl:ssl.obj
 0001:00033330       yaSSLeay_add_ssl_algorithms 0000000140034330 f   yassl:ssl.obj
 0001:00033340       yaERR_remove_state         0000000140034340 f   yassl:ssl.obj
 0001:00033360       yaERR_GET_REASON           0000000140034360 f   yassl:ssl.obj
 0001:00033370       err_helper                 0000000140034370 f   yassl:ssl.obj
 0001:000333a0       yaERR_peek_error           00000001400343a0 f   yassl:ssl.obj
 0001:000333b0       yaERR_get_error            00000001400343b0 f   yassl:ssl.obj
 0001:000333c0       yaRAND_screen              00000001400343c0 f   yassl:ssl.obj
 0001:000333d0       yaRAND_file_name           00000001400343d0 f   yassl:ssl.obj
 0001:000333e0       yaRAND_write_file          00000001400343e0 f   yassl:ssl.obj
 0001:000333f0       yaRAND_load_file           00000001400343f0 f   yassl:ssl.obj
 0001:00033400       yaRSA_free                 0000000140034400 f   yassl:ssl.obj
 0001:00033410       yaRSA_generate_key         0000000140034410 f   yassl:ssl.obj
 0001:00033420       yaX509_LOOKUP_add_dir      0000000140034420 f   yassl:ssl.obj
 0001:00033430       yaX509_LOOKUP_load_file    0000000140034430 f   yassl:ssl.obj
 0001:00033440       yaX509_LOOKUP_hash_dir     0000000140034440 f   yassl:ssl.obj
 0001:00033450       yaX509_LOOKUP_file         0000000140034450 f   yassl:ssl.obj
 0001:00033460       yaX509_STORE_add_lookup    0000000140034460 f   yassl:ssl.obj
 0001:00033470       yaX509_STORE_get_by_subject 0000000140034470 f   yassl:ssl.obj
 0001:00033480       yaX509_STORE_new           0000000140034480 f   yassl:ssl.obj
 0001:00033490       yaSSL_alert_type_string_long 0000000140034490 f   yassl:ssl.obj
 0001:000334a0       yaSSL_alert_desc_string_long 00000001400344a0 f   yassl:ssl.obj
 0001:000334b0       yaSSL_state_string_long    00000001400344b0 f   yassl:ssl.obj
 0001:000334c0       yaSSL_CTX_set_tmp_rsa_callback 00000001400344c0 f   yassl:ssl.obj
 0001:000334d0       yaSSL_CTX_set_timeout      00000001400344d0 f   yassl:ssl.obj
 0001:000334e0       yaSSL_CTX_use_certificate_chain_file 00000001400344e0 f   yassl:ssl.obj
 0001:000334f0       yaSSL_CTX_use_RSAPrivateKey_file 00000001400344f0 f   yassl:ssl.obj
 0001:00033500       yaSSL_set_rfd              0000000140034500 f   yassl:ssl.obj
 0001:00033510       yaSSL_set_wfd              0000000140034510 f   yassl:ssl.obj
 0001:00033520       yaSSL_want_read            0000000140034520 f   yassl:ssl.obj
 0001:00033530       yaSSL_want_write           0000000140034530 f   yassl:ssl.obj
 0001:00033540       yaSSL_set_shutdown         0000000140034540 f   yassl:ssl.obj
 0001:00033550       yaSSL_get_current_cipher   0000000140034550 f   yassl:ssl.obj
 0001:00033560       yaSSL_CIPHER_description   0000000140034560 f   yassl:ssl.obj
 0001:00033570       ?size@?$Block@EV?$AllocatorWithCleanup@E@TaoCrypt@@@TaoCrypt@@QEBAIXZ 0000000140034570 f i yassl:ssl.obj
 0001:00033580       ?get_buffer@?$Block@EV?$AllocatorWithCleanup@E@TaoCrypt@@@TaoCrypt@@QEBAPEAEXZ 0000000140034580 f i yassl:ssl.obj
 0001:00033590       ??0?$auto_ptr@UBulkCipher@yaSSL@@@mySTL@@QEAA@PEAUBulkCipher@yaSSL@@@Z 0000000140034590 f i yassl:ssl.obj
 0001:000335a0       ??C?$auto_ptr@UBulkCipher@yaSSL@@@mySTL@@QEBAPEAUBulkCipher@yaSSL@@XZ 00000001400345a0 f i yassl:ssl.obj
 0001:000335b0       ??0?$auto_ptr@Vx509@yaSSL@@@mySTL@@QEAA@PEAVx509@yaSSL@@@Z 00000001400345b0 f i yassl:ssl.obj
 0001:000335c0       ??C?$auto_ptr@Vx509@yaSSL@@@mySTL@@QEBAPEAVx509@yaSSL@@XZ 00000001400345c0 f i yassl:ssl.obj
 0001:000335d0       ?release@?$auto_ptr@Vx509@yaSSL@@@mySTL@@QEAAPEAVx509@yaSSL@@XZ 00000001400345d0 f i yassl:ssl.obj
 0001:000335e0       ??0?$auto_ptr@UBIGNUM@yaSSL@@@mySTL@@QEAA@PEAUBIGNUM@yaSSL@@@Z 00000001400345e0 f i yassl:ssl.obj
 0001:000335f0       ?get@?$auto_ptr@UBIGNUM@yaSSL@@@mySTL@@QEBAPEAUBIGNUM@yaSSL@@XZ 00000001400345f0 f i yassl:ssl.obj
 0001:00033600       ?release@?$auto_ptr@UBIGNUM@yaSSL@@@mySTL@@QEAAPEAUBIGNUM@yaSSL@@XZ 0000000140034600 f i yassl:ssl.obj
 0001:00033610       ?max_size@?$AllocatorBase@E@TaoCrypt@@QEBA_KXZ 0000000140034610 f i yassl:ssl.obj
 0001:00033620       ??$min@I@TaoCrypt@@YAAEBIAEBI0@Z 0000000140034620 f i yassl:ssl.obj
 0001:00033630       ??$tcArrayDelete@E@TaoCrypt@@YAXPEAE@Z 0000000140034630 f i yassl:ssl.obj
 0001:00033640       ??$ysDelete@UDH@yaSSL@@@yaSSL@@YAXPEAUDH@0@@Z 0000000140034640 f i yassl:ssl.obj
 0001:00033650       ??$swap@V?$AllocatorWithCleanup@E@TaoCrypt@@@mySTL@@YAXAEAV?$AllocatorWithCleanup@E@TaoCrypt@@0@Z 0000000140034650 f i yassl:ssl.obj
 0001:00033660       ??$ysDelete@UBulkCipher@yaSSL@@@yaSSL@@YAXPEAUBulkCipher@0@@Z 0000000140034660 f i yassl:ssl.obj
 0001:00033680       ??_Gx509@yaSSL@@QEAAPEAXI@Z 0000000140034680 f i yassl:ssl.obj
 0001:000336b0       ??_GSSL_CTX@yaSSL@@QEAAPEAXI@Z 00000001400346b0 f i yassl:ssl.obj
 0001:000336e0       ??1BIGNUM@yaSSL@@QEAA@XZ   00000001400346e0 f i yassl:ssl.obj
 0001:000336f0       ??1Security@yaSSL@@QEAA@XZ 00000001400346f0 f i yassl:ssl.obj
 0001:00033720       ??1sslHashes@yaSSL@@QEAA@XZ 0000000140034720 f i yassl:ssl.obj
 0001:00033750       ??_GMD5@TaoCrypt@@UEAAPEAXI@Z 0000000140034750 f i yassl:ssl.obj
 0001:00033750       ??_EMD5@TaoCrypt@@UEAAPEAXI@Z 0000000140034750 f i yassl:ssl.obj
 0001:00033780       ??_EMD4@TaoCrypt@@UEAAPEAXI@Z 0000000140034780 f i yassl:ssl.obj
 0001:00033780       ??_GMD4@TaoCrypt@@UEAAPEAXI@Z 0000000140034780 f i yassl:ssl.obj
 0001:000337b0       ?size@Source@TaoCrypt@@QEBAIXZ 00000001400347b0 f i yassl:ssl.obj
 0001:000337c0       ?get_buffer@Source@TaoCrypt@@QEBAPEBEXZ 00000001400347c0 f i yassl:ssl.obj
 0001:000337d0       yaSSLv3_method             00000001400347d0 f   yassl:ssl.obj
 0001:000337e0       yaSSL_read                 00000001400347e0 f   yassl:ssl.obj
 0001:00033820       yaSSL_get_cipher_name      0000000140034820 f   yassl:ssl.obj
 0001:00033830       ?allocate@?$AllocatorWithCleanup@E@TaoCrypt@@QEAAPEAE_KPEBX@Z 0000000140034830 f i yassl:ssl.obj
 0001:00033850       ?deallocate@?$AllocatorWithCleanup@E@TaoCrypt@@QEAAXPEAX_K@Z 0000000140034850 f i yassl:ssl.obj
 0001:00033870       ?Destroy@?$auto_ptr@UBulkCipher@yaSSL@@@mySTL@@AEAAXXZ 0000000140034870 f i yassl:ssl.obj
 0001:00033880       ??$ysDelete@Vx509@yaSSL@@@yaSSL@@YAXPEAVx509@0@@Z 0000000140034880 f i yassl:ssl.obj
 0001:000338b0       ??$ysDelete@VSSL_CTX@yaSSL@@@yaSSL@@YAXPEAVSSL_CTX@0@@Z 00000001400348b0 f i yassl:ssl.obj
 0001:000338e0       ??$StdReallocate@EV?$AllocatorWithCleanup@E@TaoCrypt@@@TaoCrypt@@YAPEAEAEAV?$AllocatorWithCleanup@E@0@PEAE_K2_N@Z 00000001400348e0 f i yassl:ssl.obj
 0001:000339c0       ??_GBIGNUM@yaSSL@@QEAAPEAXI@Z 00000001400349c0 f i yassl:ssl.obj
 0001:000339f0       ??1SSL@yaSSL@@QEAA@XZ      00000001400349f0 f i yassl:ssl.obj
 0001:00033a80       yaSSL_CTX_free             0000000140034a80 f   yassl:ssl.obj
 0001:00033a90       ??0?$Block@EV?$AllocatorWithCleanup@E@TaoCrypt@@@TaoCrypt@@QEAA@PEBEI@Z 0000000140034a90 f i yassl:ssl.obj
 0001:00033ae0       ??1?$Block@EV?$AllocatorWithCleanup@E@TaoCrypt@@@TaoCrypt@@QEAA@XZ 0000000140034ae0 f i yassl:ssl.obj
 0001:00033b10       ??1?$auto_ptr@UBulkCipher@yaSSL@@@mySTL@@QEAA@XZ 0000000140034b10 f i yassl:ssl.obj
 0001:00033b20       ?reset@?$auto_ptr@UBulkCipher@yaSSL@@@mySTL@@QEAAXPEAUBulkCipher@yaSSL@@@Z 0000000140034b20 f i yassl:ssl.obj
 0001:00033b50       ?reallocate@?$AllocatorWithCleanup@E@TaoCrypt@@QEAAPEAEPEAE_K1_N@Z 0000000140034b50 f i yassl:ssl.obj
 0001:00033b70       ?Destroy@?$auto_ptr@Vx509@yaSSL@@@mySTL@@AEAAXXZ 0000000140034b70 f i yassl:ssl.obj
 0001:00033b80       ?New@?$Block@EV?$AllocatorWithCleanup@E@TaoCrypt@@@TaoCrypt@@QEAAXI@Z 0000000140034b80 f i yassl:ssl.obj
 0001:00033bc0       ??$ysDelete@UBIGNUM@yaSSL@@@yaSSL@@YAXPEAUBIGNUM@0@@Z 0000000140034bc0 f i yassl:ssl.obj
 0001:00033bf0       ??_GSSL@yaSSL@@QEAAPEAXI@Z 0000000140034bf0 f i yassl:ssl.obj
 0001:00033c90       ??0Source@TaoCrypt@@QEAA@PEBEI@Z 0000000140034c90 f i yassl:ssl.obj
 0001:00033cf0       ??1Source@TaoCrypt@@QEAA@XZ 0000000140034cf0 f i yassl:ssl.obj
 0001:00033d20       ??1HexDecoder@TaoCrypt@@QEAA@XZ 0000000140034d20 f i yassl:ssl.obj
 0001:00033d50       yaDH_free                  0000000140034d50 f   yassl:ssl.obj
 0001:00033d80       ??1?$auto_ptr@Vx509@yaSSL@@@mySTL@@QEAA@XZ 0000000140034d80 f i yassl:ssl.obj
 0001:00033d90       ?CleanNew@?$Block@EV?$AllocatorWithCleanup@E@TaoCrypt@@@TaoCrypt@@QEAAXI@Z 0000000140034d90 f i yassl:ssl.obj
 0001:00033de0       ?Destroy@?$auto_ptr@UBIGNUM@yaSSL@@@mySTL@@AEAAXXZ 0000000140034de0 f i yassl:ssl.obj
 0001:00033df0       ??$ysDelete@VSSL@yaSSL@@@yaSSL@@YAXPEAVSSL@0@@Z 0000000140034df0 f i yassl:ssl.obj
 0001:00033e90       yaSSL_free                 0000000140034e90 f   yassl:ssl.obj
 0001:00033ea0       ??0?$Block@EV?$AllocatorWithCleanup@E@TaoCrypt@@@TaoCrypt@@QEAA@I@Z 0000000140034ea0 f i yassl:ssl.obj
 0001:00033f10       ??1?$auto_ptr@UBIGNUM@yaSSL@@@mySTL@@QEAA@XZ 0000000140034f10 f i yassl:ssl.obj
 0001:00033f20       ?reset@?$auto_ptr@UBIGNUM@yaSSL@@@mySTL@@QEAAXPEAUBIGNUM@yaSSL@@@Z 0000000140034f20 f i yassl:ssl.obj
 0001:00033f50       ??0HexDecoder@TaoCrypt@@QEAA@AEAVSource@1@@Z 0000000140034f50 f i yassl:ssl.obj
 0001:00033fb0       ?read_file@yaSSL@@YAHPEAVSSL_CTX@1@PEBDHW4CertType@1@@Z 0000000140034fb0 f   yassl:ssl.obj
 0001:00034590       yaSSL_CTX_use_certificate_file 0000000140035590 f   yassl:ssl.obj
 0001:000345a0       yaSSL_CTX_use_PrivateKey_file 00000001400355a0 f   yassl:ssl.obj
 0001:000345b0       yaSSL_CTX_load_verify_locations 00000001400355b0 f   yassl:ssl.obj
 0001:00034710       yaBN_bin2bn                0000000140035710 f   yassl:ssl.obj
 0001:000347b0       ??0Ciphers@yaSSL@@QEAA@XZ  00000001400357b0 f i yassl:yassl_int.obj
 0001:000347d0       ??0DH_Parms@yaSSL@@QEAA@XZ 00000001400357d0 f i yassl:yassl_int.obj
 0001:00034800       ??0Stats@yaSSL@@QEAA@XZ    0000000140035800 f i yassl:yassl_int.obj
 0001:00034840       ?c32to24@yaSSL@@YAXIAEAY02E@Z 0000000140035840 f   yassl:yassl_int.obj
 0001:00034860       ?c24to32@yaSSL@@YAXQEBEAEAI@Z 0000000140035860 f   yassl:yassl_int.obj
 0001:00034890       ?c24to32@yaSSL@@YAIQEBE@Z  0000000140035890 f   yassl:yassl_int.obj
 0001:000348b0       ?ato16@yaSSL@@YAXPEBEAEAG@Z 00000001400358b0 f   yassl:yassl_int.obj
 0001:000348d0       ?ato24@yaSSL@@YAXPEBEAEAY02E@Z 00000001400358d0 f   yassl:yassl_int.obj
 0001:000348f0       ?c16toa@yaSSL@@YAXGPEAE@Z  00000001400358f0 f   yassl:yassl_int.obj
 0001:00034900       ?c24toa@yaSSL@@YAXQEBEPEAE@Z 0000000140035900 f   yassl:yassl_int.obj
 0001:00034920       ?c32toa@yaSSL@@YAXIPEAE@Z  0000000140035920 f   yassl:yassl_int.obj
 0001:00034940       ??0States@yaSSL@@QEAA@XZ   0000000140035940 f   yassl:yassl_int.obj
 0001:00034970       ?getRecord@States@yaSSL@@QEBAAEBW4RecordLayerState@2@XZ 0000000140035970 f   yassl:yassl_int.obj
 0001:00034980       ?getHandShake@States@yaSSL@@QEBAAEBW4HandShakeState@2@XZ 0000000140035980 f   yassl:yassl_int.obj
 0001:00034990       ?getClient@States@yaSSL@@QEBAAEBW4ClientState@2@XZ 0000000140035990 f   yassl:yassl_int.obj
 0001:000349a0       ?getServer@States@yaSSL@@QEBAAEBW4ServerState@2@XZ 00000001400359a0 f   yassl:yassl_int.obj
 0001:000349b0       ?GetConnect@States@yaSSL@@QEBAAEBW4ConnectState@2@XZ 00000001400359b0 f   yassl:yassl_int.obj
 0001:000349c0       ?GetAccept@States@yaSSL@@QEBAAEBW4AcceptState@2@XZ 00000001400359c0 f   yassl:yassl_int.obj
 0001:000349d0       ?getString@States@yaSSL@@QEBAPEBDXZ 00000001400359d0 f   yassl:yassl_int.obj
 0001:000349e0       ?What@States@yaSSL@@QEBA?AW4YasslError@2@XZ 00000001400359e0 f   yassl:yassl_int.obj
 0001:000349f0       ?useRecord@States@yaSSL@@QEAAAEAW4RecordLayerState@2@XZ 00000001400359f0 f   yassl:yassl_int.obj
 0001:00034a00       ?useHandShake@States@yaSSL@@QEAAAEAW4HandShakeState@2@XZ 0000000140035a00 f   yassl:yassl_int.obj
 0001:00034a10       ?useClient@States@yaSSL@@QEAAAEAW4ClientState@2@XZ 0000000140035a10 f   yassl:yassl_int.obj
 0001:00034a20       ?useServer@States@yaSSL@@QEAAAEAW4ServerState@2@XZ 0000000140035a20 f   yassl:yassl_int.obj
 0001:00034a30       ?UseConnect@States@yaSSL@@QEAAAEAW4ConnectState@2@XZ 0000000140035a30 f   yassl:yassl_int.obj
 0001:00034a40       ?UseAccept@States@yaSSL@@QEAAAEAW4AcceptState@2@XZ 0000000140035a40 f   yassl:yassl_int.obj
 0001:00034a50       ?useString@States@yaSSL@@QEAAPEADXZ 0000000140035a50 f   yassl:yassl_int.obj
 0001:00034a60       ?SetError@States@yaSSL@@QEAAXW4YasslError@2@@Z 0000000140035a60 f   yassl:yassl_int.obj
 0001:00034a70       ?getMessage@sslFactory@yaSSL@@QEBAAEBV?$Factory@UMessage@yaSSL@@HP6APEAU12@XZ@2@XZ 0000000140035a70 f   yassl:yassl_int.obj
 0001:00034a80       ?getHandShake@sslFactory@yaSSL@@QEBAAEBV?$Factory@VHandShakeBase@yaSSL@@HP6APEAV12@XZ@2@XZ 0000000140035a80 f   yassl:yassl_int.obj
 0001:00034a90       ?getServerKey@sslFactory@yaSSL@@QEBAAEBV?$Factory@UServerKeyBase@yaSSL@@HP6APEAU12@XZ@2@XZ 0000000140035a90 f   yassl:yassl_int.obj
 0001:00034aa0       ?getClientKey@sslFactory@yaSSL@@QEBAAEBV?$Factory@UClientKeyBase@yaSSL@@HP6APEAU12@XZ@2@XZ 0000000140035aa0 f   yassl:yassl_int.obj
 0001:00034ab0       ?SetCompression@SSL@yaSSL@@QEAAHXZ 0000000140035ab0 f   yassl:yassl_int.obj
 0001:00034ac0       ?SetError@SSL@yaSSL@@QEAAXW4YasslError@2@@Z 0000000140035ac0 f   yassl:yassl_int.obj
 0001:00034ad0       ?SetQuietShutdown@SSL@yaSSL@@QEAAX_N@Z 0000000140035ad0 f   yassl:yassl_int.obj
 0001:00034ae0       ?useBuffers@SSL@yaSSL@@QEAAAEAVBuffers@2@XZ 0000000140035ae0 f   yassl:yassl_int.obj
 0001:00034bb0       ?order_error@SSL@yaSSL@@QEAAXXZ 0000000140035bb0 f   yassl:yassl_int.obj
 0001:00034bc0       ??0SumData@yassl_int_cpp_local1@yaSSL@@QEAA@XZ 0000000140035bc0 f i yassl:yassl_int.obj
 0001:00034bd0       ??RSumData@yassl_int_cpp_local1@yaSSL@@QEAAXPEAVinput_buffer@2@@Z 0000000140035bd0 f i yassl:yassl_int.obj
 0001:00034bf0       ??0SumBuffer@yassl_int_cpp_local1@yaSSL@@QEAA@XZ 0000000140035bf0 f i yassl:yassl_int.obj
 0001:00034c00       ??RSumBuffer@yassl_int_cpp_local1@yaSSL@@QEAAXPEAVoutput_buffer@2@@Z 0000000140035c00 f i yassl:yassl_int.obj
 0001:00034c20       ?getCrypto@SSL@yaSSL@@QEBAAEBVCrypto@2@XZ 0000000140035c20 f   yassl:yassl_int.obj
 0001:00034c30       ?getSecurity@SSL@yaSSL@@QEBAAEBVSecurity@2@XZ 0000000140035c30 f   yassl:yassl_int.obj
 0001:00034c40       ?getStates@SSL@yaSSL@@QEBAAEBVStates@2@XZ 0000000140035c40 f   yassl:yassl_int.obj
 0001:00034c50       ?getHashes@SSL@yaSSL@@QEBAAEBVsslHashes@2@XZ 0000000140035c50 f   yassl:yassl_int.obj
 0001:00034c60       ?getSocket@SSL@yaSSL@@QEBAAEBVSocket@2@XZ 0000000140035c60 f   yassl:yassl_int.obj
 0001:00034c70       ?GetError@SSL@yaSSL@@QEBA?AW4YasslError@2@XZ 0000000140035c70 f   yassl:yassl_int.obj
 0001:00034c80       ?GetQuietShutdown@SSL@yaSSL@@QEBA_NXZ 0000000140035c80 f   yassl:yassl_int.obj
 0001:00034c90       ?useCrypto@SSL@yaSSL@@QEAAAEAVCrypto@2@XZ 0000000140035c90 f   yassl:yassl_int.obj
 0001:00034ca0       ?useSecurity@SSL@yaSSL@@QEAAAEAVSecurity@2@XZ 0000000140035ca0 f   yassl:yassl_int.obj
 0001:00034cb0       ?useStates@SSL@yaSSL@@QEAAAEAVStates@2@XZ 0000000140035cb0 f   yassl:yassl_int.obj
 0001:00034cc0       ?useHashes@SSL@yaSSL@@QEAAAEAVsslHashes@2@XZ 0000000140035cc0 f   yassl:yassl_int.obj
 0001:00034cd0       ?useSocket@SSL@yaSSL@@QEAAAEAVSocket@2@XZ 0000000140035cd0 f   yassl:yassl_int.obj
 0001:00034ce0       ?useLog@SSL@yaSSL@@QEAAAEAVLog@2@XZ 0000000140035ce0 f   yassl:yassl_int.obj
 0001:00034cf0       ?HasData@SSL@yaSSL@@QEBA_NXZ 0000000140035cf0 f   yassl:yassl_int.obj
 0001:00034d00       ??0SSL_SESSION@yaSSL@@QEAA@AEAVRandomPool@1@@Z 0000000140035d00 f   yassl:yassl_int.obj
 0001:00034d40       ?GetID@SSL_SESSION@yaSSL@@QEBAPEBEXZ 0000000140035d40 f   yassl:yassl_int.obj
 0001:00034d50       ?GetSecret@SSL_SESSION@yaSSL@@QEBAPEBEXZ 0000000140035d50 f   yassl:yassl_int.obj
 0001:00034d60       ?GetSuite@SSL_SESSION@yaSSL@@QEBAPEBEXZ 0000000140035d60 f   yassl:yassl_int.obj
 0001:00034d70       ?GetPeerX509@SSL_SESSION@yaSSL@@QEBAPEAVX509@2@XZ 0000000140035d70 f   yassl:yassl_int.obj
 0001:00034d80       ?GetBornOn@SSL_SESSION@yaSSL@@QEBAIXZ 0000000140035d80 f   yassl:yassl_int.obj
 0001:00034d90       ?GetTimeOut@SSL_SESSION@yaSSL@@QEBAIXZ 0000000140035d90 f   yassl:yassl_int.obj
 0001:00034da0       ?SetTimeOut@SSL_SESSION@yaSSL@@QEAAXI@Z 0000000140035da0 f   yassl:yassl_int.obj
 0001:00034db0       ??0sess_match@yassl_int_cpp_local2@yaSSL@@QEAA@PEBE@Z 0000000140035db0 f i yassl:yassl_int.obj
 0001:00034dc0       ??Rsess_match@yassl_int_cpp_local2@yaSSL@@QEAA_NPEAVSSL_SESSION@2@@Z 0000000140035dc0 f i yassl:yassl_int.obj
 0001:00034df0       ?GetSelf@yassl_int_cpp_local2@yaSSL@@YAKXZ 0000000140035df0 f   yassl:yassl_int.obj
 0001:00034e00       ??0thr_match@yassl_int_cpp_local2@yaSSL@@QEAA@XZ 0000000140035e00 f i yassl:yassl_int.obj
 0001:00034e20       ??Rthr_match@yassl_int_cpp_local2@yaSSL@@QEAA_NUThreadError@2@@Z 0000000140035e20 f i yassl:yassl_int.obj
 0001:00034e30       ??0SSL_METHOD@yaSSL@@QEAA@W4ConnectionEnd@1@UProtocolVersion@1@_N@Z 0000000140035e30 f   yassl:yassl_int.obj
 0001:00034e50       ?getVersion@SSL_METHOD@yaSSL@@QEBA?AUProtocolVersion@2@XZ 0000000140035e50 f   yassl:yassl_int.obj
 0001:00034e60       ?getSide@SSL_METHOD@yaSSL@@QEBA?AW4ConnectionEnd@2@XZ 0000000140035e60 f   yassl:yassl_int.obj
 0001:00034e70       ?setVerifyPeer@SSL_METHOD@yaSSL@@QEAAXXZ 0000000140035e70 f   yassl:yassl_int.obj
 0001:00034e80       ?setVerifyNone@SSL_METHOD@yaSSL@@QEAAXXZ 0000000140035e80 f   yassl:yassl_int.obj
 0001:00034e90       ?setFailNoCert@SSL_METHOD@yaSSL@@QEAAXXZ 0000000140035e90 f   yassl:yassl_int.obj
 0001:00034ea0       ?verifyPeer@SSL_METHOD@yaSSL@@QEBA_NXZ 0000000140035ea0 f   yassl:yassl_int.obj
 0001:00034eb0       ?verifyNone@SSL_METHOD@yaSSL@@QEBA_NXZ 0000000140035eb0 f   yassl:yassl_int.obj
 0001:00034ec0       ?failNoCert@SSL_METHOD@yaSSL@@QEBA_NXZ 0000000140035ec0 f   yassl:yassl_int.obj
 0001:00034ed0       ?multipleProtocol@SSL_METHOD@yaSSL@@QEBA_NXZ 0000000140035ed0 f   yassl:yassl_int.obj
 0001:00034ee0       ??1DH_Parms@yaSSL@@QEAA@XZ 0000000140035ee0 f i yassl:yassl_int.obj
 0001:00034f00       ?GetCA_List@SSL_CTX@yaSSL@@QEBAAEBV?$list@PEAVx509@yaSSL@@@mySTL@@XZ 0000000140035f00 f   yassl:yassl_int.obj
 0001:00034f10       ?getVerifyCallback@SSL_CTX@yaSSL@@QEBAQ6AHHPEAUX509_STORE_CTX@2@@ZXZ 0000000140035f10 f   yassl:yassl_int.obj
 0001:00034f20       ?getCert@SSL_CTX@yaSSL@@QEBAPEBVx509@2@XZ 0000000140035f20 f   yassl:yassl_int.obj
 0001:00034f30       ?getKey@SSL_CTX@yaSSL@@QEBAPEBVx509@2@XZ 0000000140035f30 f   yassl:yassl_int.obj
 0001:00034f40       ?getMethod@SSL_CTX@yaSSL@@QEBAPEBVSSL_METHOD@2@XZ 0000000140035f40 f   yassl:yassl_int.obj
 0001:00034f50       ?GetCiphers@SSL_CTX@yaSSL@@QEBAAEBUCiphers@2@XZ 0000000140035f50 f   yassl:yassl_int.obj
 0001:00034f60       ?GetDH_Parms@SSL_CTX@yaSSL@@QEBAAEBUDH_Parms@2@XZ 0000000140035f60 f   yassl:yassl_int.obj
 0001:00034f70       ?GetStats@SSL_CTX@yaSSL@@QEBAAEBUStats@2@XZ 0000000140035f70 f   yassl:yassl_int.obj
 0001:00034f80       ?GetPasswordCb@SSL_CTX@yaSSL@@QEBAP6AHPEADHHPEAX@ZXZ 0000000140035f80 f   yassl:yassl_int.obj
 0001:00034f90       ?SetPasswordCb@SSL_CTX@yaSSL@@QEAAXP6AHPEADHHPEAX@Z@Z 0000000140035f90 f   yassl:yassl_int.obj
 0001:00034fa0       ?GetUserData@SSL_CTX@yaSSL@@QEBAPEAXXZ 0000000140035fa0 f   yassl:yassl_int.obj
 0001:00034fb0       ?GetSessionCacheOff@SSL_CTX@yaSSL@@QEBA_NXZ 0000000140035fb0 f   yassl:yassl_int.obj
 0001:00034fc0       ?GetSessionCacheFlushOff@SSL_CTX@yaSSL@@QEBA_NXZ 0000000140035fc0 f   yassl:yassl_int.obj
 0001:00034fd0       ?SetUserData@SSL_CTX@yaSSL@@QEAAXPEAX@Z 0000000140035fd0 f   yassl:yassl_int.obj
 0001:00034fe0       ?SetSessionCacheOff@SSL_CTX@yaSSL@@QEAAXXZ 0000000140035fe0 f   yassl:yassl_int.obj
 0001:00034ff0       ?SetSessionCacheFlushOff@SSL_CTX@yaSSL@@QEAAXXZ 0000000140035ff0 f   yassl:yassl_int.obj
 0001:00035000       ?setVerifyPeer@SSL_CTX@yaSSL@@QEAAXXZ 0000000140036000 f   yassl:yassl_int.obj
 0001:00035010       ?setVerifyNone@SSL_CTX@yaSSL@@QEAAXXZ 0000000140036010 f   yassl:yassl_int.obj
 0001:00035020       ?setFailNoCert@SSL_CTX@yaSSL@@QEAAXXZ 0000000140036020 f   yassl:yassl_int.obj
 0001:00035030       ?setVerifyCallback@SSL_CTX@yaSSL@@QEAAXP6AHHPEAUX509_STORE_CTX@2@@Z@Z 0000000140036030 f   yassl:yassl_int.obj
 0001:00035040       ?SetDH@SSL_CTX@yaSSL@@QEAA_NAEBUDH@2@@Z 0000000140036040 f   yassl:yassl_int.obj
 0001:00035090       ?SetCipherList@SSL_CTX@yaSSL@@QEAA_NPEBD@Z 0000000140036090 f   yassl:yassl_int.obj
 0001:00035220       ?IncrementStats@SSL_CTX@yaSSL@@QEAAXW4StatsField@2@@Z 0000000140036220 f   yassl:yassl_int.obj
 0001:00035340       ??0Crypto@yaSSL@@QEAA@XZ   0000000140036340 f   yassl:yassl_int.obj
 0001:00035380       ?get_digest@Crypto@yaSSL@@QEBAAEBUDigest@2@XZ 0000000140036380 f   yassl:yassl_int.obj
 0001:00035390       ?get_cipher@Crypto@yaSSL@@QEBAAEBUBulkCipher@2@XZ 0000000140036390 f   yassl:yassl_int.obj
 0001:000353a0       ?get_dh@Crypto@yaSSL@@QEBAAEBVDiffieHellman@2@XZ 00000001400363a0 f   yassl:yassl_int.obj
 0001:000353b0       ?get_random@Crypto@yaSSL@@QEBAAEBVRandomPool@2@XZ 00000001400363b0 f   yassl:yassl_int.obj
 0001:000353c0       ?get_certManager@Crypto@yaSSL@@QEBAAEBVCertManager@2@XZ 00000001400363c0 f   yassl:yassl_int.obj
 0001:000353d0       ?use_digest@Crypto@yaSSL@@QEAAAEAUDigest@2@XZ 00000001400363d0 f   yassl:yassl_int.obj
 0001:000353e0       ?use_cipher@Crypto@yaSSL@@QEAAAEAUBulkCipher@2@XZ 00000001400363e0 f   yassl:yassl_int.obj
 0001:000353f0       ?use_dh@Crypto@yaSSL@@QEAAAEAVDiffieHellman@2@XZ 00000001400363f0 f   yassl:yassl_int.obj
 0001:00035400       ?use_random@Crypto@yaSSL@@QEAAAEAVRandomPool@2@XZ 0000000140036400 f   yassl:yassl_int.obj
 0001:00035410       ?use_certManager@Crypto@yaSSL@@QEAAAEAVCertManager@2@XZ 0000000140036410 f   yassl:yassl_int.obj
 0001:00035420       ?SetDH@Crypto@yaSSL@@QEAAXPEAVDiffieHellman@2@@Z 0000000140036420 f   yassl:yassl_int.obj
 0001:00035430       ?SetDH@Crypto@yaSSL@@QEAAXAEBUDH_Parms@2@@Z 0000000140036430 f   yassl:yassl_int.obj
 0001:00035490       ?DhSet@Crypto@yaSSL@@QEAA_NXZ 0000000140036490 f   yassl:yassl_int.obj
 0001:000354a0       ?setDigest@Crypto@yaSSL@@QEAAXPEAUDigest@2@@Z 00000001400364a0 f   yassl:yassl_int.obj
 0001:000354b0       ?setCipher@Crypto@yaSSL@@QEAAXPEAUBulkCipher@2@@Z 00000001400364b0 f   yassl:yassl_int.obj
 0001:000354c0       ?get_MD5@sslHashes@yaSSL@@QEBAAEBVMD5@2@XZ 00000001400364c0 f   yassl:yassl_int.obj
 0001:000354d0       ?get_SHA@sslHashes@yaSSL@@QEBAAEBVSHA@2@XZ 00000001400364d0 f   yassl:yassl_int.obj
 0001:000354e0       ?get_verify@sslHashes@yaSSL@@QEBAAEBVFinished@2@XZ 00000001400364e0 f   yassl:yassl_int.obj
 0001:000354f0       ?get_certVerify@sslHashes@yaSSL@@QEBAAEBUHashes@2@XZ 00000001400364f0 f   yassl:yassl_int.obj
 0001:00035500       ?use_MD5@sslHashes@yaSSL@@QEAAAEAVMD5@2@XZ 0000000140036500 f   yassl:yassl_int.obj
 0001:00035510       ?use_SHA@sslHashes@yaSSL@@QEAAAEAVSHA@2@XZ 0000000140036510 f   yassl:yassl_int.obj
 0001:00035520       ?use_verify@sslHashes@yaSSL@@QEAAAEAVFinished@2@XZ 0000000140036520 f   yassl:yassl_int.obj
 0001:00035530       ?use_certVerify@sslHashes@yaSSL@@QEAAAEAUHashes@2@XZ 0000000140036530 f   yassl:yassl_int.obj
 0001:00035540       ?SetOutput@Buffers@yaSSL@@QEAAXPEAVoutput_buffer@2@@Z 0000000140036540 f   yassl:yassl_int.obj
 0001:00035550       ?SetRawInput@Buffers@yaSSL@@QEAAXPEAVinput_buffer@2@@Z 0000000140036550 f   yassl:yassl_int.obj
 0001:00035560       ?TakeRawInput@Buffers@yaSSL@@QEAAPEAVinput_buffer@2@XZ 0000000140036560 f   yassl:yassl_int.obj
 0001:00035570       ?TakeOutput@Buffers@yaSSL@@QEAAPEAVoutput_buffer@2@XZ 0000000140036570 f   yassl:yassl_int.obj
 0001:00035580       ?getData@Buffers@yaSSL@@QEBAAEBV?$list@PEAVinput_buffer@yaSSL@@@mySTL@@XZ 0000000140036580 f   yassl:yassl_int.obj
 0001:00035590       ?getHandShake@Buffers@yaSSL@@QEBAAEBV?$list@PEAVoutput_buffer@yaSSL@@@mySTL@@XZ 0000000140036590 f   yassl:yassl_int.obj
 0001:000355a0       ?useData@Buffers@yaSSL@@QEAAAEAV?$list@PEAVinput_buffer@yaSSL@@@mySTL@@XZ 00000001400365a0 f   yassl:yassl_int.obj
 0001:000355b0       ?useHandShake@Buffers@yaSSL@@QEAAAEAV?$list@PEAVoutput_buffer@yaSSL@@@mySTL@@XZ 00000001400365b0 f   yassl:yassl_int.obj
 0001:000355c0       ?get_connection@Security@yaSSL@@QEBAAEBUConnection@2@XZ 00000001400365c0 f   yassl:yassl_int.obj
 0001:000355d0       ?GetContext@Security@yaSSL@@QEBAPEBVSSL_CTX@2@XZ 00000001400365d0 f   yassl:yassl_int.obj
 0001:000355e0       ?get_parms@Security@yaSSL@@QEBAAEBUParameters@2@XZ 00000001400365e0 f   yassl:yassl_int.obj
 0001:000355f0       ?get_resume@Security@yaSSL@@QEBAAEBVSSL_SESSION@2@XZ 00000001400365f0 f   yassl:yassl_int.obj
 0001:00035600       ?get_resuming@Security@yaSSL@@QEBA_NXZ 0000000140036600 f   yassl:yassl_int.obj
 0001:00035610       ?use_connection@Security@yaSSL@@QEAAAEAUConnection@2@XZ 0000000140036610 f   yassl:yassl_int.obj
 0001:00035620       ?use_parms@Security@yaSSL@@QEAAAEAUParameters@2@XZ 0000000140036620 f   yassl:yassl_int.obj
 0001:00035630       ?use_resume@Security@yaSSL@@QEAAAEAVSSL_SESSION@2@XZ 0000000140036630 f   yassl:yassl_int.obj
 0001:00035640       ?set_resuming@Security@yaSSL@@QEAAX_N@Z 0000000140036640 f   yassl:yassl_int.obj
 0001:00035650       ??0X509_NAME@yaSSL@@QEAA@PEBD_K@Z 0000000140036650 f   yassl:yassl_int.obj
 0001:000356d0       ?GetName@X509_NAME@yaSSL@@QEBAPEBDXZ 00000001400366d0 f   yassl:yassl_int.obj
 0001:000356e0       ?GetLength@X509_NAME@yaSSL@@QEBA_KXZ 00000001400366e0 f   yassl:yassl_int.obj
 0001:000356f0       ?GetIssuer@X509@yaSSL@@QEAAPEAVX509_NAME@2@XZ 00000001400366f0 f   yassl:yassl_int.obj
 0001:00035700       ?GetSubject@X509@yaSSL@@QEAAPEAVX509_NAME@2@XZ 0000000140036700 f   yassl:yassl_int.obj
 0001:00035710       ??0StringHolder@yaSSL@@QEAA@PEBDH@Z 0000000140036710 f   yassl:yassl_int.obj
 0001:00035770       ?GetString@StringHolder@yaSSL@@QEAAPEAUASN1_STRING@2@XZ 0000000140036770 f   yassl:yassl_int.obj
 0001:00035780       ?Compress@yaSSL@@YAHPEBEHAEAVinput_buffer@1@@Z 0000000140036780 f   yassl:yassl_int.obj
 0001:00035790       ?DeCompress@yaSSL@@YAHAEAVinput_buffer@1@H0@Z 0000000140036790 f   yassl:yassl_int.obj
 0001:000357a0       ??0?$list@PEAVx509@yaSSL@@@mySTL@@QEAA@XZ 00000001400367a0 f i yassl:yassl_int.obj
 0001:000357c0       ??0?$list@PEAVSSL_SESSION@yaSSL@@@mySTL@@QEAA@XZ 00000001400367c0 f i yassl:yassl_int.obj
 0001:000357e0       ??0?$list@UThreadError@yaSSL@@@mySTL@@QEAA@XZ 00000001400367e0 f i yassl:yassl_int.obj
 0001:00035800       ??0?$list@PEAVinput_buffer@yaSSL@@@mySTL@@QEAA@XZ 0000000140036800 f i yassl:yassl_int.obj
 0001:00035820       ?size@?$list@PEAVinput_buffer@yaSSL@@@mySTL@@QEBA_KXZ 0000000140036820 f i yassl:yassl_int.obj
 0001:00035830       ??0?$list@PEAVoutput_buffer@yaSSL@@@mySTL@@QEAA@XZ 0000000140036830 f i yassl:yassl_int.obj
 0001:00035850       ?size@?$list@PEAVoutput_buffer@yaSSL@@@mySTL@@QEBA_KXZ 0000000140036850 f i yassl:yassl_int.obj
 0001:00035860       ??Diterator@?$list@PEAVx509@yaSSL@@@mySTL@@QEBAAEAPEAVx509@yaSSL@@XZ 0000000140036860 f i yassl:yassl_int.obj
 0001:00035870       ??Eiterator@?$list@PEAVx509@yaSSL@@@mySTL@@QEAAAEAV012@XZ 0000000140036870 f i yassl:yassl_int.obj
 0001:00035880       ??9iterator@?$list@PEAVx509@yaSSL@@@mySTL@@QEBA_NAEBV012@@Z 0000000140036880 f i yassl:yassl_int.obj
 0001:00035890       ??Diterator@?$list@PEAVinput_buffer@yaSSL@@@mySTL@@QEBAAEAPEAVinput_buffer@yaSSL@@XZ 0000000140036890 f i yassl:yassl_int.obj
 0001:000358a0       ??Eiterator@?$list@PEAVinput_buffer@yaSSL@@@mySTL@@QEAA?AV012@H@Z 00000001400368a0 f i yassl:yassl_int.obj
 0001:000358c0       ??0?$auto_ptr@Voutput_buffer@yaSSL@@@mySTL@@QEAA@PEAVoutput_buffer@yaSSL@@@Z 00000001400368c0 f i yassl:yassl_int.obj
 0001:000358d0       ??Diterator@?$list@PEAVSSL_SESSION@yaSSL@@@mySTL@@QEBAAEAPEAVSSL_SESSION@yaSSL@@XZ 00000001400368d0 f i yassl:yassl_int.obj
 0001:000358e0       ??Eiterator@?$list@PEAVSSL_SESSION@yaSSL@@@mySTL@@QEAAAEAV012@XZ 00000001400368e0 f i yassl:yassl_int.obj
 0001:000358f0       ??9iterator@?$list@PEAVSSL_SESSION@yaSSL@@@mySTL@@QEBA_NAEBV012@@Z 00000001400368f0 f i yassl:yassl_int.obj
 0001:00035900       ??9iterator@?$list@UThreadError@yaSSL@@@mySTL@@QEBA_NAEBV012@@Z 0000000140036900 f i yassl:yassl_int.obj
 0001:00035910       ??0iterator@?$list@PEAVx509@yaSSL@@@mySTL@@QEAA@PEAUnode@12@@Z 0000000140036910 f i yassl:yassl_int.obj
 0001:00035920       ??0iterator@?$list@PEAVinput_buffer@yaSSL@@@mySTL@@QEAA@PEAUnode@12@@Z 0000000140036920 f i yassl:yassl_int.obj
 0001:00035930       ??0iterator@?$list@PEAVoutput_buffer@yaSSL@@@mySTL@@QEAA@PEAUnode@12@@Z 0000000140036930 f i yassl:yassl_int.obj
 0001:00035940       ??0iterator@?$list@PEAVSSL_SESSION@yaSSL@@@mySTL@@QEAA@PEAUnode@12@@Z 0000000140036940 f i yassl:yassl_int.obj
 0001:00035950       ??0iterator@?$list@UThreadError@yaSSL@@@mySTL@@QEAA@PEAUnode@12@@Z 0000000140036950 f i yassl:yassl_int.obj
 0001:00035960       ??Diterator@?$list@UThreadError@yaSSL@@@mySTL@@QEBAAEAUThreadError@yaSSL@@XZ 0000000140036960 f i yassl:yassl_int.obj
 0001:00035970       ??0?$vector_base@U?$pair@HP6APEAUMessage@yaSSL@@XZ@mySTL@@@mySTL@@QEAA@XZ 0000000140036970 f i yassl:yassl_int.obj
 0001:00035990       ??0?$vector_base@U?$pair@HP6APEAVHandShakeBase@yaSSL@@XZ@mySTL@@@mySTL@@QEAA@XZ 0000000140036990 f i yassl:yassl_int.obj
 0001:000359b0       ??0?$vector_base@U?$pair@HP6APEAUServerKeyBase@yaSSL@@XZ@mySTL@@@mySTL@@QEAA@XZ 00000001400369b0 f i yassl:yassl_int.obj
 0001:000359d0       ??0?$vector_base@U?$pair@HP6APEAUClientKeyBase@yaSSL@@XZ@mySTL@@@mySTL@@QEAA@XZ 00000001400369d0 f i yassl:yassl_int.obj
 0001:000359f0       ??$GetArrayMemory@E@mySTL@@YAPEAE_K@Z 00000001400369f0 f i yassl:yassl_int.obj
 0001:00035a00       ?front@?$list@PEAVinput_buffer@yaSSL@@@mySTL@@QEBAPEAVinput_buffer@yaSSL@@XZ 0000000140036a00 f i yassl:yassl_int.obj
 0001:00035a10       ?front@?$list@PEAVoutput_buffer@yaSSL@@@mySTL@@QEBAPEAVoutput_buffer@yaSSL@@XZ 0000000140036a10 f i yassl:yassl_int.obj
 0001:00035a20       ??$find_if@Viterator@?$list@PEAVSSL_SESSION@yaSSL@@@mySTL@@Usess_match@yassl_int_cpp_local2@yaSSL@@@mySTL@@YA?AViterator@?$list@PEAVSSL_SESSION@yaSSL@@@0@V120@0Usess_match@yassl_int_cpp_local2@yaSSL@@@Z 0000000140036a20 f i yassl:yassl_int.obj
 0001:00035a90       ??$ysDelete@VSSL_METHOD@yaSSL@@@yaSSL@@YAXPEAVSSL_METHOD@0@@Z 0000000140036a90 f i yassl:yassl_int.obj
 0001:00035aa0       ??$ysDelete@UDigest@yaSSL@@@yaSSL@@YAXPEAUDigest@0@@Z 0000000140036aa0 f i yassl:yassl_int.obj
 0001:00035ac0       ??$ysArrayDelete@D@yaSSL@@YAXPEAD@Z 0000000140036ac0 f i yassl:yassl_int.obj
 0001:00035ad0       ??$ysArrayDelete@E@yaSSL@@YAXPEAE@Z 0000000140036ad0 f i yassl:yassl_int.obj
 0001:00035ae0       ??$FreeArrayMemory@U?$pair@HP6APEAUMessage@yaSSL@@XZ@mySTL@@@mySTL@@YAXPEAU?$pair@HP6APEAUMessage@yaSSL@@XZ@0@@Z 0000000140036ae0 f i yassl:yassl_int.obj
 0001:00035af0       ??$FreeArrayMemory@U?$pair@HP6APEAVHandShakeBase@yaSSL@@XZ@mySTL@@@mySTL@@YAXPEAU?$pair@HP6APEAVHandShakeBase@yaSSL@@XZ@0@@Z 0000000140036af0 f i yassl:yassl_int.obj
 0001:00035b00       ??$FreeArrayMemory@U?$pair@HP6APEAUServerKeyBase@yaSSL@@XZ@mySTL@@@mySTL@@YAXPEAU?$pair@HP6APEAUServerKeyBase@yaSSL@@XZ@0@@Z 0000000140036b00 f i yassl:yassl_int.obj
 0001:00035b10       ??$FreeArrayMemory@U?$pair@HP6APEAUClientKeyBase@yaSSL@@XZ@mySTL@@@mySTL@@YAXPEAU?$pair@HP6APEAUClientKeyBase@yaSSL@@XZ@0@@Z 0000000140036b10 f i yassl:yassl_int.obj
 0001:00035b20       ??_Ginput_buffer@yaSSL@@QEAAPEAXI@Z 0000000140036b20 f i yassl:yassl_int.obj
 0001:00035b50       ??_Goutput_buffer@yaSSL@@QEAAPEAXI@Z 0000000140036b50 f i yassl:yassl_int.obj
 0001:00035b80       ??_GDiffieHellman@yaSSL@@QEAAPEAXI@Z 0000000140036b80 f i yassl:yassl_int.obj
 0001:00035bb0       ??Eiterator@?$list@PEAVinput_buffer@yaSSL@@@mySTL@@QEAAAEAV012@XZ 0000000140036bb0 f i yassl:yassl_int.obj
 0001:00035bc0       ??9iterator@?$list@PEAVinput_buffer@yaSSL@@@mySTL@@QEBA_NAEBV012@@Z 0000000140036bc0 f i yassl:yassl_int.obj
 0001:00035bd0       ??Diterator@?$list@PEAVoutput_buffer@yaSSL@@@mySTL@@QEBAAEAPEAVoutput_buffer@yaSSL@@XZ 0000000140036bd0 f i yassl:yassl_int.obj
 0001:00035be0       ??Eiterator@?$list@PEAVoutput_buffer@yaSSL@@@mySTL@@QEAAAEAV012@XZ 0000000140036be0 f i yassl:yassl_int.obj
 0001:00035bf0       ??9iterator@?$list@PEAVoutput_buffer@yaSSL@@@mySTL@@QEBA_NAEBV012@@Z 0000000140036bf0 f i yassl:yassl_int.obj
 0001:00035c00       ??Eiterator@?$list@UThreadError@yaSSL@@@mySTL@@QEAAAEAV012@XZ 0000000140036c00 f i yassl:yassl_int.obj
 0001:00035c10       ??0node@?$list@PEAVx509@yaSSL@@@mySTL@@QEAA@PEAVx509@yaSSL@@@Z 0000000140036c10 f i yassl:yassl_int.obj
 0001:00035c30       ??0node@?$list@PEAVinput_buffer@yaSSL@@@mySTL@@QEAA@PEAVinput_buffer@yaSSL@@@Z 0000000140036c30 f i yassl:yassl_int.obj
 0001:00035c50       ??0node@?$list@PEAVSSL_SESSION@yaSSL@@@mySTL@@QEAA@PEAVSSL_SESSION@yaSSL@@@Z 0000000140036c50 f i yassl:yassl_int.obj
 0001:00035c70       ??0node@?$list@UThreadError@yaSSL@@@mySTL@@QEAA@UThreadError@yaSSL@@@Z 0000000140036c70 f i yassl:yassl_int.obj
 0001:00035c90       ??0node@?$list@PEAVoutput_buffer@yaSSL@@@mySTL@@QEAA@PEAVoutput_buffer@yaSSL@@@Z 0000000140036c90 f i yassl:yassl_int.obj
 0001:00035cb0       ??$destroy@Unode@?$list@PEAVx509@yaSSL@@@mySTL@@@mySTL@@YAXPEAUnode@?$list@PEAVx509@yaSSL@@@0@@Z 0000000140036cb0 f i yassl:yassl_int.obj
 0001:00035cc0       ??$destroy@Unode@?$list@PEAVSSL_SESSION@yaSSL@@@mySTL@@@mySTL@@YAXPEAUnode@?$list@PEAVSSL_SESSION@yaSSL@@@0@@Z 0000000140036cc0 f i yassl:yassl_int.obj
 0001:00035cd0       ??$destroy@Unode@?$list@UThreadError@yaSSL@@@mySTL@@@mySTL@@YAXPEAUnode@?$list@UThreadError@yaSSL@@@0@@Z 0000000140036cd0 f i yassl:yassl_int.obj
 0001:00035ce0       ??$destroy@Unode@?$list@PEAVinput_buffer@yaSSL@@@mySTL@@@mySTL@@YAXPEAUnode@?$list@PEAVinput_buffer@yaSSL@@@0@@Z 0000000140036ce0 f i yassl:yassl_int.obj
 0001:00035cf0       ??$destroy@Unode@?$list@PEAVoutput_buffer@yaSSL@@@mySTL@@@mySTL@@YAXPEAUnode@?$list@PEAVoutput_buffer@yaSSL@@@0@@Z 0000000140036cf0 f i yassl:yassl_int.obj
 0001:00035d00       ??$swap@PEAVSSL_SESSION@yaSSL@@@mySTL@@YAXAEAPEAVSSL_SESSION@yaSSL@@0@Z 0000000140036d00 f i yassl:yassl_int.obj
 0001:00035d10       ??$destroy@U?$pair@HP6APEAUMessage@yaSSL@@XZ@mySTL@@@mySTL@@YAXPEAU?$pair@HP6APEAUMessage@yaSSL@@XZ@0@@Z 0000000140036d10 f i yassl:yassl_int.obj
 0001:00035d20       ??$destroy@U?$pair@HP6APEAVHandShakeBase@yaSSL@@XZ@mySTL@@@mySTL@@YAXPEAU?$pair@HP6APEAVHandShakeBase@yaSSL@@XZ@0@@Z 0000000140036d20 f i yassl:yassl_int.obj
 0001:00035d30       ??$destroy@U?$pair@HP6APEAUServerKeyBase@yaSSL@@XZ@mySTL@@@mySTL@@YAXPEAU?$pair@HP6APEAUServerKeyBase@yaSSL@@XZ@0@@Z 0000000140036d30 f i yassl:yassl_int.obj
 0001:00035d40       ??$destroy@U?$pair@HP6APEAUClientKeyBase@yaSSL@@XZ@mySTL@@@mySTL@@YAXPEAU?$pair@HP6APEAUClientKeyBase@yaSSL@@XZ@0@@Z 0000000140036d40 f i yassl:yassl_int.obj
 0001:00035d50       ??$swap@PEAVx509@yaSSL@@@mySTL@@YAXAEAPEAVx509@yaSSL@@0@Z 0000000140036d50 f i yassl:yassl_int.obj
 0001:00035d60       ??$swap@PEAVoutput_buffer@yaSSL@@@mySTL@@YAXAEAPEAVoutput_buffer@yaSSL@@0@Z 0000000140036d60 f i yassl:yassl_int.obj
 0001:00035d70       ??$swap@PEAVinput_buffer@yaSSL@@@mySTL@@YAXAEAPEAVinput_buffer@yaSSL@@0@Z 0000000140036d70 f i yassl:yassl_int.obj
 0001:00035d80       ?GetMemory@mySTL@@YAPEAX_K@Z 0000000140036d80 f i yassl:yassl_int.obj
 0001:00035d90       ??0sslHashes@yaSSL@@QEAA@XZ 0000000140036d90 f i yassl:yassl_int.obj
 0001:00035dc0       ?set_pending@SSL@yaSSL@@QEAAXE@Z 0000000140036dc0 f   yassl:yassl_int.obj
 0001:00036e80       ?set_random@SSL@yaSSL@@QEAAXPEBEW4ConnectionEnd@2@@Z 0000000140037e80 f   yassl:yassl_int.obj
 0001:00036ee0       ?set_preMaster@SSL@yaSSL@@QEAAXPEBEI@Z 0000000140037ee0 f   yassl:yassl_int.obj
 0001:00036f30       ?UnSetCompression@SSL@yaSSL@@QEAAXXZ 0000000140037f30 f   yassl:yassl_int.obj
 0001:00036f50       ?CompressionOn@SSL@yaSSL@@QEBA_NXZ 0000000140037f50 f   yassl:yassl_int.obj
 0001:00036f70       ?set_masterSecret@SSL@yaSSL@@QEAAXPEBE@Z 0000000140037f70 f   yassl:yassl_int.obj
 0001:00036fc0       ?set_sessionID@SSL@yaSSL@@QEAAXPEBE@Z 0000000140037fc0 f   yassl:yassl_int.obj
 0001:00037010       ?setKeys@SSL@yaSSL@@AEAAXXZ 0000000140038010 f   yassl:yassl_int.obj
 0001:000370c0       ?Send@SSL@yaSSL@@QEAAXPEBEI@Z 00000001400380c0 f   yassl:yassl_int.obj
 0001:00037170       ?get_SEQIncrement@SSL@yaSSL@@QEAAI_N@Z 0000000140038170 f   yassl:yassl_int.obj
 0001:000371b0       ?get_macSecret@SSL@yaSSL@@QEAAPEBE_N@Z 00000001400381b0 f   yassl:yassl_int.obj
 0001:00037200       ?verifyState@SSL@yaSSL@@QEAAXAEBURecordLayerHeader@2@@Z 0000000140038200 f   yassl:yassl_int.obj
 0001:00037260       ?verifyState@SSL@yaSSL@@QEAAXW4ClientState@2@@Z 0000000140038260 f   yassl:yassl_int.obj
 0001:00037290       ?verifyState@SSL@yaSSL@@QEAAXW4ServerState@2@@Z 0000000140038290 f   yassl:yassl_int.obj
 0001:000372c0       ?verfiyHandShakeComplete@SSL@yaSSL@@QEAAXXZ 00000001400382c0 f   yassl:yassl_int.obj
 0001:000372f0       ?verifyClientState@SSL@yaSSL@@AEAAXW4HandShakeType@2@@Z 00000001400382f0 f   yassl:yassl_int.obj
 0001:000373f0       ?verifyServerState@SSL@yaSSL@@AEAAXW4HandShakeType@2@@Z 00000001400383f0 f   yassl:yassl_int.obj
 0001:00037480       ?matchSuite@SSL@yaSSL@@QEAAXPEBEI@Z 0000000140038480 f   yassl:yassl_int.obj
 0001:00037560       ?GetMultiProtocol@SSL@yaSSL@@QEBA_NXZ 0000000140038560 f   yassl:yassl_int.obj
 0001:00037590       ?isTLS@SSL@yaSSL@@QEBA_NXZ 0000000140038590 f   yassl:yassl_int.obj
 0001:000375b0       ?isTLSv1_1@SSL@yaSSL@@QEBA_NXZ 00000001400385b0 f   yassl:yassl_int.obj
 0001:000375d0       ??1X509_NAME@yaSSL@@QEAA@XZ 00000001400385d0 f   yassl:yassl_int.obj
 0001:000375f0       ?GetBefore@X509@yaSSL@@QEAAPEAUASN1_STRING@2@XZ 00000001400385f0 f   yassl:yassl_int.obj
 0001:00037600       ?GetAfter@X509@yaSSL@@QEAAPEAUASN1_STRING@2@XZ 0000000140038600 f   yassl:yassl_int.obj
 0001:00037610       ?GetEntry@X509_NAME@yaSSL@@QEAAPEAUASN1_STRING@2@H@Z 0000000140038610 f   yassl:yassl_int.obj
 0001:000376d0       ??1StringHolder@yaSSL@@QEAA@XZ 00000001400386d0 f   yassl:yassl_int.obj
 0001:000376e0       ?begin@?$list@PEAVx509@yaSSL@@@mySTL@@QEBA?AViterator@12@XZ 00000001400386e0 f i yassl:yassl_int.obj
 0001:000376f0       ?end@?$list@PEAVx509@yaSSL@@@mySTL@@QEBA?AViterator@12@XZ 00000001400386f0 f i yassl:yassl_int.obj
 0001:00037700       ?begin@?$list@PEAVSSL_SESSION@yaSSL@@@mySTL@@QEBA?AViterator@12@XZ 0000000140038700 f i yassl:yassl_int.obj
 0001:00037710       ?end@?$list@PEAVSSL_SESSION@yaSSL@@@mySTL@@QEBA?AViterator@12@XZ 0000000140038710 f i yassl:yassl_int.obj
 0001:00037720       ?begin@?$list@UThreadError@yaSSL@@@mySTL@@QEBA?AViterator@12@XZ 0000000140038720 f i yassl:yassl_int.obj
 0001:00037730       ?end@?$list@UThreadError@yaSSL@@@mySTL@@QEBA?AViterator@12@XZ 0000000140038730 f i yassl:yassl_int.obj
 0001:00037740       ?begin@?$list@PEAVinput_buffer@yaSSL@@@mySTL@@QEBA?AViterator@12@XZ 0000000140038740 f i yassl:yassl_int.obj
 0001:00037750       ?end@?$list@PEAVinput_buffer@yaSSL@@@mySTL@@QEBA?AViterator@12@XZ 0000000140038750 f i yassl:yassl_int.obj
 0001:00037760       ?begin@?$list@PEAVoutput_buffer@yaSSL@@@mySTL@@QEBA?AViterator@12@XZ 0000000140038760 f i yassl:yassl_int.obj
 0001:00037770       ?end@?$list@PEAVoutput_buffer@yaSSL@@@mySTL@@QEBA?AViterator@12@XZ 0000000140038770 f i yassl:yassl_int.obj
 0001:00037780       ??Citerator@?$list@UThreadError@yaSSL@@@mySTL@@QEBAPEAUThreadError@yaSSL@@XZ 0000000140038780 f i yassl:yassl_int.obj
 0001:00037790       ??1?$vector_base@U?$pair@HP6APEAUMessage@yaSSL@@XZ@mySTL@@@mySTL@@QEAA@XZ 0000000140038790 f i yassl:yassl_int.obj
 0001:000377a0       ??1?$vector_base@U?$pair@HP6APEAVHandShakeBase@yaSSL@@XZ@mySTL@@@mySTL@@QEAA@XZ 00000001400387a0 f i yassl:yassl_int.obj
 0001:000377b0       ??1?$vector_base@U?$pair@HP6APEAUServerKeyBase@yaSSL@@XZ@mySTL@@@mySTL@@QEAA@XZ 00000001400387b0 f i yassl:yassl_int.obj
 0001:000377c0       ??1?$vector_base@U?$pair@HP6APEAUClientKeyBase@yaSSL@@XZ@mySTL@@@mySTL@@QEAA@XZ 00000001400387c0 f i yassl:yassl_int.obj
 0001:000377d0       ??$FreeArrayMemory@X@mySTL@@YAXPEAX@Z 00000001400387d0 f i yassl:yassl_int.obj
 0001:000377e0       ?push_back@?$list@PEAVx509@yaSSL@@@mySTL@@QEAAXPEAVx509@yaSSL@@@Z 00000001400387e0 f i yassl:yassl_int.obj
 0001:00037850       ?push_back@?$list@PEAVSSL_SESSION@yaSSL@@@mySTL@@QEAAXPEAVSSL_SESSION@yaSSL@@@Z 0000000140038850 f i yassl:yassl_int.obj
 0001:000378c0       ?push_back@?$list@UThreadError@yaSSL@@@mySTL@@QEAAXUThreadError@yaSSL@@@Z 00000001400388c0 f i yassl:yassl_int.obj
 0001:00037930       ?push_back@?$list@PEAVinput_buffer@yaSSL@@@mySTL@@QEAAXPEAVinput_buffer@yaSSL@@@Z 0000000140038930 f i yassl:yassl_int.obj
 0001:000379a0       ?push_back@?$list@PEAVoutput_buffer@yaSSL@@@mySTL@@QEAAXPEAVoutput_buffer@yaSSL@@@Z 00000001400389a0 f i yassl:yassl_int.obj
 0001:00037a10       ??$for_each@Viterator@?$list@PEAVinput_buffer@yaSSL@@@mySTL@@USumData@yassl_int_cpp_local1@yaSSL@@@mySTL@@YA?AUSumData@yassl_int_cpp_local1@yaSSL@@Viterator@?$list@PEAVinput_buffer@yaSSL@@@0@0U123@@Z 0000000140038a10 f i yassl:yassl_int.obj
 0001:00037a70       ??$ysDelete@Vinput_buffer@yaSSL@@@yaSSL@@YAXPEAVinput_buffer@0@@Z 0000000140038a70 f i yassl:yassl_int.obj
 0001:00037aa0       ??$for_each@Viterator@?$list@PEAVoutput_buffer@yaSSL@@@mySTL@@USumBuffer@yassl_int_cpp_local1@yaSSL@@@mySTL@@YA?AUSumBuffer@yassl_int_cpp_local1@yaSSL@@Viterator@?$list@PEAVoutput_buffer@yaSSL@@@0@0U123@@Z 0000000140038aa0 f i yassl:yassl_int.obj
 0001:00037b00       ??$ysDelete@Voutput_buffer@yaSSL@@@yaSSL@@YAXPEAVoutput_buffer@0@@Z 0000000140038b00 f i yassl:yassl_int.obj
 0001:00037b30       ??$find_if@Viterator@?$list@UThreadError@yaSSL@@@mySTL@@Uthr_match@yassl_int_cpp_local2@yaSSL@@@mySTL@@YA?AViterator@?$list@UThreadError@yaSSL@@@0@V120@0Uthr_match@yassl_int_cpp_local2@yaSSL@@@Z 0000000140038b30 f i yassl:yassl_int.obj
 0001:00037b50       ??$ysDelete@VDiffieHellman@yaSSL@@@yaSSL@@YAXPEAVDiffieHellman@0@@Z 0000000140038b50 f i yassl:yassl_int.obj
 0001:00037b80       ??$destroy@PEAU?$pair@HP6APEAUMessage@yaSSL@@XZ@mySTL@@@mySTL@@YAXPEAU?$pair@HP6APEAUMessage@yaSSL@@XZ@0@0@Z 0000000140038b80 f i yassl:yassl_int.obj
 0001:00037b90       ??$destroy@PEAU?$pair@HP6APEAVHandShakeBase@yaSSL@@XZ@mySTL@@@mySTL@@YAXPEAU?$pair@HP6APEAVHandShakeBase@yaSSL@@XZ@0@0@Z 0000000140038b90 f i yassl:yassl_int.obj
 0001:00037ba0       ??$destroy@PEAU?$pair@HP6APEAUServerKeyBase@yaSSL@@XZ@mySTL@@@mySTL@@YAXPEAU?$pair@HP6APEAUServerKeyBase@yaSSL@@XZ@0@0@Z 0000000140038ba0 f i yassl:yassl_int.obj
 0001:00037bb0       ??$destroy@PEAU?$pair@HP6APEAUClientKeyBase@yaSSL@@XZ@mySTL@@@mySTL@@YAXPEAU?$pair@HP6APEAUClientKeyBase@yaSSL@@XZ@0@0@Z 0000000140038bb0 f i yassl:yassl_int.obj
 0001:00037bc0       ??$checked_delete@Vx509@yaSSL@@@yaSSL@@YAXPEAVx509@0@@Z 0000000140038bc0 f i yassl:yassl_int.obj
 0001:00037bd0       ??$checked_delete@Voutput_buffer@yaSSL@@@yaSSL@@YAXPEAVoutput_buffer@0@@Z 0000000140038bd0 f i yassl:yassl_int.obj
 0001:00037be0       ??$checked_delete@Vinput_buffer@yaSSL@@@yaSSL@@YAXPEAVinput_buffer@0@@Z 0000000140038be0 f i yassl:yassl_int.obj
 0001:00037bf0       ?FreeMemory@mySTL@@YAXPEAX@Z 0000000140038bf0 f i yassl:yassl_int.obj
 0001:00037c00       ??1X509@yaSSL@@QEAA@XZ     0000000140038c00 f i yassl:yassl_int.obj
 0001:00037c40       ?storeKeys@SSL@yaSSL@@AEAAXPEBE@Z 0000000140038c40 f   yassl:yassl_int.obj
 0001:00037d40       ?bufferedData@SSL@yaSSL@@QEAAIXZ 0000000140038d40 f   yassl:yassl_int.obj
 0001:00037d70       ?PeekData@SSL@yaSSL@@QEAAXAEAVData@2@@Z 0000000140038d70 f   yassl:yassl_int.obj
 0001:00037ed0       ?verifyState@SSL@yaSSL@@QEAAXAEBVHandShakeHeader@2@@Z 0000000140038ed0 f   yassl:yassl_int.obj
 0001:00037f50       ?addData@SSL@yaSSL@@QEAAXPEAVinput_buffer@2@@Z 0000000140038f50 f   yassl:yassl_int.obj
 0001:00037f90       ?addBuffer@SSL@yaSSL@@QEAAXPEAVoutput_buffer@2@@Z 0000000140038f90 f   yassl:yassl_int.obj
 0001:00037fb0       ?AddCA@SSL_CTX@yaSSL@@QEAAXPEAVx509@2@@Z 0000000140038fb0 f   yassl:yassl_int.obj
 0001:00037fc0       ??1Crypto@yaSSL@@QEAA@XZ   0000000140038fc0 f   yassl:yassl_int.obj
 0001:00038000       ??0X509@yaSSL@@QEAA@PEBD_K010H0H@Z 0000000140039000 f   yassl:yassl_int.obj
 0001:00038060       ??1?$vector@U?$pair@HP6APEAUMessage@yaSSL@@XZ@mySTL@@@mySTL@@QEAA@XZ 0000000140039060 f i yassl:yassl_int.obj
 0001:00038070       ??1?$vector@U?$pair@HP6APEAVHandShakeBase@yaSSL@@XZ@mySTL@@@mySTL@@QEAA@XZ 0000000140039070 f i yassl:yassl_int.obj
 0001:00038080       ??1?$vector@U?$pair@HP6APEAUServerKeyBase@yaSSL@@XZ@mySTL@@@mySTL@@QEAA@XZ 0000000140039080 f i yassl:yassl_int.obj
 0001:00038090       ??1?$vector@U?$pair@HP6APEAUClientKeyBase@yaSSL@@XZ@mySTL@@@mySTL@@QEAA@XZ 0000000140039090 f i yassl:yassl_int.obj
 0001:000380a0       ??0?$vector@U?$pair@HP6APEAUMessage@yaSSL@@XZ@mySTL@@@mySTL@@QEAA@XZ 00000001400390a0 f i yassl:yassl_int.obj
 0001:000380c0       ??0?$vector@U?$pair@HP6APEAVHandShakeBase@yaSSL@@XZ@mySTL@@@mySTL@@QEAA@XZ 00000001400390c0 f i yassl:yassl_int.obj
 0001:000380e0       ??0?$vector@U?$pair@HP6APEAUServerKeyBase@yaSSL@@XZ@mySTL@@@mySTL@@QEAA@XZ 00000001400390e0 f i yassl:yassl_int.obj
 0001:00038100       ??0?$vector@U?$pair@HP6APEAUClientKeyBase@yaSSL@@XZ@mySTL@@@mySTL@@QEAA@XZ 0000000140039100 f i yassl:yassl_int.obj
 0001:00038120       ?Destroy@?$auto_ptr@Voutput_buffer@yaSSL@@@mySTL@@AEAAXXZ 0000000140039120 f i yassl:yassl_int.obj
 0001:00038130       ??1?$list@PEAVx509@yaSSL@@@mySTL@@QEAA@XZ 0000000140039130 f i yassl:yassl_int.obj
 0001:00038160       ??1?$list@PEAVSSL_SESSION@yaSSL@@@mySTL@@QEAA@XZ 0000000140039160 f i yassl:yassl_int.obj
 0001:00038190       ??1?$list@UThreadError@yaSSL@@@mySTL@@QEAA@XZ 0000000140039190 f i yassl:yassl_int.obj
 0001:000381c0       ??1?$list@PEAVinput_buffer@yaSSL@@@mySTL@@QEAA@XZ 00000001400391c0 f i yassl:yassl_int.obj
 0001:000381f0       ?pop_front@?$list@PEAVinput_buffer@yaSSL@@@mySTL@@QEAAXXZ 00000001400391f0 f i yassl:yassl_int.obj
 0001:00038240       ??1?$list@PEAVoutput_buffer@yaSSL@@@mySTL@@QEAA@XZ 0000000140039240 f i yassl:yassl_int.obj
 0001:00038270       ?pop_front@?$list@PEAVoutput_buffer@yaSSL@@@mySTL@@QEAAXXZ 0000000140039270 f i yassl:yassl_int.obj
 0001:000382c0       ??_GX509@yaSSL@@QEAAPEAXI@Z 00000001400392c0 f i yassl:yassl_int.obj
 0001:00038310       ?pop_front@?$list@PEAVSSL_SESSION@yaSSL@@@mySTL@@QEAAXXZ 0000000140039310 f i yassl:yassl_int.obj
 0001:00038360       ?pop_back@?$list@PEAVSSL_SESSION@yaSSL@@@mySTL@@QEAAXXZ 0000000140039360 f i yassl:yassl_int.obj
 0001:000383c0       ?pop_front@?$list@UThreadError@yaSSL@@@mySTL@@QEAAXXZ 00000001400393c0 f i yassl:yassl_int.obj
 0001:00038410       ?pop_back@?$list@UThreadError@yaSSL@@@mySTL@@QEAAXXZ 0000000140039410 f i yassl:yassl_int.obj
 0001:00038470       ??$?RVx509@yaSSL@@@del_ptr_zero@yaSSL@@QEBAXAEAPEAVx509@1@@Z 0000000140039470 f i yassl:yassl_int.obj
 0001:00038480       ??$?RVoutput_buffer@yaSSL@@@del_ptr_zero@yaSSL@@QEBAXAEAPEAVoutput_buffer@1@@Z 0000000140039480 f i yassl:yassl_int.obj
 0001:00038490       ??$?RVinput_buffer@yaSSL@@@del_ptr_zero@yaSSL@@QEBAXAEAPEAVinput_buffer@1@@Z 0000000140039490 f i yassl:yassl_int.obj
 0001:000384a0       ??0Sessions@yaSSL@@AEAA@XZ 00000001400394a0 f i yassl:yassl_int.obj
 0001:000384e0       ??0Errors@yaSSL@@AEAA@XZ   00000001400394e0 f i yassl:yassl_int.obj
 0001:00038510       ??1Errors@yaSSL@@QEAA@XZ   0000000140039510 f i yassl:yassl_int.obj
 0001:00038530       ??1?$Factory@UMessage@yaSSL@@HP6APEAU12@XZ@yaSSL@@QEAA@XZ 0000000140039530 f i yassl:yassl_int.obj
 0001:00038540       ??1?$Factory@VHandShakeBase@yaSSL@@HP6APEAV12@XZ@yaSSL@@QEAA@XZ 0000000140039540 f i yassl:yassl_int.obj
 0001:00038550       ??1?$Factory@UServerKeyBase@yaSSL@@HP6APEAU12@XZ@yaSSL@@QEAA@XZ 0000000140039550 f i yassl:yassl_int.obj
 0001:00038560       ??1?$Factory@UClientKeyBase@yaSSL@@HP6APEAU12@XZ@yaSSL@@QEAA@XZ 0000000140039560 f i yassl:yassl_int.obj
 0001:00038570       ?deriveKeys@SSL@yaSSL@@QEAAXXZ 0000000140039570 f   yassl:yassl_int.obj
 0001:000387f0       ?deriveTLSKeys@SSL@yaSSL@@QEAAXXZ 00000001400397f0 f   yassl:yassl_int.obj
 0001:00038930       ?fillData@SSL@yaSSL@@QEAAXAEAVData@2@@Z 0000000140039930 f   yassl:yassl_int.obj
 0001:00038ad0       ?flushBuffer@SSL@yaSSL@@QEAAXXZ 0000000140039ad0 f   yassl:yassl_int.obj
 0001:00038be0       ?CopyX509@SSL_SESSION@yaSSL@@AEAAXPEAVX509@2@@Z 0000000140039be0 f   yassl:yassl_int.obj
 0001:00038cc0       ??0SSL_SESSION@yaSSL@@QEAA@AEBVSSL@1@AEAVRandomPool@1@@Z 0000000140039cc0 f   yassl:yassl_int.obj
 0001:00038da0       ?GetSessions@yaSSL@@YAAEAVSessions@1@XZ 0000000140039da0 f   yassl:yassl_int.obj
 0001:00038e20       ?GetErrors@yaSSL@@YAAEAVErrors@1@XZ 0000000140039e20 f   yassl:yassl_int.obj
 0001:00038e90       ??0SSL_CTX@yaSSL@@QEAA@PEAVSSL_METHOD@1@@Z 0000000140039e90 f   yassl:yassl_int.obj
 0001:00038f80       ??0Buffers@yaSSL@@QEAA@XZ  0000000140039f80 f   yassl:yassl_int.obj
 0001:00038fb0       ??0?$Factory@UMessage@yaSSL@@HP6APEAU12@XZ@yaSSL@@QEAA@P6AXAEAV01@@Z@Z 0000000140039fb0 f i yassl:yassl_int.obj
 0001:00038fe0       ??0?$Factory@VHandShakeBase@yaSSL@@HP6APEAV12@XZ@yaSSL@@QEAA@P6AXAEAV01@@Z@Z 0000000140039fe0 f i yassl:yassl_int.obj
 0001:00039010       ??0?$Factory@UServerKeyBase@yaSSL@@HP6APEAU12@XZ@yaSSL@@QEAA@P6AXAEAV01@@Z@Z 000000014003a010 f i yassl:yassl_int.obj
 0001:00039040       ??0?$Factory@UClientKeyBase@yaSSL@@HP6APEAU12@XZ@yaSSL@@QEAA@P6AXAEAV01@@Z@Z 000000014003a040 f i yassl:yassl_int.obj
 0001:00039070       ??1?$auto_ptr@Voutput_buffer@yaSSL@@@mySTL@@QEAA@XZ 000000014003a070 f i yassl:yassl_int.obj
 0001:00039080       ?erase@?$list@PEAVSSL_SESSION@yaSSL@@@mySTL@@QEAA_NViterator@12@@Z 000000014003a080 f i yassl:yassl_int.obj
 0001:000390f0       ?erase@?$list@UThreadError@yaSSL@@@mySTL@@QEAA_NViterator@12@@Z 000000014003a0f0 f i yassl:yassl_int.obj
 0001:00039160       ??$ysDelete@VX509@yaSSL@@@yaSSL@@YAXPEAVX509@0@@Z 000000014003a160 f i yassl:yassl_int.obj
 0001:000391a0       ??$for_each@Viterator@?$list@PEAVx509@yaSSL@@@mySTL@@Udel_ptr_zero@yaSSL@@@mySTL@@YA?AUdel_ptr_zero@yaSSL@@Viterator@?$list@PEAVx509@yaSSL@@@0@0U12@@Z 000000014003a1a0 f i yassl:yassl_int.obj
 0001:00039200       ??$for_each@Viterator@?$list@PEAVoutput_buffer@yaSSL@@@mySTL@@Udel_ptr_zero@yaSSL@@@mySTL@@YA?AUdel_ptr_zero@yaSSL@@Viterator@?$list@PEAVoutput_buffer@yaSSL@@@0@0U12@@Z 000000014003a200 f i yassl:yassl_int.obj
 0001:00039260       ??$for_each@Viterator@?$list@PEAVinput_buffer@yaSSL@@@mySTL@@Udel_ptr_zero@yaSSL@@@mySTL@@YA?AUdel_ptr_zero@yaSSL@@Viterator@?$list@PEAVinput_buffer@yaSSL@@@0@0U12@@Z 000000014003a260 f i yassl:yassl_int.obj
 0001:000392c0       ??_GErrors@yaSSL@@QEAAPEAXI@Z 000000014003a2c0 f i yassl:yassl_int.obj
 0001:00039300       ??1sslFactory@yaSSL@@QEAA@XZ 000000014003a300 f i yassl:yassl_int.obj
 0001:00039340       ??0sslFactory@yaSSL@@AEAA@XZ 000000014003a340 f   yassl:yassl_int.obj
 0001:000393b0       ?makeTLSMasterSecret@SSL@yaSSL@@QEAAXXZ 000000014003a3b0 f   yassl:yassl_int.obj
 0001:00039490       ?SendWriteBuffered@SSL@yaSSL@@QEAAXXZ 000000014003a490 f   yassl:yassl_int.obj
 0001:000394f0       ??4SSL_SESSION@yaSSL@@QEAAAEAV01@AEBV01@@Z 000000014003a4f0 f   yassl:yassl_int.obj
 0001:000395a0       ??1SSL_SESSION@yaSSL@@QEAA@XZ 000000014003a5a0 f   yassl:yassl_int.obj
 0001:000395d0       ?GetSSL_Factory@yaSSL@@YAAEAVsslFactory@1@XZ 000000014003a5d0 f   yassl:yassl_int.obj
 0001:00039620       ?Remove@Errors@yaSSL@@QEAAXXZ 000000014003a620 f   yassl:yassl_int.obj
 0001:00039680       ?Lookup@Errors@yaSSL@@QEAAH_N@Z 000000014003a680 f   yassl:yassl_int.obj
 0001:00039710       ?Add@Errors@yaSSL@@QEAAXH@Z 000000014003a710 f   yassl:yassl_int.obj
 0001:00039760       ??1SSL_CTX@yaSSL@@QEAA@XZ  000000014003a760 f   yassl:yassl_int.obj
 0001:000397d0       ??1Buffers@yaSSL@@QEAA@XZ  000000014003a7d0 f   yassl:yassl_int.obj
 0001:00039840       ??0Security@yaSSL@@QEAA@UProtocolVersion@1@AEAVRandomPool@1@W4ConnectionEnd@1@AEBUCiphers@1@PEAVSSL_CTX@1@_N@Z 000000014003a840 f   yassl:yassl_int.obj
 0001:000398c0       ??$ysDelete@VErrors@yaSSL@@@yaSSL@@YAXPEAVErrors@0@@Z 000000014003a8c0 f i yassl:yassl_int.obj
 0001:000398f0       ??_GsslFactory@yaSSL@@QEAAPEAXI@Z 000000014003a8f0 f i yassl:yassl_int.obj
 0001:00039940       ??_GSSL_SESSION@yaSSL@@QEAAPEAXI@Z 000000014003a940 f i yassl:yassl_int.obj
 0001:00039970       ?makeMasterSecret@SSL@yaSSL@@QEAAXXZ 000000014003a970 f   yassl:yassl_int.obj
 0001:00039be0       ?getFactory@SSL@yaSSL@@QEBAAEBVsslFactory@2@XZ 000000014003abe0 f   yassl:yassl_int.obj
 0001:00039bf0       ??$ysDelete@VsslFactory@yaSSL@@@yaSSL@@YAXPEAVsslFactory@0@@Z 000000014003abf0 f i yassl:yassl_int.obj
 0001:00039c30       ??$ysDelete@VSSL_SESSION@yaSSL@@@yaSSL@@YAXPEAVSSL_SESSION@0@@Z 000000014003ac30 f i yassl:yassl_int.obj
 0001:00039c60       ??0SSL@yaSSL@@QEAA@PEAVSSL_CTX@1@@Z 000000014003ac60 f   yassl:yassl_int.obj
 0001:00039f40       ??$checked_delete@VSSL_SESSION@yaSSL@@@yaSSL@@YAXPEAVSSL_SESSION@0@@Z 000000014003af40 f i yassl:yassl_int.obj
 0001:00039f50       ??$?RVSSL_SESSION@yaSSL@@@del_ptr_zero@yaSSL@@QEBAXAEAPEAVSSL_SESSION@1@@Z 000000014003af50 f i yassl:yassl_int.obj
 0001:00039f60       ?lookup@Sessions@yaSSL@@QEAAPEAVSSL_SESSION@2@PEBEPEAV32@@Z 000000014003af60 f   yassl:yassl_int.obj
 0001:0003a030       ?remove@Sessions@yaSSL@@QEAAXPEBE@Z 000000014003b030 f   yassl:yassl_int.obj
 0001:0003a0a0       ?Flush@Sessions@yaSSL@@QEAAXXZ 000000014003b0a0 f   yassl:yassl_int.obj
 0001:0003a140       ??$for_each@Viterator@?$list@PEAVSSL_SESSION@yaSSL@@@mySTL@@Udel_ptr_zero@yaSSL@@@mySTL@@YA?AUdel_ptr_zero@yaSSL@@Viterator@?$list@PEAVSSL_SESSION@yaSSL@@@0@0U12@@Z 000000014003b140 f i yassl:yassl_int.obj
 0001:0003a1a0       ?set_session@SSL@yaSSL@@QEAAXPEAVSSL_SESSION@2@@Z 000000014003b1a0 f   yassl:yassl_int.obj
 0001:0003a260       ?add@Sessions@yaSSL@@QEAAXAEBVSSL@2@@Z 000000014003b260 f   yassl:yassl_int.obj
 0001:0003a310       ??1Sessions@yaSSL@@QEAA@XZ 000000014003b310 f   yassl:yassl_int.obj
 0001:0003a350       ??_GSessions@yaSSL@@QEAAPEAXI@Z 000000014003b350 f i yassl:yassl_int.obj
 0001:0003a380       ??$ysDelete@VSessions@yaSSL@@@yaSSL@@YAXPEAVSessions@0@@Z 000000014003b380 f i yassl:yassl_int.obj
 0001:0003a3b0       yayaSSL_CleanUp            000000014003b3b0 f   yassl:yassl_int.obj
 0001:0003a400       ??1Digest@yaSSL@@UEAA@XZ   000000014003b400 f i yassl:crypto_wrapper.obj
 0001:0003a410       ??_GDigest@yaSSL@@UEAAPEAXI@Z 000000014003b410 f i yassl:crypto_wrapper.obj
 0001:0003a410       ??_EDigest@yaSSL@@UEAAPEAXI@Z 000000014003b410 f i yassl:crypto_wrapper.obj
 0001:0003a440       ??1BulkCipher@yaSSL@@UEAA@XZ 000000014003b440 f i yassl:crypto_wrapper.obj
 0001:0003a450       ??_EBulkCipher@yaSSL@@UEAAPEAXI@Z 000000014003b450 f i yassl:crypto_wrapper.obj
 0001:0003a450       ??_GBulkCipher@yaSSL@@UEAAPEAXI@Z 000000014003b450 f i yassl:crypto_wrapper.obj
 0001:0003a480       ??1Auth@yaSSL@@UEAA@XZ     000000014003b480 f i yassl:crypto_wrapper.obj
 0001:0003a490       ??_EAuth@yaSSL@@UEAAPEAXI@Z 000000014003b490 f i yassl:crypto_wrapper.obj
 0001:0003a490       ??_GAuth@yaSSL@@UEAAPEAXI@Z 000000014003b490 f i yassl:crypto_wrapper.obj
 0001:0003a4c0       ?BitsToBytes@TaoCrypt@@YAII@Z 000000014003b4c0 f i yassl:crypto_wrapper.obj
 0001:0003a4d0       ?What@Error@TaoCrypt@@QEBA?AW4ErrorNumber@2@XZ 000000014003b4d0 f i yassl:crypto_wrapper.obj
 0001:0003a4e0       ??0SHA@TaoCrypt@@QEAA@XZ   000000014003b4e0 f i yassl:crypto_wrapper.obj
 0001:0003a520       ?getByteOrder@SHA@TaoCrypt@@UEBA?AW4ByteOrder@2@XZ 000000014003b520 f i yassl:crypto_wrapper.obj
 0001:0003a530       ?getBlockSize@SHA@TaoCrypt@@UEBAIXZ 000000014003b530 f i yassl:crypto_wrapper.obj
 0001:0003a540       ?getDigestSize@SHA@TaoCrypt@@UEBAIXZ 000000014003b540 f i yassl:crypto_wrapper.obj
 0001:0003a550       ?getPadSize@SHA@TaoCrypt@@UEBAIXZ 000000014003b550 f i yassl:crypto_wrapper.obj
 0001:0003a560       ??1SHA@TaoCrypt@@UEAA@XZ   000000014003b560 f i yassl:crypto_wrapper.obj
 0001:0003a570       ??0RIPEMD160@TaoCrypt@@QEAA@XZ 000000014003b570 f i yassl:crypto_wrapper.obj
 0001:0003a5b0       ?getByteOrder@RIPEMD160@TaoCrypt@@UEBA?AW4ByteOrder@2@XZ 000000014003b5b0 f i yassl:crypto_wrapper.obj
 0001:0003a5c0       ?getBlockSize@RIPEMD160@TaoCrypt@@UEBAIXZ 000000014003b5c0 f i yassl:crypto_wrapper.obj
 0001:0003a5d0       ?getDigestSize@RIPEMD160@TaoCrypt@@UEBAIXZ 000000014003b5d0 f i yassl:crypto_wrapper.obj
 0001:0003a5e0       ?getPadSize@RIPEMD160@TaoCrypt@@UEBAIXZ 000000014003b5e0 f i yassl:crypto_wrapper.obj
 0001:0003a5f0       ??1RIPEMD160@TaoCrypt@@UEAA@XZ 000000014003b5f0 f i yassl:crypto_wrapper.obj
 0001:0003a600       ??0Mode_BASE@TaoCrypt@@QEAA@HW4CipherDir@1@W4Mode@1@@Z 000000014003b600 f i yassl:crypto_wrapper.obj
 0001:0003a630       ??1Mode_BASE@TaoCrypt@@UEAA@XZ 000000014003b630 f i yassl:crypto_wrapper.obj
 0001:0003a640       ?SetIV@Mode_BASE@TaoCrypt@@QEAAXPEBE@Z 000000014003b640 f i yassl:crypto_wrapper.obj
 0001:0003a650       ??_GMode_BASE@TaoCrypt@@UEAAPEAXI@Z 000000014003b650 f i yassl:crypto_wrapper.obj
 0001:0003a650       ??_EMode_BASE@TaoCrypt@@UEAAPEAXI@Z 000000014003b650 f i yassl:crypto_wrapper.obj
 0001:0003a680       ?ECB_Process@Mode_BASE@TaoCrypt@@IEAAXPEAEPEBEI@Z 000000014003b680 f i yassl:crypto_wrapper.obj
 0001:0003a6f0       ?CBC_Encrypt@Mode_BASE@TaoCrypt@@IEAAXPEAEPEBEI@Z 000000014003b6f0 f i yassl:crypto_wrapper.obj
 0001:0003a780       ?CBC_Decrypt@Mode_BASE@TaoCrypt@@IEAAXPEAEPEBEI@Z 000000014003b780 f i yassl:crypto_wrapper.obj
 0001:0003a880       ??0DES@TaoCrypt@@QEAA@W4CipherDir@1@W4Mode@1@@Z 000000014003b880 f i yassl:crypto_wrapper.obj
 0001:0003a8b0       ??1DES@TaoCrypt@@UEAA@XZ   000000014003b8b0 f i yassl:crypto_wrapper.obj
 0001:0003a8c0       ??0DES_EDE3@TaoCrypt@@QEAA@W4CipherDir@1@W4Mode@1@@Z 000000014003b8c0 f i yassl:crypto_wrapper.obj
 0001:0003a8f0       ?SetIV@DES_EDE3@TaoCrypt@@QEAAXPEBE@Z 000000014003b8f0 f i yassl:crypto_wrapper.obj
 0001:0003a900       ??1DES_EDE3@TaoCrypt@@UEAA@XZ 000000014003b900 f i yassl:crypto_wrapper.obj
 0001:0003a910       ??0ARC4@TaoCrypt@@QEAA@XZ  000000014003b910 f i yassl:crypto_wrapper.obj
 0001:0003a920       ??0AES@TaoCrypt@@QEAA@W4CipherDir@1@W4Mode@1@@Z 000000014003b920 f i yassl:crypto_wrapper.obj
 0001:0003a950       ?SetIV@AES@TaoCrypt@@QEAAXPEBE@Z 000000014003b950 f i yassl:crypto_wrapper.obj
 0001:0003a960       ??1AES@TaoCrypt@@UEAA@XZ   000000014003b960 f i yassl:crypto_wrapper.obj
 0001:0003a970       ?GetError@OS_Seed@TaoCrypt@@QEBA?AUError@2@XZ 000000014003b970 f i yassl:crypto_wrapper.obj
 0001:0003a980       ??1RandomNumberGenerator@TaoCrypt@@QEAA@XZ 000000014003b980 f i yassl:crypto_wrapper.obj
 0001:0003a990       ?GetError@RandomNumberGenerator@TaoCrypt@@QEBA?AW4ErrorNumber@2@XZ 000000014003b990 f i yassl:crypto_wrapper.obj
 0001:0003a9a0       ?Ref@Integer@TaoCrypt@@QEAAAEAV12@XZ 000000014003b9a0 f i yassl:crypto_wrapper.obj
 0001:0003a9b0       ??0PK_Lengths@TaoCrypt@@QEAA@AEBVInteger@1@@Z 000000014003b9b0 f i yassl:crypto_wrapper.obj
 0001:0003a9c0       ?PaddedBlockBitLength@PK_Lengths@TaoCrypt@@QEBAIXZ 000000014003b9c0 f i yassl:crypto_wrapper.obj
 0001:0003a9e0       ?PaddedBlockByteLength@PK_Lengths@TaoCrypt@@QEBAIXZ 000000014003b9e0 f i yassl:crypto_wrapper.obj
 0001:0003aa00       ?FixedCiphertextLength@PK_Lengths@TaoCrypt@@QEBAIXZ 000000014003ba00 f i yassl:crypto_wrapper.obj
 0001:0003aa10       ?Initialize@RSA_PublicKey@TaoCrypt@@QEAAXAEBVInteger@2@0@Z 000000014003ba10 f i yassl:crypto_wrapper.obj
 0001:0003aa40       ?GetModulus@RSA_PublicKey@TaoCrypt@@QEBAAEBVInteger@2@XZ 000000014003ba40 f i yassl:crypto_wrapper.obj
 0001:0003aa50       ?FixedCiphertextLength@RSA_PublicKey@TaoCrypt@@QEAAIXZ 000000014003ba50 f i yassl:crypto_wrapper.obj
 0001:0003aa60       ?Swap@RSA_PublicKey@TaoCrypt@@QEAAXAEAV12@@Z 000000014003ba60 f i yassl:crypto_wrapper.obj
 0001:0003aa90       ?GetPrivateExponent@RSA_PrivateKey@TaoCrypt@@QEBAAEBVInteger@2@XZ 000000014003ba90 f i yassl:crypto_wrapper.obj
 0001:0003aaa0       ?Swap@DH@TaoCrypt@@QEAAXAEAV12@@Z 000000014003baa0 f i yassl:crypto_wrapper.obj
 0001:0003aad0       ?SetP@DH@TaoCrypt@@QEAAXAEBVInteger@2@@Z 000000014003bad0 f i yassl:crypto_wrapper.obj
 0001:0003aae0       ?SetG@DH@TaoCrypt@@QEAAXAEBVInteger@2@@Z 000000014003bae0 f i yassl:crypto_wrapper.obj
 0001:0003aaf0       ?GetP@DH@TaoCrypt@@QEAAAEAVInteger@2@XZ 000000014003baf0 f i yassl:crypto_wrapper.obj
 0001:0003ab00       ?GetG@DH@TaoCrypt@@QEAAAEAVInteger@2@XZ 000000014003bb00 f i yassl:crypto_wrapper.obj
 0001:0003ab10       ?GetByteLength@DH@TaoCrypt@@QEBAIXZ 000000014003bb10 f i yassl:crypto_wrapper.obj
 0001:0003ab20       ??0MD5Impl@MD5@yaSSL@@QEAA@XZ 000000014003bb20 f i yassl:crypto_wrapper.obj
 0001:0003ab60       ??0MD5Impl@MD5@yaSSL@@QEAA@AEBV1TaoCrypt@@@Z 000000014003bb60 f i yassl:crypto_wrapper.obj
 0001:0003ab80       ??0Digest@yaSSL@@QEAA@XZ   000000014003bb80 f i yassl:crypto_wrapper.obj
 0001:0003ab90       ??0MD5@yaSSL@@QEAA@AEBV01@@Z 000000014003bb90 f   yassl:crypto_wrapper.obj
 0001:0003ac00       ??4MD5@yaSSL@@QEAAAEAV01@AEBV01@@Z 000000014003bc00 f   yassl:crypto_wrapper.obj
 0001:0003ac20       ?get_digestSize@MD5@yaSSL@@UEBAIXZ 000000014003bc20 f   yassl:crypto_wrapper.obj
 0001:0003ac30       ?get_padSize@MD5@yaSSL@@UEBAIXZ 000000014003bc30 f   yassl:crypto_wrapper.obj
 0001:0003ac40       ?get_digest@MD5@yaSSL@@UEAAXPEAEPEBEI@Z 000000014003bc40 f   yassl:crypto_wrapper.obj
 0001:0003ac80       ?get_digest@MD5@yaSSL@@UEAAXPEAE@Z 000000014003bc80 f   yassl:crypto_wrapper.obj
 0001:0003ac90       ?update@MD5@yaSSL@@UEAAXPEBEI@Z 000000014003bc90 f   yassl:crypto_wrapper.obj
 0001:0003aca0       ??0SHAImpl@SHA@yaSSL@@QEAA@XZ 000000014003bca0 f i yassl:crypto_wrapper.obj
 0001:0003ace0       ??0SHAImpl@SHA@yaSSL@@QEAA@AEBV1TaoCrypt@@@Z 000000014003bce0 f i yassl:crypto_wrapper.obj
 0001:0003ad00       ??0SHA@yaSSL@@QEAA@XZ      000000014003bd00 f   yassl:crypto_wrapper.obj
 0001:0003ad80       ??0SHA@yaSSL@@QEAA@AEBV01@@Z 000000014003bd80 f   yassl:crypto_wrapper.obj
 0001:0003adf0       ??4SHA@yaSSL@@QEAAAEAV01@AEBV01@@Z 000000014003bdf0 f   yassl:crypto_wrapper.obj
 0001:0003ae10       ?get_digestSize@SHA@yaSSL@@UEBAIXZ 000000014003be10 f   yassl:crypto_wrapper.obj
 0001:0003ae20       ?get_padSize@SHA@yaSSL@@UEBAIXZ 000000014003be20 f   yassl:crypto_wrapper.obj
 0001:0003ae30       ?get_digest@SHA@yaSSL@@UEAAXPEAEPEBEI@Z 000000014003be30 f   yassl:crypto_wrapper.obj
 0001:0003ae70       ?get_digest@SHA@yaSSL@@UEAAXPEAE@Z 000000014003be70 f   yassl:crypto_wrapper.obj
 0001:0003ae80       ?update@SHA@yaSSL@@UEAAXPEBEI@Z 000000014003be80 f   yassl:crypto_wrapper.obj
 0001:0003ae90       ??0RMDImpl@RMD@yaSSL@@QEAA@XZ 000000014003be90 f i yassl:crypto_wrapper.obj
 0001:0003aed0       ??0RMDImpl@RMD@yaSSL@@QEAA@AEBVRIPEMD160@TaoCrypt@@@Z 000000014003bed0 f i yassl:crypto_wrapper.obj
 0001:0003aef0       ??0RMD@yaSSL@@QEAA@XZ      000000014003bef0 f   yassl:crypto_wrapper.obj
 0001:0003af70       ??0RMD@yaSSL@@QEAA@AEBV01@@Z 000000014003bf70 f   yassl:crypto_wrapper.obj
 0001:0003afe0       ??4RMD@yaSSL@@QEAAAEAV01@AEBV01@@Z 000000014003bfe0 f   yassl:crypto_wrapper.obj
 0001:0003b000       ?get_digestSize@RMD@yaSSL@@UEBAIXZ 000000014003c000 f   yassl:crypto_wrapper.obj
 0001:0003b010       ?get_padSize@RMD@yaSSL@@UEBAIXZ 000000014003c010 f   yassl:crypto_wrapper.obj
 0001:0003b020       ?get_digest@RMD@yaSSL@@UEAAXPEAEPEBEI@Z 000000014003c020 f   yassl:crypto_wrapper.obj
 0001:0003b060       ?get_digest@RMD@yaSSL@@UEAAXPEAE@Z 000000014003c060 f   yassl:crypto_wrapper.obj
 0001:0003b070       ?update@RMD@yaSSL@@UEAAXPEBEI@Z 000000014003c070 f   yassl:crypto_wrapper.obj
 0001:0003b080       ??1?$HMAC@VMD5@TaoCrypt@@@TaoCrypt@@QEAA@XZ 000000014003c080 f i yassl:crypto_wrapper.obj
 0001:0003b090       ?get_digestSize@HMAC_MD5@yaSSL@@UEBAIXZ 000000014003c090 f   yassl:crypto_wrapper.obj
 0001:0003b0a0       ?get_padSize@HMAC_MD5@yaSSL@@UEBAIXZ 000000014003c0a0 f   yassl:crypto_wrapper.obj
 0001:0003b0b0       ??1?$HMAC@VSHA@TaoCrypt@@@TaoCrypt@@QEAA@XZ 000000014003c0b0 f i yassl:crypto_wrapper.obj
 0001:0003b0c0       ?get_digestSize@HMAC_SHA@yaSSL@@UEBAIXZ 000000014003c0c0 f   yassl:crypto_wrapper.obj
 0001:0003b0d0       ?get_padSize@HMAC_SHA@yaSSL@@UEBAIXZ 000000014003c0d0 f   yassl:crypto_wrapper.obj
 0001:0003b0e0       ??1?$HMAC@VRIPEMD160@TaoCrypt@@@TaoCrypt@@QEAA@XZ 000000014003c0e0 f i yassl:crypto_wrapper.obj
 0001:0003b0f0       ?get_digestSize@HMAC_RMD@yaSSL@@UEBAIXZ 000000014003c0f0 f   yassl:crypto_wrapper.obj
 0001:0003b100       ?get_padSize@HMAC_RMD@yaSSL@@UEBAIXZ 000000014003c100 f   yassl:crypto_wrapper.obj
 0001:0003b110       ??0BulkCipher@yaSSL@@QEAA@XZ 000000014003c110 f i yassl:crypto_wrapper.obj
 0001:0003b120       ??1?$BlockCipher@$0A@VDES@TaoCrypt@@$00@TaoCrypt@@QEAA@XZ 000000014003c120 f i yassl:crypto_wrapper.obj
 0001:0003b130       ??1?$BlockCipher@$00VDES@TaoCrypt@@$00@TaoCrypt@@QEAA@XZ 000000014003c130 f i yassl:crypto_wrapper.obj
 0001:0003b140       ??1?$BlockCipher@$0A@VDES_EDE3@TaoCrypt@@$00@TaoCrypt@@QEAA@XZ 000000014003c140 f i yassl:crypto_wrapper.obj
 0001:0003b150       ??1?$BlockCipher@$00VDES_EDE3@TaoCrypt@@$00@TaoCrypt@@QEAA@XZ 000000014003c150 f i yassl:crypto_wrapper.obj
 0001:0003b160       ??0RC4Impl@RC4@yaSSL@@QEAA@XZ 000000014003c160 f i yassl:crypto_wrapper.obj
 0001:0003b170       ?set_encryptKey@RC4@yaSSL@@UEAAXPEBE0@Z 000000014003c170 f   yassl:crypto_wrapper.obj
 0001:0003b180       ?set_decryptKey@RC4@yaSSL@@UEAAXPEBE0@Z 000000014003c180 f   yassl:crypto_wrapper.obj
 0001:0003b1a0       ?encrypt@RC4@yaSSL@@UEAAXPEAEPEBEI@Z 000000014003c1a0 f   yassl:crypto_wrapper.obj
 0001:0003b1b0       ?decrypt@RC4@yaSSL@@UEAAXPEAEPEBEI@Z 000000014003c1b0 f   yassl:crypto_wrapper.obj
 0001:0003b1c0       ??1?$BlockCipher@$0A@VAES@TaoCrypt@@$00@TaoCrypt@@QEAA@XZ 000000014003c1c0 f i yassl:crypto_wrapper.obj
 0001:0003b1d0       ??1?$BlockCipher@$00VAES@TaoCrypt@@$00@TaoCrypt@@QEAA@XZ 000000014003c1d0 f i yassl:crypto_wrapper.obj
 0001:0003b1e0       ?get_keySize@AES@yaSSL@@UEBAHXZ 000000014003c1e0 f   yassl:crypto_wrapper.obj
 0001:0003b1f0       ??0RandomImpl@RandomPool@yaSSL@@QEAA@XZ 000000014003c1f0 f i yassl:crypto_wrapper.obj
 0001:0003b210       ?GetError@RandomPool@yaSSL@@QEBAHXZ 000000014003c210 f   yassl:crypto_wrapper.obj
 0001:0003b220       ?Fill@RandomPool@yaSSL@@QEBAXPEAEI@Z 000000014003c220 f   yassl:crypto_wrapper.obj
 0001:0003b230       ??0Auth@yaSSL@@QEAA@XZ     000000014003c230 f i yassl:crypto_wrapper.obj
 0001:0003b240       ?get_signatureLength@DSS@yaSSL@@UEBAIXZ 000000014003c240 f   yassl:crypto_wrapper.obj
 0001:0003b250       ?get_cipherLength@RSA@yaSSL@@QEBAIXZ 000000014003c250 f   yassl:crypto_wrapper.obj
 0001:0003b260       ?get_signatureLength@RSA@yaSSL@@UEBAIXZ 000000014003c260 f   yassl:crypto_wrapper.obj
 0001:0003b270       ??4Integer@yaSSL@@QEAAAEAV01@AEBV01@@Z 000000014003c270 f   yassl:crypto_wrapper.obj
 0001:0003b290       ?AllocKeys@DHImpl@DiffieHellman@yaSSL@@QEAAXIII@Z 000000014003c290 f i yassl:crypto_wrapper.obj
 0001:0003b2e0       ?makeAgreement@DiffieHellman@yaSSL@@QEAAXPEBEI@Z 000000014003c2e0 f   yassl:crypto_wrapper.obj
 0001:0003b310       ?get_agreedKeyLength@DiffieHellman@yaSSL@@QEBAIXZ 000000014003c310 f   yassl:crypto_wrapper.obj
 0001:0003b320       ?get_agreedKey@DiffieHellman@yaSSL@@QEBAPEBEXZ 000000014003c320 f   yassl:crypto_wrapper.obj
 0001:0003b330       ?get_publicKey@DiffieHellman@yaSSL@@QEBAPEBEXZ 000000014003c330 f   yassl:crypto_wrapper.obj
 0001:0003b340       ??0?$BlockCipher@$0A@VDES@TaoCrypt@@$00@TaoCrypt@@QEAA@XZ 000000014003c340 f i yassl:crypto_wrapper.obj
 0001:0003b380       ?Process@?$BlockCipher@$0A@VDES@TaoCrypt@@$00@TaoCrypt@@QEAAXPEAEPEBEI@Z 000000014003c380 f i yassl:crypto_wrapper.obj
 0001:0003b390       ?SetKey@?$BlockCipher@$0A@VDES@TaoCrypt@@$00@TaoCrypt@@QEAAXPEBEI0@Z 000000014003c390 f i yassl:crypto_wrapper.obj
 0001:0003b3d0       ??0?$BlockCipher@$00VDES@TaoCrypt@@$00@TaoCrypt@@QEAA@XZ 000000014003c3d0 f i yassl:crypto_wrapper.obj
 0001:0003b410       ?Process@?$BlockCipher@$00VDES@TaoCrypt@@$00@TaoCrypt@@QEAAXPEAEPEBEI@Z 000000014003c410 f i yassl:crypto_wrapper.obj
 0001:0003b420       ?SetKey@?$BlockCipher@$00VDES@TaoCrypt@@$00@TaoCrypt@@QEAAXPEBEI0@Z 000000014003c420 f i yassl:crypto_wrapper.obj
 0001:0003b460       ??0?$BlockCipher@$0A@VDES_EDE3@TaoCrypt@@$00@TaoCrypt@@QEAA@XZ 000000014003c460 f i yassl:crypto_wrapper.obj
 0001:0003b4a0       ?Process@?$BlockCipher@$0A@VDES_EDE3@TaoCrypt@@$00@TaoCrypt@@QEAAXPEAEPEBEI@Z 000000014003c4a0 f i yassl:crypto_wrapper.obj
 0001:0003b4b0       ?SetKey@?$BlockCipher@$0A@VDES_EDE3@TaoCrypt@@$00@TaoCrypt@@QEAAXPEBEI0@Z 000000014003c4b0 f i yassl:crypto_wrapper.obj
 0001:0003b4e0       ??0?$BlockCipher@$00VDES_EDE3@TaoCrypt@@$00@TaoCrypt@@QEAA@XZ 000000014003c4e0 f i yassl:crypto_wrapper.obj
 0001:0003b520       ?Process@?$BlockCipher@$00VDES_EDE3@TaoCrypt@@$00@TaoCrypt@@QEAAXPEAEPEBEI@Z 000000014003c520 f i yassl:crypto_wrapper.obj
 0001:0003b530       ?SetKey@?$BlockCipher@$00VDES_EDE3@TaoCrypt@@$00@TaoCrypt@@QEAAXPEBEI0@Z 000000014003c530 f i yassl:crypto_wrapper.obj
 0001:0003b560       ??0?$BlockCipher@$0A@VAES@TaoCrypt@@$00@TaoCrypt@@QEAA@XZ 000000014003c560 f i yassl:crypto_wrapper.obj
 0001:0003b5a0       ?Process@?$BlockCipher@$0A@VAES@TaoCrypt@@$00@TaoCrypt@@QEAAXPEAEPEBEI@Z 000000014003c5a0 f i yassl:crypto_wrapper.obj
 0001:0003b5b0       ?SetKey@?$BlockCipher@$0A@VAES@TaoCrypt@@$00@TaoCrypt@@QEAAXPEBEI0@Z 000000014003c5b0 f i yassl:crypto_wrapper.obj
 0001:0003b5f0       ??0?$BlockCipher@$00VAES@TaoCrypt@@$00@TaoCrypt@@QEAA@XZ 000000014003c5f0 f i yassl:crypto_wrapper.obj
 0001:0003b630       ?Process@?$BlockCipher@$00VAES@TaoCrypt@@$00@TaoCrypt@@QEAAXPEAEPEBEI@Z 000000014003c630 f i yassl:crypto_wrapper.obj
 0001:0003b640       ?SetKey@?$BlockCipher@$00VAES@TaoCrypt@@$00@TaoCrypt@@QEAAXPEBEI0@Z 000000014003c640 f i yassl:crypto_wrapper.obj
 0001:0003b680       ??0?$RSA_Decryptor@VRSA_BlockType2@TaoCrypt@@@TaoCrypt@@QEAA@AEBVRSA_PrivateKey@1@@Z 000000014003c680 f i yassl:crypto_wrapper.obj
 0001:0003b690       ??0?$RSA_Encryptor@VRSA_BlockType2@TaoCrypt@@@TaoCrypt@@QEAA@AEBVRSA_PublicKey@1@@Z 000000014003c690 f i yassl:crypto_wrapper.obj
 0001:0003b6a0       ??$SaturatingSubtract@II@TaoCrypt@@YAIII@Z 000000014003c6a0 f i yassl:crypto_wrapper.obj
 0001:0003b6b0       ?Init@?$HMAC@VMD5@TaoCrypt@@@TaoCrypt@@QEAAXXZ 000000014003c6b0 f i yassl:crypto_wrapper.obj
 0001:0003b6d0       ?SetKey@?$HMAC@VMD5@TaoCrypt@@@TaoCrypt@@QEAAXPEBEI@Z 000000014003c6d0 f i yassl:crypto_wrapper.obj
 0001:0003b7f0       ?Init@?$HMAC@VSHA@TaoCrypt@@@TaoCrypt@@QEAAXXZ 000000014003c7f0 f i yassl:crypto_wrapper.obj
 0001:0003b810       ?SetKey@?$HMAC@VSHA@TaoCrypt@@@TaoCrypt@@QEAAXPEBEI@Z 000000014003c810 f i yassl:crypto_wrapper.obj
 0001:0003b920       ?Init@?$HMAC@VRIPEMD160@TaoCrypt@@@TaoCrypt@@QEAAXXZ 000000014003c920 f i yassl:crypto_wrapper.obj
 0001:0003b940       ?SetKey@?$HMAC@VRIPEMD160@TaoCrypt@@@TaoCrypt@@QEAAXPEBEI@Z 000000014003c940 f i yassl:crypto_wrapper.obj
 0001:0003ba50       ??$ysDelete@URC4Impl@RC4@yaSSL@@@yaSSL@@YAXPEAURC4Impl@RC4@0@@Z 000000014003ca50 f i yassl:crypto_wrapper.obj
 0001:0003ba60       ??$tcArrayDelete@_K@TaoCrypt@@YAXPEA_K@Z 000000014003ca60 f i yassl:crypto_wrapper.obj
 0001:0003ba70       ??1MD5Impl@MD5@yaSSL@@QEAA@XZ 000000014003ca70 f i yassl:crypto_wrapper.obj
 0001:0003ba80       ??1SHAImpl@SHA@yaSSL@@QEAA@XZ 000000014003ca80 f i yassl:crypto_wrapper.obj
 0001:0003ba90       ??1RMDImpl@RMD@yaSSL@@QEAA@XZ 000000014003ca90 f i yassl:crypto_wrapper.obj
 0001:0003baa0       ??1HMAC_MD5Impl@HMAC_MD5@yaSSL@@QEAA@XZ 000000014003caa0 f i yassl:crypto_wrapper.obj
 0001:0003bab0       ??1HMAC_SHAImpl@HMAC_SHA@yaSSL@@QEAA@XZ 000000014003cab0 f i yassl:crypto_wrapper.obj
 0001:0003bac0       ??1HMAC_RMDImpl@HMAC_RMD@yaSSL@@QEAA@XZ 000000014003cac0 f i yassl:crypto_wrapper.obj
 0001:0003bad0       ??1DESImpl@DES@yaSSL@@QEAA@XZ 000000014003cad0 f i yassl:crypto_wrapper.obj
 0001:0003baf0       ??1DES_EDEImpl@DES_EDE@yaSSL@@QEAA@XZ 000000014003caf0 f i yassl:crypto_wrapper.obj
 0001:0003bb10       ??1AESImpl@AES@yaSSL@@QEAA@XZ 000000014003cb10 f i yassl:crypto_wrapper.obj
 0001:0003bb30       ??1RandomImpl@RandomPool@yaSSL@@QEAA@XZ 000000014003cb30 f i yassl:crypto_wrapper.obj
 0001:0003bb40       ??0?$RSA_Encryptor@VRSA_BlockType1@TaoCrypt@@@TaoCrypt@@QEAA@AEBVRSA_PublicKey@1@@Z 000000014003cb40 f i yassl:crypto_wrapper.obj
 0001:0003bb50       ?KeyInnerHash@?$HMAC@VMD5@TaoCrypt@@@TaoCrypt@@AEAAXXZ 000000014003cb50 f i yassl:crypto_wrapper.obj
 0001:0003bb80       ?KeyInnerHash@?$HMAC@VSHA@TaoCrypt@@@TaoCrypt@@AEAAXXZ 000000014003cb80 f i yassl:crypto_wrapper.obj
 0001:0003bbb0       ?KeyInnerHash@?$HMAC@VRIPEMD160@TaoCrypt@@@TaoCrypt@@AEAAXXZ 000000014003cbb0 f i yassl:crypto_wrapper.obj
 0001:0003bbe0       ??_ESHA@TaoCrypt@@UEAAPEAXI@Z 000000014003cbe0 f i yassl:crypto_wrapper.obj
 0001:0003bbe0       ??_GSHA@TaoCrypt@@UEAAPEAXI@Z 000000014003cbe0 f i yassl:crypto_wrapper.obj
 0001:0003bc10       ??_ERIPEMD160@TaoCrypt@@UEAAPEAXI@Z 000000014003cc10 f i yassl:crypto_wrapper.obj
 0001:0003bc10       ??_GRIPEMD160@TaoCrypt@@UEAAPEAXI@Z 000000014003cc10 f i yassl:crypto_wrapper.obj
 0001:0003bc40       ?Process@Mode_BASE@TaoCrypt@@UEAAXPEAEPEBEI@Z 000000014003cc40 f i yassl:crypto_wrapper.obj
 0001:0003bd20       ??_EDES@TaoCrypt@@UEAAPEAXI@Z 000000014003cd20 f i yassl:crypto_wrapper.obj
 0001:0003bd20       ??_GDES@TaoCrypt@@UEAAPEAXI@Z 000000014003cd20 f i yassl:crypto_wrapper.obj
 0001:0003bd50       ??_EDES_EDE3@TaoCrypt@@UEAAPEAXI@Z 000000014003cd50 f i yassl:crypto_wrapper.obj
 0001:0003bd50       ??_GDES_EDE3@TaoCrypt@@UEAAPEAXI@Z 000000014003cd50 f i yassl:crypto_wrapper.obj
 0001:0003bd80       ??_EAES@TaoCrypt@@UEAAPEAXI@Z 000000014003cd80 f i yassl:crypto_wrapper.obj
 0001:0003bd80       ??_GAES@TaoCrypt@@UEAAPEAXI@Z 000000014003cd80 f i yassl:crypto_wrapper.obj
 0001:0003bdb0       ?FixedMaxPlaintextLength@PK_Lengths@TaoCrypt@@QEBAIXZ 000000014003cdb0 f i yassl:crypto_wrapper.obj
 0001:0003bde0       ?Initialize@DH@TaoCrypt@@QEAAXAEAVInteger@2@0@Z 000000014003cde0 f i yassl:crypto_wrapper.obj
 0001:0003be10       ??0MD5@yaSSL@@QEAA@XZ      000000014003ce10 f   yassl:crypto_wrapper.obj
 0001:0003be90       ??0DESImpl@DES@yaSSL@@QEAA@XZ 000000014003ce90 f i yassl:crypto_wrapper.obj
 0001:0003bf10       ?set_encryptKey@DES@yaSSL@@UEAAXPEBE0@Z 000000014003cf10 f   yassl:crypto_wrapper.obj
 0001:0003bf50       ?set_decryptKey@DES@yaSSL@@UEAAXPEBE0@Z 000000014003cf50 f   yassl:crypto_wrapper.obj
 0001:0003bfa0       ?encrypt@DES@yaSSL@@UEAAXPEAEPEBEI@Z 000000014003cfa0 f   yassl:crypto_wrapper.obj
 0001:0003bfb0       ?decrypt@DES@yaSSL@@UEAAXPEAEPEBEI@Z 000000014003cfb0 f   yassl:crypto_wrapper.obj
 0001:0003bfd0       ??0DES_EDEImpl@DES_EDE@yaSSL@@QEAA@XZ 000000014003cfd0 f i yassl:crypto_wrapper.obj
 0001:0003c050       ?set_encryptKey@DES_EDE@yaSSL@@UEAAXPEBE0@Z 000000014003d050 f   yassl:crypto_wrapper.obj
 0001:0003c090       ?set_decryptKey@DES_EDE@yaSSL@@UEAAXPEBE0@Z 000000014003d090 f   yassl:crypto_wrapper.obj
 0001:0003c0d0       ?encrypt@DES_EDE@yaSSL@@UEAAXPEAEPEBEI@Z 000000014003d0d0 f   yassl:crypto_wrapper.obj
 0001:0003c0e0       ?decrypt@DES_EDE@yaSSL@@UEAAXPEAEPEBEI@Z 000000014003d0e0 f   yassl:crypto_wrapper.obj
 0001:0003c100       ??0RC4@yaSSL@@QEAA@XZ      000000014003d100 f   yassl:crypto_wrapper.obj
 0001:0003c130       ?get_blockSize@RC4@yaSSL@@UEBAIXZ 000000014003d130 f i yassl:crypto_wrapper.obj
 0001:0003c140       ?get_keySize@RC4@yaSSL@@UEBAHXZ 000000014003d140 f i yassl:crypto_wrapper.obj
 0001:0003c150       ?get_ivSize@RC4@yaSSL@@UEBAHXZ 000000014003d150 f i yassl:crypto_wrapper.obj
 0001:0003c160       ??1RC4@yaSSL@@UEAA@XZ      000000014003d160 f   yassl:crypto_wrapper.obj
 0001:0003c190       ??0AESImpl@AES@yaSSL@@QEAA@I@Z 000000014003d190 f i yassl:crypto_wrapper.obj
 0001:0003c210       ??0AES@yaSSL@@QEAA@I@Z     000000014003d210 f   yassl:crypto_wrapper.obj
 0001:0003c2f0       ?get_blockSize@AES@yaSSL@@UEBAIXZ 000000014003d2f0 f i yassl:crypto_wrapper.obj
 0001:0003c300       ?get_ivSize@AES@yaSSL@@UEBAHXZ 000000014003d300 f i yassl:crypto_wrapper.obj
 0001:0003c310       ?set_encryptKey@AES@yaSSL@@UEAAXPEBE0@Z 000000014003d310 f   yassl:crypto_wrapper.obj
 0001:0003c350       ?set_decryptKey@AES@yaSSL@@UEAAXPEBE0@Z 000000014003d350 f   yassl:crypto_wrapper.obj
 0001:0003c3a0       ?encrypt@AES@yaSSL@@UEAAXPEAEPEBEI@Z 000000014003d3a0 f   yassl:crypto_wrapper.obj
 0001:0003c3b0       ?decrypt@AES@yaSSL@@UEAAXPEAEPEBEI@Z 000000014003d3b0 f   yassl:crypto_wrapper.obj
 0001:0003c3d0       ??0RandomPool@yaSSL@@QEAA@XZ 000000014003d3d0 f   yassl:crypto_wrapper.obj
 0001:0003c420       ??0?$HMAC@VMD5@TaoCrypt@@@TaoCrypt@@QEAA@XZ 000000014003d420 f i yassl:crypto_wrapper.obj
 0001:0003c490       ??0?$HMAC@VSHA@TaoCrypt@@@TaoCrypt@@QEAA@XZ 000000014003d490 f i yassl:crypto_wrapper.obj
 0001:0003c500       ??0?$HMAC@VRIPEMD160@TaoCrypt@@@TaoCrypt@@QEAA@XZ 000000014003d500 f i yassl:crypto_wrapper.obj
 0001:0003c570       ?deallocate@?$AllocatorWithCleanup@_K@TaoCrypt@@QEAAXPEAX_K@Z 000000014003d570 f i yassl:crypto_wrapper.obj
 0001:0003c5a0       ?Update@?$HMAC@VMD5@TaoCrypt@@@TaoCrypt@@QEAAXPEBEI@Z 000000014003d5a0 f i yassl:crypto_wrapper.obj
 0001:0003c5f0       ?Final@?$HMAC@VMD5@TaoCrypt@@@TaoCrypt@@QEAAXPEAE@Z 000000014003d5f0 f i yassl:crypto_wrapper.obj
 0001:0003c670       ?Update@?$HMAC@VSHA@TaoCrypt@@@TaoCrypt@@QEAAXPEBEI@Z 000000014003d670 f i yassl:crypto_wrapper.obj
 0001:0003c6c0       ?Final@?$HMAC@VSHA@TaoCrypt@@@TaoCrypt@@QEAAXPEAE@Z 000000014003d6c0 f i yassl:crypto_wrapper.obj
 0001:0003c740       ?Update@?$HMAC@VRIPEMD160@TaoCrypt@@@TaoCrypt@@QEAAXPEBEI@Z 000000014003d740 f i yassl:crypto_wrapper.obj
 0001:0003c790       ?Final@?$HMAC@VRIPEMD160@TaoCrypt@@@TaoCrypt@@QEAAXPEAE@Z 000000014003d790 f i yassl:crypto_wrapper.obj
 0001:0003c810       ??_GMD5Impl@MD5@yaSSL@@QEAAPEAXI@Z 000000014003d810 f i yassl:crypto_wrapper.obj
 0001:0003c840       ??_GSHAImpl@SHA@yaSSL@@QEAAPEAXI@Z 000000014003d840 f i yassl:crypto_wrapper.obj
 0001:0003c870       ??_GRMDImpl@RMD@yaSSL@@QEAAPEAXI@Z 000000014003d870 f i yassl:crypto_wrapper.obj
 0001:0003c8a0       ??_GHMAC_MD5Impl@HMAC_MD5@yaSSL@@QEAAPEAXI@Z 000000014003d8a0 f i yassl:crypto_wrapper.obj
 0001:0003c8d0       ??_GHMAC_SHAImpl@HMAC_SHA@yaSSL@@QEAAPEAXI@Z 000000014003d8d0 f i yassl:crypto_wrapper.obj
 0001:0003c900       ??_GHMAC_RMDImpl@HMAC_RMD@yaSSL@@QEAAPEAXI@Z 000000014003d900 f i yassl:crypto_wrapper.obj
 0001:0003c930       ??_GDESImpl@DES@yaSSL@@QEAAPEAXI@Z 000000014003d930 f i yassl:crypto_wrapper.obj
 0001:0003c960       ??_GDES_EDEImpl@DES_EDE@yaSSL@@QEAAPEAXI@Z 000000014003d960 f i yassl:crypto_wrapper.obj
 0001:0003c990       ??_GAESImpl@AES@yaSSL@@QEAAPEAXI@Z 000000014003d990 f i yassl:crypto_wrapper.obj
 0001:0003c9c0       ??_GRandomImpl@RandomPool@yaSSL@@QEAAPEAXI@Z 000000014003d9c0 f i yassl:crypto_wrapper.obj
 0001:0003c9f0       ??0HMAC_MD5Impl@HMAC_MD5@yaSSL@@QEAA@XZ 000000014003d9f0 f i yassl:crypto_wrapper.obj
 0001:0003ca60       ??0HMAC_MD5@yaSSL@@QEAA@PEBEI@Z 000000014003da60 f   yassl:crypto_wrapper.obj
 0001:0003cb30       ?get_digest@HMAC_MD5@yaSSL@@UEAAXPEAEPEBEI@Z 000000014003db30 f   yassl:crypto_wrapper.obj
 0001:0003cb70       ?get_digest@HMAC_MD5@yaSSL@@UEAAXPEAE@Z 000000014003db70 f   yassl:crypto_wrapper.obj
 0001:0003cb80       ?update@HMAC_MD5@yaSSL@@UEAAXPEBEI@Z 000000014003db80 f   yassl:crypto_wrapper.obj
 0001:0003cb90       ??0HMAC_SHAImpl@HMAC_SHA@yaSSL@@QEAA@XZ 000000014003db90 f i yassl:crypto_wrapper.obj
 0001:0003cc00       ??0HMAC_SHA@yaSSL@@QEAA@PEBEI@Z 000000014003dc00 f   yassl:crypto_wrapper.obj
 0001:0003ccd0       ?get_digest@HMAC_SHA@yaSSL@@UEAAXPEAEPEBEI@Z 000000014003dcd0 f   yassl:crypto_wrapper.obj
 0001:0003cd10       ?get_digest@HMAC_SHA@yaSSL@@UEAAXPEAE@Z 000000014003dd10 f   yassl:crypto_wrapper.obj
 0001:0003cd20       ?update@HMAC_SHA@yaSSL@@UEAAXPEBEI@Z 000000014003dd20 f   yassl:crypto_wrapper.obj
 0001:0003cd30       ??0HMAC_RMDImpl@HMAC_RMD@yaSSL@@QEAA@XZ 000000014003dd30 f i yassl:crypto_wrapper.obj
 0001:0003cda0       ??0HMAC_RMD@yaSSL@@QEAA@PEBEI@Z 000000014003dda0 f   yassl:crypto_wrapper.obj
 0001:0003ce70       ?get_digest@HMAC_RMD@yaSSL@@UEAAXPEAEPEBEI@Z 000000014003de70 f   yassl:crypto_wrapper.obj
 0001:0003ceb0       ?get_digest@HMAC_RMD@yaSSL@@UEAAXPEAE@Z 000000014003deb0 f   yassl:crypto_wrapper.obj
 0001:0003cec0       ?update@HMAC_RMD@yaSSL@@UEAAXPEBEI@Z 000000014003dec0 f   yassl:crypto_wrapper.obj
 0001:0003ced0       ??0DES@yaSSL@@QEAA@XZ      000000014003ded0 f   yassl:crypto_wrapper.obj
 0001:0003cf90       ?get_blockSize@DES@yaSSL@@UEBAIXZ 000000014003df90 f i yassl:crypto_wrapper.obj
 0001:0003cfa0       ?get_keySize@DES@yaSSL@@UEBAHXZ 000000014003dfa0 f i yassl:crypto_wrapper.obj
 0001:0003cfb0       ?get_ivSize@DES@yaSSL@@UEBAHXZ 000000014003dfb0 f i yassl:crypto_wrapper.obj
 0001:0003cfc0       ??0DES_EDE@yaSSL@@QEAA@XZ  000000014003dfc0 f   yassl:crypto_wrapper.obj
 0001:0003d080       ?get_blockSize@DES_EDE@yaSSL@@UEBAIXZ 000000014003e080 f i yassl:crypto_wrapper.obj
 0001:0003d090       ?get_keySize@DES_EDE@yaSSL@@UEBAHXZ 000000014003e090 f i yassl:crypto_wrapper.obj
 0001:0003d0a0       ?get_ivSize@DES_EDE@yaSSL@@UEBAHXZ 000000014003e0a0 f i yassl:crypto_wrapper.obj
 0001:0003d0b0       ??_GRC4@yaSSL@@UEAAPEAXI@Z 000000014003e0b0 f i yassl:crypto_wrapper.obj
 0001:0003d0b0       ??_ERC4@yaSSL@@UEAAPEAXI@Z 000000014003e0b0 f i yassl:crypto_wrapper.obj
 0001:0003d0e0       ??1?$Block@_KV?$AllocatorWithCleanup@_K@TaoCrypt@@@TaoCrypt@@QEAA@XZ 000000014003e0e0 f i yassl:crypto_wrapper.obj
 0001:0003d110       ??$ysDelete@UMD5Impl@MD5@yaSSL@@@yaSSL@@YAXPEAUMD5Impl@MD5@0@@Z 000000014003e110 f i yassl:crypto_wrapper.obj
 0001:0003d130       ??$ysDelete@USHAImpl@SHA@yaSSL@@@yaSSL@@YAXPEAUSHAImpl@SHA@0@@Z 000000014003e130 f i yassl:crypto_wrapper.obj
 0001:0003d150       ??$ysDelete@URMDImpl@RMD@yaSSL@@@yaSSL@@YAXPEAURMDImpl@RMD@0@@Z 000000014003e150 f i yassl:crypto_wrapper.obj
 0001:0003d170       ??$ysDelete@UHMAC_MD5Impl@HMAC_MD5@yaSSL@@@yaSSL@@YAXPEAUHMAC_MD5Impl@HMAC_MD5@0@@Z 000000014003e170 f i yassl:crypto_wrapper.obj
 0001:0003d190       ??$ysDelete@UHMAC_SHAImpl@HMAC_SHA@yaSSL@@@yaSSL@@YAXPEAUHMAC_SHAImpl@HMAC_SHA@0@@Z 000000014003e190 f i yassl:crypto_wrapper.obj
 0001:0003d1b0       ??$ysDelete@UHMAC_RMDImpl@HMAC_RMD@yaSSL@@@yaSSL@@YAXPEAUHMAC_RMDImpl@HMAC_RMD@0@@Z 000000014003e1b0 f i yassl:crypto_wrapper.obj
 0001:0003d1d0       ??$ysDelete@UDESImpl@DES@yaSSL@@@yaSSL@@YAXPEAUDESImpl@DES@0@@Z 000000014003e1d0 f i yassl:crypto_wrapper.obj
 0001:0003d200       ??$ysDelete@UDES_EDEImpl@DES_EDE@yaSSL@@@yaSSL@@YAXPEAUDES_EDEImpl@DES_EDE@0@@Z 000000014003e200 f i yassl:crypto_wrapper.obj
 0001:0003d230       ??$ysDelete@UAESImpl@AES@yaSSL@@@yaSSL@@YAXPEAUAESImpl@AES@0@@Z 000000014003e230 f i yassl:crypto_wrapper.obj
 0001:0003d260       ??$ysDelete@URandomImpl@RandomPool@yaSSL@@@yaSSL@@YAXPEAURandomImpl@RandomPool@0@@Z 000000014003e260 f i yassl:crypto_wrapper.obj
 0001:0003d290       ??1Integer@TaoCrypt@@QEAA@XZ 000000014003e290 f i yassl:crypto_wrapper.obj
 0001:0003d2c0       ??0RSA_PublicKey@TaoCrypt@@QEAA@XZ 000000014003e2c0 f i yassl:crypto_wrapper.obj
 0001:0003d2e0       ??0RSA_PublicKey@TaoCrypt@@QEAA@AEBV01@@Z 000000014003e2e0 f i yassl:crypto_wrapper.obj
 0001:0003d310       ??1RSA_PublicKey@TaoCrypt@@QEAA@XZ 000000014003e310 f i yassl:crypto_wrapper.obj
 0001:0003d370       ??0RSA_PrivateKey@TaoCrypt@@QEAA@XZ 000000014003e370 f i yassl:crypto_wrapper.obj
 0001:0003d3e0       ??0DSA_PublicKey@TaoCrypt@@QEAA@XZ 000000014003e3e0 f i yassl:crypto_wrapper.obj
 0001:0003d420       ??1DSA_PublicKey@TaoCrypt@@QEAA@XZ 000000014003e420 f i yassl:crypto_wrapper.obj
 0001:0003d4b0       ??0DH@TaoCrypt@@QEAA@XZ    000000014003e4b0 f i yassl:crypto_wrapper.obj
 0001:0003d4d0       ??0DH@TaoCrypt@@QEAA@AEBV01@@Z 000000014003e4d0 f i yassl:crypto_wrapper.obj
 0001:0003d500       ??1DH@TaoCrypt@@QEAA@XZ    000000014003e500 f i yassl:crypto_wrapper.obj
 0001:0003d560       ??1MD5@yaSSL@@UEAA@XZ      000000014003e560 f   yassl:crypto_wrapper.obj
 0001:0003d590       ??1SHA@yaSSL@@UEAA@XZ      000000014003e590 f   yassl:crypto_wrapper.obj
 0001:0003d5c0       ??1RMD@yaSSL@@UEAA@XZ      000000014003e5c0 f   yassl:crypto_wrapper.obj
 0001:0003d5f0       ??1HMAC_MD5@yaSSL@@UEAA@XZ 000000014003e5f0 f   yassl:crypto_wrapper.obj
 0001:0003d620       ??1HMAC_SHA@yaSSL@@UEAA@XZ 000000014003e620 f   yassl:crypto_wrapper.obj
 0001:0003d650       ??1HMAC_RMD@yaSSL@@UEAA@XZ 000000014003e650 f   yassl:crypto_wrapper.obj
 0001:0003d680       ??1DES@yaSSL@@UEAA@XZ      000000014003e680 f   yassl:crypto_wrapper.obj
 0001:0003d6b0       ??1DES_EDE@yaSSL@@UEAA@XZ  000000014003e6b0 f   yassl:crypto_wrapper.obj
 0001:0003d6e0       ??1AES@yaSSL@@UEAA@XZ      000000014003e6e0 f   yassl:crypto_wrapper.obj
 0001:0003d710       ??1RandomPool@yaSSL@@QEAA@XZ 000000014003e710 f   yassl:crypto_wrapper.obj
 0001:0003d720       ?SetPublic@DSSImpl@DSS@yaSSL@@QEAAXPEBEI@Z 000000014003e720 f   yassl:crypto_wrapper.obj
 0001:0003d7b0       ?SetPrivate@DSSImpl@DSS@yaSSL@@QEAAXPEBEI@Z 000000014003e7b0 f   yassl:crypto_wrapper.obj
 0001:0003d8f0       ??1DSA_PrivateKey@TaoCrypt@@QEAA@XZ 000000014003e8f0 f i yassl:crypto_wrapper.obj
 0001:0003d9b0       ??1DSA_Signer@TaoCrypt@@QEAA@XZ 000000014003e9b0 f i yassl:crypto_wrapper.obj
 0001:0003da10       ??1DSA_Verifier@TaoCrypt@@QEAA@XZ 000000014003ea10 f i yassl:crypto_wrapper.obj
 0001:0003da70       ?SetPublic@RSAImpl@RSA@yaSSL@@QEAAXPEBEI@Z 000000014003ea70 f   yassl:crypto_wrapper.obj
 0001:0003db00       ??1RSA_PrivateKey@TaoCrypt@@QEAA@XZ 000000014003eb00 f i yassl:crypto_wrapper.obj
 0001:0003dc20       ??0IntegerImpl@Integer@yaSSL@@QEAA@XZ 000000014003ec20 f i yassl:crypto_wrapper.obj
 0001:0003dc40       ??0IntegerImpl@Integer@yaSSL@@QEAA@AEBV1TaoCrypt@@@Z 000000014003ec40 f i yassl:crypto_wrapper.obj
 0001:0003dc60       ??0Integer@yaSSL@@QEAA@XZ  000000014003ec60 f   yassl:crypto_wrapper.obj
 0001:0003dcb0       ??0Integer@yaSSL@@QEAA@AEBV01@@Z 000000014003ecb0 f   yassl:crypto_wrapper.obj
 0001:0003dd20       ?assign@Integer@yaSSL@@QEAAXPEBEI@Z 000000014003ed20 f   yassl:crypto_wrapper.obj
 0001:0003dd70       ??0DHImpl@DiffieHellman@yaSSL@@QEAA@AEAVRandomNumberGenerator@TaoCrypt@@@Z 000000014003ed70 f i yassl:crypto_wrapper.obj
 0001:0003ddb0       ??1DHImpl@DiffieHellman@yaSSL@@QEAA@XZ 000000014003edb0 f i yassl:crypto_wrapper.obj
 0001:0003de20       ??0DHImpl@DiffieHellman@yaSSL@@QEAA@AEBU012@@Z 000000014003ee20 f i yassl:crypto_wrapper.obj
 0001:0003dea0       ??0DiffieHellman@yaSSL@@QEAA@PEBEI0I0IAEBVRandomPool@1@@Z 000000014003eea0 f   yassl:crypto_wrapper.obj
 0001:0003dfe0       ??0DiffieHellman@yaSSL@@QEAA@AEBVInteger@1@0AEBVRandomPool@1@@Z 000000014003efe0 f   yassl:crypto_wrapper.obj
 0001:0003e0d0       ??0DiffieHellman@yaSSL@@QEAA@AEBV01@@Z 000000014003f0d0 f   yassl:crypto_wrapper.obj
 0001:0003e190       ?set_sizes@DiffieHellman@yaSSL@@QEBAXAEAH00@Z 000000014003f190 f   yassl:crypto_wrapper.obj
 0001:0003e250       ?get_parms@DiffieHellman@yaSSL@@QEBAXPEAE00@Z 000000014003f250 f   yassl:crypto_wrapper.obj
 0001:0003e340       ??1Base64Decoder@TaoCrypt@@QEAA@XZ 000000014003f340 f i yassl:crypto_wrapper.obj
 0001:0003e370       ??_GDHImpl@DiffieHellman@yaSSL@@QEAAPEAXI@Z 000000014003f370 f i yassl:crypto_wrapper.obj
 0001:0003e400       ??1DSSImpl@DSS@yaSSL@@QEAA@XZ 000000014003f400 f i yassl:crypto_wrapper.obj
 0001:0003e550       ??1RSAImpl@RSA@yaSSL@@QEAA@XZ 000000014003f550 f i yassl:crypto_wrapper.obj
 0001:0003e5b0       ??1IntegerImpl@Integer@yaSSL@@QEAA@XZ 000000014003f5b0 f i yassl:crypto_wrapper.obj
 0001:0003e5e0       ??4RSA_PublicKey@TaoCrypt@@QEAAAEAV01@AEBV01@@Z 000000014003f5e0 f i yassl:crypto_wrapper.obj
 0001:0003e680       ??0DSA_PrivateKey@TaoCrypt@@QEAA@XZ 000000014003f680 f i yassl:crypto_wrapper.obj
 0001:0003e6c0       ??4DH@TaoCrypt@@QEAAAEAV01@AEBV01@@Z 000000014003f6c0 f i yassl:crypto_wrapper.obj
 0001:0003e760       ??_GMD5@yaSSL@@UEAAPEAXI@Z 000000014003f760 f i yassl:crypto_wrapper.obj
 0001:0003e760       ??_EMD5@yaSSL@@UEAAPEAXI@Z 000000014003f760 f i yassl:crypto_wrapper.obj
 0001:0003e790       ??_GSHA@yaSSL@@UEAAPEAXI@Z 000000014003f790 f i yassl:crypto_wrapper.obj
 0001:0003e790       ??_ESHA@yaSSL@@UEAAPEAXI@Z 000000014003f790 f i yassl:crypto_wrapper.obj
 0001:0003e7c0       ??_ERMD@yaSSL@@UEAAPEAXI@Z 000000014003f7c0 f i yassl:crypto_wrapper.obj
 0001:0003e7c0       ??_GRMD@yaSSL@@UEAAPEAXI@Z 000000014003f7c0 f i yassl:crypto_wrapper.obj
 0001:0003e7f0       ??_GHMAC_MD5@yaSSL@@UEAAPEAXI@Z 000000014003f7f0 f i yassl:crypto_wrapper.obj
 0001:0003e7f0       ??_EHMAC_MD5@yaSSL@@UEAAPEAXI@Z 000000014003f7f0 f i yassl:crypto_wrapper.obj
 0001:0003e820       ??_EHMAC_SHA@yaSSL@@UEAAPEAXI@Z 000000014003f820 f i yassl:crypto_wrapper.obj
 0001:0003e820       ??_GHMAC_SHA@yaSSL@@UEAAPEAXI@Z 000000014003f820 f i yassl:crypto_wrapper.obj
 0001:0003e850       ??_GHMAC_RMD@yaSSL@@UEAAPEAXI@Z 000000014003f850 f i yassl:crypto_wrapper.obj
 0001:0003e850       ??_EHMAC_RMD@yaSSL@@UEAAPEAXI@Z 000000014003f850 f i yassl:crypto_wrapper.obj
 0001:0003e880       ??_EDES@yaSSL@@UEAAPEAXI@Z 000000014003f880 f i yassl:crypto_wrapper.obj
 0001:0003e880       ??_GDES@yaSSL@@UEAAPEAXI@Z 000000014003f880 f i yassl:crypto_wrapper.obj
 0001:0003e8b0       ??_EDES_EDE@yaSSL@@UEAAPEAXI@Z 000000014003f8b0 f i yassl:crypto_wrapper.obj
 0001:0003e8b0       ??_GDES_EDE@yaSSL@@UEAAPEAXI@Z 000000014003f8b0 f i yassl:crypto_wrapper.obj
 0001:0003e8e0       ??_EAES@yaSSL@@UEAAPEAXI@Z 000000014003f8e0 f i yassl:crypto_wrapper.obj
 0001:0003e8e0       ??_GAES@yaSSL@@UEAAPEAXI@Z 000000014003f8e0 f i yassl:crypto_wrapper.obj
 0001:0003e910       ??0DSSImpl@DSS@yaSSL@@QEAA@XZ 000000014003f910 f i yassl:crypto_wrapper.obj
 0001:0003e990       ?sign@DSS@yaSSL@@UEAAXPEAEPEBEIAEBVRandomPool@2@@Z 000000014003f990 f   yassl:crypto_wrapper.obj
 0001:0003ea20       ?verify@DSS@yaSSL@@UEAA_NPEBEI0I@Z 000000014003fa20 f   yassl:crypto_wrapper.obj
 0001:0003eab0       ?SetPrivate@RSAImpl@RSA@yaSSL@@QEAAXPEBEI@Z 000000014003fab0 f   yassl:crypto_wrapper.obj
 0001:0003ec30       ??0RSAImpl@RSA@yaSSL@@QEAA@XZ 000000014003fc30 f i yassl:crypto_wrapper.obj
 0001:0003ecc0       ??4DiffieHellman@yaSSL@@QEAAAEAV01@AEBV01@@Z 000000014003fcc0 f   yassl:crypto_wrapper.obj
 0001:0003ed80       ?Decrypt@?$RSA_Decryptor@VRSA_BlockType2@TaoCrypt@@@TaoCrypt@@QEAAIPEBEIPEAEAEAVRandomNumberGenerator@2@@Z 000000014003fd80 f i yassl:crypto_wrapper.obj
 0001:0003ef30       ?Encrypt@?$RSA_Encryptor@VRSA_BlockType2@TaoCrypt@@@TaoCrypt@@QEAAXPEBEIPEAEAEAVRandomNumberGenerator@2@@Z 000000014003ff30 f i yassl:crypto_wrapper.obj
 0001:0003f0c0       ?SSL_Verify@?$RSA_Encryptor@VRSA_BlockType2@TaoCrypt@@@TaoCrypt@@QEAA_NPEBEI0@Z 00000001400400c0 f i yassl:crypto_wrapper.obj
 0001:0003f1c0       ??$ysDelete@UDHImpl@DiffieHellman@yaSSL@@@yaSSL@@YAXPEAUDHImpl@DiffieHellman@0@@Z 00000001400401c0 f i yassl:crypto_wrapper.obj
 0001:0003f240       ??_GDSSImpl@DSS@yaSSL@@QEAAPEAXI@Z 0000000140040240 f i yassl:crypto_wrapper.obj
 0001:0003f270       ??_GRSAImpl@RSA@yaSSL@@QEAAPEAXI@Z 0000000140040270 f i yassl:crypto_wrapper.obj
 0001:0003f2f0       ??_GIntegerImpl@Integer@yaSSL@@QEAAPEAXI@Z 00000001400402f0 f i yassl:crypto_wrapper.obj
 0001:0003f350       ?Encrypt@?$RSA_Encryptor@VRSA_BlockType1@TaoCrypt@@@TaoCrypt@@QEAAXPEBEIPEAEAEAVRandomNumberGenerator@2@@Z 0000000140040350 f i yassl:crypto_wrapper.obj
 0001:0003f4e0       ??0Base64Decoder@TaoCrypt@@QEAA@AEAVSource@1@@Z 00000001400404e0 f i yassl:crypto_wrapper.obj
 0001:0003f540       ??0DSS@yaSSL@@QEAA@PEBEI_N@Z 0000000140040540 f   yassl:crypto_wrapper.obj
 0001:0003f640       ??0RSA@yaSSL@@QEAA@PEBEI_N@Z 0000000140040640 f   yassl:crypto_wrapper.obj
 0001:0003f740       ?verify@RSA@yaSSL@@UEAA_NPEBEI0I@Z 0000000140040740 f   yassl:crypto_wrapper.obj
 0001:0003f760       ?encrypt@RSA@yaSSL@@QEAAXPEAEPEBEIAEBVRandomPool@2@@Z 0000000140040760 f   yassl:crypto_wrapper.obj
 0001:0003f7a0       ?decrypt@RSA@yaSSL@@QEAAXPEAEPEBEIAEBVRandomPool@2@@Z 00000001400407a0 f   yassl:crypto_wrapper.obj
 0001:0003f7e0       ??1DiffieHellman@yaSSL@@QEAA@XZ 00000001400407e0 f   yassl:crypto_wrapper.obj
 0001:0003f7f0       ?PemToDer@yaSSL@@YAPEAVx509@1@PEAU_iobuf@@W4CertType@1@PEAUEncryptedInfo@1@@Z 00000001400407f0 f   yassl:crypto_wrapper.obj
 0001:0003fcd0       ??$ysDelete@UDSSImpl@DSS@yaSSL@@@yaSSL@@YAXPEAUDSSImpl@DSS@0@@Z 0000000140040cd0 f i yassl:crypto_wrapper.obj
 0001:0003fd00       ??$ysDelete@URSAImpl@RSA@yaSSL@@@yaSSL@@YAXPEAURSAImpl@RSA@0@@Z 0000000140040d00 f i yassl:crypto_wrapper.obj
 0001:0003fd70       ?SSL_Sign@?$RSA_Decryptor@VRSA_BlockType2@TaoCrypt@@@TaoCrypt@@QEAAXPEBEIPEAEAEAVRandomNumberGenerator@2@@Z 0000000140040d70 f i yassl:crypto_wrapper.obj
 0001:0003fe50       ??$ysDelete@UIntegerImpl@Integer@yaSSL@@@yaSSL@@YAXPEAUIntegerImpl@Integer@0@@Z 0000000140040e50 f i yassl:crypto_wrapper.obj
 0001:0003fea0       ??1DSS@yaSSL@@UEAA@XZ      0000000140040ea0 f   yassl:crypto_wrapper.obj
 0001:0003fed0       ??1RSA@yaSSL@@UEAA@XZ      0000000140040ed0 f   yassl:crypto_wrapper.obj
 0001:0003ff00       ?sign@RSA@yaSSL@@UEAAXPEAEPEBEIAEBVRandomPool@2@@Z 0000000140040f00 f   yassl:crypto_wrapper.obj
 0001:0003ff40       ??1Integer@yaSSL@@QEAA@XZ  0000000140040f40 f   yassl:crypto_wrapper.obj
 0001:0003ff50       ??_GDSS@yaSSL@@UEAAPEAXI@Z 0000000140040f50 f i yassl:crypto_wrapper.obj
 0001:0003ff50       ??_EDSS@yaSSL@@UEAAPEAXI@Z 0000000140040f50 f i yassl:crypto_wrapper.obj
 0001:0003ff80       ??_GRSA@yaSSL@@UEAAPEAXI@Z 0000000140040f80 f i yassl:crypto_wrapper.obj
 0001:0003ff80       ??_ERSA@yaSSL@@UEAAPEAXI@Z 0000000140040f80 f i yassl:crypto_wrapper.obj
 0001:0003ffb0       ??0Message@yaSSL@@QEAA@XZ  0000000140040fb0 f i yassl:yassl_imp.obj
 0001:0003ffc0       ??0HandShakeHeader@yaSSL@@QEAA@XZ 0000000140040fc0 f i yassl:yassl_imp.obj
 0001:0003ffd0       ??1HandShakeHeader@yaSSL@@UEAA@XZ 0000000140040fd0 f i yassl:yassl_imp.obj
 0001:0003ffe0       ??1ServerKeyBase@yaSSL@@UEAA@XZ 0000000140040fe0 f i yassl:yassl_imp.obj
 0001:0003fff0       ?build@ServerKeyBase@yaSSL@@UEAAXAEAVSSL@2@@Z 0000000140040ff0 f i yassl:yassl_imp.obj
 0001:00040000       ?read@ServerKeyBase@yaSSL@@UEAAXAEAVSSL@2@AEAVinput_buffer@2@@Z 0000000140041000 f i yassl:yassl_imp.obj
 0001:00040010       ??_EServerKeyBase@yaSSL@@UEAAPEAXI@Z 0000000140041010 f i yassl:yassl_imp.obj
 0001:00040010       ??_GServerKeyBase@yaSSL@@UEAAPEAXI@Z 0000000140041010 f i yassl:yassl_imp.obj
 0001:00040040       ??1ClientKeyBase@yaSSL@@UEAA@XZ 0000000140041040 f i yassl:yassl_imp.obj
 0001:00040050       ?build@ClientKeyBase@yaSSL@@UEAAXAEAVSSL@2@@Z 0000000140041050 f i yassl:yassl_imp.obj
 0001:00040060       ?read@ClientKeyBase@yaSSL@@UEAAXAEAVSSL@2@AEAVinput_buffer@2@@Z 0000000140041060 f i yassl:yassl_imp.obj
 0001:00040070       ??_EClientKeyBase@yaSSL@@UEAAPEAXI@Z 0000000140041070 f i yassl:yassl_imp.obj
 0001:00040070       ??_GClientKeyBase@yaSSL@@UEAAPEAXI@Z 0000000140041070 f i yassl:yassl_imp.obj
 0001:000400a0       ?isTLS@?A0xcd0c9aaf@yaSSL@@YA_NUProtocolVersion@2@@Z 00000001400410a0 f   yassl:yassl_imp.obj
 0001:000400c0       ??0ProtocolVersion@yaSSL@@QEAA@EE@Z 00000001400410c0 f   yassl:yassl_imp.obj
 0001:000400d0       ??0ClientKeyBase@yaSSL@@QEAA@XZ 00000001400410d0 f i yassl:yassl_imp.obj
 0001:000400e0       ?get_length@EncryptedPreMasterSecret@yaSSL@@UEBAHXZ 00000001400410e0 f   yassl:yassl_imp.obj
 0001:000400f0       ?get_clientKey@EncryptedPreMasterSecret@yaSSL@@UEBAPEAEXZ 00000001400410f0 f   yassl:yassl_imp.obj
 0001:00040100       ?alloc@EncryptedPreMasterSecret@yaSSL@@QEAAXH@Z 0000000140041100 f   yassl:yassl_imp.obj
 0001:00040120       ??0ClientDiffieHellmanPublic@yaSSL@@QEAA@XZ 0000000140041120 f   yassl:yassl_imp.obj
 0001:00040140       ?get_length@ClientDiffieHellmanPublic@yaSSL@@UEBAHXZ 0000000140041140 f   yassl:yassl_imp.obj
 0001:00040150       ?get_clientKey@ClientDiffieHellmanPublic@yaSSL@@UEBAPEAEXZ 0000000140041150 f   yassl:yassl_imp.obj
 0001:00040160       ?alloc@ClientDiffieHellmanPublic@yaSSL@@QEAAXH_N@Z 0000000140041160 f   yassl:yassl_imp.obj
 0001:00040190       ??0ServerKeyBase@yaSSL@@QEAA@XZ 0000000140041190 f i yassl:yassl_imp.obj
 0001:000401a0       ?get_length@DH_Server@yaSSL@@UEBAHXZ 00000001400411a0 f   yassl:yassl_imp.obj
 0001:000401b0       ?get_serverKey@DH_Server@yaSSL@@UEBAPEAEXZ 00000001400411b0 f   yassl:yassl_imp.obj
 0001:000401c0       ?SetCipherNames@Parameters@yaSSL@@QEAAXXZ 00000001400411c0 f   yassl:yassl_imp.obj
 0001:00040260       ??5yaSSL@@YAAEAVinput_buffer@0@AEAV10@AEAURecordLayerHeader@0@@Z 0000000140041260 f   yassl:yassl_imp.obj
 0001:000402f0       ??6yaSSL@@YAAEAVoutput_buffer@0@AEAV10@AEBURecordLayerHeader@0@@Z 00000001400412f0 f   yassl:yassl_imp.obj
 0001:00040380       ??5yaSSL@@YAAEAVinput_buffer@0@AEAV10@AEAUMessage@0@@Z 0000000140041380 f   yassl:yassl_imp.obj
 0001:00040390       ??6yaSSL@@YAAEAVoutput_buffer@0@AEAV10@AEBUMessage@0@@Z 0000000140041390 f   yassl:yassl_imp.obj
 0001:000403a0       ??5yaSSL@@YAAEAVinput_buffer@0@AEAV10@AEAVHandShakeHeader@0@@Z 00000001400413a0 f   yassl:yassl_imp.obj
 0001:00040410       ??6yaSSL@@YAAEAVoutput_buffer@0@AEAV10@AEBVHandShakeHeader@0@@Z 0000000140041410 f   yassl:yassl_imp.obj
 0001:00040460       ?get_type@HandShakeHeader@yaSSL@@UEBA?AW4ContentType@2@XZ 0000000140041460 f   yassl:yassl_imp.obj
 0001:00040470       ?get_length@HandShakeHeader@yaSSL@@UEBAGXZ 0000000140041470 f   yassl:yassl_imp.obj
 0001:00040480       ?get_handshakeType@HandShakeHeader@yaSSL@@QEBA?AW4HandShakeType@2@XZ 0000000140041480 f   yassl:yassl_imp.obj
 0001:00040490       ?set_type@HandShakeHeader@yaSSL@@QEAAXW4HandShakeType@2@@Z 0000000140041490 f   yassl:yassl_imp.obj
 0001:000404a0       ?set_length@HandShakeHeader@yaSSL@@QEAAXI@Z 00000001400414a0 f   yassl:yassl_imp.obj
 0001:000404b0       ?set@HandShakeHeader@yaSSL@@UEAAAEAVinput_buffer@2@AEAV32@@Z 00000001400414b0 f   yassl:yassl_imp.obj
 0001:000404c0       ?get@HandShakeHeader@yaSSL@@UEBAAEAVoutput_buffer@2@AEAV32@@Z 00000001400414c0 f   yassl:yassl_imp.obj
 0001:000404d0       ?get_length@HandShakeBase@yaSSL@@QEBAHXZ 00000001400414d0 f   yassl:yassl_imp.obj
 0001:000404e0       ?set_length@HandShakeBase@yaSSL@@QEAAXH@Z 00000001400414e0 f   yassl:yassl_imp.obj
 0001:000404f0       ?get_type@HandShakeBase@yaSSL@@UEBA?AW4HandShakeType@2@XZ 00000001400414f0 f   yassl:yassl_imp.obj
 0001:00040500       ?set@HandShakeBase@yaSSL@@UEAAAEAVinput_buffer@2@AEAV32@@Z 0000000140041500 f   yassl:yassl_imp.obj
 0001:00040510       ?get@HandShakeBase@yaSSL@@UEBAAEAVoutput_buffer@2@AEAV32@@Z 0000000140041510 f   yassl:yassl_imp.obj
 0001:00040520       ?Process@HandShakeBase@yaSSL@@UEAAXAEAVinput_buffer@2@AEAVSSL@2@@Z 0000000140041520 f   yassl:yassl_imp.obj
 0001:00040530       ?set@HelloRequest@yaSSL@@UEAAAEAVinput_buffer@2@AEAV32@@Z 0000000140041530 f   yassl:yassl_imp.obj
 0001:00040540       ?get@HelloRequest@yaSSL@@UEBAAEAVoutput_buffer@2@AEAV32@@Z 0000000140041540 f   yassl:yassl_imp.obj
 0001:00040550       ?Process@HelloRequest@yaSSL@@UEAAXAEAVinput_buffer@2@AEAVSSL@2@@Z 0000000140041550 f   yassl:yassl_imp.obj
 0001:00040560       ?get_type@HelloRequest@yaSSL@@UEBA?AW4HandShakeType@2@XZ 0000000140041560 f   yassl:yassl_imp.obj
 0001:00040570       ??5yaSSL@@YAAEAVinput_buffer@0@AEAV10@AEAVChangeCipherSpec@0@@Z 0000000140041570 f   yassl:yassl_imp.obj
 0001:000405a0       ??6yaSSL@@YAAEAVoutput_buffer@0@AEAV10@AEBVChangeCipherSpec@0@@Z 00000001400415a0 f   yassl:yassl_imp.obj
 0001:000405d0       ??0ChangeCipherSpec@yaSSL@@QEAA@XZ 00000001400415d0 f   yassl:yassl_imp.obj
 0001:000405f0       ??1ChangeCipherSpec@yaSSL@@UEAA@XZ 00000001400415f0 f i yassl:yassl_imp.obj
 0001:00040600       ?set@ChangeCipherSpec@yaSSL@@UEAAAEAVinput_buffer@2@AEAV32@@Z 0000000140041600 f   yassl:yassl_imp.obj
 0001:00040610       ?get@ChangeCipherSpec@yaSSL@@UEBAAEAVoutput_buffer@2@AEAV32@@Z 0000000140041610 f   yassl:yassl_imp.obj
 0001:00040620       ?get_type@ChangeCipherSpec@yaSSL@@UEBA?AW4ContentType@2@XZ 0000000140041620 f   yassl:yassl_imp.obj
 0001:00040630       ?get_length@ChangeCipherSpec@yaSSL@@UEBAGXZ 0000000140041630 f   yassl:yassl_imp.obj
 0001:00040640       ?Process@ChangeCipherSpec@yaSSL@@UEAAXAEAVinput_buffer@2@AEAVSSL@2@@Z 0000000140041640 f   yassl:yassl_imp.obj
 0001:000406f0       ??0Alert@yaSSL@@QEAA@W4AlertLevel@1@W4AlertDescription@1@@Z 00000001400416f0 f   yassl:yassl_imp.obj
 0001:00040710       ?get_type@Alert@yaSSL@@UEBA?AW4ContentType@2@XZ 0000000140041710 f   yassl:yassl_imp.obj
 0001:00040720       ?get_length@Alert@yaSSL@@UEBAGXZ 0000000140041720 f   yassl:yassl_imp.obj
 0001:00040730       ??5yaSSL@@YAAEAVinput_buffer@0@AEAV10@AEAVAlert@0@@Z 0000000140041730 f   yassl:yassl_imp.obj
 0001:00040780       ??6yaSSL@@YAAEAVoutput_buffer@0@AEAV10@AEBVAlert@0@@Z 0000000140041780 f   yassl:yassl_imp.obj
 0001:000407d0       ?Process@Alert@yaSSL@@UEAAXAEAVinput_buffer@2@AEAVSSL@2@@Z 00000001400417d0 f   yassl:yassl_imp.obj
 0001:000409d0       ??0Data@yaSSL@@QEAA@XZ     00000001400419d0 f   yassl:yassl_imp.obj
 0001:000409f0       ??0Data@yaSSL@@QEAA@GPEAE@Z 00000001400419f0 f   yassl:yassl_imp.obj
 0001:00040a10       ?SetData@Data@yaSSL@@QEAAXGPEBE@Z 0000000140041a10 f   yassl:yassl_imp.obj
 0001:00040a20       ?set@Data@yaSSL@@UEAAAEAVinput_buffer@2@AEAV32@@Z 0000000140041a20 f   yassl:yassl_imp.obj
 0001:00040a30       ?get_type@Data@yaSSL@@UEBA?AW4ContentType@2@XZ 0000000140041a30 f   yassl:yassl_imp.obj
 0001:00040a40       ?get_length@Data@yaSSL@@UEBAGXZ 0000000140041a40 f   yassl:yassl_imp.obj
 0001:00040a50       ?set_length@Data@yaSSL@@QEAAXG@Z 0000000140041a50 f   yassl:yassl_imp.obj
 0001:00040a60       ?set_buffer@Data@yaSSL@@QEAAPEAEXZ 0000000140041a60 f   yassl:yassl_imp.obj
 0001:00040a70       ??6yaSSL@@YAAEAVoutput_buffer@0@AEAV10@AEBVData@0@@Z 0000000140041a70 f   yassl:yassl_imp.obj
 0001:00040a90       ?Process@Data@yaSSL@@UEAAXAEAVinput_buffer@2@AEAVSSL@2@@Z 0000000140041a90 f   yassl:yassl_imp.obj
 0001:00040d60       ??5yaSSL@@YAAEAVinput_buffer@0@AEAV10@AEAVHandShakeBase@0@@Z 0000000140041d60 f   yassl:yassl_imp.obj
 0001:00040d70       ??6yaSSL@@YAAEAVoutput_buffer@0@AEAV10@AEBVHandShakeBase@0@@Z 0000000140041d70 f   yassl:yassl_imp.obj
 0001:00040d80       ??0HandShakeBase@yaSSL@@QEAA@XZ 0000000140041d80 f i yassl:yassl_imp.obj
 0001:00040d90       ?get_buffer@Certificate@yaSSL@@QEBAPEBEXZ 0000000140041d90 f   yassl:yassl_imp.obj
 0001:00040da0       ??6yaSSL@@YAAEAVoutput_buffer@0@AEAV10@AEBVCertificate@0@@Z 0000000140041da0 f   yassl:yassl_imp.obj
 0001:00040e30       ?Process@Certificate@yaSSL@@UEAAXAEAVinput_buffer@2@AEAVSSL@2@@Z 0000000140041e30 f   yassl:yassl_imp.obj
 0001:00041030       ??0Certificate@yaSSL@@QEAA@XZ 0000000140042030 f   yassl:yassl_imp.obj
 0001:00041050       ??1Certificate@yaSSL@@UEAA@XZ 0000000140042050 f i yassl:yassl_imp.obj
 0001:00041060       ?set@Certificate@yaSSL@@UEAAAEAVinput_buffer@2@AEAV32@@Z 0000000140042060 f   yassl:yassl_imp.obj
 0001:00041070       ?get@Certificate@yaSSL@@UEBAAEAVoutput_buffer@2@AEAV32@@Z 0000000140042070 f   yassl:yassl_imp.obj
 0001:00041080       ?get_type@Certificate@yaSSL@@UEBA?AW4HandShakeType@2@XZ 0000000140042080 f   yassl:yassl_imp.obj
 0001:00041090       ??0ServerDHParams@yaSSL@@QEAA@XZ 0000000140042090 f   yassl:yassl_imp.obj
 0001:000410b0       ?get_pSize@ServerDHParams@yaSSL@@QEBAHXZ 00000001400420b0 f   yassl:yassl_imp.obj
 0001:000410c0       ?get_gSize@ServerDHParams@yaSSL@@QEBAHXZ 00000001400420c0 f   yassl:yassl_imp.obj
 0001:000410d0       ?get_pubSize@ServerDHParams@yaSSL@@QEBAHXZ 00000001400420d0 f   yassl:yassl_imp.obj
 0001:000410e0       ?get_p@ServerDHParams@yaSSL@@QEBAPEBEXZ 00000001400420e0 f   yassl:yassl_imp.obj
 0001:000410f0       ?get_g@ServerDHParams@yaSSL@@QEBAPEBEXZ 00000001400420f0 f   yassl:yassl_imp.obj
 0001:00041100       ?get_pub@ServerDHParams@yaSSL@@QEBAPEBEXZ 0000000140042100 f   yassl:yassl_imp.obj
 0001:00041110       ?alloc_p@ServerDHParams@yaSSL@@QEAAPEAEH@Z 0000000140042110 f   yassl:yassl_imp.obj
 0001:00041130       ?alloc_g@ServerDHParams@yaSSL@@QEAAPEAEH@Z 0000000140042130 f   yassl:yassl_imp.obj
 0001:00041150       ?alloc_pub@ServerDHParams@yaSSL@@QEAAPEAEH@Z 0000000140042150 f   yassl:yassl_imp.obj
 0001:00041170       ?get_length@ServerKeyBase@yaSSL@@UEBAHXZ 0000000140042170 f   yassl:yassl_imp.obj
 0001:00041180       ?get_serverKey@ServerKeyBase@yaSSL@@UEBAPEAEXZ 0000000140042180 f   yassl:yassl_imp.obj
 0001:00041190       ??5yaSSL@@YAAEAVinput_buffer@0@AEAV10@AEAVServerHello@0@@Z 0000000140042190 f   yassl:yassl_imp.obj
 0001:00041250       ??6yaSSL@@YAAEAVoutput_buffer@0@AEAV10@AEBVServerHello@0@@Z 0000000140042250 f   yassl:yassl_imp.obj
 0001:00041310       ??0ServerHello@yaSSL@@QEAA@XZ 0000000140042310 f   yassl:yassl_imp.obj
 0001:00041360       ??1ServerHello@yaSSL@@UEAA@XZ 0000000140042360 f i yassl:yassl_imp.obj
 0001:00041370       ??0ServerHello@yaSSL@@QEAA@UProtocolVersion@1@_N@Z 0000000140042370 f   yassl:yassl_imp.obj
 0001:000413c0       ?set@ServerHello@yaSSL@@UEAAAEAVinput_buffer@2@AEAV32@@Z 00000001400423c0 f   yassl:yassl_imp.obj
 0001:000413d0       ?get@ServerHello@yaSSL@@UEBAAEAVoutput_buffer@2@AEAV32@@Z 00000001400423d0 f   yassl:yassl_imp.obj
 0001:000413e0       ?get_type@ServerHello@yaSSL@@UEBA?AW4HandShakeType@2@XZ 00000001400423e0 f   yassl:yassl_imp.obj
 0001:000413f0       ?get_random@ServerHello@yaSSL@@QEBAPEBEXZ 00000001400423f0 f   yassl:yassl_imp.obj
 0001:00041400       ?Process@ServerHelloDone@yaSSL@@UEAAXAEAVinput_buffer@2@AEAVSSL@2@@Z 0000000140042400 f   yassl:yassl_imp.obj
 0001:00041420       ??0ServerHelloDone@yaSSL@@QEAA@XZ 0000000140042420 f   yassl:yassl_imp.obj
 0001:00041440       ??1ServerHelloDone@yaSSL@@UEAA@XZ 0000000140042440 f i yassl:yassl_imp.obj
 0001:00041450       ?set@ServerHelloDone@yaSSL@@UEAAAEAVinput_buffer@2@AEAV32@@Z 0000000140042450 f   yassl:yassl_imp.obj
 0001:00041460       ?get@ServerHelloDone@yaSSL@@UEBAAEAVoutput_buffer@2@AEAV32@@Z 0000000140042460 f   yassl:yassl_imp.obj
 0001:00041470       ?get_type@ServerHelloDone@yaSSL@@UEBA?AW4HandShakeType@2@XZ 0000000140042470 f   yassl:yassl_imp.obj
 0001:00041480       ?get_length@ClientKeyBase@yaSSL@@UEBAHXZ 0000000140042480 f   yassl:yassl_imp.obj
 0001:00041490       ?get_clientKey@ClientKeyBase@yaSSL@@UEBAPEAEXZ 0000000140042490 f   yassl:yassl_imp.obj
 0001:000414a0       ??5yaSSL@@YAAEAVinput_buffer@0@AEAV10@AEAVClientHello@0@@Z 00000001400424a0 f   yassl:yassl_imp.obj
 0001:00041650       ??6yaSSL@@YAAEAVoutput_buffer@0@AEAV10@AEBVClientHello@0@@Z 0000000140042650 f   yassl:yassl_imp.obj
 0001:00041750       ?set@ClientHello@yaSSL@@UEAAAEAVinput_buffer@2@AEAV32@@Z 0000000140042750 f   yassl:yassl_imp.obj
 0001:00041760       ?get@ClientHello@yaSSL@@UEBAAEAVoutput_buffer@2@AEAV32@@Z 0000000140042760 f   yassl:yassl_imp.obj
 0001:00041770       ?get_type@ClientHello@yaSSL@@UEBA?AW4HandShakeType@2@XZ 0000000140042770 f   yassl:yassl_imp.obj
 0001:00041780       ?get_random@ClientHello@yaSSL@@QEBAPEBEXZ 0000000140042780 f   yassl:yassl_imp.obj
 0001:00041790       ??0ClientHello@yaSSL@@QEAA@XZ 0000000140042790 f   yassl:yassl_imp.obj
 0001:000417d0       ??1ClientHello@yaSSL@@UEAA@XZ 00000001400427d0 f i yassl:yassl_imp.obj
 0001:000417e0       ??0ClientHello@yaSSL@@QEAA@UProtocolVersion@1@_N@Z 00000001400427e0 f   yassl:yassl_imp.obj
 0001:00041820       ??0ServerKeyExchange@yaSSL@@QEAA@XZ 0000000140042820 f   yassl:yassl_imp.obj
 0001:00041840       ?build@ServerKeyExchange@yaSSL@@QEAAXAEAVSSL@2@@Z 0000000140042840 f   yassl:yassl_imp.obj
 0001:00041870       ?getKey@ServerKeyExchange@yaSSL@@QEBAPEBEXZ 0000000140042870 f   yassl:yassl_imp.obj
 0001:00041880       ?getKeyLength@ServerKeyExchange@yaSSL@@QEBAHXZ 0000000140042880 f   yassl:yassl_imp.obj
 0001:00041890       ?set@ServerKeyExchange@yaSSL@@UEAAAEAVinput_buffer@2@AEAV32@@Z 0000000140042890 f   yassl:yassl_imp.obj
 0001:000418a0       ?get_type@ServerKeyExchange@yaSSL@@UEBA?AW4HandShakeType@2@XZ 00000001400428a0 f   yassl:yassl_imp.obj
 0001:000418b0       ?Process@CertificateRequest@yaSSL@@UEAAXAEAVinput_buffer@2@AEAVSSL@2@@Z 00000001400428b0 f   yassl:yassl_imp.obj
 0001:00041900       ?get_type@CertificateRequest@yaSSL@@UEBA?AW4HandShakeType@2@XZ 0000000140042900 f   yassl:yassl_imp.obj
 0001:00041910       ??0CertificateVerify@yaSSL@@QEAA@XZ 0000000140042910 f   yassl:yassl_imp.obj
 0001:00041930       ??5yaSSL@@YAAEAVinput_buffer@0@AEAV10@AEAVCertificateVerify@0@@Z 0000000140042930 f   yassl:yassl_imp.obj
 0001:000419b0       ??6yaSSL@@YAAEAVoutput_buffer@0@AEAV10@AEBVCertificateVerify@0@@Z 00000001400429b0 f   yassl:yassl_imp.obj
 0001:000419e0       ?Process@CertificateVerify@yaSSL@@UEAAXAEAVinput_buffer@2@AEAVSSL@2@@Z 00000001400429e0 f   yassl:yassl_imp.obj
 0001:00041b40       ?get_type@CertificateVerify@yaSSL@@UEBA?AW4HandShakeType@2@XZ 0000000140042b40 f   yassl:yassl_imp.obj
 0001:00041b50       ??0ClientKeyExchange@yaSSL@@QEAA@XZ 0000000140042b50 f   yassl:yassl_imp.obj
 0001:00041b70       ?build@ClientKeyExchange@yaSSL@@QEAAXAEAVSSL@2@@Z 0000000140042b70 f   yassl:yassl_imp.obj
 0001:00041ba0       ?getKey@ClientKeyExchange@yaSSL@@QEBAPEBEXZ 0000000140042ba0 f   yassl:yassl_imp.obj
 0001:00041bb0       ?getKeyLength@ClientKeyExchange@yaSSL@@QEBAHXZ 0000000140042bb0 f   yassl:yassl_imp.obj
 0001:00041bc0       ?set@ClientKeyExchange@yaSSL@@UEAAAEAVinput_buffer@2@AEAV32@@Z 0000000140042bc0 f   yassl:yassl_imp.obj
 0001:00041bd0       ?get_type@ClientKeyExchange@yaSSL@@UEBA?AW4HandShakeType@2@XZ 0000000140042bd0 f   yassl:yassl_imp.obj
 0001:00041be0       ??5yaSSL@@YAAEAVinput_buffer@0@AEAV10@AEAVFinished@0@@Z 0000000140042be0 f   yassl:yassl_imp.obj
 0001:00041bf0       ??6yaSSL@@YAAEAVoutput_buffer@0@AEAV10@AEBVFinished@0@@Z 0000000140042bf0 f   yassl:yassl_imp.obj
 0001:00041c60       ?Process@Finished@yaSSL@@UEAAXAEAVinput_buffer@2@AEAVSSL@2@@Z 0000000140042c60 f   yassl:yassl_imp.obj
 0001:00041ea0       ??0Finished@yaSSL@@QEAA@XZ 0000000140042ea0 f   yassl:yassl_imp.obj
 0001:00041ec0       ??_GFinished@yaSSL@@UEAAPEAXI@Z 0000000140042ec0 f i yassl:yassl_imp.obj
 0001:00041ec0       ??_EFinished@yaSSL@@UEAAPEAXI@Z 0000000140042ec0 f i yassl:yassl_imp.obj
 0001:00041ef0       ?set_md5@Finished@yaSSL@@QEAAPEAEXZ 0000000140042ef0 f   yassl:yassl_imp.obj
 0001:00041f00       ?set_sha@Finished@yaSSL@@QEAAPEAEXZ 0000000140042f00 f   yassl:yassl_imp.obj
 0001:00041f10       ?set@Finished@yaSSL@@UEAAAEAVinput_buffer@2@AEAV32@@Z 0000000140042f10 f   yassl:yassl_imp.obj
 0001:00041f20       ?get@Finished@yaSSL@@UEBAAEAVoutput_buffer@2@AEAV32@@Z 0000000140042f20 f   yassl:yassl_imp.obj
 0001:00041f30       ?get_type@Finished@yaSSL@@UEBA?AW4HandShakeType@2@XZ 0000000140042f30 f   yassl:yassl_imp.obj
 0001:00041f40       ?clean@yaSSL@@YAXPECEIAEAVRandomPool@1@@Z 0000000140042f40 f   yassl:yassl_imp.obj
 0001:00041fa0       ??0Connection@yaSSL@@QEAA@UProtocolVersion@1@AEAVRandomPool@1@@Z 0000000140042fa0 f   yassl:yassl_imp.obj
 0001:00042060       ?AllocPreSecret@Connection@yaSSL@@QEAAXI@Z 0000000140043060 f   yassl:yassl_imp.obj
 0001:00042080       ?TurnOffTLS@Connection@yaSSL@@QEAAXXZ 0000000140043080 f   yassl:yassl_imp.obj
 0001:00042090       ?TurnOffTLS1_1@Connection@yaSSL@@QEAAXXZ 0000000140043090 f   yassl:yassl_imp.obj
 0001:000420a0       ?CleanMaster@Connection@yaSSL@@QEAAXXZ 00000001400430a0 f   yassl:yassl_imp.obj
 0001:000420e0       ?CreateCipherSpec@yaSSL@@YAPEAUMessage@1@XZ 00000001400430e0 f   yassl:yassl_imp.obj
 0001:00042110       ?CreateHandShake@yaSSL@@YAPEAUMessage@1@XZ 0000000140043110 f   yassl:yassl_imp.obj
 0001:00042140       ?CreateData@yaSSL@@YAPEAUMessage@1@XZ 0000000140043140 f   yassl:yassl_imp.obj
 0001:00042170       ??0HelloRequest@yaSSL@@QEAA@XZ 0000000140043170 f i yassl:yassl_imp.obj
 0001:00042180       ??1HelloRequest@yaSSL@@UEAA@XZ 0000000140043180 f i yassl:yassl_imp.obj
 0001:00042190       ?CreateClientHello@yaSSL@@YAPEAVHandShakeBase@1@XZ 0000000140043190 f   yassl:yassl_imp.obj
 0001:000421c0       ?CreateServerHello@yaSSL@@YAPEAVHandShakeBase@1@XZ 00000001400431c0 f   yassl:yassl_imp.obj
 0001:000421f0       ?CreateCertificate@yaSSL@@YAPEAVHandShakeBase@1@XZ 00000001400431f0 f   yassl:yassl_imp.obj
 0001:00042220       ?CreateServerKeyExchange@yaSSL@@YAPEAVHandShakeBase@1@XZ 0000000140043220 f   yassl:yassl_imp.obj
 0001:00042250       ?CreateServerHelloDone@yaSSL@@YAPEAVHandShakeBase@1@XZ 0000000140043250 f   yassl:yassl_imp.obj
 0001:00042280       ?CreateCertificateVerify@yaSSL@@YAPEAVHandShakeBase@1@XZ 0000000140043280 f   yassl:yassl_imp.obj
 0001:000422b0       ?CreateClientKeyExchange@yaSSL@@YAPEAVHandShakeBase@1@XZ 00000001400432b0 f   yassl:yassl_imp.obj
 0001:000422e0       ?CreateFinished@yaSSL@@YAPEAVHandShakeBase@1@XZ 00000001400432e0 f   yassl:yassl_imp.obj
 0001:00042310       ??0RSA_Server@yaSSL@@QEAA@XZ 0000000140043310 f i yassl:yassl_imp.obj
 0001:00042320       ??1RSA_Server@yaSSL@@UEAA@XZ 0000000140043320 f i yassl:yassl_imp.obj
 0001:00042330       ??0Fortezza_Server@yaSSL@@QEAA@XZ 0000000140043330 f i yassl:yassl_imp.obj
 0001:00042340       ??1Fortezza_Server@yaSSL@@UEAA@XZ 0000000140043340 f i yassl:yassl_imp.obj
 0001:00042350       ?CreateDHClient@yaSSL@@YAPEAUClientKeyBase@1@XZ 0000000140043350 f   yassl:yassl_imp.obj
 0001:00042380       ??0FortezzaKeys@yaSSL@@QEAA@XZ 0000000140043380 f i yassl:yassl_imp.obj
 0001:00042390       ??1FortezzaKeys@yaSSL@@UEAA@XZ 0000000140043390 f i yassl:yassl_imp.obj
 0001:000423a0       ??0?$list@PEAE@mySTL@@QEAA@XZ 00000001400433a0 f i yassl:yassl_imp.obj
 0001:000423c0       ??0?$auto_ptr@UAuth@yaSSL@@@mySTL@@QEAA@PEAUAuth@yaSSL@@@Z 00000001400433c0 f i yassl:yassl_imp.obj
 0001:000423d0       ??C?$auto_ptr@UAuth@yaSSL@@@mySTL@@QEBAPEAUAuth@yaSSL@@XZ 00000001400433d0 f i yassl:yassl_imp.obj
 0001:000423e0       ??0?$auto_ptr@VHandShakeBase@yaSSL@@@mySTL@@QEAA@PEAVHandShakeBase@yaSSL@@@Z 00000001400433e0 f i yassl:yassl_imp.obj
 0001:000423f0       ??C?$auto_ptr@VHandShakeBase@yaSSL@@@mySTL@@QEBAPEAVHandShakeBase@yaSSL@@XZ 00000001400433f0 f i yassl:yassl_imp.obj
 0001:00042400       ??D?$auto_ptr@VHandShakeBase@yaSSL@@@mySTL@@QEBAAEAVHandShakeBase@yaSSL@@XZ 0000000140043400 f i yassl:yassl_imp.obj
 0001:00042410       ?get@?$auto_ptr@VHandShakeBase@yaSSL@@@mySTL@@QEBAPEAVHandShakeBase@yaSSL@@XZ 0000000140043410 f i yassl:yassl_imp.obj
 0001:00042420       ??Diterator@?$list@PEAE@mySTL@@QEBAAEAPEAEXZ 0000000140043420 f i yassl:yassl_imp.obj
 0001:00042430       ??Eiterator@?$list@PEAE@mySTL@@QEAAAEAV012@XZ 0000000140043430 f i yassl:yassl_imp.obj
 0001:00042440       ??9iterator@?$list@PEAE@mySTL@@QEBA_NAEBV012@@Z 0000000140043440 f i yassl:yassl_imp.obj
 0001:00042450       ??0?$auto_array@E@mySTL@@QEAA@PEAE@Z 0000000140043450 f i yassl:yassl_imp.obj
 0001:00042460       ?get@?$auto_array@E@mySTL@@QEBAPEAEXZ 0000000140043460 f i yassl:yassl_imp.obj
 0001:00042470       ?release@?$auto_array@E@mySTL@@QEAAPEAEXZ 0000000140043470 f i yassl:yassl_imp.obj
 0001:00042480       ?begin@?$vector@U?$pair@HP6APEAVHandShakeBase@yaSSL@@XZ@mySTL@@@mySTL@@QEBAPEBU?$pair@HP6APEAVHandShakeBase@yaSSL@@XZ@2@XZ 0000000140043480 f i yassl:yassl_imp.obj
 0001:00042490       ?end@?$vector@U?$pair@HP6APEAVHandShakeBase@yaSSL@@XZ@mySTL@@@mySTL@@QEBAPEBU?$pair@HP6APEAVHandShakeBase@yaSSL@@XZ@2@XZ 0000000140043490 f i yassl:yassl_imp.obj
 0001:000424a0       ?begin@?$vector@U?$pair@HP6APEAUServerKeyBase@yaSSL@@XZ@mySTL@@@mySTL@@QEBAPEBU?$pair@HP6APEAUServerKeyBase@yaSSL@@XZ@2@XZ 00000001400434a0 f i yassl:yassl_imp.obj
 0001:000424b0       ?end@?$vector@U?$pair@HP6APEAUServerKeyBase@yaSSL@@XZ@mySTL@@@mySTL@@QEBAPEBU?$pair@HP6APEAUServerKeyBase@yaSSL@@XZ@2@XZ 00000001400434b0 f i yassl:yassl_imp.obj
 0001:000424c0       ?begin@?$vector@U?$pair@HP6APEAUClientKeyBase@yaSSL@@XZ@mySTL@@@mySTL@@QEBAPEBU?$pair@HP6APEAUClientKeyBase@yaSSL@@XZ@2@XZ 00000001400434c0 f i yassl:yassl_imp.obj
 0001:000424d0       ?end@?$vector@U?$pair@HP6APEAUClientKeyBase@yaSSL@@XZ@mySTL@@@mySTL@@QEBAPEBU?$pair@HP6APEAUClientKeyBase@yaSSL@@XZ@2@XZ 00000001400434d0 f i yassl:yassl_imp.obj
 0001:000424e0       ??0iterator@?$list@PEAE@mySTL@@QEAA@PEAUnode@12@@Z 00000001400434e0 f i yassl:yassl_imp.obj
 0001:000424f0       ?capacity@?$vector@U?$pair@HP6APEAUMessage@yaSSL@@XZ@mySTL@@@mySTL@@QEBA_KXZ 00000001400434f0 f i yassl:yassl_imp.obj
 0001:00042500       ?size@?$vector@U?$pair@HP6APEAUMessage@yaSSL@@XZ@mySTL@@@mySTL@@QEBA_KXZ 0000000140043500 f i yassl:yassl_imp.obj
 0001:00042510       ?capacity@?$vector@U?$pair@HP6APEAVHandShakeBase@yaSSL@@XZ@mySTL@@@mySTL@@QEBA_KXZ 0000000140043510 f i yassl:yassl_imp.obj
 0001:00042520       ?size@?$vector@U?$pair@HP6APEAVHandShakeBase@yaSSL@@XZ@mySTL@@@mySTL@@QEBA_KXZ 0000000140043520 f i yassl:yassl_imp.obj
 0001:00042530       ?capacity@?$vector@U?$pair@HP6APEAUServerKeyBase@yaSSL@@XZ@mySTL@@@mySTL@@QEBA_KXZ 0000000140043530 f i yassl:yassl_imp.obj
 0001:00042540       ?size@?$vector@U?$pair@HP6APEAUServerKeyBase@yaSSL@@XZ@mySTL@@@mySTL@@QEBA_KXZ 0000000140043540 f i yassl:yassl_imp.obj
 0001:00042550       ?capacity@?$vector@U?$pair@HP6APEAUClientKeyBase@yaSSL@@XZ@mySTL@@@mySTL@@QEBA_KXZ 0000000140043550 f i yassl:yassl_imp.obj
 0001:00042560       ?size@?$vector@U?$pair@HP6APEAUClientKeyBase@yaSSL@@XZ@mySTL@@@mySTL@@QEBA_KXZ 0000000140043560 f i yassl:yassl_imp.obj
 0001:00042570       ??$ysDelete@UServerKeyBase@yaSSL@@@yaSSL@@YAXPEAUServerKeyBase@0@@Z 0000000140043570 f i yassl:yassl_imp.obj
 0001:00042590       ??$ysDelete@UClientKeyBase@yaSSL@@@yaSSL@@YAXPEAUClientKeyBase@0@@Z 0000000140043590 f i yassl:yassl_imp.obj
 0001:000425b0       ??$construct@U?$pair@HP6APEAUMessage@yaSSL@@XZ@mySTL@@U12@@mySTL@@YAXPEAU?$pair@HP6APEAUMessage@yaSSL@@XZ@0@AEBU10@@Z 00000001400435b0 f i yassl:yassl_imp.obj
 0001:000425d0       ??$construct@U?$pair@HP6APEAVHandShakeBase@yaSSL@@XZ@mySTL@@U12@@mySTL@@YAXPEAU?$pair@HP6APEAVHandShakeBase@yaSSL@@XZ@0@AEBU10@@Z 00000001400435d0 f i yassl:yassl_imp.obj
 0001:000425f0       ??$construct@U?$pair@HP6APEAUServerKeyBase@yaSSL@@XZ@mySTL@@U12@@mySTL@@YAXPEAU?$pair@HP6APEAUServerKeyBase@yaSSL@@XZ@0@AEBU10@@Z 00000001400435f0 f i yassl:yassl_imp.obj
 0001:00042610       ??$construct@U?$pair@HP6APEAUClientKeyBase@yaSSL@@XZ@mySTL@@U12@@mySTL@@YAXPEAU?$pair@HP6APEAUClientKeyBase@yaSSL@@XZ@0@AEBU10@@Z 0000000140043610 f i yassl:yassl_imp.obj
 0001:00042630       ??$ysDelete@UAuth@yaSSL@@@yaSSL@@YAXPEAUAuth@0@@Z 0000000140043630 f i yassl:yassl_imp.obj
 0001:00042650       ??$ysDelete@VHandShakeBase@yaSSL@@@yaSSL@@YAXPEAVHandShakeBase@0@@Z 0000000140043650 f i yassl:yassl_imp.obj
 0001:00042670       ??$uninit_copy@PEAU?$pair@HP6APEAUMessage@yaSSL@@XZ@mySTL@@PEAU12@@mySTL@@YAPEAU?$pair@HP6APEAUMessage@yaSSL@@XZ@0@PEAU10@00@Z 0000000140043670 f i yassl:yassl_imp.obj
 0001:000426a0       ??$uninit_copy@PEAU?$pair@HP6APEAVHandShakeBase@yaSSL@@XZ@mySTL@@PEAU12@@mySTL@@YAPEAU?$pair@HP6APEAVHandShakeBase@yaSSL@@XZ@0@PEAU10@00@Z 00000001400436a0 f i yassl:yassl_imp.obj
 0001:000426d0       ??$uninit_copy@PEAU?$pair@HP6APEAUServerKeyBase@yaSSL@@XZ@mySTL@@PEAU12@@mySTL@@YAPEAU?$pair@HP6APEAUServerKeyBase@yaSSL@@XZ@0@PEAU10@00@Z 00000001400436d0 f i yassl:yassl_imp.obj
 0001:00042700       ??$uninit_copy@PEAU?$pair@HP6APEAUClientKeyBase@yaSSL@@XZ@mySTL@@PEAU12@@mySTL@@YAPEAU?$pair@HP6APEAUClientKeyBase@yaSSL@@XZ@0@PEAU10@00@Z 0000000140043700 f i yassl:yassl_imp.obj
 0001:00042730       ??$GetArrayMemory@U?$pair@HP6APEAUMessage@yaSSL@@XZ@mySTL@@@mySTL@@YAPEAU?$pair@HP6APEAUMessage@yaSSL@@XZ@0@_K@Z 0000000140043730 f i yassl:yassl_imp.obj
 0001:00042740       ??$swap@PEAU?$pair@HP6APEAUMessage@yaSSL@@XZ@mySTL@@@mySTL@@YAXAEAPEAU?$pair@HP6APEAUMessage@yaSSL@@XZ@0@0@Z 0000000140043740 f i yassl:yassl_imp.obj
 0001:00042750       ??$GetArrayMemory@U?$pair@HP6APEAVHandShakeBase@yaSSL@@XZ@mySTL@@@mySTL@@YAPEAU?$pair@HP6APEAVHandShakeBase@yaSSL@@XZ@0@_K@Z 0000000140043750 f i yassl:yassl_imp.obj
 0001:00042760       ??$swap@PEAU?$pair@HP6APEAVHandShakeBase@yaSSL@@XZ@mySTL@@@mySTL@@YAXAEAPEAU?$pair@HP6APEAVHandShakeBase@yaSSL@@XZ@0@0@Z 0000000140043760 f i yassl:yassl_imp.obj
 0001:00042770       ??$GetArrayMemory@U?$pair@HP6APEAUServerKeyBase@yaSSL@@XZ@mySTL@@@mySTL@@YAPEAU?$pair@HP6APEAUServerKeyBase@yaSSL@@XZ@0@_K@Z 0000000140043770 f i yassl:yassl_imp.obj
 0001:00042780       ??$swap@PEAU?$pair@HP6APEAUServerKeyBase@yaSSL@@XZ@mySTL@@@mySTL@@YAXAEAPEAU?$pair@HP6APEAUServerKeyBase@yaSSL@@XZ@0@0@Z 0000000140043780 f i yassl:yassl_imp.obj
 0001:00042790       ??$GetArrayMemory@U?$pair@HP6APEAUClientKeyBase@yaSSL@@XZ@mySTL@@@mySTL@@YAPEAU?$pair@HP6APEAUClientKeyBase@yaSSL@@XZ@0@_K@Z 0000000140043790 f i yassl:yassl_imp.obj
 0001:000427a0       ??$swap@PEAU?$pair@HP6APEAUClientKeyBase@yaSSL@@XZ@mySTL@@@mySTL@@YAXAEAPEAU?$pair@HP6APEAUClientKeyBase@yaSSL@@XZ@0@0@Z 00000001400437a0 f i yassl:yassl_imp.obj
 0001:000427b0       ??0?$pair@HP6APEAUMessage@yaSSL@@XZ@mySTL@@QEAA@AEBHAEBQ6APEAUMessage@yaSSL@@XZ@Z 00000001400437b0 f i yassl:yassl_imp.obj
 0001:000427c0       ??0?$pair@HP6APEAVHandShakeBase@yaSSL@@XZ@mySTL@@QEAA@AEBHAEBQ6APEAVHandShakeBase@yaSSL@@XZ@Z 00000001400437c0 f i yassl:yassl_imp.obj
 0001:000427d0       ??0?$pair@HP6APEAUServerKeyBase@yaSSL@@XZ@mySTL@@QEAA@AEBHAEBQ6APEAUServerKeyBase@yaSSL@@XZ@Z 00000001400437d0 f i yassl:yassl_imp.obj
 0001:000427e0       ??0?$pair@HP6APEAUClientKeyBase@yaSSL@@XZ@mySTL@@QEAA@AEBHAEBQ6APEAUClientKeyBase@yaSSL@@XZ@Z 00000001400437e0 f i yassl:yassl_imp.obj
 0001:000427f0       ??0node@?$list@PEAE@mySTL@@QEAA@PEAE@Z 00000001400437f0 f i yassl:yassl_imp.obj
 0001:00042810       ??$destroy@Unode@?$list@PEAE@mySTL@@@mySTL@@YAXPEAUnode@?$list@PEAE@0@@Z 0000000140043810 f i yassl:yassl_imp.obj
 0001:00042820       ??$swap@PEAE@mySTL@@YAXAEAPEAE0@Z 0000000140043820 f i yassl:yassl_imp.obj
 0001:00042830       ??$ysDelete@E@yaSSL@@YAXPEAE@Z 0000000140043830 f i yassl:yassl_imp.obj
 0001:00042840       ??0Alert@yaSSL@@QEAA@XZ    0000000140043840 f i yassl:yassl_imp.obj
 0001:00042850       ??_GAlert@yaSSL@@UEAAPEAXI@Z 0000000140043850 f i yassl:yassl_imp.obj
 0001:00042850       ??_EAlert@yaSSL@@UEAAPEAXI@Z 0000000140043850 f i yassl:yassl_imp.obj
 0001:00042880       ??_EHandShakeHeader@yaSSL@@UEAAPEAXI@Z 0000000140043880 f i yassl:yassl_imp.obj
 0001:00042880       ??_GHandShakeHeader@yaSSL@@UEAAPEAXI@Z 0000000140043880 f i yassl:yassl_imp.obj
 0001:000428b0       ?build@EncryptedPreMasterSecret@yaSSL@@UEAAXAEAVSSL@2@@Z 00000001400438b0 f   yassl:yassl_imp.obj
 0001:00042a30       ?build@ClientDiffieHellmanPublic@yaSSL@@UEAAXAEAVSSL@2@@Z 0000000140043a30 f   yassl:yassl_imp.obj
 0001:00042b20       ?read@EncryptedPreMasterSecret@yaSSL@@UEAAXAEAVSSL@2@AEAVinput_buffer@2@@Z 0000000140043b20 f   yassl:yassl_imp.obj
 0001:00042c80       ??0EncryptedPreMasterSecret@yaSSL@@QEAA@XZ 0000000140043c80 f   yassl:yassl_imp.obj
 0001:00042ca0       ??1EncryptedPreMasterSecret@yaSSL@@UEAA@XZ 0000000140043ca0 f   yassl:yassl_imp.obj
 0001:00042cd0       ?read@ClientDiffieHellmanPublic@yaSSL@@UEAAXAEAVSSL@2@AEAVinput_buffer@2@@Z 0000000140043cd0 f   yassl:yassl_imp.obj
 0001:00042dc0       ??1ClientDiffieHellmanPublic@yaSSL@@UEAA@XZ 0000000140043dc0 f   yassl:yassl_imp.obj
 0001:00042df0       ?read@DH_Server@yaSSL@@UEAAXAEAVSSL@2@AEAVinput_buffer@2@@Z 0000000140043df0 f   yassl:yassl_imp.obj
 0001:000432c0       ?SetSuites@Parameters@yaSSL@@QEAAXUProtocolVersion@2@_N11@Z 00000001400442c0 f   yassl:yassl_imp.obj
 0001:00043580       ??_GChangeCipherSpec@yaSSL@@UEAAPEAXI@Z 0000000140044580 f i yassl:yassl_imp.obj
 0001:00043580       ??_EChangeCipherSpec@yaSSL@@UEAAPEAXI@Z 0000000140044580 f i yassl:yassl_imp.obj
 0001:000435b0       ?set@Alert@yaSSL@@UEAAAEAVinput_buffer@2@AEAV32@@Z 00000001400445b0 f   yassl:yassl_imp.obj
 0001:000435c0       ?get@Alert@yaSSL@@UEBAAEAVoutput_buffer@2@AEAV32@@Z 00000001400445c0 f   yassl:yassl_imp.obj
 0001:000435d0       ??_EData@yaSSL@@UEAAPEAXI@Z 00000001400445d0 f i yassl:yassl_imp.obj
 0001:000435d0       ??_GData@yaSSL@@UEAAPEAXI@Z 00000001400445d0 f i yassl:yassl_imp.obj
 0001:00043600       ?get@Data@yaSSL@@UEBAAEAVoutput_buffer@2@AEAV32@@Z 0000000140044600 f   yassl:yassl_imp.obj
 0001:00043610       ??0Certificate@yaSSL@@QEAA@PEBVx509@1@@Z 0000000140044610 f   yassl:yassl_imp.obj
 0001:00043650       ??_ECertificate@yaSSL@@UEAAPEAXI@Z 0000000140044650 f i yassl:yassl_imp.obj
 0001:00043650       ??_GCertificate@yaSSL@@UEAAPEAXI@Z 0000000140044650 f i yassl:yassl_imp.obj
 0001:00043680       ??1ServerDHParams@yaSSL@@QEAA@XZ 0000000140044680 f   yassl:yassl_imp.obj
 0001:000436b0       ?Process@ServerHello@yaSSL@@UEAAXAEAVinput_buffer@2@AEAVSSL@2@@Z 00000001400446b0 f   yassl:yassl_imp.obj
 0001:000438c0       ??_EServerHello@yaSSL@@UEAAPEAXI@Z 00000001400448c0 f i yassl:yassl_imp.obj
 0001:000438c0       ??_GServerHello@yaSSL@@UEAAPEAXI@Z 00000001400448c0 f i yassl:yassl_imp.obj
 0001:000438f0       ??_GServerHelloDone@yaSSL@@UEAAPEAXI@Z 00000001400448f0 f i yassl:yassl_imp.obj
 0001:000438f0       ??_EServerHelloDone@yaSSL@@UEAAPEAXI@Z 00000001400448f0 f i yassl:yassl_imp.obj
 0001:00043920       ?Process@ClientHello@yaSSL@@UEAAXAEAVinput_buffer@2@AEAVSSL@2@@Z 0000000140044920 f   yassl:yassl_imp.obj
 0001:00043ca0       ??_GClientHello@yaSSL@@UEAAPEAXI@Z 0000000140044ca0 f i yassl:yassl_imp.obj
 0001:00043ca0       ??_EClientHello@yaSSL@@UEAAPEAXI@Z 0000000140044ca0 f i yassl:yassl_imp.obj
 0001:00043cd0       ??6yaSSL@@YAAEAVoutput_buffer@0@AEAV10@AEBVServerKeyExchange@0@@Z 0000000140044cd0 f   yassl:yassl_imp.obj
 0001:00043d20       ??1ServerKeyExchange@yaSSL@@UEAA@XZ 0000000140044d20 f   yassl:yassl_imp.obj
 0001:00043d50       ?get@ServerKeyExchange@yaSSL@@UEBAAEAVoutput_buffer@2@AEAV32@@Z 0000000140044d50 f   yassl:yassl_imp.obj
 0001:00043d60       ??1CertificateVerify@yaSSL@@UEAA@XZ 0000000140044d60 f   yassl:yassl_imp.obj
 0001:00043d90       ?set@CertificateVerify@yaSSL@@UEAAAEAVinput_buffer@2@AEAV32@@Z 0000000140044d90 f   yassl:yassl_imp.obj
 0001:00043da0       ?get@CertificateVerify@yaSSL@@UEBAAEAVoutput_buffer@2@AEAV32@@Z 0000000140044da0 f   yassl:yassl_imp.obj
 0001:00043db0       ??6yaSSL@@YAAEAVoutput_buffer@0@AEAV10@AEBVClientKeyExchange@0@@Z 0000000140044db0 f   yassl:yassl_imp.obj
 0001:00043e00       ??1ClientKeyExchange@yaSSL@@UEAA@XZ 0000000140044e00 f   yassl:yassl_imp.obj
 0001:00043e30       ?get@ClientKeyExchange@yaSSL@@UEBAAEAVoutput_buffer@2@AEAV32@@Z 0000000140044e30 f   yassl:yassl_imp.obj
 0001:00043e40       ?CleanPreMaster@Connection@yaSSL@@QEAAXXZ 0000000140044e40 f   yassl:yassl_imp.obj
 0001:00043e80       ?CreateAlert@yaSSL@@YAPEAUMessage@1@XZ 0000000140044e80 f   yassl:yassl_imp.obj
 0001:00043eb0       ?CreateHelloRequest@yaSSL@@YAPEAVHandShakeBase@1@XZ 0000000140044eb0 f   yassl:yassl_imp.obj
 0001:00043ee0       ??_EHelloRequest@yaSSL@@UEAAPEAXI@Z 0000000140044ee0 f i yassl:yassl_imp.obj
 0001:00043ee0       ??_GHelloRequest@yaSSL@@UEAAPEAXI@Z 0000000140044ee0 f i yassl:yassl_imp.obj
 0001:00043f10       ?CreateRSAServerKEA@yaSSL@@YAPEAUServerKeyBase@1@XZ 0000000140044f10 f   yassl:yassl_imp.obj
 0001:00043f40       ??_GRSA_Server@yaSSL@@UEAAPEAXI@Z 0000000140044f40 f i yassl:yassl_imp.obj
 0001:00043f40       ??_ERSA_Server@yaSSL@@UEAAPEAXI@Z 0000000140044f40 f i yassl:yassl_imp.obj
 0001:00043f70       ?CreateFortezzaServerKEA@yaSSL@@YAPEAUServerKeyBase@1@XZ 0000000140044f70 f   yassl:yassl_imp.obj
 0001:00043fa0       ??_EFortezza_Server@yaSSL@@UEAAPEAXI@Z 0000000140044fa0 f i yassl:yassl_imp.obj
 0001:00043fa0       ??_GFortezza_Server@yaSSL@@UEAAPEAXI@Z 0000000140044fa0 f i yassl:yassl_imp.obj
 0001:00043fd0       ?CreateRSAClient@yaSSL@@YAPEAUClientKeyBase@1@XZ 0000000140044fd0 f   yassl:yassl_imp.obj
 0001:00044000       ?CreateFortezzaClient@yaSSL@@YAPEAUClientKeyBase@1@XZ 0000000140045000 f   yassl:yassl_imp.obj
 0001:00044030       ??_EFortezzaKeys@yaSSL@@UEAAPEAXI@Z 0000000140045030 f i yassl:yassl_imp.obj
 0001:00044030       ??_GFortezzaKeys@yaSSL@@UEAAPEAXI@Z 0000000140045030 f i yassl:yassl_imp.obj
 0001:00044060       ?begin@?$list@PEAE@mySTL@@QEBA?AViterator@12@XZ 0000000140045060 f i yassl:yassl_imp.obj
 0001:00044070       ?end@?$list@PEAE@mySTL@@QEBA?AViterator@12@XZ 0000000140045070 f i yassl:yassl_imp.obj
 0001:00044080       ?CreateObject@?$Factory@VHandShakeBase@yaSSL@@HP6APEAV12@XZ@yaSSL@@QEBAPEAVHandShakeBase@2@AEBH@Z 0000000140045080 f i yassl:yassl_imp.obj
 0001:000440b0       ?CreateObject@?$Factory@UServerKeyBase@yaSSL@@HP6APEAU12@XZ@yaSSL@@QEBAPEAUServerKeyBase@2@AEBH@Z 00000001400450b0 f i yassl:yassl_imp.obj
 0001:000440e0       ?CreateObject@?$Factory@UClientKeyBase@yaSSL@@HP6APEAU12@XZ@yaSSL@@QEBAPEAUClientKeyBase@2@AEBH@Z 00000001400450e0 f i yassl:yassl_imp.obj
 0001:00044110       ?Destroy@?$auto_ptr@UAuth@yaSSL@@@mySTL@@AEAAXXZ 0000000140045110 f i yassl:yassl_imp.obj
 0001:00044120       ?Destroy@?$auto_ptr@VHandShakeBase@yaSSL@@@mySTL@@AEAAXXZ 0000000140045120 f i yassl:yassl_imp.obj
 0001:00044130       ?Destroy@?$auto_array@E@mySTL@@AEAAXXZ 0000000140045130 f i yassl:yassl_imp.obj
 0001:00044140       ??0?$vector_base@U?$pair@HP6APEAUMessage@yaSSL@@XZ@mySTL@@@mySTL@@QEAA@_K@Z 0000000140045140 f i yassl:yassl_imp.obj
 0001:00044180       ?Swap@?$vector_base@U?$pair@HP6APEAUMessage@yaSSL@@XZ@mySTL@@@mySTL@@QEAAXAEAU12@@Z 0000000140045180 f i yassl:yassl_imp.obj
 0001:000441b0       ??0?$vector_base@U?$pair@HP6APEAVHandShakeBase@yaSSL@@XZ@mySTL@@@mySTL@@QEAA@_K@Z 00000001400451b0 f i yassl:yassl_imp.obj
 0001:000441f0       ?Swap@?$vector_base@U?$pair@HP6APEAVHandShakeBase@yaSSL@@XZ@mySTL@@@mySTL@@QEAAXAEAU12@@Z 00000001400451f0 f i yassl:yassl_imp.obj
 0001:00044220       ??0?$vector_base@U?$pair@HP6APEAUServerKeyBase@yaSSL@@XZ@mySTL@@@mySTL@@QEAA@_K@Z 0000000140045220 f i yassl:yassl_imp.obj
 0001:00044260       ?Swap@?$vector_base@U?$pair@HP6APEAUServerKeyBase@yaSSL@@XZ@mySTL@@@mySTL@@QEAAXAEAU12@@Z 0000000140045260 f i yassl:yassl_imp.obj
 0001:00044290       ??0?$vector_base@U?$pair@HP6APEAUClientKeyBase@yaSSL@@XZ@mySTL@@@mySTL@@QEAA@_K@Z 0000000140045290 f i yassl:yassl_imp.obj
 0001:000442d0       ?Swap@?$vector_base@U?$pair@HP6APEAUClientKeyBase@yaSSL@@XZ@mySTL@@@mySTL@@QEAAXAEAU12@@Z 00000001400452d0 f i yassl:yassl_imp.obj
 0001:00044300       ?push_back@?$list@PEAE@mySTL@@QEAAXPEAE@Z 0000000140045300 f i yassl:yassl_imp.obj
 0001:00044370       ??$make_pair@HP6APEAUMessage@yaSSL@@XZ@mySTL@@YA?AU?$pair@HP6APEAUMessage@yaSSL@@XZ@0@AEBHAEBQ6APEAUMessage@yaSSL@@XZ@Z 0000000140045370 f i yassl:yassl_imp.obj
 0001:00044380       ??$make_pair@HP6APEAVHandShakeBase@yaSSL@@XZ@mySTL@@YA?AU?$pair@HP6APEAVHandShakeBase@yaSSL@@XZ@0@AEBHAEBQ6APEAVHandShakeBase@yaSSL@@XZ@Z 0000000140045380 f i yassl:yassl_imp.obj
 0001:00044390       ??$make_pair@HP6APEAUServerKeyBase@yaSSL@@XZ@mySTL@@YA?AU?$pair@HP6APEAUServerKeyBase@yaSSL@@XZ@0@AEBHAEBQ6APEAUServerKeyBase@yaSSL@@XZ@Z 0000000140045390 f i yassl:yassl_imp.obj
 0001:000443a0       ??$make_pair@HP6APEAUClientKeyBase@yaSSL@@XZ@mySTL@@YA?AU?$pair@HP6APEAUClientKeyBase@yaSSL@@XZ@0@AEBHAEBQ6APEAUClientKeyBase@yaSSL@@XZ@Z 00000001400453a0 f i yassl:yassl_imp.obj
 0001:000443b0       ??$checked_delete@E@yaSSL@@YAXPEAE@Z 00000001400453b0 f i yassl:yassl_imp.obj
 0001:000443c0       ?createKey@ClientKeyExchange@yaSSL@@QEAAXAEAVSSL@2@@Z 00000001400453c0 f   yassl:yassl_imp.obj
 0001:00044450       ?createKey@ServerKeyExchange@yaSSL@@QEAAXAEAVSSL@2@@Z 0000000140045450 f   yassl:yassl_imp.obj
 0001:000444e0       ??_GEncryptedPreMasterSecret@yaSSL@@UEAAPEAXI@Z 00000001400454e0 f i yassl:yassl_imp.obj
 0001:000444e0       ??_EEncryptedPreMasterSecret@yaSSL@@UEAAPEAXI@Z 00000001400454e0 f i yassl:yassl_imp.obj
 0001:00044510       ??_EClientDiffieHellmanPublic@yaSSL@@UEAAPEAXI@Z 0000000140045510 f i yassl:yassl_imp.obj
 0001:00044510       ??_GClientDiffieHellmanPublic@yaSSL@@UEAAPEAXI@Z 0000000140045510 f i yassl:yassl_imp.obj
 0001:00044540       ??0DH_Server@yaSSL@@QEAA@XZ 0000000140045540 f   yassl:yassl_imp.obj
 0001:00044570       ??1DH_Server@yaSSL@@UEAA@XZ 0000000140045570 f   yassl:yassl_imp.obj
 0001:000445b0       ??0Parameters@yaSSL@@QEAA@W4ConnectionEnd@1@AEBUCiphers@1@UProtocolVersion@1@_N@Z 00000001400455b0 f   yassl:yassl_imp.obj
 0001:00044670       ?Process@ServerKeyExchange@yaSSL@@UEAAXAEAVinput_buffer@2@AEAVSSL@2@@Z 0000000140045670 f   yassl:yassl_imp.obj
 0001:000446e0       ??0ServerKeyExchange@yaSSL@@QEAA@AEAVSSL@1@@Z 00000001400456e0 f   yassl:yassl_imp.obj
 0001:00044710       ??_GServerKeyExchange@yaSSL@@UEAAPEAXI@Z 0000000140045710 f i yassl:yassl_imp.obj
 0001:00044710       ??_EServerKeyExchange@yaSSL@@UEAAPEAXI@Z 0000000140045710 f i yassl:yassl_imp.obj
 0001:00044740       ?Build@CertificateRequest@yaSSL@@QEAAXXZ 0000000140045740 f   yassl:yassl_imp.obj
 0001:00044760       ??5yaSSL@@YAAEAVinput_buffer@0@AEAV10@AEAVCertificateRequest@0@@Z 0000000140045760 f   yassl:yassl_imp.obj
 0001:00044860       ??6yaSSL@@YAAEAVoutput_buffer@0@AEAV10@AEBVCertificateRequest@0@@Z 0000000140045860 f   yassl:yassl_imp.obj
 0001:00044930       ??_ECertificateVerify@yaSSL@@UEAAPEAXI@Z 0000000140045930 f i yassl:yassl_imp.obj
 0001:00044930       ??_GCertificateVerify@yaSSL@@UEAAPEAXI@Z 0000000140045930 f i yassl:yassl_imp.obj
 0001:00044960       ?Process@ClientKeyExchange@yaSSL@@UEAAXAEAVinput_buffer@2@AEAVSSL@2@@Z 0000000140045960 f   yassl:yassl_imp.obj
 0001:00044a00       ??0ClientKeyExchange@yaSSL@@QEAA@AEAVSSL@1@@Z 0000000140045a00 f   yassl:yassl_imp.obj
 0001:00044a30       ??_EClientKeyExchange@yaSSL@@UEAAPEAXI@Z 0000000140045a30 f i yassl:yassl_imp.obj
 0001:00044a30       ??_GClientKeyExchange@yaSSL@@UEAAPEAXI@Z 0000000140045a30 f i yassl:yassl_imp.obj
 0001:00044a60       ??1Connection@yaSSL@@QEAA@XZ 0000000140045a60 f   yassl:yassl_imp.obj
 0001:00044a90       ?CreateDHServerKEA@yaSSL@@YAPEAUServerKeyBase@1@XZ 0000000140045a90 f   yassl:yassl_imp.obj
 0001:00044ac0       ??1?$auto_ptr@UAuth@yaSSL@@@mySTL@@QEAA@XZ 0000000140045ac0 f i yassl:yassl_imp.obj
 0001:00044ad0       ?reset@?$auto_ptr@UAuth@yaSSL@@@mySTL@@QEAAXPEAUAuth@yaSSL@@@Z 0000000140045ad0 f i yassl:yassl_imp.obj
 0001:00044b00       ??1?$auto_ptr@VHandShakeBase@yaSSL@@@mySTL@@QEAA@XZ 0000000140045b00 f i yassl:yassl_imp.obj
 0001:00044b10       ??1?$auto_array@E@mySTL@@QEAA@XZ 0000000140045b10 f i yassl:yassl_imp.obj
 0001:00044b20       ?reset@?$auto_array@E@mySTL@@QEAAXPEAE@Z 0000000140045b20 f i yassl:yassl_imp.obj
 0001:00044b50       ?Swap@?$vector@U?$pair@HP6APEAUMessage@yaSSL@@XZ@mySTL@@@mySTL@@QEAAXAEAV12@@Z 0000000140045b50 f i yassl:yassl_imp.obj
 0001:00044b80       ??0?$vector@U?$pair@HP6APEAUMessage@yaSSL@@XZ@mySTL@@@mySTL@@AEAA@_KAEBV01@@Z 0000000140045b80 f i yassl:yassl_imp.obj
 0001:00044bf0       ?Swap@?$vector@U?$pair@HP6APEAVHandShakeBase@yaSSL@@XZ@mySTL@@@mySTL@@QEAAXAEAV12@@Z 0000000140045bf0 f i yassl:yassl_imp.obj
 0001:00044c20       ??0?$vector@U?$pair@HP6APEAVHandShakeBase@yaSSL@@XZ@mySTL@@@mySTL@@AEAA@_KAEBV01@@Z 0000000140045c20 f i yassl:yassl_imp.obj
 0001:00044c90       ?Swap@?$vector@U?$pair@HP6APEAUServerKeyBase@yaSSL@@XZ@mySTL@@@mySTL@@QEAAXAEAV12@@Z 0000000140045c90 f i yassl:yassl_imp.obj
 0001:00044cc0       ??0?$vector@U?$pair@HP6APEAUServerKeyBase@yaSSL@@XZ@mySTL@@@mySTL@@AEAA@_KAEBV01@@Z 0000000140045cc0 f i yassl:yassl_imp.obj
 0001:00044d30       ?Swap@?$vector@U?$pair@HP6APEAUClientKeyBase@yaSSL@@XZ@mySTL@@@mySTL@@QEAAXAEAV12@@Z 0000000140045d30 f i yassl:yassl_imp.obj
 0001:00044d60       ??0?$vector@U?$pair@HP6APEAUClientKeyBase@yaSSL@@XZ@mySTL@@@mySTL@@AEAA@_KAEBV01@@Z 0000000140045d60 f i yassl:yassl_imp.obj
 0001:00044dd0       ??1?$list@PEAE@mySTL@@QEAA@XZ 0000000140045dd0 f i yassl:yassl_imp.obj
 0001:00044e00       ??$?RE@del_ptr_zero@yaSSL@@QEBAXAEAPEAE@Z 0000000140045e00 f i yassl:yassl_imp.obj
 0001:00044e10       ?build@DH_Server@yaSSL@@UEAAXAEAVSSL@2@@Z 0000000140045e10 f   yassl:yassl_imp.obj
 0001:00045320       ??_EDH_Server@yaSSL@@UEAAPEAXI@Z 0000000140046320 f i yassl:yassl_imp.obj
 0001:00045320       ??_GDH_Server@yaSSL@@UEAAPEAXI@Z 0000000140046320 f i yassl:yassl_imp.obj
 0001:00045350       ?Process@HandShakeHeader@yaSSL@@UEAAXAEAVinput_buffer@2@AEAVSSL@2@@Z 0000000140046350 f   yassl:yassl_imp.obj
 0001:00045450       ??0CertificateRequest@yaSSL@@QEAA@XZ 0000000140046450 f   yassl:yassl_imp.obj
 0001:00045490       ?set@CertificateRequest@yaSSL@@UEAAAEAVinput_buffer@2@AEAV32@@Z 0000000140046490 f   yassl:yassl_imp.obj
 0001:000454a0       ?get@CertificateRequest@yaSSL@@UEBAAEAVoutput_buffer@2@AEAV32@@Z 00000001400464a0 f   yassl:yassl_imp.obj
 0001:000454b0       ?Build@CertificateVerify@yaSSL@@QEAAXAEAVSSL@2@@Z 00000001400464b0 f   yassl:yassl_imp.obj
 0001:000456c0       ?CreateCertificateRequest@yaSSL@@YAPEAVHandShakeBase@1@XZ 00000001400466c0 f   yassl:yassl_imp.obj
 0001:000456f0       ?push_back@?$vector@U?$pair@HP6APEAUMessage@yaSSL@@XZ@mySTL@@@mySTL@@QEAAXAEBU?$pair@HP6APEAUMessage@yaSSL@@XZ@2@@Z 00000001400466f0 f i yassl:yassl_imp.obj
 0001:000457d0       ?reserve@?$vector@U?$pair@HP6APEAUMessage@yaSSL@@XZ@mySTL@@@mySTL@@QEAAX_K@Z 00000001400467d0 f i yassl:yassl_imp.obj
 0001:00045860       ?push_back@?$vector@U?$pair@HP6APEAVHandShakeBase@yaSSL@@XZ@mySTL@@@mySTL@@QEAAXAEBU?$pair@HP6APEAVHandShakeBase@yaSSL@@XZ@2@@Z 0000000140046860 f i yassl:yassl_imp.obj
 0001:00045940       ?reserve@?$vector@U?$pair@HP6APEAVHandShakeBase@yaSSL@@XZ@mySTL@@@mySTL@@QEAAX_K@Z 0000000140046940 f i yassl:yassl_imp.obj
 0001:000459d0       ?push_back@?$vector@U?$pair@HP6APEAUServerKeyBase@yaSSL@@XZ@mySTL@@@mySTL@@QEAAXAEBU?$pair@HP6APEAUServerKeyBase@yaSSL@@XZ@2@@Z 00000001400469d0 f i yassl:yassl_imp.obj
 0001:00045ab0       ?reserve@?$vector@U?$pair@HP6APEAUServerKeyBase@yaSSL@@XZ@mySTL@@@mySTL@@QEAAX_K@Z 0000000140046ab0 f i yassl:yassl_imp.obj
 0001:00045b40       ?push_back@?$vector@U?$pair@HP6APEAUClientKeyBase@yaSSL@@XZ@mySTL@@@mySTL@@QEAAXAEBU?$pair@HP6APEAUClientKeyBase@yaSSL@@XZ@2@@Z 0000000140046b40 f i yassl:yassl_imp.obj
 0001:00045c20       ?reserve@?$vector@U?$pair@HP6APEAUClientKeyBase@yaSSL@@XZ@mySTL@@@mySTL@@QEAAX_K@Z 0000000140046c20 f i yassl:yassl_imp.obj
 0001:00045cb0       ??$for_each@Viterator@?$list@PEAE@mySTL@@Udel_ptr_zero@yaSSL@@@mySTL@@YA?AUdel_ptr_zero@yaSSL@@Viterator@?$list@PEAE@0@0U12@@Z 0000000140046cb0 f i yassl:yassl_imp.obj
 0001:00045d10       ??1CertificateRequest@yaSSL@@UEAA@XZ 0000000140046d10 f   yassl:yassl_imp.obj
 0001:00045d60       ?Reserve@?$Factory@UMessage@yaSSL@@HP6APEAU12@XZ@yaSSL@@QEAAX_K@Z 0000000140046d60 f i yassl:yassl_imp.obj
 0001:00045df0       ?Register@?$Factory@UMessage@yaSSL@@HP6APEAU12@XZ@yaSSL@@QEAAXAEBHP6APEAUMessage@2@XZ@Z 0000000140046df0 f i yassl:yassl_imp.obj
 0001:00045ed0       ?Reserve@?$Factory@VHandShakeBase@yaSSL@@HP6APEAV12@XZ@yaSSL@@QEAAX_K@Z 0000000140046ed0 f i yassl:yassl_imp.obj
 0001:00045f60       ?Register@?$Factory@VHandShakeBase@yaSSL@@HP6APEAV12@XZ@yaSSL@@QEAAXAEBHP6APEAVHandShakeBase@2@XZ@Z 0000000140046f60 f i yassl:yassl_imp.obj
 0001:00046040       ?Reserve@?$Factory@UServerKeyBase@yaSSL@@HP6APEAU12@XZ@yaSSL@@QEAAX_K@Z 0000000140047040 f i yassl:yassl_imp.obj
 0001:000460d0       ?Register@?$Factory@UServerKeyBase@yaSSL@@HP6APEAU12@XZ@yaSSL@@QEAAXAEBHP6APEAUServerKeyBase@2@XZ@Z 00000001400470d0 f i yassl:yassl_imp.obj
 0001:000461b0       ?Reserve@?$Factory@UClientKeyBase@yaSSL@@HP6APEAU12@XZ@yaSSL@@QEAAX_K@Z 00000001400471b0 f i yassl:yassl_imp.obj
 0001:00046240       ?Register@?$Factory@UClientKeyBase@yaSSL@@HP6APEAU12@XZ@yaSSL@@QEAAXAEBHP6APEAUClientKeyBase@2@XZ@Z 0000000140047240 f i yassl:yassl_imp.obj
 0001:00046320       ??_ECertificateRequest@yaSSL@@UEAAPEAXI@Z 0000000140047320 f i yassl:yassl_imp.obj
 0001:00046320       ??_GCertificateRequest@yaSSL@@UEAAPEAXI@Z 0000000140047320 f i yassl:yassl_imp.obj
 0001:00046350       ?InitMessageFactory@yaSSL@@YAXAEAV?$Factory@UMessage@yaSSL@@HP6APEAU12@XZ@1@@Z 0000000140047350 f   yassl:yassl_imp.obj
 0001:00046680       ?InitHandShakeFactory@yaSSL@@YAXAEAV?$Factory@VHandShakeBase@yaSSL@@HP6APEAV12@XZ@1@@Z 0000000140047680 f   yassl:yassl_imp.obj
 0001:00046dc0       ?InitServerKeyFactory@yaSSL@@YAXAEAV?$Factory@UServerKeyBase@yaSSL@@HP6APEAU12@XZ@1@@Z 0000000140047dc0 f   yassl:yassl_imp.obj
 0001:00047050       ?InitClientKeyFactory@yaSSL@@YAXAEAV?$Factory@UClientKeyBase@yaSSL@@HP6APEAU12@XZ@1@@Z 0000000140048050 f   yassl:yassl_imp.obj
 0001:000472e0       ??0Socket@yaSSL@@QEAA@_K@Z 00000001400482e0 f   yassl:socket_wrapper.obj
 0001:000472f0       ?set_fd@Socket@yaSSL@@QEAAX_K@Z 00000001400482f0 f   yassl:socket_wrapper.obj
 0001:00047300       ?get_fd@Socket@yaSSL@@QEBA_KXZ 0000000140048300 f   yassl:socket_wrapper.obj
 0001:00047310       ??1Socket@yaSSL@@QEAA@XZ   0000000140048310 f   yassl:socket_wrapper.obj
 0001:00047320       ?closeSocket@Socket@yaSSL@@QEAAXXZ 0000000140048320 f   yassl:socket_wrapper.obj
 0001:00047350       ?get_ready@Socket@yaSSL@@QEBAIXZ 0000000140048350 f   yassl:socket_wrapper.obj
 0001:00047380       ?shutDown@Socket@yaSSL@@QEAAXH@Z 0000000140048380 f   yassl:socket_wrapper.obj
 0001:00047390       ?get_lastError@Socket@yaSSL@@SAHXZ 0000000140048390 f   yassl:socket_wrapper.obj
 0001:000473a0       ?WouldBlock@Socket@yaSSL@@QEBA_NXZ 00000001400483a0 f   yassl:socket_wrapper.obj
 0001:000473b0       ?IsNonBlocking@Socket@yaSSL@@QEBA_NXZ 00000001400483b0 f   yassl:socket_wrapper.obj
 0001:000473c0       ?set_lastError@Socket@yaSSL@@SAXH@Z 00000001400483c0 f   yassl:socket_wrapper.obj
 0001:000473d0       ?send@Socket@yaSSL@@QEAAIPEBEIAEAIH@Z 00000001400483d0 f   yassl:socket_wrapper.obj
 0001:00047480       ?receive@Socket@yaSSL@@QEAAIPEAEIH@Z 0000000140048480 f   yassl:socket_wrapper.obj
 0001:000474f0       ?wait@Socket@yaSSL@@QEAA_NXZ 00000001400484f0 f   yassl:socket_wrapper.obj
 0001:00047520       ??0Log@yaSSL@@QEAA@PEBD@Z  0000000140048520 f   yassl:log.obj
 0001:00047530       ??1Log@yaSSL@@QEAA@XZ      0000000140048530 f   yassl:log.obj
 0001:00047540       ?Trace@Log@yaSSL@@QEAAXPEBD@Z 0000000140048540 f   yassl:log.obj
 0001:00047550       ?ShowTCP@Log@yaSSL@@QEAAX_K_N@Z 0000000140048550 f   yassl:log.obj
 0001:00047560       ?ShowData@Log@yaSSL@@QEAAXI_N@Z 0000000140048560 f   yassl:log.obj
 0001:00047570       ?buildClientHello@yaSSL@@YAXAEAVSSL@1@AEAVClientHello@1@@Z 0000000140048570 f   yassl:handshake.obj
 0001:00047680       ?buildServerHello@yaSSL@@YAXAEAVSSL@1@AEAVServerHello@1@@Z 0000000140048680 f   yassl:handshake.obj
 0001:000477b0       ?hashHandShake@yaSSL@@YAXAEAVSSL@1@AEBVinput_buffer@1@I@Z 00000001400487b0 f   yassl:handshake.obj
 0001:00047840       ?buildOutput@?A0x5c10b036@yaSSL@@YAXAEAVoutput_buffer@2@AEBURecordLayerHeader@2@AEBUMessage@2@@Z 0000000140048840 f   yassl:handshake.obj
 0001:00047890       ?buildOutput@?A0x5c10b036@yaSSL@@YAXAEAVoutput_buffer@2@AEBURecordLayerHeader@2@AEBVHandShakeHeader@2@AEBVHandShakeBase@2@@Z 0000000140048890 f   yassl:handshake.obj
 0001:00047900       ?buildHeader@?A0x5c10b036@yaSSL@@YAXAEAVSSL@2@AEAURecordLayerHeader@2@AEBUMessage@2@@Z 0000000140048900 f   yassl:handshake.obj
 0001:00047970       ?buildHeaders@?A0x5c10b036@yaSSL@@YAXAEAVSSL@2@AEAVHandShakeHeader@2@AEAURecordLayerHeader@2@AEBVHandShakeBase@2@@Z 0000000140048970 f   yassl:handshake.obj
 0001:00047a10       ?hashHandShake@?A0x5c10b036@yaSSL@@YAXAEAVSSL@2@AEBVoutput_buffer@2@_N@Z 0000000140048a10 f   yassl:handshake.obj
 0001:00047ac0       ?buildMD5@?A0x5c10b036@yaSSL@@YAXAEAVSSL@2@AEAVFinished@2@PEBE@Z 0000000140048ac0 f   yassl:handshake.obj
 0001:00047c70       ?buildSHA@?A0x5c10b036@yaSSL@@YAXAEAVSSL@2@AEAVFinished@2@PEBE@Z 0000000140048c70 f   yassl:handshake.obj
 0001:00047e20       ?decrypt_message@?A0x5c10b036@yaSSL@@YAXAEAVSSL@2@AEAVinput_buffer@2@I@Z 0000000140048e20 f   yassl:handshake.obj
 0001:00047f20       ??6?A0x5c10b036@yaSSL@@YAAEAVoutput_buffer@1@AEAV21@AEBVinput_buffer@1@@Z 0000000140048f20 f   yassl:handshake.obj
 0001:00047f70       ??0RecordLayerHeader@yaSSL@@QEAA@XZ 0000000140048f70 f i yassl:handshake.obj
 0001:00047f90       ?get_xor@?A0x5c10b036@yaSSL@@YAXPEAEIAEAVoutput_buffer@2@1@Z 0000000140048f90 f   yassl:handshake.obj
 0001:00048010       ?buildMD5_CertVerify@?A0x5c10b036@yaSSL@@YAXAEAVSSL@2@PEAE@Z 0000000140049010 f   yassl:handshake.obj
 0001:000481e0       ?buildSHA_CertVerify@?A0x5c10b036@yaSSL@@YAXAEAVSSL@2@PEAE@Z 00000001400491e0 f   yassl:handshake.obj
 0001:000483a0       ?hmac@yaSSL@@YAXAEAVSSL@1@PEAEPEBEIW4ContentType@1@_N@Z 00000001400493a0 f   yassl:handshake.obj
 0001:00048560       ?build_certHashes@yaSSL@@YAXAEAVSSL@1@AEAUHashes@1@@Z 0000000140049560 f   yassl:handshake.obj
 0001:00048660       ?sendClientHello@yaSSL@@YAXAEAVSSL@1@@Z 0000000140049660 f   yassl:handshake.obj
 0001:000487c0       ??0?$auto_ptr@UDigest@yaSSL@@@mySTL@@QEAA@PEAUDigest@yaSSL@@@Z 00000001400497c0 f i yassl:handshake.obj
 0001:000487d0       ??C?$auto_ptr@UDigest@yaSSL@@@mySTL@@QEBAPEAUDigest@yaSSL@@XZ 00000001400497d0 f i yassl:handshake.obj
 0001:000487e0       ??0?$auto_ptr@UMessage@yaSSL@@@mySTL@@QEAA@PEAUMessage@yaSSL@@@Z 00000001400497e0 f i yassl:handshake.obj
 0001:000487f0       ??C?$auto_ptr@UMessage@yaSSL@@@mySTL@@QEBAPEAUMessage@yaSSL@@XZ 00000001400497f0 f i yassl:handshake.obj
 0001:00048800       ??D?$auto_ptr@UMessage@yaSSL@@@mySTL@@QEBAAEAUMessage@yaSSL@@XZ 0000000140049800 f i yassl:handshake.obj
 0001:00048810       ?get@?$auto_ptr@UMessage@yaSSL@@@mySTL@@QEBAPEAUMessage@yaSSL@@XZ 0000000140049810 f i yassl:handshake.obj
 0001:00048820       ??C?$auto_ptr@Voutput_buffer@yaSSL@@@mySTL@@QEBAPEAVoutput_buffer@yaSSL@@XZ 0000000140049820 f i yassl:handshake.obj
 0001:00048830       ?get@?$auto_ptr@Voutput_buffer@yaSSL@@@mySTL@@QEBAPEAVoutput_buffer@yaSSL@@XZ 0000000140049830 f i yassl:handshake.obj
 0001:00048840       ?release@?$auto_ptr@Voutput_buffer@yaSSL@@@mySTL@@QEAAPEAVoutput_buffer@yaSSL@@XZ 0000000140049840 f i yassl:handshake.obj
 0001:00048850       ?begin@?$vector@U?$pair@HP6APEAUMessage@yaSSL@@XZ@mySTL@@@mySTL@@QEBAPEBU?$pair@HP6APEAUMessage@yaSSL@@XZ@2@XZ 0000000140049850 f i yassl:handshake.obj
 0001:00048860       ?end@?$vector@U?$pair@HP6APEAUMessage@yaSSL@@XZ@mySTL@@@mySTL@@QEBAPEBU?$pair@HP6APEAUMessage@yaSSL@@XZ@2@XZ 0000000140049860 f i yassl:handshake.obj
 0001:00048870       ??$ysDelete@UMessage@yaSSL@@@yaSSL@@YAXPEAUMessage@0@@Z 0000000140049870 f i yassl:handshake.obj
 0001:00048890       ?ProcessOldClientHello@yaSSL@@YAXAEAVinput_buffer@1@AEAVSSL@1@@Z 0000000140049890 f   yassl:handshake.obj
 0001:00048b90       ?CreateObject@?$Factory@UMessage@yaSSL@@HP6APEAU12@XZ@yaSSL@@QEBAPEAUMessage@2@AEBH@Z 0000000140049b90 f i yassl:handshake.obj
 0001:00048bc0       ?Destroy@?$auto_ptr@UDigest@yaSSL@@@mySTL@@AEAAXXZ 0000000140049bc0 f i yassl:handshake.obj
 0001:00048bd0       ?Destroy@?$auto_ptr@UMessage@yaSSL@@@mySTL@@AEAAXXZ 0000000140049bd0 f i yassl:handshake.obj
 0001:00048be0       ??1?$auto_ptr@UDigest@yaSSL@@@mySTL@@QEAA@XZ 0000000140049be0 f i yassl:handshake.obj
 0001:00048bf0       ?reset@?$auto_ptr@UDigest@yaSSL@@@mySTL@@QEAAXPEAUDigest@yaSSL@@@Z 0000000140049bf0 f i yassl:handshake.obj
 0001:00048c20       ??1?$auto_ptr@UMessage@yaSSL@@@mySTL@@QEAA@XZ 0000000140049c20 f i yassl:handshake.obj
 0001:00048c30       ?p_hash@?A0x5c10b036@yaSSL@@YAXAEAVoutput_buffer@2@AEBV32@1W4MACAlgorithm@2@@Z 0000000140049c30 f   yassl:handshake.obj
 0001:00048e10       ?TLS_hmac@yaSSL@@YAXAEAVSSL@1@PEAEPEBEIW4ContentType@1@_N@Z 0000000140049e10 f   yassl:handshake.obj
 0001:00048ff0       ?PRF@yaSSL@@YAXPEAEIPEBEI1I1I@Z 0000000140049ff0 f   yassl:handshake.obj
 0001:00049190       ?DoProcessReply@yaSSL@@YAHAEAVSSL@1@@Z 000000014004a190 f   yassl:handshake.obj
 0001:00049540       ?processReply@yaSSL@@YAXAEAVSSL@1@@Z 000000014004a540 f   yassl:handshake.obj
 0001:000495b0       ?receiveData@yaSSL@@YAHAEAVSSL@1@AEAVData@1@_N@Z 000000014004a5b0 f   yassl:handshake.obj
 0001:000496c0       ?cipherFinished@?A0x5c10b036@yaSSL@@YAXAEAVSSL@2@AEAVFinished@2@AEAVoutput_buffer@2@@Z 000000014004a6c0 f   yassl:handshake.obj
 0001:00049a10       ?buildMessage@?A0x5c10b036@yaSSL@@YAXAEAVSSL@2@AEAVoutput_buffer@2@AEBUMessage@2@@Z 000000014004aa10 f   yassl:handshake.obj
 0001:00049d30       ?buildAlert@?A0x5c10b036@yaSSL@@YAXAEAVSSL@2@AEAVoutput_buffer@2@AEBVAlert@2@@Z 000000014004ad30 f   yassl:handshake.obj
 0001:00049dc0       ?buildFinishedTLS@?A0x5c10b036@yaSSL@@YAXAEAVSSL@2@AEAVFinished@2@PEBE@Z 000000014004adc0 f   yassl:handshake.obj
 0001:00049ed0       ?buildFinished@yaSSL@@YAXAEAVSSL@1@AEAVFinished@1@PEBE@Z 000000014004aed0 f   yassl:handshake.obj
 0001:00049fb0       ?sendClientKeyExchange@yaSSL@@YAXAEAVSSL@1@W4BufferOutput@1@@Z 000000014004afb0 f   yassl:handshake.obj
 0001:0004a110       ?sendServerKeyExchange@yaSSL@@YAXAEAVSSL@1@W4BufferOutput@1@@Z 000000014004b110 f   yassl:handshake.obj
 0001:0004a270       ?sendChangeCipher@yaSSL@@YAXAEAVSSL@1@W4BufferOutput@1@@Z 000000014004b270 f   yassl:handshake.obj
 0001:0004a390       ?sendFinished@yaSSL@@YAXAEAVSSL@1@W4ConnectionEnd@1@W4BufferOutput@1@@Z 000000014004b390 f   yassl:handshake.obj
 0001:0004a540       ?sendData@yaSSL@@YAHAEAVSSL@1@PEBXH@Z 000000014004b540 f   yassl:handshake.obj
 0001:0004a7a0       ?sendAlert@yaSSL@@YAHAEAVSSL@1@AEBVAlert@1@@Z 000000014004b7a0 f   yassl:handshake.obj
 0001:0004a820       ?sendServerHello@yaSSL@@YAXAEAVSSL@1@W4BufferOutput@1@@Z 000000014004b820 f   yassl:handshake.obj
 0001:0004a9e0       ?sendServerHelloDone@yaSSL@@YAXAEAVSSL@1@W4BufferOutput@1@@Z 000000014004b9e0 f   yassl:handshake.obj
 0001:0004ab00       ?sendCertificate@yaSSL@@YAXAEAVSSL@1@W4BufferOutput@1@@Z 000000014004bb00 f   yassl:handshake.obj
 0001:0004ac40       ?sendCertificateRequest@yaSSL@@YAXAEAVSSL@1@W4BufferOutput@1@@Z 000000014004bc40 f   yassl:handshake.obj
 0001:0004ada0       ?sendCertificateVerify@yaSSL@@YAXAEAVSSL@1@W4BufferOutput@1@@Z 000000014004bda0 f   yassl:handshake.obj
 0001:0004af00       ?GetKey@PublicKey@TaoCrypt@@QEBAPEBEXZ 000000014004bf00 f i yassl:cert_wrapper.obj
 0001:0004af10       ?size@PublicKey@TaoCrypt@@QEBAIXZ 000000014004bf10 f i yassl:cert_wrapper.obj
 0001:0004af20       ?GetPublicKey@CertDecoder@TaoCrypt@@QEBAAEBVPublicKey@2@XZ 000000014004bf20 f i yassl:cert_wrapper.obj
 0001:0004af30       ?GetKeyType@CertDecoder@TaoCrypt@@QEBA?AW4KeyType@2@XZ 000000014004bf30 f i yassl:cert_wrapper.obj
 0001:0004af40       ?GetIssuer@CertDecoder@TaoCrypt@@QEBAPEBDXZ 000000014004bf40 f i yassl:cert_wrapper.obj
 0001:0004af50       ?GetCommonName@CertDecoder@TaoCrypt@@QEBAPEBDXZ 000000014004bf50 f i yassl:cert_wrapper.obj
 0001:0004af60       ?GetHash@CertDecoder@TaoCrypt@@QEBAPEBEXZ 000000014004bf60 f i yassl:cert_wrapper.obj
 0001:0004af70       ?GetBeforeDate@CertDecoder@TaoCrypt@@QEBAPEBDXZ 000000014004bf70 f i yassl:cert_wrapper.obj
 0001:0004af80       ?GetAfterDate@CertDecoder@TaoCrypt@@QEBAPEBDXZ 000000014004bf80 f i yassl:cert_wrapper.obj
 0001:0004af90       ??0x509@yaSSL@@QEAA@I@Z    000000014004bf90 f   yassl:cert_wrapper.obj
 0001:0004afb0       ??0x509@yaSSL@@QEAA@AEBV01@@Z 000000014004bfb0 f   yassl:cert_wrapper.obj
 0001:0004aff0       ?get_length@x509@yaSSL@@QEBAIXZ 000000014004bff0 f   yassl:cert_wrapper.obj
 0001:0004b000       ?get_buffer@x509@yaSSL@@QEBAPEBEXZ 000000014004c000 f   yassl:cert_wrapper.obj
 0001:0004b010       ?use_buffer@x509@yaSSL@@QEAAPEAEXZ 000000014004c010 f   yassl:cert_wrapper.obj
 0001:0004b020       ?verifyPeer@CertManager@yaSSL@@QEBA_NXZ 000000014004c020 f   yassl:cert_wrapper.obj
 0001:0004b030       ?verifyNone@CertManager@yaSSL@@QEBA_NXZ 000000014004c030 f   yassl:cert_wrapper.obj
 0001:0004b040       ?failNoCert@CertManager@yaSSL@@QEBA_NXZ 000000014004c040 f   yassl:cert_wrapper.obj
 0001:0004b050       ?sendVerify@CertManager@yaSSL@@QEBA_NXZ 000000014004c050 f   yassl:cert_wrapper.obj
 0001:0004b060       ?setVerifyPeer@CertManager@yaSSL@@QEAAXXZ 000000014004c060 f   yassl:cert_wrapper.obj
 0001:0004b070       ?setVerifyNone@CertManager@yaSSL@@QEAAXXZ 000000014004c070 f   yassl:cert_wrapper.obj
 0001:0004b080       ?setFailNoCert@CertManager@yaSSL@@QEAAXXZ 000000014004c080 f   yassl:cert_wrapper.obj
 0001:0004b090       ?setSendVerify@CertManager@yaSSL@@QEAAXXZ 000000014004c090 f   yassl:cert_wrapper.obj
 0001:0004b0a0       ?setVerifyCallback@CertManager@yaSSL@@QEAAXP6AHHPEAUX509_STORE_CTX@2@@Z@Z 000000014004c0a0 f   yassl:cert_wrapper.obj
 0001:0004b0b0       ?get_peerKey@CertManager@yaSSL@@QEBAPEBEXZ 000000014004c0b0 f   yassl:cert_wrapper.obj
 0001:0004b0c0       ?get_peerX509@CertManager@yaSSL@@QEBAPEAVX509@2@XZ 000000014004c0c0 f   yassl:cert_wrapper.obj
 0001:0004b0d0       ?get_peerKeyType@CertManager@yaSSL@@QEBA?AW4SignatureAlgorithm@2@XZ 000000014004c0d0 f   yassl:cert_wrapper.obj
 0001:0004b0e0       ?get_keyType@CertManager@yaSSL@@QEBA?AW4SignatureAlgorithm@2@XZ 000000014004c0e0 f   yassl:cert_wrapper.obj
 0001:0004b0f0       ?get_peerKeyLength@CertManager@yaSSL@@QEBAIXZ 000000014004c0f0 f   yassl:cert_wrapper.obj
 0001:0004b100       ?get_privateKey@CertManager@yaSSL@@QEBAPEBEXZ 000000014004c100 f   yassl:cert_wrapper.obj
 0001:0004b110       ?get_privateKeyLength@CertManager@yaSSL@@QEBAIXZ 000000014004c110 f   yassl:cert_wrapper.obj
 0001:0004b120       ?setPeerX509@CertManager@yaSSL@@QEAAXPEAVX509@2@@Z 000000014004c120 f   yassl:cert_wrapper.obj
 0001:0004b230       ?size@?$list@PEAVx509@yaSSL@@@mySTL@@QEBA_KXZ 000000014004c230 f i yassl:cert_wrapper.obj
 0001:0004b240       ??0?$list@PEAVSigner@TaoCrypt@@@mySTL@@QEAA@XZ 000000014004c240 f i yassl:cert_wrapper.obj
 0001:0004b260       ??Dreverse_iterator@?$list@PEAVx509@yaSSL@@@mySTL@@QEBAAEAPEAVx509@yaSSL@@XZ 000000014004c260 f i yassl:cert_wrapper.obj
 0001:0004b270       ??Ereverse_iterator@?$list@PEAVx509@yaSSL@@@mySTL@@QEAAAEAV012@XZ 000000014004c270 f i yassl:cert_wrapper.obj
 0001:0004b280       ??0iterator@?$list@PEAVSigner@TaoCrypt@@@mySTL@@QEAA@PEAUnode@12@@Z 000000014004c280 f i yassl:cert_wrapper.obj
 0001:0004b290       ??0reverse_iterator@?$list@PEAVx509@yaSSL@@@mySTL@@QEAA@PEAUnode@12@@Z 000000014004c290 f i yassl:cert_wrapper.obj
 0001:0004b2a0       ?front@?$list@PEAVx509@yaSSL@@@mySTL@@QEBAPEAVx509@yaSSL@@XZ 000000014004c2a0 f i yassl:cert_wrapper.obj
 0001:0004b2b0       ??$swap@I@mySTL@@YAXAEAI0@Z 000000014004c2b0 f i yassl:cert_wrapper.obj
 0001:0004b2c0       ??Diterator@?$list@PEAVSigner@TaoCrypt@@@mySTL@@QEBAAEAPEAVSigner@TaoCrypt@@XZ 000000014004c2c0 f i yassl:cert_wrapper.obj
 0001:0004b2d0       ??Eiterator@?$list@PEAVSigner@TaoCrypt@@@mySTL@@QEAAAEAV012@XZ 000000014004c2d0 f i yassl:cert_wrapper.obj
 0001:0004b2e0       ??9iterator@?$list@PEAVSigner@TaoCrypt@@@mySTL@@QEBA_NAEBV012@@Z 000000014004c2e0 f i yassl:cert_wrapper.obj
 0001:0004b2f0       ??0node@?$list@PEAVSigner@TaoCrypt@@@mySTL@@QEAA@PEAVSigner@TaoCrypt@@@Z 000000014004c2f0 f i yassl:cert_wrapper.obj
 0001:0004b310       ??$destroy@Unode@?$list@PEAVSigner@TaoCrypt@@@mySTL@@@mySTL@@YAXPEAUnode@?$list@PEAVSigner@TaoCrypt@@@0@@Z 000000014004c310 f i yassl:cert_wrapper.obj
 0001:0004b320       ??$swap@PEAVSigner@TaoCrypt@@@mySTL@@YAXAEAPEAVSigner@TaoCrypt@@0@Z 000000014004c320 f i yassl:cert_wrapper.obj
 0001:0004b330       ??_GSigner@TaoCrypt@@QEAAPEAXI@Z 000000014004c330 f i yassl:cert_wrapper.obj
 0001:0004b360       ??1x509@yaSSL@@QEAA@XZ     000000014004c360 f   yassl:cert_wrapper.obj
 0001:0004b370       ?Swap@x509@yaSSL@@AEAAXAEAV12@@Z 000000014004c370 f   yassl:cert_wrapper.obj
 0001:0004b390       ??4x509@yaSSL@@QEAAAEAV01@AEBV01@@Z 000000014004c390 f   yassl:cert_wrapper.obj
 0001:0004b3d0       ?get_cert@CertManager@yaSSL@@QEBAPEBVx509@2@XZ 000000014004c3d0 f   yassl:cert_wrapper.obj
 0001:0004b3e0       ?rbegin@?$list@PEAVx509@yaSSL@@@mySTL@@QEBA?AVreverse_iterator@12@XZ 000000014004c3e0 f i yassl:cert_wrapper.obj
 0001:0004b3f0       ?begin@?$list@PEAVSigner@TaoCrypt@@@mySTL@@QEBA?AViterator@12@XZ 000000014004c3f0 f i yassl:cert_wrapper.obj
 0001:0004b400       ?end@?$list@PEAVSigner@TaoCrypt@@@mySTL@@QEBA?AViterator@12@XZ 000000014004c400 f i yassl:cert_wrapper.obj
 0001:0004b410       ?push_back@?$list@PEAVSigner@TaoCrypt@@@mySTL@@QEAAXPEAVSigner@TaoCrypt@@@Z 000000014004c410 f i yassl:cert_wrapper.obj
 0001:0004b480       ??$ysDelete@VSigner@TaoCrypt@@@yaSSL@@YAXPEAVSigner@TaoCrypt@@@Z 000000014004c480 f i yassl:cert_wrapper.obj
 0001:0004b4b0       ?AddPeerCert@CertManager@yaSSL@@QEAAXPEAVx509@2@@Z 000000014004c4b0 f   yassl:cert_wrapper.obj
 0001:0004b4c0       ?CopySelfCert@CertManager@yaSSL@@QEAAXPEBVx509@2@@Z 000000014004c4c0 f   yassl:cert_wrapper.obj
 0001:0004b510       ??1?$list@PEAVSigner@TaoCrypt@@@mySTL@@QEAA@XZ 000000014004c510 f i yassl:cert_wrapper.obj
 0001:0004b540       ??$checked_delete@VSigner@TaoCrypt@@@yaSSL@@YAXPEAVSigner@TaoCrypt@@@Z 000000014004c540 f i yassl:cert_wrapper.obj
 0001:0004b550       ??0CertManager@yaSSL@@QEAA@XZ 000000014004c550 f   yassl:cert_wrapper.obj
 0001:0004b5d0       ?CopyCaCert@CertManager@yaSSL@@QEAAHPEBVx509@2@@Z 000000014004c5d0 f   yassl:cert_wrapper.obj
 0001:0004b720       ?Validate@CertManager@yaSSL@@QEAAHXZ 000000014004c720 f   yassl:cert_wrapper.obj
 0001:0004bb60       ?SetPrivateKey@CertManager@yaSSL@@QEAAHAEBVx509@2@@Z 000000014004cb60 f   yassl:cert_wrapper.obj
 0001:0004bcf0       ??$?RVSigner@TaoCrypt@@@del_ptr_zero@yaSSL@@QEBAXAEAPEAVSigner@TaoCrypt@@@Z 000000014004ccf0 f i yassl:cert_wrapper.obj
 0001:0004bd00       ??$for_each@Viterator@?$list@PEAVSigner@TaoCrypt@@@mySTL@@Udel_ptr_zero@yaSSL@@@mySTL@@YA?AUdel_ptr_zero@yaSSL@@Viterator@?$list@PEAVSigner@TaoCrypt@@@0@0U12@@Z 000000014004cd00 f i yassl:cert_wrapper.obj
 0001:0004bd60       ??1CertManager@yaSSL@@QEAA@XZ 000000014004cd60 f   yassl:cert_wrapper.obj
 0001:0004bdf0       ?SetErrorString@yaSSL@@YAXKPEAD@Z 000000014004cdf0 f   yassl:yassl_error.obj
 0001:0004c230       ?check@NoCheck@yaSSL@@QEAAXII@Z 000000014004d230 f   yassl:buffer.obj
 0001:0004c240       ??0input_buffer@yaSSL@@QEAA@XZ 000000014004d240 f   yassl:buffer.obj
 0001:0004c260       ??0input_buffer@yaSSL@@QEAA@I@Z 000000014004d260 f   yassl:buffer.obj
 0001:0004c2a0       ?allocate@input_buffer@yaSSL@@QEAAXI@Z 000000014004d2a0 f   yassl:buffer.obj
 0001:0004c2d0       ?get_buffer@input_buffer@yaSSL@@QEBAPEAEXZ 000000014004d2d0 f   yassl:buffer.obj
 0001:0004c2e0       ?get_capacity@input_buffer@yaSSL@@QEBAIXZ 000000014004d2e0 f   yassl:buffer.obj
 0001:0004c2f0       ?get_current@input_buffer@yaSSL@@QEBAIXZ 000000014004d2f0 f   yassl:buffer.obj
 0001:0004c300       ?get_size@input_buffer@yaSSL@@QEBAIXZ 000000014004d300 f   yassl:buffer.obj
 0001:0004c310       ?get_remaining@input_buffer@yaSSL@@QEBAIXZ 000000014004d310 f   yassl:buffer.obj
 0001:0004c320       ?set_current@input_buffer@yaSSL@@QEAAXI@Z 000000014004d320 f   yassl:buffer.obj
 0001:0004c330       ??Ainput_buffer@yaSSL@@QEAAAEBEI@Z 000000014004d330 f   yassl:buffer.obj
 0001:0004c350       ?eof@input_buffer@yaSSL@@QEAA_NXZ 000000014004d350 f   yassl:buffer.obj
 0001:0004c360       ?peek@input_buffer@yaSSL@@QEBAEXZ 000000014004d360 f   yassl:buffer.obj
 0001:0004c370       ?read@input_buffer@yaSSL@@QEAAXPEAEI@Z 000000014004d370 f   yassl:buffer.obj
 0001:0004c3b0       ??0output_buffer@yaSSL@@QEAA@XZ 000000014004d3b0 f   yassl:buffer.obj
 0001:0004c3c0       ??0output_buffer@yaSSL@@QEAA@I@Z 000000014004d3c0 f   yassl:buffer.obj
 0001:0004c400       ?get_size@output_buffer@yaSSL@@QEBAIXZ 000000014004d400 f   yassl:buffer.obj
 0001:0004c410       ?get_capacity@output_buffer@yaSSL@@QEBAIXZ 000000014004d410 f   yassl:buffer.obj
 0001:0004c420       ?set_current@output_buffer@yaSSL@@QEAAXI@Z 000000014004d420 f   yassl:buffer.obj
 0001:0004c430       ?allocate@output_buffer@yaSSL@@QEAAXI@Z 000000014004d430 f   yassl:buffer.obj
 0001:0004c460       ?get_buffer@output_buffer@yaSSL@@QEBAPEBEXZ 000000014004d460 f   yassl:buffer.obj
 0001:0004c470       ??Aoutput_buffer@yaSSL@@QEAAAEAEI@Z 000000014004d470 f   yassl:buffer.obj
 0001:0004c480       ?eof@output_buffer@yaSSL@@QEAA_NXZ 000000014004d480 f   yassl:buffer.obj
 0001:0004c4a0       ?write@output_buffer@yaSSL@@QEAAXPEBEI@Z 000000014004d4a0 f   yassl:buffer.obj
 0001:0004c4d0       ??1input_buffer@yaSSL@@QEAA@XZ 000000014004d4d0 f   yassl:buffer.obj
 0001:0004c4e0       ?add_size@input_buffer@yaSSL@@QEAAXI@Z 000000014004d4e0 f   yassl:buffer.obj
 0001:0004c4f0       ?assign@input_buffer@yaSSL@@QEAAXPEBEI@Z 000000014004d4f0 f   yassl:buffer.obj
 0001:0004c520       ??0output_buffer@yaSSL@@QEAA@IPEBEI@Z 000000014004d520 f   yassl:buffer.obj
 0001:0004c580       ??1output_buffer@yaSSL@@QEAA@XZ 000000014004d580 f   yassl:buffer.obj
 0001:0004c590       ??0input_buffer@yaSSL@@QEAA@IPEBEI@Z 000000014004d590 f   yassl:buffer.obj
 0001:0004c5f0       ??0Mutex@yaSSL@@QEAA@XZ    000000014004d5f0 f   yassl:lock.obj
 0001:0004c610       ??1Mutex@yaSSL@@QEAA@XZ    000000014004d610 f   yassl:lock.obj
 0001:0004c620       ??0Lock@Mutex@yaSSL@@QEAA@AEAV12@@Z 000000014004d620 f   yassl:lock.obj
 0001:0004c640       ??1Lock@Mutex@yaSSL@@QEAA@XZ 000000014004d640 f   yassl:lock.obj
 0001:0004c650       ?timer@yaSSL@@YANXZ        000000014004d650 f   yassl:timer.obj
 0001:0004c6a0       ?lowResTimer@yaSSL@@YAIXZ  000000014004d6a0 f   yassl:timer.obj
 0001:0004c6c0       compress2                  000000014004d6c0 f   zlib:compress.obj
 0001:0004c780       compress                   000000014004d780 f   zlib:compress.obj
 0001:0004c7a0       compressBound              000000014004d7a0 f   zlib:compress.obj
 0001:0004c7c0       uncompress                 000000014004d7c0 f   zlib:uncompr.obj
 0001:0004c890       deflateSetDictionary       000000014004d890 f   zlib:deflate.obj
 0001:0004c9f0       deflateSetHeader           000000014004d9f0 f   zlib:deflate.obj
 0001:0004ca20       deflatePrime               000000014004da20 f   zlib:deflate.obj
 0001:0004ca60       deflateTune                000000014004da60 f   zlib:deflate.obj
 0001:0004caa0       deflateBound               000000014004daa0 f   zlib:deflate.obj
 0001:0004cb90       deflate                    000000014004db90 f   zlib:deflate.obj
 0001:0004d440       deflateEnd                 000000014004e440 f   zlib:deflate.obj
 0001:0004d520       deflateCopy                000000014004e520 f   zlib:deflate.obj
 0001:0004e730       deflateReset               000000014004f730 f   zlib:deflate.obj
 0001:0004e810       deflateParams              000000014004f810 f   zlib:deflate.obj
 0001:0004e920       deflateInit2_              000000014004f920 f   zlib:deflate.obj
 0001:0004ebb0       deflateInit_               000000014004fbb0 f   zlib:deflate.obj
 0001:0004ebf0       inflateReset               000000014004fbf0 f   zlib:inflate.obj
 0001:0004ec60       inflatePrime               000000014004fc60 f   zlib:inflate.obj
 0001:0004ecb0       inflateInit2_              000000014004fcb0 f   zlib:inflate.obj
 0001:0004edd0       inflateInit_               000000014004fdd0 f   zlib:inflate.obj
 0001:0004ef20       inflate                    000000014004ff20 f   zlib:inflate.obj
 0001:00050970       inflateEnd                 0000000140051970 f   zlib:inflate.obj
 0001:000509d0       inflateSetDictionary       00000001400519d0 f   zlib:inflate.obj
 0001:00050ac0       inflateGetHeader           0000000140051ac0 f   zlib:inflate.obj
 0001:00050b60       inflateSync                0000000140051b60 f   zlib:inflate.obj
 0001:00050c80       inflateSyncPoint           0000000140051c80 f   zlib:inflate.obj
 0001:00050cb0       inflateCopy                0000000140051cb0 f   zlib:inflate.obj
 0001:00050e40       adler32                    0000000140051e40 f   zlib:adler32.obj
 0001:00051150       adler32_combine            0000000140052150 f   zlib:adler32.obj
 0001:00051f40       _tr_tally                  0000000140052f40 f   zlib:trees.obj
 0001:00052720       _tr_init                   0000000140053720 f   zlib:trees.obj
 0001:00052b10       _tr_stored_block           0000000140053b10 f   zlib:trees.obj
 0001:00052bb0       _tr_align                  0000000140053bb0 f   zlib:trees.obj
 0001:00052de0       _tr_flush_block            0000000140053de0 f   zlib:trees.obj
 0001:00053010       get_crc_table              0000000140054010 f   zlib:crc32.obj
 0001:00053730       crc32_combine              0000000140054730 f   zlib:crc32.obj
 0001:00053820       crc32                      0000000140054820 f   zlib:crc32.obj
 0001:00053830       zlibVersion                0000000140054830 f   zlib:zutil.obj
 0001:00053840       zlibCompileFlags           0000000140054840 f   zlib:zutil.obj
 0001:00053850       zError                     0000000140054850 f   zlib:zutil.obj
 0001:00053870       zcalloc                    0000000140054870 f   zlib:zutil.obj
 0001:00053880       zcfree                     0000000140054880 f   zlib:zutil.obj
 0001:00053890       inflate_fast               0000000140054890 f   zlib:inffast.obj
 0001:00053d80       inflate_table              0000000140054d80 f   zlib:inftrees.obj
 0001:00054250       gethostname                0000000140055250 f   wsock32:WSOCK32.dll
 0001:00054256       ioctlsocket                0000000140055256 f   wsock32:WSOCK32.dll
 0001:0005425c       closesocket                000000014005525c f   wsock32:WSOCK32.dll
 0001:00054262       listen                     0000000140055262 f   wsock32:WSOCK32.dll
 0001:00054268       bind                       0000000140055268 f   wsock32:WSOCK32.dll
 0001:0005426e       setsockopt                 000000014005526e f   wsock32:WSOCK32.dll
 0001:00054274       htons                      0000000140055274 f   wsock32:WSOCK32.dll
 0001:0005427a       htonl                      000000014005527a f   wsock32:WSOCK32.dll
 0001:00054280       inet_addr                  0000000140055280 f   wsock32:WSOCK32.dll
 0001:00054286       socket                     0000000140055286 f   wsock32:WSOCK32.dll
 0001:0005428c       shutdown                   000000014005528c f   wsock32:WSOCK32.dll
 0001:00054292       accept                     0000000140055292 f   wsock32:WSOCK32.dll
 0001:00054298       __WSAFDIsSet               0000000140055298 f   wsock32:WSOCK32.dll
 0001:0005429e       select                     000000014005529e f   wsock32:WSOCK32.dll
 0001:000542a4       connect                    00000001400552a4 f   wsock32:WSOCK32.dll
 0001:000542aa       WSAGetLastError            00000001400552aa f   wsock32:WSOCK32.dll
 0001:000542b0       WSACleanup                 00000001400552b0 f   wsock32:WSOCK32.dll
 0001:000542b6       WSAStartup                 00000001400552b6 f   wsock32:WSOCK32.dll
 0001:000542bc       inet_ntoa                  00000001400552bc f   wsock32:WSOCK32.dll
 0001:000542c2       gethostbyname              00000001400552c2 f   wsock32:WSOCK32.dll
 0001:000542c8       recv                       00000001400552c8 f   wsock32:WSOCK32.dll
 0001:000542ce       send                       00000001400552ce f   wsock32:WSOCK32.dll
 0001:000542d4       ntohs                      00000001400552d4 f   wsock32:WSOCK32.dll
 0001:000542da       getpeername                00000001400552da f   wsock32:WSOCK32.dll
 0001:000542e0       WSASetLastError            00000001400552e0 f   wsock32:WSOCK32.dll
 0001:000542f0       _fpclear                   00000001400552f0 f   LIBCMT:fpinit.obj
 0001:00054300       _cfltcvt_init              0000000140055300 f   LIBCMT:fpinit.obj
 0001:00054390       __setfflag                 0000000140055390 f   LIBCMT:fpinit.obj
 0001:000543a0       _fpmath                    00000001400553a0 f   LIBCMT:fpinit.obj
 0001:00054430       ?name@type_info@@QEBAPEBDPEAU__type_info_node@@@Z 0000000140055430 f   LIBCMT:typinfo.obj
 0001:00054440       ??1type_info@@UEAA@XZ      0000000140055440 f   LIBCMT:typinfo.obj
 0001:00054450       ??_Gtype_info@@UEAAPEAXI@Z 0000000140055450 f i LIBCMT:typinfo.obj
 0001:00054450       ??_Etype_info@@UEAAPEAXI@Z 0000000140055450 f i LIBCMT:typinfo.obj
 0001:00054490       ?_name_internal_method@type_info@@QEBAPEBDPEAU__type_info_node@@@Z 0000000140055490 f   LIBCMT:typinfo.obj
 0001:000544a0       ?_type_info_dtor_internal_method@type_info@@QEAAXXZ 00000001400554a0 f   LIBCMT:typinfo.obj
 0001:000544b0       ??8type_info@@QEBA_NAEBV0@@Z 00000001400554b0 f   LIBCMT:typinfo.obj
 0001:000544e0       ??9type_info@@QEBA_NAEBV0@@Z 00000001400554e0 f   LIBCMT:typinfo.obj
 0001:00054510       ?before@type_info@@QEBAHAEBV1@@Z 0000000140055510 f   LIBCMT:typinfo.obj
 0001:00054540       ?raw_name@type_info@@QEBAPEBDXZ 0000000140055540 f   LIBCMT:typinfo.obj
 0001:00054550       ??0type_info@@AEAA@AEBV0@@Z 0000000140055550 f   LIBCMT:typinfo.obj
 0001:00054560       ??4type_info@@AEAAAEAV0@AEBV0@@Z 0000000140055560 f   LIBCMT:typinfo.obj
 0001:00054570       _purecall                  0000000140055570 f   LIBCMT:purevirt.obj
 0001:000545b0       _set_purecall_handler      00000001400555b0 f   LIBCMT:purevirt.obj
 0001:000545f0       _get_purecall_handler      00000001400555f0 f   LIBCMT:purevirt.obj
 0001:00054600       ??3@YAXPEAX@Z              0000000140055600 f   LIBCMT:delete.obj
 0001:00054610       strchr                     0000000140055610 f   LIBCMT:strchr.obj
 0001:000547a0       _stat64i32                 00000001400557a0 f   LIBCMT:stati32.obj
 0001:00054c10       atol                       0000000140055c10 f   LIBCMT:atox.obj
 0001:00054c20       _atol_l                    0000000140055c20 f   LIBCMT:atox.obj
 0001:00054c30       atoi                       0000000140055c30 f   LIBCMT:atox.obj
 0001:00054c40       _atoi_l                    0000000140055c40 f   LIBCMT:atox.obj
 0001:00054c50       _atoi64                    0000000140055c50 f   LIBCMT:atox.obj
 0001:00054c60       _atoi64_l                  0000000140055c60 f   LIBCMT:atox.obj
 0001:00054c70       __GSHandlerCheckCommon     0000000140055c70 f   LIBCMT:gshandler.obj
 0001:00054ce0       __GSHandlerCheck           0000000140055ce0 f   LIBCMT:gshandler.obj
 0001:00054d60       __security_check_cookie    0000000140055d60 f   LIBCMT:amdsecgs.obj
 0001:00054d80       _time64                    0000000140055d80 f   LIBCMT:time64.obj
 0001:00054dd0       ??0bad_alloc@std@@QEAA@XZ  0000000140055dd0 f i LIBCMT:new.obj
 0001:00054e00       ??1bad_alloc@std@@UEAA@XZ  0000000140055e00 f i LIBCMT:new.obj
 0001:00054e10       ??_Ebad_alloc@std@@UEAAPEAXI@Z 0000000140055e10 f i LIBCMT:new.obj
 0001:00054e10       ??_Gbad_alloc@std@@UEAAPEAXI@Z 0000000140055e10 f i LIBCMT:new.obj
 0001:00054e50       ??0bad_alloc@std@@QEAA@AEBV01@@Z 0000000140055e50 f i LIBCMT:new.obj
 0001:00054e80       ??2@YAPEAX_K@Z             0000000140055e80 f   LIBCMT:new.obj
 0001:00054f30       memset                     0000000140055f30 f   LIBCMT:memset.obj
 0001:00055030       strncmp                    0000000140056030 f   LIBCMT:strncmp.obj
 0001:000550f0       _snprintf                  00000001400560f0 f   LIBCMT:snprintf.obj
 0001:000551c0       _snprintf_l                00000001400561c0 f   LIBCMT:snprintf.obj
 0001:000551e0       strstr                     00000001400561e0 f   LIBCMT:strstr.obj
 0001:00055250       vfscanf                    0000000140056250 f   LIBCMT:fscanf.obj
 0001:00055430       fscanf                     0000000140056430 f   LIBCMT:fscanf.obj
 0001:00055470       _fscanf_l                  0000000140056470 f   LIBCMT:fscanf.obj
 0001:000554b0       fscanf_s                   00000001400564b0 f   LIBCMT:fscanf.obj
 0001:000554f0       _fscanf_s_l                00000001400564f0 f   LIBCMT:fscanf.obj
 0001:00055530       printf                     0000000140056530 f   LIBCMT:printf.obj
 0001:00055620       _printf_l                  0000000140056620 f   LIBCMT:printf.obj
 0001:00055650       _printf_s_l                0000000140056650 f   LIBCMT:printf.obj
 0001:00055680       printf_s                   0000000140056680 f   LIBCMT:printf.obj
 0001:000556b0       _printf_p_l                00000001400566b0 f   LIBCMT:printf.obj
 0001:000556e0       _printf_p                  00000001400566e0 f   LIBCMT:printf.obj
 0001:00055710       _set_printf_count_output   0000000140056710 f   LIBCMT:printf.obj
 0001:00055740       _get_printf_count_output   0000000140056740 f   LIBCMT:printf.obj
 0001:00055770       memmove                    0000000140056770     LIBCMT:memcpy.obj
 0001:00055770       memcpy                     0000000140056770 f   LIBCMT:memcpy.obj
 0001:00055ab0       _invoke_watson_if_error    0000000140056ab0 f i LIBCMT:strerror.obj
 0001:00055af0       _get_sys_err_msg           0000000140056af0 f i LIBCMT:strerror.obj
 0001:00055b30       strerror                   0000000140056b30 f   LIBCMT:strerror.obj
 0001:00055be0       strerror_s                 0000000140056be0 f   LIBCMT:strerror.obj
 0001:00055ca0       _get_errno_from_oserr      0000000140056ca0 f   LIBCMT:dosmap.obj
 0001:00055cf0       _errno                     0000000140056cf0 f   LIBCMT:dosmap.obj
 0001:00055d20       __doserrno                 0000000140056d20 f   LIBCMT:dosmap.obj
 0001:00055d50       _dosmaperr                 0000000140056d50 f   LIBCMT:dosmap.obj
 0001:00055de0       _set_errno                 0000000140056de0 f   LIBCMT:dosmap.obj
 0001:00055e30       _get_errno                 0000000140056e30 f   LIBCMT:dosmap.obj
 0001:00055e90       _set_doserrno              0000000140056e90 f   LIBCMT:dosmap.obj
 0001:00055ee0       _get_doserrno              0000000140056ee0 f   LIBCMT:dosmap.obj
 0001:00055f40       fprintf                    0000000140056f40 f   LIBCMT:fprintf.obj
 0001:00056120       _fprintf_l                 0000000140057120 f   LIBCMT:fprintf.obj
 0001:00056140       _fprintf_s_l               0000000140057140 f   LIBCMT:fprintf.obj
 0001:00056160       fprintf_s                  0000000140057160 f   LIBCMT:fprintf.obj
 0001:00056190       _fprintf_p_l               0000000140057190 f   LIBCMT:fprintf.obj
 0001:000561b0       _fprintf_p                 00000001400571b0 f   LIBCMT:fprintf.obj
 0001:000561e0       _vsnprintf_l               00000001400571e0 f   LIBCMT:vsnprint.obj
 0001:000562b0       _vsnprintf                 00000001400572b0 f   LIBCMT:vsnprint.obj
 0001:00056370       sprintf                    0000000140057370 f   LIBCMT:sprintf.obj
 0001:00056420       _sprintf_l                 0000000140057420 f   LIBCMT:sprintf.obj
 0001:00056440       sprintf_s                  0000000140057440 f   LIBCMT:sprintf.obj
 0001:00056470       _sprintf_s_l               0000000140057470 f   LIBCMT:sprintf.obj
 0001:00056490       _snprintf_s                0000000140057490 f   LIBCMT:sprintf.obj
 0001:000564c0       _snprintf_s_l              00000001400574c0 f   LIBCMT:sprintf.obj
 0001:000564f0       _sprintf_p                 00000001400574f0 f   LIBCMT:sprintf.obj
 0001:00056520       _sprintf_p_l               0000000140057520 f   LIBCMT:sprintf.obj
 0001:00056540       _scprintf                  0000000140057540 f   LIBCMT:sprintf.obj
 0001:00056570       _scprintf_p                0000000140057570 f   LIBCMT:sprintf.obj
 0001:000565a0       _scprintf_l                00000001400575a0 f   LIBCMT:sprintf.obj
 0001:000565d0       _scprintf_p_l              00000001400575d0 f   LIBCMT:sprintf.obj
 0001:00056600       __iob_func                 0000000140057600 f   LIBCMT:_file.obj
 0001:00056610       __initstdio                0000000140057610 f   LIBCMT:_file.obj
 0001:00056710       __endstdio                 0000000140057710 f   LIBCMT:_file.obj
 0001:00056740       _lock_file                 0000000140057740 f   LIBCMT:_file.obj
 0001:000567b0       _lock_file2                00000001400577b0 f   LIBCMT:_file.obj
 0001:000567f0       _unlock_file               00000001400577f0 f   LIBCMT:_file.obj
 0001:00056840       _unlock_file2              0000000140057840 f   LIBCMT:_file.obj
 0001:00056860       vfprintf_helper            0000000140057860 f   LIBCMT:vfprintf.obj
 0001:00056a50       _vfprintf_l                0000000140057a50 f   LIBCMT:vfprintf.obj
 0001:00056a80       _vfprintf_s_l              0000000140057a80 f   LIBCMT:vfprintf.obj
 0001:00056ab0       _vfprintf_p_l              0000000140057ab0 f   LIBCMT:vfprintf.obj
 0001:00056ae0       vfprintf                   0000000140057ae0 f   LIBCMT:vfprintf.obj
 0001:00056b10       vfprintf_s                 0000000140057b10 f   LIBCMT:vfprintf.obj
 0001:00056b40       _vfprintf_p                0000000140057b40 f   LIBCMT:vfprintf.obj
 0001:00056b70       setbuf                     0000000140057b70 f   LIBCMT:setbuf.obj
 0001:00056b90       _amsg_exit                 0000000140057b90 f   LIBCMT:crt0dat.obj
 0001:00056bc0       __crtCorExitProcess        0000000140057bc0 f   LIBCMT:crt0dat.obj
 0001:00056c00       __crtExitProcess           0000000140057c00 f   LIBCMT:crt0dat.obj
 0001:00056c40       _lockexit                  0000000140057c40 f   LIBCMT:crt0dat.obj
 0001:00056c50       _unlockexit                0000000140057c50 f   LIBCMT:crt0dat.obj
 0001:00056ca0       _initterm_e                0000000140057ca0 f   LIBCMT:crt0dat.obj
 0001:00056ce0       _get_osplatform            0000000140057ce0 f   LIBCMT:crt0dat.obj
 0001:00056d30       _get_osver                 0000000140057d30 f   LIBCMT:crt0dat.obj
 0001:00056d80       _get_winver                0000000140057d80 f   LIBCMT:crt0dat.obj
 0001:00056dd0       _get_winmajor              0000000140057dd0 f   LIBCMT:crt0dat.obj
 0001:00056e20       _get_winminor              0000000140057e20 f   LIBCMT:crt0dat.obj
 0001:00056e70       _get_wpgmptr               0000000140057e70 f   LIBCMT:crt0dat.obj
 0001:00056ec0       _get_pgmptr                0000000140057ec0 f   LIBCMT:crt0dat.obj
 0001:00056f10       _cinit                     0000000140057f10 f   LIBCMT:crt0dat.obj
 0001:00057120       exit                       0000000140058120 f   LIBCMT:crt0dat.obj
 0001:00057130       _exit                      0000000140058130 f   LIBCMT:crt0dat.obj
 0001:00057140       _cexit                     0000000140058140 f   LIBCMT:crt0dat.obj
 0001:00057150       _c_exit                    0000000140058150 f   LIBCMT:crt0dat.obj
 0001:00057160       _init_pointers             0000000140058160 f   LIBCMT:crt0dat.obj
 0001:000571d0       _initp_misc_winsig         00000001400581d0 f   LIBCMT:winsig.obj
 0001:000572f0       __get_sigabrt              00000001400582f0 f   LIBCMT:winsig.obj
 0001:00057300       __fpecode                  0000000140058300 f   LIBCMT:winsig.obj
 0001:00057320       __pxcptinfoptrs            0000000140058320 f   LIBCMT:winsig.obj
 0001:00057340       signal                     0000000140058340 f   LIBCMT:winsig.obj
 0001:00057600       raise                      0000000140058600 f   LIBCMT:winsig.obj
 0001:000578b0       srand                      00000001400588b0 f   LIBCMT:rand.obj
 0001:000578d0       rand                       00000001400588d0 f   LIBCMT:rand.obj
 0001:00057900       strrchr                    0000000140058900 f   LIBCMT:strrchr.obj
 0001:00057930       fgets                      0000000140058930 f   LIBCMT:fgets.obj
 0001:00057b90       _invoke_watson_if_oneof    0000000140058b90 f i LIBCMT:popen.obj
 0001:00057c80       _popen                     0000000140058c80 f   LIBCMT:popen.obj
 0001:00058460       _pclose                    0000000140059460 f   LIBCMT:popen.obj
 0001:00058580       setvbuf                    0000000140059580 f   LIBCMT:setvbuf.obj
 0001:00058720       feof                       0000000140059720 f   LIBCMT:feoferr.obj
 0001:00058760       ferror                     0000000140059760 f   LIBCMT:feoferr.obj
 0001:000587a0       floor                      00000001400597a0 f   LIBCMT:floor.obj
 0001:000588c0       memcmp                     00000001400598c0 f   LIBCMT:memcmp.obj
 0001:00058990       _getenv_helper_nolock      0000000140059990 f   LIBCMT:getenv.obj
 0001:00058c80       getenv                     0000000140059c80 f   LIBCMT:getenv.obj
 0001:00058d50       getenv_s                   0000000140059d50 f   LIBCMT:getenv.obj
 0001:00058eb0       _dupenv_s                  0000000140059eb0 f   LIBCMT:getenv.obj
 0001:00059010       ??0_LocaleUpdate@@QEAA@PEAUlocaleinfo_struct@@@Z 000000014005a010 f i LIBCMT:strtol.obj
 0001:000590d0       ??1_LocaleUpdate@@QEAA@XZ  000000014005a0d0 f i LIBCMT:strtol.obj
 0001:000590f0       ?GetLocaleT@_LocaleUpdate@@QEAAPEAUlocaleinfo_struct@@XZ 000000014005a0f0 f i LIBCMT:strtol.obj
 0001:00059490       strtol                     000000014005a490 f   LIBCMT:strtol.obj
 0001:000594d0       _strtol_l                  000000014005a4d0 f   LIBCMT:strtol.obj
 0001:00059500       strtoul                    000000014005a500 f   LIBCMT:strtol.obj
 0001:00059540       _strtoul_l                 000000014005a540 f   LIBCMT:strtol.obj
 0001:00059570       _isalpha_l                 000000014005a570 f i LIBCMT:_ctype.obj
 0001:00059680       isalpha                    000000014005a680 f i LIBCMT:_ctype.obj
 0001:000597a0       _isupper_l                 000000014005a7a0 f i LIBCMT:_ctype.obj
 0001:000598b0       isupper                    000000014005a8b0 f i LIBCMT:_ctype.obj
 0001:000599c0       _islower_l                 000000014005a9c0 f i LIBCMT:_ctype.obj
 0001:00059ad0       islower                    000000014005aad0 f i LIBCMT:_ctype.obj
 0001:00059be0       _isdigit_l                 000000014005abe0 f i LIBCMT:_ctype.obj
 0001:00059cf0       isdigit                    000000014005acf0 f i LIBCMT:_ctype.obj
 0001:00059e00       _isxdigit_l                000000014005ae00 f i LIBCMT:_ctype.obj
 0001:00059f10       isxdigit                   000000014005af10 f i LIBCMT:_ctype.obj
 0001:0005a020       _isspace_l                 000000014005b020 f i LIBCMT:_ctype.obj
 0001:0005a130       isspace                    000000014005b130 f i LIBCMT:_ctype.obj
 0001:0005a240       _ispunct_l                 000000014005b240 f i LIBCMT:_ctype.obj
 0001:0005a350       ispunct                    000000014005b350 f i LIBCMT:_ctype.obj
 0001:0005a460       _isalnum_l                 000000014005b460 f i LIBCMT:_ctype.obj
 0001:0005a570       isalnum                    000000014005b570 f i LIBCMT:_ctype.obj
 0001:0005a690       _isprint_l                 000000014005b690 f i LIBCMT:_ctype.obj
 0001:0005a7a0       isprint                    000000014005b7a0 f i LIBCMT:_ctype.obj
 0001:0005a8c0       _isgraph_l                 000000014005b8c0 f i LIBCMT:_ctype.obj
 0001:0005a9d0       isgraph                    000000014005b9d0 f i LIBCMT:_ctype.obj
 0001:0005aaf0       _iscntrl_l                 000000014005baf0 f i LIBCMT:_ctype.obj
 0001:0005ac00       iscntrl                    000000014005bc00 f i LIBCMT:_ctype.obj
 0001:0005ad10       __isascii                  000000014005bd10 f i LIBCMT:_ctype.obj
 0001:0005ad20       __toascii                  000000014005bd20 f i LIBCMT:_ctype.obj
 0001:0005ad30       _iscsymf_l                 000000014005bd30 f i LIBCMT:_ctype.obj
 0001:0005ad60       __iscsymf                  000000014005bd60 f i LIBCMT:_ctype.obj
 0001:0005ad90       _iscsym_l                  000000014005bd90 f i LIBCMT:_ctype.obj
 0001:0005adc0       __iscsym                   000000014005bdc0 f i LIBCMT:_ctype.obj
 0001:0005adf0       _MarkAllocaS               000000014005bdf0 f i LIBCMT:getch.obj
 0001:0005ae00       _freea                     000000014005be00 f i LIBCMT:getch.obj
 0001:0005ae20       _ungetch_nolock            000000014005be20 f   LIBCMT:getch.obj
 0001:0005ae40       _getextendedkeycode        000000014005be40 f   LIBCMT:getch.obj
 0001:0005aef0       _getch_nolock              000000014005bef0 f   LIBCMT:getch.obj
 0001:0005b0e0       _getche_nolock             000000014005c0e0 f   LIBCMT:getch.obj
 0001:0005b140       _kbhit_nolock              000000014005c140 f   LIBCMT:getch.obj
 0001:0005b2d0       _ungetch                   000000014005c2d0 f   LIBCMT:getch.obj
 0001:0005b320       _getch                     000000014005c320 f   LIBCMT:getch.obj
 0001:0005b370       _getche                    000000014005c370 f   LIBCMT:getch.obj
 0001:0005b3c0       _kbhit                     000000014005c3c0 f   LIBCMT:getch.obj
 0001:0005b410       _cputs                     000000014005c410 f   LIBCMT:cputs.obj
 0001:0005b4d0       _set_osplatform            000000014005c4d0 f i LIBCMT:crt0.obj
 0001:0005b4e0       _set_osver                 000000014005c4e0 f i LIBCMT:crt0.obj
 0001:0005b4f0       _set_winver                000000014005c4f0 f i LIBCMT:crt0.obj
 0001:0005b500       _set_winmajor              000000014005c500 f i LIBCMT:crt0.obj
 0001:0005b510       _set_winminor              000000014005c510 f i LIBCMT:crt0.obj
 0001:0005b840       mainCRTStartup             000000014005c840 f   LIBCMT:crt0.obj
 0001:0005b860       realloc                    000000014005c860 f   LIBCMT:realloc.obj
 0001:0005b950       _recalloc                  000000014005c950 f   LIBCMT:realloc.obj
 0001:0005ba00       _heap_alloc                000000014005ca00 f i LIBCMT:malloc.obj
 0001:0005ba50       malloc                     000000014005ca50 f   LIBCMT:malloc.obj
 0001:0005bb20       free                       000000014005cb20 f   LIBCMT:free.obj
 0001:0005bb70       _lseeki64_nolock           000000014005cb70 f   LIBCMT:lseeki64.obj
 0001:0005bc20       _lseeki64                  000000014005cc20 f   LIBCMT:lseeki64.obj
 0001:0005bd70       _telli64                   000000014005cd70 f   LIBCMT:telli64.obj
 0001:0005bd80       _fstat64i32                000000014005cd80 f   LIBCMT:fstati32.obj
 0001:0005c210       _findclose                 000000014005d210 f   LIBCMT:findfile.obj
 0001:0005c240       __timet_from_ft            000000014005d240 f   LIBCMT:findfile.obj
 0001:0005c2c0       _findfirst32               000000014005d2c0 f   LIBCMT:findfile.obj
 0001:0005c550       _findnext32                000000014005d550 f   LIBCMT:findfile.obj
 0001:0005c7d0       __time64_t_from_ft         000000014005d7d0 f   LIBCMT:findfi32.obj
 0001:0005c850       _findfirst64i32            000000014005d850 f   LIBCMT:findfi32.obj
 0001:0005caf0       _findnext64i32             000000014005daf0 f   LIBCMT:findfi32.obj
 0001:0005cd80       _set_osfhnd                000000014005dd80 f   LIBCMT:osfinfo.obj
 0001:0005ce40       _free_osfhnd               000000014005de40 f   LIBCMT:osfinfo.obj
 0001:0005cf10       _get_osfhandle             000000014005df10 f   LIBCMT:osfinfo.obj
 0001:0005cfb0       __lock_fhandle             000000014005dfb0 f   LIBCMT:osfinfo.obj
 0001:0005d080       _unlock_fhandle            000000014005e080 f   LIBCMT:osfinfo.obj
 0001:0005d0b0       _alloc_osfhnd              000000014005e0b0 f   LIBCMT:osfinfo.obj
 0001:0005d320       _open_osfhandle            000000014005e320 f   LIBCMT:osfinfo.obj
 0001:0005d470       _umask_s                   000000014005e470 f   LIBCMT:umask.obj
 0001:0005d4d0       _umask                     000000014005e4d0 f   LIBCMT:umask.obj
 0001:0005d4d0       umask                      000000014005e4d0 f   LIBCMT:umask.obj
 0001:0005d530       _localtime64_s             000000014005e530 f   LIBCMT:loctim64.obj
 0001:0005d8b0       _localtime64               000000014005e8b0 f   LIBCMT:loctim64.obj
 0001:0005d900       _endthread                 000000014005e900 f   LIBCMT:thread.obj
 0001:0005da50       _beginthread               000000014005ea50 f   LIBCMT:thread.obj
 0001:0005db70       _gmtime64_s                000000014005eb70 f   LIBCMT:gmtime64.obj
 0001:0005dea0       _gmtime64                  000000014005eea0 f   LIBCMT:gmtime64.obj
 0001:0005def0       fputs                      000000014005eef0 f   LIBCMT:fputs.obj
 0001:0005e0f0       puts                       000000014005f0f0 f   LIBCMT:puts.obj
 0001:0005e330       fputc                      000000014005f330 f   LIBCMT:fputc.obj
 0001:0005e4d0       putc                       000000014005f4d0 f   LIBCMT:fputc.obj
 0001:0005e670       _fclose_nolock             000000014005f670 f   LIBCMT:fclose.obj
 0001:0005e710       fclose                     000000014005f710 f   LIBCMT:fclose.obj
 0001:0005e7b0       _fsopen                    000000014005f7b0 f   LIBCMT:fopen.obj
 0001:0005e910       fopen                      000000014005f910 f   LIBCMT:fopen.obj
 0001:0005e920       fopen_s                    000000014005f920 f   LIBCMT:fopen.obj
 0001:0005e990       _set_daylight              000000014005f990 f i LIBCMT:tzset.obj
 0001:0005e9b0       _set_dstbias               000000014005f9b0 f i LIBCMT:tzset.obj
 0001:0005e9d0       _set_timezone              000000014005f9d0 f i LIBCMT:tzset.obj
 0001:0005f6c0       __tzset                    00000001400606c0 f   LIBCMT:tzset.obj
 0001:0005f720       _tzset                     0000000140060720 f   LIBCMT:tzset.obj
 0001:0005f770       _isindst                   0000000140060770 f   LIBCMT:tzset.obj
 0001:0005f7c0       _initp_misc_invarg         00000001400607c0 f   LIBCMT:invarg.obj
 0001:0005f7d0       _invoke_watson             00000001400607d0 f   LIBCMT:invarg.obj
 0001:0005f870       _set_invalid_parameter_handler 0000000140060870 f   LIBCMT:invarg.obj
 0001:0005f8b0       _get_invalid_parameter_handler 00000001400608b0 f   LIBCMT:invarg.obj
 0001:0005f8c0       ?_invoke_watson@@YAXPEBG00I_K@Z 00000001400608c0 f   LIBCMT:invarg.obj
 0001:0005f960       _invalid_parameter         0000000140060960 f   LIBCMT:invarg.obj
 0001:0005fa70       _invalid_parameter_noinfo  0000000140060a70 f   LIBCMT:invarg.obj
 0001:0005fb60       ?_invalid_parameter@@YAXPEBG00I_K@Z 0000000140060b60 f   LIBCMT:invarg.obj
 0001:0005fb80       _flush                     0000000140060b80 f   LIBCMT:fflush.obj
 0001:0005fc00       _fflush_nolock             0000000140060c00 f   LIBCMT:fflush.obj
 0001:0005fe10       fflush                     0000000140060e10 f   LIBCMT:fflush.obj
 0001:0005fe80       _flushall                  0000000140060e80 f   LIBCMT:fflush.obj
 0001:0005fe90       _fputchar                  0000000140060e90 f   LIBCMT:fputchar.obj
 0001:0005feb0       putchar                    0000000140060eb0 f   LIBCMT:fputchar.obj
 0001:0005fed0       _fread_nolock_s            0000000140060ed0 f   LIBCMT:fread.obj
 0001:000601b0       _fread_nolock              00000001400611b0 f   LIBCMT:fread.obj
 0001:000601d0       fread_s                    00000001400611d0 f   LIBCMT:fread.obj
 0001:000602b0       fread                      00000001400612b0 f   LIBCMT:fread.obj
 0001:000602d0       _ftell_nolock              00000001400612d0 f   LIBCMT:ftell.obj
 0001:000604f0       ftell                      00000001400614f0 f   LIBCMT:ftell.obj
 0001:00060580       _fseek_nolock              0000000140061580 f   LIBCMT:fseek.obj
 0001:00060640       fseek                      0000000140061640 f   LIBCMT:fseek.obj
 0001:00060720       _fwrite_nolock             0000000140061720 f   LIBCMT:fwrite.obj
 0001:000608e0       fwrite                     00000001400618e0 f   LIBCMT:fwrite.obj
 0001:000609b0       ldiv                       00000001400619b0 f   LIBCMT:ldiv.obj
 0001:00060ad0       qsort                      0000000140061ad0 f   LIBCMT:qsort.obj
 0001:00060e40       _isnan                     0000000140061e40 f   LIBCMT:ieeemisc.obj
 0001:00060e70       _isnanf                    0000000140061e70 f   LIBCMT:ieeemisc.obj
 0001:00060e90       _fpclass                   0000000140061e90 f   LIBCMT:ieeemisc.obj
 0001:00060f50       _fpclassf                  0000000140061f50 f   LIBCMT:ieeemisc.obj
 0001:00060fe0       _nextafter                 0000000140061fe0 f   LIBCMT:ieeemisc.obj
 0001:000611c0       _nextafterf                00000001400621c0 f   LIBCMT:ieeemisc.obj
 0001:00061370       _scalb                     0000000140062370 f   LIBCMT:ieeemisc.obj
 0001:000615c0       _scalbf                    00000001400625c0 f   LIBCMT:ieeemisc.obj
 0001:000617b0       _finite                    00000001400627b0 f   LIBCMT:_finite.obj
 0001:000617f0       strncpy                    00000001400627f0 f   LIBCMT:strncpy.obj
 0001:00061960       ??_V@YAXPEAX@Z             0000000140062960 f   LIBCMT:delete2.obj
 0001:00061970       ??_U@YAPEAX_K@Z            0000000140062970 f   LIBCMT:new2.obj
 0001:00061980       rewind                     0000000140062980 f   LIBCMT:rewind.obj
 0001:00061a90       strncat                    0000000140062a90 f   LIBCMT:strncat.obj
 0001:00061c30       _forcdecpt_l               0000000140062c30 f   LIBCMT:cvt.obj
 0001:00061d70       _cropzeros_l               0000000140062d70 f   LIBCMT:cvt.obj
 0001:00061ee0       _positive                  0000000140062ee0 f   LIBCMT:cvt.obj
 0001:00061f00       _fassign_l                 0000000140062f00 f   LIBCMT:cvt.obj
 0001:00061f50       _fassign                   0000000140062f50 f   LIBCMT:cvt.obj
 0001:00061fe0       _forcdecpt                 0000000140062fe0 f   LIBCMT:cvt.obj
 0001:00061ff0       _cropzeros                 0000000140062ff0 f   LIBCMT:cvt.obj
 0001:00062340       _cftoe_l                   0000000140063340 f   LIBCMT:cvt.obj
 0001:00062460       _cftoe                     0000000140063460 f   LIBCMT:cvt.obj
 0001:00062480       _cftoa_l                   0000000140063480 f   LIBCMT:cvt.obj
 0001:00062940       _cftoa                     0000000140063940 f   LIBCMT:cvt.obj
 0001:00062bc0       _cftof_l                   0000000140063bc0 f   LIBCMT:cvt.obj
 0001:00062cb0       _cftof                     0000000140063cb0 f   LIBCMT:cvt.obj
 0001:00062da0       _cftog_l                   0000000140063da0 f   LIBCMT:cvt.obj
 0001:00062f10       _cftog                     0000000140063f10 f   LIBCMT:cvt.obj
 0001:00062f30       _cfltcvt_l                 0000000140063f30 f   LIBCMT:cvt.obj
 0001:00062fd0       _cfltcvt                   0000000140063fd0 f   LIBCMT:cvt.obj
 0001:00063070       _initp_misc_cfltcvt_tab    0000000140064070 f   LIBCMT:cmiscdat.obj
 0001:000630b0       ?_Type_info_dtor@type_info@@CAXPEAV1@@Z 00000001400640b0 f   LIBCMT:typname.obj
 0001:00063150       ?_Name_base@type_info@@CAPEBDPEBV1@PEAU__type_info_node@@@Z 0000000140064150 f   LIBCMT:typname.obj
 0001:000632b0       ?_Type_info_dtor_internal@type_info@@CAXPEAV1@@Z 00000001400642b0 f   LIBCMT:typname.obj
 0001:00063350       __unDNameHelper            0000000140064350 f   LIBCMT:typname.obj
 0001:00063390       ?_Name_base_internal@type_info@@CAPEBDPEBV1@PEAU__type_info_node@@@Z 0000000140064390 f   LIBCMT:typname.obj
 0001:000634f0       __clean_type_info_names_internal 00000001400644f0 f   LIBCMT:typname.obj
 0001:00063570       abort                      0000000140064570 f   LIBCMT:abort.obj
 0001:00063620       _set_abort_behavior        0000000140064620 f   LIBCMT:abort.obj
 0001:00063640       _NMSG_WRITE                0000000140064640 f   LIBCMT:crt0msg.obj
 0001:00063880       _GET_RTERRMSG              0000000140064880 f   LIBCMT:crt0msg.obj
 0001:000638b0       _FF_MSGBANNER              00000001400648b0 f   LIBCMT:crt0msg.obj
 0001:00063a40       _encode_pointer            0000000140064a40 f   LIBCMT:tidtable.obj
 0001:00063b10       _encoded_null              0000000140064b10 f   LIBCMT:tidtable.obj
 0001:00063c00       _decode_pointer            0000000140064c00 f   LIBCMT:tidtable.obj
 0001:00063cd0       __crtTlsAlloc              0000000140064cd0 f   LIBCMT:tidtable.obj
 0001:00063ce0       __fls_getvalue             0000000140064ce0 f   LIBCMT:tidtable.obj
 0001:00063cf0       __get_flsindex             0000000140064cf0 f   LIBCMT:tidtable.obj
 0001:00063d00       __set_flsgetvalue          0000000140064d00 f   LIBCMT:tidtable.obj
 0001:00063d10       __fls_setvalue             0000000140064d10 f   LIBCMT:tidtable.obj
 0001:00063d20       _mtterm                    0000000140064d20 f   LIBCMT:tidtable.obj
 0001:00063d70       _initptd                   0000000140064d70 f   LIBCMT:tidtable.obj
 0001:00063f00       _getptd_noexit             0000000140064f00 f   LIBCMT:tidtable.obj
 0001:00063f90       _getptd                    0000000140064f90 f   LIBCMT:tidtable.obj
 0001:00064030       _freefls                   0000000140065030 f   LIBCMT:tidtable.obj
 0001:000641a0       _freeptd                   00000001400651a0 f   LIBCMT:tidtable.obj
 0001:00064200       __threadid                 0000000140065200 f   LIBCMT:tidtable.obj
 0001:00064210       __threadhandle             0000000140065210 f   LIBCMT:tidtable.obj
 0001:00064220       _mtinit                    0000000140065220 f   LIBCMT:tidtable.obj
 0001:00064340       __getlocaleinfo            0000000140065340 f   LIBCMT:inithelp.obj
 0001:00064520       _initp_misc_purevirt       0000000140065520 f   LIBCMT:inithelp.obj
 0001:00064530       _fullpath                  0000000140065530 f   LIBCMT:fullpath.obj
 0001:00064680       __dtoxmode                 0000000140065680 f   LIBCMT:stat.obj
 0001:000648c0       _stat32                    00000001400658c0 f   LIBCMT:stat.obj
 0001:00064d20       __loctotime64_t            0000000140065d20 f   LIBCMT:dtoxtm64.obj
 0001:00065030       _getdrive                  0000000140066030 f   LIBCMT:drive.obj
 0001:00065130       _chdrive                   0000000140066130 f   LIBCMT:drive.obj
 0001:000651f0       _mbctolower_l              00000001400661f0 f   LIBCMT:mbtolwr.obj
 0001:000653b0       _mbctolower                00000001400663b0 f   LIBCMT:mbtolwr.obj
 0001:000653c0       _mbspbrk_l                 00000001400663c0 f   LIBCMT:mbspbrk.obj
 0001:00065570       _mbspbrk                   0000000140066570 f   LIBCMT:mbspbrk.obj
 0001:00065900       _strtoi64                  0000000140066900 f   LIBCMT:strtoq.obj
 0001:00065940       _strtoi64_l                0000000140066940 f   LIBCMT:strtoq.obj
 0001:00065970       _strtoui64                 0000000140066970 f   LIBCMT:strtoq.obj
 0001:000659b0       _strtoui64_l               00000001400669b0 f   LIBCMT:strtoq.obj
 0001:000659e0       __report_gsfailure         00000001400669e0 f   LIBCMT:gs_report.obj
 0001:00065b30       ??0exception@std@@QEAA@XZ  0000000140066b30 f   LIBCMT:stdexcpt.obj
 0001:00065b50       ??0exception@std@@QEAA@AEBQEBD@Z 0000000140066b50 f   LIBCMT:stdexcpt.obj
 0001:00065be0       ??0exception@std@@QEAA@AEBQEBDH@Z 0000000140066be0 f   LIBCMT:stdexcpt.obj
 0001:00065c00       ??0exception@std@@QEAA@AEBV01@@Z 0000000140066c00 f   LIBCMT:stdexcpt.obj
 0001:00065cb0       ??4exception@std@@QEAAAEAV01@AEBV01@@Z 0000000140066cb0 f   LIBCMT:stdexcpt.obj
 0001:00065d50       ??1exception@std@@UEAA@XZ  0000000140066d50 f   LIBCMT:stdexcpt.obj
 0001:00065d80       ?what@exception@std@@UEBAPEBDXZ 0000000140066d80 f   LIBCMT:stdexcpt.obj
 0001:00065da0       ??0bad_cast@std@@QEAA@PEBD@Z 0000000140066da0 f   LIBCMT:stdexcpt.obj
 0001:00065e30       ??0bad_cast@std@@QEAA@AEBV01@@Z 0000000140066e30 f   LIBCMT:stdexcpt.obj
 0001:00065ec0       ??1bad_cast@std@@UEAA@XZ   0000000140066ec0 f   LIBCMT:stdexcpt.obj
 0001:00065ef0       ??0bad_typeid@std@@QEAA@PEBD@Z 0000000140066ef0 f   LIBCMT:stdexcpt.obj
 0001:00065f80       ??0bad_typeid@std@@QEAA@AEBV01@@Z 0000000140066f80 f   LIBCMT:stdexcpt.obj
 0001:00066010       ??1bad_typeid@std@@UEAA@XZ 0000000140067010 f   LIBCMT:stdexcpt.obj
 0001:00066040       ??0__non_rtti_object@std@@QEAA@PEBD@Z 0000000140067040 f   LIBCMT:stdexcpt.obj
 0001:000660d0       ??0__non_rtti_object@std@@QEAA@AEBV01@@Z 00000001400670d0 f   LIBCMT:stdexcpt.obj
 0001:00066160       ??1__non_rtti_object@std@@UEAA@XZ 0000000140067160 f   LIBCMT:stdexcpt.obj
 0001:00066190       ??_Gexception@std@@UEAAPEAXI@Z 0000000140067190 f i LIBCMT:stdexcpt.obj
 0001:00066190       ??_Eexception@std@@UEAAPEAXI@Z 0000000140067190 f i LIBCMT:stdexcpt.obj
 0001:000661e0       ??_Gbad_cast@std@@UEAAPEAXI@Z 00000001400671e0 f i LIBCMT:stdexcpt.obj
 0001:000661e0       ??_Ebad_cast@std@@UEAAPEAXI@Z 00000001400671e0 f i LIBCMT:stdexcpt.obj
 0001:00066230       ??_Ebad_typeid@std@@UEAAPEAXI@Z 0000000140067230 f i LIBCMT:stdexcpt.obj
 0001:00066230       ??_Gbad_typeid@std@@UEAAPEAXI@Z 0000000140067230 f i LIBCMT:stdexcpt.obj
 0001:00066280       ??_G__non_rtti_object@std@@UEAAPEAXI@Z 0000000140067280 f i LIBCMT:stdexcpt.obj
 0001:00066280       ??_E__non_rtti_object@std@@UEAAPEAXI@Z 0000000140067280 f i LIBCMT:stdexcpt.obj
 0001:000663d0       __onexitinit               00000001400673d0 f   LIBCMT:onexit.obj
 0001:00066420       _onexit                    0000000140067420 f   LIBCMT:onexit.obj
 0001:00066550       atexit                     0000000140067550 f   LIBCMT:onexit.obj
 0001:00066570       _initp_heap_handler        0000000140067570 f   LIBCMT:handler.obj
 0001:00066580       ?_set_new_handler@@YAP6AH_K@ZP6AH0@Z@Z 0000000140067580 f   LIBCMT:handler.obj
 0001:000665d0       ?_set_new_handler@@YAP6AH_K@ZH@Z 00000001400675d0 f   LIBCMT:handler.obj
 0001:00066610       ?_query_new_handler@@YAP6AH_K@ZXZ 0000000140067610 f   LIBCMT:handler.obj
 0001:00066620       _callnewh                  0000000140067620 f   LIBCMT:handler.obj
 0001:00066660       _CxxThrowException         0000000140067660 f   LIBCMT:throw.obj
 0001:00066730       _flsbuf                    0000000140067730 f   LIBCMT:_flsbuf.obj
 0001:00066ae0       get_int_arg                0000000140067ae0 f i LIBCMT:output.obj
 0001:00066af0       get_int64_arg              0000000140067af0 f i LIBCMT:output.obj
 0001:00066b00       get_short_arg              0000000140067b00 f i LIBCMT:output.obj
 0001:00066b10       _output_l                  0000000140067b10 f   LIBCMT:output.obj
 0001:00067ae0       __C_specific_handler       0000000140068ae0 f   LIBCMT:chandler.obj
 0001:00067ca0       _ioinit                    0000000140068ca0 f   LIBCMT:ioinit.obj
 0001:00067fe0       _ioterm                    0000000140068fe0 f   LIBCMT:ioinit.obj
 0001:00068070       _fileno                    0000000140069070 f   LIBCMT:fileno.obj
 0001:00068070       fileno                     0000000140069070 f   LIBCMT:fileno.obj
 0001:00068160       _INTRN_LOCALE_CONV         0000000140069160 f i LIBCMT:input.obj
 0001:00068240       _input_l                   0000000140069240 f   LIBCMT:input.obj
 0001:00069d10       _input_s_l                 000000014006ad10 f   LIBCMT:inputs.obj
 0001:0006b830       _stbuf                     000000014006c830 f   LIBCMT:_sftbuf.obj
 0001:0006b910       _ftbuf                     000000014006c910 f   LIBCMT:_sftbuf.obj
 0001:0006b950       vprintf_helper             000000014006c950 f   LIBCMT:vprintf.obj
 0001:0006ba30       _vprintf_l                 000000014006ca30 f   LIBCMT:vprintf.obj
 0001:0006ba50       _vprintf_s_l               000000014006ca50 f   LIBCMT:vprintf.obj
 0001:0006ba70       _vprintf_p_l               000000014006ca70 f   LIBCMT:vprintf.obj
 0001:0006ba90       vprintf                    000000014006ca90 f   LIBCMT:vprintf.obj
 0001:0006bab0       vprintf_s                  000000014006cab0 f   LIBCMT:vprintf.obj
 0001:0006bad0       _vprintf_p                 000000014006cad0 f   LIBCMT:vprintf.obj
 0001:0006baf0       __sys_nerr                 000000014006caf0 f   LIBCMT:syserr.obj
 0001:0006bb00       __sys_errlist              000000014006cb00 f   LIBCMT:syserr.obj
 0001:0006bb10       strcpy_s                   000000014006cb10 f   LIBCMT:strcpy_s.obj
 0001:0006bbc0       wait_a_bit                 000000014006cbc0 f i LIBCMT:crtheap.obj
 0001:0006bbf0       _set_malloc_crt_max_wait   000000014006cbf0 f   LIBCMT:crtheap.obj
 0001:0006bc00       _malloc_crt                000000014006cc00 f   LIBCMT:crtheap.obj
 0001:0006bc70       _calloc_crt                000000014006cc70 f   LIBCMT:crtheap.obj
 0001:0006bd00       _realloc_crt               000000014006cd00 f   LIBCMT:crtheap.obj
 0001:0006bd90       _recalloc_crt              000000014006cd90 f   LIBCMT:crtheap.obj
 0001:0006be30       strncpy_s                  000000014006ce30 f   LIBCMT:strncpy_s.obj
 0001:0006bf50       _vsprintf_l                000000014006cf50 f   LIBCMT:vsprintf.obj
 0001:0006bff0       vsprintf                   000000014006cff0 f   LIBCMT:vsprintf.obj
 0001:0006c090       _vscprintf_helper          000000014006d090 f   LIBCMT:vsprintf.obj
 0001:0006c0f0       _vscprintf                 000000014006d0f0 f   LIBCMT:vsprintf.obj
 0001:0006c160       _vscprintf_l               000000014006d160 f   LIBCMT:vsprintf.obj
 0001:0006c1d0       _vscprintf_p               000000014006d1d0 f   LIBCMT:vsprintf.obj
 0001:0006c240       _vscprintf_p_l             000000014006d240 f   LIBCMT:vsprintf.obj
 0001:0006c2b0       _vsnprintf_helper          000000014006d2b0 f   LIBCMT:vsnprnc.obj
 0001:0006c3c0       _vsnprintf_c               000000014006d3c0 f   LIBCMT:vsnprnc.obj
 0001:0006c4b0       _vsnprintf_c_l             000000014006d4b0 f   LIBCMT:vsnprnc.obj
 0001:0006c5b0       _vsprintf_s_l              000000014006d5b0 f   LIBCMT:vsnprnc.obj
 0001:0006c640       vsprintf_s                 000000014006d640 f   LIBCMT:vsnprnc.obj
 0001:0006c6c0       _vsnprintf_s_l             000000014006d6c0 f   LIBCMT:vsnprnc.obj
 0001:0006c830       _vsnprintf_s               000000014006d830 f   LIBCMT:vsnprnc.obj
 0001:0006c860       _vsprintf_p                000000014006d860 f   LIBCMT:vsnprnc.obj
 0001:0006c950       _vsprintf_p_l              000000014006d950 f   LIBCMT:vsnprnc.obj
 0001:0006ca50       _fcloseall                 000000014006da50 f   LIBCMT:closeall.obj
 0001:0006cb40       _mtinitlocks               000000014006db40 f   LIBCMT:mlock.obj
 0001:0006cbe0       _mtdeletelocks             000000014006dbe0 f   LIBCMT:mlock.obj
 0001:0006cc80       _unlock                    000000014006dc80 f   LIBCMT:mlock.obj
 0001:0006cca0       _lockerr_exit              000000014006dca0 f   LIBCMT:mlock.obj
 0001:0006ccc0       _mtinitlocknum             000000014006dcc0 f   LIBCMT:mlock.obj
 0001:0006cdd0       _lock                      000000014006ddd0 f   LIBCMT:mlock.obj
 0001:0006d000       _output_s_l                000000014006e000 f   LIBCMT:outputs.obj
 0001:0006e010       _validate_param_reuseA     000000014006f010 f   LIBCMT:outputp.obj
 0001:0006e360       get_crtdouble_arg          000000014006f360 f i LIBCMT:outputp.obj
 0001:0006e370       _output_p_l                000000014006f370 f   LIBCMT:outputp.obj
 0001:000701c0       _RTC_Initialize            00000001400711c0 f   LIBCMT:initsect.obj
 0001:00070200       _RTC_Terminate             0000000140071200 f   LIBCMT:initsect.obj
 0001:00070240       _ValidateImageBase         0000000140071240 f   LIBCMT:pesect.obj
 0001:00070270       _FindPESection             0000000140071270 f   LIBCMT:pesect.obj
 0001:000702c0       _IsNonwritableInCurrentImage 00000001400712c0 f   LIBCMT:pesect.obj
 0001:00070330       ?terminate@@YAXXZ          0000000140071330 f   LIBCMT:hooks.obj
 0001:00070360       ?unexpected@@YAXXZ         0000000140071360 f   LIBCMT:hooks.obj
 0001:00070380       ?_inconsistency@@YAXXZ     0000000140071380 f   LIBCMT:hooks.obj
 0001:000703b0       _initp_eh_hooks            00000001400713b0 f   LIBCMT:hooks.obj
 0001:000703d0       _initp_misc_winxfltr       00000001400713d0 f   LIBCMT:winxfltr.obj
 0001:00070420       _XcptFilter                0000000140071420 f   LIBCMT:winxfltr.obj
 0001:00070630       __CppXcptFilter            0000000140071630 f   LIBCMT:winxfltr.obj
 0001:00070640       _initp_misc_rand_s         0000000140071640 f   LIBCMT:rand_s.obj
 0001:00070650       rand_s                     0000000140071650 f   LIBCMT:rand_s.obj
 0001:000707b0       _initp_misc_initcrit       00000001400717b0 f   LIBCMT:initcrit.obj
 0001:000707e0       __crtInitCritSecAndSpinCount 00000001400717e0 f   LIBCMT:initcrit.obj
 0001:00070900       _filbuf                    0000000140071900 f   LIBCMT:_filbuf.obj
 0001:00070a80       _mbsrchr_l                 0000000140071a80 f   LIBCMT:mbsrchr.obj
 0001:00070c10       _mbsrchr                   0000000140071c10 f   LIBCMT:mbsrchr.obj
 0001:00070c20       _getpath                   0000000140071c20 f   LIBCMT:getpath.obj
 0001:00070cf0       _access_s                  0000000140071cf0 f   LIBCMT:access.obj
 0001:00070da0       _access                    0000000140071da0 f   LIBCMT:access.obj
 0001:00070e60       strcat_s                   0000000140071e60 f   LIBCMT:strcat_s.obj
 0001:00070f20       fdopen                     0000000140071f20 f   LIBCMT:fdopen.obj
 0001:00070f20       _fdopen                    0000000140071f20 f   LIBCMT:fdopen.obj
 0001:00071240       _close_nolock              0000000140072240 f   LIBCMT:close.obj
 0001:00071310       close                      0000000140072310 f   LIBCMT:close.obj
 0001:00071310       _close                     0000000140072310 f   LIBCMT:close.obj
 0001:00071440       _pipe                      0000000140072440 f   LIBCMT:pipe.obj
 0001:00071790       _cwait                     0000000140072790 f   LIBCMT:wait.obj
 0001:00071860       _freebuf                   0000000140072860 f   LIBCMT:_freebuf.obj
 0001:000719d0       _handle_errorf             00000001400729d0 f   LIBCMT:libm_error.obj
 0001:00071be0       _handle_error              0000000140072be0 f   LIBCMT:libm_error.obj
 0001:00071df0       _mbsnbicoll_l              0000000140072df0 f   LIBCMT:mbsnbico.obj
 0001:00071fb0       _mbsnbicoll                0000000140072fb0 f   LIBCMT:mbsnbico.obj
 0001:00071fc0       __wtomb_environ            0000000140072fc0 f   LIBCMT:wtombenv.obj
 0001:000720d0       _calloc_impl               00000001400730d0 f   LIBCMT:calloc.obj
 0001:000721a0       calloc                     00000001400731a0 f   LIBCMT:calloc.obj
 0001:00072290       strnlen                    0000000140073290 f   LIBCMT:strlen_s.obj
 0001:000725c0       __updatetmbcinfo           00000001400735c0 f   LIBCMT:mbctype.obj
 0001:000727b0       _setmbcp_nolock            00000001400737b0 f   LIBCMT:mbctype.obj
 0001:00072b70       _getmbcp                   0000000140073b70 f   LIBCMT:mbctype.obj
 0001:00072c30       _setmbcp                   0000000140073c30 f   LIBCMT:mbctype.obj
 0001:00072e60       __initmbctable             0000000140073e60 f   LIBCMT:mbctype.obj
 0001:00072e90       ___setlc_active_func       0000000140073e90 f   LIBCMT:setlocal.obj
 0001:00072ea0       ___unguarded_readlc_active_add_func 0000000140073ea0 f   LIBCMT:setlocal.obj
 0001:00072eb0       __freetlocinfo             0000000140073eb0 f   LIBCMT:setlocal.obj
 0001:00073040       __addlocaleref             0000000140074040 f   LIBCMT:setlocal.obj
 0001:000730e0       __removelocaleref          00000001400740e0 f   LIBCMT:setlocal.obj
 0001:00073230       __updatetlocinfo           0000000140074230 f   LIBCMT:setlocal.obj
 0001:000732d0       _configthreadlocale        00000001400742d0 f   LIBCMT:setlocal.obj
 0001:000733d0       _free_locale               00000001400743d0 f   LIBCMT:setlocal.obj
 0001:00073490       __free_locale              0000000140074490 f   LIBCMT:setlocal.obj
 0001:000734a0       _get_current_locale        00000001400744a0 f   LIBCMT:setlocal.obj
 0001:00073550       __get_current_locale       0000000140074550 f   LIBCMT:setlocal.obj
 0001:00073560       __init_dummy               0000000140074560 f   LIBCMT:setlocal.obj
 0001:00073570       _strcats                   0000000140074570 f   LIBCMT:setlocal.obj
 0001:000735f0       __lc_strtolc               00000001400745f0 f   LIBCMT:setlocal.obj
 0001:000737d0       __lc_lctostr               00000001400747d0 f   LIBCMT:setlocal.obj
 0001:00073a90       _expandlocale              0000000140074a90 f   LIBCMT:setlocal.obj
 0001:00074300       _create_locale             0000000140075300 f   LIBCMT:setlocal.obj
 0001:00074490       __create_locale            0000000140075490 f   LIBCMT:setlocal.obj
 0001:000744a0       setlocale                  00000001400754a0 f   LIBCMT:setlocal.obj
 0001:00074740       _isctype_l                 0000000140075740 f   LIBCMT:isctype.obj
 0001:00074930       _isctype                   0000000140075930 f   LIBCMT:isctype.obj
 0001:00074960       __initconin                0000000140075960 f   LIBCMT:initcon.obj
 0001:000749a0       __initconout               00000001400759a0 f   LIBCMT:initcon.obj
 0001:000749e0       __termcon                  00000001400759e0 f   LIBCMT:initcon.obj
 0001:00074a20       _putch_nolock              0000000140075a20 f   LIBCMT:putch.obj
 0001:00074ae0       _putch                     0000000140075ae0 f   LIBCMT:putch.obj
 0001:00074b30       ?__CxxUnhandledExceptionFilter@@YAJPEAU_EXCEPTION_POINTERS@@@Z 0000000140075b30 f   LIBCMT:unhandld.obj
 0001:00074b80       __CxxSetUnhandledExceptionFilter 0000000140075b80 f   LIBCMT:unhandld.obj
 0001:00074ba0       _setenvp                   0000000140075ba0 f   LIBCMT:stdenvp.obj
 0001:00074d10       _set_pgmptr                0000000140075d10 f i LIBCMT:stdargv.obj
 0001:00074f40       _setargv                   0000000140075f40 f   LIBCMT:stdargv.obj
 0001:00075050       __crtGetEnvironmentStringsA 0000000140076050 f   LIBCMT:a_env.obj
 0001:00075220       _heap_init                 0000000140076220 f   LIBCMT:heapinit.obj
 0001:00075280       _heap_term                 0000000140076280 f   LIBCMT:heapinit.obj
 0001:000752b0       _get_heap_handle           00000001400762b0 f   LIBCMT:heapinit.obj
 0001:000752c0       __security_init_cookie     00000001400762c0 f   LIBCMT:gs_support.obj
 0001:00075380       _msize                     0000000140076380 f   LIBCMT:msize.obj
 0001:000753d0       __loctotime32_t            00000001400763d0 f   LIBCMT:dtoxtime.obj
 0001:000756c0       _get_daylight              00000001400766c0 f   LIBCMT:timeset.obj
 0001:00075710       _get_dstbias               0000000140076710 f   LIBCMT:timeset.obj
 0001:00075760       _get_timezone              0000000140076760 f   LIBCMT:timeset.obj
 0001:000757b0       _get_tzname                00000001400767b0 f   LIBCMT:timeset.obj
 0001:00075860       __daylight                 0000000140076860 f   LIBCMT:timeset.obj
 0001:00075870       __dstbias                  0000000140076870 f   LIBCMT:timeset.obj
 0001:00075880       __timezone                 0000000140076880 f   LIBCMT:timeset.obj
 0001:00075890       __tzname                   0000000140076890 f   LIBCMT:timeset.obj
 0001:000758a0       _gmtime32_s                00000001400768a0 f   LIBCMT:gmtime.obj
 0001:00075ab0       __getgmtimebuf             0000000140076ab0 f   LIBCMT:gmtime.obj
 0001:00075b10       _gmtime32                  0000000140076b10 f   LIBCMT:gmtime.obj
 0001:00075bb0       _openfile                  0000000140076bb0 f   LIBCMT:_open.obj
 0001:00075f10       _getstream                 0000000140076f10 f   LIBCMT:stream.obj
 0001:000760c0       _local_unwind              00000001400770c0 f   LIBCMT:jmpuwind.obj
 0001:000760f0       _NLG_Notify                00000001400770f0 f   LIBCMT:jmpuwind.obj
 0001:00076110       __NLG_Dispatch2            0000000140077110 f   LIBCMT:jmpuwind.obj
 0001:00076120       __NLG_Return2              0000000140077120 f   LIBCMT:jmpuwind.obj
 0001:00076130       __init_ctype               0000000140077130 f   LIBCMT:initctyp.obj
 0001:000765c0       ___mb_cur_max_func         00000001400775c0 f   LIBCMT:initctyp.obj
 0001:00076610       ___mb_cur_max_l_func       0000000140077610 f   LIBCMT:initctyp.obj
 0001:00076660       ___lc_codepage_func        0000000140077660 f   LIBCMT:initctyp.obj
 0001:000766a0       ___lc_collate_cp_func      00000001400776a0 f   LIBCMT:initctyp.obj
 0001:000766e0       ___lc_handle_func          00000001400776e0 f   LIBCMT:initctyp.obj
 0001:00076720       __crt_debugger_hook        0000000140077720 f   LIBCMT:dbghook.obj
 0001:00076730       _write_nolock              0000000140077730 f   LIBCMT:write.obj
 0001:00076f40       write                      0000000140077f40 f   LIBCMT:write.obj
 0001:00076f40       _write                     0000000140077f40 f   LIBCMT:write.obj
 0001:00077090       _commit                    0000000140078090 f   LIBCMT:commit.obj
 0001:000771d0       _read_nolock               00000001400781d0 f   LIBCMT:read.obj
 0001:00077ae0       read                       0000000140078ae0 f   LIBCMT:read.obj
 0001:00077ae0       _read                      0000000140078ae0 f   LIBCMT:read.obj
 0001:00077c80       memcpy_s                   0000000140078c80 f   LIBCMT:memcpy_s.obj
 0001:00077d50       _lseek_nolock              0000000140078d50 f   LIBCMT:lseek.obj
 0001:00077e00       _lseek                     0000000140078e00 f   LIBCMT:lseek.obj
 0001:00077f50       _tolower                   0000000140078f50 f   LIBCMT:tolower.obj
 0001:00077f60       _tolower_l                 0000000140078f60 f   LIBCMT:tolower.obj
 0001:000781d0       tolower                    00000001400791d0 f   LIBCMT:tolower.obj
 0001:000781f0       _atodbl_l                  00000001400791f0 f   LIBCMT:atodbl.obj
 0001:00078380       _atodbl                    0000000140079380 f   LIBCMT:atodbl.obj
 0001:00078390       _atoldbl_l                 0000000140079390 f   LIBCMT:atodbl.obj
 0001:00078530       _atoldbl                   0000000140079530 f   LIBCMT:atodbl.obj
 0001:00078540       _atoflt_l                  0000000140079540 f   LIBCMT:atodbl.obj
 0001:000786d0       _atoflt                    00000001400796d0 f   LIBCMT:atodbl.obj
 0001:000786e0       _set_output_format         00000001400796e0 f   LIBCMT:outputformat.obj
 0001:00078730       _get_output_format         0000000140079730 f   LIBCMT:outputformat.obj
 0001:00078740       _fptostr                   0000000140079740 f   LIBCMT:_fptostr.obj
 0001:00078860       __dtold                    0000000140079860 f   LIBCMT:cfout.obj
 0001:00078920       _fltout2                   0000000140079920 f   LIBCMT:cfout.obj
 0001:00078a90       _fptrap                    0000000140079a90 f   LIBCMT:crt0fp.obj
 0001:00078aa0       ??0Block@HeapManager@@QEAA@XZ 0000000140079aa0 f i LIBCMT:undname.obj
 0001:00078ab0       ?Constructor@HeapManager@@QEAAXP6APEAX_K@ZP6AXPEAX@Z@Z 0000000140079ab0 f i LIBCMT:undname.obj
 0001:00078ad0       ?Destructor@HeapManager@@QEAAXXZ 0000000140079ad0 f i LIBCMT:undname.obj
 0001:00078b20       ?getNumberOfDimensions@UnDecorator@@CAHXZ 0000000140079b20 f   LIBCMT:undname.obj
 0001:00078b90       ?getTypeEncoding@UnDecorator@@CAHXZ 0000000140079b90 f i LIBCMT:undname.obj
 0001:000791b0       ?doUnderScore@UnDecorator@@SAHXZ 000000014007a1b0 f i LIBCMT:undname.obj
 0001:000791c0       ?doMSKeywords@UnDecorator@@SAHXZ 000000014007a1c0 f i LIBCMT:undname.obj
 0001:000791d0       ?doPtr64@UnDecorator@@SAHXZ 000000014007a1d0 f i LIBCMT:undname.obj
 0001:000791e0       ?doFunctionReturns@UnDecorator@@SAHXZ 000000014007a1e0 f i LIBCMT:undname.obj
 0001:000791f0       ?doAllocationModel@UnDecorator@@SAHXZ 000000014007a1f0 f i LIBCMT:undname.obj
 0001:00079200       ?doAllocationLanguage@UnDecorator@@SAHXZ 000000014007a200 f i LIBCMT:undname.obj
 0001:00079210       ?doThisTypes@UnDecorator@@SAHXZ 000000014007a210 f i LIBCMT:undname.obj
 0001:00079230       ?doAccessSpecifiers@UnDecorator@@SAHXZ 000000014007a230 f i LIBCMT:undname.obj
 0001:00079240       ?doThrowTypes@UnDecorator@@SAHXZ 000000014007a240 f i LIBCMT:undname.obj
 0001:00079250       ?doMemberTypes@UnDecorator@@SAHXZ 000000014007a250 f i LIBCMT:undname.obj
 0001:00079260       ?doNameOnly@UnDecorator@@SAHXZ 000000014007a260 f i LIBCMT:undname.obj
 0001:00079270       ?doTypeOnly@UnDecorator@@SAHXZ 000000014007a270 f i LIBCMT:undname.obj
 0001:00079280       ?haveTemplateParameters@UnDecorator@@SAHXZ 000000014007a280 f i LIBCMT:undname.obj
 0001:00079290       ?doEcsu@UnDecorator@@SAHXZ 000000014007a290 f i LIBCMT:undname.obj
 0001:000792a0       ?doNoIdentCharCheck@UnDecorator@@SAHXZ 000000014007a2a0 f i LIBCMT:undname.obj
 0001:000792b0       ?doEllipsis@UnDecorator@@SAHXZ 000000014007a2b0 f i LIBCMT:undname.obj
 0001:000792c0       ?UScore@UnDecorator@@SAPEBDW4Tokens@@@Z 000000014007a2c0 f   LIBCMT:undname.obj
 0001:000792f0       ?getMemory@HeapManager@@QEAAPEAX_KH@Z 000000014007a2f0 f   LIBCMT:undname.obj
 0001:000793d0       ??0DName@@QEAA@XZ          000000014007a3d0 f i LIBCMT:undname.obj
 0001:000793f0       ??0DName@@QEAA@PEAVDNameNode@@@Z 000000014007a3f0 f i LIBCMT:undname.obj
 0001:00079400       ??0DName@@QEAA@AEBV0@@Z    000000014007a400 f i LIBCMT:undname.obj
 0001:000794b0       ?status@DName@@QEBA?AW4DNameStatus@@XZ 000000014007a4b0 f i LIBCMT:undname.obj
 0001:000794c0       ?clearStatus@DName@@QEAAXXZ 000000014007a4c0 f i LIBCMT:undname.obj
 0001:000794d0       ?setPtrRef@DName@@QEAAAEAV1@XZ 000000014007a4d0 f i LIBCMT:undname.obj
 0001:000794e0       ?isPtrRef@DName@@QEBAHXZ   000000014007a4e0 f i LIBCMT:undname.obj
 0001:000794f0       ?setIsArray@DName@@QEAAXXZ 000000014007a4f0 f i LIBCMT:undname.obj
 0001:00079500       ?isArray@DName@@QEBAHXZ    000000014007a500 f i LIBCMT:undname.obj
 0001:00079510       ?isNoTE@DName@@QEBAHXZ     000000014007a510 f i LIBCMT:undname.obj
 0001:00079520       ?setIsNoTE@DName@@QEAAXXZ  000000014007a520 f i LIBCMT:undname.obj
 0001:00079530       ?isPinPtr@DName@@QEBAHXZ   000000014007a530 f i LIBCMT:undname.obj
 0001:00079540       ?setIsPinPtr@DName@@QEAAXXZ 000000014007a540 f i LIBCMT:undname.obj
 0001:00079550       ?isComArray@DName@@QEBAHXZ 000000014007a550 f i LIBCMT:undname.obj
 0001:00079560       ?setIsComArray@DName@@QEAAXXZ 000000014007a560 f i LIBCMT:undname.obj
 0001:00079570       ?isVCallThunk@DName@@QEBAHXZ 000000014007a570 f i LIBCMT:undname.obj
 0001:00079580       ?setIsVCallThunk@DName@@QEAAXXZ 000000014007a580 f i LIBCMT:undname.obj
 0001:00079590       ??4DName@@QEAAAEAV0@AEBV0@@Z 000000014007a590 f   LIBCMT:undname.obj
 0001:00079620       ?isFull@Replicator@@QEBAHXZ 000000014007a620 f i LIBCMT:undname.obj
 0001:00079630       ??AReplicator@@QEBAAEBVDName@@H@Z 000000014007a630 f   LIBCMT:undname.obj
 0001:00079660       ??0DNameNode@@IEAA@XZ      000000014007a660 f   LIBCMT:undname.obj
 0001:00079680       ?nextNode@DNameNode@@QEBAPEAV1@XZ 000000014007a680 f i LIBCMT:undname.obj
 0001:00079690       ??YDNameNode@@QEAAAEAV0@PEAV0@@Z 000000014007a690 f   LIBCMT:undname.obj
 0001:000796d0       ??0charNode@@QEAA@D@Z      000000014007a6d0 f   LIBCMT:undname.obj
 0001:000796f0       ?length@charNode@@UEBAHXZ  000000014007a6f0 f i LIBCMT:undname.obj
 0001:00079700       ?getLastChar@charNode@@UEBADXZ 000000014007a700 f i LIBCMT:undname.obj
 0001:00079710       ?getString@charNode@@UEBAPEADPEADH@Z 000000014007a710 f   LIBCMT:undname.obj
 0001:00079730       ?length@pcharNode@@UEBAHXZ 000000014007a730 f i LIBCMT:undname.obj
 0001:00079740       ??0pDNameNode@@QEAA@PEAVDName@@@Z 000000014007a740 f   LIBCMT:undname.obj
 0001:00079780       ??0DNameStatusNode@@QEAA@W4DNameStatus@@@Z 000000014007a780 f   LIBCMT:undname.obj
 0001:000797b0       ?length@DNameStatusNode@@UEBAHXZ 000000014007a7b0 f i LIBCMT:undname.obj
 0001:000797c0       ?getLastChar@DNameStatusNode@@UEBADXZ 000000014007a7c0 f i LIBCMT:undname.obj
 0001:00079860       ?getDataIndirectType@UnDecorator@@CA?AVDName@@XZ 000000014007a860 f i LIBCMT:undname.obj
 0001:000798b0       ?getThisType@UnDecorator@@CA?AVDName@@XZ 000000014007a8b0 f i LIBCMT:undname.obj
 0001:00079900       ??2@YAPEAX_KAEAVHeapManager@@H@Z 000000014007a900 f i LIBCMT:undname.obj
 0001:000799c0       ??0DName@@QEAA@PEAV0@@Z    000000014007a9c0 f   LIBCMT:undname.obj
 0001:00079ad0       ??0DName@@QEAA@W4DNameStatus@@@Z 000000014007aad0 f   LIBCMT:undname.obj
 0001:00079bc0       ?isValid@DName@@QEBAHXZ    000000014007abc0 f   LIBCMT:undname.obj
 0001:00079be0       ?isEmpty@DName@@QEBAHXZ    000000014007abe0 f   LIBCMT:undname.obj
 0001:00079c00       ?isUDC@DName@@QEBAHXZ      000000014007ac00 f i LIBCMT:undname.obj
 0001:00079c30       ?setIsUDC@DName@@QEAAXXZ   000000014007ac30 f i LIBCMT:undname.obj
 0001:00079c60       ?isUDTThunk@DName@@QEBAHXZ 000000014007ac60 f i LIBCMT:undname.obj
 0001:00079c90       ?length@DName@@QEBAHXZ     000000014007ac90 f   LIBCMT:undname.obj
 0001:00079ce0       ?getLastChar@DName@@QEBADXZ 000000014007ace0 f   LIBCMT:undname.obj
 0001:00079d50       ?getString@DName@@QEBAPEADPEADH@Z 000000014007ad50 f   LIBCMT:undname.obj
 0001:00079ef0       ??_5DName@@QEAAAEAV0@AEBV0@@Z 000000014007aef0 f   LIBCMT:undname.obj
 0001:00079f20       ??4DName@@QEAAAEAV0@W4DNameStatus@@@Z 000000014007af20 f   LIBCMT:undname.obj
 0001:0007a050       ??0Replicator@@QEAA@XZ     000000014007b050 f i LIBCMT:undname.obj
 0001:0007a1f0       ??YReplicator@@QEAAAEAV0@AEBVDName@@@Z 000000014007b1f0 f   LIBCMT:undname.obj
 0001:0007a360       ?clone@DNameNode@@QEAAPEAV1@XZ 000000014007b360 f   LIBCMT:undname.obj
 0001:0007a4b0       ??0pcharNode@@QEAA@PEBDH@Z 000000014007b4b0 f   LIBCMT:undname.obj
 0001:0007a610       ?getLastChar@pcharNode@@UEBADXZ 000000014007b610 f i LIBCMT:undname.obj
 0001:0007a630       ?getString@pcharNode@@UEBAPEADPEADH@Z 000000014007b630 f   LIBCMT:undname.obj
 0001:0007a670       ?length@pDNameNode@@UEBAHXZ 000000014007b670 f i LIBCMT:undname.obj
 0001:0007a6f0       ?getLastChar@pDNameNode@@UEBADXZ 000000014007b6f0 f i LIBCMT:undname.obj
 0001:0007a780       ?getString@pDNameNode@@UEBAPEADPEADH@Z 000000014007b780 f   LIBCMT:undname.obj
 0001:0007a7a0       ?getString@DNameStatusNode@@UEBAPEADPEADH@Z 000000014007b7a0 f   LIBCMT:undname.obj
 0001:0007a7f0       ??0UnDecorator@@QEAA@PEADPEBDHP6APEADJ@ZK@Z 000000014007b7f0 f i LIBCMT:undname.obj
 0001:0007a8a0       ?getReturnType@UnDecorator@@CA?AVDName@@PEAV2@@Z 000000014007b8a0 f   LIBCMT:undname.obj
 0001:0007a8e0       ?getStorageConvention@UnDecorator@@CA?AVDName@@XZ 000000014007b8e0 f i LIBCMT:undname.obj
 0001:0007a930       ??YDName@@QEAAAEAV0@W4DNameStatus@@@Z 000000014007b930 f   LIBCMT:undname.obj
 0001:0007aaa0       ??4DName@@QEAAAEAV0@PEAV0@@Z 000000014007baa0 f   LIBCMT:undname.obj
 0001:0007abc0       ?doPchar@DName@@AEAAXPEBDH@Z 000000014007bbc0 f   LIBCMT:undname.obj
 0001:0007ada0       ??0DName@@QEAA@D@Z         000000014007bda0 f   LIBCMT:undname.obj
 0001:0007aeb0       ??0DName@@QEAA@PEBD@Z      000000014007beb0 f   LIBCMT:undname.obj
 0001:0007aef0       ??0DName@@QEAA@AEAPEBDD@Z  000000014007bef0 f   LIBCMT:undname.obj
 0001:0007b050       ??0DName@@QEAA@_K@Z        000000014007c050 f   LIBCMT:undname.obj
 0001:0007b0f0       ??0DName@@QEAA@_J@Z        000000014007c0f0 f   LIBCMT:undname.obj
 0001:0007b1b0       ??HDName@@QEBA?AV0@W4DNameStatus@@@Z 000000014007c1b0 f   LIBCMT:undname.obj
 0001:0007b290       ??YDName@@QEAAAEAV0@AEBV0@@Z 000000014007c290 f   LIBCMT:undname.obj
 0001:0007b3f0       ??YDName@@QEAAAEAV0@PEAV0@@Z 000000014007c3f0 f   LIBCMT:undname.obj
 0001:0007b5a0       ??4DName@@QEAAAEAV0@D@Z    000000014007c5a0 f   LIBCMT:undname.obj
 0001:0007b6b0       ??4DName@@QEAAAEAV0@PEBD@Z 000000014007c6b0 f   LIBCMT:undname.obj
 0001:0007b6f0       ?getCallingConvention@UnDecorator@@CA?AVDName@@XZ 000000014007c6f0 f   LIBCMT:undname.obj
 0001:0007bae0       ?getVCallThunkType@UnDecorator@@CA?AVDName@@XZ 000000014007cae0 f i LIBCMT:undname.obj
 0001:0007bcc0       ??HDName@@QEBA?AV0@AEBV0@@Z 000000014007ccc0 f   LIBCMT:undname.obj
 0001:0007be40       ??HDName@@QEBA?AV0@PEAV0@@Z 000000014007ce40 f   LIBCMT:undname.obj
 0001:0007bf20       ??YDName@@QEAAAEAV0@D@Z    000000014007cf20 f   LIBCMT:undname.obj
 0001:0007c080       ??YDName@@QEAAAEAV0@PEBD@Z 000000014007d080 f   LIBCMT:undname.obj
 0001:0007c230       ?getArgumentList@UnDecorator@@CA?AVDName@@XZ 000000014007d230 f   LIBCMT:undname.obj
 0001:0007c590       ?getVdispMapType@UnDecorator@@CA?AVDName@@AEBV2@@Z 000000014007d590 f i LIBCMT:undname.obj
 0001:0007c690       ??H@YA?AVDName@@DAEBV0@@Z  000000014007d690 f i LIBCMT:undname.obj
 0001:0007c750       ??H@YA?AVDName@@W4DNameStatus@@AEBV0@@Z 000000014007d750 f i LIBCMT:undname.obj
 0001:0007c880       ??H@YA?AVDName@@PEBDAEBV0@@Z 000000014007d880 f i LIBCMT:undname.obj
 0001:0007c900       ??HDName@@QEBA?AV0@D@Z     000000014007d900 f   LIBCMT:undname.obj
 0001:0007c9e0       ??HDName@@QEBA?AV0@PEBD@Z  000000014007d9e0 f   LIBCMT:undname.obj
 0001:0007caf0       ?getDimension@UnDecorator@@CA?AVDName@@_N@Z 000000014007daf0 f   LIBCMT:undname.obj
 0001:0007d0a0       ?getEnumType@UnDecorator@@CA?AVDName@@XZ 000000014007e0a0 f i LIBCMT:undname.obj
 0001:0007d570       ?getArgumentTypes@UnDecorator@@CA?AVDName@@XZ 000000014007e570 f   LIBCMT:undname.obj
 0001:0007d730       ?getThrowTypes@UnDecorator@@CA?AVDName@@XZ 000000014007e730 f   LIBCMT:undname.obj
 0001:0007dad0       ?getExtendedDataIndirectType@UnDecorator@@CA?AVDName@@AEADAEA_NH@Z 000000014007ead0 f   LIBCMT:undname.obj
 0001:0007df10       ?getArrayType@UnDecorator@@CA?AVDName@@AEBV2@@Z 000000014007ef10 f i LIBCMT:undname.obj
 0001:0007f110       ?getLexicalFrame@UnDecorator@@CA?AVDName@@XZ 0000000140080110 f i LIBCMT:undname.obj
 0001:0007f240       ?getDisplacement@UnDecorator@@CA?AVDName@@XZ 0000000140080240 f i LIBCMT:undname.obj
 0001:0007f260       ?getCallIndex@UnDecorator@@CA?AVDName@@XZ 0000000140080260 f i LIBCMT:undname.obj
 0001:0007f280       ?getGuardNumber@UnDecorator@@CA?AVDName@@XZ 0000000140080280 f i LIBCMT:undname.obj
 0001:0007f2a0       ?getVfTableType@UnDecorator@@CA?AVDName@@AEBV2@@Z 00000001400802a0 f i LIBCMT:undname.obj
 0001:0007f890       ?getStringEncoding@UnDecorator@@CA?AVDName@@PEADH@Z 0000000140080890 f   LIBCMT:undname.obj
 0001:0007fb50       ?getSignedDimension@UnDecorator@@CA?AVDName@@XZ 0000000140080b50 f   LIBCMT:undname.obj
 0001:0007fd20       ?getTemplateConstant@UnDecorator@@CA?AVDName@@XZ 0000000140080d20 f   LIBCMT:undname.obj
 0001:00080580       ?getPtrRefDataType@UnDecorator@@CA?AVDName@@AEBV2@H@Z 0000000140081580 f i LIBCMT:undname.obj
 0001:00080a60       ?getVbTableType@UnDecorator@@CA?AVDName@@AEBV2@@Z 0000000140081a60 f i LIBCMT:undname.obj
 0001:00080a80       ?getTemplateArgumentList@UnDecorator@@CA?AVDName@@XZ 0000000140081a80 f   LIBCMT:undname.obj
 0001:000814b0       ?getOperatorName@UnDecorator@@CA?AVDName@@_NPEA_N@Z 00000001400824b0 f i LIBCMT:undname.obj
 0001:000823c0       ?getTemplateName@UnDecorator@@CA?AVDName@@_N@Z 00000001400833c0 f   LIBCMT:undname.obj
 0001:000827d0       ?getZName@UnDecorator@@CA?AVDName@@_N@Z 00000001400837d0 f   LIBCMT:undname.obj
 0001:00082f20       ?getScopedName@UnDecorator@@CA?AVDName@@XZ 0000000140083f20 f   LIBCMT:undname.obj
 0001:000833f0       ?getECSUName@UnDecorator@@CA?AVDName@@XZ 00000001400843f0 f i LIBCMT:undname.obj
 0001:00083410       ?getECSUDataType@UnDecorator@@CA?AVDName@@XZ 0000000140084410 f   LIBCMT:undname.obj
 0001:000838c0       ?getSymbolName@UnDecorator@@CA?AVDName@@XZ 00000001400848c0 f i LIBCMT:undname.obj
 0001:00083920       ?getBasedType@UnDecorator@@CA?AVDName@@XZ 0000000140084920 f   LIBCMT:undname.obj
 0001:00083bf0       ?composeDeclaration@UnDecorator@@CA?AVDName@@AEBV2@@Z 0000000140084bf0 f i LIBCMT:undname.obj
 0001:00085a90       ?getDecoratedName@UnDecorator@@CA?AVDName@@XZ 0000000140086a90 f   LIBCMT:undname.obj
 0001:00086040       ?getScope@UnDecorator@@CA?AVDName@@XZ 0000000140087040 f   LIBCMT:undname.obj
 0001:00086fe0       ?getFunctionIndirectType@UnDecorator@@CA?AVDName@@AEBV2@@Z 0000000140087fe0 f   LIBCMT:undname.obj
 0001:00087f30       ?getDataIndirectType@UnDecorator@@CA?AVDName@@AEBV2@D0H@Z 0000000140088f30 f   LIBCMT:undname.obj
 0001:00089590       ??BUnDecorator@@QEAAPEADXZ 000000014008a590 f i LIBCMT:undname.obj
 0001:00089910       ?getPtrRefType@UnDecorator@@CA?AVDName@@AEBV2@0D@Z 000000014008a910 f   LIBCMT:undname.obj
 0001:00089bb0       ?getPointerType@UnDecorator@@CA?AVDName@@AEBV2@0@Z 000000014008abb0 f i LIBCMT:undname.obj
 0001:00089bd0       ?getPointerTypeArray@UnDecorator@@CA?AVDName@@AEBV2@0@Z 000000014008abd0 f i LIBCMT:undname.obj
 0001:00089bf0       ?getReferenceType@UnDecorator@@CA?AVDName@@AEBV2@0@Z 000000014008abf0 f i LIBCMT:undname.obj
 0001:00089c10       __unDName                  000000014008ac10 f   LIBCMT:undname.obj
 0001:00089d40       __unDNameEx                000000014008ad40 f   LIBCMT:undname.obj
 0001:00089e80       ?getBasicDataType@UnDecorator@@CA?AVDName@@AEBV2@@Z 000000014008ae80 f   LIBCMT:undname.obj
 0001:0008aa30       ?getPrimaryDataType@UnDecorator@@CA?AVDName@@AEBV2@@Z 000000014008ba30 f   LIBCMT:undname.obj
 0001:0008acd0       ?getDataType@UnDecorator@@CA?AVDName@@PEAV2@@Z 000000014008bcd0 f   LIBCMT:undname.obj
 0001:0008b010       ?getExternalDataType@UnDecorator@@CA?AVDName@@AEBV2@@Z 000000014008c010 f i LIBCMT:undname.obj
 0001:0008b270       __crtMessageBoxA           000000014008c270 f   LIBCMT:crtmbox.obj
 0001:0008b4d0       _set_error_mode            000000014008c4d0 f   LIBCMT:errmode.obj
 0001:0008b530       __set_app_type             000000014008c530 f   LIBCMT:errmode.obj
 0001:0008b540       __get_app_type             000000014008c540 f   LIBCMT:errmode.obj
 0001:0008b730       __crtGetLocaleInfoW        000000014008c730 f   LIBCMT:w_loc.obj
 0001:0008ba30       __crtGetLocaleInfoA        000000014008ca30 f   LIBCMT:a_loc.obj
 0001:0008bb60       _validdrive                000000014008cb60 f   LIBCMT:getcwd.obj
 0001:0008bbb0       _getdcwd_nolock            000000014008cbb0 f   LIBCMT:getcwd.obj
 0001:0008bd80       _getcwd                    000000014008cd80 f   LIBCMT:getcwd.obj
 0001:0008bd80       getcwd                     000000014008cd80 f   LIBCMT:getcwd.obj
 0001:0008bdf0       _getdcwd                   000000014008cdf0 f   LIBCMT:getcwd.obj
 0001:0008be60       _mbsicmp_l                 000000014008ce60 f   LIBCMT:mbsicmp.obj
 0001:0008c1c0       _mbsicmp                   000000014008d1c0 f   LIBCMT:mbsicmp.obj
 0001:0008c1d0       _toupper                   000000014008d1d0 f   LIBCMT:toupper.obj
 0001:0008c1e0       _toupper_l                 000000014008d1e0 f   LIBCMT:toupper.obj
 0001:0008c450       toupper                    000000014008d450 f   LIBCMT:toupper.obj
 0001:0008c9d0       __crtLCMapStringA          000000014008d9d0 f   LIBCMT:a_map.obj
 0001:0008cb30       strpbrk                    000000014008db30 f   LIBCMT:strpbrk.obj
 0001:0008cc00       _getbuf                    000000014008dc00 f   LIBCMT:_getbuf.obj
 0001:0008cc60       _isatty                    000000014008dc60 f   LIBCMT:isatty.obj
 0001:0008cce0       _wctomb_s_l                000000014008dce0 f   LIBCMT:wctomb.obj
 0001:0008cf90       wctomb_s                   000000014008df90 f   LIBCMT:wctomb.obj
 0001:0008cfb0       _wctomb_l                  000000014008dfb0 f   LIBCMT:wctomb.obj
 0001:0008d100       wctomb                     000000014008e100 f   LIBCMT:wctomb.obj
 0001:0008d160       _isleadbyte_l              000000014008e160 f i LIBCMT:_wctype.obj
 0001:0008d250       isleadbyte                 000000014008e250 f i LIBCMT:_wctype.obj
 0001:0008d320       _iswalpha_l                000000014008e320 f i LIBCMT:_wctype.obj
 0001:0008d330       iswalpha                   000000014008e330 f i LIBCMT:_wctype.obj
 0001:0008d340       _iswupper_l                000000014008e340 f i LIBCMT:_wctype.obj
 0001:0008d350       iswupper                   000000014008e350 f i LIBCMT:_wctype.obj
 0001:0008d360       _iswlower_l                000000014008e360 f i LIBCMT:_wctype.obj
 0001:0008d370       iswlower                   000000014008e370 f i LIBCMT:_wctype.obj
 0001:0008d380       _iswdigit_l                000000014008e380 f i LIBCMT:_wctype.obj
 0001:0008d390       iswdigit                   000000014008e390 f i LIBCMT:_wctype.obj
 0001:0008d3a0       _iswxdigit_l               000000014008e3a0 f i LIBCMT:_wctype.obj
 0001:0008d3b0       iswxdigit                  000000014008e3b0 f i LIBCMT:_wctype.obj
 0001:0008d3c0       _iswspace_l                000000014008e3c0 f i LIBCMT:_wctype.obj
 0001:0008d3d0       iswspace                   000000014008e3d0 f i LIBCMT:_wctype.obj
 0001:0008d3e0       _iswpunct_l                000000014008e3e0 f i LIBCMT:_wctype.obj
 0001:0008d3f0       iswpunct                   000000014008e3f0 f i LIBCMT:_wctype.obj
 0001:0008d400       _iswalnum_l                000000014008e400 f i LIBCMT:_wctype.obj
 0001:0008d410       iswalnum                   000000014008e410 f i LIBCMT:_wctype.obj
 0001:0008d420       _iswprint_l                000000014008e420 f i LIBCMT:_wctype.obj
 0001:0008d430       iswprint                   000000014008e430 f i LIBCMT:_wctype.obj
 0001:0008d440       _iswgraph_l                000000014008e440 f i LIBCMT:_wctype.obj
 0001:0008d450       iswgraph                   000000014008e450 f i LIBCMT:_wctype.obj
 0001:0008d460       _iswcntrl_l                000000014008e460 f i LIBCMT:_wctype.obj
 0001:0008d470       iswcntrl                   000000014008e470 f i LIBCMT:_wctype.obj
 0001:0008d480       iswascii                   000000014008e480 f i LIBCMT:_wctype.obj
 0001:0008d490       _iswcsym_l                 000000014008e490 f i LIBCMT:_wctype.obj
 0001:0008d4c0       __iswcsym                  000000014008e4c0 f i LIBCMT:_wctype.obj
 0001:0008d4f0       _iswcsymf_l                000000014008e4f0 f i LIBCMT:_wctype.obj
 0001:0008d520       __iswcsymf                 000000014008e520 f i LIBCMT:_wctype.obj
 0001:0008d550       _ungetc_nolock             000000014008e550 f   LIBCMT:ungetc.obj
 0001:0008d6d0       ungetc                     000000014008e6d0 f   LIBCMT:ungetc.obj
 0001:0008d770       _mbtowc_l                  000000014008e770 f   LIBCMT:mbtowc.obj
 0001:0008d9d0       mbtowc                     000000014008e9d0 f   LIBCMT:mbtowc.obj
 0001:0008d9e0       _setmode_nolock            000000014008e9e0 f   LIBCMT:setmode.obj
 0001:0008dae0       _set_fmode                 000000014008eae0 f   LIBCMT:setmode.obj
 0001:0008db40       _get_fmode                 000000014008eb40 f   LIBCMT:setmode.obj
 0001:0008db90       _setmode                   000000014008eb90 f   LIBCMT:setmode.obj
 0001:0008dd10       _raise_exc_ex              000000014008ed10 f   LIBCMT:fpexcept.obj
 0001:0008e060       _raise_exc                 000000014008f060 f   LIBCMT:fpexcept.obj
 0001:0008e090       _raise_excf                000000014008f090 f   LIBCMT:fpexcept.obj
 0001:0008e0c0       _handle_exc                000000014008f0c0 f   LIBCMT:fpexcept.obj
 0001:0008e3b0       _set_errno_from_matherr    000000014008f3b0 f   LIBCMT:fpexcept.obj
 0001:0008e420       _errcode                   000000014008f420 f   LIBCMT:fpexcept.obj
 0001:0008e460       _umatherr                  000000014008f460 f   LIBCMT:fpexcept.obj
 0001:0008e5a0       _handle_qnan1              000000014008f5a0 f   LIBCMT:fpexcept.obj
 0001:0008e6e0       _handle_qnan2              000000014008f6e0 f   LIBCMT:fpexcept.obj
 0001:0008e820       _except1                   000000014008f820 f   LIBCMT:fpexcept.obj
 0001:0008e980       _except2                   000000014008f980 f   LIBCMT:fpexcept.obj
 0001:0008eb10       _matherr                   000000014008fb10 f   LIBCMT:matherr.obj
 0001:0008eb20       _statfp                    000000014008fb20 f   LIBCMT:fpctrl.obj
 0001:0008eb40       _clrfp                     000000014008fb40 f   LIBCMT:fpctrl.obj
 0001:0008eb60       _ctrlfp                    000000014008fb60 f   LIBCMT:fpctrl.obj
 0001:0008ec10       _set_statfp                000000014008fc10 f   LIBCMT:fpctrl.obj
 0001:0008f130       __crtCompareStringA        0000000140090130 f   LIBCMT:a_cmp.obj
 0001:0008f270       _strnicoll_l               0000000140090270 f   LIBCMT:strnicol.obj
 0001:0008f450       _strnicoll                 0000000140090450 f   LIBCMT:strnicol.obj
 0001:0008f5b0       __crtsetenv                00000001400905b0 f   LIBCMT:setenv.obj
 0001:0008fb60       __crtGetStringTypeA        0000000140090b60 f   LIBCMT:a_str.obj
 0001:0008fcb0       __pwctype_func             0000000140090cb0 f   LIBCMT:ctype.obj
 0001:0008fcc0       __pctype_func              0000000140090cc0 f   LIBCMT:ctype.obj
 0001:000903a0       __free_lc_time             00000001400913a0 f   LIBCMT:inittime.obj
 0001:00090590       __init_time                0000000140091590 f   LIBCMT:inittime.obj
 0001:00090690       __free_lconv_num           0000000140091690 f   LIBCMT:initnum.obj
 0001:000906e0       __init_numeric             00000001400916e0 f   LIBCMT:initnum.obj
 0001:00090990       __free_lconv_mon           0000000140091990 f   LIBCMT:initmon.obj
 0001:00090a30       __init_monetary            0000000140091a30 f   LIBCMT:initmon.obj
 0001:00090e20       __init_collate             0000000140091e20 f   LIBCMT:initcoll.obj
 0001:00090e30       _Getdays_l                 0000000140091e30 f   LIBCMT:strftime.obj
 0001:00091050       _Getdays                   0000000140092050 f   LIBCMT:strftime.obj
 0001:00091060       _Getmonths_l               0000000140092060 f   LIBCMT:strftime.obj
 0001:00091290       _Getmonths                 0000000140092290 f   LIBCMT:strftime.obj
 0001:000912a0       _Gettnames_l               00000001400922a0 f   LIBCMT:strftime.obj
 0001:000917f0       _Gettnames                 00000001400927f0 f   LIBCMT:strftime.obj
 0001:00092630       _Strftime_l                0000000140093630 f   LIBCMT:strftime.obj
 0001:00092990       _strftime_l                0000000140093990 f   LIBCMT:strftime.obj
 0001:000929c0       strftime                   00000001400939c0 f   LIBCMT:strftime.obj
 0001:000929e0       _Strftime                  00000001400939e0 f   LIBCMT:strftime.obj
 0001:00092a10       localeconv                 0000000140093a10 f   LIBCMT:lconv.obj
 0001:00092a50       strcspn                    0000000140093a50 f   LIBCMT:strcspn.obj
 0001:00093550       __get_qualified_locale     0000000140094550 f   LIBCMT:getqloc.obj
 0001:00093920       _putwch_nolock             0000000140094920 f   LIBCMT:putwch.obj
 0001:00093a50       _cputws                    0000000140094a50 f   LIBCMT:putwch.obj
 0001:00093b30       _putwch                    0000000140094b30 f   LIBCMT:putwch.obj
 0001:00093cc0       _ismbbkalnum_l             0000000140094cc0 f   LIBCMT:ismbbyte.obj
 0001:00093da0       _ismbbkalnum               0000000140094da0 f   LIBCMT:ismbbyte.obj
 0001:00093e50       _ismbbkprint_l             0000000140094e50 f   LIBCMT:ismbbyte.obj
 0001:00093f40       _ismbbkprint               0000000140094f40 f   LIBCMT:ismbbyte.obj
 0001:00094000       _ismbbkpunct_l             0000000140095000 f   LIBCMT:ismbbyte.obj
 0001:000940e0       _ismbbkpunct               00000001400950e0 f   LIBCMT:ismbbyte.obj
 0001:00094190       _ismbbalnum_l              0000000140095190 f   LIBCMT:ismbbyte.obj
 0001:000942a0       _ismbbalnum                00000001400952a0 f   LIBCMT:ismbbyte.obj
 0001:00094380       _ismbbalpha_l              0000000140095380 f   LIBCMT:ismbbyte.obj
 0001:00094490       _ismbbalpha                0000000140095490 f   LIBCMT:ismbbyte.obj
 0001:00094570       _ismbbgraph_l              0000000140095570 f   LIBCMT:ismbbyte.obj
 0001:00094680       _ismbbgraph                0000000140095680 f   LIBCMT:ismbbyte.obj
 0001:00094760       _ismbbprint_l              0000000140095760 f   LIBCMT:ismbbyte.obj
 0001:00094870       _ismbbprint                0000000140095870 f   LIBCMT:ismbbyte.obj
 0001:00094950       _ismbbpunct_l              0000000140095950 f   LIBCMT:ismbbyte.obj
 0001:00094a60       _ismbbpunct                0000000140095a60 f   LIBCMT:ismbbyte.obj
 0001:00094b40       _ismbblead_l               0000000140095b40 f   LIBCMT:ismbbyte.obj
 0001:00094c20       _ismbblead                 0000000140095c20 f   LIBCMT:ismbbyte.obj
 0001:00094ce0       _ismbbtrail_l              0000000140095ce0 f   LIBCMT:ismbbyte.obj
 0001:00094dc0       _ismbbtrail                0000000140095dc0 f   LIBCMT:ismbbyte.obj
 0001:00094e80       _ismbbkana_l               0000000140095e80 f   LIBCMT:ismbbyte.obj
 0001:00094fa0       _ismbbkana                 0000000140095fa0 f   LIBCMT:ismbbyte.obj
 0001:00095a20       _open                      0000000140096a20 f   LIBCMT:open.obj
 0001:00095b60       _sopen_helper              0000000140096b60 f   LIBCMT:open.obj
 0001:00095d00       _sopen                     0000000140096d00 f   LIBCMT:open.obj
 0001:00095d50       _sopen_s                   0000000140096d50 f   LIBCMT:open.obj
 0001:00095d90       _mbsnbcmp_l                0000000140096d90 f   LIBCMT:mbsnbcmp.obj
 0001:00095fa0       _mbsnbcmp                  0000000140096fa0 f   LIBCMT:mbsnbcmp.obj
 0001:00095fb0       __addl                     0000000140096fb0 f i LIBCMT:intrncvt.obj
 0001:00095fd0       _ZeroTail                  0000000140096fd0 f i LIBCMT:intrncvt.obj
 0001:00096030       _IncMan                    0000000140097030 f i LIBCMT:intrncvt.obj
 0001:000960b0       _RoundMan                  00000001400970b0 f i LIBCMT:intrncvt.obj
 0001:00096210       _CopyMan                   0000000140097210 f i LIBCMT:intrncvt.obj
 0001:00096230       _FillZeroMan               0000000140097230 f i LIBCMT:intrncvt.obj
 0001:00096240       _IsZeroMan                 0000000140097240 f i LIBCMT:intrncvt.obj
 0001:00096260       _ShrMan                    0000000140097260 f i LIBCMT:intrncvt.obj
 0001:00096310       _ld12cvt                   0000000140097310 f i LIBCMT:intrncvt.obj
 0001:000969d0       _ld12tod                   00000001400979d0 f   LIBCMT:intrncvt.obj
 0001:00097090       _ld12tof                   0000000140098090 f   LIBCMT:intrncvt.obj
 0001:00097750       _ld12told                  0000000140098750 f   LIBCMT:intrncvt.obj
 0001:00097820       __shl_12                   0000000140098820 f i LIBCMT:strgtold.obj
 0001:00097850       __shr_12                   0000000140098850 f i LIBCMT:strgtold.obj
 0001:00097880       __ld12mul                  0000000140098880 f i LIBCMT:strgtold.obj
 0001:00097c20       __multtenpow12             0000000140098c20 f i LIBCMT:strgtold.obj
 0001:000980b0       __strgtold12_l             00000001400990b0 f   LIBCMT:strgtold.obj
 0001:00098ae0       __STRINGTOLD_L             0000000140099ae0 f   LIBCMT:strgtold.obj
 0001:00098b50       __add_12                   0000000140099b50 f i LIBCMT:x10fout.obj
 0001:00098be0       $I10_OUTPUT                0000000140099be0 f   LIBCMT:x10fout.obj
 0001:000999e0       __ascii_stricmp            000000014009a9e0 f   LIBCMT:stricmp.obj
 0001:00099a30       _stricmp_l                 000000014009aa30 f   LIBCMT:stricmp.obj
 0001:00099c10       _stricmp                   000000014009ac10 f   LIBCMT:stricmp.obj
 0001:00099c10       stricmp                    000000014009ac10 f   LIBCMT:stricmp.obj
 0001:00099cb0       __ansicp                   000000014009acb0 f   LIBCMT:convrtcp.obj
 0001:00099d20       __convertcp                000000014009ad20 f   LIBCMT:convrtcp.obj
 0001:00099fb0       _iswctype_l                000000014009afb0 f   LIBCMT:iswctype.obj
 0001:0009a120       iswctype                   000000014009b120 f   LIBCMT:iswctype.obj
 0001:0009a1c0       is_wctype                  000000014009b1c0 f   LIBCMT:iswctype.obj
 0001:0009a270       _set_exp                   000000014009b270 f   LIBCMT:util.obj
 0001:0009a2b0       _get_exp                   000000014009b2b0 f   LIBCMT:util.obj
 0001:0009a2d0       _add_exp                   000000014009b2d0 f   LIBCMT:util.obj
 0001:0009a320       _set_bexp                  000000014009b320 f   LIBCMT:util.obj
 0001:0009a350       _sptype                    000000014009b350 f   LIBCMT:util.obj
 0001:0009a3c0       _decomp                    000000014009b3c0 f   LIBCMT:util.obj
 0001:0009a4e0       _set_fpsr                  000000014009b4e0 f   LIBCMT:fpsr.obj
 0001:0009a4ea       _fclrf                     000000014009b4ea f   LIBCMT:fpsr.obj
 0001:0009a500       __ascii_strnicmp           000000014009b500 f   LIBCMT:strnicmp.obj
 0001:0009a560       _strnicmp_l                000000014009b560 f   LIBCMT:strnicmp.obj
 0001:0009a760       _strnicmp                  000000014009b760 f   LIBCMT:strnicmp.obj
 0001:0009a820       _strdup                    000000014009b820 f   LIBCMT:strdup.obj
 0001:0009a820       strdup                     000000014009b820 f   LIBCMT:strdup.obj
 0001:0009a8b0       _mbschr_l                  000000014009b8b0 f   LIBCMT:mbschr.obj
 0001:0009aa50       _mbschr                    000000014009ba50 f   LIBCMT:mbschr.obj
 0001:0009abb0       _itoa_s                    000000014009bbb0 f   LIBCMT:xtoas.obj
 0001:0009ace0       _ltoa_s                    000000014009bce0 f   LIBCMT:xtoas.obj
 0001:0009ad20       _ultoa_s                   000000014009bd20 f   LIBCMT:xtoas.obj
 0001:0009af80       _i64toa_s                  000000014009bf80 f   LIBCMT:xtoas.obj
 0001:0009afc0       _ui64toa_s                 000000014009bfc0 f   LIBCMT:xtoas.obj
 0001:0009b0d0       _chsize_nolock             000000014009c0d0 f   LIBCMT:chsize.obj
 0001:0009b290       _chsize_s                  000000014009c290 f   LIBCMT:chsize.obj
 0001:0009b400       _chsize                    000000014009c400 f   LIBCMT:chsize.obj
 0001:0009b420       __mtold12                  000000014009c420 f   LIBCMT:mantold.obj
 0001:0009b980       __crtGetStringTypeW        000000014009c980 f   LIBCMT:w_str.obj
 0001:0009babe       CreateEventA               000000014009cabe f   kernel32:KERNEL32.dll
 0001:0009bac4       SetEvent                   000000014009cac4 f   kernel32:KERNEL32.dll
 0001:0009baca       ResetEvent                 000000014009caca f   kernel32:KERNEL32.dll
 0001:0009bad0       WaitForMultipleObjects     000000014009cad0 f   kernel32:KERNEL32.dll
 0001:0009bad6       TryEnterCriticalSection    000000014009cad6 f   kernel32:KERNEL32.dll
 0001:0009badc       SetThreadPriority          000000014009cadc f   kernel32:KERNEL32.dll
 0001:0009bae2       GetLocaleInfoA             000000014009cae2 f   kernel32:KERNEL32.dll
 0001:0009bae8       GetSystemDirectoryA        000000014009cae8 f   kernel32:KERNEL32.dll
 0001:0009baee       GetWindowsDirectoryA       000000014009caee f   kernel32:KERNEL32.dll
 0001:0009baf4       DeleteFileA                000000014009caf4 f   kernel32:KERNEL32.dll
 0001:0009bafa       MoveFileA                  000000014009cafa f   kernel32:KERNEL32.dll
 0001:0009bb00       GetTickCount               000000014009cb00 f   kernel32:KERNEL32.dll
 0001:0009bb06       GetFileAttributesExA       000000014009cb06 f   kernel32:KERNEL32.dll
 0001:0009bb0c       SetEndOfFile               000000014009cb0c f   kernel32:KERNEL32.dll
 0001:0009bb12       SetFilePointer             000000014009cb12 f   kernel32:KERNEL32.dll
 0001:0009bb18       GetFileAttributesA         000000014009cb18 f   kernel32:KERNEL32.dll
 0001:0009bb1e       GetFullPathNameA           000000014009cb1e f   kernel32:KERNEL32.dll
 0001:0009bb24       ReadFile                   000000014009cb24 f   kernel32:KERNEL32.dll
 0001:0009bb2a       WriteFile                  000000014009cb2a f   kernel32:KERNEL32.dll
 0001:0009bb30       UnmapViewOfFile            000000014009cb30 f   kernel32:KERNEL32.dll
 0001:0009bb36       FindClose                  000000014009cb36 f   kernel32:KERNEL32.dll
 0001:0009bb3c       FindNextFileA              000000014009cb3c f   kernel32:KERNEL32.dll
 0001:0009bb42       FindFirstFileA             000000014009cb42 f   kernel32:KERNEL32.dll
 0001:0009bb48       QueryPerformanceCounter    000000014009cb48 f   kernel32:KERNEL32.dll
 0001:0009bb4e       QueryPerformanceFrequency  000000014009cb4e f   kernel32:KERNEL32.dll
 0001:0009bb54       FileTimeToSystemTime       000000014009cb54 f   kernel32:KERNEL32.dll
 0001:0009bb5a       FileTimeToLocalFileTime    000000014009cb5a f   kernel32:KERNEL32.dll
 0001:0009bb60       GetDriveTypeA              000000014009cb60 f   kernel32:KERNEL32.dll
 0001:0009bb66       ExitProcess                000000014009cb66 f   kernel32:KERNEL32.dll
 0001:0009bb6c       SetConsoleCtrlHandler      000000014009cb6c f   kernel32:KERNEL32.dll
 0001:0009bb72       ReadConsoleInputA          000000014009cb72 f   kernel32:KERNEL32.dll
 0001:0009bb78       SetConsoleMode             000000014009cb78 f   kernel32:KERNEL32.dll
 0001:0009bb7e       GetConsoleMode             000000014009cb7e f   kernel32:KERNEL32.dll
 0001:0009bb84       PeekConsoleInputA          000000014009cb84 f   kernel32:KERNEL32.dll
 0001:0009bb8a       GetNumberOfConsoleInputEvents 000000014009cb8a f   kernel32:KERNEL32.dll
 0001:0009bb90       GetCommandLineA            000000014009cb90 f   kernel32:KERNEL32.dll
 0001:0009bb96       HeapFree                   000000014009cb96 f   kernel32:KERNEL32.dll
 0001:0009bb9c       GetVersionExA              000000014009cb9c f   kernel32:KERNEL32.dll
 0001:0009bba2       HeapAlloc                  000000014009cba2 f   kernel32:KERNEL32.dll
 0001:0009bba8       GetProcessHeap             000000014009cba8 f   kernel32:KERNEL32.dll
 0001:0009bbae       HeapReAlloc                000000014009cbae f   kernel32:KERNEL32.dll
 0001:0009bbb4       GetFileInformationByHandle 000000014009cbb4 f   kernel32:KERNEL32.dll
 0001:0009bbba       PeekNamedPipe              000000014009cbba f   kernel32:KERNEL32.dll
 0001:0009bbc0       GetFileType                000000014009cbc0 f   kernel32:KERNEL32.dll
 0001:0009bbc6       SetStdHandle               000000014009cbc6 f   kernel32:KERNEL32.dll
 0001:0009bbcc       ExitThread                 000000014009cbcc f   kernel32:KERNEL32.dll
 0001:0009bbd2       ResumeThread               000000014009cbd2 f   kernel32:KERNEL32.dll
 0001:0009bbd8       CreateThread               000000014009cbd8 f   kernel32:KERNEL32.dll
 0001:0009bbde       WideCharToMultiByte        000000014009cbde f   kernel32:KERNEL32.dll
 0001:0009bbe4       GetTimeZoneInformation     000000014009cbe4 f   kernel32:KERNEL32.dll
 0001:0009bbea       UnhandledExceptionFilter   000000014009cbea f   kernel32:KERNEL32.dll
 0001:0009bbf0       SetUnhandledExceptionFilter 000000014009cbf0 f   kernel32:KERNEL32.dll
 0001:0009bbf6       IsDebuggerPresent          000000014009cbf6 f   kernel32:KERNEL32.dll
 0001:0009bbfc       RtlCaptureContext          000000014009cbfc f   kernel32:KERNEL32.dll
 0001:0009bc02       GetStdHandle               000000014009cc02 f   kernel32:KERNEL32.dll
 0001:0009bc08       FlsGetValue                000000014009cc08 f   kernel32:KERNEL32.dll
 0001:0009bc0e       TlsAlloc                   000000014009cc0e f   kernel32:KERNEL32.dll
 0001:0009bc14       FlsSetValue                000000014009cc14 f   kernel32:KERNEL32.dll
 0001:0009bc1a       TlsFree                    000000014009cc1a f   kernel32:KERNEL32.dll
 0001:0009bc20       FlsFree                    000000014009cc20 f   kernel32:KERNEL32.dll
 0001:0009bc26       TlsSetValue                000000014009cc26 f   kernel32:KERNEL32.dll
 0001:0009bc2c       GetCurrentThread           000000014009cc2c f   kernel32:KERNEL32.dll
 0001:0009bc32       FlsAlloc                   000000014009cc32 f   kernel32:KERNEL32.dll
 0001:0009bc38       GetCurrentDirectoryA       000000014009cc38 f   kernel32:KERNEL32.dll
 0001:0009bc3e       SetCurrentDirectoryA       000000014009cc3e f   kernel32:KERNEL32.dll
 0001:0009bc44       RtlVirtualUnwind           000000014009cc44 f   kernel32:KERNEL32.dll
 0001:0009bc4a       RtlLookupFunctionEntry     000000014009cc4a f   kernel32:KERNEL32.dll
 0001:0009bc50       RaiseException             000000014009cc50 f   kernel32:KERNEL32.dll
 0001:0009bc56       RtlPcToFileHeader          000000014009cc56 f   kernel32:KERNEL32.dll
 0001:0009bc5c       RtlUnwindEx                000000014009cc5c f   kernel32:KERNEL32.dll
 0001:0009bc62       SetHandleCount             000000014009cc62 f   kernel32:KERNEL32.dll
 0001:0009bc68       GetStartupInfoA            000000014009cc68 f   kernel32:KERNEL32.dll
 0001:0009bc6e       FatalAppExitA              000000014009cc6e f   kernel32:KERNEL32.dll
 0001:0009bc74       FreeLibrary                000000014009cc74 f   kernel32:KERNEL32.dll
 0001:0009bc7a       LoadLibraryA               000000014009cc7a f   kernel32:KERNEL32.dll
 0001:0009bc80       CreatePipe                 000000014009cc80 f   kernel32:KERNEL32.dll
 0001:0009bc86       GetCPInfo                  000000014009cc86 f   kernel32:KERNEL32.dll
 0001:0009bc8c       GetACP                     000000014009cc8c f   kernel32:KERNEL32.dll
 0001:0009bc92       GetOEMCP                   000000014009cc92 f   kernel32:KERNEL32.dll
 0001:0009bc98       IsValidCodePage            000000014009cc98 f   kernel32:KERNEL32.dll
 0001:0009bc9e       FreeEnvironmentStringsA    000000014009cc9e f   kernel32:KERNEL32.dll
 0001:0009bca4       GetEnvironmentStrings      000000014009cca4 f   kernel32:KERNEL32.dll
 0001:0009bcaa       FreeEnvironmentStringsW    000000014009ccaa f   kernel32:KERNEL32.dll
 0001:0009bcb0       GetEnvironmentStringsW     000000014009ccb0 f   kernel32:KERNEL32.dll
 0001:0009bcb6       HeapSetInformation         000000014009ccb6 f   kernel32:KERNEL32.dll
 0001:0009bcbc       HeapCreate                 000000014009ccbc f   kernel32:KERNEL32.dll
 0001:0009bcc2       HeapDestroy                000000014009ccc2 f   kernel32:KERNEL32.dll
 0001:0009bcc8       GetCurrentProcessId        000000014009ccc8 f   kernel32:KERNEL32.dll
 0001:0009bcce       HeapSize                   000000014009ccce f   kernel32:KERNEL32.dll
 0001:0009bcd4       GetConsoleCP               000000014009ccd4 f   kernel32:KERNEL32.dll
 0001:0009bcda       FlushFileBuffers           000000014009ccda f   kernel32:KERNEL32.dll
 0001:0009bce0       MultiByteToWideChar        000000014009cce0 f   kernel32:KERNEL32.dll
 0001:0009bce6       GetLocaleInfoW             000000014009cce6 f   kernel32:KERNEL32.dll
 0001:0009bcec       LCMapStringA               000000014009ccec f   kernel32:KERNEL32.dll
 0001:0009bcf2       LCMapStringW               000000014009ccf2 f   kernel32:KERNEL32.dll
 0001:0009bcf8       CompareStringA             000000014009ccf8 f   kernel32:KERNEL32.dll
 0001:0009bcfe       CompareStringW             000000014009ccfe f   kernel32:KERNEL32.dll
 0001:0009bd04       SetEnvironmentVariableA    000000014009cd04 f   kernel32:KERNEL32.dll
 0001:0009bd0a       GetStringTypeA             000000014009cd0a f   kernel32:KERNEL32.dll
 0001:0009bd10       GetStringTypeW             000000014009cd10 f   kernel32:KERNEL32.dll
 0001:0009bd16       GetDateFormatA             000000014009cd16 f   kernel32:KERNEL32.dll
 0001:0009bd1c       GetTimeFormatA             000000014009cd1c f   kernel32:KERNEL32.dll
 0001:0009bd22       GetUserDefaultLCID         000000014009cd22 f   kernel32:KERNEL32.dll
 0001:0009bd28       EnumSystemLocalesA         000000014009cd28 f   kernel32:KERNEL32.dll
 0001:0009bd2e       IsValidLocale              000000014009cd2e f   kernel32:KERNEL32.dll
 0001:0009bd34       WriteConsoleA              000000014009cd34 f   kernel32:KERNEL32.dll
 0001:0009bd3a       GetConsoleOutputCP         000000014009cd3a f   kernel32:KERNEL32.dll
 0001:0009bd40       WriteConsoleW              000000014009cd40 f   kernel32:KERNEL32.dll
 0001:0009bd46       SetTimer                   000000014009cd46 f   user32:USER32.dll
 0001:0009bd4c       KillTimer                  000000014009cd4c f   user32:USER32.dll
 0001:0009bd52       PeekMessageA               000000014009cd52 f   user32:USER32.dll
 0001:0009bd58       RegCloseKey                000000014009cd58 f   advapi32:ADVAPI32.dll
 0001:0009bd5e       RegEnumValueA              000000014009cd5e f   advapi32:ADVAPI32.dll
 0001:0009bd64       RegOpenKeyExA              000000014009cd64 f   advapi32:ADVAPI32.dll
 0001:0009bd70       ??$rotlFixed@I@TaoCrypt@@YAIII@Z 000000014009cd70 f i taocrypt:md5.obj
 0001:0009bd80       ?Init@MD5@TaoCrypt@@UEAAXXZ 000000014009cd80 f   taocrypt:md5.obj
 0001:0009bdb0       ??0MD5@TaoCrypt@@QEAA@AEBV01@@Z 000000014009cdb0 f   taocrypt:md5.obj
 0001:0009be30       ?Transform@MD5@TaoCrypt@@EEAAXXZ 000000014009ce30 f   taocrypt:md5.obj
 0001:0009c5b0       ?Swap@MD5@TaoCrypt@@QEAAXAEAV12@@Z 000000014009d5b0 f   taocrypt:md5.obj
 0001:0009c610       ??4MD5@TaoCrypt@@QEAAAEAV01@AEBV01@@Z 000000014009d610 f   taocrypt:md5.obj
 0001:0009c640       ??$rotrFixed@I@TaoCrypt@@YAIII@Z 000000014009d640 f i taocrypt:hash.obj
 0001:0009c650       ?ByteReverse@TaoCrypt@@YAII@Z 000000014009d650 f i taocrypt:hash.obj
 0001:0009c670       ?GetBitCountLo@HASHwithTransform@TaoCrypt@@QEBAIXZ 000000014009d670 f i taocrypt:hash.obj
 0001:0009c680       ?GetBitCountHi@HASHwithTransform@TaoCrypt@@QEBAIXZ 000000014009d680 f i taocrypt:hash.obj
 0001:0009c690       ?GetBitCountLo@HASH64withTransform@TaoCrypt@@QEBAIXZ 000000014009d690 f i taocrypt:hash.obj
 0001:0009c6a0       ?GetBitCountHi@HASH64withTransform@TaoCrypt@@QEBAIXZ 000000014009d6a0 f i taocrypt:hash.obj
 0001:0009c6b0       ??0HASH@TaoCrypt@@QEAA@XZ  000000014009d6b0 f i taocrypt:hash.obj
 0001:0009c6c0       ??0HASH64withTransform@TaoCrypt@@QEAA@II@Z 000000014009d6c0 f   taocrypt:hash.obj
 0001:0009c6d0       ??1HASH64withTransform@TaoCrypt@@UEAA@XZ 000000014009d6d0 f i taocrypt:hash.obj
 0001:0009c6e0       ??_EHASH64withTransform@TaoCrypt@@UEAAPEAXI@Z 000000014009d6e0 f i taocrypt:hash.obj
 0001:0009c6e0       ??_GHASH64withTransform@TaoCrypt@@UEAAPEAXI@Z 000000014009d6e0 f i taocrypt:hash.obj
 0001:0009c710       ?ToEnum@?$EnumToType@W4ByteOrder@TaoCrypt@@$0A@@TaoCrypt@@SA?AW4ByteOrder@2@XZ 000000014009d710 f i taocrypt:hash.obj
 0001:0009c720       ??$rotlFixed@_K@TaoCrypt@@YA_K_KI@Z 000000014009d720 f i taocrypt:hash.obj
 0001:0009c730       ??$ByteReverse@I@TaoCrypt@@YAXPEAIPEBII@Z 000000014009d730 f i taocrypt:hash.obj
 0001:0009c770       ??$RightShift@I@?$SafeShifter@$00@TaoCrypt@@SAIII@Z 000000014009d770 f i taocrypt:hash.obj
 0001:0009c780       ?GetHostByteOrder@TaoCrypt@@YA?AW4ByteOrder@1@XZ 000000014009d780 f i taocrypt:hash.obj
 0001:0009c790       ?HostByteOrderIs@TaoCrypt@@YA_NW4ByteOrder@1@@Z 000000014009d790 f i taocrypt:hash.obj
 0001:0009c7a0       ?ByteReverse@TaoCrypt@@YA_K_K@Z 000000014009d7a0 f i taocrypt:hash.obj
 0001:0009c7f0       ?ByteReverse@TaoCrypt@@YAXPEAEPEBEI@Z 000000014009d7f0 f i taocrypt:hash.obj
 0001:0009c830       ??0HASHwithTransform@TaoCrypt@@QEAA@II@Z 000000014009d830 f   taocrypt:hash.obj
 0001:0009c840       ??_GHASHwithTransform@TaoCrypt@@UEAAPEAXI@Z 000000014009d840 f i taocrypt:hash.obj
 0001:0009c840       ??_EHASHwithTransform@TaoCrypt@@UEAAPEAXI@Z 000000014009d840 f i taocrypt:hash.obj
 0001:0009c870       ??$SafeRightShift@$0CA@I@TaoCrypt@@YAII@Z 000000014009d870 f i taocrypt:hash.obj
 0001:0009c880       ??$ByteReverseIf@E@TaoCrypt@@YAXPEAEPEBEIW4ByteOrder@0@@Z 000000014009d880 f i taocrypt:hash.obj
 0001:0009c8e0       ??$ByteReverseIf@I@TaoCrypt@@YAXPEAIPEBIIW4ByteOrder@0@@Z 000000014009d8e0 f i taocrypt:hash.obj
 0001:0009c940       ??$ByteReverse@_K@TaoCrypt@@YAXPEA_KPEB_KI@Z 000000014009d940 f i taocrypt:hash.obj
 0001:0009c9d0       ?AddLength@HASHwithTransform@TaoCrypt@@IEAAXI@Z 000000014009d9d0 f   taocrypt:hash.obj
 0001:0009c9f0       ?Update@HASHwithTransform@TaoCrypt@@UEAAXPEBEI@Z 000000014009d9f0 f   taocrypt:hash.obj
 0001:0009caf0       ?Final@HASHwithTransform@TaoCrypt@@UEAAXPEAE@Z 000000014009daf0 f   taocrypt:hash.obj
 0001:0009ccf0       ?AddLength@HASH64withTransform@TaoCrypt@@IEAAXI@Z 000000014009dcf0 f   taocrypt:hash.obj
 0001:0009cd10       ??$ByteReverseIf@_K@TaoCrypt@@YAXPEA_KPEB_KIW4ByteOrder@0@@Z 000000014009dd10 f i taocrypt:hash.obj
 0001:0009cdc0       ?Update@HASH64withTransform@TaoCrypt@@UEAAXPEBEI@Z 000000014009ddc0 f   taocrypt:hash.obj
 0001:0009cf30       ?Final@HASH64withTransform@TaoCrypt@@UEAAXPEAE@Z 000000014009df30 f   taocrypt:hash.obj
 0001:0009d230       ?Init@MD4@TaoCrypt@@UEAAXXZ 000000014009e230 f   taocrypt:md4.obj
 0001:0009d260       ??0MD4@TaoCrypt@@QEAA@AEBV01@@Z 000000014009e260 f   taocrypt:md4.obj
 0001:0009d2e0       ?Transform@MD4@TaoCrypt@@EEAAXXZ 000000014009e2e0 f   taocrypt:md4.obj
 0001:0009d800       ?Swap@MD4@TaoCrypt@@QEAAXAEAV12@@Z 000000014009e800 f   taocrypt:md4.obj
 0001:0009d860       ??4MD4@TaoCrypt@@QEAAAEAV01@AEBV01@@Z 000000014009e860 f   taocrypt:md4.obj
 0001:0009d890       ?SetError@Error@TaoCrypt@@QEAAXW4ErrorNumber@2@@Z 000000014009e890 f i taocrypt:coding.obj
 0001:0009d8a0       ?GetError@Source@TaoCrypt@@QEAA?AUError@2@XZ 000000014009e8a0 f i taocrypt:coding.obj
 0001:0009d8b0       ?SetError@Source@TaoCrypt@@QEAAXW4ErrorNumber@2@@Z 000000014009e8b0 f i taocrypt:coding.obj
 0001:0009d8c0       ??A?$Block@EV?$AllocatorWithCleanup@E@TaoCrypt@@@TaoCrypt@@QEAAAEAEI@Z 000000014009e8c0 f i taocrypt:coding.obj
 0001:0009d8d0       ?remaining@Source@TaoCrypt@@QEAAIXZ 000000014009e8d0 f i taocrypt:coding.obj
 0001:0009d8e0       ?IsLeft@Source@TaoCrypt@@QEAA_NI@Z 000000014009e8e0 f i taocrypt:coding.obj
 0001:0009d900       ?next@Source@TaoCrypt@@QEAAEXZ 000000014009e900 f i taocrypt:coding.obj
 0001:0009d930       ?resize@?$Block@EV?$AllocatorWithCleanup@E@TaoCrypt@@@TaoCrypt@@QEAAXI@Z 000000014009e930 f i taocrypt:coding.obj
 0001:0009d970       ?Encode@HexEncoder@TaoCrypt@@AEAAXXZ 000000014009e970 f   taocrypt:coding.obj
 0001:0009da50       ?Decode@HexDecoder@TaoCrypt@@AEAAXXZ 000000014009ea50 f   taocrypt:coding.obj
 0001:0009db50       ?Encode@Base64Encoder@TaoCrypt@@AEAAXXZ 000000014009eb50 f   taocrypt:coding.obj
 0001:0009de30       ?Decode@Base64Decoder@TaoCrypt@@AEAAXXZ 000000014009ee30 f   taocrypt:coding.obj
 0001:0009e140       ?BytesToWords@TaoCrypt@@YAII@Z 000000014009f140 f i taocrypt:integer.obj
 0001:0009e150       ?BitsToWords@TaoCrypt@@YAII@Z 000000014009f150 f i taocrypt:integer.obj
 0001:0009e160       ?CopyWords@TaoCrypt@@YAXPEA_KPEB_KI@Z 000000014009f160 f i taocrypt:integer.obj
 0001:0009e190       ?CountWords@TaoCrypt@@YAIPEB_KI@Z 000000014009f190 f i taocrypt:integer.obj
 0001:0009e1c0       ?SetWords@TaoCrypt@@YAXPEA_K_KI@Z 000000014009f1c0 f i taocrypt:integer.obj
 0001:0009e1e0       ?ShiftWordsLeftByBits@TaoCrypt@@YA_KPEA_KII@Z 000000014009f1e0 f i taocrypt:integer.obj
 0001:0009e250       ?ShiftWordsRightByBits@TaoCrypt@@YA_KPEA_KII@Z 000000014009f250 f i taocrypt:integer.obj
 0001:0009e2b0       ?IsNegative@Integer@TaoCrypt@@QEBA_NXZ 000000014009f2b0 f i taocrypt:integer.obj
 0001:0009e2c0       ?NotNegative@Integer@TaoCrypt@@QEBA_NXZ 000000014009f2c0 f i taocrypt:integer.obj
 0001:0009e2d0       ??1AbstractGroup@TaoCrypt@@UEAA@XZ 000000014009f2d0 f i taocrypt:integer.obj
 0001:0009e2e0       ??0AbstractGroup@TaoCrypt@@QEAA@XZ 000000014009f2e0 f i taocrypt:integer.obj
 0001:0009e2f0       ??0MultiplicativeGroupT@AbstractRing@TaoCrypt@@QEAA@XZ 000000014009f2f0 f i taocrypt:integer.obj
 0001:0009e300       ?InversionIsFast@AbstractGroup@TaoCrypt@@UEBA_NXZ 000000014009f300 f i taocrypt:integer.obj
 0001:0009e310       ?GetRing@MultiplicativeGroupT@AbstractRing@TaoCrypt@@QEBAAEBV23@XZ 000000014009f310 f i taocrypt:integer.obj
 0001:0009e320       ?Equal@MultiplicativeGroupT@AbstractRing@TaoCrypt@@UEBA_NAEBVInteger@3@0@Z 000000014009f320 f i taocrypt:integer.obj
 0001:0009e330       ?Identity@MultiplicativeGroupT@AbstractRing@TaoCrypt@@UEBAAEBVInteger@3@XZ 000000014009f330 f i taocrypt:integer.obj
 0001:0009e340       ?Add@MultiplicativeGroupT@AbstractRing@TaoCrypt@@UEBAAEBVInteger@3@AEBV43@0@Z 000000014009f340 f i taocrypt:integer.obj
 0001:0009e350       ?Inverse@MultiplicativeGroupT@AbstractRing@TaoCrypt@@UEBAAEBVInteger@3@AEBV43@@Z 000000014009f350 f i taocrypt:integer.obj
 0001:0009e360       ?Subtract@MultiplicativeGroupT@AbstractRing@TaoCrypt@@UEBAAEBVInteger@3@AEBV43@0@Z 000000014009f360 f i taocrypt:integer.obj
 0001:0009e370       ?Double@MultiplicativeGroupT@AbstractRing@TaoCrypt@@UEBAAEBVInteger@3@AEBV43@@Z 000000014009f370 f i taocrypt:integer.obj
 0001:0009e380       ?SimultaneousMultiply@MultiplicativeGroupT@AbstractRing@TaoCrypt@@UEBAXPEAVInteger@3@AEBV43@PEBV43@I@Z 000000014009f380 f i taocrypt:integer.obj
 0001:0009e3a0       ??1MultiplicativeGroupT@AbstractRing@TaoCrypt@@UEAA@XZ 000000014009f3a0 f i taocrypt:integer.obj
 0001:0009e3b0       ??1AbstractRing@TaoCrypt@@UEAA@XZ 000000014009f3b0 f i taocrypt:integer.obj
 0001:0009e3c0       ??_GMultiplicativeGroupT@AbstractRing@TaoCrypt@@UEAAPEAXI@Z 000000014009f3c0 f i taocrypt:integer.obj
 0001:0009e3c0       ??_EMultiplicativeGroupT@AbstractRing@TaoCrypt@@UEAAPEAXI@Z 000000014009f3c0 f i taocrypt:integer.obj
 0001:0009e3e0       ?SimultaneousExponentiate@MontgomeryRepresentation@TaoCrypt@@UEBAXPEAVInteger@2@AEBV32@PEBV32@I@Z 000000014009f3e0 f i taocrypt:integer.obj
 0001:0009e400       ??0DWord@TaoCrypt@@QEAA@XZ 000000014009f400 f i taocrypt:integer.obj
 0001:0009e410       ??0DWord@TaoCrypt@@QEAA@_K@Z 000000014009f410 f i taocrypt:integer.obj
 0001:0009e420       ??0DWord@TaoCrypt@@QEAA@_K0@Z 000000014009f420 f i taocrypt:integer.obj
 0001:0009e430       ?Multiply@DWord@TaoCrypt@@SA?AV12@_K0@Z 000000014009f430 f i taocrypt:integer.obj
 0001:0009e450       ??YDWord@TaoCrypt@@QEAAAEAV01@_K@Z 000000014009f450 f i taocrypt:integer.obj
 0001:0009e460       ??HDWord@TaoCrypt@@QEAA?AV01@_K@Z 000000014009f460 f i taocrypt:integer.obj
 0001:0009e480       ??GDWord@TaoCrypt@@QEAA?AV01@V01@@Z 000000014009f480 f i taocrypt:integer.obj
 0001:0009e4b0       ??GDWord@TaoCrypt@@QEAA?AV01@_K@Z 000000014009f4b0 f i taocrypt:integer.obj
 0001:0009e4e0       ??7DWord@TaoCrypt@@QEBA_NXZ 000000014009f4e0 f i taocrypt:integer.obj
 0001:0009e500       ?GetLowHalf@DWord@TaoCrypt@@QEBA_KXZ 000000014009f500 f i taocrypt:integer.obj
 0001:0009e510       ?GetHighHalf@DWord@TaoCrypt@@QEBA_KXZ 000000014009f510 f i taocrypt:integer.obj
 0001:0009e520       ?GetHighHalfAsBorrow@DWord@TaoCrypt@@QEBA_KXZ 000000014009f520 f i taocrypt:integer.obj
 0001:0009e530       ??0Word@TaoCrypt@@QEAA@XZ  000000014009f530 f i taocrypt:integer.obj
 0001:0009e540       ??0Word@TaoCrypt@@QEAA@_K@Z 000000014009f540 f i taocrypt:integer.obj
 0001:0009e550       ??0Word@TaoCrypt@@QEAA@II@Z 000000014009f550 f i taocrypt:integer.obj
 0001:0009e570       ?Multiply@Word@TaoCrypt@@SA?AV12@II@Z 000000014009f570 f i taocrypt:integer.obj
 0001:0009e590       ??GWord@TaoCrypt@@QEAA?AV01@V01@@Z 000000014009f590 f i taocrypt:integer.obj
 0001:0009e5a0       ??GWord@TaoCrypt@@QEAA?AV01@I@Z 000000014009f5a0 f i taocrypt:integer.obj
 0001:0009e5b0       ??KWord@TaoCrypt@@QEAAII@Z 000000014009f5b0 f i taocrypt:integer.obj
 0001:0009e5c0       ??7Word@TaoCrypt@@QEBA_NXZ 000000014009f5c0 f i taocrypt:integer.obj
 0001:0009e5d0       ?GetWhole@Word@TaoCrypt@@QEBA_KXZ 000000014009f5d0 f i taocrypt:integer.obj
 0001:0009e5e0       ?GetLowHalf@Word@TaoCrypt@@QEBAIXZ 000000014009f5e0 f i taocrypt:integer.obj
 0001:0009e5f0       ?GetHighHalf@Word@TaoCrypt@@QEBAIXZ 000000014009f5f0 f i taocrypt:integer.obj
 0001:0009e600       ?GetHighHalfAsBorrow@Word@TaoCrypt@@QEBAIXZ 000000014009f600 f i taocrypt:integer.obj
 0001:0009e7c0       ?MultiplyRecursionLimit@Portable@TaoCrypt@@SAIXZ 000000014009f7c0 f i taocrypt:integer.obj
 0001:0009e7d0       ?MultiplyBottomRecursionLimit@Portable@TaoCrypt@@SAIXZ 000000014009f7d0 f i taocrypt:integer.obj
 0001:0009e7e0       ?SquareRecursionLimit@Portable@TaoCrypt@@SAIXZ 000000014009f7e0 f i taocrypt:integer.obj
 0001:0009e7f0       ?Add@Portable@TaoCrypt@@SA_KPEA_KPEB_K1I@Z 000000014009f7f0 f   taocrypt:integer.obj
 0001:0009e8e0       ?Subtract@Portable@TaoCrypt@@SA_KPEA_KPEB_K1I@Z 000000014009f8e0 f   taocrypt:integer.obj
 0001:0009e9e0       ?Multiply2@Portable@TaoCrypt@@SAXPEA_KPEB_K1@Z 000000014009f9e0 f   taocrypt:integer.obj
 0001:0009eb20       ?Multiply2Bottom@Portable@TaoCrypt@@SAXPEA_KPEB_K1@Z 000000014009fb20 f   taocrypt:integer.obj
 0001:0009eb50       ?Multiply2Add@Portable@TaoCrypt@@SA_KPEA_KPEB_K1@Z 000000014009fb50 f   taocrypt:integer.obj
 0001:0009ecf0       ?Add@TaoCrypt@@YA_KPEA_KPEB_K1I@Z 000000014009fcf0 f i taocrypt:integer.obj
 0001:0009ed00       ?Subtract@TaoCrypt@@YA_KPEA_KPEB_K1I@Z 000000014009fd00 f i taocrypt:integer.obj
 0001:0009ed40       ?DivideByPower2Mod@TaoCrypt@@YAXPEA_KPEB_KI1I@Z 000000014009fd40 f   taocrypt:integer.obj
 0001:0009ee40       ?MultiplyByPower2Mod@TaoCrypt@@YAXPEA_KPEB_KI1I@Z 000000014009fe40 f   taocrypt:integer.obj
 0001:0009ef00       ??A?$Block@_KV?$AllocatorWithCleanup@_K@TaoCrypt@@@TaoCrypt@@QEAAAEA_KI@Z 000000014009ff00 f i taocrypt:integer.obj
 0001:0009ef10       ??A?$Block@_KV?$AllocatorWithCleanup@_K@TaoCrypt@@@TaoCrypt@@QEBAAEB_KI@Z 000000014009ff10 f i taocrypt:integer.obj
 0001:0009ef20       ??H?$Block@_KV?$AllocatorWithCleanup@_K@TaoCrypt@@@TaoCrypt@@QEAAPEA_KI@Z 000000014009ff20 f i taocrypt:integer.obj
 0001:0009ef30       ??H?$Block@_KV?$AllocatorWithCleanup@_K@TaoCrypt@@@TaoCrypt@@QEBAPEB_KI@Z 000000014009ff30 f i taocrypt:integer.obj
 0001:0009ef40       ?size@?$Block@_KV?$AllocatorWithCleanup@_K@TaoCrypt@@@TaoCrypt@@QEBAIXZ 000000014009ff40 f i taocrypt:integer.obj
 0001:0009ef50       ?get_buffer@?$Block@_KV?$AllocatorWithCleanup@_K@TaoCrypt@@@TaoCrypt@@QEBAPEA_KXZ 000000014009ff50 f i taocrypt:integer.obj
 0001:0009ef60       ?begin@?$Block@_KV?$AllocatorWithCleanup@_K@TaoCrypt@@@TaoCrypt@@QEBAPEA_KXZ 000000014009ff60 f i taocrypt:integer.obj
 0001:0009ef70       ?max_size@?$AllocatorBase@_K@TaoCrypt@@QEBA_KXZ 000000014009ff70 f i taocrypt:integer.obj
 0001:0009ef80       ??$swap@PEB_K@mySTL@@YAXAEAPEB_K0@Z 000000014009ff80 f i taocrypt:integer.obj
 0001:0009ef90       ??$swap@PEA_K@mySTL@@YAXAEAPEA_K0@Z 000000014009ff90 f i taocrypt:integer.obj
 0001:0009efa0       ??$max@I@TaoCrypt@@YAAEBIAEBI0@Z 000000014009ffa0 f i taocrypt:integer.obj
 0001:0009efb0       ??$swap@W4Sign@Integer@TaoCrypt@@@mySTL@@YAXAEAW4Sign@Integer@TaoCrypt@@0@Z 000000014009ffb0 f i taocrypt:integer.obj
 0001:0009efc0       ??$swap@V?$AllocatorWithCleanup@_K@TaoCrypt@@@mySTL@@YAXAEAV?$AllocatorWithCleanup@_K@TaoCrypt@@0@Z 000000014009ffc0 f i taocrypt:integer.obj
 0001:0009efd0       ??$DivideThreeWordsByTwo@IVWord@TaoCrypt@@@TaoCrypt@@YAIPEAIIIPEAVWord@0@@Z 000000014009ffd0 f i taocrypt:integer.obj
 0001:0009f0b0       ??$RightShift@K@?$SafeShifter@$00@TaoCrypt@@SAKKI@Z 00000001400a00b0 f i taocrypt:integer.obj
 0001:0009f0c0       ??$LeftShift@K@?$SafeShifter@$00@TaoCrypt@@SAKKI@Z 00000001400a00c0 f i taocrypt:integer.obj
 0001:0009f0d0       ?ShiftWordsLeftByWords@TaoCrypt@@YAXPEA_KII@Z 00000001400a00d0 f i taocrypt:integer.obj
 0001:0009f150       ?ShiftWordsRightByWords@TaoCrypt@@YAXPEA_KII@Z 00000001400a0150 f i taocrypt:integer.obj
 0001:0009f1d0       ?prev@Source@TaoCrypt@@QEAAEXZ 00000001400a01d0 f i taocrypt:integer.obj
 0001:0009f1f0       ??0AbstractRing@TaoCrypt@@QEAA@XZ 00000001400a01f0 f i taocrypt:integer.obj
 0001:0009f210       ?MultiplyAndAdd@DWord@TaoCrypt@@SA?AV12@_K00@Z 00000001400a0210 f i taocrypt:integer.obj
 0001:0009f2a0       ?Multiply4@Portable@TaoCrypt@@SAXPEA_KPEB_K1@Z 00000001400a02a0 f   taocrypt:integer.obj
 0001:0009f4f0       ?Square2@Portable@TaoCrypt@@SAXPEA_KPEB_K@Z 00000001400a04f0 f   taocrypt:integer.obj
 0001:0009f570       ?Square4@Portable@TaoCrypt@@SAXPEA_KPEB_K@Z 00000001400a0570 f   taocrypt:integer.obj
 0001:0009f580       ?Multiply8@Portable@TaoCrypt@@SAXPEA_KPEB_K1@Z 00000001400a0580 f   taocrypt:integer.obj
 0001:0009fe60       ?Multiply4Bottom@Portable@TaoCrypt@@SAXPEA_KPEB_K1@Z 00000001400a0e60 f   taocrypt:integer.obj
 0001:0009ff30       ?Multiply8Bottom@Portable@TaoCrypt@@SAXPEA_KPEB_K1@Z 00000001400a0f30 f   taocrypt:integer.obj
 0001:000a0350       ?RecursiveMultiply@TaoCrypt@@YAXPEA_K0PEB_K1I@Z 00000001400a1350 f   taocrypt:integer.obj
 0001:000a0690       ?RecursiveSquare@TaoCrypt@@YAXPEA_K0PEB_KI@Z 00000001400a1690 f   taocrypt:integer.obj
 0001:000a07c0       ?RecursiveMultiplyBottom@TaoCrypt@@YAXPEA_K0PEB_K1I@Z 00000001400a17c0 f   taocrypt:integer.obj
 0001:000a08c0       ?RecursiveMultiplyTop@TaoCrypt@@YAXPEA_K0PEB_K11I@Z 00000001400a18c0 f   taocrypt:integer.obj
 0001:000a0c60       ?Multiply@TaoCrypt@@YAXPEA_K0PEB_K1I@Z 00000001400a1c60 f i taocrypt:integer.obj
 0001:000a0c80       ?Square@TaoCrypt@@YAXPEA_K0PEB_KI@Z 00000001400a1c80 f i taocrypt:integer.obj
 0001:000a0c90       ?AsymmetricMultiply@TaoCrypt@@YAXPEA_K0PEB_KI1I@Z 00000001400a1c90 f   taocrypt:integer.obj
 0001:000a0ee0       ?AlmostInverse@TaoCrypt@@YAIPEA_K0PEB_KI1I@Z 00000001400a1ee0 f   taocrypt:integer.obj
 0001:000a13b0       ?GetBit@Integer@TaoCrypt@@QEBA_NI@Z 00000001400a23b0 f   taocrypt:integer.obj
 0001:000a13e0       ?GetBits@Integer@TaoCrypt@@QEBAKII@Z 00000001400a23e0 f   taocrypt:integer.obj
 0001:000a1440       ?GetByte@Integer@TaoCrypt@@QEBAEI@Z 00000001400a2440 f   taocrypt:integer.obj
 0001:000a1470       ?WordCount@Integer@TaoCrypt@@QEBAIXZ 00000001400a2470 f   taocrypt:integer.obj
 0001:000a1640       ?IsUnit@Integer@TaoCrypt@@QEBA_NXZ 00000001400a2640 f   taocrypt:integer.obj
 0001:000a1670       ?MultiplyBottom@TaoCrypt@@YAXPEA_K0PEB_K1I@Z 00000001400a2670 f i taocrypt:integer.obj
 0001:000a1690       ?MultiplyTop@TaoCrypt@@YAXPEA_K0PEB_K11I@Z 00000001400a2690 f i taocrypt:integer.obj
 0001:000a16b0       ?MontgomeryReduce@TaoCrypt@@YAXPEA_K0PEB_K11I@Z 00000001400a26b0 f   taocrypt:integer.obj
 0001:000a1790       ?RecursiveInverseModPower2@TaoCrypt@@YAXPEA_K0PEB_KI@Z 00000001400a2790 f   taocrypt:integer.obj
 0001:000a18c0       ?Multiply@MontgomeryRepresentation@TaoCrypt@@UEBAAEBVInteger@2@AEBV32@0@Z 00000001400a28c0 f   taocrypt:integer.obj
 0001:000a1990       ?Square@MontgomeryRepresentation@TaoCrypt@@UEBAAEBVInteger@2@AEBV32@@Z 00000001400a2990 f   taocrypt:integer.obj
 0001:000a1a40       ?MultiplicativeInverse@MontgomeryRepresentation@TaoCrypt@@UEBAAEBVInteger@2@AEBV32@@Z 00000001400a2a40 f   taocrypt:integer.obj
 0001:000a1b60       ?Swap@?$Block@_KV?$AllocatorWithCleanup@_K@TaoCrypt@@@TaoCrypt@@QEAAXAEAV12@@Z 00000001400a2b60 f i taocrypt:integer.obj
 0001:000a1b80       ?allocate@?$AllocatorWithCleanup@_K@TaoCrypt@@QEAAPEA_K_KPEBX@Z 00000001400a2b80 f i taocrypt:integer.obj
 0001:000a1bc0       ??$DivideFourWordsByTwo@IVWord@TaoCrypt@@@TaoCrypt@@YA?AVWord@0@PEAIAEBV10@11@Z 00000001400a2bc0 f i taocrypt:integer.obj
 0001:000a1c80       ??$SafeRightShift@$0EA@K@TaoCrypt@@YAKK@Z 00000001400a2c80 f i taocrypt:integer.obj
 0001:000a1c90       ??$SafeLeftShift@$0EA@K@TaoCrypt@@YAKK@Z 00000001400a2c90 f i taocrypt:integer.obj
 0001:000a1ca0       ??$StdReallocate@_KV?$AllocatorWithCleanup@_K@TaoCrypt@@@TaoCrypt@@YAPEA_KAEAV?$AllocatorWithCleanup@_K@0@PEA_K_K2_N@Z 00000001400a2ca0 f i taocrypt:integer.obj
 0001:000a1dd0       ?IsEven@Integer@TaoCrypt@@QEBA_NXZ 00000001400a2dd0 f i taocrypt:integer.obj
 0001:000a1df0       ?IsOdd@Integer@TaoCrypt@@QEBA_NXZ 00000001400a2df0 f i taocrypt:integer.obj
 0001:000a1e10       ??KDWord@TaoCrypt@@QEAA_K_K@Z 00000001400a2e10 f i taocrypt:integer.obj
 0001:000a1eb0       ??LDWord@TaoCrypt@@QEAA_K_K@Z 00000001400a2eb0 f i taocrypt:integer.obj
 0001:000a1f70       ??7Integer@TaoCrypt@@QEBA_NXZ 00000001400a2f70 f   taocrypt:integer.obj
 0001:000a1fa0       ?PositiveSubtract@TaoCrypt@@YAXAEAVInteger@1@AEBV21@1@Z 00000001400a2fa0 f   taocrypt:integer.obj
 0001:000a2120       ?PositiveCompare@Integer@TaoCrypt@@AEBAHAEBV12@@Z 00000001400a3120 f   taocrypt:integer.obj
 0001:000a2170       ?BitCount@Integer@TaoCrypt@@QEBAIXZ 00000001400a3170 f   taocrypt:integer.obj
 0001:000a21b0       ?ByteCount@Integer@TaoCrypt@@QEBAIXZ 00000001400a31b0 f   taocrypt:integer.obj
 0001:000a21f0       ?IsConvertableToLong@Integer@TaoCrypt@@QEBA_NXZ 00000001400a31f0 f   taocrypt:integer.obj
 0001:000a2240       ?ConvertToLong@Integer@TaoCrypt@@QEBAJXZ 00000001400a3240 f   taocrypt:integer.obj
 0001:000a2260       ?Swap@Integer@TaoCrypt@@QEAAXAEAV12@@Z 00000001400a3260 f   taocrypt:integer.obj
 0001:000a2290       ?Modulo@Integer@TaoCrypt@@QEBA_K_K@Z 00000001400a3290 f   taocrypt:integer.obj
 0001:000a24c0       ?Inverse@ModularArithmetic@TaoCrypt@@UEBAAEBVInteger@2@AEBV32@@Z 00000001400a34c0 f   taocrypt:integer.obj
 0001:000a2560       ?reallocate@?$AllocatorWithCleanup@_K@TaoCrypt@@QEAAPEA_KPEA_K_K1_N@Z 00000001400a3560 f i taocrypt:integer.obj
 0001:000a2580       ??$DivideThreeWordsByTwo@_KVDWord@TaoCrypt@@@TaoCrypt@@YA_KPEA_K_K1PEAVDWord@0@@Z 00000001400a3580 f i taocrypt:integer.obj
 0001:000a2720       ?IsZero@Integer@TaoCrypt@@QEBA_NXZ 00000001400a3720 f i taocrypt:integer.obj
 0001:000a2730       ?NotZero@Integer@TaoCrypt@@QEBA_NXZ 00000001400a3730 f i taocrypt:integer.obj
 0001:000a2750       ?IsPositive@Integer@TaoCrypt@@QEBA_NXZ 00000001400a3750 f i taocrypt:integer.obj
 0001:000a2780       ??LTaoCrypt@@YA_KAEBVInteger@0@_K@Z 00000001400a3780 f i taocrypt:integer.obj
 0001:000a2790       ?ScalarMultiply@MultiplicativeGroupT@AbstractRing@TaoCrypt@@UEBA?AVInteger@3@AEBV43@0@Z 00000001400a3790 f i taocrypt:integer.obj
 0001:000a27b0       ?CascadeScalarMultiply@MultiplicativeGroupT@AbstractRing@TaoCrypt@@UEBA?AVInteger@3@AEBV43@000@Z 00000001400a37b0 f i taocrypt:integer.obj
 0001:000a27f0       ??1AbstractEuclideanDomain@TaoCrypt@@UEAA@XZ 00000001400a37f0 f i taocrypt:integer.obj
 0001:000a2820       ??1EuclideanDomainOf@TaoCrypt@@UEAA@XZ 00000001400a3820 f i taocrypt:integer.obj
 0001:000a2880       ??1ModularArithmetic@TaoCrypt@@UEAA@XZ 00000001400a3880 f i taocrypt:integer.obj
 0001:000a2900       ?CascadeExponentiate@MontgomeryRepresentation@TaoCrypt@@UEBA?AVInteger@2@AEBV32@000@Z 00000001400a3900 f i taocrypt:integer.obj
 0001:000a2930       ?Negate@Integer@TaoCrypt@@QEAAXXZ 00000001400a3930 f   taocrypt:integer.obj
 0001:000a2960       ?Compare@Integer@TaoCrypt@@QEBAHAEBV12@@Z 00000001400a3960 f   taocrypt:integer.obj
 0001:000a29a0       ?InverseMod@Integer@TaoCrypt@@QEBA_K_K@Z 00000001400a39a0 f   taocrypt:integer.obj
 0001:000a2a30       ??1MontgomeryRepresentation@TaoCrypt@@UEAA@XZ 00000001400a3a30 f i taocrypt:integer.obj
 0001:000a2af0       ?CleanGrow@?$Block@_KV?$AllocatorWithCleanup@_K@TaoCrypt@@@TaoCrypt@@QEAAXI@Z 00000001400a3af0 f i taocrypt:integer.obj
 0001:000a2b50       ?New@?$Block@_KV?$AllocatorWithCleanup@_K@TaoCrypt@@@TaoCrypt@@QEAAXI@Z 00000001400a3b50 f i taocrypt:integer.obj
 0001:000a2b90       ?resize@?$Block@_KV?$AllocatorWithCleanup@_K@TaoCrypt@@@TaoCrypt@@QEAAXI@Z 00000001400a3b90 f i taocrypt:integer.obj
 0001:000a2bd0       ??$DivideFourWordsByTwo@_KVDWord@TaoCrypt@@@TaoCrypt@@YA?AVDWord@0@PEA_KAEBV10@11@Z 00000001400a3bd0 f i taocrypt:integer.obj
 0001:000a2c80       ??_GInteger@TaoCrypt@@QEAAPEAXI@Z 00000001400a3c80 f i taocrypt:integer.obj
 0001:000a2ce0       ??8TaoCrypt@@YA_NAEBVInteger@0@0@Z 00000001400a3ce0 f i taocrypt:integer.obj
 0001:000a2d00       ??OTaoCrypt@@YA_NAEBVInteger@0@0@Z 00000001400a3d00 f i taocrypt:integer.obj
 0001:000a2d20       ??PTaoCrypt@@YA_NAEBVInteger@0@0@Z 00000001400a3d20 f i taocrypt:integer.obj
 0001:000a2d40       ??MTaoCrypt@@YA_NAEBVInteger@0@0@Z 00000001400a3d40 f i taocrypt:integer.obj
 0001:000a2d60       ?SetBit@Integer@TaoCrypt@@QEAAXI_N@Z 00000001400a3d60 f   taocrypt:integer.obj
 0001:000a2e80       ?SetByte@Integer@TaoCrypt@@QEAAXIE@Z 00000001400a3e80 f   taocrypt:integer.obj
 0001:000a2f70       ??4Integer@TaoCrypt@@QEAAAEAV01@AEBV01@@Z 00000001400a3f70 f   taocrypt:integer.obj
 0001:000a3050       ??_3Integer@TaoCrypt@@QEAAAEAV01@I@Z 00000001400a4050 f   taocrypt:integer.obj
 0001:000a31f0       ?PositiveAdd@TaoCrypt@@YAXAEAVInteger@1@AEBV21@1@Z 00000001400a41f0 f   taocrypt:integer.obj
 0001:000a3400       ?Divide@TaoCrypt@@YAXPEA_K00PEB_KI1I@Z 00000001400a4400 f   taocrypt:integer.obj
 0001:000a3820       ?CleanNew@?$Block@_KV?$AllocatorWithCleanup@_K@TaoCrypt@@@TaoCrypt@@QEAAXI@Z 00000001400a4820 f i taocrypt:integer.obj
 0001:000a3880       ??$tcDelete@VInteger@TaoCrypt@@@TaoCrypt@@YAXPEAVInteger@0@@Z 00000001400a4880 f i taocrypt:integer.obj
 0001:000a38d0       ?Accumulate@MultiplicativeGroupT@AbstractRing@TaoCrypt@@UEBAAEAVInteger@3@AEAV43@AEBV43@@Z 00000001400a48d0 f i taocrypt:integer.obj
 0001:000a3900       ?Reduce@MultiplicativeGroupT@AbstractRing@TaoCrypt@@UEBAAEAVInteger@3@AEAV43@AEBV43@@Z 00000001400a4900 f i taocrypt:integer.obj
 0001:000a3930       ?Decode@Integer@TaoCrypt@@QEAAXAEAVSource@2@@Z 00000001400a4930 f   taocrypt:integer.obj
 0001:000a3a90       ?Decode@Integer@TaoCrypt@@QEAAXPEBEIW4Signedness@12@@Z 00000001400a4a90 f   taocrypt:integer.obj
 0001:000a3c20       ?CleanUp@TaoCrypt@@YAXXZ   00000001400a4c20 f   taocrypt:integer.obj
 0001:000a3c60       ?Randomize@Integer@TaoCrypt@@QEAAXAEAVRandomNumberGenerator@2@I@Z 00000001400a4c60 f   taocrypt:integer.obj
 0001:000a3d30       ??YInteger@TaoCrypt@@QEAAAEAV01@AEBV01@@Z 00000001400a4d30 f   taocrypt:integer.obj
 0001:000a3e00       ??ZInteger@TaoCrypt@@QEAAAEAV01@AEBV01@@Z 00000001400a4e00 f   taocrypt:integer.obj
 0001:000a3ed0       ?Accumulate@ModularArithmetic@TaoCrypt@@UEBAAEAVInteger@2@AEAV32@AEBV32@@Z 00000001400a4ed0 f   taocrypt:integer.obj
 0001:000a3f80       ?Reduce@ModularArithmetic@TaoCrypt@@UEBAAEAVInteger@2@AEAV32@AEBV32@@Z 00000001400a4f80 f   taocrypt:integer.obj
 0001:000a4010       ??0?$Block@_KV?$AllocatorWithCleanup@_K@TaoCrypt@@@TaoCrypt@@QEAA@I@Z 00000001400a5010 f i taocrypt:integer.obj
 0001:000a40b0       ?PositiveMultiply@TaoCrypt@@YAXAEAVInteger@1@AEBV21@1@Z 00000001400a50b0 f   taocrypt:integer.obj
 0001:000a42a0       ?Multiply@TaoCrypt@@YAXAEAVInteger@1@AEBV21@1@Z 00000001400a52a0 f   taocrypt:integer.obj
 0001:000a42f0       ??0Integer@TaoCrypt@@QEAA@XZ 00000001400a52f0 f   taocrypt:integer.obj
 0001:000a4390       ??0Integer@TaoCrypt@@QEAA@AEBV01@@Z 00000001400a5390 f   taocrypt:integer.obj
 0001:000a44c0       ??0Integer@TaoCrypt@@QEAA@J@Z 00000001400a54c0 f   taocrypt:integer.obj
 0001:000a4570       ??0Integer@TaoCrypt@@QEAA@W4Sign@01@_K1@Z 00000001400a5570 f   taocrypt:integer.obj
 0001:000a4630       ??0Integer@TaoCrypt@@AEAA@_KI@Z 00000001400a5630 f   taocrypt:integer.obj
 0001:000a4760       ??0Integer@TaoCrypt@@QEAA@PEBEIW4Signedness@01@@Z 00000001400a5760 f   taocrypt:integer.obj
 0001:000a47e0       ??0Integer@TaoCrypt@@QEAA@AEAVSource@1@@Z 00000001400a57e0 f   taocrypt:integer.obj
 0001:000a4880       ?Zero@Integer@TaoCrypt@@SAAEBV12@XZ 00000001400a5880 f   taocrypt:integer.obj
 0001:000a48d0       ?One@Integer@TaoCrypt@@SAAEBV12@XZ 00000001400a58d0 f   taocrypt:integer.obj
 0001:000a4920       ?Power2@Integer@TaoCrypt@@SA?AV12@I@Z 00000001400a5920 f   taocrypt:integer.obj
 0001:000a4960       ??GInteger@TaoCrypt@@QEBA?AV01@XZ 00000001400a5960 f   taocrypt:integer.obj
 0001:000a4990       ??EInteger@TaoCrypt@@QEAAAEAV01@XZ 00000001400a5990 f   taocrypt:integer.obj
 0001:000a4a60       ??FInteger@TaoCrypt@@QEAAAEAV01@XZ 00000001400a5a60 f   taocrypt:integer.obj
 0001:000a4b40       ??_2Integer@TaoCrypt@@QEAAAEAV01@I@Z 00000001400a5b40 f   taocrypt:integer.obj
 0001:000a4c50       ?MinEncodedSize@Integer@TaoCrypt@@QEBAIW4Signedness@12@@Z 00000001400a5c50 f   taocrypt:integer.obj
 0001:000a4d70       ?Plus@Integer@TaoCrypt@@QEBA?AV12@AEBV12@@Z 00000001400a5d70 f   taocrypt:integer.obj
 0001:000a4e30       ?Minus@Integer@TaoCrypt@@QEBA?AV12@AEBV12@@Z 00000001400a5e30 f   taocrypt:integer.obj
 0001:000a4ef0       ?Times@Integer@TaoCrypt@@QEBA?AV12@AEBV12@@Z 00000001400a5ef0 f   taocrypt:integer.obj
 0001:000a4f40       ?PositiveDivide@TaoCrypt@@YAXAEAVInteger@1@0AEBV21@1@Z 00000001400a5f40 f   taocrypt:integer.obj
 0001:000a51a0       ?AbsoluteValue@Integer@TaoCrypt@@QEBA?AV12@XZ 00000001400a61a0 f   taocrypt:integer.obj
 0001:000a51d0       ?MultiplicativeInverse@Integer@TaoCrypt@@QEBA?AV12@XZ 00000001400a61d0 f   taocrypt:integer.obj
 0001:000a5210       ?ConvertOut@MontgomeryRepresentation@TaoCrypt@@UEBA?AVInteger@2@AEBV32@@Z 00000001400a6210 f   taocrypt:integer.obj
 0001:000a52d0       ??5Integer@TaoCrypt@@QEBA?AV01@I@Z 00000001400a62d0 f i taocrypt:integer.obj
 0001:000a5330       ??6Integer@TaoCrypt@@QEBA?AV01@I@Z 00000001400a6330 f i taocrypt:integer.obj
 0001:000a5390       ?Squared@Integer@TaoCrypt@@QEBA?AV12@XZ 00000001400a6390 f i taocrypt:integer.obj
 0001:000a53b0       ??HTaoCrypt@@YA?AVInteger@0@AEBV10@0@Z 00000001400a63b0 f i taocrypt:integer.obj
 0001:000a53d0       ??GTaoCrypt@@YA?AVInteger@0@AEBV10@0@Z 00000001400a63d0 f i taocrypt:integer.obj
 0001:000a53f0       ??DTaoCrypt@@YA?AVInteger@0@AEBV10@0@Z 00000001400a63f0 f i taocrypt:integer.obj
 0001:000a5410       ??0AbstractEuclideanDomain@TaoCrypt@@QEAA@XZ 00000001400a6410 f i taocrypt:integer.obj
 0001:000a5440       ??0ModularArithmetic@TaoCrypt@@QEAA@AEBVInteger@1@@Z 00000001400a6440 f i taocrypt:integer.obj
 0001:000a54a0       ?MultiplicativeGroup@AbstractRing@TaoCrypt@@UEBAAEBVAbstractGroup@2@XZ 00000001400a64a0 f i taocrypt:integer.obj
 0001:000a54b0       ?IsMontgomeryRepresentation@ModularArithmetic@TaoCrypt@@UEBA_NXZ 00000001400a64b0 f i taocrypt:integer.obj
 0001:000a54c0       ?Double@ModularArithmetic@TaoCrypt@@UEBAAEBVInteger@2@AEBV32@@Z 00000001400a64c0 f i taocrypt:integer.obj
 0001:000a54d0       ?Divide@ModularArithmetic@TaoCrypt@@UEBAAEBVInteger@2@AEBV32@0@Z 00000001400a64d0 f i taocrypt:integer.obj
 0001:000a5510       ?Equal@ModularArithmetic@TaoCrypt@@UEBA_NAEBVInteger@2@0@Z 00000001400a6510 f i taocrypt:integer.obj
 0001:000a5530       ??_GModularArithmetic@TaoCrypt@@UEAAPEAXI@Z 00000001400a6530 f i taocrypt:integer.obj
 0001:000a5530       ??_EModularArithmetic@TaoCrypt@@UEAAPEAXI@Z 00000001400a6530 f i taocrypt:integer.obj
 0001:000a55c0       ?ConvertOut@ModularArithmetic@TaoCrypt@@UEBA?AVInteger@2@AEBV32@@Z 00000001400a65c0 f i taocrypt:integer.obj
 0001:000a55e0       ?Identity@ModularArithmetic@TaoCrypt@@UEBAAEBVInteger@2@XZ 00000001400a65e0 f i taocrypt:integer.obj
 0001:000a55f0       ?MultiplicativeIdentity@ModularArithmetic@TaoCrypt@@UEBAAEBVInteger@2@XZ 00000001400a65f0 f i taocrypt:integer.obj
 0001:000a5600       ?Encode@Integer@TaoCrypt@@QEBAIPEAEIW4Signedness@12@@Z 00000001400a6600 f   taocrypt:integer.obj
 0001:000a5730       ?Randomize@Integer@TaoCrypt@@QEAAXAEAVRandomNumberGenerator@2@AEBV12@1@Z 00000001400a6730 f   taocrypt:integer.obj
 0001:000a57d0       ?Divide@Integer@TaoCrypt@@SAXAEAV12@0AEBV12@1@Z 00000001400a67d0 f   taocrypt:integer.obj
 0001:000a58b0       ?DivideByPowerOf2@Integer@TaoCrypt@@SAXAEAV12@0AEBV12@I@Z 00000001400a68b0 f   taocrypt:integer.obj
 0001:000a5b30       ?DividedBy@Integer@TaoCrypt@@QEBA?AV12@AEBV12@@Z 00000001400a6b30 f   taocrypt:integer.obj
 0001:000a5ba0       ?Modulo@Integer@TaoCrypt@@QEBA?AV12@AEBV12@@Z 00000001400a6ba0 f   taocrypt:integer.obj
 0001:000a5c10       ?Divide@Integer@TaoCrypt@@SAXAEA_KAEAV12@AEBV12@_K@Z 00000001400a6c10 f   taocrypt:integer.obj
 0001:000a5f10       ?DividedBy@Integer@TaoCrypt@@QEBA?AV12@_K@Z 00000001400a6f10 f   taocrypt:integer.obj
 0001:000a5f60       ?a_exp_b_mod_c@TaoCrypt@@YA?AVInteger@1@AEBV21@00@Z 00000001400a6f60 f   taocrypt:integer.obj
 0001:000a6060       ?Half@ModularArithmetic@TaoCrypt@@QEBAAEBVInteger@2@AEBV32@@Z 00000001400a7060 f   taocrypt:integer.obj
 0001:000a6220       ?Add@ModularArithmetic@TaoCrypt@@UEBAAEBVInteger@2@AEBV32@0@Z 00000001400a7220 f   taocrypt:integer.obj
 0001:000a6310       ?Subtract@ModularArithmetic@TaoCrypt@@UEBAAEBVInteger@2@AEBV32@0@Z 00000001400a7310 f   taocrypt:integer.obj
 0001:000a63e0       ??0MontgomeryRepresentation@TaoCrypt@@QEAA@AEBVInteger@1@@Z 00000001400a73e0 f   taocrypt:integer.obj
 0001:000a6510       ?IsMontgomeryRepresentation@MontgomeryRepresentation@TaoCrypt@@UEBA_NXZ 00000001400a7510 f i taocrypt:integer.obj
 0001:000a6520       ??_EMontgomeryRepresentation@TaoCrypt@@UEAAPEAXI@Z 00000001400a7520 f i taocrypt:integer.obj
 0001:000a6520       ??_GMontgomeryRepresentation@TaoCrypt@@UEAAPEAXI@Z 00000001400a7520 f i taocrypt:integer.obj
 0001:000a6600       ??KTaoCrypt@@YA?AVInteger@0@AEBV10@0@Z 00000001400a7600 f i taocrypt:integer.obj
 0001:000a6620       ??LTaoCrypt@@YA?AVInteger@0@AEBV10@0@Z 00000001400a7620 f i taocrypt:integer.obj
 0001:000a6640       ?ModularExponentiation@TaoCrypt@@YA?AVInteger@1@AEBV21@00@Z 00000001400a7640 f i taocrypt:integer.obj
 0001:000a6660       ??0EuclideanDomainOf@TaoCrypt@@QEAA@XZ 00000001400a7660 f i taocrypt:integer.obj
 0001:000a66a0       ?IsUnit@EuclideanDomainOf@TaoCrypt@@UEBA_NAEBVInteger@2@@Z 00000001400a76a0 f i taocrypt:integer.obj
 0001:000a66b0       ?Equal@EuclideanDomainOf@TaoCrypt@@UEBA_NAEBVInteger@2@0@Z 00000001400a76b0 f i taocrypt:integer.obj
 0001:000a66d0       ??_GEuclideanDomainOf@TaoCrypt@@UEAAPEAXI@Z 00000001400a76d0 f i taocrypt:integer.obj
 0001:000a66d0       ??_EEuclideanDomainOf@TaoCrypt@@UEAAPEAXI@Z 00000001400a76d0 f i taocrypt:integer.obj
 0001:000a6750       ?Accumulate@EuclideanDomainOf@TaoCrypt@@UEBAAEAVInteger@2@AEAV32@AEBV32@@Z 00000001400a7750 f i taocrypt:integer.obj
 0001:000a6760       ?Reduce@EuclideanDomainOf@TaoCrypt@@UEBAAEAVInteger@2@AEAV32@AEBV32@@Z 00000001400a7760 f i taocrypt:integer.obj
 0001:000a6770       ?Doubled@Integer@TaoCrypt@@QEBA?AV12@XZ 00000001400a7770 f i taocrypt:integer.obj
 0001:000a6790       ?Identity@EuclideanDomainOf@TaoCrypt@@UEBAAEBVInteger@2@XZ 00000001400a7790 f i taocrypt:integer.obj
 0001:000a67a0       ?Add@EuclideanDomainOf@TaoCrypt@@UEBAAEBVInteger@2@AEBV32@0@Z 00000001400a77a0 f i taocrypt:integer.obj
 0001:000a6800       ?Inverse@EuclideanDomainOf@TaoCrypt@@UEBAAEBVInteger@2@AEBV32@@Z 00000001400a7800 f i taocrypt:integer.obj
 0001:000a6860       ?Subtract@EuclideanDomainOf@TaoCrypt@@UEBAAEBVInteger@2@AEBV32@0@Z 00000001400a7860 f i taocrypt:integer.obj
 0001:000a68c0       ?Double@EuclideanDomainOf@TaoCrypt@@UEBAAEBVInteger@2@AEBV32@@Z 00000001400a78c0 f i taocrypt:integer.obj
 0001:000a6920       ?MultiplicativeIdentity@EuclideanDomainOf@TaoCrypt@@UEBAAEBVInteger@2@XZ 00000001400a7920 f i taocrypt:integer.obj
 0001:000a6930       ?Multiply@EuclideanDomainOf@TaoCrypt@@UEBAAEBVInteger@2@AEBV32@0@Z 00000001400a7930 f i taocrypt:integer.obj
 0001:000a6990       ?Square@EuclideanDomainOf@TaoCrypt@@UEBAAEBVInteger@2@AEBV32@@Z 00000001400a7990 f i taocrypt:integer.obj
 0001:000a69f0       ?MultiplicativeInverse@EuclideanDomainOf@TaoCrypt@@UEBAAEBVInteger@2@AEBV32@@Z 00000001400a79f0 f i taocrypt:integer.obj
 0001:000a6a50       ?Divide@EuclideanDomainOf@TaoCrypt@@UEBAAEBVInteger@2@AEBV32@0@Z 00000001400a7a50 f i taocrypt:integer.obj
 0001:000a6ab0       ?Mod@EuclideanDomainOf@TaoCrypt@@UEBAAEBVInteger@2@AEBV32@0@Z 00000001400a7ab0 f i taocrypt:integer.obj
 0001:000a6b10       ?DivisionAlgorithm@EuclideanDomainOf@TaoCrypt@@UEBAXAEAVInteger@2@0AEBV32@1@Z 00000001400a7b10 f i taocrypt:integer.obj
 0001:000a6b30       ?ConvertIn@ModularArithmetic@TaoCrypt@@UEBA?AVInteger@2@AEBV32@@Z 00000001400a7b30 f i taocrypt:integer.obj
 0001:000a6b60       ?Multiply@ModularArithmetic@TaoCrypt@@UEBAAEBVInteger@2@AEBV32@0@Z 00000001400a7b60 f i taocrypt:integer.obj
 0001:000a6bf0       ?Square@ModularArithmetic@TaoCrypt@@UEBAAEBVInteger@2@AEBV32@@Z 00000001400a7bf0 f i taocrypt:integer.obj
 0001:000a6c90       ?ConvertIn@MontgomeryRepresentation@TaoCrypt@@UEBA?AVInteger@2@AEBV32@@Z 00000001400a7c90 f i taocrypt:integer.obj
 0001:000a6d40       ?MultiplicativeIdentity@MontgomeryRepresentation@TaoCrypt@@UEBAAEBVInteger@2@XZ 00000001400a7d40 f i taocrypt:integer.obj
 0001:000a6dd0       ??0Integer@TaoCrypt@@QEAA@AEAVRandomNumberGenerator@1@AEBV01@1@Z 00000001400a7dd0 f   taocrypt:integer.obj
 0001:000a6e50       ?SquareRoot@Integer@TaoCrypt@@QEBA?AV12@XZ 00000001400a7e50 f   taocrypt:integer.obj
 0001:000a7050       ?IsSquare@Integer@TaoCrypt@@QEBA_NXZ 00000001400a8050 f   taocrypt:integer.obj
 0001:000a70e0       ?a_times_b_mod_c@TaoCrypt@@YA?AVInteger@1@AEBV21@00@Z 00000001400a80e0 f   taocrypt:integer.obj
 0001:000a7140       ?Gcd@Integer@TaoCrypt@@SA?AV12@AEBV12@0@Z 00000001400a8140 f   taocrypt:integer.obj
 0001:000a7210       ?InverseMod@Integer@TaoCrypt@@QEBA?AV12@AEBV12@@Z 00000001400a8210 f   taocrypt:integer.obj
 0001:000a75c0       ?CascadeExponentiate@ModularArithmetic@TaoCrypt@@UEBA?AVInteger@2@AEBV32@000@Z 00000001400a85c0 f   taocrypt:integer.obj
 0001:000a78f0       ?SimultaneousExponentiate@ModularArithmetic@TaoCrypt@@UEBAXPEAVInteger@2@AEBV32@PEBV32@I@Z 00000001400a88f0 f   taocrypt:integer.obj
 0001:000a7b50       ?CRT@TaoCrypt@@YA?AVInteger@1@AEBV21@0000@Z 00000001400a8b50 f   taocrypt:integer.obj
 0001:000a7c70       ?IsUnit@ModularArithmetic@TaoCrypt@@UEBA_NAEBVInteger@2@@Z 00000001400a8c70 f i taocrypt:integer.obj
 0001:000a7cd0       ?MultiplicativeInverse@ModularArithmetic@TaoCrypt@@UEBAAEBVInteger@2@AEBV32@@Z 00000001400a8cd0 f i taocrypt:integer.obj
 0001:000a7d30       ?ModularRoot@TaoCrypt@@YA?AVInteger@1@AEBV21@00000@Z 00000001400a8d30 f   taocrypt:integer.obj
 0001:000a7e90       ??1SHA256@TaoCrypt@@UEAA@XZ 00000001400a8e90 f i taocrypt:sha.obj
 0001:000a7ea0       ??1SHA224@TaoCrypt@@UEAA@XZ 00000001400a8ea0 f i taocrypt:sha.obj
 0001:000a7eb0       ??1SHA512@TaoCrypt@@UEAA@XZ 00000001400a8eb0 f i taocrypt:sha.obj
 0001:000a7ec0       ??1SHA384@TaoCrypt@@UEAA@XZ 00000001400a8ec0 f i taocrypt:sha.obj
 0001:000a7ed0       ?Init@SHA@TaoCrypt@@UEAAXXZ 00000001400a8ed0 f   taocrypt:sha.obj
 0001:000a7f00       ?Init@SHA256@TaoCrypt@@UEAAXXZ 00000001400a8f00 f   taocrypt:sha.obj
 0001:000a7f50       ?Init@SHA224@TaoCrypt@@UEAAXXZ 00000001400a8f50 f   taocrypt:sha.obj
 0001:000a7fa0       ?Init@SHA512@TaoCrypt@@UEAAXXZ 00000001400a8fa0 f   taocrypt:sha.obj
 0001:000a8020       ?Init@SHA384@TaoCrypt@@UEAAXXZ 00000001400a9020 f   taocrypt:sha.obj
 0001:000a80a0       ??0SHA@TaoCrypt@@QEAA@AEBV01@@Z 00000001400a90a0 f   taocrypt:sha.obj
 0001:000a8120       ??0SHA256@TaoCrypt@@QEAA@AEBV01@@Z 00000001400a9120 f   taocrypt:sha.obj
 0001:000a81b0       ?getByteOrder@SHA256@TaoCrypt@@UEBA?AW4ByteOrder@2@XZ 00000001400a91b0 f i taocrypt:sha.obj
 0001:000a81c0       ?getBlockSize@SHA256@TaoCrypt@@UEBAIXZ 00000001400a91c0 f i taocrypt:sha.obj
 0001:000a81d0       ?getDigestSize@SHA256@TaoCrypt@@UEBAIXZ 00000001400a91d0 f i taocrypt:sha.obj
 0001:000a81e0       ?getPadSize@SHA256@TaoCrypt@@UEBAIXZ 00000001400a91e0 f i taocrypt:sha.obj
 0001:000a81f0       ??0SHA224@TaoCrypt@@QEAA@AEBV01@@Z 00000001400a91f0 f   taocrypt:sha.obj
 0001:000a8280       ?getByteOrder@SHA224@TaoCrypt@@UEBA?AW4ByteOrder@2@XZ 00000001400a9280 f i taocrypt:sha.obj
 0001:000a8290       ?getBlockSize@SHA224@TaoCrypt@@UEBAIXZ 00000001400a9290 f i taocrypt:sha.obj
 0001:000a82a0       ?getDigestSize@SHA224@TaoCrypt@@UEBAIXZ 00000001400a92a0 f i taocrypt:sha.obj
 0001:000a82b0       ?getPadSize@SHA224@TaoCrypt@@UEBAIXZ 00000001400a92b0 f i taocrypt:sha.obj
 0001:000a82c0       ??0SHA512@TaoCrypt@@QEAA@AEBV01@@Z 00000001400a92c0 f   taocrypt:sha.obj
 0001:000a8360       ?getByteOrder@SHA512@TaoCrypt@@UEBA?AW4ByteOrder@2@XZ 00000001400a9360 f i taocrypt:sha.obj
 0001:000a8370       ?getBlockSize@SHA512@TaoCrypt@@UEBAIXZ 00000001400a9370 f i taocrypt:sha.obj
 0001:000a8380       ?getDigestSize@SHA512@TaoCrypt@@UEBAIXZ 00000001400a9380 f i taocrypt:sha.obj
 0001:000a8390       ?getPadSize@SHA512@TaoCrypt@@UEBAIXZ 00000001400a9390 f i taocrypt:sha.obj
 0001:000a83a0       ??0SHA384@TaoCrypt@@QEAA@AEBV01@@Z 00000001400a93a0 f   taocrypt:sha.obj
 0001:000a8430       ?getByteOrder@SHA384@TaoCrypt@@UEBA?AW4ByteOrder@2@XZ 00000001400a9430 f i taocrypt:sha.obj
 0001:000a8440       ?getBlockSize@SHA384@TaoCrypt@@UEBAIXZ 00000001400a9440 f i taocrypt:sha.obj
 0001:000a8450       ?getDigestSize@SHA384@TaoCrypt@@UEBAIXZ 00000001400a9450 f i taocrypt:sha.obj
 0001:000a8460       ?getPadSize@SHA384@TaoCrypt@@UEBAIXZ 00000001400a9460 f i taocrypt:sha.obj
 0001:000a8470       ?Transform@SHA@TaoCrypt@@EEAAXXZ 00000001400a9470 f   taocrypt:sha.obj
 0001:000aa220       ?Transform@SHA256@TaoCrypt@@EEAAXXZ 00000001400ab220 f   taocrypt:sha.obj
 0001:000aa230       ?Transform@SHA224@TaoCrypt@@EEAAXXZ 00000001400ab230 f   taocrypt:sha.obj
 0001:000aa240       ??$rotrFixed@_K@TaoCrypt@@YA_K_KI@Z 00000001400ab240 f i taocrypt:sha.obj
 0001:000aa250       ??_ESHA256@TaoCrypt@@UEAAPEAXI@Z 00000001400ab250 f i taocrypt:sha.obj
 0001:000aa250       ??_GSHA256@TaoCrypt@@UEAAPEAXI@Z 00000001400ab250 f i taocrypt:sha.obj
 0001:000aa280       ??_ESHA224@TaoCrypt@@UEAAPEAXI@Z 00000001400ab280 f i taocrypt:sha.obj
 0001:000aa280       ??_GSHA224@TaoCrypt@@UEAAPEAXI@Z 00000001400ab280 f i taocrypt:sha.obj
 0001:000aa2b0       ??_GSHA512@TaoCrypt@@UEAAPEAXI@Z 00000001400ab2b0 f i taocrypt:sha.obj
 0001:000aa2b0       ??_ESHA512@TaoCrypt@@UEAAPEAXI@Z 00000001400ab2b0 f i taocrypt:sha.obj
 0001:000aa2e0       ??_ESHA384@TaoCrypt@@UEAAPEAXI@Z 00000001400ab2e0 f i taocrypt:sha.obj
 0001:000aa2e0       ??_GSHA384@TaoCrypt@@UEAAPEAXI@Z 00000001400ab2e0 f i taocrypt:sha.obj
 0001:000aa310       ?Swap@SHA@TaoCrypt@@QEAAXAEAV12@@Z 00000001400ab310 f   taocrypt:sha.obj
 0001:000aa380       ?Swap@SHA256@TaoCrypt@@QEAAXAEAV12@@Z 00000001400ab380 f   taocrypt:sha.obj
 0001:000aa400       ?Swap@SHA224@TaoCrypt@@QEAAXAEAV12@@Z 00000001400ab400 f   taocrypt:sha.obj
 0001:000aa470       ?Swap@SHA512@TaoCrypt@@QEAAXAEAV12@@Z 00000001400ab470 f   taocrypt:sha.obj
 0001:000aa4f0       ?Swap@SHA384@TaoCrypt@@QEAAXAEAV12@@Z 00000001400ab4f0 f   taocrypt:sha.obj
 0001:000ab470       ?Transform@SHA512@TaoCrypt@@EEAAXXZ 00000001400ac470 f   taocrypt:sha.obj
 0001:000ab480       ?Transform@SHA384@TaoCrypt@@EEAAXXZ 00000001400ac480 f   taocrypt:sha.obj
 0001:000ab490       ??4SHA@TaoCrypt@@QEAAAEAV01@AEBV01@@Z 00000001400ac490 f   taocrypt:sha.obj
 0001:000ab4c0       ??4SHA256@TaoCrypt@@QEAAAEAV01@AEBV01@@Z 00000001400ac4c0 f   taocrypt:sha.obj
 0001:000ab4f0       ??4SHA224@TaoCrypt@@QEAAAEAV01@AEBV01@@Z 00000001400ac4f0 f   taocrypt:sha.obj
 0001:000ab520       ??4SHA512@TaoCrypt@@QEAAAEAV01@AEBV01@@Z 00000001400ac520 f   taocrypt:sha.obj
 0001:000ab550       ??4SHA384@TaoCrypt@@QEAAAEAV01@AEBV01@@Z 00000001400ac550 f   taocrypt:sha.obj
 0001:000ab580       ?Init@RIPEMD160@TaoCrypt@@UEAAXXZ 00000001400ac580 f   taocrypt:ripemd.obj
 0001:000ab5b0       ??0RIPEMD160@TaoCrypt@@QEAA@AEBV01@@Z 00000001400ac5b0 f   taocrypt:ripemd.obj
 0001:000ab630       ?Transform@RIPEMD160@TaoCrypt@@EEAAXXZ 00000001400ac630 f   taocrypt:ripemd.obj
 0001:000acad0       ?Swap@RIPEMD160@TaoCrypt@@QEAAXAEAV12@@Z 00000001400adad0 f   taocrypt:ripemd.obj
 0001:000acb40       ??4RIPEMD160@TaoCrypt@@QEAAAEAV01@AEBV01@@Z 00000001400adb40 f   taocrypt:ripemd.obj
 0001:000acb70       ?XorWords@TaoCrypt@@YAXPEA_KPEB_KI@Z 00000001400adb70 f i taocrypt:misc.obj
 0001:000acba0       ?xorbuf@TaoCrypt@@YAXPEAEPEBEI@Z 00000001400adba0 f   taocrypt:misc.obj
 0001:000acc00       ?BytePrecision@TaoCrypt@@YAI_K@Z 00000001400adc00 f   taocrypt:misc.obj
 0001:000acc30       ?BitPrecision@TaoCrypt@@YAI_K@Z 00000001400adc30 f   taocrypt:misc.obj
 0001:000acc80       ?Crop@TaoCrypt@@YA_K_KI@Z  00000001400adc80 f   taocrypt:misc.obj
 0001:000acca0       ?ReverseDir@TaoCrypt@@YA?AW4CipherDir@1@W421@@Z 00000001400adca0 f i taocrypt:des.obj
 0001:000accb0       ?UnalignedGetWordNonTemplate@TaoCrypt@@YAIW4ByteOrder@1@PEBEPEAI@Z 00000001400adcb0 f i taocrypt:des.obj
 0001:000acd00       ?UnalignedPutWord@TaoCrypt@@YAXW4ByteOrder@1@PEAEIPEBE@Z 00000001400add00 f i taocrypt:des.obj
 0001:000acea0       ?RawProcessBlock@BasicDES@TaoCrypt@@QEBAXAEAI0@Z 00000001400adea0 f   taocrypt:des.obj
 0001:000ad020       ??0?$PutBlock@IU?$EnumToType@W4ByteOrder@TaoCrypt@@$00@TaoCrypt@@$00@TaoCrypt@@QEAA@PEBXPEAX@Z 00000001400ae020 f i taocrypt:des.obj
 0001:000ad030       ??0?$GetBlock@IU?$EnumToType@W4ByteOrder@TaoCrypt@@$00@TaoCrypt@@$00@TaoCrypt@@QEAA@PEBX@Z 00000001400ae030 f i taocrypt:des.obj
 0001:000ad040       ?ToEnum@?$EnumToType@W4ByteOrder@TaoCrypt@@$00@TaoCrypt@@SA?AW4ByteOrder@2@XZ 00000001400ae040 f i taocrypt:des.obj
 0001:000ad050       ??$UnalignedGetWord@I@TaoCrypt@@YAIW4ByteOrder@0@PEBEPEAI@Z 00000001400ae050 f i taocrypt:des.obj
 0001:000ad0a0       ?SetKey@BasicDES@TaoCrypt@@QEAAXPEBEIW4CipherDir@2@@Z 00000001400ae0a0 f   taocrypt:des.obj
 0001:000ad330       ?SetKey@DES_EDE2@TaoCrypt@@QEAAXPEBEIW4CipherDir@2@@Z 00000001400ae330 f   taocrypt:des.obj
 0001:000ad390       ?SetKey@DES_EDE3@TaoCrypt@@QEAAXPEBEIW4CipherDir@2@@Z 00000001400ae390 f   taocrypt:des.obj
 0001:000ad430       ?Get@?$BlockGetAndPut@IU?$EnumToType@W4ByteOrder@TaoCrypt@@$00@TaoCrypt@@$00@TaoCrypt@@SA?AV?$GetBlock@IU?$EnumToType@W4ByteOrder@TaoCrypt@@$00@TaoCrypt@@$00@2@PEBX@Z 00000001400ae430 f i taocrypt:des.obj
 0001:000ad440       ??$ByteReverseIf@I@TaoCrypt@@YAIIW4ByteOrder@0@@Z 00000001400ae440 f i taocrypt:des.obj
 0001:000ad460       ??$GetWord@I@TaoCrypt@@YAI_NW4ByteOrder@0@PEBE@Z 00000001400ae460 f i taocrypt:des.obj
 0001:000ad4e0       ??$PutWord@I@TaoCrypt@@YAX_NW4ByteOrder@0@PEAEIPEBE@Z 00000001400ae4e0 f i taocrypt:des.obj
 0001:000ad5a0       ??$?RI@?$GetBlock@IU?$EnumToType@W4ByteOrder@TaoCrypt@@$00@TaoCrypt@@$00@TaoCrypt@@QEAAAEAV01@AEAI@Z 00000001400ae5a0 f i taocrypt:des.obj
 0001:000ad5d0       ??$?RI@?$PutBlock@IU?$EnumToType@W4ByteOrder@TaoCrypt@@$00@TaoCrypt@@$00@TaoCrypt@@QEAAAEAV01@I@Z 00000001400ae5d0 f i taocrypt:des.obj
 0001:000ad610       ?ProcessAndXorBlock@DES@TaoCrypt@@EEBAXPEBE0PEAE@Z 00000001400ae610 f   taocrypt:des.obj
 0001:000ad7b0       ?ProcessAndXorBlock@DES_EDE2@TaoCrypt@@EEBAXPEBE0PEAE@Z 00000001400ae7b0 f   taocrypt:des.obj
 0001:000ad980       ?ProcessAndXorBlock@DES_EDE3@TaoCrypt@@EEBAXPEBE0PEAE@Z 00000001400ae980 f   taocrypt:des.obj
 0001:000adb60       ??$IsPowerOf2@I@TaoCrypt@@YA_NI@Z 00000001400aeb60 f i taocrypt:aes.obj
 0001:000adb80       ??$ModPowerOf2@II@TaoCrypt@@YAIII@Z 00000001400aeb80 f i taocrypt:aes.obj
 0001:000adb90       ??$RoundDownToMultipleOf@I@TaoCrypt@@YAIII@Z 00000001400aeb90 f i taocrypt:aes.obj
 0001:000adbc0       ??$RoundUpToMultipleOf@I@TaoCrypt@@YAIII@Z 00000001400aebc0 f i taocrypt:aes.obj
 0001:000adbf0       ??$GetUserKey@I@TaoCrypt@@YAXW4ByteOrder@0@PEAIIPEBEI@Z 00000001400aebf0 f i taocrypt:aes.obj
 0001:000adca0       ?SetKey@AES@TaoCrypt@@QEAAXPEBEIW4CipherDir@2@@Z 00000001400aeca0 f   taocrypt:aes.obj
 0001:000ae3e0       ?encrypt@AES@TaoCrypt@@AEBAXPEBE0PEAE@Z 00000001400af3e0 f   taocrypt:aes.obj
 0001:000ae990       ?decrypt@AES@TaoCrypt@@AEBAXPEBE0PEAE@Z 00000001400af990 f   taocrypt:aes.obj
 0001:000aef40       ?ProcessAndXorBlock@AES@TaoCrypt@@EEBAXPEBE0PEAE@Z 00000001400aff40 f   taocrypt:aes.obj
 0001:000aef50       ?GenerateBlock@RandomNumberGenerator@TaoCrypt@@QEAAXPEAEI@Z 00000001400aff50 f   taocrypt:random.obj
 0001:000aefa0       ?GenerateByte@RandomNumberGenerator@TaoCrypt@@QEAAEXZ 00000001400affa0 f   taocrypt:random.obj
 0001:000aefc0       ??0OS_Seed@TaoCrypt@@QEAA@XZ 00000001400affc0 f   taocrypt:random.obj
 0001:000af000       ??1OS_Seed@TaoCrypt@@QEAA@XZ 00000001400b0000 f   taocrypt:random.obj
 0001:000af010       ?GenerateSeed@OS_Seed@TaoCrypt@@QEAAXPEAEI@Z 00000001400b0010 f   taocrypt:random.obj
 0001:000af040       ??0RandomNumberGenerator@TaoCrypt@@QEAA@XZ 00000001400b0040 f   taocrypt:random.obj
 0001:000af0c0       ?SetKey@ARC4@TaoCrypt@@QEAAXPEBEI@Z 00000001400b00c0 f   taocrypt:arc4.obj
 0001:000af160       ?MakeByte@?A0x45194f11@TaoCrypt@@YAIAEAI0PEAE@Z 00000001400b0160 f i taocrypt:arc4.obj
 0001:000af1a0       ?Process@ARC4@TaoCrypt@@QEAAXPEAEPEBEI@Z 00000001400b01a0 f   taocrypt:arc4.obj
 0001:000af280       ??0BER_Decoder@TaoCrypt@@QEAA@AEAVSource@1@@Z 00000001400b0280 f i taocrypt:dsa.obj
 0001:000af2a0       ??1BER_Decoder@TaoCrypt@@UEAA@XZ 00000001400b02a0 f i taocrypt:dsa.obj
 0001:000af2b0       ??_EBER_Decoder@TaoCrypt@@UEAAPEAXI@Z 00000001400b02b0 f i taocrypt:dsa.obj
 0001:000af2b0       ??_GBER_Decoder@TaoCrypt@@UEAAPEAXI@Z 00000001400b02b0 f i taocrypt:dsa.obj
 0001:000af2e0       ??0DSA_Private_Decoder@TaoCrypt@@QEAA@AEAVSource@1@@Z 00000001400b02e0 f i taocrypt:dsa.obj
 0001:000af300       ??1DSA_Private_Decoder@TaoCrypt@@UEAA@XZ 00000001400b0300 f i taocrypt:dsa.obj
 0001:000af310       ??0DSA_Public_Decoder@TaoCrypt@@QEAA@AEAVSource@1@@Z 00000001400b0310 f i taocrypt:dsa.obj
 0001:000af330       ??1DSA_Public_Decoder@TaoCrypt@@UEAA@XZ 00000001400b0330 f i taocrypt:dsa.obj
 0001:000af340       ?Swap@DSA_PublicKey@TaoCrypt@@QEAAXAEAV12@@Z 00000001400b0340 f   taocrypt:dsa.obj
 0001:000af390       ?Initialize@DSA_PublicKey@TaoCrypt@@QEAAXAEAVSource@2@@Z 00000001400b0390 f   taocrypt:dsa.obj
 0001:000af3c0       ?Initialize@DSA_PublicKey@TaoCrypt@@QEAAXAEBVInteger@2@000@Z 00000001400b03c0 f   taocrypt:dsa.obj
 0001:000af420       ?GetModulus@DSA_PublicKey@TaoCrypt@@QEBAAEBVInteger@2@XZ 00000001400b0420 f   taocrypt:dsa.obj
 0001:000af430       ?GetSubGroupOrder@DSA_PublicKey@TaoCrypt@@QEBAAEBVInteger@2@XZ 00000001400b0430 f   taocrypt:dsa.obj
 0001:000af440       ?GetSubGroupGenerator@DSA_PublicKey@TaoCrypt@@QEBAAEBVInteger@2@XZ 00000001400b0440 f   taocrypt:dsa.obj
 0001:000af450       ?GetPublicPart@DSA_PublicKey@TaoCrypt@@QEBAAEBVInteger@2@XZ 00000001400b0450 f   taocrypt:dsa.obj
 0001:000af460       ?SetModulus@DSA_PublicKey@TaoCrypt@@QEAAXAEBVInteger@2@@Z 00000001400b0460 f   taocrypt:dsa.obj
 0001:000af470       ?SetSubGroupOrder@DSA_PublicKey@TaoCrypt@@QEAAXAEBVInteger@2@@Z 00000001400b0470 f   taocrypt:dsa.obj
 0001:000af480       ?SetSubGroupGenerator@DSA_PublicKey@TaoCrypt@@QEAAXAEBVInteger@2@@Z 00000001400b0480 f   taocrypt:dsa.obj
 0001:000af490       ?SetPublicPart@DSA_PublicKey@TaoCrypt@@QEAAXAEBVInteger@2@@Z 00000001400b0490 f   taocrypt:dsa.obj
 0001:000af4a0       ?SignatureLength@DSA_PublicKey@TaoCrypt@@QEBAIXZ 00000001400b04a0 f   taocrypt:dsa.obj
 0001:000af4c0       ?Initialize@DSA_PrivateKey@TaoCrypt@@QEAAXAEAVSource@2@@Z 00000001400b04c0 f   taocrypt:dsa.obj
 0001:000af4f0       ?Initialize@DSA_PrivateKey@TaoCrypt@@QEAAXAEBVInteger@2@0000@Z 00000001400b04f0 f   taocrypt:dsa.obj
 0001:000af520       ?GetPrivatePart@DSA_PrivateKey@TaoCrypt@@QEBAAEBVInteger@2@XZ 00000001400b0520 f   taocrypt:dsa.obj
 0001:000af530       ?SetPrivatePart@DSA_PrivateKey@TaoCrypt@@QEAAXAEBVInteger@2@@Z 00000001400b0530 f   taocrypt:dsa.obj
 0001:000af540       ?GetR@DSA_Signer@TaoCrypt@@QEBAAEBVInteger@2@XZ 00000001400b0540 f   taocrypt:dsa.obj
 0001:000af550       ?GetS@DSA_Signer@TaoCrypt@@QEBAAEBVInteger@2@XZ 00000001400b0550 f   taocrypt:dsa.obj
 0001:000af560       ?GetR@DSA_Verifier@TaoCrypt@@QEBAAEBVInteger@2@XZ 00000001400b0560 f   taocrypt:dsa.obj
 0001:000af570       ?GetS@DSA_Verifier@TaoCrypt@@QEBAAEBVInteger@2@XZ 00000001400b0570 f   taocrypt:dsa.obj
 0001:000af580       ??_EDSA_Private_Decoder@TaoCrypt@@UEAAPEAXI@Z 00000001400b0580 f i taocrypt:dsa.obj
 0001:000af580       ??_GDSA_Private_Decoder@TaoCrypt@@UEAAPEAXI@Z 00000001400b0580 f i taocrypt:dsa.obj
 0001:000af5b0       ??_GDSA_Public_Decoder@TaoCrypt@@UEAAPEAXI@Z 00000001400b05b0 f i taocrypt:dsa.obj
 0001:000af5b0       ??_EDSA_Public_Decoder@TaoCrypt@@UEAAPEAXI@Z 00000001400b05b0 f i taocrypt:dsa.obj
 0001:000af5e0       ??_1Integer@TaoCrypt@@QEAAAEAV01@AEBV01@@Z 00000001400b05e0 f i taocrypt:dsa.obj
 0001:000af640       ??0DSA_PublicKey@TaoCrypt@@QEAA@AEBV01@@Z 00000001400b0640 f   taocrypt:dsa.obj
 0001:000af690       ??4DSA_PublicKey@TaoCrypt@@QEAAAEAV01@AEBV01@@Z 00000001400b0690 f   taocrypt:dsa.obj
 0001:000af760       ??0DSA_PublicKey@TaoCrypt@@QEAA@AEAVSource@1@@Z 00000001400b0760 f   taocrypt:dsa.obj
 0001:000af7b0       ??0DSA_PrivateKey@TaoCrypt@@QEAA@AEAVSource@1@@Z 00000001400b07b0 f   taocrypt:dsa.obj
 0001:000af810       ??0DSA_Signer@TaoCrypt@@QEAA@AEBVDSA_PrivateKey@1@@Z 00000001400b0810 f   taocrypt:dsa.obj
 0001:000af840       ?Sign@DSA_Signer@TaoCrypt@@QEAAIPEBEPEAEAEAVRandomNumberGenerator@2@@Z 00000001400b0840 f   taocrypt:dsa.obj
 0001:000afc70       ??0DSA_Verifier@TaoCrypt@@QEAA@AEBVDSA_PublicKey@1@@Z 00000001400b0c70 f   taocrypt:dsa.obj
 0001:000afca0       ?Verify@DSA_Verifier@TaoCrypt@@QEAA_NPEBE0@Z 00000001400b0ca0 f   taocrypt:dsa.obj
 0001:000b00f0       ??0DH_Decoder@TaoCrypt@@QEAA@AEAVSource@1@@Z 00000001400b10f0 f i taocrypt:dh.obj
 0001:000b0110       ??1DH_Decoder@TaoCrypt@@UEAA@XZ 00000001400b1110 f i taocrypt:dh.obj
 0001:000b0120       ?DiscreteLogWorkFactor@?A0x4eb909e7@TaoCrypt@@YAII@Z 00000001400b1120 f   taocrypt:dh.obj
 0001:000b01a0       ?Initialize@DH@TaoCrypt@@QEAAXAEAVSource@2@@Z 00000001400b11a0 f   taocrypt:dh.obj
 0001:000b01d0       ??$min@VInteger@TaoCrypt@@@TaoCrypt@@YAAEBVInteger@0@AEBV10@0@Z 00000001400b11d0 f i taocrypt:dh.obj
 0001:000b0200       ??_GDH_Decoder@TaoCrypt@@UEAAPEAXI@Z 00000001400b1200 f i taocrypt:dh.obj
 0001:000b0200       ??_EDH_Decoder@TaoCrypt@@UEAAPEAXI@Z 00000001400b1200 f i taocrypt:dh.obj
 0001:000b0230       ?GeneratePrivate@DH@TaoCrypt@@AEAAXAEAVRandomNumberGenerator@2@PEAE@Z 00000001400b1230 f   taocrypt:dh.obj
 0001:000b0390       ?GeneratePublic@DH@TaoCrypt@@AEAAXPEBEPEAE@Z 00000001400b1390 f   taocrypt:dh.obj
 0001:000b0450       ?Agree@DH@TaoCrypt@@QEAAXPEAEPEBE1I@Z 00000001400b1450 f   taocrypt:dh.obj
 0001:000b0570       ??0DH@TaoCrypt@@QEAA@AEAVSource@1@@Z 00000001400b1570 f   taocrypt:dh.obj
 0001:000b05b0       ?GenerateKeyPair@DH@TaoCrypt@@QEAAXAEAVRandomNumberGenerator@2@PEAE1@Z 00000001400b15b0 f   taocrypt:dh.obj
 0001:000b05f0       ??0RSA_Private_Decoder@TaoCrypt@@QEAA@AEAVSource@1@@Z 00000001400b15f0 f i taocrypt:rsa.obj
 0001:000b0610       ??1RSA_Private_Decoder@TaoCrypt@@UEAA@XZ 00000001400b1610 f i taocrypt:rsa.obj
 0001:000b0620       ??0RSA_Public_Decoder@TaoCrypt@@QEAA@AEAVSource@1@@Z 00000001400b1620 f i taocrypt:rsa.obj
 0001:000b0640       ??1RSA_Public_Decoder@TaoCrypt@@UEAA@XZ 00000001400b1640 f i taocrypt:rsa.obj
 0001:000b0650       ?Initialize@RSA_PublicKey@TaoCrypt@@QEAAXAEAVSource@2@@Z 00000001400b1650 f   taocrypt:rsa.obj
 0001:000b0680       ?Initialize@RSA_PrivateKey@TaoCrypt@@QEAAXAEAVSource@2@@Z 00000001400b1680 f   taocrypt:rsa.obj
 0001:000b06b0       ?Pad@RSA_BlockType2@TaoCrypt@@QEBAXPEBEIPEAEIAEAVRandomNumberGenerator@2@@Z 00000001400b16b0 f   taocrypt:rsa.obj
 0001:000b0760       ?Pad@RSA_BlockType1@TaoCrypt@@QEBAXPEBEIPEAEIAEAVRandomNumberGenerator@2@@Z 00000001400b1760 f   taocrypt:rsa.obj
 0001:000b07f0       ??_GRSA_Private_Decoder@TaoCrypt@@UEAAPEAXI@Z 00000001400b17f0 f i taocrypt:rsa.obj
 0001:000b07f0       ??_ERSA_Private_Decoder@TaoCrypt@@UEAAPEAXI@Z 00000001400b17f0 f i taocrypt:rsa.obj
 0001:000b0820       ??_GRSA_Public_Decoder@TaoCrypt@@UEAAPEAXI@Z 00000001400b1820 f i taocrypt:rsa.obj
 0001:000b0820       ??_ERSA_Public_Decoder@TaoCrypt@@UEAAPEAXI@Z 00000001400b1820 f i taocrypt:rsa.obj
 0001:000b0850       ?UnPad@RSA_BlockType2@TaoCrypt@@QEBAIPEBEIPEAE@Z 00000001400b1850 f   taocrypt:rsa.obj
 0001:000b08f0       ?UnPad@RSA_BlockType1@TaoCrypt@@QEBAIPEBEIPEAE@Z 00000001400b18f0 f   taocrypt:rsa.obj
 0001:000b0990       ?ApplyFunction@RSA_PublicKey@TaoCrypt@@QEBA?AVInteger@2@AEBV32@@Z 00000001400b1990 f   taocrypt:rsa.obj
 0001:000b09c0       ??0RSA_PublicKey@TaoCrypt@@QEAA@AEAVSource@1@@Z 00000001400b19c0 f   taocrypt:rsa.obj
 0001:000b0a00       ?CalculateInverse@RSA_PrivateKey@TaoCrypt@@QEBA?AVInteger@2@AEAVRandomNumberGenerator@2@AEBV32@@Z 00000001400b1a00 f   taocrypt:rsa.obj
 0001:000b0cd0       ??0RSA_PrivateKey@TaoCrypt@@QEAA@AEAVSource@1@@Z 00000001400b1cd0 f   taocrypt:rsa.obj
 0001:000b0d50       ?SSL_Decrypt@TaoCrypt@@YAIAEBVRSA_PublicKey@1@PEBEPEAE@Z 00000001400b1d50 f   taocrypt:rsa.obj
 0001:000b0eb0       ?GetPublicKey@Signer@TaoCrypt@@QEBAAEBVPublicKey@2@XZ 00000001400b1eb0 f i taocrypt:asn.obj
 0001:000b0ec0       ?GetHash@Signer@TaoCrypt@@QEBAPEBEXZ 00000001400b1ec0 f i taocrypt:asn.obj
 0001:000b0ed0       ??0DER_Encoder@TaoCrypt@@QEAA@XZ 00000001400b1ed0 f i taocrypt:asn.obj
 0001:000b0ef0       ??1DER_Encoder@TaoCrypt@@UEAA@XZ 00000001400b1ef0 f i taocrypt:asn.obj
 0001:000b0f00       ??_GDER_Encoder@TaoCrypt@@UEAAPEAXI@Z 00000001400b1f00 f i taocrypt:asn.obj
 0001:000b0f00       ??_EDER_Encoder@TaoCrypt@@UEAAPEAXI@Z 00000001400b1f00 f i taocrypt:asn.obj
 0001:000b0f30       ?get_index@Source@TaoCrypt@@QEBAIXZ 00000001400b1f30 f i taocrypt:asn.obj
 0001:000b0f40       ?SetModulus@RSA_PublicKey@TaoCrypt@@QEAAXAEBVInteger@2@@Z 00000001400b1f40 f i taocrypt:asn.obj
 0001:000b0f50       ?SetPublicExponent@RSA_PublicKey@TaoCrypt@@QEAAXAEBVInteger@2@@Z 00000001400b1f50 f i taocrypt:asn.obj
 0001:000b0f60       ?SetPrime1@RSA_PrivateKey@TaoCrypt@@QEAAXAEBVInteger@2@@Z 00000001400b1f60 f i taocrypt:asn.obj
 0001:000b0f70       ?SetPrime2@RSA_PrivateKey@TaoCrypt@@QEAAXAEBVInteger@2@@Z 00000001400b1f70 f i taocrypt:asn.obj
 0001:000b0f80       ?SetPrivateExponent@RSA_PrivateKey@TaoCrypt@@QEAAXAEBVInteger@2@@Z 00000001400b1f80 f i taocrypt:asn.obj
 0001:000b0f90       ?SetModPrime1PrivateExponent@RSA_PrivateKey@TaoCrypt@@QEAAXAEBVInteger@2@@Z 00000001400b1f90 f i taocrypt:asn.obj
 0001:000b0fa0       ?SetModPrime2PrivateExponent@RSA_PrivateKey@TaoCrypt@@QEAAXAEBVInteger@2@@Z 00000001400b1fa0 f i taocrypt:asn.obj
 0001:000b0fb0       ?SetMultiplicativeInverseOfPrime2ModPrime1@RSA_PrivateKey@TaoCrypt@@QEAAXAEBVInteger@2@@Z 00000001400b1fb0 f i taocrypt:asn.obj
 0001:000b0fe0       ??O?A0xd1b11f91@TaoCrypt@@YA_NAEAUtm@@0@Z 00000001400b1fe0 f   taocrypt:asn.obj
 0001:000b1060       ??M?A0xd1b11f91@TaoCrypt@@YA_NAEAUtm@@0@Z 00000001400b2060 f   taocrypt:asn.obj
 0001:000b1080       ?btoi@?A0xd1b11f91@TaoCrypt@@YAIE@Z 00000001400b2080 f   taocrypt:asn.obj
 0001:000b1090       ?GetTime@?A0xd1b11f91@TaoCrypt@@YAXAEAHPEBE0@Z 00000001400b2090 f   taocrypt:asn.obj
 0001:000b10e0       ?ValidateDate@?A0xd1b11f91@TaoCrypt@@YA_NPEBEEW4DateType@CertDecoder@2@@Z 00000001400b20e0 f   taocrypt:asn.obj
 0001:000b1250       ?SetLength@TaoCrypt@@YAIIPEAE@Z 00000001400b2250 f   taocrypt:asn.obj
 0001:000b12e0       ?SetSize@PublicKey@TaoCrypt@@QEAAXI@Z 00000001400b22e0 f   taocrypt:asn.obj
 0001:000b1300       ?SetKey@PublicKey@TaoCrypt@@QEAAXPEBE@Z 00000001400b2300 f   taocrypt:asn.obj
 0001:000b1310       ?GetError@BER_Decoder@TaoCrypt@@QEAA?AUError@2@XZ 00000001400b2310 f   taocrypt:asn.obj
 0001:000b1320       ?GetInteger@BER_Decoder@TaoCrypt@@QEAAAEAVInteger@2@AEAV32@@Z 00000001400b2320 f   taocrypt:asn.obj
 0001:000b1350       ??1Signature_Encoder@TaoCrypt@@UEAA@XZ 00000001400b2350 f i taocrypt:asn.obj
 0001:000b1360       ?SetDigest@Signature_Encoder@TaoCrypt@@AEAAIPEBEIPEAE@Z 00000001400b2360 f   taocrypt:asn.obj
 0001:000b1390       ?SetSequence@TaoCrypt@@YAIIPEAE@Z 00000001400b2390 f   taocrypt:asn.obj
 0001:000b13b0       ?EncodeDSA_Signature@TaoCrypt@@YAIAEBVInteger@1@0PEAE@Z 00000001400b23b0 f   taocrypt:asn.obj
 0001:000b14f0       ??A?$Block@EV?$AllocatorWithCleanup@E@TaoCrypt@@@TaoCrypt@@QEBAAEBEI@Z 00000001400b24f0 f i taocrypt:asn.obj
 0001:000b1500       ??0?$auto_ptr@VHASH@TaoCrypt@@@mySTL@@QEAA@PEAVHASH@TaoCrypt@@@Z 00000001400b2500 f i taocrypt:asn.obj
 0001:000b1510       ??C?$auto_ptr@VHASH@TaoCrypt@@@mySTL@@QEBAPEAVHASH@TaoCrypt@@XZ 00000001400b2510 f i taocrypt:asn.obj
 0001:000b1520       ??$tcDelete@VHASH@TaoCrypt@@@TaoCrypt@@YAXPEAVHASH@0@@Z 00000001400b2520 f i taocrypt:asn.obj
 0001:000b1540       ??1PublicKey@TaoCrypt@@QEAA@XZ 00000001400b2540 f i taocrypt:asn.obj
 0001:000b1550       ?get_current@Source@TaoCrypt@@QEBAPEBEXZ 00000001400b2550 f i taocrypt:asn.obj
 0001:000b1560       ?set_index@Source@TaoCrypt@@QEAAXI@Z 00000001400b2560 f i taocrypt:asn.obj
 0001:000b1570       ?add@Source@TaoCrypt@@QEAAXPEBEI@Z 00000001400b2570 f i taocrypt:asn.obj
 0001:000b15d0       ?advance@Source@TaoCrypt@@QEAAXI@Z 00000001400b25d0 f i taocrypt:asn.obj
 0001:000b15f0       ?GetLength@TaoCrypt@@YAIAEAVSource@1@@Z 00000001400b25f0 f   taocrypt:asn.obj
 0001:000b16b0       ??0PublicKey@TaoCrypt@@QEAA@PEBEI@Z 00000001400b26b0 f   taocrypt:asn.obj
 0001:000b16f0       ??0Signer@TaoCrypt@@QEAA@PEBEIPEBD0@Z 00000001400b26f0 f   taocrypt:asn.obj
 0001:000b1770       ??1Signer@TaoCrypt@@QEAA@XZ 00000001400b2770 f   taocrypt:asn.obj
 0001:000b1780       ?GetSequence@BER_Decoder@TaoCrypt@@QEAAIXZ 00000001400b2780 f   taocrypt:asn.obj
 0001:000b17d0       ?GetSet@BER_Decoder@TaoCrypt@@QEAAIXZ 00000001400b27d0 f   taocrypt:asn.obj
 0001:000b1820       ?GetVersion@BER_Decoder@TaoCrypt@@QEAAIXZ 00000001400b2820 f   taocrypt:asn.obj
 0001:000b18f0       ?GetExplicitVersion@BER_Decoder@TaoCrypt@@QEAAIXZ 00000001400b28f0 f   taocrypt:asn.obj
 0001:000b1970       ?ReadHeader@RSA_Private_Decoder@TaoCrypt@@EEAAXXZ 00000001400b2970 f   taocrypt:asn.obj
 0001:000b1990       ?ReadHeader@DSA_Private_Decoder@TaoCrypt@@EEAAXXZ 00000001400b2990 f   taocrypt:asn.obj
 0001:000b19b0       ?ReadHeaderOpenSSL@RSA_Public_Decoder@TaoCrypt@@AEAAXXZ 00000001400b29b0 f   taocrypt:asn.obj
 0001:000b1bb0       ?ReadHeader@RSA_Public_Decoder@TaoCrypt@@EEAAXXZ 00000001400b2bb0 f   taocrypt:asn.obj
 0001:000b1bc0       ?ReadHeader@DSA_Public_Decoder@TaoCrypt@@EEAAXXZ 00000001400b2bc0 f   taocrypt:asn.obj
 0001:000b1bd0       ?ReadHeader@DH_Decoder@TaoCrypt@@EEAAXXZ 00000001400b2bd0 f   taocrypt:asn.obj
 0001:000b1be0       ??1CertDecoder@TaoCrypt@@UEAA@XZ 00000001400b2be0 f   taocrypt:asn.obj
 0001:000b1c20       ?StoreKey@CertDecoder@TaoCrypt@@AEAAXXZ 00000001400b2c20 f   taocrypt:asn.obj
 0001:000b1d10       ?GetAlgoId@CertDecoder@TaoCrypt@@AEAAIXZ 00000001400b2d10 f   taocrypt:asn.obj
 0001:000b1e90       ?GetSignature@CertDecoder@TaoCrypt@@AEAAIXZ 00000001400b2e90 f   taocrypt:asn.obj
 0001:000b1fe0       ?GetDigest@CertDecoder@TaoCrypt@@AEAAIXZ 00000001400b2fe0 f   taocrypt:asn.obj
 0001:000b20a0       ?AddTag@CertDecoder@TaoCrypt@@AEAAPEADPEADPEBD1II@Z 00000001400b30a0 f   taocrypt:asn.obj
 0001:000b2120       ?GetName@CertDecoder@TaoCrypt@@AEAAXW4NameType@12@@Z 00000001400b3120 f   taocrypt:asn.obj
 0001:000b2690       ?GetDate@CertDecoder@TaoCrypt@@AEAAXW4DateType@12@@Z 00000001400b3690 f   taocrypt:asn.obj
 0001:000b2850       ?GetValidity@CertDecoder@TaoCrypt@@AEAAXXZ 00000001400b3850 f   taocrypt:asn.obj
 0001:000b2890       ?SetAlgoID@DER_Encoder@TaoCrypt@@QEAAIW4HashType@2@PEAE@Z 00000001400b3890 f   taocrypt:asn.obj
 0001:000b29b0       ?Destroy@?$auto_ptr@VHASH@TaoCrypt@@@mySTL@@AEAAXXZ 00000001400b39b0 f i taocrypt:asn.obj
 0001:000b29c0       ??_GCertDecoder@TaoCrypt@@UEAAPEAXI@Z 00000001400b39c0 f i taocrypt:asn.obj
 0001:000b29c0       ??_ECertDecoder@TaoCrypt@@UEAAPEAXI@Z 00000001400b39c0 f i taocrypt:asn.obj
 0001:000b29f0       ??1?$auto_ptr@VHASH@TaoCrypt@@@mySTL@@QEAA@XZ 00000001400b39f0 f i taocrypt:asn.obj
 0001:000b2a00       ?reset@?$auto_ptr@VHASH@TaoCrypt@@@mySTL@@QEAAXPEAVHASH@TaoCrypt@@@Z 00000001400b3a00 f i taocrypt:asn.obj
 0001:000b2a30       ?AddToEnd@PublicKey@TaoCrypt@@QEAAXPEBEI@Z 00000001400b3a30 f   taocrypt:asn.obj
 0001:000b2ab0       ?Decode@RSA_Private_Decoder@TaoCrypt@@QEAAXAEAVRSA_PrivateKey@2@@Z 00000001400b3ab0 f   taocrypt:asn.obj
 0001:000b2d00       ?Decode@DSA_Private_Decoder@TaoCrypt@@QEAAXAEAVDSA_PrivateKey@2@@Z 00000001400b3d00 f   taocrypt:asn.obj
 0001:000b2e80       ?Decode@RSA_Public_Decoder@TaoCrypt@@QEAAXAEAVRSA_PublicKey@2@@Z 00000001400b3e80 f   taocrypt:asn.obj
 0001:000b2f60       ?Decode@DSA_Public_Decoder@TaoCrypt@@QEAAXAEAVDSA_PublicKey@2@@Z 00000001400b3f60 f   taocrypt:asn.obj
 0001:000b30a0       ?Decode@DH_Decoder@TaoCrypt@@QEAAXAEAVDH@2@@Z 00000001400b40a0 f   taocrypt:asn.obj
 0001:000b3160       ?ReadHeader@CertDecoder@TaoCrypt@@EEAAXXZ 00000001400b4160 f   taocrypt:asn.obj
 0001:000b31e0       ?AddDSA@CertDecoder@TaoCrypt@@AEAAXXZ 00000001400b41e0 f   taocrypt:asn.obj
 0001:000b3370       ?EncodeDSA_Signature@TaoCrypt@@YAIPEBEPEAE@Z 00000001400b4370 f   taocrypt:asn.obj
 0001:000b3410       ?DecodeDSA_Signature@TaoCrypt@@YAIPEAEPEBEI@Z 00000001400b4410 f   taocrypt:asn.obj
 0001:000b36a0       ?CleanGrow@?$Block@EV?$AllocatorWithCleanup@E@TaoCrypt@@@TaoCrypt@@QEAAXI@Z 00000001400b46a0 f i taocrypt:asn.obj
 0001:000b36f0       ?grow@Source@TaoCrypt@@QEAAXI@Z 00000001400b46f0 f i taocrypt:asn.obj
 0001:000b3740       ?GetKey@CertDecoder@TaoCrypt@@AEAAXXZ 00000001400b4740 f   taocrypt:asn.obj
 0001:000b3870       ??0Signature_Encoder@TaoCrypt@@QEAA@PEBEIW4HashType@1@AEAVSource@1@@Z 00000001400b4870 f   taocrypt:asn.obj
 0001:000b39d0       ??_GSignature_Encoder@TaoCrypt@@UEAAPEAXI@Z 00000001400b49d0 f i taocrypt:asn.obj
 0001:000b39d0       ??_ESignature_Encoder@TaoCrypt@@UEAAPEAXI@Z 00000001400b49d0 f i taocrypt:asn.obj
 0001:000b3a00       ??0Source@TaoCrypt@@QEAA@I@Z 00000001400b4a00 f i taocrypt:asn.obj
 0001:000b3a80       ?DecodeToKey@CertDecoder@TaoCrypt@@QEAAXXZ 00000001400b4a80 f   taocrypt:asn.obj
 0001:000b3ad0       ?ConfirmSignature@CertDecoder@TaoCrypt@@AEAA_NAEAVSource@2@@Z 00000001400b4ad0 f   taocrypt:asn.obj
 0001:000b3eb0       ?ValidateSelfSignature@CertDecoder@TaoCrypt@@AEAA_NXZ 00000001400b4eb0 f   taocrypt:asn.obj
 0001:000b3f40       ?ValidateSignature@CertDecoder@TaoCrypt@@AEAA_NPEAV?$list@PEAVSigner@TaoCrypt@@@mySTL@@@Z 00000001400b4f40 f   taocrypt:asn.obj
 0001:000b4040       ?Decode@CertDecoder@TaoCrypt@@AEAAXPEAV?$list@PEAVSigner@TaoCrypt@@@mySTL@@W4CertType@12@@Z 00000001400b5040 f   taocrypt:asn.obj
 0001:000b4100       ??0CertDecoder@TaoCrypt@@QEAA@AEAVSource@1@_NPEAV?$list@PEAVSigner@TaoCrypt@@@mySTL@@1W4CertType@01@@Z 00000001400b5100 f   taocrypt:asn.obj
 0001:000b4190       ?GetCompareHash@CertDecoder@TaoCrypt@@AEAAXPEBEIPEAEI@Z 00000001400b5190 f   taocrypt:asn.obj
 0001:000b42c0       ??1FileSource@TaoCrypt@@QEAA@XZ 00000001400b52c0 f   taocrypt:file.obj
 0001:000b42e0       ?size@FileSource@TaoCrypt@@QEAAI_N@Z 00000001400b52e0 f   taocrypt:file.obj
 0001:000b4360       ?size_left@FileSource@TaoCrypt@@AEAAIXZ 00000001400b5360 f   taocrypt:file.obj
 0001:000b4370       ??1FileSink@TaoCrypt@@QEAA@XZ 00000001400b5370 f   taocrypt:file.obj
 0001:000b4390       ?put@FileSink@TaoCrypt@@AEAAXAEAVSource@2@@Z 00000001400b5390 f   taocrypt:file.obj
 0001:000b43b0       ?Swap@?$Block@EV?$AllocatorWithCleanup@E@TaoCrypt@@@TaoCrypt@@QEAAXAEAV12@@Z 00000001400b53b0 f i taocrypt:file.obj
 0001:000b43d0       ??0FileSink@TaoCrypt@@QEAA@PEBDAEAVSource@1@@Z 00000001400b53d0 f   taocrypt:file.obj
 0001:000b4420       ?reset@Source@TaoCrypt@@QEAAXAEAV?$Block@EV?$AllocatorWithCleanup@E@TaoCrypt@@@2@@Z 00000001400b5420 f   taocrypt:file.obj
 0001:000b4450       ?get@FileSource@TaoCrypt@@AEAAIAEAVSource@2@@Z 00000001400b5450 f   taocrypt:file.obj
 0001:000b44e0       ??0FileSource@TaoCrypt@@QEAA@PEBDAEAVSource@1@@Z 00000001400b54e0 f   taocrypt:file.obj
 0001:000b4530       ?Double@AbstractGroup@TaoCrypt@@UEBAAEBVInteger@2@AEBV32@@Z 00000001400b5530 f   taocrypt:algebra.obj
 0001:000b4540       ?Accumulate@AbstractGroup@TaoCrypt@@UEBAAEAVInteger@2@AEAV32@AEBV32@@Z 00000001400b5540 f   taocrypt:algebra.obj
 0001:000b4560       ?Reduce@AbstractGroup@TaoCrypt@@UEBAAEAVInteger@2@AEAV32@AEBV32@@Z 00000001400b5560 f   taocrypt:algebra.obj
 0001:000b4580       ?Square@AbstractRing@TaoCrypt@@UEBAAEBVInteger@2@AEBV32@@Z 00000001400b5580 f   taocrypt:algebra.obj
 0001:000b4590       ?FindNextWindow@WindowSlider@TaoCrypt@@QEAAXXZ 00000001400b5590 f i taocrypt:algebra.obj
 0001:000b4680       ?size@?$vector@VInteger@TaoCrypt@@@mySTL@@QEBA_KXZ 00000001400b5680 f i taocrypt:algebra.obj
 0001:000b4690       ??A?$vector@VInteger@TaoCrypt@@@mySTL@@QEAAAEAVInteger@TaoCrypt@@_K@Z 00000001400b5690 f i taocrypt:algebra.obj
 0001:000b46a0       ??A?$vector@V?$vector@VInteger@TaoCrypt@@@mySTL@@@mySTL@@QEAAAEAV?$vector@VInteger@TaoCrypt@@@1@_K@Z 00000001400b56a0 f i taocrypt:algebra.obj
 0001:000b46b0       ??A?$vector@UWindowSlider@TaoCrypt@@@mySTL@@QEAAAEAUWindowSlider@TaoCrypt@@_K@Z 00000001400b56b0 f i taocrypt:algebra.obj
 0001:000b46c0       ?capacity@?$vector@UWindowSlider@TaoCrypt@@@mySTL@@QEBA_KXZ 00000001400b56c0 f i taocrypt:algebra.obj
 0001:000b46f0       ?size@?$vector@UWindowSlider@TaoCrypt@@@mySTL@@QEBA_KXZ 00000001400b56f0 f i taocrypt:algebra.obj
 0001:000b4720       ??0?$vector_base@UWindowSlider@TaoCrypt@@@mySTL@@QEAA@XZ 00000001400b5720 f i taocrypt:algebra.obj
 0001:000b4740       ??0?$vector_base@VInteger@TaoCrypt@@@mySTL@@QEAA@XZ 00000001400b5740 f i taocrypt:algebra.obj
 0001:000b4760       ??$GetArrayMemory@VInteger@TaoCrypt@@@mySTL@@YAPEAVInteger@TaoCrypt@@_K@Z 00000001400b5760 f i taocrypt:algebra.obj
 0001:000b4770       ??$FreeArrayMemory@VInteger@TaoCrypt@@@mySTL@@YAXPEAVInteger@TaoCrypt@@@Z 00000001400b5770 f i taocrypt:algebra.obj
 0001:000b4780       ??$GetArrayMemory@V?$vector@VInteger@TaoCrypt@@@mySTL@@@mySTL@@YAPEAV?$vector@VInteger@TaoCrypt@@@0@_K@Z 00000001400b5780 f i taocrypt:algebra.obj
 0001:000b4790       ??$FreeArrayMemory@V?$vector@VInteger@TaoCrypt@@@mySTL@@@mySTL@@YAXPEAV?$vector@VInteger@TaoCrypt@@@0@@Z 00000001400b5790 f i taocrypt:algebra.obj
 0001:000b47a0       ??$FreeArrayMemory@UWindowSlider@TaoCrypt@@@mySTL@@YAXPEAUWindowSlider@TaoCrypt@@@Z 00000001400b57a0 f i taocrypt:algebra.obj
 0001:000b47b0       ??$swap@PEAVInteger@TaoCrypt@@@mySTL@@YAXAEAPEAVInteger@TaoCrypt@@0@Z 00000001400b57b0 f i taocrypt:algebra.obj
 0001:000b47c0       ??$GetArrayMemory@UWindowSlider@TaoCrypt@@@mySTL@@YAPEAUWindowSlider@TaoCrypt@@_K@Z 00000001400b57c0 f i taocrypt:algebra.obj
 0001:000b47d0       ??$swap@PEAUWindowSlider@TaoCrypt@@@mySTL@@YAXAEAPEAUWindowSlider@TaoCrypt@@0@Z 00000001400b57d0 f i taocrypt:algebra.obj
 0001:000b47e0       ??$construct@VInteger@TaoCrypt@@V12@@mySTL@@YAXPEAVInteger@TaoCrypt@@AEBV12@@Z 00000001400b57e0 f i taocrypt:algebra.obj
 0001:000b4800       ??0?$vector_base@VInteger@TaoCrypt@@@mySTL@@QEAA@_K@Z 00000001400b5800 f i taocrypt:algebra.obj
 0001:000b4840       ??1?$vector_base@VInteger@TaoCrypt@@@mySTL@@QEAA@XZ 00000001400b5840 f i taocrypt:algebra.obj
 0001:000b4850       ??0?$vector_base@V?$vector@VInteger@TaoCrypt@@@mySTL@@@mySTL@@QEAA@_K@Z 00000001400b5850 f i taocrypt:algebra.obj
 0001:000b4890       ??1?$vector_base@V?$vector@VInteger@TaoCrypt@@@mySTL@@@mySTL@@QEAA@XZ 00000001400b5890 f i taocrypt:algebra.obj
 0001:000b48a0       ??1?$vector_base@UWindowSlider@TaoCrypt@@@mySTL@@QEAA@XZ 00000001400b58a0 f i taocrypt:algebra.obj
 0001:000b48b0       ?Swap@?$vector_base@VInteger@TaoCrypt@@@mySTL@@QEAAXAEAU12@@Z 00000001400b58b0 f i taocrypt:algebra.obj
 0001:000b48e0       ??0?$vector_base@UWindowSlider@TaoCrypt@@@mySTL@@QEAA@_K@Z 00000001400b58e0 f i taocrypt:algebra.obj
 0001:000b4920       ?Swap@?$vector_base@UWindowSlider@TaoCrypt@@@mySTL@@QEAAXAEAU12@@Z 00000001400b5920 f i taocrypt:algebra.obj
 0001:000b4950       ??$uninit_fill_n@PEAVInteger@TaoCrypt@@_KV12@@mySTL@@YAPEAVInteger@TaoCrypt@@PEAV12@_KAEBV12@@Z 00000001400b5950 f i taocrypt:algebra.obj
 0001:000b49a0       ??$uninit_copy@PEAVInteger@TaoCrypt@@PEAV12@@mySTL@@YAPEAVInteger@TaoCrypt@@PEAV12@00@Z 00000001400b59a0 f i taocrypt:algebra.obj
 0001:000b49f0       ??0?$vector@VInteger@TaoCrypt@@@mySTL@@QEAA@AEBV01@@Z 00000001400b59f0 f i taocrypt:algebra.obj
 0001:000b4a50       ??0?$vector@UWindowSlider@TaoCrypt@@@mySTL@@QEAA@XZ 00000001400b5a50 f i taocrypt:algebra.obj
 0001:000b4a70       ??0?$vector@VInteger@TaoCrypt@@@mySTL@@QEAA@XZ 00000001400b5a70 f i taocrypt:algebra.obj
 0001:000b4a90       ?Swap@?$vector@VInteger@TaoCrypt@@@mySTL@@QEAAXAEAV12@@Z 00000001400b5a90 f i taocrypt:algebra.obj
 0001:000b4ac0       ??0?$vector@VInteger@TaoCrypt@@@mySTL@@AEAA@_KAEBV01@@Z 00000001400b5ac0 f i taocrypt:algebra.obj
 0001:000b4b30       ?Swap@?$vector@UWindowSlider@TaoCrypt@@@mySTL@@QEAAXAEAV12@@Z 00000001400b5b30 f i taocrypt:algebra.obj
 0001:000b4b60       ??$construct@V?$vector@VInteger@TaoCrypt@@@mySTL@@V12@@mySTL@@YAXPEAV?$vector@VInteger@TaoCrypt@@@0@AEBV10@@Z 00000001400b5b60 f i taocrypt:algebra.obj
 0001:000b4bd0       ?Subtract@AbstractGroup@TaoCrypt@@UEBAAEBVInteger@2@AEBV32@0@Z 00000001400b5bd0 f   taocrypt:algebra.obj
 0001:000b4c40       ?Divide@AbstractRing@TaoCrypt@@UEBAAEBVInteger@2@AEBV32@0@Z 00000001400b5c40 f   taocrypt:algebra.obj
 0001:000b4cc0       ?Mod@AbstractEuclideanDomain@TaoCrypt@@UEBAAEBVInteger@2@AEBV32@0@Z 00000001400b5cc0 f   taocrypt:algebra.obj
 0001:000b4d40       ?ScalarMultiply@AbstractGroup@TaoCrypt@@UEBA?AVInteger@2@AEBV32@0@Z 00000001400b5d40 f   taocrypt:algebra.obj
 0001:000b4da0       ??0WindowSlider@TaoCrypt@@QEAA@AEBVInteger@1@_NI@Z 00000001400b5da0 f i taocrypt:algebra.obj
 0001:000b4e70       ??1WindowSlider@TaoCrypt@@QEAA@XZ 00000001400b5e70 f i taocrypt:algebra.obj
 0001:000b4ed0       ?Exponentiate@AbstractRing@TaoCrypt@@UEBA?AVInteger@2@AEBV32@0@Z 00000001400b5ed0 f   taocrypt:algebra.obj
 0001:000b4f30       ??0?$vector@VInteger@TaoCrypt@@@mySTL@@QEAA@_K@Z 00000001400b5f30 f i taocrypt:algebra.obj
 0001:000b4fb0       ??$uninit_fill_n@PEAV?$vector@VInteger@TaoCrypt@@@mySTL@@_KV12@@mySTL@@YAPEAV?$vector@VInteger@TaoCrypt@@@0@PEAV10@_KAEBV10@@Z 00000001400b5fb0 f i taocrypt:algebra.obj
 0001:000b5040       ??0WindowSlider@TaoCrypt@@QEAA@AEBU01@@Z 00000001400b6040 f i taocrypt:algebra.obj
 0001:000b50a0       ??_GWindowSlider@TaoCrypt@@QEAAPEAXI@Z 00000001400b60a0 f i taocrypt:algebra.obj
 0001:000b5110       ??$construct@UWindowSlider@TaoCrypt@@U12@@mySTL@@YAXPEAUWindowSlider@TaoCrypt@@AEBU12@@Z 00000001400b6110 f i taocrypt:algebra.obj
 0001:000b5180       ??$uninit_copy@PEAUWindowSlider@TaoCrypt@@PEAU12@@mySTL@@YAPEAUWindowSlider@TaoCrypt@@PEAU12@00@Z 00000001400b6180 f i taocrypt:algebra.obj
 0001:000b5210       ??$destroy@VInteger@TaoCrypt@@@mySTL@@YAXPEAVInteger@TaoCrypt@@@Z 00000001400b6210 f i taocrypt:algebra.obj
 0001:000b5240       ??$destroy@UWindowSlider@TaoCrypt@@@mySTL@@YAXPEAUWindowSlider@TaoCrypt@@@Z 00000001400b6240 f i taocrypt:algebra.obj
 0001:000b52a0       ??0?$vector@UWindowSlider@TaoCrypt@@@mySTL@@AEAA@_KAEBV01@@Z 00000001400b62a0 f i taocrypt:algebra.obj
 0001:000b5330       ??$destroy@PEAVInteger@TaoCrypt@@@mySTL@@YAXPEAVInteger@TaoCrypt@@0@Z 00000001400b6330 f i taocrypt:algebra.obj
 0001:000b5390       ??$destroy@PEAUWindowSlider@TaoCrypt@@@mySTL@@YAXPEAUWindowSlider@TaoCrypt@@0@Z 00000001400b6390 f i taocrypt:algebra.obj
 0001:000b5410       ??1?$vector@VInteger@TaoCrypt@@@mySTL@@QEAA@XZ 00000001400b6410 f i taocrypt:algebra.obj
 0001:000b5440       ?resize@?$vector@VInteger@TaoCrypt@@@mySTL@@QEAAX_KAEBVInteger@TaoCrypt@@@Z 00000001400b6440 f i taocrypt:algebra.obj
 0001:000b5550       ??0?$vector@V?$vector@VInteger@TaoCrypt@@@mySTL@@@mySTL@@QEAA@_K@Z 00000001400b6550 f i taocrypt:algebra.obj
 0001:000b55c0       ??1?$vector@UWindowSlider@TaoCrypt@@@mySTL@@QEAA@XZ 00000001400b65c0 f i taocrypt:algebra.obj
 0001:000b55f0       ?push_back@?$vector@UWindowSlider@TaoCrypt@@@mySTL@@QEAAXAEBUWindowSlider@TaoCrypt@@@Z 00000001400b65f0 f i taocrypt:algebra.obj
 0001:000b5780       ?reserve@?$vector@UWindowSlider@TaoCrypt@@@mySTL@@QEAAX_K@Z 00000001400b6780 f i taocrypt:algebra.obj
 0001:000b5860       ??_G?$vector@VInteger@TaoCrypt@@@mySTL@@QEAAPEAXI@Z 00000001400b6860 f i taocrypt:algebra.obj
 0001:000b58a0       ?Gcd@AbstractEuclideanDomain@TaoCrypt@@UEBAAEBVInteger@2@AEBV32@0@Z 00000001400b68a0 f   taocrypt:algebra.obj
 0001:000b5a00       ?CascadeScalarMultiply@AbstractGroup@TaoCrypt@@UEBA?AVInteger@2@AEBV32@000@Z 00000001400b6a00 f   taocrypt:algebra.obj
 0001:000b5ee0       ?CascadeExponentiate@AbstractRing@TaoCrypt@@UEBA?AVInteger@2@AEBV32@000@Z 00000001400b6ee0 f   taocrypt:algebra.obj
 0001:000b5f40       ??$destroy@V?$vector@VInteger@TaoCrypt@@@mySTL@@@mySTL@@YAXPEAV?$vector@VInteger@TaoCrypt@@@0@@Z 00000001400b6f40 f i taocrypt:algebra.obj
 0001:000b5f70       ??$destroy@PEAV?$vector@VInteger@TaoCrypt@@@mySTL@@@mySTL@@YAXPEAV?$vector@VInteger@TaoCrypt@@@0@0@Z 00000001400b6f70 f i taocrypt:algebra.obj
 0001:000b5fc0       ??1?$vector@V?$vector@VInteger@TaoCrypt@@@mySTL@@@mySTL@@QEAA@XZ 00000001400b6fc0 f i taocrypt:algebra.obj
 0001:000b5ff0       ?SimultaneousMultiply@AbstractGroup@TaoCrypt@@UEBAXPEAVInteger@2@AEBV32@PEBV32@I@Z 00000001400b6ff0 f   taocrypt:algebra.obj
 0001:000b6710       ?SimultaneousExponentiate@AbstractRing@TaoCrypt@@UEBAXPEAVInteger@2@AEBV32@PEBV32@I@Z 00000001400b7710 f   taocrypt:algebra.obj
 0001:000b6760       ?Init@MD2@TaoCrypt@@UEAAXXZ 00000001400b7760 f   taocrypt:md2.obj
 0001:000b67a0       ?Update@MD2@TaoCrypt@@UEAAXPEBEI@Z 00000001400b77a0 f   taocrypt:md2.obj
 0001:000b6980       ?Final@MD2@TaoCrypt@@UEAAXPEAE@Z 00000001400b7980 f   taocrypt:md2.obj
 0001:000b6a20       ??0MD2@TaoCrypt@@QEAA@XZ   00000001400b7a20 f   taocrypt:md2.obj
 0001:000b6b30       ?getBlockSize@MD2@TaoCrypt@@UEBAIXZ 00000001400b7b30 f i taocrypt:md2.obj
 0001:000b6b40       ?getDigestSize@MD2@TaoCrypt@@UEBAIXZ 00000001400b7b40 f i taocrypt:md2.obj
 0001:000b6b50       ??1MD2@TaoCrypt@@UEAA@XZ   00000001400b7b50 f i taocrypt:md2.obj
 0001:000b6bc0       ??_GMD2@TaoCrypt@@UEAAPEAXI@Z 00000001400b7bc0 f i taocrypt:md2.obj
 0001:000b6bc0       ??_EMD2@TaoCrypt@@UEAAPEAXI@Z 00000001400b7bc0 f i taocrypt:md2.obj
 0001:000b6c50       remove                     00000001400b7c50 f   LIBCMT:unlink.obj
 0001:000b6c80       _unlink                    00000001400b7c80 f   LIBCMT:unlink.obj
 0001:000b6c80       unlink                     00000001400b7c80 f   LIBCMT:unlink.obj
 0001:000b7000       _putenv                    00000001400b8000 f   LIBCMT:putenv.obj
 0001:000b7000       putenv                     00000001400b8000 f   LIBCMT:putenv.obj
 0001:000b7060       _putenv_s                  00000001400b8060 f   LIBCMT:putenv.obj
 0001:000b7110       _chdir                     00000001400b8110 f   LIBCMT:chdir.obj
 0001:000b7110       chdir                      00000001400b8110 f   LIBCMT:chdir.obj
 0001:000b7260       log                        00000001400b8260 f   LIBCMT:log.obj
 0001:000b7570       pow                        00000001400b8570 f   LIBCMT:pow.obj
 0001:000b7b5a       __clear_x87_state          00000001400b8b5a f   LIBCMT:pow.obj
 0001:000b7ca0       __crtwsetenv               00000001400b8ca0 f   LIBCMT:wsetenv.obj
 0001:000b8190       _mbctoupper_l              00000001400b9190 f   LIBCMT:mbtoupr.obj
 0001:000b8350       _mbctoupper                00000001400b9350 f   LIBCMT:mbtoupr.obj
 0001:000b8360       __pow_error                00000001400b9360 f   LIBCMT:pow_error.obj
 0001:000b86a0       _wcsnicoll_l               00000001400b96a0 f   LIBCMT:wcsnicol.obj
 0001:000b8810       _wcsnicoll                 00000001400b9810 f   LIBCMT:wcsnicol.obj
 0001:000b88c0       _wcsdup                    00000001400b98c0 f   LIBCMT:wcsdup.obj
 0001:000b8960       wcscpy_s                   00000001400b9960 f   LIBCMT:wcscpy_s.obj
 0001:000b8a10       __mbtow_environ            00000001400b9a10 f   LIBCMT:mbtowenv.obj
 0001:000b8b10       _wsetenvp                  00000001400b9b10 f   LIBCMT:wstdenvp.obj
 0001:000b8c80       __crtGetEnvironmentStringsW 00000001400b9c80 f   LIBCMT:w_env.obj
 0001:000b8e80       wcschr                     00000001400b9e80 f   LIBCMT:wcschr.obj
 0001:000b9260       __crtCompareStringW        00000001400ba260 f   LIBCMT:w_cmp.obj
 0001:000b93a8       SetEnvironmentVariableW    00000001400ba3a8 f   kernel32:KERNEL32.dll
 0001:000b93ae       CryptAcquireContextA       00000001400ba3ae f   advapi32:ADVAPI32.dll
 0001:000b93b4       CryptReleaseContext        00000001400ba3b4 f   advapi32:ADVAPI32.dll
 0001:000b93ba       CryptGenRandom             00000001400ba3ba f   advapi32:ADVAPI32.dll
 0001:000e42c0       _frnd                      00000001400e52c0 f   LIBCMT:fpsr.obj
 0001:000e5300       __chkstk                   00000001400e6300 f   LIBCMT:chkstk.obj
 0001:000e5300       _alloca_probe              00000001400e6300     LIBCMT:chkstk.obj
 0001:000e5360       _get_fpsr                  00000001400e6360 f   LIBCMT:fpsr.obj
 0002:00000000       __xc_a                     00000001400e9000     LIBCMT:crt0init.obj
 0002:00000110       __xc_z                     00000001400e9110     LIBCMT:crt0init.obj
 0002:00000220       __xi_a                     00000001400e9220     LIBCMT:crt0init.obj
 0002:00000560       __xi_z                     00000001400e9560     LIBCMT:crt0init.obj
 0002:00000670       __xl_a                     00000001400e9670     LIBCMT:tlssup.obj
 0002:00000678       __xl_z                     00000001400e9678     LIBCMT:tlssup.obj
 0002:00000680       __xp_a                     00000001400e9680     LIBCMT:crt0init.obj
 0002:000009b0       __xp_z                     00000001400e99b0     LIBCMT:crt0init.obj
 0002:00000ac0       __xt_a                     00000001400e9ac0     LIBCMT:crt0init.obj
 0002:00000bd0       __xt_z                     00000001400e9bd0     LIBCMT:crt0init.obj
 0002:00000cfc       ?BUFFER_INITIAL_SIZE@Buffer@@0IB 00000001400e9cfc     buffer.obj
 0002:00000d00       ?MAX_BUFFER_SIZE@Buffer@@0IB 00000001400e9d00     buffer.obj
 0002:00000d08       __real@3ff8000000000000    00000001400e9d08     buffer.obj
 0002:00000d18       __real@43f0000000000000    00000001400e9d18     buffer.obj
 0002:00000d30       ??_7Command@@6B@           00000001400e9d30     command.obj
 0002:00000d48       ??_C@_07OFPCFMBE@offline?$AA@ 00000001400e9d48     commands.obj
 0002:00000d54       ??_C@_06GNLMCJKK@online?$AA@ 00000001400e9d54     commands.obj
 0002:00000d5c       ??_C@_06DJIHEMFI@status?$AA@ 00000001400e9d5c     commands.obj
 0002:00000d68       ??_C@_0O@MIFOIHFB@instance_name?$AA@ 00000001400e9d68     commands.obj
 0002:00000d80       ??_7Show_instance_status@@6B@ 00000001400e9d80     commands.obj
 0002:00000d98       ??_C@_07CIFAGBMG@unknown?$AA@ 00000001400e9d98     commands.obj
 0002:00000da8       ??_C@_07CPCPJPKL@version?$AA@ 00000001400e9da8     commands.obj
 0002:00000dc0       ??_7Show_instance_options@@6B@ 00000001400e9dc0     commands.obj
 0002:00000dd4       ??_C@_00CNPNBAHC@?$AA@     00000001400e9dd4     commands.obj
 0002:00000dd8       ??_C@_0L@PNJKAIKE@nonguarded?$AA@ 00000001400e9dd8     commands.obj
 0002:00000de8       ??_C@_0M@IKAFELGN@mysqld?9path?$AA@ 00000001400e9de8     commands.obj
 0002:00000df8       ??_C@_05MFEJDJP@value?$AA@ 00000001400e9df8     commands.obj
 0002:00000e00       ??_C@_0M@PNCLCLFB@option_name?$AA@ 00000001400e9e00     commands.obj
 0002:00000e18       ??_7Start_instance@@6B@    00000001400e9e18     commands.obj
 0002:00000e30       ??_C@_0BB@EIFMIEBH@Instance?5started?$AA@ 00000001400e9e30     commands.obj
 0002:00000e50       ??_7Show_instance_log@@6B@ 00000001400e9e50     commands.obj
 0002:00000e64       ??_C@_03GGEOLGBL@Log?$AA@  00000001400e9e64     commands.obj
 0002:00000e70       ??_7Show_instance_log_files@@6B@ 00000001400e9e70     commands.obj
 0002:00000e84       ??_C@_01GBGANLPD@0?$AA@    00000001400e9e84     commands.obj
 0002:00000e88       ??_C@_08FLCOKHCB@SLOW?5LOG?$AA@ 00000001400e9e88     commands.obj
 0002:00000e98       ??_C@_0M@CKKADIMG@GENERAL?5LOG?$AA@ 00000001400e9e98     commands.obj
 0002:00000ea8       ??_C@_09ILJLBPE@ERROR?5LOG?$AA@ 00000001400e9ea8     commands.obj
 0002:00000eb8       ??_C@_09JPMHFEOD@File?5size?$AA@ 00000001400e9eb8     commands.obj
 0002:00000ec4       ??_C@_04HMIIHGGM@Path?$AA@ 00000001400e9ec4     commands.obj
 0002:00000ed0       ??_C@_07IFPLGDBI@Logfile?$AA@ 00000001400e9ed0     commands.obj
 0002:00000ee8       ??_7Set_option@@6B@        00000001400e9ee8     commands.obj
 0002:00000f20       ??_7Stop_instance@@6B@     00000001400e9f20     commands.obj
 0002:00000f38       ??_C@_0CE@KLOLAHDE@guardian?3?5starting?5instance?5?8?$CFs?8@ 00000001400e9f38     guardian.obj
 0002:00000f68       ??_C@_0CG@PFEDLDCH@guardian?3?5restarting?5instance?5?8?$CF@ 00000001400e9f68     guardian.obj
 0002:00000f98       ??_C@_0DK@BHAMDBAE@guardian?3?5instance?5?8?$CFs?8?5is?5runni@ 00000001400e9f98     guardian.obj
 0002:00000fe0       ??_C@_02KOPDJAMB@?$CC?5?$AA@ 00000001400e9fe0     instance.obj
 0002:00000fe4       ??_C@_01BJJEKLCA@?$CC?$AA@ 00000001400e9fe4     instance.obj
 0002:00000ff0       ??_C@_0HP@LKGFAABM@cannot?5remove?5pidfile?5for?5instan@ 00000001400e9ff0     instance.obj
 0002:00001090       ??_C@_0JC@DPNOFBGO@The?5Instance?5Manager?5was?5able?5to@ 00000001400ea090     instance.obj
 0002:00001140       ??_C@_09IPAEKDAI@localhost?$AA@ 00000001400ea140     instance.obj
 0002:00001150       ??_C@_0BB@GHJAIMGF@check_connection?$AA@ 00000001400ea150     instance.obj
 0002:00001168       ??_C@_0BH@JBEJIMON@MySQL_Instance_Manager?$AA@ 00000001400ea168     instance.obj
 0002:00001188       ??_C@_0BH@KOCPJDOG@Access?5denied?5for?5user?$AA@ 00000001400ea188     instance.obj
 0002:000011a8       ??_C@_0M@LPAKIOHO@ExitProcess?$AA@ 00000001400ea1a8     instance.obj
 0002:000011b8       ??_C@_08HPEMMIEC@Kernel32?$AA@ 00000001400ea1b8     instance.obj
 0002:000011d0       ??_C@_0JG@DJCPAHAF@The?5instance?5?8?$CFs?8?5is?5being?5stopp@ 00000001400ea1d0     instance.obj
 0002:00001288       ??_C@_0BK@BFPPEPOA@starting?5instance?5?8?$CFs?8?4?4?4?$AA@ 00000001400ea288     instance.obj
 0002:000012a8       ??_C@_0DA@NOPFEENC@Instance?3?3start?$CI?$CJ?3?5pthread_creat@ 00000001400ea2a8     instance.obj
 0002:000012ec       ??_C@_06IJHCJAKM@mysqld?$AA@ 00000001400ea2ec     instance_map.obj
 0002:000012f8       ??_C@_0CF@CIPOJFHL@Falling?5back?5to?5compiled?9in?5defa@ 00000001400ea2f8     instance_map.obj
 0002:00001328       ??_C@_0BD@BMHFPFCK@?9?9defaults?9file?$DN?$CFs?$AA@ 00000001400ea328     instance_map.obj
 0002:00001340       ??_C@_0N@MBMMAPDF@mysqlmanager?$AA@ 00000001400ea340     instance_map.obj
 0002:00001350       ??_C@_0CA@PNOFEODE@?5?9?9no?9defaults?5?9?9verbose?5?9?9help?$AA@ 00000001400ea350     instance_options.obj
 0002:00001378       ??_C@_0DF@IIJHIFPH@fill_instance_version?3?5Failed?5to@ 00000001400ea378     instance_options.obj
 0002:000013b8       ??_C@_0BJ@HDFDNOPO@?5?9?9no?9defaults?5?9?9version?$AA@ 00000001400ea3b8     instance_options.obj
 0002:000013d8       ??_C@_0DJ@OGJADNHA@fill_mysqld_real_path?3?5Failed?5to@ 00000001400ea3d8     instance_options.obj
 0002:00001420       ??_C@_09DGMGBAEA@?$FLOPTIONS?$FN?$AA@ 00000001400ea420     instance_options.obj
 0002:00001430       ??_C@_07CKBCDPF@Usage?3?5?$AA@ 00000001400ea430     instance_options.obj
 0002:00001440       ??_C@_0BG@FCNLNJKD@?5?9?9no?9defaults?5?9?9help?$AA@ 00000001400ea440     instance_options.obj
 0002:0000145c       ??_C@_05OLGEOJNI@mysql?$AA@ 00000001400ea45c     instance_options.obj
 0002:00001468       ??_C@_09HGKCAJKI@?9?9datadir?$AA@ 00000001400ea468     instance_options.obj
 0002:00001478       ??_C@_09OFFDPMNL@?9slow?4log?$AA@ 00000001400ea478     instance_options.obj
 0002:00001488       ??_C@_0BD@OPICEAGD@?9?9log?9slow?9queries?$AA@ 00000001400ea488     instance_options.obj
 0002:000014a0       ??_C@_04FPOLKAEB@?4log?$AA@ 00000001400ea4a0     instance_options.obj
 0002:000014a8       ??_C@_05NEJJJKMH@?9?9log?$AA@ 00000001400ea4a8     instance_options.obj
 0002:000014b0       ??_C@_04BKIDJPM@?4err?$AA@ 00000001400ea4b0     instance_options.obj
 0002:000014b8       ??_C@_0M@DHGGKIBL@?9?9log?9error?$AA@ 00000001400ea4b8     instance_options.obj
 0002:000014c8       ??_C@_01KMDKNFGN@?1?$AA@   00000001400ea4c8     instance_options.obj
 0002:000014cc       ??_C@_02IKAHHCAI@?$CFi?$AA@ 00000001400ea4cc     instance_options.obj
 0002:000014d0       ??_C@_0BB@HMNJCLE@?9?9shutdown?9delay?$AA@ 00000001400ea4d0     instance_options.obj
 0002:000014e8       ??_C@_0N@OLKFAOFH@?9?9nonguarded?$AA@ 00000001400ea4e8     instance_options.obj
 0002:000014f8       ??_C@_0P@IPJDFBGE@?9?9mysqld?9path?$DN?$AA@ 00000001400ea4f8     instance_options.obj
 0002:00001510       ??_C@_0M@KMHFJFJJ@?9?9pid?9file?$DN?$AA@ 00000001400ea510     instance_options.obj
 0002:00001520       ??_C@_0BA@DEEPBOIA@?9?9bind?9address?$DN?$AA@ 00000001400ea520     instance_options.obj
 0002:00001538       ??_C@_0L@LCJDMBGN@?9?9datadir?$DN?$AA@ 00000001400ea538     instance_options.obj
 0002:00001548       ??_C@_07LOKCACDF@?9?9port?$DN?$AA@ 00000001400ea548     instance_options.obj
 0002:00001558       ??_C@_09NPCDGEMJ@?9?9socket?$DN?$AA@ 00000001400ea558     instance_options.obj
 0002:00001568       ??_C@_09PGAHDFGH@argv?3?5?$CFs?6?$AA@ 00000001400ea568     instance_options.obj
 0002:00001578       ??_C@_0CD@NLOANHMJ@printing?5out?5an?5instance?5?$CFs?5argv@ 00000001400ea578     instance_options.obj
 0002:000015a4       ??_C@_01JOAMLHOP@?9?$AA@   00000001400ea5a4     instance_options.obj
 0002:000015a8       ??_C@_04GKIEGHBH@?4pid?$AA@ 00000001400ea5a8     instance_options.obj
 0002:000015b0       ??_C@_0O@LNAGOGFC@?9?9no?9defaults?$AA@ 00000001400ea5b0     instance_options.obj
 0002:000015c0       ?LISTEN_BACK_LOG_SIZE@Listener_thread@@0HB 00000001400ea5c0     listener.obj
 0002:000015c8       ??_C@_0CO@ENBOPDEJ@accepting?5connections?5on?5ip?5sock@ 00000001400ea5c8     listener.obj
 0002:00001600       ??_C@_0DF@KMJLFBDJ@Listener_thread?3?3run?$CI?$CJ?3?5listen?$CIi@ 00000001400ea600     listener.obj
 0002:00001640       ??_C@_0DF@LHPONHCM@Listener_thread?3?3run?$CI?$CJ?3?5bind?$CIip?5@ 00000001400ea640     listener.obj
 0002:00001680       ??_C@_0DC@GOJKIMBC@Listener_thead?3?3run?$CI?$CJ?3?5socket?$CIAF@ 00000001400ea680     listener.obj
 0002:000016c0       ??_C@_0EK@BNCDEHPC@handle_one_mysql_connection?$CI?$CJ?3se@ 00000001400ea6c0     listener.obj
 0002:00001718       ??_C@_0DH@NJKJOHPK@Listener_thread?3?3run?$CI?$CJ?3?5shutdown@ 00000001400ea718     listener.obj
 0002:00001760       ??_C@_0CM@GOLGPCHM@Listener_thread?3?3run?$CI?$CJ?3?5select?$CI?$CJ@ 00000001400ea760     listener.obj
 0002:00001798       ??_C@_0DF@HKOKJDHM@Listener?3?5failed?5to?5initialize?4?5@ 00000001400ea798     listener.obj
 0002:000017d8       ??_C@_05JMJKDBEJ@?$CFs?$CFs?6?$AA@ 00000001400ea7d8     log.obj
 0002:000017e0       ??_C@_0CO@EMDKHBOI@log?$CI?$CJ?3?5message?5is?5too?5big?0?5my_ma@ 00000001400ea7e0     log.obj
 0002:00001818       ??_C@_0BM@FGPIOMJK@?$CF02d?$CF02d?$CF02d?5?$CF2d?3?$CF02d?3?$CF02d?7?$AA@ 00000001400ea818     log.obj
 0002:0000183c       ??_C@_01EEMJAFIK@?6?$AA@   00000001400ea83c     log.obj
 0002:00001840       ??_C@_04PFAOODAA@?$CFs?3?5?$AA@ 00000001400ea840     log.obj
 0002:00001848       ??_C@_0CH@BHKFELIG@can?8t?5create?5pid?5file?5?$CFs?3?5errno?$DN@ 00000001400ea848     manager.obj
 0002:00001878       ??_C@_03PMGGPEJJ@?$CFd?6?$AA@ 00000001400ea878     manager.obj
 0002:00001880       ??_C@_0BB@JBMDHFOG@sigwait?$CI?$CJ?5failed?$AA@ 00000001400ea880     manager.obj
 0002:00001898       ??_C@_0DK@CMFIJLOI@manager?$CI?$CJ?3?5set_stacksize_n_creat@ 00000001400ea898     manager.obj
 0002:000018e0       ??_C@_0II@IINGEECN@Cannot?5init?5instances?5repository@ 00000001400ea8e0     manager.obj
 0002:00001988       ??_C@_0DK@OILECFCC@manager?$CI?$CJ?3?5set_stacksize_n_creat@ 00000001400ea988     manager.obj
 0002:000019d0       ??_C@_0BM@EJGDIPGI@IM?5pid?5file?3?5?8?$CFs?8?$DL?5PID?3?5?$CFd?4?$AA@ 00000001400ea9d0     manager.obj
 0002:000019f8       ??_C@_0DH@OLEIDFFJ@Cannot?5open?5the?5option?5file?5to?5e@ 00000001400ea9f8     messages.obj
 0002:00001a40       ??_C@_0FE@PBJNMGMK@Cannot?5guess?5the?5log?5filename?4?5T@ 00000001400eaa40     messages.obj
 0002:00001aa8       ??_C@_0BF@CCAMAPAA@Cannot?5open?5log?5file?$AA@ 00000001400eaaa8     messages.obj
 0002:00001ac8       ??_C@_0CF@HGFDHMPH@The?5instance?5has?5no?5such?5log?5ena@ 00000001400eaac8     messages.obj
 0002:00001af8       ??_C@_0CK@BDCIGLMK@Cannot?5read?5requested?5part?5of?5th@ 00000001400eaaf8     messages.obj
 0002:00001b30       ??_C@_0BF@BOFNNLAC@Cannot?5stop?5instance?$AA@ 00000001400eab30     messages.obj
 0002:00001b50       ??_C@_0CF@EPBEMJMO@Cannot?5read?5negative?5number?5of?5b@ 00000001400eab50     messages.obj
 0002:00001b80       ??_C@_0FJ@FAEFAGFE@Cannot?5start?5instance?4?5Possible?5@ 00000001400eab80     messages.obj
 0002:00001bf0       ??_C@_0CA@OIEOKEDL@The?5instance?5is?5already?5started?$AA@ 00000001400eabf0     messages.obj
 0002:00001c20       ??_C@_0HD@GGDAMBEA@Cannot?5stop?5instance?4?5Perhaps?5th@ 00000001400eac20     messages.obj
 0002:00001cb0       ??_C@_0ED@IPKHLHCN@Bad?5instance?5name?4?5Check?5that?5th@ 00000001400eacb0     messages.obj
 0002:00001d00       ??_C@_0IP@BELLFNGA@You?5have?5an?5error?5in?5your?5comman@ 00000001400ead00     messages.obj
 0002:00001db0       ??_C@_0BA@MPOJHAMO@Unknown?5command?$AA@ 00000001400eadb0     messages.obj
 0002:00001dd0       ??_C@_0GF@CPHLBCPM@Client?5does?5not?5support?5authenti@ 00000001400eadd0     messages.obj
 0002:00001e50       ??_C@_0CK@DOCEONGH@Access?5denied?4?5Bad?5username?1pass@ 00000001400eae50     messages.obj
 0002:00001e90       ??_C@_0LH@OBGNHNPK@Out?5of?5memory?$DL?5?5Check?5if?5mysqld?5@ 00000001400eae90     messages.obj
 0002:00001f70       ??_C@_0O@DIOIANKF@Bad?5handshake?$AA@ 00000001400eaf70     messages.obj
 0002:00001f80       ??_C@_0CP@BJKIJCH@query?5for?5connection?5?$CFlu?5receive@ 00000001400eaf80     mysql_connection.obj
 0002:00001fb8       ??_C@_0CJ@LMHBIBIE@query?5for?5connection?5?$CFlu?5execute@ 00000001400eafb8     mysql_connection.obj
 0002:00001ff0       ??_C@_0CF@BKMEOAHD@query?5for?5connection?5?$CFlu?5execute@ 00000001400eaff0     mysql_connection.obj
 0002:00002020       ??_C@_0CO@HBIOCLGM@query?5for?5connection?5?$CFlu?5success@ 00000001400eb020     mysql_connection.obj
 0002:00002058       ??_C@_0DN@KOGIBOEA@query?5for?5connection?5?$CFlu?5?3?5?9?9?9?9?6@ 00000001400eb058     mysql_connection.obj
 0002:000020a8       ??_C@_0CP@DALMNPLH@query?5for?5connection?5?$CFlu?5receive@ 00000001400eb0a8     mysql_connection.obj
 0002:000020e0       ??_C@_0DC@HELMMJKC@query?5for?5connection?5?$CFlu?5receive@ 00000001400eb0e0     mysql_connection.obj
 0002:00002120       ??_C@_0CO@KLKKOBCE@connection?5?$CFlu?3?5packet_length?$DN?$CFl@ 00000001400eb120     mysql_connection.obj
 0002:00002158       ??_C@_0CH@PBJKGPOJ@connection?5?$CFlu?5is?5checked?5succes@ 00000001400eb158     mysql_connection.obj
 0002:00002188       ??_C@_0BO@LOPJDLBA@accepted?5mysql?5connection?5?$CFlu?$AA@ 00000001400eb188     mysql_connection.obj
 0002:000021b0       ??_C@_0CO@FMCLIPDB@mysql_connection?$CI?$CJ?3?5error?5initia@ 00000001400eb1b0     mysql_connection.obj
 0002:000021e8       ??_C@_07JPLKDPHP@manager?$AA@ 00000001400eb1e8     options.obj
 0002:00002200       ??_C@_0EP@PDDIBNOH@The?5number?5of?5seconds?5IM?5waits?5f@ 00000001400eb200     options.obj
 0002:00002260       ??_C@_0N@IKNOIIJE@wait?9timeout?$AA@ 00000001400eb260     options.obj
 0002:00002270       ??_C@_0CF@PMNNCCFJ@Output?5version?5information?5and?5e@ 00000001400eb270     options.obj
 0002:000022a0       ??_C@_0CJ@IONBCKIB@Run?5the?5application?5in?5stand?5alo@ 00000001400eb2a0     options.obj
 0002:000022d8       ??_C@_0L@FLHGMILF@standalone?$AA@ 00000001400eb2d8     options.obj
 0002:000022e8       ??_C@_0BH@DMOGDMLA@Remove?5system?5service?4?$AA@ 00000001400eb2e8     options.obj
 0002:00002304       ??_C@_06LEMKAMD@remove?$AA@ 00000001400eb304     options.obj
 0002:00002310       ??_C@_0BL@KHPAFIOP@Install?5as?5system?5service?4?$AA@ 00000001400eb310     options.obj
 0002:00002330       ??_C@_07EALBDFH@install?$AA@ 00000001400eb330     options.obj
 0002:00002340       ??_C@_0CK@FMEHMJFO@Interval?5to?5monitor?5instances?5in@ 00000001400eb340     options.obj
 0002:00002378       ??_C@_0BE@INENLLN@monitoring?9interval?$AA@ 00000001400eb378     options.obj
 0002:00002390       ??_C@_0CH@LIAINEMB@Where?5to?5look?5for?5MySQL?5Server?5b@ 00000001400eb390     options.obj
 0002:000023c0       ??_C@_0BE@HCHLGHAI@default?9mysqld?9path?$AA@ 00000001400eb3c0     options.obj
 0002:000023d8       ??_C@_0DE@HMCHLBBP@Look?5for?5Instance?5Manager?5users?5@ 00000001400eb3d8     options.obj
 0002:00002418       ??_C@_0O@JHLAPOPF@password?9file?$AA@ 00000001400eb418     options.obj
 0002:00002428       ??_C@_0CD@MHHOJIKI@Port?5number?5to?5use?5for?5connectio@ 00000001400eb428     options.obj
 0002:00002454       ??_C@_04LPGMAPLE@port?$AA@ 00000001400eb454     options.obj
 0002:00002460       ??_C@_0CE@LKPLDHBK@Bind?5address?5to?5use?5for?5connecti@ 00000001400eb460     options.obj
 0002:00002490       ??_C@_0N@KPFNDBAM@bind?9address?$AA@ 00000001400eb490     options.obj
 0002:000024a0       ??_C@_0CI@LGIDHNND@Prepare?5entry?5for?5passwd?5file?5an@ 00000001400eb4a0     options.obj
 0002:000024d0       ??_C@_06NKIEGJEO@passwd?$AA@ 00000001400eb4d0     options.obj
 0002:000024d8       ??_C@_0BB@DGOMPFMC@Pid?5file?5to?5use?4?$AA@ 00000001400eb4d8     options.obj
 0002:000024f0       ??_C@_08OLCBHKMI@pid?9file?$AA@ 00000001400eb4f0     options.obj
 0002:00002500       ??_C@_0DD@PCDFCKMG@Path?5to?5log?5file?4?5Used?5only?5with@ 00000001400eb500     options.obj
 0002:00002540       ??_C@_03MGHMBJCF@log?$AA@  00000001400eb540     options.obj
 0002:00002548       ??_C@_0BM@BKPKLHCC@Display?5this?5help?5and?5exit?4?$AA@ 00000001400eb548     options.obj
 0002:0000256c       ??_C@_04PCJFHION@help?$AA@ 00000001400eb56c     options.obj
 0002:00002578       ??_C@_0L@MFNJLFIO@?4angel?4pid?$AA@ 00000001400eb578     options.obj
 0002:00002588       ??_C@_0BE@FKMKPPAN@DEFAULT_MYSQLD_PATH?$AA@ 00000001400eb588     options.obj
 0002:000025a0       ??_C@_0BG@GNGCPKDM@DEFAULT_PID_FILE_NAME?$AA@ 00000001400eb5a0     options.obj
 0002:000025d0       ??_C@_0BI@DFCIJINN@?$CFs?5Ver?5?$CFs?5for?5?$CFs?5on?5?$CFs?6?$AA@ 00000001400eb5d0     options.obj
 0002:000025ec       ??_C@_05ILKBJJMK@Win64?$AA@ 00000001400eb5ec     options.obj
 0002:00002600       ??_C@_0BHM@GIOFNEGN@?6The?5following?5options?5may?5be?5gi@ 00000001400eb600     options.obj
 0002:000027c8       ??_C@_0BG@GNEAPHGE@Usage?3?5?$CFs?5?$FLOPTIONS?$FN?5?6?$AA@ 00000001400eb7c8     options.obj
 0002:000027f0       ??_C@_0MP@IAOBOCIK@Copyright?5?$CIC?$CJ?52003?92007?5MySQL?5AB@ 00000001400eb7f0     options.obj
 0002:000028e8       ??_C@_06KCIFIIHN@?$CFs?3?$CFs?6?$AA@ 00000001400eb8e8     options.obj
 0002:000028f0       ??_C@_0CA@GHLPBOBI@Sorry?0?5passwords?5do?5not?5match?4?6?$AA@ 00000001400eb8f0     options.obj
 0002:00002918       ??_C@_0BG@FABKDGBO@Unable?5to?5read?5user?4?6?$AA@ 00000001400eb918     options.obj
 0002:00002938       ??_C@_0BC@DEAECJAP@Enter?5user?5name?3?5?$AA@ 00000001400eb938     options.obj
 0002:00002950       ??_C@_0BP@NJIBNPLM@Creating?5record?5for?5new?5user?4?6?$AA@ 00000001400eb950     options.obj
 0002:00002978       ??_C@_0BD@NKGLHMFK@Re?9type?5password?3?5?$AA@ 00000001400eb978     options.obj
 0002:00002990       ??_C@_0BB@LAEJCAEB@Enter?5password?3?5?$AA@ 00000001400eb990     options.obj
 0002:000029a4       ??_C@_04JLMDILM@?4exe?$AA@ 00000001400eb9a4     options.obj
 0002:000029b0       ??_C@_0GN@NBIDIJLJ@The?5?9?9defaults?9extra?9file?5and?5?9?9@ 00000001400eb9b0     options.obj
 0002:00002a38       ??_C@_0BH@HNKMCPPG@?9?9defaults?9extra?9file?$DN?$AA@ 00000001400eba38     options.obj
 0002:00002a58       ??_C@_0BB@LDHKPEKC@?9?9defaults?9file?$DN?$AA@ 00000001400eba58     options.obj
 0002:00002a6c       ??_C@_05IEIDFGAH@UNSET?$AA@ 00000001400eba6c     parse.obj
 0002:00002a74       ??_C@_04JGPCMMEF@SHOW?$AA@ 00000001400eba74     parse.obj
 0002:00002a7c       ??_C@_04MDHMLCKF@STOP?$AA@ 00000001400eba7c     parse.obj
 0002:00002a84       ??_C@_06DNKMJCIK@STATUS?$AA@ 00000001400eba84     parse.obj
 0002:00002a8c       ??_C@_05JLPDBANI@START?$AA@ 00000001400eba8c     parse.obj
 0002:00002a94       ??_C@_04BJJAFLBC@SLOW?$AA@ 00000001400eba94     parse.obj
 0002:00002a9c       ??_C@_03KPIFFHNE@SET?$AA@  00000001400eba9c     parse.obj
 0002:00002aa0       ??_C@_07KDKMIPIP@OPTIONS?$AA@ 00000001400ebaa0     parse.obj
 0002:00002aac       ??_C@_03MLIHNEFJ@LOG?$AA@  00000001400ebaac     parse.obj
 0002:00002ab0       ??_C@_09CJBINDHJ@INSTANCES?$AA@ 00000001400ebab0     parse.obj
 0002:00002ac0       ??_C@_08DDHIOBDH@INSTANCE?$AA@ 00000001400ebac0     parse.obj
 0002:00002ad0       ??_C@_07EGGHCNEO@GENERAL?$AA@ 00000001400ebad0     parse.obj
 0002:00002adc       ??_C@_05KALGKIBB@FLUSH?$AA@ 00000001400ebadc     parse.obj
 0002:00002ae4       ??_C@_05PENKCLCM@FILES?$AA@ 00000001400ebae4     parse.obj
 0002:00002aec       ??_C@_05MBDEGLCK@ERROR?$AA@ 00000001400ebaec     parse.obj
 0002:00002b00       ??_7Show_instances@@6B@    00000001400ebb00     parse.obj
 0002:00002b20       ??_7Flush_instances@@6B@   00000001400ebb20     parse.obj
 0002:00002b40       ??_7Syntax_error@@6B@      00000001400ebb40     parse.obj
 0002:00002b60       ??_7Unset_option@@6B@      00000001400ebb60     parse.obj
 0002:00002b80       ??_C@_01KDCPPGHE@r?$AA@    00000001400ebb80     parse_output.obj
 0002:00002b88       ?mysqlmanager_version@@3QBDB 00000001400ebb88     priv.obj
 0002:00002b92       ?protocol_version@@3EB     00000001400ebb92     priv.obj
 0002:00002b94       ?mysqlmanager_version_length@@3HB 00000001400ebb94     priv.obj
 0002:00002ba0       ??_C@_0CL@EMLLAKPP@error?5parsing?5user?5and?5password?5@ 00000001400ebba0     user_map.obj
 0002:00002bd8       ??_C@_0P@OFMBKLL@loaded?5user?5?$CFs?$AA@ 00000001400ebbd8     user_map.obj
 0002:00002bf0       ??_C@_0DE@NNMOOOEE@?$FLWARNING?$FN?5can?8t?5open?5password?5fi@ 00000001400ebbf0     user_map.obj
 0002:00002c38       ??_7IMService@@6B@         00000001400ebc38     IMService.obj
 0002:00002c78       ??_C@_0O@ONNFOFNE@MySQL?5Manager?$AA@ 00000001400ebc78     IMService.obj
 0002:00002c88       ??_C@_0N@NFIKJEB@MySqlManager?$AA@ 00000001400ebc88     IMService.obj
 0002:00002c98       ??_C@_0BJ@FAGHJNJN@Service?5failed?5to?5remove?$AA@ 00000001400ebc98     IMService.obj
 0002:00002cb8       ??_C@_0BN@CIDKMPML@Service?5removed?5successfully?$AA@ 00000001400ebcb8     IMService.obj
 0002:00002ce0       ??_C@_0BJ@FCKPKBPE@Service?5is?5not?5installed?$AA@ 00000001400ebce0     IMService.obj
 0002:00002d00       ??_C@_0BK@IIIDEEJJ@Service?5failed?5to?5install?$AA@ 00000001400ebd00     IMService.obj
 0002:00002d20       ??_C@_0BP@PFCIEMND@Service?5installed?5successfully?$AA@ 00000001400ebd20     IMService.obj
 0002:00002d48       ??_C@_0BN@DCHLHDND@Service?5is?5already?5installed?$AA@ 00000001400ebd48     IMService.obj
 0002:00002d78       ??_7WindowsService@@6B@    00000001400ebd78     WindowsService.obj
 0002:00002db8       ??_C@_0BE@GPLHKCHK@ReportStatus?5failed?$AA@ 00000001400ebdb8     WindowsService.obj
 0002:00002dd0       ??_C@_0L@KDJOJLDL@?$CF08lx?$CF08lx?$AA@ 00000001400ebdd0     password.obj
 0002:00002de0       __real@4050000000000000    00000001400ebde0     password.obj
 0002:00002df0       __real@403f000000000000    00000001400ebdf0     password.obj
 0002:00002e00       __real@4040800000000000    00000001400ebe00     password.obj
 0002:00002e10       __real@4057800000000000    00000001400ebe10     password.obj
 0002:00002e1c       ??_C@_05EKPPILBK@XA102?$AA@ 00000001400ebe1c     sql_state.obj
 0002:00002e24       ??_C@_05COJDEOBO@XA106?$AA@ 00000001400ebe24     sql_state.obj
 0002:00002e2c       ??_C@_05BPLBLCNG@22008?$AA@ 00000001400ebe2c     sql_state.obj
 0002:00002e34       ??_C@_05FEENFEFL@XAE08?$AA@ 00000001400ebe34     sql_state.obj
 0002:00002e3c       ??_C@_05MOHDAJJP@22001?$AA@ 00000001400ebe3c     sql_state.obj
 0002:00002e44       ??_C@_05HIMJOJJI@XA100?$AA@ 00000001400ebe44     sql_state.obj
 0002:00002e4c       ??_C@_05LHLJINJA@XAE03?$AA@ 00000001400ebe4c     sql_state.obj
 0002:00002e54       ??_C@_05ENFGGFBK@XAE09?$AA@ 00000001400ebe54     sql_state.obj
 0002:00002e5c       ??_C@_05NDNFEIJE@XAE07?$AA@ 00000001400ebe5c     sql_state.obj
 0002:00002e64       ??_C@_05OBODCKBG@XAE05?$AA@ 00000001400ebe64     sql_state.obj
 0002:00002e6c       ??_C@_05PIPIBLFH@XAE04?$AA@ 00000001400ebe6c     sql_state.obj
 0002:00002e74       ??_C@_05OEJMDAGL@22012?$AA@ 00000001400ebe74     sql_state.obj
 0002:00002e7c       ??_C@_05KNKIGLLO@20000?$AA@ 00000001400ebe7c     sql_state.obj
 0002:00002e84       ??_C@_05JKKAJJNF@02000?$AA@ 00000001400ebe84     sql_state.obj
 0002:00002e8c       ??_C@_05FICIMNHO@24000?$AA@ 00000001400ebe8c     sql_state.obj
 0002:00002e94       ??_C@_05KGENIKJE@2F005?$AA@ 00000001400ebe94     sql_state.obj
 0002:00002e9c       ??_C@_05EFNJJNGI@70100?$AA@ 00000001400ebe9c     sql_state.obj
 0002:00002ea4       ??_C@_05CENCADMK@0A000?$AA@ 00000001400ebea4     sql_state.obj
 0002:00002eac       ??_C@_05PABHCNBC@2F003?$AA@ 00000001400ebeac     sql_state.obj
 0002:00002eb4       ??_C@_05JICJKOBJ@22007?$AA@ 00000001400ebeb4     sql_state.obj
 0002:00002ebc       ??_C@_05PMEFGLBN@22003?$AA@ 00000001400ebebc     sql_state.obj
 0002:00002ec4       ??_C@_05NNAAODAF@01000?$AA@ 00000001400ebec4     sql_state.obj
 0002:00002ecc       ??_C@_05JAMIECAO@21000?$AA@ 00000001400ebecc     sql_state.obj
 0002:00002ed4       ??_C@_05GCOKLJOC@40001?$AA@ 00000001400ebed4     sql_state.obj
 0002:00002edc       ??_C@_05GFEIOEMO@25000?$AA@ 00000001400ebedc     sql_state.obj
 0002:00002ee4       ??_C@_05LDAEPNNK@22004?$AA@ 00000001400ebee4     sql_state.obj
 0002:00002eec       ??_C@_05BLFGILJL@42S12?$AA@ 00000001400ebeec     sql_state.obj
 0002:00002ef4       ??_C@_05DCDNGGAB@42S21?$AA@ 00000001400ebef4     sql_state.obj
 0002:00002efc       ??_C@_05KAEACLKC@21S01?$AA@ 00000001400ebefc     sql_state.obj
 0002:00002f04       ??_C@_05ICKCCFLI@S1009?$AA@ 00000001400ebf04     sql_state.obj
 0002:00002f0c       ??_C@_05FPLCABKN@S0022?$AA@ 00000001400ebf0c     sql_state.obj
 0002:00002f14       ??_C@_05BJBADFMC@42S22?$AA@ 00000001400ebf14     sql_state.obj
 0002:00002f1c       ??_C@_05BKJEOBKM@42S02?$AA@ 00000001400ebf1c     sql_state.obj
 0002:00002f24       ??_C@_05DBLJLCGP@42S01?$AA@ 00000001400ebf24     sql_state.obj
 0002:00002f2c       ??_C@_05GKKGPOBE@3D000?$AA@ 00000001400ebf2c     sql_state.obj
 0002:00002f34       ??_C@_05JNNICAHP@28000?$AA@ 00000001400ebf34     sql_state.obj
 0002:00002f3c       ??_C@_05BDBNLMD@42000?$AA@ 00000001400ebf3c     sql_state.obj
 0002:00002f44       ??_C@_05OAJIOINI@08S01?$AA@ 00000001400ebf44     sql_state.obj
 0002:00002f4c       ??_C@_05LEHMEEHA@08004?$AA@ 00000001400ebf4c     sql_state.obj
 0002:00002f54       ??_C@_05EKHLKPLA@S1001?$AA@ 00000001400ebf54     sql_state.obj
 0002:00002f5c       ??_C@_05IKCIGBGE@HY001?$AA@ 00000001400ebf5c     sql_state.obj
 0002:00002f64       ??_C@_05OKAIBBGO@23000?$AA@ 00000001400ebf64     sql_state.obj
 0002:00002f6c       ??_C@_05JDDDFACF@HY000?$AA@ 00000001400ebf6c     sql_state.obj
 0002:00002f74       ??_C@_06HPIPGHLH@MEMORY?$AA@ 00000001400ebf74     client.obj
 0002:00002f7c       ??_C@_04GGAEFGO@PIPE?$AA@  00000001400ebf7c     client.obj
 0002:00002f84       ??_C@_06HFGAEBMM@SOCKET?$AA@ 00000001400ebf84     client.obj
 0002:00002f8c       ??_C@_03FCLDNGNL@TCP?$AA@  00000001400ebf8c     client.obj
 0002:00002f90       ??_C@_07FOPBDDAL@options?$AA@ 00000001400ebf90     client.obj
 0002:00002fa0       ??_C@_0BH@BONNBGIA@report?9data?9truncation?$AA@ 00000001400ebfa0     client.obj
 0002:00002fc0       ??_C@_0M@PMDPKFDA@secure?9auth?$AA@ 00000001400ebfc0     client.obj
 0002:00002fd0       ??_C@_0O@IGPGCENI@multi?9queries?$AA@ 00000001400ebfd0     client.obj
 0002:00002fe0       ??_C@_0BB@ECMBLIEH@multi?9statements?$AA@ 00000001400ebfe0     client.obj
 0002:00002ff8       ??_C@_0O@CCDCLLBG@multi?9results?$AA@ 00000001400ebff8     client.obj
 0002:00003008       ??_C@_0BI@FOKNPLJP@shared?9memory?9base?9name?$AA@ 00000001400ec008     client.obj
 0002:00003028       ??_C@_08FCFPNNHF@protocol?$AA@ 00000001400ec028     client.obj
 0002:00003038       ??_C@_0BD@OFGLABCB@max?9allowed?9packet?$AA@ 00000001400ec038     client.obj
 0002:00003050       ??_C@_0L@PHBCGEDL@ssl?9cipher?$AA@ 00000001400ec050     client.obj
 0002:00003060       ??_C@_0BB@HNHJLDBF@repl?9parse?9query?$AA@ 00000001400ec060     client.obj
 0002:00003078       ??_C@_0BJ@JAEAFHJM@enable?9reads?9from?9master?$AA@ 00000001400ec078     client.obj
 0002:00003098       ??_C@_0BC@BKIPLOIH@replication?9probe?$AA@ 00000001400ec098     client.obj
 0002:000030b0       ??_C@_0BF@DNHMICAO@disable?9local?9infile?$AA@ 00000001400ec0b0     client.obj
 0002:000030d0       ??_C@_0N@DEPIEDDP@local?9infile?$AA@ 00000001400ec0d0     client.obj
 0002:000030e0       ??_C@_0BA@PKFDCPCI@connect?9timeout?$AA@ 00000001400ec0e0     client.obj
 0002:000030f8       ??_C@_0BE@PKKGFOHM@interactive?9timeout?$AA@ 00000001400ec0f8     client.obj
 0002:00003110       ??_C@_0BG@BMMCDGOA@default?9character?9set?$AA@ 00000001400ec110     client.obj
 0002:00003130       ??_C@_0BD@HPLEKGGN@character?9sets?9dir?$AA@ 00000001400ec130     client.obj
 0002:00003148       ??_C@_0L@MLIAJKEA@ssl?9capath?$AA@ 00000001400ec148     client.obj
 0002:00003158       ??_C@_06KEIFHGI@ssl?9ca?$AA@ 00000001400ec158     client.obj
 0002:00003160       ??_C@_08MLGPLICL@ssl?9cert?$AA@ 00000001400ec160     client.obj
 0002:00003170       ??_C@_07HPCDODLB@ssl?9key?$AA@ 00000001400ec170     client.obj
 0002:00003180       ??_C@_0BC@CPNNNMD@return?9found?9rows?$AA@ 00000001400ec180     client.obj
 0002:00003198       ??_C@_05GFCDIDHO@debug?$AA@ 00000001400ec198     client.obj
 0002:000031a0       ??_C@_08PBOCEOLL@database?$AA@ 00000001400ec1a0     client.obj
 0002:000031ac       ??_C@_04OODOLJMA@host?$AA@ 00000001400ec1ac     client.obj
 0002:000031b8       ??_C@_0N@CJBLNCLF@init?9command?$AA@ 00000001400ec1b8     client.obj
 0002:000031c8       ??_C@_04CCHAHKJA@user?$AA@ 00000001400ec1c8     client.obj
 0002:000031d0       ??_C@_07DDHNKDGP@timeout?$AA@ 00000001400ec1d0     client.obj
 0002:000031dc       ??_C@_04MKFKKHBG@pipe?$AA@ 00000001400ec1dc     client.obj
 0002:000031e8       ??_C@_08NLHBPEGP@password?$AA@ 00000001400ec1e8     client.obj
 0002:000031f8       ??_C@_08EJNPIMGB@compress?$AA@ 00000001400ec1f8     client.obj
 0002:00003204       ??_C@_06HBELJPBO@socket?$AA@ 00000001400ec204     client.obj
 0002:0000320c       ??_C@_05MJALLADF@08001?$AA@ 00000001400ec20c     client.obj
 0002:00003214       ??_C@_05OAGAMKLF@00000?$AA@ 00000001400ec214     client.obj
 0002:0000321c       ??_C@_02HDBGODGB@?2?2?$AA@ 00000001400ec21c     client.obj
 0002:00003220       ??_C@_06CKMLAALA@?2pipe?2?$AA@ 00000001400ec220     client.obj
 0002:00003228       ??_C@_01LFCBOECM@?4?$AA@   00000001400ec228     client.obj
 0002:00003230       ??_C@_0L@MKBJOBHN@Windows_NT?$AA@ 00000001400ec230     client.obj
 0002:00003240       ??_C@_02OKOOOCIH@OS?$AA@   00000001400ec240     client.obj
 0002:00003248       ??_C@_0CA@ONJAFPFC@Unknown?5option?5to?5protocol?3?5?$CFs?6?$AA@ 00000001400ec248     client.obj
 0002:00003270       ??_C@_06DGDLPBAN@client?$AA@ 00000001400ec270     client.obj
 0002:00003278       ??_C@_04ODABKPJA@?1CN?$DN?$AA@ 00000001400ec278     client.obj
 0002:00003280       ??_C@_0CP@EINHLMKL@COLLATION?5?$CFs?5is?5not?5valid?5for?5CH@ 00000001400ec280     client.obj
 0002:000032b8       ??_C@_0BC@BNNCKLMG@latin1_swedish_ci?$AA@ 00000001400ec2b8     client.obj
 0002:000032d0       ??_C@_06CDEFMFPB@latin1?$AA@ 00000001400ec2d0     client.obj
 0002:000032d8       ??_C@_0N@HAKKOMP@SET?5NAMES?5?$CFs?$AA@ 00000001400ec2d8     client.obj
 0002:000032e8       ??_C@_0CD@CIHNPOGB@sending?5authentication?5informati@ 00000001400ec2e8     client.obj
 0002:00003318       ??_C@_0BJ@EDEHFNCE@Setting?5intital?5database?$AA@ 00000001400ec318     client.obj
 0002:00003338       ??_C@_0BN@NHONKCFH@sending?5password?5information?$AA@ 00000001400ec338     client.obj
 0002:00003360       ??_C@_0CC@FOKDGKNL@reading?5final?5connect?5informatio@ 00000001400ec360     client.obj
 0002:00003388       ??_C@_0BN@IKPBBPKC@reading?5authorization?5packet?$AA@ 00000001400ec388     client.obj
 0002:000033b0       ??_C@_0CJ@OKBDLPBM@sending?5connection?5information?5t@ 00000001400ec3b0     client.obj
 0002:000033e8       ??_C@_0CF@JIJHEKCB@reading?5initial?5communication?5pa@ 00000001400ec3e8     client.obj
 0002:00003418       ??_C@_0CJ@GFOPAJCF@waiting?5for?5initial?5communicatio@ 00000001400ec418     client.obj
 0002:0000344c       ??_C@_05OBDDCBJC@MySQL?$AA@ 00000001400ec44c     client.obj
 0002:00003454       ??_C@_02LOEMLMCB@my?$AA@   00000001400ec454     client.obj
 0002:00003458       ??_C@_01NBENCBCI@?$CK?$AA@ 00000001400ec458     get_password.obj
 0002:0000345c       ??_C@_03OLJLMEOE@?$AI?5?$AI?$AA@ 00000001400ec45c     get_password.obj
 0002:00003460       ??_C@_0DK@NDNCLJNI@Lost?5connection?5to?5MySQL?5server?5@ 00000001400ec460     errmsg.obj
 0002:000034a8       ??_C@_0CE@HBOGEKGA@This?5feature?5is?5not?5implemented?5@ 00000001400ec4a8     errmsg.obj
 0002:000034e0       ??_C@_0FB@FBBFBAHN@Attempt?5to?5read?5a?5row?5while?5ther@ 00000001400ec4e0     errmsg.obj
 0002:00003548       ??_C@_0CI@HALOFLAE@Prepared?5statement?5contains?5no?5m@ 00000001400ec548     errmsg.obj
 0002:00003578       ??_C@_0CP@CONJDJBD@Attempt?5to?5read?5column?5without?5p@ 00000001400ec578     errmsg.obj
 0002:000035b0       ??_C@_0DG@NCJJHECB@Row?5retrieval?5was?5canceled?5by?5my@ 00000001400ec5b0     errmsg.obj
 0002:000035f0       ??_C@_0GH@LCEGFGKM@Connection?5using?5old?5?$CIpre?94?41?41?$CJ@ 00000001400ec5f0     errmsg.obj
 0002:00003670       ??_C@_0BK@JMIMHFDF@Invalid?5connection?5handle?$AA@ 00000001400ec670     errmsg.obj
 0002:00003690       ??_C@_0BK@GLFMEDLO@Wrong?5or?5unknown?5protocol?$AA@ 00000001400ec690     errmsg.obj
 0002:000036b0       ??_C@_0EE@IPCCLOKB@Can?8t?5open?5shared?5memory?$DL?5cannot@ 00000001400ec6b0     errmsg.obj
 0002:00003708       ??_C@_0DG@KGBHPOJD@Can?8t?5open?5shared?5memory?$DL?5no?5ans@ 00000001400ec708     errmsg.obj
 0002:00003750       ??_C@_0EB@MDFKCBGN@Can?8t?5open?5shared?5memory?$DL?5client@ 00000001400ec750     errmsg.obj
 0002:000037a0       ??_C@_0EN@FCGLLCJK@Can?8t?5open?5shared?5memory?$DL?5client@ 00000001400ec7a0     errmsg.obj
 0002:00003800       ??_C@_0EH@LNAOKCEE@Can?8t?5open?5shared?5memory?$DL?5client@ 00000001400ec800     errmsg.obj
 0002:00003860       ??_C@_0EN@PMIKFHIB@Can?8t?5open?5shared?5memory?$DL?5server@ 00000001400ec860     errmsg.obj
 0002:000038c0       ??_C@_0EH@KCLOIILK@Can?8t?5open?5shared?5memory?$DL?5server@ 00000001400ec8c0     errmsg.obj
 0002:00003920       ??_C@_0EF@KIGDFHBB@Can?8t?5open?5shared?5memory?$DL?5no?5ans@ 00000001400ec920     errmsg.obj
 0002:00003980       ??_C@_0EG@BEPMLGLN@Can?8t?5open?5shared?5memory?$DL?5client@ 00000001400ec980     errmsg.obj
 0002:000039d8       ??_C@_0BH@OHMIMHCN@Shared?5memory?3?5?$CF?9?4100s?$AA@ 00000001400ec9d8     errmsg.obj
 0002:000039f8       ??_C@_0DD@HBOCKDGH@Using?5unsupported?5buffer?5type?3?5?$CF@ 00000001400ec9f8     errmsg.obj
 0002:00003a40       ??_C@_0EK@GGAINION@Can?8t?5send?5long?5data?5for?5non?9str@ 00000001400eca40     errmsg.obj
 0002:00003a98       ??_C@_0BJ@LEKCEENG@Invalid?5parameter?5number?$AA@ 00000001400eca98     errmsg.obj
 0002:00003ab8       ??_C@_0CF@OAFCOHEP@No?5parameters?5exist?5in?5the?5state@ 00000001400ecab8     errmsg.obj
 0002:00003ae8       ??_C@_0P@KJHDOAKM@Data?5truncated?$AA@ 00000001400ecae8     errmsg.obj
 0002:00003b00       ??_C@_0DG@PGNJOEPP@No?5data?5supplied?5for?5parameters?5@ 00000001400ecb00     errmsg.obj
 0002:00003b40       ??_C@_0BH@OCBFPEOC@Statement?5not?5prepared?$AA@ 00000001400ecb40     errmsg.obj
 0002:00003b60       ??_C@_0BM@EEGCMMPG@Invalid?5use?5of?5null?5pointer?$AA@ 00000001400ecb60     errmsg.obj
 0002:00003b90       ??_C@_0FE@HLHPGJMI@This?5client?5library?5is?5licensed?5@ 00000001400ecb90     errmsg.obj
 0002:00003bf8       ??_C@_0BB@DAKKIOKN@Malformed?5packet?$AA@ 00000001400ecbf8     errmsg.obj
 0002:00003c10       ??_C@_0BF@GNKPEKCC@SSL?5connection?5error?$AA@ 00000001400ecc10     errmsg.obj
 0002:00003c30       ??_C@_0BM@DBHHCLGE@Error?5connecting?5to?5master?3?$AA@ 00000001400ecc30     errmsg.obj
 0002:00003c58       ??_C@_0BL@NMFPGPDF@Error?5connecting?5to?5slave?3?$AA@ 00000001400ecc58     errmsg.obj
 0002:00003c78       ??_C@_0BL@BDOEBOAG@Error?5on?5SHOW?5SLAVE?5HOSTS?3?$AA@ 00000001400ecc78     errmsg.obj
 0002:00003c98       ??_C@_0BM@KEKCHGPI@Error?5on?5SHOW?5SLAVE?5STATUS?3?$AA@ 00000001400ecc98     errmsg.obj
 0002:00003cc0       ??_C@_0BA@JILIEPGI@Embedded?5server?$AA@ 00000001400eccc0     errmsg.obj
 0002:00003cd8       ??_C@_0DC@PLGHDHHE@Got?5packet?5bigger?5than?5?8max_allo@ 00000001400eccd8     errmsg.obj
 0002:00003d18       ??_C@_0DG@MMIKLOLE@Can?8t?5initialize?5character?5set?5?$CF@ 00000001400ecd18     errmsg.obj
 0002:00003d60       ??_C@_0EC@JBHOMNCI@Can?8t?5set?5state?5of?5named?5pipe?5to@ 00000001400ecd60     errmsg.obj
 0002:00003db0       ??_C@_0DK@DGFLNGLM@Can?8t?5open?5named?5pipe?5to?5host?3?5?$CF@ 00000001400ecdb0     errmsg.obj
 0002:00003df8       ??_C@_0DO@MCIKAJJD@Can?8t?5wait?5for?5named?5pipe?5to?5hos@ 00000001400ecdf8     errmsg.obj
 0002:00003e48       ??_C@_0BD@MONBAMLI@Named?5pipe?3?5?$CF?9?432s?$AA@ 00000001400ece48     errmsg.obj
 0002:00003e60       ??_C@_0DF@GGAOFKDM@Commands?5out?5of?5sync?$DL?5you?5can?8t?5@ 00000001400ece60     errmsg.obj
 0002:00003ea0       ??_C@_0CN@MCPHLMHK@Lost?5connection?5to?5MySQL?5server?5@ 00000001400ecea0     errmsg.obj
 0002:00003ed8       ??_C@_0BK@OPFAEJOB@Error?5in?5server?5handshake?$AA@ 00000001400eced8     errmsg.obj
 0002:00003ef8       ??_C@_0BD@JHCOEEJ@?$CF?9?4100s?5via?5TCP?1IP?$AA@ 00000001400ecef8     errmsg.obj
 0002:00003f10       ??_C@_0BK@OAJGGGIC@Localhost?5via?5UNIX?5socket?$AA@ 00000001400ecf10     errmsg.obj
 0002:00003f30       ??_C@_0BA@OBGODAJN@Wrong?5host?5info?$AA@ 00000001400ecf30     errmsg.obj
 0002:00003f48       ??_C@_0BP@LPGLBKOF@MySQL?5client?5ran?5out?5of?5memory?$AA@ 00000001400ecf48     errmsg.obj
 0002:00003f70       ??_C@_0DM@BHKAADIN@Protocol?5mismatch?$DL?5server?5versio@ 00000001400ecf70     errmsg.obj
 0002:00003fb8       ??_C@_0BL@GGNHAOJF@MySQL?5server?5has?5gone?5away?$AA@ 00000001400ecfb8     errmsg.obj
 0002:00003fd8       ??_C@_0CJ@MGNDPAC@Unknown?5MySQL?5server?5host?5?8?$CF?9?410@ 00000001400ecfd8     errmsg.obj
 0002:00004010       ??_C@_0CA@NNJEMGCD@Can?8t?5create?5TCP?1IP?5socket?5?$CI?$CFd?$CJ?$AA@ 00000001400ed010     errmsg.obj
 0002:00004038       ??_C@_0DA@DGOLCCI@Can?8t?5connect?5to?5MySQL?5server?5on@ 00000001400ed038     errmsg.obj
 0002:00004080       ??_C@_0EC@FCNCJBBO@Can?8t?5connect?5to?5local?5MySQL?5ser@ 00000001400ed080     errmsg.obj
 0002:000040d0       ??_C@_0BO@EGFBLII@Can?8t?5create?5UNIX?5socket?5?$CI?$CFd?$CJ?$AA@ 00000001400ed0d0     errmsg.obj
 0002:000040f8       ??_C@_0BE@OOMFAHBF@Unknown?5MySQL?5error?$AA@ 00000001400ed0f8     errmsg.obj
 0002:00004110       ??_C@_02PCIJFNDE@?$AN?6?$AA@ 00000001400ed110     mysys:default_modify.obj
 0002:00004118       ??_C@_07CCIHIKOK@no_name?$AA@ 00000001400ed118     mysys:my_thr_init.obj
 0002:00004120       ??_C@_0CE@CLEEBIJB@Can?8t?5initialize?5threads?3?5error?5@ 00000001400ed120     mysys:my_thr_init.obj
 0002:00004144       ??_C@_04LHHHFLPP@utf8?$AA@ 00000001400ed144     mysys:charset.obj
 0002:0000414c       ??_C@_04JKLLLNMI@ucs2?$AA@ 00000001400ed14c     mysys:charset.obj
 0002:00004158       ??_C@_09NKDKDEJM@charsets?1?$AA@ 00000001400ed158     mysys:charset.obj
 0002:00004168       ??_C@_0CJ@GOPBAPMO@c?3?1Program?5Files?1MySQL?1MySQL?5Ser@ 00000001400ed168     mysys:charset.obj
 0002:00004194       ??_C@_05KGKMKOAF@share?$AA@ 00000001400ed194     mysys:charset.obj
 0002:000041a0       ??_C@_09NJBIMGLE@Index?4xml?$AA@ 00000001400ed1a0     mysys:charset.obj
 0002:000041ac       ??_C@_01OGPIMHDM@?$DP?$AA@ 00000001400ed1ac     mysys:charset.obj
 0002:000041b0       ??_C@_04GAOAGNCM@?4xml?$AA@ 00000001400ed1b0     mysys:charset.obj
 0002:000041b8       ??_C@_05HPPBHLPE@cp932?$AA@ 00000001400ed1b8     mysys:charset.obj
 0002:000041c0       ??_C@_02GFBACKGC@cp?$AA@   00000001400ed1c0     mysys:charset.obj
 0002:000041c4       ??_C@_04BPFBOLGB@?4cnf?$AA@ 00000001400ed1c4     mysys:default.obj
 0002:000041cc       ??_C@_04PHHEBHMK@?4ini?$AA@ 00000001400ed1cc     mysys:default.obj
 0002:000041f0       ??_C@_0BJ@KIKAGLAC@?9?9defaults?9group?9suffix?$DN?$AA@ 00000001400ed1f0     mysys:default.obj
 0002:00004210       ??_C@_0DM@LOBIDFGL@error?3?5Wrong?5?8?$CB?$CFs?8?5directive?5in?5@ 00000001400ed210     mysys:default.obj
 0002:00004250       ??_C@_09FJGNFLHN@?2System32?$AA@ 00000001400ed250     mysys:default.obj
 0002:00004260       ??_C@_0BL@CAKPALPI@GetSystemWindowsDirectoryA?$AA@ 00000001400ed260     mysys:default.obj
 0002:00004280       ??_C@_0N@MDJJJHMB@kernel32?4dll?$AA@ 00000001400ed280     mysys:default.obj
 0002:00004290       ??_C@_0L@DODNGCIN@MYSQL_HOME?$AA@ 00000001400ed290     mysys:default.obj
 0002:0000429c       ??_C@_03GMPKIPBL@C?3?1?$AA@ 00000001400ed29c     mysys:default.obj
 0002:000042a0       ??_C@_0EM@DMHOPFHM@error?3?5Found?5option?5without?5prec@ 00000001400ed2a0     mysys:default.obj
 0002:000042f0       ??_C@_0DN@MBLPBICC@error?3?5Wrong?5group?5definition?5in@ 00000001400ed2f0     mysys:default.obj
 0002:00004330       ??_C@_02BAABKJLB@?9?9?$AA@ 00000001400ed330     mysys:default.obj
 0002:00004340       ??_C@_0GG@GBLJMDFL@Warning?3?5skipping?5?8?$CFs?8?5directive@ 00000001400ed340     mysys:default.obj
 0002:000043a8       ??_C@_01CLKCMJKC@?5?$AA@   00000001400ed3a8     mysys:default.obj
 0002:000043b0       ??_C@_0DF@OKDAKIKM@Internal?5error?5initializing?5defa@ 00000001400ed3b0     mysys:default.obj
 0002:000043f0       ??_C@_0EH@NKGMIPDP@?6Default?5options?5are?5read?5from?5t@ 00000001400ed3f0     mysys:default.obj
 0002:00004440       ??_C@_0BDO@PJIJBBOO@?6The?5following?5options?5may?5be?5gi@ 00000001400ed440     mysys:default.obj
 0002:00004580       ??_C@_0BP@MNBILDMG@The?5following?5groups?5are?5read?3?$AA@ 00000001400ed580     mysys:default.obj
 0002:000045a0       ??_C@_0DD@BMIFLCG@Fatal?5error?5in?5defaults?5handling@ 00000001400ed5a0     mysys:default.obj
 0002:000045d8       ??_C@_0CL@DPGKONAJ@Could?5not?5open?5required?5defaults@ 00000001400ed5d8     mysys:default.obj
 0002:00004608       ??_C@_0BD@GMCINPDE@MYSQL_GROUP_SUFFIX?$AA@ 00000001400ed608     mysys:default.obj
 0002:0000461c       ??_C@_03IKGEINEE@?$CFs?5?$AA@ 00000001400ed61c     mysys:default.obj
 0002:00004620       ??_C@_0DK@MHCNAEBD@?$CFs?5would?5have?5been?5started?5with?5@ 00000001400ed620     mysys:default.obj
 0002:00004660       ??_C@_0BB@BKNLJB@?9?9print?9defaults?$AA@ 00000001400ed660     mysys:default.obj
 0002:00004678       ??_C@_08LMJEPNLL@defaults?$AA@ 00000001400ed678     mysys:default.obj
 0002:00004684       ??_C@_02DJGKEECL@?4?4?$AA@ 00000001400ed684     mysys:mf_loadpath.obj
 0002:00004688       ??_C@_07FGFPPMNP@striped?$AA@ 00000001400ed688     mysys:my_static.obj
 0002:00004690       ??_C@_04CGFJFPFD@none?$AA@ 00000001400ed690     mysys:my_static.obj
 0002:00004698       ??_C@_0BL@LPICHLF@01230120022455012623010202?$AA@ 00000001400ed698     mysys:my_static.obj
 0002:000046b8       ??_C@_0BA@KPMGBOMG@?$CFs?4?$CF08X?4deleted?$AA@ 00000001400ed6b8     mysys:my_delete.obj
 0002:000046c8       ??_C@_01NEMOKFLO@?$DN?$AA@ 00000001400ed6c8     mysys:my_init.obj
 0002:000046d0       ??_C@_0P@MCGHDL@Software?2MySQL?$AA@ 00000001400ed6d0     mysys:my_init.obj
 0002:000046e0       ??_C@_0L@LKJCDLMN@HAVE_TCPIP?$AA@ 00000001400ed6e0     mysys:my_init.obj
 0002:000046f0       ??_C@_0DF@KNCKAEOE@SYSTEM?2CurrentControlSet?2Service@ 00000001400ed6f0     mysys:my_init.obj
 0002:00004728       ??_C@_0DG@NPLBFMIJ@SYSTEM?2CurrentControlSet?2Service@ 00000001400ed728     mysys:my_init.obj
 0002:00004760       ??_C@_0DD@IKBMIFKO@SYSTEM?2CurrentControlSet?2Service@ 00000001400ed760     mysys:my_init.obj
 0002:00004798       ??_C@_09KHPDOLMK@UMASK_DIR?$AA@ 00000001400ed798     mysys:my_init.obj
 0002:000047a4       ??_C@_05OMMCGCJP@UMASK?$AA@ 00000001400ed7a4     mysys:my_init.obj
 0002:000047ac       ??_C@_04GHGFPGNC@HOME?$AA@ 00000001400ed7ac     mysys:my_init.obj
 0002:000047b4       ??_C@_05HBBNPFP@loose?$AA@ 00000001400ed7b4     mysys:my_getopt.obj
 0002:000047c0       ??_C@_07MEIENILC@maximum?$AA@ 00000001400ed7c0     mysys:my_getopt.obj
 0002:000047c8       ??_C@_06OFNJOBDK@enable?$AA@ 00000001400ed7c8     mysys:my_getopt.obj
 0002:000047d0       ??_C@_07DBNODEFN@disable?$AA@ 00000001400ed7d0     mysys:my_getopt.obj
 0002:000047d8       ??_C@_04DLBGLKG@skip?$AA@  00000001400ed7d8     mysys:my_getopt.obj
 0002:000047f8       ??_C@_02DKCKIIND@?$CFs?$AA@ 00000001400ed7f8     mysys:my_getopt.obj
 0002:000047fc       ??_C@_06EILBFPFN@Info?3?5?$AA@ 00000001400ed7fc     mysys:my_getopt.obj
 0002:00004808       ??_C@_09CKCJCCOK@Warning?3?5?$AA@ 00000001400ed808     mysys:my_getopt.obj
 0002:00004818       ??_C@_0DJ@LCKGBNKC@Unknown?5suffix?5?8?$CFc?8?5used?5for?5var@ 00000001400ed818     mysys:my_getopt.obj
 0002:00004858       ??_C@_0BO@MNLPLDPE@Incorrect?5integer?5value?3?5?8?$CFs?8?$AA@ 00000001400ed858     mysys:my_getopt.obj
 0002:00004878       ??_C@_0CM@CINNIGFM@option?5?8?$CFs?8?3?5signed?5value?5?$CFs?5adj@ 00000001400ed878     mysys:my_getopt.obj
 0002:000048a8       ??_C@_0CO@JEKLPIGP@option?5?8?$CFs?8?3?5unsigned?5value?5?$CFs?5a@ 00000001400ed8a8     mysys:my_getopt.obj
 0002:000048d8       ??_C@_0L@PIHEMIFO@?$CFs?$DNname?$CFs?5?$AA@ 00000001400ed8d8     mysys:my_getopt.obj
 0002:000048e8       ??_C@_07JMJBGKBC@?$CFs?$DN?$CD?$CFs?5?$AA@ 00000001400ed8e8     mysys:my_getopt.obj
 0002:000048f0       ??_C@_04GIEADKIK@?9?9?$CFs?$AA@ 00000001400ed8f0     mysys:my_getopt.obj
 0002:000048f8       ??_C@_07NACDLBD@?5?5?9?$CFc?$CFs?$AA@ 00000001400ed8f8     mysys:my_getopt.obj
 0002:00004900       ??_C@_02KNHHEEKP@?5?5?$AA@ 00000001400ed900     mysys:my_getopt.obj
 0002:00004904       ??_C@_01OHGJGJJP@?$FL?$AA@ 00000001400ed904     mysys:my_getopt.obj
 0002:00004908       ??_C@_01LBDDMOBJ@?$FN?$AA@ 00000001400ed908     mysys:my_getopt.obj
 0002:0000490c       ??_C@_02KEGNLNML@?0?5?$AA@ 00000001400ed90c     mysys:my_getopt.obj
 0002:00004910       ??_C@_0M@EPOBBBBF@?$CIDisabled?$CJ?6?$AA@ 00000001400ed910     mysys:my_getopt.obj
 0002:0000491c       ??_C@_04OJNJKCBM@?$CFlu?6?$AA@ 00000001400ed91c     mysys:my_getopt.obj
 0002:00004924       ??_C@_04PEDNGLFL@?$CFld?6?$AA@ 00000001400ed924     mysys:my_getopt.obj
 0002:0000492c       ??_C@_05MAJJAKPI@FALSE?$AA@ 00000001400ed92c     mysys:my_getopt.obj
 0002:00004934       ??_C@_03OFAPEBGM@?$CFs?6?$AA@ 00000001400ed934     mysys:my_getopt.obj
 0002:00004938       ??_C@_0BD@IAAJELIC@?$CINo?5default?5value?$CJ?$AA@ 00000001400ed938     mysys:my_getopt.obj
 0002:0000494c       ??_C@_04HCDDPBNL@TRUE?$AA@ 00000001400ed94c     mysys:my_getopt.obj
 0002:00004960       ??_C@_0EB@DLNDDEIC@?9?9?9?9?9?9?9?9?9?9?9?9?9?9?9?9?9?9?9?9?9?9?9?9?9?9?9?9?9?9?9?9@ 00000001400ed960     mysys:my_getopt.obj
 0002:000049b0       ??_C@_0EB@MLHGNKOO@and?5boolean?5options?5?$HLFALSE?$HMTRUE?$HN@ 00000001400ed9b0     mysys:my_getopt.obj
 0002:000049f8       ??_C@_0CE@PGFPJDHK@?6Variables?5?$CI?9?9variable?9name?$DNvalu@ 00000001400ed9f8     mysys:my_getopt.obj
 0002:00004a20       ??_C@_0CF@LIKIEIBC@?$CFs?3?5ambiguous?5option?5?8?9?9?$CFs?8?5?$CI?$CFs?0@ 00000001400eda20     mysys:my_getopt.obj
 0002:00004a48       ??_C@_0CH@NLLNKKKI@?$CFs?3?5variable?5prefix?5?8?$CFs?8?5is?5not?5@ 00000001400eda48     mysys:my_getopt.obj
 0002:00004a70       ??_C@_0CH@FPNHAJDD@?$CFs?3?5option?5?8?9?9?$CFs?8?5requires?5an?5ar@ 00000001400eda70     mysys:my_getopt.obj
 0002:00004a98       ??_C@_0CK@KELFDMIH@?$CFs?3?5option?5?8?9?9?$CFs?8?5cannot?5take?5an@ 00000001400eda98     mysys:my_getopt.obj
 0002:00004ac8       ??_C@_0CI@IFAFNNJB@?$CFs?3?5option?5?8?$CFs?8?5cannot?5take?5an?5a@ 00000001400edac8     mysys:my_getopt.obj
 0002:00004af0       ??_C@_0CJ@FNGIKGPP@?$CFs?3?5ambiguous?5option?5?8?9?9?$CFs?9?$CFs?8?5?$CI@ 00000001400edaf0     mysys:my_getopt.obj
 0002:00004b20       ??_C@_0CF@MFEIKBHA@?$CFs?3?5Option?5?8?9O?8?5requires?5an?5argu@ 00000001400edb20     mysys:my_getopt.obj
 0002:00004b48       ??_C@_0BJ@PLKIKLOO@?$CFs?3?5unknown?5option?5?8?9?$CFc?8?$AA@ 00000001400edb48     mysys:my_getopt.obj
 0002:00004b68       ??_C@_0CP@OAGPFOL@?$CFs?3?5ERROR?3?5Option?5?8?9?$CFc?8?5used?0?5bu@ 00000001400edb68     mysys:my_getopt.obj
 0002:00004b98       ??_C@_0CL@CIFFNEPP@?$CFs?3?5Error?5while?5setting?5value?5?8?$CF@ 00000001400edb98     mysys:my_getopt.obj
 0002:00004bc8       ??_C@_0CG@OPCNLHEP@?$CFs?3?5option?5?8?9?$CFc?8?5requires?5an?5arg@ 00000001400edbc8     mysys:my_getopt.obj
 0002:00004bf0       ??_C@_0DF@NCABEMAI@?$CFs?3?5ignoring?5option?5?8?9?9?$CFs?8?5due?5t@ 00000001400edbf0     mysys:my_getopt.obj
 0002:00004c28       ??_C@_05LAPONLG@false?$AA@ 00000001400edc28     mysys:my_getopt.obj
 0002:00004c30       ??_C@_04LOAJBDKD@true?$AA@ 00000001400edc30     mysys:my_getopt.obj
 0002:00004c38       ??_C@_0CL@BLOGDLDC@?$CFs?3?5?$CFs?3?5Option?5?8?$CFs?8?5used?0?5but?5is@ 00000001400edc38     mysys:my_getopt.obj
 0002:00004c68       ??_C@_07KCOHIFOP@WARNING?$AA@ 00000001400edc68     mysys:my_getopt.obj
 0002:00004c70       ??_C@_0BK@HIDGBPPN@?$CFs?3?5unknown?5option?5?8?9?9?$CFs?8?$AA@ 00000001400edc70     mysys:my_getopt.obj
 0002:00004c90       ??_C@_0BK@JFALHNEE@?$CFs?3?5unknown?5variable?5?8?$CFs?8?$AA@ 00000001400edc90     mysys:my_getopt.obj
 0002:00004cac       ??_C@_01HIHLOKLC@1?$AA@    00000001400edcac     mysys:my_getopt.obj
 0002:00004cb0       ??_C@_0DB@OBCAMIPA@?$CFs?3?5Option?5?8?9?9set?9variable?8?5requ@ 00000001400edcb0     mysys:my_getopt.obj
 0002:00004ce8       ??_C@_0O@LAIDGFMB@?9set?9variable?$AA@ 00000001400edce8     mysys:my_getopt.obj
 0002:00004cf8       sha_const_key              00000001400edcf8     mysys:sha1.obj
 0002:00004d20       ??_C@_0BB@BIKLJNJD@Unknown?5error?5?$CFd?$AA@ 00000001400edd20     mysys:my_error.obj
 0002:00004d38       ??_C@_08KKHFAPMN@UNOPENED?$AA@ 00000001400edd38     mysys:my_div.obj
 0002:00004d48       ??_C@_07NFANNNEC@UNKNOWN?$AA@ 00000001400edd48     mysys:my_div.obj
 0002:00004d50       ??_C@_06LBMPDOLO@CLOCK$?$AA@ 00000001400edd50     mysys:my_access.obj
 0002:00004d58       ??_C@_04KOCLJNO@LPT9?$AA@  00000001400edd58     mysys:my_access.obj
 0002:00004d60       ??_C@_04BDPJIIJP@LPT8?$AA@ 00000001400edd60     mysys:my_access.obj
 0002:00004d68       ??_C@_04JEGBJEFA@LPT7?$AA@ 00000001400edd68     mysys:my_access.obj
 0002:00004d70       ??_C@_04INHKKFBB@LPT6?$AA@ 00000001400edd70     mysys:my_access.obj
 0002:00004d78       ??_C@_04KGFHPGNC@LPT5?$AA@ 00000001400edd78     mysys:my_access.obj
 0002:00004d80       ??_C@_04LPEMMHJD@LPT4?$AA@ 00000001400edd80     mysys:my_access.obj
 0002:00004d88       ??_C@_04PAANFBFE@LPT3?$AA@ 00000001400edd88     mysys:my_access.obj
 0002:00004d90       ??_C@_04OJBGGABF@LPT2?$AA@ 00000001400edd90     mysys:my_access.obj
 0002:00004d98       ??_C@_04MCDLDDNG@LPT1?$AA@ 00000001400edd98     mysys:my_access.obj
 0002:00004da0       ??_C@_04JDDPPBDJ@COM9?$AA@ 00000001400edda0     mysys:my_access.obj
 0002:00004da8       ??_C@_04IKCEMAHI@COM8?$AA@ 00000001400edda8     mysys:my_access.obj
 0002:00004db0       ??_C@_04NLMNMLH@COM7?$AA@  00000001400eddb0     mysys:my_access.obj
 0002:00004db8       ??_C@_04BEKHONPG@COM6?$AA@ 00000001400eddb8     mysys:my_access.obj
 0002:00004dc0       ??_C@_04DPIKLODF@COM5?$AA@ 00000001400eddc0     mysys:my_access.obj
 0002:00004dc8       ??_C@_04CGJBIPHE@COM4?$AA@ 00000001400eddc8     mysys:my_access.obj
 0002:00004dd0       ??_C@_04GJNABJLD@COM3?$AA@ 00000001400eddd0     mysys:my_access.obj
 0002:00004dd8       ??_C@_04HAMLCIPC@COM2?$AA@ 00000001400eddd8     mysys:my_access.obj
 0002:00004de0       ??_C@_04FLOGHLDB@COM1?$AA@ 00000001400edde0     mysys:my_access.obj
 0002:00004de8       ??_C@_03JDMLODLP@NUL?$AA@  00000001400edde8     mysys:my_access.obj
 0002:00004dec       ??_C@_03OFAGCELM@AUX?$AA@  00000001400eddec     mysys:my_access.obj
 0002:00004df0       ??_C@_03BEHELHBE@PRN?$AA@  00000001400eddf0     mysys:my_access.obj
 0002:00004df4       ??_C@_03ECCGHPEG@CON?$AA@  00000001400eddf4     mysys:my_access.obj
 0002:00004df8       ??_C@_01KICIPPFI@?2?$AA@   00000001400eddf8     mysys:my_getwd.obj
 0002:00004dfc       ??_C@_04LFNFNAMA@?4sym?$AA@ 00000001400eddfc     mysys:mf_pack.obj
 0002:00004e04       ??_C@_02LMMGGCAJ@?3?5?$AA@ 00000001400ede04     mysys:my_messnc.obj
 0002:00004e08       ??_C@_0CC@POIIBGBO@File?5?8?$CFs?8?5not?5found?5?$CIErrcode?3?5?$CFd@ 00000001400ede08     mysys:errors.obj
 0002:00004e30       ??_C@_0FB@HBKGDBGI@Collation?5?8?$CFs?8?5is?5not?5a?5compiled@ 00000001400ede30     mysys:errors.obj
 0002:00004e88       ??_C@_0CL@IPPKDKJC@Can?8t?5sync?5file?5?8?$CFs?8?5to?5disk?5?$CIEr@ 00000001400ede88     mysys:errors.obj
 0002:00004eb8       ??_C@_0CH@DMNLJIAN@Error?5on?5realpath?$CI?$CJ?5on?5?8?$CFs?8?5?$CIErr@ 00000001400edeb8     mysys:errors.obj
 0002:00004ee0       ??_C@_0DG@MPBGHFJG@Can?8t?5create?5symlink?5?8?$CFs?8?5pointi@ 00000001400edee0     mysys:errors.obj
 0002:00004f18       ??_C@_0CN@FDDHNKAL@Can?8t?5read?5value?5for?5symlink?5?8?$CFs@ 00000001400edf18     mysys:errors.obj
 0002:00004f48       ??_C@_0DG@HFJCEGGP@Out?5of?5resources?5when?5opening?5fi@ 00000001400edf48     mysys:errors.obj
 0002:00004f80       ??_C@_0FJ@LJEFGFHC@Character?5set?5?8?$CFs?8?5is?5not?5a?5comp@ 00000001400edf80     mysys:errors.obj
 0002:00004fe0       ??_C@_0CK@KAOBDLLK@Can?8t?5create?5directory?5?8?$CFs?8?5?$CIErr@ 00000001400edfe0     mysys:errors.obj
 0002:00005010       ??_C@_0JL@NKJOFGOC@Disk?5is?5full?5writing?5?8?$CFs?8?5?$CIErrco@ 00000001400ee010     mysys:errors.obj
 0002:000050b0       ??_C@_0CG@DLBAOFCG@?$CFd?5files?5and?5?$CFd?5streams?5is?5left?5@ 00000001400ee0b0     mysys:errors.obj
 0002:000050d8       ??_C@_0BL@KPAFHPFA@Warning?3?5?8?$CFs?8?5had?5?$CFd?5links?$AA@ 00000001400ee0d8     mysys:errors.obj
 0002:000050f8       ??_C@_0CH@HKPCIIFI@Can?8t?5change?5dir?5to?5?8?$CFs?8?5?$CIErrcod@ 00000001400ee0f8     mysys:errors.obj
 0002:00005120       ??_C@_0CJ@HHIGEGH@Can?8t?5get?5working?5dirctory?5?$CIErrc@ 00000001400ee120     mysys:errors.obj
 0002:00005150       ??_C@_0CM@IDOLEFDO@Can?8t?5open?5stream?5from?5handle?5?$CIE@ 00000001400ee150     mysys:errors.obj
 0002:00005180       ??_C@_0CI@JHPDBJAP@Can?8t?5change?5size?5of?5file?5?$CIErrco@ 00000001400ee180     mysys:errors.obj
 0002:000051a8       ??_C@_0CF@EBINEGNH@Can?8t?5get?5stat?5of?5?8?$CFs?8?5?$CIErrcode?3@ 00000001400ee1a8     mysys:errors.obj
 0002:000051d0       ??_C@_0CF@DKKFLCIK@Can?8t?5read?5dir?5of?5?8?$CFs?8?5?$CIErrcode?3@ 00000001400ee1d0     mysys:errors.obj
 0002:000051f8       ??_C@_0CA@NMCGOICJ@Can?8t?5unlock?5file?5?$CIErrcode?3?5?$CFd?$CJ?$AA@ 00000001400ee1f8     mysys:errors.obj
 0002:00005218       ??_C@_0BO@FABCFMMA@Can?8t?5lock?5file?5?$CIErrcode?3?5?$CFd?$CJ?$AA@ 00000001400ee218     mysys:errors.obj
 0002:00005238       ??_C@_0DK@OPEJLFLC@Unexpected?5eof?5found?5when?5readin@ 00000001400ee238     mysys:errors.obj
 0002:00005278       ??_C@_0CO@NDIKPEAP@Error?5on?5rename?5of?5?8?$CFs?8?5to?5?8?$CFs?8?5@ 00000001400ee278     mysys:errors.obj
 0002:000052a8       ??_C@_0CG@LPKMPJNP@Error?5on?5delete?5of?5?8?$CFs?8?5?$CIErrcode@ 00000001400ee2a8     mysys:errors.obj
 0002:000052d0       ??_C@_0CA@NLHLMAKD@Out?5of?5memory?5?$CINeeded?5?$CFu?5bytes?$CJ?$AA@ 00000001400ee2d0     mysys:errors.obj
 0002:000052f0       ??_C@_0CF@BEDBELLH@Error?5on?5close?5of?5?8?$CFs?8?5?$CIErrcode?3@ 00000001400ee2f0     mysys:errors.obj
 0002:00005318       ??_C@_0CG@CGPFOMKP@Error?5writing?5file?5?8?$CFs?8?5?$CIErrcode@ 00000001400ee318     mysys:errors.obj
 0002:00005340       ??_C@_0CG@NONCHHAM@Error?5reading?5file?5?8?$CFs?8?5?$CIErrcode@ 00000001400ee340     mysys:errors.obj
 0002:00005368       ??_C@_0CO@OHAAEPNE@Can?8t?5create?1write?5to?5file?5?8?$CFs?8?5@ 00000001400ee368     mysys:errors.obj
 0002:00005398       ??_C@_0CP@BPNOAMDC@Retry?5in?5?$CFd?5secs?4?5Message?5reprin@ 00000001400ee398     mysys:errors.obj
 0002:000053c8       ??_C@_0L@BBMDDOEP@latin1_bin?$AA@ 00000001400ee3c8     strings:ctype-latin1.obj
 0002:000053d8       ??_C@_0BC@JEMPBIB@latin1_german2_ci?$AA@ 00000001400ee3d8     strings:ctype-latin1.obj
 0002:000053ec       ??_C@_06OJHGLDPL@?$CInull?$CJ?$AA@ 00000001400ee3ec     strings:my_vsnprintf.obj
 0002:000053f4       ??_C@_06FNFBAEBE@binary?$AA@ 00000001400ee3f4     strings:ctype-bin.obj
 0002:00005400       ??_C@_0CD@BFGJEGID@charsets?4charset?4collation?4rules@ 00000001400ee400     strings:ctype.obj
 0002:00005428       ??_C@_0CD@FKCINAEE@charsets?4charset?4collation?4rules@ 00000001400ee428     strings:ctype.obj
 0002:00005450       ??_C@_0CD@HBAFIDIH@charsets?4charset?4collation?4rules@ 00000001400ee450     strings:ctype.obj
 0002:00005478       ??_C@_0CH@KJFHHNMJ@charsets?4charset?4collation?4rules@ 00000001400ee478     strings:ctype.obj
 0002:000054a0       ??_C@_0BP@NMDEOJPD@charsets?4charset?4collation?4map?$AA@ 00000001400ee4a0     strings:ctype.obj
 0002:000054c0       ??_C@_0CA@JGIKEKKE@charsets?4charset?4collation?4flag?$AA@ 00000001400ee4c0     strings:ctype.obj
 0002:000054e0       ??_C@_0CB@KBKKLI@charsets?4charset?4collation?4order@ 00000001400ee4e0     strings:ctype.obj
 0002:00005508       ??_C@_0BO@MIJPBBIL@charsets?4charset?4collation?4id?$AA@ 00000001400ee508     strings:ctype.obj
 0002:00005528       ??_C@_0CA@GPLMECFO@charsets?4charset?4collation?4name?$AA@ 00000001400ee528     strings:ctype.obj
 0002:00005548       ??_C@_0BL@IDKPIAPF@charsets?4charset?4collation?$AA@ 00000001400ee548     strings:ctype.obj
 0002:00005568       ??_C@_0BN@ILNCMOEP@charsets?4charset?4unicode?4map?$AA@ 00000001400ee568     strings:ctype.obj
 0002:00005588       ??_C@_0BJ@JKKCHCFM@charsets?4charset?4unicode?$AA@ 00000001400ee588     strings:ctype.obj
 0002:000055a8       ??_C@_0BL@GALBJBAL@charsets?4charset?4lower?4map?$AA@ 00000001400ee5a8     strings:ctype.obj
 0002:000055c8       ??_C@_0BH@GOLLAKNF@charsets?4charset?4lower?$AA@ 00000001400ee5c8     strings:ctype.obj
 0002:000055e0       ??_C@_0BL@MCLGLPJA@charsets?4charset?4upper?4map?$AA@ 00000001400ee5e0     strings:ctype.obj
 0002:00005600       ??_C@_0BH@DFAFGBGM@charsets?4charset?4upper?$AA@ 00000001400ee600     strings:ctype.obj
 0002:00005618       ??_C@_0BL@IBJAIFFC@charsets?4charset?4ctype?4map?$AA@ 00000001400ee618     strings:ctype.obj
 0002:00005638       ??_C@_0BH@HHGMIMKN@charsets?4charset?4ctype?$AA@ 00000001400ee638     strings:ctype.obj
 0002:00005650       ??_C@_0BH@DLFBNKOK@charsets?4charset?4alias?$AA@ 00000001400ee650     strings:ctype.obj
 0002:00005668       ??_C@_0BN@PJKOHNED@charsets?4charset?4description?$AA@ 00000001400ee668     strings:ctype.obj
 0002:00005688       ??_C@_0BI@OAGONPDB@charsets?4charset?4family?$AA@ 00000001400ee688     strings:ctype.obj
 0002:000056a0       ??_C@_0BG@OFKJCAHC@charsets?4charset?4name?$AA@ 00000001400ee6a0     strings:ctype.obj
 0002:000056b8       ??_C@_0BL@KLEDBLCK@charsets?4charset?4binary?9id?$AA@ 00000001400ee6b8     strings:ctype.obj
 0002:000056d8       ??_C@_0BM@CNFHBIFP@charsets?4charset?4primary?9id?$AA@ 00000001400ee6d8     strings:ctype.obj
 0002:000056f8       ??_C@_0BB@NIMCMEKL@charsets?4charset?$AA@ 00000001400ee6f8     strings:ctype.obj
 0002:00005710       ??_C@_0BA@BJIDBDPI@charsets?4max?9id?$AA@ 00000001400ee710     strings:ctype.obj
 0002:00005720       ??_C@_08PBFNHBDC@charsets?$AA@ 00000001400ee720     strings:ctype.obj
 0002:00005730       ??_C@_0N@HPNLKDDF@xml?4encoding?$AA@ 00000001400ee730     strings:ctype.obj
 0002:00005740       ??_C@_0M@JDGBHFH@xml?4version?$AA@ 00000001400ee740     strings:ctype.obj
 0002:0000574c       ??_C@_03PJHHNEEI@xml?$AA@  00000001400ee74c     strings:ctype.obj
 0002:00005750       ??_C@_04HHCDBDLF@?5?7?$AN?6?$AA@ 00000001400ee750     strings:ctype.obj
 0002:00005758       ??_C@_06NOJLBGIH@?5?$CFs?5?$CFs?$AA@ 00000001400ee758     strings:ctype.obj
 0002:00005760       ??_C@_03DKMEACPB@?$DM?$DM?$DM?$AA@ 00000001400ee760     strings:ctype.obj
 0002:00005764       ??_C@_02FODMEDOG@?$DM?$DM?$AA@ 00000001400ee764     strings:ctype.obj
 0002:00005768       ??_C@_01MNNFJEPP@?$DM?$AA@ 00000001400ee768     strings:ctype.obj
 0002:0000576c       ??_C@_01HNPIGOCE@?$CG?$AA@ 00000001400ee76c     strings:ctype.obj
 0002:00005770       ??_C@_08DOMPDOCM@compiled?$AA@ 00000001400ee770     strings:ctype.obj
 0002:00005780       ??_C@_07CJDBHDIN@primary?$AA@ 00000001400ee780     strings:ctype.obj
 0002:00005788       ??_C@_0BC@FAACCCJD@utf8_hungarian_ci?$AA@ 00000001400ee788     strings:ctype-uca.obj
 0002:000057a0       ??_C@_0BC@MMMDBEJH@utf8_esperanto_ci?$AA@ 00000001400ee7a0     strings:ctype-uca.obj
 0002:000057b8       ??_C@_0BA@POPDBMKL@utf8_persian_ci?$AA@ 00000001400ee7b8     strings:ctype-uca.obj
 0002:000057c8       ??_C@_0O@JCIJCIKH@utf8_roman_ci?$AA@ 00000001400ee7c8     strings:ctype-uca.obj
 0002:000057d8       ??_C@_0BB@DMDMGDOP@utf8_spanish2_ci?$AA@ 00000001400ee7d8     strings:ctype-uca.obj
 0002:000057f0       ??_C@_0P@NIJBPDBH@utf8_slovak_ci?$AA@ 00000001400ee7f0     strings:ctype-uca.obj
 0002:00005800       ??_C@_0BD@MHPAIICH@utf8_lithuanian_ci?$AA@ 00000001400ee800     strings:ctype-uca.obj
 0002:00005818       ??_C@_0P@LICOLLCI@utf8_danish_ci?$AA@ 00000001400ee818     strings:ctype-uca.obj
 0002:00005828       ??_C@_0O@OMAOFLBG@utf8_czech_ci?$AA@ 00000001400ee828     strings:ctype-uca.obj
 0002:00005838       ??_C@_0BA@HIEJCGP@utf8_turkish_ci?$AA@ 00000001400ee838     strings:ctype-uca.obj
 0002:00005848       ??_C@_0BA@DLMLGKMF@utf8_swedish_ci?$AA@ 00000001400ee848     strings:ctype-uca.obj
 0002:00005858       ??_C@_0BA@BFDLDMHI@utf8_spanish_ci?$AA@ 00000001400ee858     strings:ctype-uca.obj
 0002:00005868       ??_C@_0BB@IDIAKKIG@utf8_estonian_ci?$AA@ 00000001400ee868     strings:ctype-uca.obj
 0002:00005880       ??_C@_0P@BMIMEGFF@utf8_polish_ci?$AA@ 00000001400ee880     strings:ctype-uca.obj
 0002:00005890       ??_C@_0BC@ONGHKMPJ@utf8_slovenian_ci?$AA@ 00000001400ee890     strings:ctype-uca.obj
 0002:000058a8       ??_C@_0BB@EMJFIJEJ@utf8_romanian_ci?$AA@ 00000001400ee8a8     strings:ctype-uca.obj
 0002:000058c0       ??_C@_0BA@GIAOJNDD@utf8_latvian_ci?$AA@ 00000001400ee8c0     strings:ctype-uca.obj
 0002:000058d0       ??_C@_0BC@OLHAMMMB@utf8_icelandic_ci?$AA@ 00000001400ee8d0     strings:ctype-uca.obj
 0002:000058e8       ??_C@_0BA@GBKHDDAB@utf8_unicode_ci?$AA@ 00000001400ee8e8     strings:ctype-uca.obj
 0002:000058f8       ??_C@_0BC@JMLAFJDL@ucs2_hungarian_ci?$AA@ 00000001400ee8f8     strings:ctype-uca.obj
 0002:00005910       ??_C@_0BC@HBGPDP@ucs2_esperanto_ci?$AA@ 00000001400ee910     strings:ctype-uca.obj
 0002:00005928       ??_C@_0BA@PJNOLINJ@ucs2_persian_ci?$AA@ 00000001400ee928     strings:ctype-uca.obj
 0002:00005938       ??_C@_0O@CNOJEKEN@ucs2_roman_ci?$AA@ 00000001400ee938     strings:ctype-uca.obj
 0002:00005948       ??_C@_0BB@ICDAFOFL@ucs2_spanish2_ci?$AA@ 00000001400ee948     strings:ctype-uca.obj
 0002:00005960       ??_C@_0P@JIPBJIBD@ucs2_slovak_ci?$AA@ 00000001400ee960     strings:ctype-uca.obj
 0002:00005970       ??_C@_0BD@BPDBBBIG@ucs2_lithuanian_ci?$AA@ 00000001400ee970     strings:ctype-uca.obj
 0002:00005988       ??_C@_0P@PIEONACM@ucs2_danish_ci?$AA@ 00000001400ee988     strings:ctype-uca.obj
 0002:00005998       ??_C@_0O@FDGODJPM@ucs2_czech_ci?$AA@ 00000001400ee998     strings:ctype-uca.obj
 0002:000059a8       ??_C@_0BA@KJDGBN@ucs2_turkish_ci?$AA@ 00000001400ee9a8     strings:ctype-uca.obj
 0002:000059b8       ??_C@_0BA@DMOGMOLH@ucs2_swedish_ci?$AA@ 00000001400ee9b8     strings:ctype-uca.obj
 0002:000059c8       ??_C@_0BA@BCBGJIAK@ucs2_spanish_ci?$AA@ 00000001400ee9c8     strings:ctype-uca.obj
 0002:000059d8       ??_C@_0BB@DNIMJHDC@ucs2_estonian_ci?$AA@ 00000001400ee9d8     strings:ctype-uca.obj
 0002:000059f0       ??_C@_0P@FMOMCNFB@ucs2_polish_ci?$AA@ 00000001400ee9f0     strings:ctype-uca.obj
 0002:00005a00       ??_C@_0BC@CBNFNHFB@ucs2_slovenian_ci?$AA@ 00000001400eea00     strings:ctype-uca.obj
 0002:00005a18       ??_C@_0BB@PCJJLEPN@ucs2_romanian_ci?$AA@ 00000001400eea18     strings:ctype-uca.obj
 0002:00005a30       ??_C@_0BA@GPCDDJEB@ucs2_latvian_ci?$AA@ 00000001400eea30     strings:ctype-uca.obj
 0002:00005a40       ??_C@_0BC@CHMCLHGJ@ucs2_icelandic_ci?$AA@ 00000001400eea40     strings:ctype-uca.obj
 0002:00005a58       ??_C@_0BA@GGIKJHHD@ucs2_unicode_ci?$AA@ 00000001400eea58     strings:ctype-uca.obj
 0002:00006768       ??_C@_0L@JHIJEIOB@?$CFs?5at?5?8?$CFs?8?$AA@ 00000001400ef768     strings:ctype-uca.obj
 0002:00006778       ??_C@_0BC@FMLIFBCF@Unknown?5character?$AA@ 00000001400ef778     strings:ctype-uca.obj
 0002:00006790       ??_C@_0L@BNFOJFGF@?$CG?5expected?$AA@ 00000001400ef790     strings:ctype-uca.obj
 0002:000067a0       ??_C@_0BA@CIAPGHM@?$CG?5or?5?$DM?5expected?$AA@ 00000001400ef7a0     strings:ctype-uca.obj
 0002:000067b0       ??_C@_0BD@DBLGAKEN@character?5expected?$AA@ 00000001400ef7b0     strings:ctype-uca.obj
 0002:000067c8       ??_C@_0BE@OMJLCPFJ@Should?5never?5happen?$AA@ 00000001400ef7c8     strings:ctype-uca.obj
 0002:000067e0       ??_C@_0P@MGHCGHFF@Too?5many?5rules?$AA@ 00000001400ef7e0     strings:ctype-uca.obj
 0002:000067f0       ??_C@_09LKJGLAE@cp932_bin?$AA@ 00000001400ef7f0     strings:ctype-cp932.obj
 0002:00006800       ??_C@_0BC@CHMDDICP@cp932_japanese_ci?$AA@ 00000001400ef800     strings:ctype-cp932.obj
 0002:00006818       ??_C@_0BC@DDCCPNHL@latin1_spanish_ci?$AA@ 00000001400ef818     strings:ctype-extra.obj
 0002:00006830       ??_C@_0L@JHFHEMOB@latin2_bin?$AA@ 00000001400ef830     strings:ctype-extra.obj
 0002:00006840       ??_C@_0L@DMJAOHGP@cp1250_bin?$AA@ 00000001400ef840     strings:ctype-extra.obj
 0002:00006850       ??_C@_0BC@DDOEKG@latin1_general_cs?$AA@ 00000001400ef850     strings:ctype-extra.obj
 0002:00006868       ??_C@_0BC@LABOBOHN@latin1_general_ci?$AA@ 00000001400ef868     strings:ctype-extra.obj
 0002:00006880       ??_C@_0BD@LKINKBJP@cp1250_croatian_ci?$AA@ 00000001400ef880     strings:ctype-extra.obj
 0002:00006898       ??_C@_0BD@LCIKDBGI@latin2_croatian_ci?$AA@ 00000001400ef898     strings:ctype-extra.obj
 0002:000068b0       ??_C@_0BC@GHHJKIPO@cp1250_general_ci?$AA@ 00000001400ef8b0     strings:ctype-extra.obj
 0002:000068c4       ??_C@_06OIGKMLKM@cp1250?$AA@ 00000001400ef8c4     strings:ctype-extra.obj
 0002:000068d0       ??_C@_0BE@IGDBMPBG@latin2_hungarian_ci?$AA@ 00000001400ef8d0     strings:ctype-extra.obj
 0002:000068e8       ??_C@_0BB@HINPBEBI@latin1_danish_ci?$AA@ 00000001400ef8e8     strings:ctype-extra.obj
 0002:00006900       ??_C@_0BC@NNEHCLD@latin2_general_ci?$AA@ 00000001400ef900     strings:ctype-extra.obj
 0002:00006914       ??_C@_06IGIJGDC@latin2?$AA@ 00000001400ef914     strings:ctype-extra.obj
 0002:00006920       ??_C@_0BC@EOOMILFB@latin1_german1_ci?$AA@ 00000001400ef920     strings:ctype-extra.obj
 0002:00006938       ??_C@_08BMIDNPKK@utf8_bin?$AA@ 00000001400ef938     strings:ctype-utf8.obj
 0002:00006948       ??_C@_0BA@JGAHNPHO@utf8_general_ci?$AA@ 00000001400ef948     strings:ctype-utf8.obj
 0002:00006958       ??_C@_08OGGFHGPF@ujis_bin?$AA@ 00000001400ef958     strings:ctype-ujis.obj
 0002:00006968       ??_C@_0BB@KEGFAMFE@ujis_japanese_ci?$AA@ 00000001400ef968     strings:ctype-ujis.obj
 0002:0000697c       ??_C@_04BPGAKKKA@ujis?$AA@ 00000001400ef97c     strings:ctype-ujis.obj
 0002:00006988       ??_C@_08POIAHHJH@ucs2_bin?$AA@ 00000001400ef988     strings:ctype-ucs2.obj
 0002:00006998       ??_C@_0BA@JBCKHLAM@ucs2_general_ci?$AA@ 00000001400ef998     strings:ctype-ucs2.obj
 0002:000069a8       ??_C@_0L@NBGPIHPA@tis620_bin?$AA@ 00000001400ef9a8     strings:ctype-tis620.obj
 0002:000069b8       ??_C@_0P@GFLKKABK@tis620_thai_ci?$AA@ 00000001400ef9b8     strings:ctype-tis620.obj
 0002:000069c8       ??_C@_06MGNELAEE@tis620?$AA@ 00000001400ef9c8     strings:ctype-tis620.obj
 0002:000069d0       ??_C@_08JFHPAPHP@sjis_bin?$AA@ 00000001400ef9d0     strings:ctype-sjis.obj
 0002:000069e0       ??_C@_0BB@DFBLLFM@sjis_japanese_ci?$AA@ 00000001400ef9e0     strings:ctype-sjis.obj
 0002:000069f4       ??_C@_04JACAFPAA@sjis?$AA@ 00000001400ef9f4     strings:ctype-sjis.obj
 0002:00006a00       ??_C@_07KJPNPKHF@gbk_bin?$AA@ 00000001400efa00     strings:ctype-gbk.obj
 0002:00006a08       ??_C@_0P@GNPIDCFN@gbk_chinese_ci?$AA@ 00000001400efa08     strings:ctype-gbk.obj
 0002:00006a18       ??_C@_03LFBAECHL@gbk?$AA@  00000001400efa18     strings:ctype-gbk.obj
 0002:00006a20       ??_C@_0L@ODLCHMHL@gb2312_bin?$AA@ 00000001400efa20     strings:ctype-gb2312.obj
 0002:00006a30       ??_C@_0BC@NLCEMJAE@gb2312_chinese_ci?$AA@ 00000001400efa30     strings:ctype-gb2312.obj
 0002:00006a44       ??_C@_06JIBIJLME@gb2312?$AA@ 00000001400efa44     strings:ctype-gb2312.obj
 0002:00006a50       ??_C@_09JHKEBMLO@euckr_bin?$AA@ 00000001400efa50     strings:ctype-euc_kr.obj
 0002:00006a60       ??_C@_0BA@EKHKJCHH@euckr_korean_ci?$AA@ 00000001400efa60     strings:ctype-euc_kr.obj
 0002:00006a70       ??_C@_05FHCOMIFC@euckr?$AA@ 00000001400efa70     strings:ctype-euc_kr.obj
 0002:00006a78       ??_C@_0M@BEKAHKLO@eucjpms_bin?$AA@ 00000001400efa78     strings:ctype-eucjpms.obj
 0002:00006a88       ??_C@_0BE@GEODDEKB@eucjpms_japanese_ci?$AA@ 00000001400efa88     strings:ctype-eucjpms.obj
 0002:00006aa0       ??_C@_07MOEGLBAH@eucjpms?$AA@ 00000001400efaa0     strings:ctype-eucjpms.obj
 0002:00006aa8       ??_C@_0BA@IOACFKLD@latin2_czech_cs?$AA@ 00000001400efaa8     strings:ctype-czech.obj
 0002:00006ab8       ??_C@_04PJNGGADL@?$AF?6?$BC?$BC?$AA@ 00000001400efab8     strings:ctype-czech.obj
 0002:00006ac0       ??_C@_01GFHCPBMG@C?$AA@    00000001400efac0     strings:ctype-czech.obj
 0002:00006ac4       ??_C@_04NALNINKB@?$AF?6?$BB?$BB?$AA@ 00000001400efac4     strings:ctype-czech.obj
 0002:00006acc       ??_C@_01PAPGNFGE@c?$AA@    00000001400efacc     strings:ctype-czech.obj
 0002:00006ad0       ??_C@_04DCMIHFOD@?$AM?$BJ11?$AA@ 00000001400efad0     strings:ctype-czech.obj
 0002:00006ad8       ??_C@_02EKMCNAHJ@CH?$AA@   00000001400efad8     strings:ctype-czech.obj
 0002:00006adc       ??_C@_04CKBBCOJF@?$AM?$BJ00?$AA@ 00000001400efadc     strings:ctype-czech.obj
 0002:00006ae4       ??_C@_02NPEGPENL@Ch?$AA@   00000001400efae4     strings:ctype-czech.obj
 0002:00006ae8       ??_C@_04PADBMEEG@?$AM?$BJ?1?1?$AA@ 00000001400efae8     strings:ctype-czech.obj
 0002:00006af0       ??_C@_02OHALLCDL@ch?$AA@   00000001400efaf0     strings:ctype-czech.obj
 0002:00006b00       ??_C@_0BAB@LDKHKKBE@?$LE?$LF?$LG?$LH?$LI?$LJ?$LK?$LL?$LM?$AC?$LO?$LP?$MA?A?B?C?D?E?F?G?H?I?J?K?L?M?N?O?P?Q?R?S@ 00000001400efb00     strings:ctype-czech.obj
 0002:00006c10       ??_C@_0BAB@JENJBEPB@?$AA?$AA?$AA?$AA?$AA?$AA?$AA?$AA?$AA?$AC?$AA?$AA?$AA?$AA?$AA?$AA?$AA?$AA?$AA?$AA?$AA?$AA?$AA?$AA?$AA?$AA?$AA?$AA?$AA?$AA?$AA?$AA@ 00000001400efc10     strings:ctype-czech.obj
 0002:00006d20       ??_C@_0BAB@GIDHDAFJ@?$AA?$AA?$AA?$AA?$AA?$AA?$AA?$AA?$AA?$AC?$AA?$AA?$AA?$AA?$AA?$AA?$AA?$AA?$AA?$AA?$AA?$AA?$AA?$AA?$AA?$AA?$AA?$AA?$AA?$AA?$AA?$AA@ 00000001400efd20     strings:ctype-czech.obj
 0002:00006e30       ??_C@_0BAB@HNOGOFAJ@?$AA?$AA?$AA?$AA?$AA?$AA?$AA?$AA?$AA?$AC?$AA?$AA?$AA?$AA?$AA?$AA?$AA?$AA?$AA?$AA?$AA?$AA?$AA?$AA?$AA?$AA?$AA?$AA?$AA?$AA?$AA?$AA@ 00000001400efe30     strings:ctype-czech.obj
 0002:00006f38       ??_C@_0BA@MDKNCPKD@cp1250_czech_cs?$AA@ 00000001400eff38     strings:ctype-win1250ch.obj
 0002:00006f48       ??_C@_08CJHFMMIC@big5_bin?$AA@ 00000001400eff48     strings:ctype-big5.obj
 0002:00006f58       ??_C@_0BA@HCMNJPNC@big5_chinese_ci?$AA@ 00000001400eff58     strings:ctype-big5.obj
 0002:00006f68       ??_C@_04HDKIILFF@big5?$AA@ 00000001400eff68     strings:ctype-big5.obj
 0002:00006f70       log_10                     00000001400eff70     strings:strtod.obj
 0002:00007918       __real@8000000000000000    00000001400f0918     strings:strtod.obj
 0002:00007920       __real@7fefffffffffffff    00000001400f0920     strings:strtod.obj
 0002:00007928       __real@3ffcc359e067a348    00000001400f0928     strings:strtod.obj
 0002:00007930       __real@4024000000000000    00000001400f0930     strings:strtod.obj
 0002:00007938       __real@3ff0000000000000    00000001400f0938     strings:strtod.obj
 0002:00007940       ??_C@_03BECJNG@?8?$CB?8?$AA@ 00000001400f0940     strings:xml.obj
 0002:00007944       ??_C@_03BGKMKHKM@?8?$DP?8?$AA@ 00000001400f0944     strings:xml.obj
 0002:00007948       ??_C@_04OEPMCOLO@TEXT?$AA@ 00000001400f0948     strings:xml.obj
 0002:00007950       ??_C@_07JEDAPFNH@COMMENT?$AA@ 00000001400f0950     strings:xml.obj
 0002:00007958       ??_C@_03KIKAENM@?8?1?8?$AA@ 00000001400f0958     strings:xml.obj
 0002:0000795c       ??_C@_03BHGOMNJL@?8?$DO?8?$AA@ 00000001400f095c     strings:xml.obj
 0002:00007960       ??_C@_03BEOKBJPF@?8?$DM?8?$AA@ 00000001400f0960     strings:xml.obj
 0002:00007964       ??_C@_03BFCIHDMC@?8?$DN?8?$AA@ 00000001400f0964     strings:xml.obj
 0002:00007968       ??_C@_05MDAAGLOE@IDENT?$AA@ 00000001400f0968     strings:xml.obj
 0002:00007970       ??_C@_06IGECGLFO@STRING?$AA@ 00000001400f0970     strings:xml.obj
 0002:00007978       ??_C@_03KPJEKKJC@EOF?$AA@  00000001400f0978     strings:xml.obj
 0002:00007980       ??_C@_0M@OGPNDMIP@?$DP?8?$CC?$DN?1?$DM?$DO?5?7?$AN?6?$AA@ 00000001400f0980     strings:xml.obj
 0002:0000798c       ??_C@_06NPFKMDPM@?$DP?$DN?1?$DM?$DO?$CB?$AA@ 00000001400f098c     strings:xml.obj
 0002:00007994       ??_C@_03PNLDJJMO@?9?9?$DO?$AA@ 00000001400f0994     strings:xml.obj
 0002:00007998       ??_C@_04FFDNBKGC@?$DM?$CB?9?9?$AA@ 00000001400f0998     strings:xml.obj
 0002:000079a0       ??_C@_0M@JHPIDPOK@To?5deep?5XML?$AA@ 00000001400f09a0     strings:xml.obj
 0002:000079b0       ??_C@_0CE@HIBBMALO@?8?$DM?1?$CFs?$DO?8?5unexpected?5?$CI?8?$DM?1?$CFs?$DO?8?5want@ 00000001400f09b0     strings:xml.obj
 0002:000079d8       ??_C@_0CH@HIBKOAJO@3?3?5?$CFs?5unexpected?5?$CIident?5or?5?8?1?8?5w@ 00000001400f09d8     strings:xml.obj
 0002:00007a00       ??_C@_0BO@DNBFCJAM@6?3?5?$CFs?5unexpected?5?$CI?8?$DP?8?5wanted?$CJ?$AA@ 00000001400f0a00     strings:xml.obj
 0002:00007a20       ??_C@_0CK@ICCLNHGI@4?3?5?$CFs?5unexpected?5?$CIident?5or?5strin@ 00000001400f0a20     strings:xml.obj
 0002:00007a50       ??_C@_0CA@MOCEIADI@1?3?5?$CFs?5unexpected?5?$CIident?5wanted?$CJ?$AA@ 00000001400f0a50     strings:xml.obj
 0002:00007a70       ??_C@_0BO@LIDKNDNE@5?3?5?$CFs?5unexpected?5?$CI?8?$DO?8?5wanted?$CJ?$AA@ 00000001400f0a70     strings:xml.obj
 0002:00007a90       ??_C@_0M@GPMPBOKO@TCP?1IP?5?$CI?$CFd?$CJ?$AA@ 00000001400f0a90     vio:vio.obj
 0002:00007aa0       ??_C@_0M@BKHBDAGP@socket?5?$CI?$CFd?$CJ?$AA@ 00000001400f0aa0     vio:vio.obj
 0002:00007ab0       ??_C@_0L@BGAKJGHL@named?5pipe?$AA@ 00000001400f0ab0     vio:vio.obj
 0002:00007ac0       ??_C@_0O@CPADDGOO@shared?5memory?$AA@ 00000001400f0ac0     vio:vio.obj
 0002:00007ad0       ??_C@_09PFCHIMEP@127?40?40?41?$AA@ 00000001400f0ad0     vio:viosocket.obj
 0002:00007ae0       ??_C@_0BD@JKAKBJG@SSL_CTX_new?5failed?$AA@ 00000001400f0ae0     vio:viosslfactories.obj
 0002:00007af8       ??_C@_0BN@EHNEHPHI@Failed?5to?5set?5ciphers?5to?5use?$AA@ 00000001400f0af8     vio:viosslfactories.obj
 0002:00007b20       ??_C@_0FN@GPPKHFPO@Private?5key?5does?5not?5match?5the?5c@ 00000001400f0b20     vio:viosslfactories.obj
 0002:00007b80       ??_C@_0BK@OJIINBMD@Unable?5to?5get?5private?5key?$AA@ 00000001400f0b80     vio:viosslfactories.obj
 0002:00007ba0       ??_C@_0BK@DLGAGNNA@Unable?5to?5get?5certificate?$AA@ 00000001400f0ba0     vio:viosslfactories.obj
 0002:00007bc0       ??_C@_08INEPGKHH@No?5error?$AA@ 00000001400f0bc0     vio:viosslfactories.obj
 0002:00007bd0       ??_C@_0P@PDGGPCGE@SSL?5error?3?5?$CFs?6?$AA@ 00000001400f0bd0     vio:viosslfactories.obj
 0002:00007be0       ??_C@_0BJ@DBKDBMMN@SSL?5error?3?5?$CFs?5from?5?8?$CFs?8?6?$AA@ 00000001400f0be0     vio:viosslfactories.obj
 0002:00007c00       ??_C@_0P@GHFPNOJB@bad?5allocation?$AA@ 00000001400f0c00     yassl:ssl.obj
 0002:00007c20       ??_7Message@yaSSL@@6B@     00000001400f0c20     yassl:ssl.obj
 0002:00007c58       ??_7HandShakeBase@yaSSL@@6B@ 00000001400f0c58     yassl:ssl.obj
 0002:00007c88       ??_7HASH@TaoCrypt@@6B@     00000001400f0c88     yassl:ssl.obj
 0002:00007cc8       ??_7MD5@TaoCrypt@@6B@      00000001400f0cc8     yassl:ssl.obj
 0002:00007d18       ??_7MD4@TaoCrypt@@6B@      00000001400f0d18     yassl:ssl.obj
 0002:00007d60       ??_C@_0BM@CIPOPOID@Not?5Implemented?0?5SSLv2?5only?$AA@ 00000001400f0d60     yassl:ssl.obj
 0002:00007d7c       ??_C@_05MOEBAHEJ@SSLv3?$AA@ 00000001400f0d7c     yassl:ssl.obj
 0002:00007d84       ??_C@_05LLIBCOJ@TLSv1?$AA@ 00000001400f0d84     yassl:ssl.obj
 0002:00007d90       ??_C@_0BL@IAMLJBHP@SSLeay?5yaSSL?5compatibility?$AA@ 00000001400f0d90     yassl:ssl.obj
 0002:00007db0       ??_C@_0CI@BCOALAL@Please?5supply?5a?5buffer?5for?5error@ 00000001400f0db0     yassl:ssl.obj
 0002:00007dd8       ??_C@_0BA@JGKGKAME@Not?5Implemented?$AA@ 00000001400f0dd8     yassl:ssl.obj
 0002:00007de8       ??_C@_03GCGHEHKJ@MD5?$AA@  00000001400f0de8     yassl:ssl.obj
 0002:00007df0       ??_C@_0N@MLDFENGJ@DES?9EDE3?9CBC?$AA@ 00000001400f0df0     yassl:ssl.obj
 0002:00007e00       ??_C@_0M@FOEEEMFG@AES?9256?9CBC?$AA@ 00000001400f0e00     yassl:ssl.obj
 0002:00007e10       ??_C@_0M@IMPKGDNH@AES?9192?9CBC?$AA@ 00000001400f0e10     yassl:ssl.obj
 0002:00007e20       ??_C@_0M@CPGGBEEL@AES?9128?9CBC?$AA@ 00000001400f0e20     yassl:ssl.obj
 0002:00007e30       ??_C@_07LDJJJFAI@DES?9CBC?$AA@ 00000001400f0e30     yassl:ssl.obj
 0002:00007e38       ??_C@_02JDPG@rb?$AA@       00000001400f0e38     yassl:ssl.obj
 0002:00007e3c       ??_C@_02KHDDNBB@?2?$CK?$AA@ 00000001400f0e3c     yassl:ssl.obj
 0002:00007e40       ??_C@_07OCFLHCIN@RC4?9MD5?$AA@ 00000001400f0e40     yassl:ssl.obj
 0002:00007e48       ??_C@_07BANEBHLH@RC4?9SHA?$AA@ 00000001400f0e48     yassl:ssl.obj
 0002:00007e50       ??_C@_0M@LLIFGIFE@DES?9CBC?9SHA?$AA@ 00000001400f0e50     yassl:ssl.obj
 0002:00007e60       ??_C@_0N@HCCILIJF@DES?9CBC3?9SHA?$AA@ 00000001400f0e60     yassl:ssl.obj
 0002:00007e70       ??_C@_0BE@COMFBKAK@EDH?9DSS?9DES?9CBC?9SHA?$AA@ 00000001400f0e70     yassl:ssl.obj
 0002:00007e88       ??_C@_0BF@POGOIEBE@EDH?9DSS?9DES?9CBC3?9SHA?$AA@ 00000001400f0e88     yassl:ssl.obj
 0002:00007ea0       ??_C@_0BE@BMKPLFLB@EDH?9RSA?9DES?9CBC?9SHA?$AA@ 00000001400f0ea0     yassl:ssl.obj
 0002:00007eb8       ??_C@_0BF@KCOPIELP@EDH?9RSA?9DES?9CBC3?9SHA?$AA@ 00000001400f0eb8     yassl:ssl.obj
 0002:00007ed0       ??_C@_0L@FJECLCPG@AES128?9SHA?$AA@ 00000001400f0ed0     yassl:ssl.obj
 0002:00007ee0       ??_C@_0BD@HPNPDEHO@DHE?9DSS?9AES128?9SHA?$AA@ 00000001400f0ee0     yassl:ssl.obj
 0002:00007ef8       ??_C@_0BD@MNBMGMFC@DHE?9RSA?9AES128?9SHA?$AA@ 00000001400f0ef8     yassl:ssl.obj
 0002:00007f10       ??_C@_0L@CIGAOKOL@AES256?9SHA?$AA@ 00000001400f0f10     yassl:ssl.obj
 0002:00007f20       ??_C@_0BD@OPNGMGD@DHE?9DSS?9AES256?9SHA?$AA@ 00000001400f0f20     yassl:ssl.obj
 0002:00007f38       ??_C@_0BD@LMDODEEP@DHE?9RSA?9AES256?9SHA?$AA@ 00000001400f0f38     yassl:ssl.obj
 0002:00007f50       ??_C@_0BF@EGKJPLJF@DHE?9DSS?9DES?9CBC3?9RMD?$AA@ 00000001400f0f50     yassl:ssl.obj
 0002:00007f68       ??_C@_0BD@LMNPGFLF@DHE?9DSS?9AES128?9RMD?$AA@ 00000001400f0f68     yassl:ssl.obj
 0002:00007f80       ??_C@_0BD@MNPNDNKI@DHE?9DSS?9AES256?9RMD?$AA@ 00000001400f0f80     yassl:ssl.obj
 0002:00007f98       ??_C@_0BF@BKCIPLDO@DHE?9RSA?9DES?9CBC3?9RMD?$AA@ 00000001400f0f98     yassl:ssl.obj
 0002:00007fb0       ??_C@_0BD@OBMDNJJ@DHE?9RSA?9AES128?9RMD?$AA@ 00000001400f0fb0     yassl:ssl.obj
 0002:00007fc8       ??_C@_0BD@HPDOGFIE@DHE?9RSA?9AES256?9RMD?$AA@ 00000001400f0fc8     yassl:ssl.obj
 0002:00007fe0       ??_C@_0N@LBCIOJFO@DES?9CBC3?9RMD?$AA@ 00000001400f0fe0     yassl:ssl.obj
 0002:00007ff0       ??_C@_0L@JKECODDN@AES128?9RMD?$AA@ 00000001400f0ff0     yassl:ssl.obj
 0002:00008000       ??_C@_0L@OLGALLCA@AES256?9RMD?$AA@ 00000001400f1000     yassl:ssl.obj
 0002:00008038       ??_C@_07MIJDMBL@GGGGGGG?$AA@ 00000001400f1038     yassl:yassl_int.obj
 0002:00008040       ??_C@_06CHLBDKEK@FFFFFF?$AA@ 00000001400f1040     yassl:yassl_int.obj
 0002:00008048       ??_C@_05NGCOEONO@EEEEE?$AA@ 00000001400f1048     yassl:yassl_int.obj
 0002:00008050       ??_C@_03POJCPIGP@CCC?$AA@  00000001400f1050     yassl:yassl_int.obj
 0002:00008058       ??_C@_09IKAJMJIH@yaSSL?4log?$AA@ 00000001400f1058     yassl:yassl_int.obj
 0002:00008078       ??_7Digest@yaSSL@@6B@      00000001400f1078     yassl:crypto_wrapper.obj
 0002:000080b8       ??_7BulkCipher@yaSSL@@6B@  00000001400f10b8     yassl:crypto_wrapper.obj
 0002:00008100       ??_7Auth@yaSSL@@6B@        00000001400f1100     yassl:crypto_wrapper.obj
 0002:00008128       ??_7SHA@TaoCrypt@@6B@      00000001400f1128     yassl:crypto_wrapper.obj
 0002:00008178       ??_7RIPEMD160@TaoCrypt@@6B@ 00000001400f1178     yassl:crypto_wrapper.obj
 0002:000081c8       ??_7Mode_BASE@TaoCrypt@@6B@ 00000001400f11c8     yassl:crypto_wrapper.obj
 0002:000081e8       ??_7DES@TaoCrypt@@6B@      00000001400f11e8     yassl:crypto_wrapper.obj
 0002:00008208       ??_7DES_EDE3@TaoCrypt@@6B@ 00000001400f1208     yassl:crypto_wrapper.obj
 0002:00008228       ??_7AES@TaoCrypt@@6B@      00000001400f1228     yassl:crypto_wrapper.obj
 0002:00008248       ??_7MD5@yaSSL@@6B@         00000001400f1248     yassl:crypto_wrapper.obj
 0002:00008280       ??_7SHA@yaSSL@@6B@         00000001400f1280     yassl:crypto_wrapper.obj
 0002:000082b8       ??_7RMD@yaSSL@@6B@         00000001400f12b8     yassl:crypto_wrapper.obj
 0002:000082f8       ??_7RC4@yaSSL@@6B@         00000001400f12f8     yassl:crypto_wrapper.obj
 0002:00008348       ??_7AES@yaSSL@@6B@         00000001400f1348     yassl:crypto_wrapper.obj
 0002:00008390       ??_7HMAC_MD5@yaSSL@@6B@    00000001400f1390     yassl:crypto_wrapper.obj
 0002:000083c8       ??_7HMAC_SHA@yaSSL@@6B@    00000001400f13c8     yassl:crypto_wrapper.obj
 0002:00008400       ??_7HMAC_RMD@yaSSL@@6B@    00000001400f1400     yassl:crypto_wrapper.obj
 0002:00008438       ??_7DES@yaSSL@@6B@         00000001400f1438     yassl:crypto_wrapper.obj
 0002:00008488       ??_7DES_EDE@yaSSL@@6B@     00000001400f1488     yassl:crypto_wrapper.obj
 0002:000084d0       ??_7DSS@yaSSL@@6B@         00000001400f14d0     yassl:crypto_wrapper.obj
 0002:000084f8       ??_7RSA@yaSSL@@6B@         00000001400f14f8     yassl:crypto_wrapper.obj
 0002:00008518       ??_C@_01LIIJDEN@?$AN?$AA@  00000001400f1518     yassl:crypto_wrapper.obj
 0002:0000851c       ??_C@_03BKNEFOAH@AES?$AA@  00000001400f151c     yassl:crypto_wrapper.obj
 0002:00008520       ??_C@_01IHBHIGKO@?0?$AA@   00000001400f1520     yassl:crypto_wrapper.obj
 0002:00008524       ??_C@_03CNAKKODF@DES?$AA@  00000001400f1524     yassl:crypto_wrapper.obj
 0002:00008528       ??_C@_09OEEMHJLK@Proc?9Type?$AA@ 00000001400f1528     yassl:crypto_wrapper.obj
 0002:00008538       ??_C@_0BO@KNLPBMJG@?9?9?9?9?9END?5RSA?5PRIVATE?5KEY?9?9?9?9?9?$AA@ 00000001400f1538     yassl:crypto_wrapper.obj
 0002:00008558       ??_C@_0CA@PEOGIGIM@?9?9?9?9?9BEGIN?5RSA?5PRIVATE?5KEY?9?9?9?9?9?$AA@ 00000001400f1558     yassl:crypto_wrapper.obj
 0002:00008578       ??_C@_0BK@LPPAEOGJ@?9?9?9?9?9END?5CERTIFICATE?9?9?9?9?9?$AA@ 00000001400f1578     yassl:crypto_wrapper.obj
 0002:00008598       ??_C@_0BM@CPJANAAJ@?9?9?9?9?9BEGIN?5CERTIFICATE?9?9?9?9?9?$AA@ 00000001400f1598     yassl:crypto_wrapper.obj
 0002:000085d0       ??_7HandShakeHeader@yaSSL@@6B@ 00000001400f15d0     yassl:yassl_imp.obj
 0002:00008608       ??_7ServerKeyBase@yaSSL@@6B@ 00000001400f1608     yassl:yassl_imp.obj
 0002:00008638       ??_7ClientKeyBase@yaSSL@@6B@ 00000001400f1638     yassl:yassl_imp.obj
 0002:00008668       ??_7ClientDiffieHellmanPublic@yaSSL@@6B@ 00000001400f1668     yassl:yassl_imp.obj
 0002:00008698       ??_7ChangeCipherSpec@yaSSL@@6B@ 00000001400f1698     yassl:yassl_imp.obj
 0002:000086d0       ??_7Alert@yaSSL@@6B@       00000001400f16d0     yassl:yassl_imp.obj
 0002:00008708       ??_7Data@yaSSL@@6B@        00000001400f1708     yassl:yassl_imp.obj
 0002:00008740       ??_7Certificate@yaSSL@@6B@ 00000001400f1740     yassl:yassl_imp.obj
 0002:00008770       ??_7ServerHello@yaSSL@@6B@ 00000001400f1770     yassl:yassl_imp.obj
 0002:000087a0       ??_7ServerHelloDone@yaSSL@@6B@ 00000001400f17a0     yassl:yassl_imp.obj
 0002:000087d0       ??_7ClientHello@yaSSL@@6B@ 00000001400f17d0     yassl:yassl_imp.obj
 0002:00008800       ??_7ServerKeyExchange@yaSSL@@6B@ 00000001400f1800     yassl:yassl_imp.obj
 0002:00008830       ??_7CertificateVerify@yaSSL@@6B@ 00000001400f1830     yassl:yassl_imp.obj
 0002:00008860       ??_7ClientKeyExchange@yaSSL@@6B@ 00000001400f1860     yassl:yassl_imp.obj
 0002:00008890       ??_7Finished@yaSSL@@6B@    00000001400f1890     yassl:yassl_imp.obj
 0002:000088c0       ??_7HelloRequest@yaSSL@@6B@ 00000001400f18c0     yassl:yassl_imp.obj
 0002:000088f0       ??_7RSA_Server@yaSSL@@6B@  00000001400f18f0     yassl:yassl_imp.obj
 0002:00008920       ??_7Fortezza_Server@yaSSL@@6B@ 00000001400f1920     yassl:yassl_imp.obj
 0002:00008950       ??_7FortezzaKeys@yaSSL@@6B@ 00000001400f1950     yassl:yassl_imp.obj
 0002:00008980       ??_7EncryptedPreMasterSecret@yaSSL@@6B@ 00000001400f1980     yassl:yassl_imp.obj
 0002:000089a8       ??_C@_0BJ@MIAIEIAP@server?5denied?5resumption?$AA@ 00000001400f19a8     yassl:yassl_imp.obj
 0002:000089c8       ??_C@_0BG@NFGEHEFF@session?5lookup?5failed?$AA@ 00000001400f19c8     yassl:yassl_imp.obj
 0002:000089e8       ??_7DH_Server@yaSSL@@6B@   00000001400f19e8     yassl:yassl_imp.obj
 0002:00008a10       ??_C@_04OKGDLNCL@NONE?$AA@ 00000001400f1a10     yassl:yassl_imp.obj
 0002:00008a20       ??_7CertificateRequest@yaSSL@@6B@ 00000001400f1a20     yassl:yassl_imp.obj
 0002:00008ae0       ??_C@_0BF@LOHHNDDD@unknown?5error?5number?$AA@ 00000001400f1ae0     yassl:yassl_error.obj
 0002:00008af8       ??_C@_0BN@DLDIDPJM@Unable?5to?5verify?5certificate?$AA@ 00000001400f1af8     yassl:yassl_error.obj
 0002:00008b18       ??_C@_0BK@HAFIKEEK@bad?5PEM?5format?5processing?$AA@ 00000001400f1b18     yassl:yassl_error.obj
 0002:00008b38       ??_C@_0BH@PIPJPDKN@bad?5content?5processing?$AA@ 00000001400f1b38     yassl:yassl_error.obj
 0002:00008b50       ??_C@_0CG@JIHDAALO@ASN?3?5bad?5other?5signature?5confirm@ 00000001400f1b50     yassl:yassl_error.obj
 0002:00008b78       ??_C@_0CF@OCOHBCCG@ASN?3?5bad?5self?5signature?5confirma@ 00000001400f1b78     yassl:yassl_error.obj
 0002:00008ba0       ??_C@_0BM@NEHMDLJI@ASN?3?5after?5date?5in?5the?5past?$AA@ 00000001400f1ba0     yassl:yassl_error.obj
 0002:00008bc0       ??_C@_0BP@BJJDPHIA@ASN?3?5before?5date?5in?5the?5future?$AA@ 00000001400f1bc0     yassl:yassl_error.obj
 0002:00008be0       ??_C@_0BJ@HLIMONLK@ASN?3?5bad?5DSA?5r?5or?5s?5size?$AA@ 00000001400f1be0     yassl:yassl_error.obj
 0002:00008c00       ??_C@_0BG@DKPAPHGN@ASN?3?5unknown?5hash?5OID?$AA@ 00000001400f1c00     yassl:yassl_error.obj
 0002:00008c18       ??_C@_0BL@LEANJGE@ASN?3?5unknown?5signature?5OID?$AA@ 00000001400f1c18     yassl:yassl_error.obj
 0002:00008c38       ??_C@_0BK@DFPFLNHD@ASN?3?5bad?5Signature?5Length?$AA@ 00000001400f1c38     yassl:yassl_error.obj
 0002:00008c58       ??_C@_0BD@BBKHNDOD@ASN?3?5bad?5Date?5Size?$AA@ 00000001400f1c58     yassl:yassl_error.obj
 0002:00008c70       ??_C@_0O@NCDKAAAO@ASN?3?5bad?5TIME?$AA@ 00000001400f1c70     yassl:yassl_error.obj
 0002:00008c80       ??_C@_0BN@GPGLBGJG@ASN?3?5bad?5Octet?5String?5Header?$AA@ 00000001400f1c80     yassl:yassl_error.obj
 0002:00008ca0       ??_C@_0BA@CHEGMMMD@ASN?3?5expected?50?$AA@ 00000001400f1ca0     yassl:yassl_error.obj
 0002:00008cb0       ??_C@_0BH@CNGNFALI@ASN?3?5expected?5TAG?5NULL?$AA@ 00000001400f1cb0     yassl:yassl_error.obj
 0002:00008cc8       ??_C@_0BK@EHIEHJHJ@ASN?3?5bad?5Ojbect?5ID?5Header?$AA@ 00000001400f1cc8     yassl:yassl_error.obj
 0002:00008ce8       ??_C@_0BK@JLGAAPDA@ASN?3?5unknown?5key?5OID?5type?$AA@ 00000001400f1ce8     yassl:yassl_error.obj
 0002:00008d08       ??_C@_0BK@NEMPKOOB@ASN?3?5bad?5BitString?5Header?$AA@ 00000001400f1d08     yassl:yassl_error.obj
 0002:00008d28       ??_C@_0BM@EABFJODO@ASN?3?5signature?5OID?5mismatch?$AA@ 00000001400f1d28     yassl:yassl_error.obj
 0002:00008d48       ??_C@_0BK@PCPPAJBM@ASN?3?5version?5length?5not?51?$AA@ 00000001400f1d48     yassl:yassl_error.obj
 0002:00008d68       ??_C@_0BE@CBIMDPIB@ASN?3?5bad?5Set?5Header?$AA@ 00000001400f1d68     yassl:yassl_error.obj
 0002:00008d80       ??_C@_0BJ@BABNHBJL@ASN?3?5bad?5Sequence?5Header?$AA@ 00000001400f1d80     yassl:yassl_error.obj
 0002:00008da0       ??_C@_0BM@MLGJJFHM@ASN?3?5bad?5DER?5Integer?5Header?$AA@ 00000001400f1da0     yassl:yassl_error.obj
 0002:00008dc0       ??_C@_0BM@EOJLGIGG@unable?5to?5use?5random?5device?$AA@ 00000001400f1dc0     yassl:yassl_error.obj
 0002:00008de0       ??_C@_0BF@OKLABNFB@CryptGenRandom?5error?$AA@ 00000001400f1de0     yassl:yassl_error.obj
 0002:00008df8       ??_C@_0BF@ONICCKFL@bad?5wincrypt?5acquire?$AA@ 00000001400f1df8     yassl:yassl_error.obj
 0002:00008e10       ??_C@_0BD@EFIDFPA@not?5in?5error?5state?$AA@ 00000001400f1e10     yassl:yassl_error.obj
 0002:00008e28       ??_C@_0CA@FBLLHEJE@the?5write?5operation?5would?5block?$AA@ 00000001400f1e28     yassl:yassl_error.obj
 0002:00008e48       ??_C@_0BP@JNLPEFPG@the?5read?5operation?5would?5block?$AA@ 00000001400f1e48     yassl:yassl_error.obj
 0002:00008e68       ??_C@_0CC@PELKPKCF@bad?5PreMasterSecret?5version?5erro@ 00000001400f1e68     yassl:yassl_error.obj
 0002:00008e90       ??_C@_0BE@IGBKENJK@decompression?5error?$AA@ 00000001400f1e90     yassl:yassl_error.obj
 0002:00008ea8       ??_C@_0BC@NKDLBFJI@compression?5error?$AA@ 00000001400f1ea8     yassl:yassl_error.obj
 0002:00008ec0       ??_C@_0BK@MGANGKEA@protocol?5version?5mismatch?$AA@ 00000001400f1ec0     yassl:yassl_error.obj
 0002:00008ee0       ??_C@_0CL@JIHDBKKF@unable?5to?5proccess?5private?5key?0?5@ 00000001400f1ee0     yassl:yassl_error.obj
 0002:00008f10       ??_C@_0BO@JFJFDJB@unable?5to?5proccess?5cerificate?$AA@ 00000001400f1f10     yassl:yassl_error.obj
 0002:00008f30       ??_C@_0BL@PNPNLENI@socket?5layer?5receive?5error?$AA@ 00000001400f1f30     yassl:yassl_error.obj
 0002:00008f50       ??_C@_0BI@IMFNBLNH@socket?5layer?5send?5error?$AA@ 00000001400f1f50     yassl:yassl_error.obj
 0002:00008f68       ??_C@_0BP@DJNJFCDO@unable?5to?5verify?5peer?5checksum?$AA@ 00000001400f1f68     yassl:yassl_error.obj
 0002:00008f88       ??_C@_0CE@JNMOHBDL@the?5server?5needs?5a?5private?5key?5f@ 00000001400f1f88     yassl:yassl_error.obj
 0002:00008fb0       ??_C@_0CJ@MGMCLLGF@unable?5to?5match?5a?5supported?5ciph@ 00000001400f1fb0     yassl:yassl_error.obj
 0002:00008fe0       ??_C@_0BH@BJAEIFLP@bad?5cipher?5suite?5input?$AA@ 00000001400f1fe0     yassl:yassl_error.obj
 0002:00008ff8       ??_C@_0CK@DPEGAADO@handshake?5message?5received?5in?5wr@ 00000001400f1ff8     yassl:yassl_error.obj
 0002:00009028       ??_C@_0BO@MDNKKMLF@handshake?5layer?5not?5ready?5yet?$AA@ 00000001400f2028     yassl:yassl_error.obj
 0002:00009048       ??_C@_0BL@JKJNJCO@record?5layer?5not?5ready?5yet?$AA@ 00000001400f2048     yassl:yassl_error.obj
 0002:00009068       ??_C@_0CN@HCIHAPHI@bad?5master?5secret?5derivation?0?5pr@ 00000001400f2068     yassl:yassl_error.obj
 0002:00009098       ??_C@_0CA@ICDMIOMH@trying?5to?5use?5an?5unknown?5cipher?$AA@ 00000001400f2098     yassl:yassl_error.obj
 0002:000090b8       ??_C@_0BP@HEAJNFGH@unknown?5factory?5create?5request?$AA@ 00000001400f20b8     yassl:yassl_error.obj
 0002:000090d8       ??_C@_0CB@GDMDOMBH@trying?5to?5realloc?5a?5fixed?5buffer@ 00000001400f20d8     yassl:yassl_error.obj
 0002:00009100       ??_C@_0CB@GAKDHIMM@buffer?5index?5error?0?5out?5of?5range@ 00000001400f2100     yassl:yassl_error.obj
 0002:00009130       ??_C@_05GDHACFMB@1?42?43?$AA@ 00000001400f2130     zlib:compress.obj
 0002:00009140       deflate_copyright          00000001400f2140     zlib:deflate.obj
 0002:00009ad8       ??_C@_0BH@FGKKJGOC@incorrect?5length?5check?$AA@ 00000001400f2ad8     zlib:inflate.obj
 0002:00009af0       ??_C@_0BF@MEIGEHBE@incorrect?5data?5check?$AA@ 00000001400f2af0     zlib:inflate.obj
 0002:00009b08       ??_C@_0BO@ECPMAOGG@invalid?5distance?5too?5far?5back?$AA@ 00000001400f2b08     zlib:inflate.obj
 0002:00009b28       ??_C@_0BG@LBKINIKP@invalid?5distance?5code?$AA@ 00000001400f2b28     zlib:inflate.obj
 0002:00009b40       ??_C@_0BM@FFFLPBBC@invalid?5literal?1length?5code?$AA@ 00000001400f2b40     zlib:inflate.obj
 0002:00009b60       ??_C@_0BG@GMDFCBGP@invalid?5distances?5set?$AA@ 00000001400f2b60     zlib:inflate.obj
 0002:00009b78       ??_C@_0BK@BMMPFBBH@invalid?5bit?5length?5repeat?$AA@ 00000001400f2b78     zlib:inflate.obj
 0002:00009b98       ??_C@_0BM@IIMGAINC@invalid?5literal?1lengths?5set?$AA@ 00000001400f2b98     zlib:inflate.obj
 0002:00009bb8       ??_C@_0CE@GMIGFPBB@too?5many?5length?5or?5distance?5symb@ 00000001400f2bb8     zlib:inflate.obj
 0002:00009be0       ??_C@_0BJ@HDEPPGOH@invalid?5code?5lengths?5set?$AA@ 00000001400f2be0     zlib:inflate.obj
 0002:00009c00       ??_C@_0BN@LGAADGOK@invalid?5stored?5block?5lengths?$AA@ 00000001400f2c00     zlib:inflate.obj
 0002:00009c20       ??_C@_0BD@PJCBIDD@invalid?5block?5type?$AA@ 00000001400f2c20     zlib:inflate.obj
 0002:00009c38       ??_C@_0BE@GONKLEPM@header?5crc?5mismatch?$AA@ 00000001400f2c38     zlib:inflate.obj
 0002:00009c50       ??_C@_0BJ@BLBBCOMO@unknown?5header?5flags?5set?$AA@ 00000001400f2c50     zlib:inflate.obj
 0002:00009c70       ??_C@_0BH@LIBMMIGA@incorrect?5header?5check?$AA@ 00000001400f2c70     zlib:inflate.obj
 0002:00009c88       ??_C@_0BE@EMOGCLGO@invalid?5window?5size?$AA@ 00000001400f2c88     zlib:inflate.obj
 0002:00009ca0       ??_C@_0BL@IHKGDAEE@unknown?5compression?5method?$AA@ 00000001400f2ca0     zlib:inflate.obj
 0002:0000a330       _dist_code                 00000001400f3330     zlib:trees.obj
 0002:0000a530       _length_code               00000001400f3530     zlib:trees.obj
 0002:0000c730       ??_C@_0BF@CJFPCCEG@incompatible?5version?$AA@ 00000001400f5730     zlib:zutil.obj
 0002:0000c748       ??_C@_0N@DFPGLBGC@buffer?5error?$AA@ 00000001400f5748     zlib:zutil.obj
 0002:0000c758       ??_C@_0BE@OGGJBMCE@insufficient?5memory?$AA@ 00000001400f5758     zlib:zutil.obj
 0002:0000c770       ??_C@_0L@HAHMBNLP@data?5error?$AA@ 00000001400f5770     zlib:zutil.obj
 0002:0000c780       ??_C@_0N@MKKNPMJD@stream?5error?$AA@ 00000001400f5780     zlib:zutil.obj
 0002:0000c790       ??_C@_0L@KIJFAKBJ@file?5error?$AA@ 00000001400f5790     zlib:zutil.obj
 0002:0000c7a0       ??_C@_0L@FNAOCBOG@stream?5end?$AA@ 00000001400f57a0     zlib:zutil.obj
 0002:0000c7b0       ??_C@_0BA@MOKMMFOD@need?5dictionary?$AA@ 00000001400f57b0     zlib:zutil.obj
 0002:0000c7c0       z_errmsg                   00000001400f57c0     zlib:zutil.obj
 0002:0000c810       inflate_copyright          00000001400f5810     zlib:inftrees.obj
 0002:0000c940       _FPinit                    00000001400f5940     LIBCMT:fpinit.obj
 0002:0000c948       _FPmtinit                  00000001400f5948     LIBCMT:fpinit.obj
 0002:0000c950       _FPmtterm                  00000001400f5950     LIBCMT:fpinit.obj
 0002:0000c960       ??_7type_info@@6B@         00000001400f5960     LIBCMT:typinfo.obj
 0002:0000c968       ??_C@_03LLEJOLGL@?4?1?2?$AA@ 00000001400f5968     LIBCMT:stati32.obj
 0002:0000c96c       ??_C@_02EAOCEIGI@?$DP?$CK?$AA@ 00000001400f596c     LIBCMT:stati32.obj
 0002:0000c978       ??_7bad_alloc@std@@6B@     00000001400f5978     LIBCMT:new.obj
 0002:0000c990       ??_C@_0EA@FCLIIPNN@Visual?5C?$CL?$CL?5CRT?3?5Not?5enough?5memor@ 00000001400f5990     LIBCMT:strerror.obj
 0002:0000c9d0       ??_C@_0P@MIGLKIOC@CorExitProcess?$AA@ 00000001400f59d0     LIBCMT:crt0dat.obj
 0002:0000c9e0       ??_C@_0M@MBOPBNBK@mscoree?4dll?$AA@ 00000001400f59e0     LIBCMT:crt0dat.obj
 0002:0000c9ec       ??_C@_04HBHDLLBA@PATH?$AA@ 00000001400f59ec     LIBCMT:popen.obj
 0002:0000c9f4       ??_C@_04NPFIMJFF@?5?1c?5?$AA@ 00000001400f59f4     LIBCMT:popen.obj
 0002:0000ca00       ??_C@_07INNMNHPJ@cmd?4exe?$AA@ 00000001400f5a00     LIBCMT:popen.obj
 0002:0000ca08       ??_C@_0M@BOIIGAL@command?4com?$AA@ 00000001400f5a08     LIBCMT:popen.obj
 0002:0000ca18       ??_C@_07CFPBBAOO@COMSPEC?$AA@ 00000001400f5a18     LIBCMT:popen.obj
 0002:0000ca20       __real@bff0000000000000    00000001400f5a20     LIBCMT:floor.obj
 0002:0000ca28       ??_C@_05PBJFFIGL@floor?$AA@ 00000001400f5a28     LIBCMT:floor.obj
 0002:0000ca30       ?ProcessDetach@NativeDll@<CrtImplementationDetails>@@0IB 00000001400f5a30     LIBCMT:strtol.obj
 0002:0000ca34       ?ProcessAttach@NativeDll@<CrtImplementationDetails>@@0IB 00000001400f5a34     LIBCMT:strtol.obj
 0002:0000ca38       ?ThreadAttach@NativeDll@<CrtImplementationDetails>@@0IB 00000001400f5a38     LIBCMT:strtol.obj
 0002:0000ca3c       ?ThreadDetach@NativeDll@<CrtImplementationDetails>@@0IB 00000001400f5a3c     LIBCMT:strtol.obj
 0002:0000ca40       ?ProcessVerifier@NativeDll@<CrtImplementationDetails>@@0IB 00000001400f5a40     LIBCMT:strtol.obj
 0002:0000cd98       ??_C@_02CLFPBFFP@TZ?$AA@   00000001400f5d98     LIBCMT:tzset.obj
 0002:0000cda0       ??_C@_0L@KDOEJCKC@_nextafter?$AA@ 00000001400f5da0     LIBCMT:ieeemisc.obj
 0002:0000cdb0       ??_C@_0M@LNMOKHH@_nextafterf?$AA@ 00000001400f5db0     LIBCMT:ieeemisc.obj
 0002:0000cdbc       ??_C@_06HBLGGACK@_scalb?$AA@ 00000001400f5dbc     LIBCMT:ieeemisc.obj
 0002:0000cdc8       ??_C@_07OIGNLDJH@_scalbf?$AA@ 00000001400f5dc8     LIBCMT:ieeemisc.obj
 0002:0000cdd0       __real@0000000000000000    00000001400f5dd0     LIBCMT:cvt.obj
 0002:0000cdd8       ??_C@_05KLBDPFGC@e?$CL000?$AA@ 00000001400f5dd8     LIBCMT:cvt.obj
 0002:0000cde0       ??_C@_0P@GGKDKEEG@runtime?5error?5?$AA@ 00000001400f5de0     LIBCMT:crt0msg.obj
 0002:0000cdf0       ??_C@_0O@MJNIPGOH@TLOSS?5error?$AN?6?$AA@ 00000001400f5df0     LIBCMT:crt0msg.obj
 0002:0000ce00       ??_C@_0N@BONNPDHF@SING?5error?$AN?6?$AA@ 00000001400f5e00     LIBCMT:crt0msg.obj
 0002:0000ce10       ??_C@_0P@MBDAJNE@DOMAIN?5error?$AN?6?$AA@ 00000001400f5e10     LIBCMT:crt0msg.obj
 0002:0000ce20       ??_C@_0JL@DFDOOABL@R6034?$AN?6An?5application?5has?5made?5a@ 00000001400f5e20     LIBCMT:crt0msg.obj
 0002:0000cec0       ??_C@_0PH@EPAFIJ@R6033?$AN?6?9?5Attempt?5to?5use?5MSIL?5cod@ 00000001400f5ec0     LIBCMT:crt0msg.obj
 0002:0000cfb8       ??_C@_0DD@BKEEABMM@R6032?$AN?6?9?5not?5enough?5space?5for?5lo@ 00000001400f5fb8     LIBCMT:crt0msg.obj
 0002:0000cff0       ??_C@_0GD@OFKILIED@R6031?$AN?6?9?5Attempt?5to?5initialize?5t@ 00000001400f5ff0     LIBCMT:crt0msg.obj
 0002:0000d058       ??_C@_0BP@LPMHJOKI@R6030?$AN?6?9?5CRT?5not?5initialized?$AN?6?$AA@ 00000001400f6058     LIBCMT:crt0msg.obj
 0002:0000d078       ??_C@_0CF@KJDAIALP@R6028?$AN?6?9?5unable?5to?5initialize?5he@ 00000001400f6078     LIBCMT:crt0msg.obj
 0002:0000d0a0       ??_C@_0DF@GAKBPDFP@R6027?$AN?6?9?5not?5enough?5space?5for?5lo@ 00000001400f60a0     LIBCMT:crt0msg.obj
 0002:0000d0d8       ??_C@_0DF@IBLNNAIG@R6026?$AN?6?9?5not?5enough?5space?5for?5st@ 00000001400f60d8     LIBCMT:crt0msg.obj
 0002:0000d110       ??_C@_0CG@IOHKGFNJ@R6025?$AN?6?9?5pure?5virtual?5function?5c@ 00000001400f6110     LIBCMT:crt0msg.obj
 0002:0000d138       ??_C@_0DF@JIJJFJDC@R6024?$AN?6?9?5not?5enough?5space?5for?5_o@ 00000001400f6138     LIBCMT:crt0msg.obj
 0002:0000d170       ??_C@_0CJ@EGEJHFME@R6019?$AN?6?9?5unable?5to?5open?5console?5@ 00000001400f6170     LIBCMT:crt0msg.obj
 0002:0000d1a0       ??_C@_0CB@GNHNIELH@R6018?$AN?6?9?5unexpected?5heap?5error?$AN?6@ 00000001400f61a0     LIBCMT:crt0msg.obj
 0002:0000d1c8       ??_C@_0CN@FOLDKNG@R6017?$AN?6?9?5unexpected?5multithread?5@ 00000001400f61c8     LIBCMT:crt0msg.obj
 0002:0000d1f8       ??_C@_0CM@FAHFJNHO@R6016?$AN?6?9?5not?5enough?5space?5for?5th@ 00000001400f61f8     LIBCMT:crt0msg.obj
 0002:0000d230       ??_C@_0JG@LBKMGKLD@?$AN?6This?5application?5has?5requested@ 00000001400f6230     LIBCMT:crt0msg.obj
 0002:0000d2c8       ??_C@_0CM@FLCNIPKK@R6009?$AN?6?9?5not?5enough?5space?5for?5en@ 00000001400f62c8     LIBCMT:crt0msg.obj
 0002:0000d2f8       ??_C@_0CK@KMMJOAPP@R6008?$AN?6?9?5not?5enough?5space?5for?5ar@ 00000001400f62f8     LIBCMT:crt0msg.obj
 0002:0000d328       ??_C@_0CN@LEKKICBM@R6002?$AN?6?9?5floating?5point?5support?5@ 00000001400f6328     LIBCMT:crt0msg.obj
 0002:0000d358       ??_C@_0CF@GOGNBNAK@Microsoft?5Visual?5C?$CL?$CL?5Runtime?5Lib@ 00000001400f6358     LIBCMT:crt0msg.obj
 0002:0000d380       ??_C@_02PHMGELLB@?6?6?$AA@ 00000001400f6380     LIBCMT:crt0msg.obj
 0002:0000d384       ??_C@_03KHICJKCI@?4?4?4?$AA@ 00000001400f6384     LIBCMT:crt0msg.obj
 0002:0000d388       ??_C@_0BH@DNAGHKFM@?$DMprogram?5name?5unknown?$DO?$AA@ 00000001400f6388     LIBCMT:crt0msg.obj
 0002:0000d3a0       ??_C@_0BK@OFGJDLJJ@Runtime?5Error?$CB?6?6Program?3?5?$AA@ 00000001400f63a0     LIBCMT:crt0msg.obj
 0002:0000d3c0       ??_C@_07EPKMNAGK@?4mixcrt?$AA@ 00000001400f63c0     LIBCMT:tidtable.obj
 0002:0000d3c8       ??_C@_0O@NLDKAIKN@EncodePointer?$AA@ 00000001400f63c8     LIBCMT:tidtable.obj
 0002:0000d3d8       ??_C@_0N@NHGLKGEC@KERNEL32?4DLL?$AA@ 00000001400f63d8     LIBCMT:tidtable.obj
 0002:0000d3e8       ??_C@_0O@KBPMFGHI@DecodePointer?$AA@ 00000001400f63e8     LIBCMT:tidtable.obj
 0002:0000d3f8       ??_C@_04PNGHFIJN@?4com?$AA@ 00000001400f63f8     LIBCMT:stat.obj
 0002:0000d400       ??_C@_04NEEFLLOK@?4bat?$AA@ 00000001400f6400     LIBCMT:stat.obj
 0002:0000d408       ??_C@_04CPCBDHLK@?4cmd?$AA@ 00000001400f6408     LIBCMT:stat.obj
 0002:0000d428       ??_7exception@std@@6B@     00000001400f6428     LIBCMT:stdexcpt.obj
 0002:0000d438       ??_C@_0BC@EOODALEL@Unknown?5exception?$AA@ 00000001400f6438     LIBCMT:stdexcpt.obj
 0002:0000d458       ??_7bad_cast@std@@6B@      00000001400f6458     LIBCMT:stdexcpt.obj
 0002:0000d470       ??_7bad_typeid@std@@6B@    00000001400f6470     LIBCMT:stdexcpt.obj
 0002:0000d488       ??_7__non_rtti_object@std@@6B@ 00000001400f6488     LIBCMT:stdexcpt.obj
 0002:0000d4e0       ??_C@_1O@CEDCILHN@?$AA?$CI?$AAn?$AAu?$AAl?$AAl?$AA?$CJ?$AA?$AA@ 00000001400f64e0     LIBCMT:output.obj
 0002:0000d4f0       __lookuptable              00000001400f64f0     LIBCMT:output.obj
 0002:0000d550       ??_C@_0BG@KLEAJEFJ@Illegal?5byte?5sequence?$AA@ 00000001400f6550     LIBCMT:syserr.obj
 0002:0000d568       ??_C@_0BE@ICMCHPHH@Directory?5not?5empty?$AA@ 00000001400f6568     LIBCMT:syserr.obj
 0002:0000d580       ??_C@_0BJ@IHEHINLI@Function?5not?5implemented?$AA@ 00000001400f6580     LIBCMT:syserr.obj
 0002:0000d5a0       ??_C@_0BD@CLHBCGPB@No?5locks?5available?$AA@ 00000001400f65a0     LIBCMT:syserr.obj
 0002:0000d5b8       ??_C@_0BC@BEDIHIDK@Filename?5too?5long?$AA@ 00000001400f65b8     LIBCMT:syserr.obj
 0002:0000d5d0       ??_C@_0BK@JAEBMJJM@Resource?5deadlock?5avoided?$AA@ 00000001400f65d0     LIBCMT:syserr.obj
 0002:0000d5f0       ??_C@_0BB@FCBJFCAJ@Result?5too?5large?$AA@ 00000001400f65f0     LIBCMT:syserr.obj
 0002:0000d608       ??_C@_0N@MMJPGLJK@Domain?5error?$AA@ 00000001400f6608     LIBCMT:syserr.obj
 0002:0000d618       ??_C@_0M@LHEPIIOM@Broken?5pipe?$AA@ 00000001400f6618     LIBCMT:syserr.obj
 0002:0000d628       ??_C@_0P@PKCJJLLM@Too?5many?5links?$AA@ 00000001400f6628     LIBCMT:syserr.obj
 0002:0000d638       ??_C@_0BG@DDBFNKBH@Read?9only?5file?5system?$AA@ 00000001400f6638     LIBCMT:syserr.obj
 0002:0000d650       ??_C@_0N@FEHLOILP@Invalid?5seek?$AA@ 00000001400f6650     LIBCMT:syserr.obj
 0002:0000d660       ??_C@_0BI@FEALHKLD@No?5space?5left?5on?5device?$AA@ 00000001400f6660     LIBCMT:syserr.obj
 0002:0000d678       ??_C@_0P@LFMMIPAE@File?5too?5large?$AA@ 00000001400f6678     LIBCMT:syserr.obj
 0002:0000d688       ??_C@_0CE@ONOKNLPF@Inappropriate?5I?1O?5control?5operat@ 00000001400f6688     LIBCMT:syserr.obj
 0002:0000d6b0       ??_C@_0BE@INBJMKGG@Too?5many?5open?5files?$AA@ 00000001400f66b0     LIBCMT:syserr.obj
 0002:0000d6c8       ??_C@_0BO@IIFBODJE@Too?5many?5open?5files?5in?5system?$AA@ 00000001400f66c8     LIBCMT:syserr.obj
 0002:0000d6e8       ??_C@_0BB@HMGGCEBG@Invalid?5argument?$AA@ 00000001400f66e8     LIBCMT:syserr.obj
 0002:0000d700       ??_C@_0P@NDHGCGKE@Is?5a?5directory?$AA@ 00000001400f6700     LIBCMT:syserr.obj
 0002:0000d710       ??_C@_0BA@CJBACOOL@Not?5a?5directory?$AA@ 00000001400f6710     LIBCMT:syserr.obj
 0002:0000d720       ??_C@_0P@NLEIANHE@No?5such?5device?$AA@ 00000001400f6720     LIBCMT:syserr.obj
 0002:0000d730       ??_C@_0O@OAMDNOCP@Improper?5link?$AA@ 00000001400f6730     LIBCMT:syserr.obj
 0002:0000d740       ??_C@_0M@NAAJNNGH@File?5exists?$AA@ 00000001400f6740     LIBCMT:syserr.obj
 0002:0000d750       ??_C@_0BA@BIBLIOEK@Resource?5device?$AA@ 00000001400f6750     LIBCMT:syserr.obj
 0002:0000d760       ??_C@_0O@NIPGCINC@Unknown?5error?$AA@ 00000001400f6760     LIBCMT:syserr.obj
 0002:0000d770       ??_C@_0M@LOEHLCJD@Bad?5address?$AA@ 00000001400f6770     LIBCMT:syserr.obj
 0002:0000d780       ??_C@_0BC@HFNFNKAI@Permission?5denied?$AA@ 00000001400f6780     LIBCMT:syserr.obj
 0002:0000d798       ??_C@_0BB@IMDKMPFB@Not?5enough?5space?$AA@ 00000001400f6798     LIBCMT:syserr.obj
 0002:0000d7b0       ??_C@_0CB@EPFKGNAK@Resource?5temporarily?5unavailable@ 00000001400f67b0     LIBCMT:syserr.obj
 0002:0000d7d8       ??_C@_0BD@LOHELEP@No?5child?5processes?$AA@ 00000001400f67d8     LIBCMT:syserr.obj
 0002:0000d7f0       ??_C@_0BE@NFGDDCEF@Bad?5file?5descriptor?$AA@ 00000001400f67f0     LIBCMT:syserr.obj
 0002:0000d808       ??_C@_0BC@HKPNECK@Exec?5format?5error?$AA@ 00000001400f6808     LIBCMT:syserr.obj
 0002:0000d820       ??_C@_0BC@MFFGCDFL@Arg?5list?5too?5long?$AA@ 00000001400f6820     LIBCMT:syserr.obj
 0002:0000d838       ??_C@_0BK@DPKMCKJ@No?5such?5device?5or?5address?$AA@ 00000001400f6838     LIBCMT:syserr.obj
 0002:0000d858       ??_C@_0BD@KKNFOBBD@Input?1output?5error?$AA@ 00000001400f6858     LIBCMT:syserr.obj
 0002:0000d870       ??_C@_0BK@FJBOAFDK@Interrupted?5function?5call?$AA@ 00000001400f6870     LIBCMT:syserr.obj
 0002:0000d890       ??_C@_0BA@FKIAIBGA@No?5such?5process?$AA@ 00000001400f6890     LIBCMT:syserr.obj
 0002:0000d8a0       ??_C@_0BK@FMDHKPNF@No?5such?5file?5or?5directory?$AA@ 00000001400f68a0     LIBCMT:syserr.obj
 0002:0000d8c0       ??_C@_0BI@BJFCGOHL@Operation?5not?5permitted?$AA@ 00000001400f68c0     LIBCMT:syserr.obj
 0002:0000d8e0       __lookuptable_s            00000001400f68e0     LIBCMT:outputs.obj
 0002:0000d940       ??_C@_0BC@JEAENNKH@SystemFunction036?$AA@ 00000001400f6940     LIBCMT:rand_s.obj
 0002:0000d958       ??_C@_0N@JJPEKNFO@ADVAPI32?4DLL?$AA@ 00000001400f6958     LIBCMT:rand_s.obj
 0002:0000d968       ??_C@_0CG@PKBDLMEO@InitializeCriticalSectionAndSpin@ 00000001400f6968     LIBCMT:initcrit.obj
 0002:0000d990       ??_C@_07LCBHPJJN@LC_TIME?$AA@ 00000001400f6990     LIBCMT:setlocal.obj
 0002:0000d998       ??_C@_0L@DLHIECNL@LC_NUMERIC?$AA@ 00000001400f6998     LIBCMT:setlocal.obj
 0002:0000d9a8       ??_C@_0M@MIENIKLA@LC_MONETARY?$AA@ 00000001400f69a8     LIBCMT:setlocal.obj
 0002:0000d9b8       ??_C@_08EADHIDAD@LC_CTYPE?$AA@ 00000001400f69b8     LIBCMT:setlocal.obj
 0002:0000d9c8       ??_C@_0L@KFJHEKIK@LC_COLLATE?$AA@ 00000001400f69c8     LIBCMT:setlocal.obj
 0002:0000d9d4       ??_C@_06NEFDFEKB@LC_ALL?$AA@ 00000001400f69d4     LIBCMT:setlocal.obj
 0002:0000d9e0       __lc_category              00000001400f69e0     LIBCMT:setlocal.obj
 0002:0000daf0       ??_C@_03EGDHDPFD@_?4?0?$AA@ 00000001400f6af0     LIBCMT:setlocal.obj
 0002:0000daf4       ??_C@_01IDAFKMJL@_?$AA@    00000001400f6af4     LIBCMT:setlocal.obj
 0002:0000daf8       ??_C@_01ICJEACDI@?$DL?$AA@ 00000001400f6af8     LIBCMT:setlocal.obj
 0002:0000dafc       ??_C@_02BALPLPBG@?$DN?$DL?$AA@ 00000001400f6afc     LIBCMT:setlocal.obj
 0002:0000db00       ??_C@_06GDENEHCP@CONIN$?$AA@ 00000001400f6b00     LIBCMT:initcon.obj
 0002:0000db08       ??_C@_07GPDNMNG@CONOUT$?$AA@ 00000001400f6b08     LIBCMT:initcon.obj
 0002:0000db10       __dnames                   00000001400f6b10     LIBCMT:timeset.obj
 0002:0000db28       __mnames                   00000001400f6b28     LIBCMT:timeset.obj
 0002:0000db78       ??_C@_0BK@CFCOFLF@?5Complete?5Object?5Locator?8?$AA@ 00000001400f6b78     LIBCMT:undname.obj
 0002:0000db98       ??_C@_0BN@MECKDCOJ@?5Class?5Hierarchy?5Descriptor?8?$AA@ 00000001400f6b98     LIBCMT:undname.obj
 0002:0000dbb8       ??_C@_0BD@LGICGFMM@?5Base?5Class?5Array?8?$AA@ 00000001400f6bb8     LIBCMT:undname.obj
 0002:0000dbd0       ??_C@_0BM@LDKODKLH@?5Base?5Class?5Descriptor?5at?5?$CI?$AA@ 00000001400f6bd0     LIBCMT:undname.obj
 0002:0000dbf0       ??_C@_0BC@DAFEJGAK@?5Type?5Descriptor?8?$AA@ 00000001400f6bf0     LIBCMT:undname.obj
 0002:0000dc08       ??_C@_0BM@PMGGMLDN@?$GAlocal?5static?5thread?5guard?8?$AA@ 00000001400f6c08     LIBCMT:undname.obj
 0002:0000dc28       ??_C@_0CL@FGIJHLCE@?$GAmanaged?5vector?5copy?5constructor@ 00000001400f6c28     LIBCMT:undname.obj
 0002:0000dc58       ??_C@_0CJ@GJELGAMM@?$GAvector?5vbase?5copy?5constructor?5i@ 00000001400f6c58     LIBCMT:undname.obj
 0002:0000dc88       ??_C@_0CD@CGAJBKEJ@?$GAvector?5copy?5constructor?5iterato@ 00000001400f6c88     LIBCMT:undname.obj
 0002:0000dcb0       ??_C@_0CB@PDBIFEP@?$GAdynamic?5atexit?5destructor?5for?5?8@ 00000001400f6cb0     LIBCMT:undname.obj
 0002:0000dcd8       ??_C@_0BL@CLIPGLGB@?$GAdynamic?5initializer?5for?5?8?$AA@ 00000001400f6cd8     LIBCMT:undname.obj
 0002:0000dcf8       ??_C@_0CM@FCBBDIGB@?$GAeh?5vector?5vbase?5copy?5constructo@ 00000001400f6cf8     LIBCMT:undname.obj
 0002:0000dd28       ??_C@_0CG@HLDDJMAG@?$GAeh?5vector?5copy?5constructor?5iter@ 00000001400f6d28     LIBCMT:undname.obj
 0002:0000dd50       ??_C@_0CF@IMGKMJNO@?$GAmanaged?5vector?5destructor?5itera@ 00000001400f6d50     LIBCMT:undname.obj
 0002:0000dd78       ??_C@_0CG@CFDHKGGD@?$GAmanaged?5vector?5constructor?5iter@ 00000001400f6d78     LIBCMT:undname.obj
 0002:0000dda0       ??_C@_0BN@CKNJLHMB@?$GAplacement?5delete?$FL?$FN?5closure?8?$AA@ 00000001400f6da0     LIBCMT:undname.obj
 0002:0000ddc0       ??_C@_0BL@CNOONJFP@?$GAplacement?5delete?5closure?8?$AA@ 00000001400f6dc0     LIBCMT:undname.obj
 0002:0000dde0       ??_C@_0P@HJKNJFNN@?$GAomni?5callsig?8?$AA@ 00000001400f6de0     LIBCMT:undname.obj
 0002:0000ddf0       ??_C@_09LBNFPBCA@?5delete?$FL?$FN?$AA@ 00000001400f6df0     LIBCMT:undname.obj
 0002:0000ddfc       ??_C@_06FHBGPFGH@?5new?$FL?$FN?$AA@ 00000001400f6dfc     LIBCMT:undname.obj
 0002:0000de08       ??_C@_0CE@IIHCMGGL@?$GAlocal?5vftable?5constructor?5closu@ 00000001400f6e08     LIBCMT:undname.obj
 0002:0000de30       ??_C@_0BA@KKLDJDLB@?$GAlocal?5vftable?8?$AA@ 00000001400f6e30     LIBCMT:undname.obj
 0002:0000de40       ??_C@_05KHLCHHI@?$GARTTI?$AA@ 00000001400f6e40     LIBCMT:undname.obj
 0002:0000de48       ??_C@_03KLGMFNMG@?$GAEH?$AA@ 00000001400f6e48     LIBCMT:undname.obj
 0002:0000de50       ??_C@_0BA@KBCDOMBN@?$GAudt?5returning?8?$AA@ 00000001400f6e50     LIBCMT:undname.obj
 0002:0000de60       ??_C@_0BL@LLKPOHJI@?$GAcopy?5constructor?5closure?8?$AA@ 00000001400f6e60     LIBCMT:undname.obj
 0002:0000de80       ??_C@_0CH@OOJPLCPH@?$GAeh?5vector?5vbase?5constructor?5ite@ 00000001400f6e80     LIBCMT:undname.obj
 0002:0000dea8       ??_C@_0CA@GCEOPDGL@?$GAeh?5vector?5destructor?5iterator?8?$AA@ 00000001400f6ea8     LIBCMT:undname.obj
 0002:0000dec8       ??_C@_0CB@JONCMFFK@?$GAeh?5vector?5constructor?5iterator?8@ 00000001400f6ec8     LIBCMT:undname.obj
 0002:0000def0       ??_C@_0BL@NILFHHPC@?$GAvirtual?5displacement?5map?8?$AA@ 00000001400f6ef0     LIBCMT:undname.obj
 0002:0000df10       ??_C@_0CE@IKBNEHA@?$GAvector?5vbase?5constructor?5iterat@ 00000001400f6f10     LIBCMT:undname.obj
 0002:0000df38       ??_C@_0BN@LFPFMEDL@?$GAvector?5destructor?5iterator?8?$AA@ 00000001400f6f38     LIBCMT:undname.obj
 0002:0000df58       ??_C@_0BO@PFGOCPJJ@?$GAvector?5constructor?5iterator?8?$AA@ 00000001400f6f58     LIBCMT:undname.obj
 0002:0000df78       ??_C@_0BN@IMDCHIKM@?$GAscalar?5deleting?5destructor?8?$AA@ 00000001400f6f78     LIBCMT:undname.obj
 0002:0000df98       ??_C@_0BO@OBMKPJIG@?$GAdefault?5constructor?5closure?8?$AA@ 00000001400f6f98     LIBCMT:undname.obj
 0002:0000dfb8       ??_C@_0BN@DEGPLNFK@?$GAvector?5deleting?5destructor?8?$AA@ 00000001400f6fb8     LIBCMT:undname.obj
 0002:0000dfd8       ??_C@_0BD@JDLKDPAB@?$GAvbase?5destructor?8?$AA@ 00000001400f6fd8     LIBCMT:undname.obj
 0002:0000dff0       ??_C@_08OBABFOLI@?$GAstring?8?$AA@ 00000001400f6ff0     LIBCMT:undname.obj
 0002:0000e000       ??_C@_0BF@KDPPACIK@?$GAlocal?5static?5guard?8?$AA@ 00000001400f7000     LIBCMT:undname.obj
 0002:0000e018       ??_C@_08LLFFHHDJ@?$GAtypeof?8?$AA@ 00000001400f7018     LIBCMT:undname.obj
 0002:0000e028       ??_C@_07FEEIOKP@?$GAvcall?8?$AA@ 00000001400f7028     LIBCMT:undname.obj
 0002:0000e030       ??_C@_09BLBHBJP@?$GAvbtable?8?$AA@ 00000001400f7030     LIBCMT:undname.obj
 0002:0000e040       ??_C@_09IFPLHPGF@?$GAvftable?8?$AA@ 00000001400f7040     LIBCMT:undname.obj
 0002:0000e04c       ??_C@_02MHEGNOJ@?$FO?$DN?$AA@ 00000001400f704c     LIBCMT:undname.obj
 0002:0000e050       ??_C@_02DHLNPPGH@?$HM?$DN?$AA@ 00000001400f7050     LIBCMT:undname.obj
 0002:0000e054       ??_C@_02FGJGFEAB@?$CG?$DN?$AA@ 00000001400f7054     LIBCMT:undname.obj
 0002:0000e058       ??_C@_03CDNPDDLA@?$DM?$DM?$DN?$AA@ 00000001400f7058     LIBCMT:undname.obj
 0002:0000e05c       ??_C@_03IKFCCPFF@?$DO?$DO?$DN?$AA@ 00000001400f705c     LIBCMT:undname.obj
 0002:0000e060       ??_C@_02FENAOKFI@?$CF?$DN?$AA@ 00000001400f7060     LIBCMT:undname.obj
 0002:0000e064       ??_C@_02FJEHGPIO@?1?$DN?$AA@ 00000001400f7064     LIBCMT:undname.obj
 0002:0000e068       ??_C@_02FKMDLLOA@?9?$DN?$AA@ 00000001400f7068     LIBCMT:undname.obj
 0002:0000e06c       ??_C@_02FOEOMHFC@?$CL?$DN?$AA@ 00000001400f706c     LIBCMT:undname.obj
 0002:0000e070       ??_C@_02FPIMKNGF@?$CK?$DN?$AA@ 00000001400f7070     LIBCMT:undname.obj
 0002:0000e074       ??_C@_02NONPIBCD@?$HM?$HM?$AA@ 00000001400f7074     LIBCMT:undname.obj
 0002:0000e078       ??_C@_02PPKAJPJL@?$CG?$CG?$AA@ 00000001400f7078     LIBCMT:undname.obj
 0002:0000e07c       ??_C@_01DNKMNLPK@?$HM?$AA@ 00000001400f707c     LIBCMT:undname.obj
 0002:0000e080       ??_C@_01JKBOJNNK@?$FO?$AA@ 00000001400f7080     LIBCMT:undname.obj
 0002:0000e084       ??_C@_01PJKLJHI@?$HO?$AA@  00000001400f7084     LIBCMT:undname.obj
 0002:0000e088       ??_C@_02HCKGKOFO@?$CI?$CJ?$AA@ 00000001400f7088     LIBCMT:undname.obj
 0002:0000e08c       ??_C@_02EEKDKGMJ@?$DO?$DN?$AA@ 00000001400f708c     LIBCMT:undname.obj
 0002:0000e090       ??_C@_01PPODPGHN@?$DO?$AA@ 00000001400f7090     LIBCMT:undname.obj
 0002:0000e094       ??_C@_02EHCHHCKH@?$DM?$DN?$AA@ 00000001400f7094     LIBCMT:undname.obj
 0002:0000e098       ??_C@_01FGNFDNOH@?$CF?$AA@ 00000001400f7098     LIBCMT:undname.obj
 0002:0000e09c       ??_C@_03MNHNFDLC@?9?$DO?$CK?$AA@ 00000001400f709c     LIBCMT:undname.obj
 0002:0000e0a0       ??_C@_01MIFGBAGJ@?$CL?$AA@ 00000001400f70a0     LIBCMT:undname.obj
 0002:0000e0a4       ??_C@_02ECNGHCIF@?$CL?$CL?$AA@ 00000001400f70a4     LIBCMT:undname.obj
 0002:0000e0a8       ??_C@_02HBOOOICD@?9?$DO?$AA@ 00000001400f70a8     LIBCMT:undname.obj
 0002:0000e0b0       ??_C@_08LHJFAFGD@operator?$AA@ 00000001400f70b0     LIBCMT:undname.obj
 0002:0000e0bc       ??_C@_02GPECMEKF@?$FL?$FN?$AA@ 00000001400f70bc     LIBCMT:undname.obj
 0002:0000e0c0       ??_C@_02FDNJECIE@?$CB?$DN?$AA@ 00000001400f70c0     LIBCMT:undname.obj
 0002:0000e0c4       ??_C@_02EGOFBIJA@?$DN?$DN?$AA@ 00000001400f70c4     LIBCMT:undname.obj
 0002:0000e0c8       ??_C@_01DCLJPIOD@?$CB?$AA@ 00000001400f70c8     LIBCMT:undname.obj
 0002:0000e0cc       ??_C@_02GPIOPFAK@?$DO?$DO?$AA@ 00000001400f70cc     LIBCMT:undname.obj
 0002:0000e0d0       ??_C@_07FPCDHGMM@?5delete?$AA@ 00000001400f70d0     LIBCMT:undname.obj
 0002:0000e0d8       ??_C@_04NIHEBCM@?5new?$AA@ 00000001400f70d8     LIBCMT:undname.obj
 0002:0000e0e0       ??_C@_0M@GFIIJFMG@__unaligned?$AA@ 00000001400f70e0     LIBCMT:undname.obj
 0002:0000e0f0       ??_C@_0L@PILCLIHE@__restrict?$AA@ 00000001400f70f0     LIBCMT:undname.obj
 0002:0000e100       ??_C@_07JOMMBBKO@__ptr64?$AA@ 00000001400f7100     LIBCMT:undname.obj
 0002:0000e108       ??_C@_09HIJEGCPM@__clrcall?$AA@ 00000001400f7108     LIBCMT:undname.obj
 0002:0000e118       ??_C@_0L@JMKHOMEK@__fastcall?$AA@ 00000001400f7118     LIBCMT:undname.obj
 0002:0000e128       ??_C@_0L@NPHFGOKO@__thiscall?$AA@ 00000001400f7128     LIBCMT:undname.obj
 0002:0000e138       ??_C@_09IFJBGAPI@__stdcall?$AA@ 00000001400f7138     LIBCMT:undname.obj
 0002:0000e148       ??_C@_08GHMPAG@__pascal?$AA@ 00000001400f7148     LIBCMT:undname.obj
 0002:0000e158       ??_C@_07KOLFKCDI@__cdecl?$AA@ 00000001400f7158     LIBCMT:undname.obj
 0002:0000e160       ??_C@_08EHJDFFNH@__based?$CI?$AA@ 00000001400f7160     LIBCMT:undname.obj
 0002:0000e478       ??_7DNameNode@@6B@         00000001400f7478     LIBCMT:undname.obj
 0002:0000e498       ??_7charNode@@6B@          00000001400f7498     LIBCMT:undname.obj
 0002:0000e4b8       ??_7pDNameNode@@6B@        00000001400f74b8     LIBCMT:undname.obj
 0002:0000e4d8       ??_7DNameStatusNode@@6B@   00000001400f74d8     LIBCMT:undname.obj
 0002:0000e4f8       ??_7pcharNode@@6B@         00000001400f74f8     LIBCMT:undname.obj
 0002:0000e510       ??_C@_04OKOHEJBO@?5?$DP?$DP?5?$AA@ 00000001400f7510     LIBCMT:undname.obj
 0002:0000e518       ??_C@_06EEGAIFAK@?$HLflat?$HN?$AA@ 00000001400f7518     LIBCMT:undname.obj
 0002:0000e520       ??_C@_05JIBOFOHK@?$HLfor?5?$AA@ 00000001400f7520     LIBCMT:undname.obj
 0002:0000e528       ??_C@_0BN@IBLMMFAP@?$GAnon?9type?9template?9parameter?$AA@ 00000001400f7528     LIBCMT:undname.obj
 0002:0000e548       ??_C@_09EBBEKKIH@unsigned?5?$AA@ 00000001400f7548     LIBCMT:undname.obj
 0002:0000e554       ??_C@_05CJIMAING@long?5?$AA@ 00000001400f7554     LIBCMT:undname.obj
 0002:0000e55c       ??_C@_04LAHKHJMA@int?5?$AA@ 00000001400f755c     LIBCMT:undname.obj
 0002:0000e564       ??_C@_06EHJMALKF@short?5?$AA@ 00000001400f7564     LIBCMT:undname.obj
 0002:0000e56c       ??_C@_05CIHEBHNO@char?5?$AA@ 00000001400f756c     LIBCMT:undname.obj
 0002:0000e574       ??_C@_04GKJNKENE@void?$AA@ 00000001400f7574     LIBCMT:undname.obj
 0002:0000e580       ??_C@_0L@EGPHHEKN@?$DMellipsis?$DO?$AA@ 00000001400f7580     LIBCMT:undname.obj
 0002:0000e590       ??_C@_0M@ELJOJFFH@?0?$DMellipsis?$DO?$AA@ 00000001400f7590     LIBCMT:undname.obj
 0002:0000e59c       ??_C@_04EENFHACM@?0?4?4?4?$AA@ 00000001400f759c     LIBCMT:undname.obj
 0002:0000e5a8       ??_C@_07HDJPLPEK@?5throw?$CI?$AA@ 00000001400f75a8     LIBCMT:undname.obj
 0002:0000e5b0       ??_C@_02GOGNNPBN@?$CJ?$FL?$AA@ 00000001400f75b0     LIBCMT:undname.obj
 0002:0000e5b4       ??_C@_02MDINNEEG@s?5?$AA@  00000001400f75b4     LIBCMT:undname.obj
 0002:0000e5b8       ??_C@_01GEODFPGF@?8?$AA@   00000001400f75b8     LIBCMT:undname.obj
 0002:0000e5c0       ??_C@_0BE@EODMJLIF@?$GAtemplate?9parameter?$AA@ 00000001400f75c0     LIBCMT:undname.obj
 0002:0000e5d4       ??_C@_04HIBGFPH@NULL?$AA@  00000001400f75d4     LIBCMT:undname.obj
 0002:0000e5e0       ??_C@_0O@GKABPPIF@cli?3?3pin_ptr?$DM?$AA@ 00000001400f75e0     LIBCMT:undname.obj
 0002:0000e5f0       ??_C@_0M@EALIELKG@cli?3?3array?$DM?$AA@ 00000001400f75f0     LIBCMT:undname.obj
 0002:0000e5fc       ??_C@_05BEFAKPML@void?5?$AA@ 00000001400f75fc     LIBCMT:undname.obj
 0002:0000e604       ??_C@_02OHHJMEON@?8?8?$AA@ 00000001400f7604     LIBCMT:undname.obj
 0002:0000e608       ??_C@_0BG@JNJLAMPM@?$GAanonymous?5namespace?8?$AA@ 00000001400f7608     LIBCMT:undname.obj
 0002:0000e620       ??_C@_01NLNLIGKH@?$GA?$AA@ 00000001400f7620     LIBCMT:undname.obj
 0002:0000e628       ??_C@_0O@KHGCOMHP@generic?9type?9?$AA@ 00000001400f7628     LIBCMT:undname.obj
 0002:0000e638       ??_C@_0BE@JAEOCHPE@template?9parameter?9?$AA@ 00000001400f7638     LIBCMT:undname.obj
 0002:0000e64c       ??_C@_02MOLJINC@?3?3?$AA@  00000001400f764c     LIBCMT:undname.obj
 0002:0000e650       ??_C@_05LJGMCFOG@enum?5?$AA@ 00000001400f7650     LIBCMT:undname.obj
 0002:0000e658       ??_C@_0N@DLIEFKNA@cointerface?5?$AA@ 00000001400f7658     LIBCMT:undname.obj
 0002:0000e668       ??_C@_08KOFANOFK@coclass?5?$AA@ 00000001400f7668     LIBCMT:undname.obj
 0002:0000e674       ??_C@_06LJBABKPM@class?5?$AA@ 00000001400f7674     LIBCMT:undname.obj
 0002:0000e680       ??_C@_07DIBCDNGL@struct?5?$AA@ 00000001400f7680     LIBCMT:undname.obj
 0002:0000e688       ??_C@_06MOJHIBMG@union?5?$AA@ 00000001400f7688     LIBCMT:undname.obj
 0002:0000e690       ??_C@_0P@GCIFDJCJ@?$GAunknown?5ecsu?8?$AA@ 00000001400f7690     LIBCMT:undname.obj
 0002:0000e6a0       ??_C@_02KCKGHPCA@?$CJ?5?$AA@ 00000001400f76a0     LIBCMT:undname.obj
 0002:0000e6a8       ??_C@_0M@DHNBOJMP@extern?5?$CCC?$CC?5?$AA@ 00000001400f76a8     LIBCMT:undname.obj
 0002:0000e6b8       ??_C@_08KJLFOPNE@?$FLthunk?$FN?3?$AA@ 00000001400f76b8     LIBCMT:undname.obj
 0002:0000e6c8       ??_C@_08GPDDCMKI@public?3?5?$AA@ 00000001400f76c8     LIBCMT:undname.obj
 0002:0000e6d8       ??_C@_0M@GAIFPFIP@protected?3?5?$AA@ 00000001400f76d8     LIBCMT:undname.obj
 0002:0000e6e8       ??_C@_09LAPHOOG@private?3?5?$AA@ 00000001400f76e8     LIBCMT:undname.obj
 0002:0000e6f8       ??_C@_08NIEOINHE@virtual?5?$AA@ 00000001400f76f8     LIBCMT:undname.obj
 0002:0000e708       ??_C@_07PGOEDBHP@static?5?$AA@ 00000001400f7708     LIBCMT:undname.obj
 0002:0000e710       ??_C@_0DA@HGFJFBBE@?$GAtemplate?5static?5data?5member?5des@ 00000001400f7710     LIBCMT:undname.obj
 0002:0000e740       ??_C@_0DB@ILEFOCIJ@?$GAtemplate?5static?5data?5member?5con@ 00000001400f7740     LIBCMT:undname.obj
 0002:0000e778       ??_C@_0CB@KJDOOODE@?$GAlocal?5static?5destructor?5helper?8@ 00000001400f7778     LIBCMT:undname.obj
 0002:0000e7a0       ??_C@_0L@HNGCOGAE@?$GAadjustor?$HL?$AA@ 00000001400f77a0     LIBCMT:undname.obj
 0002:0000e7b0       ??_C@_0L@GHPFDFH@?$GAvtordisp?$HL?$AA@ 00000001400f77b0     LIBCMT:undname.obj
 0002:0000e7c0       ??_C@_0N@CBHHHENL@?$GAvtordispex?$HL?$AA@ 00000001400f77c0     LIBCMT:undname.obj
 0002:0000e7d0       ??_C@_02IGFCGPIL@?$HN?8?$AA@ 00000001400f77d0     LIBCMT:undname.obj
 0002:0000e7d4       ??_C@_03OPGICMGF@?$HN?8?5?$AA@ 00000001400f77d4     LIBCMT:undname.obj
 0002:0000e7d8       ??_C@_06LIJLOJAG@const?5?$AA@ 00000001400f77d8     LIBCMT:undname.obj
 0002:0000e7e0       ??_C@_09GAIEOBLP@volatile?5?$AA@ 00000001400f77e0     LIBCMT:undname.obj
 0002:0000e7ec       ??_C@_04HEJADOOB@CV?3?5?$AA@ 00000001400f77ec     LIBCMT:undname.obj
 0002:0000e7f8       ??_C@_07EDHNAJHC@signed?5?$AA@ 00000001400f77f8     LIBCMT:undname.obj
 0002:0000e800       ??_C@_06GCICPBLB@__w64?5?$AA@ 00000001400f7800     LIBCMT:undname.obj
 0002:0000e808       ??_C@_07CLGGIAMF@wchar_t?$AA@ 00000001400f7808     LIBCMT:undname.obj
 0002:0000e810       ??_C@_08GAHOLHEO@__int128?$AA@ 00000001400f7810     LIBCMT:undname.obj
 0002:0000e820       ??_C@_07LFCOJCAC@__int64?$AA@ 00000001400f7820     LIBCMT:undname.obj
 0002:0000e828       ??_C@_07OFLPPHGP@__int32?$AA@ 00000001400f7828     LIBCMT:undname.obj
 0002:0000e830       ??_C@_07ICFHOGAF@__int16?$AA@ 00000001400f7830     LIBCMT:undname.obj
 0002:0000e838       ??_C@_06EBGKOKIG@__int8?$AA@ 00000001400f7838     LIBCMT:undname.obj
 0002:0000e840       ??_C@_04DDKJGDCM@bool?$AA@ 00000001400f7840     LIBCMT:undname.obj
 0002:0000e848       ??_C@_08PABEKFH@volatile?$AA@ 00000001400f7848     LIBCMT:undname.obj
 0002:0000e858       ??_C@_09EFNPDFFP@?5volatile?$AA@ 00000001400f7858     LIBCMT:undname.obj
 0002:0000e864       ??_C@_05BNCCCJPP@const?$AA@ 00000001400f7864     LIBCMT:undname.obj
 0002:0000e86c       ??_C@_06BNJCAIGJ@double?$AA@ 00000001400f786c     LIBCMT:undname.obj
 0002:0000e874       ??_C@_05KNFBNCOH@float?$AA@ 00000001400f7874     LIBCMT:undname.obj
 0002:0000e87c       ??_C@_04GOKPGOLB@long?$AA@ 00000001400f787c     LIBCMT:undname.obj
 0002:0000e884       ??_C@_03JBIPMCLC@int?$AA@  00000001400f7884     LIBCMT:undname.obj
 0002:0000e888       ??_C@_05BFKKPKCG@short?$AA@ 00000001400f7888     LIBCMT:undname.obj
 0002:0000e890       ??_C@_04ENMBGAPA@char?$AA@ 00000001400f7890     LIBCMT:undname.obj
 0002:0000e898       ??_C@_0BI@DFKBFLJE@GetProcessWindowStation?$AA@ 00000001400f7898     LIBCMT:crtmbox.obj
 0002:0000e8b0       ??_C@_0BK@CIDNPOGP@GetUserObjectInformationA?$AA@ 00000001400f78b0     LIBCMT:crtmbox.obj
 0002:0000e8d0       ??_C@_0BD@HHGDFDBJ@GetLastActivePopup?$AA@ 00000001400f78d0     LIBCMT:crtmbox.obj
 0002:0000e8e8       ??_C@_0BA@HNOPNCHB@GetActiveWindow?$AA@ 00000001400f78e8     LIBCMT:crtmbox.obj
 0002:0000e8f8       ??_C@_0M@CHKKJDAI@MessageBoxA?$AA@ 00000001400f78f8     LIBCMT:crtmbox.obj
 0002:0000e908       ??_C@_0L@NDEGIDAG@USER32?4DLL?$AA@ 00000001400f7908     LIBCMT:crtmbox.obj
 0002:0000e914       ??_C@_13NOLLCAOD@?$AA?$AA?$AA?$AA@ 00000001400f7914     LIBCMT:a_map.obj
 0002:0000e918       ??_C@_05JGDBENOH@_logb?$AA@ 00000001400f7918     LIBCMT:fpexcept.obj
 0002:0000e920       ??_C@_03ONILCKOB@_yn?$AA@  00000001400f7920     LIBCMT:fpexcept.obj
 0002:0000e924       ??_C@_03NAKIGLHK@_y1?$AA@  00000001400f7924     LIBCMT:fpexcept.obj
 0002:0000e928       ??_C@_03MJLDFKDL@_y0?$AA@  00000001400f7928     LIBCMT:fpexcept.obj
 0002:0000e92c       ??_C@_05GKKHEGJL@frexp?$AA@ 00000001400f792c     LIBCMT:fpexcept.obj
 0002:0000e934       ??_C@_04KEPJIHGP@fmod?$AA@ 00000001400f7934     LIBCMT:fpexcept.obj
 0002:0000e93c       ??_C@_06MEIMCGCF@_hypot?$AA@ 00000001400f793c     LIBCMT:fpexcept.obj
 0002:0000e944       ??_C@_05KBKMEMPO@_cabs?$AA@ 00000001400f7944     LIBCMT:fpexcept.obj
 0002:0000e94c       ??_C@_05CEJMAHNP@ldexp?$AA@ 00000001400f794c     LIBCMT:fpexcept.obj
 0002:0000e954       ??_C@_04EHEDPDJG@modf?$AA@ 00000001400f7954     LIBCMT:fpexcept.obj
 0002:0000e95c       ??_C@_04ODHECPBC@fabs?$AA@ 00000001400f795c     LIBCMT:fpexcept.obj
 0002:0000e964       ??_C@_04GFPJNGEK@ceil?$AA@ 00000001400f7964     LIBCMT:fpexcept.obj
 0002:0000e96c       ??_C@_03IIINPABG@tan?$AA@  00000001400f796c     LIBCMT:fpexcept.obj
 0002:0000e970       ??_C@_03LALBNOCG@cos?$AA@  00000001400f7970     LIBCMT:fpexcept.obj
 0002:0000e974       ??_C@_03BLEJJJBH@sin?$AA@  00000001400f7974     LIBCMT:fpexcept.obj
 0002:0000e978       ??_C@_04EIAKFFMI@sqrt?$AA@ 00000001400f7978     LIBCMT:fpexcept.obj
 0002:0000e980       ??_C@_05KNGEOGJB@atan2?$AA@ 00000001400f7980     LIBCMT:fpexcept.obj
 0002:0000e988       ??_C@_04MLLJIGOK@atan?$AA@ 00000001400f7988     LIBCMT:fpexcept.obj
 0002:0000e990       ??_C@_04PDIFKINK@acos?$AA@ 00000001400f7990     LIBCMT:fpexcept.obj
 0002:0000e998       ??_C@_04FIHNOPOL@asin?$AA@ 00000001400f7998     LIBCMT:fpexcept.obj
 0002:0000e9a0       ??_C@_04FJHINJAO@tanh?$AA@ 00000001400f79a0     LIBCMT:fpexcept.obj
 0002:0000e9a8       ??_C@_04HPJJNFIM@cosh?$AA@ 00000001400f79a8     LIBCMT:fpexcept.obj
 0002:0000e9b0       ??_C@_04COOMCNPB@sinh?$AA@ 00000001400f79b0     LIBCMT:fpexcept.obj
 0002:0000e9b8       ??_C@_05HGHHAHAP@log10?$AA@ 00000001400f79b8     LIBCMT:fpexcept.obj
 0002:0000e9c0       ??_C@_03JGHBODFD@pow?$AA@  00000001400f79c0     LIBCMT:fpexcept.obj
 0002:0000e9c4       ??_C@_03KHJOGHMM@exp?$AA@  00000001400f79c4     LIBCMT:fpexcept.obj
 0002:0000e9d0       __newctype                 00000001400f79d0     LIBCMT:ctype.obj
 0002:0000ecd0       _wctype                    00000001400f7cd0     LIBCMT:ctype.obj
 0002:0000eee0       __newclmap                 00000001400f7ee0     LIBCMT:ctype.obj
 0002:0000f060       __newcumap                 00000001400f8060     LIBCMT:ctype.obj
 0002:0000f1e0       ??_C@_08JCCMCCIL@HH?3mm?3ss?$AA@ 00000001400f81e0     LIBCMT:strftime.obj
 0002:0000f1f0       ??_C@_0BE@CKGJFCPC@dddd?0?5MMMM?5dd?0?5yyyy?$AA@ 00000001400f81f0     LIBCMT:strftime.obj
 0002:0000f208       ??_C@_08BPBNCDIB@MM?1dd?1yy?$AA@ 00000001400f8208     LIBCMT:strftime.obj
 0002:0000f214       ??_C@_02CJNFDJBF@PM?$AA@   00000001400f8214     LIBCMT:strftime.obj
 0002:0000f218       ??_C@_02DEDBPAFC@AM?$AA@   00000001400f8218     LIBCMT:strftime.obj
 0002:0000f220       ??_C@_08EDHMEBNP@December?$AA@ 00000001400f8220     LIBCMT:strftime.obj
 0002:0000f230       ??_C@_08HCHEGEOA@November?$AA@ 00000001400f8230     LIBCMT:strftime.obj
 0002:0000f240       ??_C@_07JJNFCEND@October?$AA@ 00000001400f8240     LIBCMT:strftime.obj
 0002:0000f248       ??_C@_09BHHEALKD@September?$AA@ 00000001400f8248     LIBCMT:strftime.obj
 0002:0000f254       ??_C@_06LBBHFDDG@August?$AA@ 00000001400f8254     LIBCMT:strftime.obj
 0002:0000f25c       ??_C@_04MIEPOIFP@July?$AA@ 00000001400f825c     LIBCMT:strftime.obj
 0002:0000f264       ??_C@_04CNLMGBGM@June?$AA@ 00000001400f8264     LIBCMT:strftime.obj
 0002:0000f26c       ??_C@_05DMJDNLEJ@April?$AA@ 00000001400f826c     LIBCMT:strftime.obj
 0002:0000f274       ??_C@_05HPCKOFNC@March?$AA@ 00000001400f8274     LIBCMT:strftime.obj
 0002:0000f280       ??_C@_08GNJGEPFN@February?$AA@ 00000001400f8280     LIBCMT:strftime.obj
 0002:0000f290       ??_C@_07CGJPFGJA@January?$AA@ 00000001400f8290     LIBCMT:strftime.obj
 0002:0000f298       ??_C@_03MKABNOCG@Dec?$AA@  00000001400f8298     LIBCMT:strftime.obj
 0002:0000f29c       ??_C@_03JPJOFNIA@Nov?$AA@  00000001400f829c     LIBCMT:strftime.obj
 0002:0000f2a0       ??_C@_03BMAOKBAD@Oct?$AA@  00000001400f82a0     LIBCMT:strftime.obj
 0002:0000f2a4       ??_C@_03GGCAPAJC@Sep?$AA@  00000001400f82a4     LIBCMT:strftime.obj
 0002:0000f2a8       ??_C@_03IFJFEIGA@Aug?$AA@  00000001400f82a8     LIBCMT:strftime.obj
 0002:0000f2ac       ??_C@_03LBGABGKK@Jul?$AA@  00000001400f82ac     LIBCMT:strftime.obj
 0002:0000f2b0       ??_C@_03IDFGHECI@Jun?$AA@  00000001400f82b0     LIBCMT:strftime.obj
 0002:0000f2b4       ??_C@_03CNMDKL@May?$AA@    00000001400f82b4     LIBCMT:strftime.obj
 0002:0000f2b8       ??_C@_03LEOLGMJP@Apr?$AA@  00000001400f82b8     LIBCMT:strftime.obj
 0002:0000f2bc       ??_C@_03ODNJBKGA@Mar?$AA@  00000001400f82bc     LIBCMT:strftime.obj
 0002:0000f2c0       ??_C@_03HJBDCHOM@Feb?$AA@  00000001400f82c0     LIBCMT:strftime.obj
 0002:0000f2c4       ??_C@_03JIHJHPIE@Jan?$AA@  00000001400f82c4     LIBCMT:strftime.obj
 0002:0000f2c8       ??_C@_08INBOOONO@Saturday?$AA@ 00000001400f82c8     LIBCMT:strftime.obj
 0002:0000f2d4       ??_C@_06JECMNKMI@Friday?$AA@ 00000001400f82d4     LIBCMT:strftime.obj
 0002:0000f2e0       ??_C@_08HACCIKIA@Thursday?$AA@ 00000001400f82e0     LIBCMT:strftime.obj
 0002:0000f2f0       ??_C@_09DLIGFAKA@Wednesday?$AA@ 00000001400f82f0     LIBCMT:strftime.obj
 0002:0000f300       ??_C@_07BAAGCFCM@Tuesday?$AA@ 00000001400f8300     LIBCMT:strftime.obj
 0002:0000f308       ??_C@_06JLEDEDGH@Monday?$AA@ 00000001400f8308     LIBCMT:strftime.obj
 0002:0000f310       ??_C@_06OOPIFAJ@Sunday?$AA@ 00000001400f8310     LIBCMT:strftime.obj
 0002:0000f318       ??_C@_03FEFJNEK@Sat?$AA@   00000001400f8318     LIBCMT:strftime.obj
 0002:0000f31c       ??_C@_03IDIOELNC@Fri?$AA@  00000001400f831c     LIBCMT:strftime.obj
 0002:0000f320       ??_C@_03IOFIKPDN@Thu?$AA@  00000001400f8320     LIBCMT:strftime.obj
 0002:0000f324       ??_C@_03MHOMLAJA@Wed?$AA@  00000001400f8324     LIBCMT:strftime.obj
 0002:0000f328       ??_C@_03NAGEINEP@Tue?$AA@  00000001400f8328     LIBCMT:strftime.obj
 0002:0000f32c       ??_C@_03PDAGKDH@Mon?$AA@   00000001400f832c     LIBCMT:strftime.obj
 0002:0000f330       ??_C@_03KOEHGMDN@Sun?$AA@  00000001400f8330     LIBCMT:strftime.obj
 0002:0000f334       ??_C@_03EBAPMIKO@a?1p?$AA@ 00000001400f8334     LIBCMT:strftime.obj
 0002:0000f338       ??_C@_05JAMEPDIN@am?1pm?$AA@ 00000001400f8338     LIBCMT:strftime.obj
 0002:0000f340       ??_C@_0O@FMJNFNKE@united?9states?$AA@ 00000001400f8340     LIBCMT:getqloc.obj
 0002:0000f350       ??_C@_0P@NDHFFKCA@united?9kingdom?$AA@ 00000001400f8350     LIBCMT:getqloc.obj
 0002:0000f360       ??_C@_0BC@HHDADLGF@trinidad?5?$CG?5tobago?$AA@ 00000001400f8360     LIBCMT:getqloc.obj
 0002:0000f378       ??_C@_0M@IOAEBDAC@south?9korea?$AA@ 00000001400f8378     LIBCMT:getqloc.obj
 0002:0000f388       ??_C@_0N@FIELFKIJ@south?9africa?$AA@ 00000001400f8388     LIBCMT:getqloc.obj
 0002:0000f398       ??_C@_0M@OPNDHCMC@south?5korea?$AA@ 00000001400f8398     LIBCMT:getqloc.obj
 0002:0000f3a8       ??_C@_0N@MDEOEPFI@south?5africa?$AA@ 00000001400f83a8     LIBCMT:getqloc.obj
 0002:0000f3b8       ??_C@_06FKAPCJLB@slovak?$AA@ 00000001400f83b8     LIBCMT:getqloc.obj
 0002:0000f3c0       ??_C@_0M@EFJANOAL@puerto?9rico?$AA@ 00000001400f83c0     LIBCMT:getqloc.obj
 0002:0000f3d0       ??_C@_08PGOJKDAI@pr?9china?$AA@ 00000001400f83d0     LIBCMT:getqloc.obj
 0002:0000f3e0       ??_C@_08JHDOMCMI@pr?5china?$AA@ 00000001400f83e0     LIBCMT:getqloc.obj
 0002:0000f3ec       ??_C@_02JHCHFBLL@nz?$AA@   00000001400f83ec     LIBCMT:getqloc.obj
 0002:0000f3f0       ??_C@_0M@LINHDHKP@new?9zealand?$AA@ 00000001400f83f0     LIBCMT:getqloc.obj
 0002:0000f400       ??_C@_09IIIPPBDB@hong?9kong?$AA@ 00000001400f8400     LIBCMT:getqloc.obj
 0002:0000f410       ??_C@_07HJLCKBG@holland?$AA@ 00000001400f8410     LIBCMT:getqloc.obj
 0002:0000f418       ??_C@_0O@LEHGMHAG@great?5britain?$AA@ 00000001400f8418     LIBCMT:getqloc.obj
 0002:0000f428       ??_C@_07FACOMELA@england?$AA@ 00000001400f8428     LIBCMT:getqloc.obj
 0002:0000f430       ??_C@_05JIHCEICB@czech?$AA@ 00000001400f8430     LIBCMT:getqloc.obj
 0002:0000f438       ??_C@_05BBJOBLGB@china?$AA@ 00000001400f8438     LIBCMT:getqloc.obj
 0002:0000f440       ??_C@_07GPKPHICP@britain?$AA@ 00000001400f8440     LIBCMT:getqloc.obj
 0002:0000f448       ??_C@_07MHIPBHMG@america?$AA@ 00000001400f8448     LIBCMT:getqloc.obj
 0002:0000f450       ??_C@_03KIALPMKC@usa?$AA@  00000001400f8450     LIBCMT:getqloc.obj
 0002:0000f454       ??_C@_02FGJGKGGD@us?$AA@   00000001400f8454     LIBCMT:getqloc.obj
 0002:0000f458       ??_C@_02NEINDODK@uk?$AA@   00000001400f8458     LIBCMT:getqloc.obj
 0002:0000f45c       ??_C@_05JMPCFJFJ@swiss?$AA@ 00000001400f845c     LIBCMT:getqloc.obj
 0002:0000f468       ??_C@_0BA@HLOCPIOD@swedish?9finland?$AA@ 00000001400f8468     LIBCMT:getqloc.obj
 0002:0000f478       ??_C@_0BC@PKCNIABK@spanish?9venezuela?$AA@ 00000001400f8478     LIBCMT:getqloc.obj
 0002:0000f490       ??_C@_0BA@GBHHMIJI@spanish?9uruguay?$AA@ 00000001400f8490     LIBCMT:getqloc.obj
 0002:0000f4a0       ??_C@_0BE@BHDOHPMC@spanish?9puerto?5rico?$AA@ 00000001400f84a0     LIBCMT:getqloc.obj
 0002:0000f4b8       ??_C@_0N@KMOIDGGN@spanish?9peru?$AA@ 00000001400f84b8     LIBCMT:getqloc.obj
 0002:0000f4c8       ??_C@_0BB@HMHLPGPH@spanish?9paraguay?$AA@ 00000001400f84c8     LIBCMT:getqloc.obj
 0002:0000f4e0       ??_C@_0P@MCPKNGFD@spanish?9panama?$AA@ 00000001400f84e0     LIBCMT:getqloc.obj
 0002:0000f4f0       ??_C@_0BC@IHOHGAIL@spanish?9nicaragua?$AA@ 00000001400f84f0     LIBCMT:getqloc.obj
 0002:0000f508       ??_C@_0P@KLMJDNFJ@spanish?9modern?$AA@ 00000001400f8508     LIBCMT:getqloc.obj
 0002:0000f518       ??_C@_0BA@BPAPGBCM@spanish?9mexican?$AA@ 00000001400f8518     LIBCMT:getqloc.obj
 0002:0000f528       ??_C@_0BB@PDECHHHE@spanish?9honduras?$AA@ 00000001400f8528     LIBCMT:getqloc.obj
 0002:0000f540       ??_C@_0BC@KLHKFGDB@spanish?9guatemala?$AA@ 00000001400f8540     LIBCMT:getqloc.obj
 0002:0000f558       ??_C@_0BE@MFOOKJAI@spanish?9el?5salvador?$AA@ 00000001400f8558     LIBCMT:getqloc.obj
 0002:0000f570       ??_C@_0BA@FCOKFPFC@spanish?9ecuador?$AA@ 00000001400f8570     LIBCMT:getqloc.obj
 0002:0000f580       ??_C@_0BL@PLMGIMOO@spanish?9dominican?5republic?$AA@ 00000001400f8580     LIBCMT:getqloc.obj
 0002:0000f5a0       ??_C@_0BD@HLGDNMHB@spanish?9costa?5rica?$AA@ 00000001400f85a0     LIBCMT:getqloc.obj
 0002:0000f5b8       ??_C@_0BB@PKCBKCPE@spanish?9colombia?$AA@ 00000001400f85b8     LIBCMT:getqloc.obj
 0002:0000f5d0       ??_C@_0O@MCBIJGNE@spanish?9chile?$AA@ 00000001400f85d0     LIBCMT:getqloc.obj
 0002:0000f5e0       ??_C@_0BA@BEFEIGJJ@spanish?9bolivia?$AA@ 00000001400f85e0     LIBCMT:getqloc.obj
 0002:0000f5f0       ??_C@_0BC@EMECMPD@spanish?9argentina?$AA@ 00000001400f85f0     LIBCMT:getqloc.obj
 0002:0000f608       ??_C@_0BF@EALFLENP@portuguese?9brazilian?$AA@ 00000001400f8608     LIBCMT:getqloc.obj
 0002:0000f620       ??_C@_0BC@HBLEBLNN@norwegian?9nynorsk?$AA@ 00000001400f8620     LIBCMT:getqloc.obj
 0002:0000f638       ??_C@_0BB@HMACDDCK@norwegian?9bokmal?$AA@ 00000001400f8638     LIBCMT:getqloc.obj
 0002:0000f650       ??_C@_09BAFFPPHE@norwegian?$AA@ 00000001400f8650     LIBCMT:getqloc.obj
 0002:0000f660       ??_C@_0O@EAJFJDFG@italian?9swiss?$AA@ 00000001400f8660     LIBCMT:getqloc.obj
 0002:0000f670       ??_C@_0O@CNOMPGD@irish?9english?$AA@ 00000001400f8670     LIBCMT:getqloc.obj
 0002:0000f680       ??_C@_0N@EDHBGCKG@german?9swiss?$AA@ 00000001400f8680     LIBCMT:getqloc.obj
 0002:0000f690       ??_C@_0BC@JACMHNBP@german?9luxembourg?$AA@ 00000001400f8690     LIBCMT:getqloc.obj
 0002:0000f6a8       ??_C@_0BE@HBGMGFEG@german?9lichtenstein?$AA@ 00000001400f86a8     LIBCMT:getqloc.obj
 0002:0000f6c0       ??_C@_0BA@HKKBIBKL@german?9austrian?$AA@ 00000001400f86c0     LIBCMT:getqloc.obj
 0002:0000f6d0       ??_C@_0N@GCAEPEBK@french?9swiss?$AA@ 00000001400f86d0     LIBCMT:getqloc.obj
 0002:0000f6e0       ??_C@_0BC@DJFJJCK@french?9luxembourg?$AA@ 00000001400f86e0     LIBCMT:getqloc.obj
 0002:0000f6f8       ??_C@_0BA@NNCEDFIC@french?9canadian?$AA@ 00000001400f86f8     LIBCMT:getqloc.obj
 0002:0000f708       ??_C@_0P@CMPOCLM@french?9belgian?$AA@ 00000001400f8708     LIBCMT:getqloc.obj
 0002:0000f718       ??_C@_0M@GHHDJOK@english?9usa?$AA@ 00000001400f8718     LIBCMT:getqloc.obj
 0002:0000f728       ??_C@_0L@PLDJKEIL@english?9us?$AA@ 00000001400f8728     LIBCMT:getqloc.obj
 0002:0000f738       ??_C@_0L@HJCCDMNC@english?9uk?$AA@ 00000001400f8738     LIBCMT:getqloc.obj
 0002:0000f748       ??_C@_0BK@CKLIAGJB@english?9trinidad?5y?5tobago?$AA@ 00000001400f8748     LIBCMT:getqloc.obj
 0002:0000f768       ??_C@_0BF@JMJMGNNF@english?9south?5africa?$AA@ 00000001400f8768     LIBCMT:getqloc.obj
 0002:0000f780       ??_C@_0L@DKIIFDFD@english?9nz?$AA@ 00000001400f8780     LIBCMT:getqloc.obj
 0002:0000f790       ??_C@_0BA@ONHGJCLH@english?9jamaica?$AA@ 00000001400f8790     LIBCMT:getqloc.obj
 0002:0000f7a0       ??_C@_0M@HJBGHOPO@english?9ire?$AA@ 00000001400f87a0     LIBCMT:getqloc.obj
 0002:0000f7b0       ??_C@_0BC@LFEKMIFB@english?9caribbean?$AA@ 00000001400f87b0     LIBCMT:getqloc.obj
 0002:0000f7c8       ??_C@_0M@OLDPFKHI@english?9can?$AA@ 00000001400f87c8     LIBCMT:getqloc.obj
 0002:0000f7d8       ??_C@_0P@OMDEHBMP@english?9belize?$AA@ 00000001400f87d8     LIBCMT:getqloc.obj
 0002:0000f7e8       ??_C@_0M@KFHFPFED@english?9aus?$AA@ 00000001400f87e8     LIBCMT:getqloc.obj
 0002:0000f7f8       ??_C@_0BB@MNMBKDFE@english?9american?$AA@ 00000001400f87f8     LIBCMT:getqloc.obj
 0002:0000f810       ??_C@_0O@KIDLNNBA@dutch?9belgian?$AA@ 00000001400f8810     LIBCMT:getqloc.obj
 0002:0000f820       ??_C@_0BE@JBKABBMH@chinese?9traditional?$AA@ 00000001400f8820     LIBCMT:getqloc.obj
 0002:0000f838       ??_C@_0BC@MJJMPKCG@chinese?9singapore?$AA@ 00000001400f8838     LIBCMT:getqloc.obj
 0002:0000f850       ??_C@_0BD@FDKADDCP@chinese?9simplified?$AA@ 00000001400f8850     LIBCMT:getqloc.obj
 0002:0000f868       ??_C@_0BB@DBEFDDME@chinese?9hongkong?$AA@ 00000001400f8868     LIBCMT:getqloc.obj
 0002:0000f880       ??_C@_07DHNMFMCI@chinese?$AA@ 00000001400f8880     LIBCMT:getqloc.obj
 0002:0000f888       ??_C@_03FNDDCHI@chi?$AA@   00000001400f8888     LIBCMT:getqloc.obj
 0002:0000f88c       ??_C@_03BMMIADDJ@chh?$AA@  00000001400f888c     LIBCMT:getqloc.obj
 0002:0000f890       ??_C@_08OAIPJDGI@canadian?$AA@ 00000001400f8890     LIBCMT:getqloc.obj
 0002:0000f8a0       ??_C@_07HBPMNPNJ@belgian?$AA@ 00000001400f88a0     LIBCMT:getqloc.obj
 0002:0000f8a8       ??_C@_0L@OEKOPBEL@australian?$AA@ 00000001400f88a8     LIBCMT:getqloc.obj
 0002:0000f8b8       ??_C@_0BB@MEIMBEDG@american?9english?$AA@ 00000001400f88b8     LIBCMT:getqloc.obj
 0002:0000f8d0       ??_C@_0BB@DFMDPDGB@american?5english?$AA@ 00000001400f88d0     LIBCMT:getqloc.obj
 0002:0000f8e8       ??_C@_08IJLOKOLL@american?$AA@ 00000001400f88e8     LIBCMT:getqloc.obj
 0002:0000f900       __rg_language              00000001400f8900     LIBCMT:getqloc.obj
 0002:0000fd10       __rg_country               00000001400f8d10     LIBCMT:getqloc.obj
 0002:0000fe80       __rglangidNotDefault       00000001400f8e80     LIBCMT:getqloc.obj
 0002:0000fe94       ??_C@_03NFKLAGEF@OCP?$AA@  00000001400f8e94     LIBCMT:getqloc.obj
 0002:0000fe98       ??_C@_03DFHEHBHG@ACP?$AA@  00000001400f8e98     LIBCMT:getqloc.obj
 0002:0000fea0       ??_C@_0BC@NFIEMBLL@Norwegian?9Nynorsk?$AA@ 00000001400f8ea0     LIBCMT:getqloc.obj
 0002:0000feb4       ??_C@_06IMKFLFPG@1?$CDQNAN?$AA@ 00000001400f8eb4     LIBCMT:x10fout.obj
 0002:0000febc       ??_C@_05DNEBIAHO@1?$CDINF?$AA@ 00000001400f8ebc     LIBCMT:x10fout.obj
 0002:0000fec4       ??_C@_05PHHOCPM@1?$CDIND?$AA@ 00000001400f8ec4     LIBCMT:x10fout.obj
 0002:0000fecc       ??_C@_06PGGFOGJG@1?$CDSNAN?$AA@ 00000001400f8ecc     LIBCMT:x10fout.obj
 0002:0000fef8       ??_7HASH64withTransform@TaoCrypt@@6B@ 00000001400f8ef8     taocrypt:hash.obj
 0002:0000ff48       ??_7HASHwithTransform@TaoCrypt@@6B@ 00000001400f8f48     taocrypt:hash.obj
 0002:00010088       ??_7MultiplicativeGroupT@AbstractRing@TaoCrypt@@6B@ 00000001400f9088     taocrypt:integer.obj
 0002:000100f8       ??_7ModularArithmetic@TaoCrypt@@6B@ 00000001400f90f8     taocrypt:integer.obj
 0002:000101d8       ??_7MontgomeryRepresentation@TaoCrypt@@6B@ 00000001400f91d8     taocrypt:integer.obj
 0002:000102b8       ??_7EuclideanDomainOf@TaoCrypt@@6B@ 00000001400f92b8     taocrypt:integer.obj
 0002:00010718       ??_7SHA256@TaoCrypt@@6B@   00000001400f9718     taocrypt:sha.obj
 0002:00010768       ??_7SHA224@TaoCrypt@@6B@   00000001400f9768     taocrypt:sha.obj
 0002:000107b8       ??_7SHA512@TaoCrypt@@6B@   00000001400f97b8     taocrypt:sha.obj
 0002:00010808       ??_7SHA384@TaoCrypt@@6B@   00000001400f9808     taocrypt:sha.obj
 0002:000110f0       ?Te@AES@TaoCrypt@@0QAY0BAA@$$CBIA 00000001400fa0f0     taocrypt:aes.obj
 0002:000124f0       ?Td@AES@TaoCrypt@@0QAY0BAA@$$CBIA 00000001400fb4f0     taocrypt:aes.obj
 0002:000138f8       ??_7BER_Decoder@TaoCrypt@@6B@ 00000001400fc8f8     taocrypt:dsa.obj
 0002:00013910       ??_7DSA_Private_Decoder@TaoCrypt@@6B@ 00000001400fc910     taocrypt:dsa.obj
 0002:00013928       ??_7DSA_Public_Decoder@TaoCrypt@@6B@ 00000001400fc928     taocrypt:dsa.obj
 0002:00013940       ??_7DH_Decoder@TaoCrypt@@6B@ 00000001400fc940     taocrypt:dh.obj
 0002:00013950       __real@4014000000000000    00000001400fc950     taocrypt:dh.obj
 0002:00013958       __real@4003333333333333    00000001400fc958     taocrypt:dh.obj
 0002:00013960       __real@3fd5555555555555    00000001400fc960     taocrypt:dh.obj
 0002:00013968       __real@3fe5555555555555    00000001400fc968     taocrypt:dh.obj
 0002:00013978       ??_7RSA_Private_Decoder@TaoCrypt@@6B@ 00000001400fc978     taocrypt:rsa.obj
 0002:00013990       ??_7RSA_Public_Decoder@TaoCrypt@@6B@ 00000001400fc990     taocrypt:rsa.obj
 0002:000139a8       ??_7DER_Encoder@TaoCrypt@@6B@ 00000001400fc9a8     taocrypt:asn.obj
 0002:000139b8       ??_7CertDecoder@TaoCrypt@@6B@ 00000001400fc9b8     taocrypt:asn.obj
 0002:000139c8       ??_C@_0P@FGCJCCJK@?1emailAddress?$DN?$AA@ 00000001400fc9c8     taocrypt:asn.obj
 0002:000139d8       ??_C@_04LJKEFMLJ@?1OU?$DN?$AA@ 00000001400fc9d8     taocrypt:asn.obj
 0002:000139e0       ??_C@_03DHMEBNMI@?1O?$DN?$AA@ 00000001400fc9e0     taocrypt:asn.obj
 0002:000139e4       ??_C@_04KCKJNOKJ@?1ST?$DN?$AA@ 00000001400fc9e4     taocrypt:asn.obj
 0002:000139ec       ??_C@_03DFICKDJB@?1L?$DN?$AA@ 00000001400fc9ec     taocrypt:asn.obj
 0002:000139f0       ??_C@_03DONOOEKM@?1C?$DN?$AA@ 00000001400fc9f0     taocrypt:asn.obj
 0002:000139f4       ??_C@_04LDBIPIAP@?1SN?$DN?$AA@ 00000001400fc9f4     taocrypt:asn.obj
 0002:00013a30       ??_7Signature_Encoder@TaoCrypt@@6B@ 00000001400fca30     taocrypt:asn.obj
 0002:00013a38       ??_C@_02GMLFBBN@wb?$AA@    00000001400fca38     taocrypt:file.obj
 0002:00013a40       ?rcon_@AES@TaoCrypt@@0QBIB 00000001400fca40     taocrypt:aestables.obj
 0002:00013b78       ??_7MD2@TaoCrypt@@6B@      00000001400fcb78     taocrypt:md2.obj
 0002:00014020       __real@3fe0000000000000    00000001400fd020     LIBCMT:log.obj
 0002:00014028       __real@3f80000000000000    00000001400fd028     LIBCMT:log.obj
 0002:00014030       __real@4000000000000000    00000001400fd030     LIBCMT:log.obj
 0002:00018010       _tls_used                  0000000140101010     LIBCMT:tlssup.obj
 0002:000182f0       ??_R4Command@@6B@          00000001401012f0     command.obj
 0002:00018318       ??_R3Command@@8            0000000140101318     command.obj
 0002:00018330       ??_R2Command@@8            0000000140101330     command.obj
 0002:00018340       ??_R1A@?0A@EA@Command@@8   0000000140101340     command.obj
 0002:00018370       ??_R4Show_instance_status@@6B@ 0000000140101370     commands.obj
 0002:00018398       ??_R3Show_instance_status@@8 0000000140101398     commands.obj
 0002:000183b0       ??_R2Show_instance_status@@8 00000001401013b0     commands.obj
 0002:000183c8       ??_R1A@?0A@EA@Show_instance_status@@8 00000001401013c8     commands.obj
 0002:000183f8       ??_R4Show_instance_options@@6B@ 00000001401013f8     commands.obj
 0002:00018420       ??_R3Show_instance_options@@8 0000000140101420     commands.obj
 0002:00018438       ??_R2Show_instance_options@@8 0000000140101438     commands.obj
 0002:00018450       ??_R1A@?0A@EA@Show_instance_options@@8 0000000140101450     commands.obj
 0002:00018480       ??_R4Start_instance@@6B@   0000000140101480     commands.obj
 0002:000184a8       ??_R3Start_instance@@8     00000001401014a8     commands.obj
 0002:000184c0       ??_R2Start_instance@@8     00000001401014c0     commands.obj
 0002:000184d8       ??_R1A@?0A@EA@Start_instance@@8 00000001401014d8     commands.obj
 0002:00018508       ??_R4Show_instance_log@@6B@ 0000000140101508     commands.obj
 0002:00018530       ??_R3Show_instance_log@@8  0000000140101530     commands.obj
 0002:00018548       ??_R2Show_instance_log@@8  0000000140101548     commands.obj
 0002:00018560       ??_R1A@?0A@EA@Show_instance_log@@8 0000000140101560     commands.obj
 0002:00018590       ??_R4Show_instance_log_files@@6B@ 0000000140101590     commands.obj
 0002:000185b8       ??_R3Show_instance_log_files@@8 00000001401015b8     commands.obj
 0002:000185d0       ??_R2Show_instance_log_files@@8 00000001401015d0     commands.obj
 0002:000185e8       ??_R1A@?0A@EA@Show_instance_log_files@@8 00000001401015e8     commands.obj
 0002:00018618       ??_R4Set_option@@6B@       0000000140101618     commands.obj
 0002:00018640       ??_R3Set_option@@8         0000000140101640     commands.obj
 0002:00018658       ??_R2Set_option@@8         0000000140101658     commands.obj
 0002:00018670       ??_R1A@?0A@EA@Set_option@@8 0000000140101670     commands.obj
 0002:000186a0       ??_R4Stop_instance@@6B@    00000001401016a0     commands.obj
 0002:000186c8       ??_R3Stop_instance@@8      00000001401016c8     commands.obj
 0002:000186e0       ??_R2Stop_instance@@8      00000001401016e0     commands.obj
 0002:000186f8       ??_R1A@?0A@EA@Stop_instance@@8 00000001401016f8     commands.obj
 0002:00018728       ??_R4Show_instances@@6B@   0000000140101728     parse.obj
 0002:00018750       ??_R3Show_instances@@8     0000000140101750     parse.obj
 0002:00018768       ??_R2Show_instances@@8     0000000140101768     parse.obj
 0002:00018780       ??_R1A@?0A@EA@Show_instances@@8 0000000140101780     parse.obj
 0002:000187b0       ??_R4Flush_instances@@6B@  00000001401017b0     parse.obj
 0002:000187d8       ??_R3Flush_instances@@8    00000001401017d8     parse.obj
 0002:000187f0       ??_R2Flush_instances@@8    00000001401017f0     parse.obj
 0002:00018808       ??_R1A@?0A@EA@Flush_instances@@8 0000000140101808     parse.obj
 0002:00018838       ??_R4Syntax_error@@6B@     0000000140101838     parse.obj
 0002:00018860       ??_R3Syntax_error@@8       0000000140101860     parse.obj
 0002:00018878       ??_R2Syntax_error@@8       0000000140101878     parse.obj
 0002:00018890       ??_R1A@?0A@EA@Syntax_error@@8 0000000140101890     parse.obj
 0002:000188c0       ??_R4Unset_option@@6B@     00000001401018c0     parse.obj
 0002:000188e8       ??_R3Unset_option@@8       00000001401018e8     parse.obj
 0002:00018900       ??_R2Unset_option@@8       0000000140101900     parse.obj
 0002:00018928       ??_R1A@?0A@EA@Unset_option@@8 0000000140101928     parse.obj
 0002:00018958       ??_R4IMService@@6B@        0000000140101958     IMService.obj
 0002:00018980       ??_R3IMService@@8          0000000140101980     IMService.obj
 0002:00018998       ??_R2IMService@@8          0000000140101998     IMService.obj
 0002:000189b0       ??_R1A@?0A@EA@IMService@@8 00000001401019b0     IMService.obj
 0002:000189e0       ??_R1A@?0A@EA@WindowsService@@8 00000001401019e0     IMService.obj
 0002:00018a10       ??_R3WindowsService@@8     0000000140101a10     IMService.obj
 0002:00018a28       ??_R2WindowsService@@8     0000000140101a28     IMService.obj
 0002:00018a38       ??_R4WindowsService@@6B@   0000000140101a38     WindowsService.obj
 0002:00018a60       ??_R4Message@yaSSL@@6B@    0000000140101a60     yassl:ssl.obj
 0002:00018a80       ??_R3Message@yaSSL@@8      0000000140101a80     yassl:ssl.obj
 0002:00018a98       ??_R2Message@yaSSL@@8      0000000140101a98     yassl:ssl.obj
 0002:00018ab0       ??_R1A@?0A@EA@Message@yaSSL@@8 0000000140101ab0     yassl:ssl.obj
 0002:00018ad8       ??_R17?0A@EA@virtual_base@yaSSL@@8 0000000140101ad8     yassl:ssl.obj
 0002:00018b00       ??_R3virtual_base@yaSSL@@8 0000000140101b00     yassl:ssl.obj
 0002:00018b18       ??_R2virtual_base@yaSSL@@8 0000000140101b18     yassl:ssl.obj
 0002:00018b28       ??_R1A@?0A@EA@virtual_base@yaSSL@@8 0000000140101b28     yassl:ssl.obj
 0002:00018b50       ??_R4HandShakeBase@yaSSL@@6B@ 0000000140101b50     yassl:ssl.obj
 0002:00018b70       ??_R3HandShakeBase@yaSSL@@8 0000000140101b70     yassl:ssl.obj
 0002:00018b88       ??_R2HandShakeBase@yaSSL@@8 0000000140101b88     yassl:ssl.obj
 0002:00018ba0       ??_R1A@?0A@EA@HandShakeBase@yaSSL@@8 0000000140101ba0     yassl:ssl.obj
 0002:00018bc8       ??_R4HASH@TaoCrypt@@6B@    0000000140101bc8     yassl:ssl.obj
 0002:00018be8       ??_R3HASH@TaoCrypt@@8      0000000140101be8     yassl:ssl.obj
 0002:00018c00       ??_R2HASH@TaoCrypt@@8      0000000140101c00     yassl:ssl.obj
 0002:00018c18       ??_R1A@?0A@EA@HASH@TaoCrypt@@8 0000000140101c18     yassl:ssl.obj
 0002:00018c40       ??_R17?0A@EA@virtual_base@TaoCrypt@@8 0000000140101c40     yassl:ssl.obj
 0002:00018c68       ??_R3virtual_base@TaoCrypt@@8 0000000140101c68     yassl:ssl.obj
 0002:00018c80       ??_R2virtual_base@TaoCrypt@@8 0000000140101c80     yassl:ssl.obj
 0002:00018c90       ??_R1A@?0A@EA@virtual_base@TaoCrypt@@8 0000000140101c90     yassl:ssl.obj
 0002:00018cb8       ??_R4MD5@TaoCrypt@@6B@     0000000140101cb8     yassl:ssl.obj
 0002:00018cd8       ??_R3MD5@TaoCrypt@@8       0000000140101cd8     yassl:ssl.obj
 0002:00018cf0       ??_R2MD5@TaoCrypt@@8       0000000140101cf0     yassl:ssl.obj
 0002:00018d18       ??_R1A@?0A@EA@MD5@TaoCrypt@@8 0000000140101d18     yassl:ssl.obj
 0002:00018d40       ??_R1A@?0A@EA@HASHwithTransform@TaoCrypt@@8 0000000140101d40     yassl:ssl.obj
 0002:00018d68       ??_R3HASHwithTransform@TaoCrypt@@8 0000000140101d68     yassl:ssl.obj
 0002:00018d80       ??_R2HASHwithTransform@TaoCrypt@@8 0000000140101d80     yassl:ssl.obj
 0002:00018da0       ??_R4MD4@TaoCrypt@@6B@     0000000140101da0     yassl:ssl.obj
 0002:00018dc0       ??_R3MD4@TaoCrypt@@8       0000000140101dc0     yassl:ssl.obj
 0002:00018dd8       ??_R2MD4@TaoCrypt@@8       0000000140101dd8     yassl:ssl.obj
 0002:00018e00       ??_R1A@?0A@EA@MD4@TaoCrypt@@8 0000000140101e00     yassl:ssl.obj
 0002:00018e28       ??_R4Digest@yaSSL@@6B@     0000000140101e28     yassl:crypto_wrapper.obj
 0002:00018e48       ??_R3Digest@yaSSL@@8       0000000140101e48     yassl:crypto_wrapper.obj
 0002:00018e60       ??_R2Digest@yaSSL@@8       0000000140101e60     yassl:crypto_wrapper.obj
 0002:00018e78       ??_R1A@?0A@EA@Digest@yaSSL@@8 0000000140101e78     yassl:crypto_wrapper.obj
 0002:00018ea0       ??_R4BulkCipher@yaSSL@@6B@ 0000000140101ea0     yassl:crypto_wrapper.obj
 0002:00018ec0       ??_R3BulkCipher@yaSSL@@8   0000000140101ec0     yassl:crypto_wrapper.obj
 0002:00018ed8       ??_R2BulkCipher@yaSSL@@8   0000000140101ed8     yassl:crypto_wrapper.obj
 0002:00018ef0       ??_R1A@?0A@EA@BulkCipher@yaSSL@@8 0000000140101ef0     yassl:crypto_wrapper.obj
 0002:00018f18       ??_R4Auth@yaSSL@@6B@       0000000140101f18     yassl:crypto_wrapper.obj
 0002:00018f38       ??_R3Auth@yaSSL@@8         0000000140101f38     yassl:crypto_wrapper.obj
 0002:00018f50       ??_R2Auth@yaSSL@@8         0000000140101f50     yassl:crypto_wrapper.obj
 0002:00018f68       ??_R1A@?0A@EA@Auth@yaSSL@@8 0000000140101f68     yassl:crypto_wrapper.obj
 0002:00018f90       ??_R4SHA@TaoCrypt@@6B@     0000000140101f90     yassl:crypto_wrapper.obj
 0002:00018fb0       ??_R3SHA@TaoCrypt@@8       0000000140101fb0     yassl:crypto_wrapper.obj
 0002:00018fc8       ??_R2SHA@TaoCrypt@@8       0000000140101fc8     yassl:crypto_wrapper.obj
 0002:00018ff0       ??_R1A@?0A@EA@SHA@TaoCrypt@@8 0000000140101ff0     yassl:crypto_wrapper.obj
 0002:00019018       ??_R4RIPEMD160@TaoCrypt@@6B@ 0000000140102018     yassl:crypto_wrapper.obj
 0002:00019038       ??_R3RIPEMD160@TaoCrypt@@8 0000000140102038     yassl:crypto_wrapper.obj
 0002:00019050       ??_R2RIPEMD160@TaoCrypt@@8 0000000140102050     yassl:crypto_wrapper.obj
 0002:00019078       ??_R1A@?0A@EA@RIPEMD160@TaoCrypt@@8 0000000140102078     yassl:crypto_wrapper.obj
 0002:000190a0       ??_R4Mode_BASE@TaoCrypt@@6B@ 00000001401020a0     yassl:crypto_wrapper.obj
 0002:000190c0       ??_R3Mode_BASE@TaoCrypt@@8 00000001401020c0     yassl:crypto_wrapper.obj
 0002:000190d8       ??_R2Mode_BASE@TaoCrypt@@8 00000001401020d8     yassl:crypto_wrapper.obj
 0002:000190f0       ??_R1A@?0A@EA@Mode_BASE@TaoCrypt@@8 00000001401020f0     yassl:crypto_wrapper.obj
 0002:00019118       ??_R4DES@TaoCrypt@@6B@     0000000140102118     yassl:crypto_wrapper.obj
 0002:00019138       ??_R3DES@TaoCrypt@@8       0000000140102138     yassl:crypto_wrapper.obj
 0002:00019150       ??_R2DES@TaoCrypt@@8       0000000140102150     yassl:crypto_wrapper.obj
 0002:00019178       ??_R1A@?0A@EA@DES@TaoCrypt@@8 0000000140102178     yassl:crypto_wrapper.obj
 0002:000191a0       ??_R1EI@?0A@EA@BasicDES@TaoCrypt@@8 00000001401021a0     yassl:crypto_wrapper.obj
 0002:000191c8       ??_R3BasicDES@TaoCrypt@@8  00000001401021c8     yassl:crypto_wrapper.obj
 0002:000191e0       ??_R2BasicDES@TaoCrypt@@8  00000001401021e0     yassl:crypto_wrapper.obj
 0002:000191f0       ??_R1A@?0A@EA@BasicDES@TaoCrypt@@8 00000001401021f0     yassl:crypto_wrapper.obj
 0002:00019218       ??_R4DES_EDE3@TaoCrypt@@6B@ 0000000140102218     yassl:crypto_wrapper.obj
 0002:00019238       ??_R3DES_EDE3@TaoCrypt@@8  0000000140102238     yassl:crypto_wrapper.obj
 0002:00019250       ??_R2DES_EDE3@TaoCrypt@@8  0000000140102250     yassl:crypto_wrapper.obj
 0002:00019270       ??_R1A@?0A@EA@DES_EDE3@TaoCrypt@@8 0000000140102270     yassl:crypto_wrapper.obj
 0002:00019298       ??_R4AES@TaoCrypt@@6B@     0000000140102298     yassl:crypto_wrapper.obj
 0002:000192b8       ??_R3AES@TaoCrypt@@8       00000001401022b8     yassl:crypto_wrapper.obj
 0002:000192d0       ??_R2AES@TaoCrypt@@8       00000001401022d0     yassl:crypto_wrapper.obj
 0002:000192f0       ??_R1A@?0A@EA@AES@TaoCrypt@@8 00000001401022f0     yassl:crypto_wrapper.obj
 0002:00019318       ??_R4MD5@yaSSL@@6B@        0000000140102318     yassl:crypto_wrapper.obj
 0002:00019338       ??_R3MD5@yaSSL@@8          0000000140102338     yassl:crypto_wrapper.obj
 0002:00019350       ??_R2MD5@yaSSL@@8          0000000140102350     yassl:crypto_wrapper.obj
 0002:00019370       ??_R1A@?0A@EA@MD5@yaSSL@@8 0000000140102370     yassl:crypto_wrapper.obj
 0002:00019398       ??_R4SHA@yaSSL@@6B@        0000000140102398     yassl:crypto_wrapper.obj
 0002:000193b8       ??_R3SHA@yaSSL@@8          00000001401023b8     yassl:crypto_wrapper.obj
 0002:000193d0       ??_R2SHA@yaSSL@@8          00000001401023d0     yassl:crypto_wrapper.obj
 0002:000193f0       ??_R1A@?0A@EA@SHA@yaSSL@@8 00000001401023f0     yassl:crypto_wrapper.obj
 0002:00019418       ??_R4RMD@yaSSL@@6B@        0000000140102418     yassl:crypto_wrapper.obj
 0002:00019438       ??_R3RMD@yaSSL@@8          0000000140102438     yassl:crypto_wrapper.obj
 0002:00019450       ??_R2RMD@yaSSL@@8          0000000140102450     yassl:crypto_wrapper.obj
 0002:00019470       ??_R1A@?0A@EA@RMD@yaSSL@@8 0000000140102470     yassl:crypto_wrapper.obj
 0002:00019498       ??_R4RC4@yaSSL@@6B@        0000000140102498     yassl:crypto_wrapper.obj
 0002:000194b8       ??_R3RC4@yaSSL@@8          00000001401024b8     yassl:crypto_wrapper.obj
 0002:000194d0       ??_R2RC4@yaSSL@@8          00000001401024d0     yassl:crypto_wrapper.obj
 0002:000194f0       ??_R1A@?0A@EA@RC4@yaSSL@@8 00000001401024f0     yassl:crypto_wrapper.obj
 0002:00019518       ??_R4AES@yaSSL@@6B@        0000000140102518     yassl:crypto_wrapper.obj
 0002:00019538       ??_R3AES@yaSSL@@8          0000000140102538     yassl:crypto_wrapper.obj
 0002:00019550       ??_R2AES@yaSSL@@8          0000000140102550     yassl:crypto_wrapper.obj
 0002:00019570       ??_R1A@?0A@EA@AES@yaSSL@@8 0000000140102570     yassl:crypto_wrapper.obj
 0002:00019598       ??_R4HMAC_MD5@yaSSL@@6B@   0000000140102598     yassl:crypto_wrapper.obj
 0002:000195b8       ??_R3HMAC_MD5@yaSSL@@8     00000001401025b8     yassl:crypto_wrapper.obj
 0002:000195d0       ??_R2HMAC_MD5@yaSSL@@8     00000001401025d0     yassl:crypto_wrapper.obj
 0002:000195f0       ??_R1A@?0A@EA@HMAC_MD5@yaSSL@@8 00000001401025f0     yassl:crypto_wrapper.obj
 0002:00019618       ??_R4HMAC_SHA@yaSSL@@6B@   0000000140102618     yassl:crypto_wrapper.obj
 0002:00019638       ??_R3HMAC_SHA@yaSSL@@8     0000000140102638     yassl:crypto_wrapper.obj
 0002:00019650       ??_R2HMAC_SHA@yaSSL@@8     0000000140102650     yassl:crypto_wrapper.obj
 0002:00019670       ??_R1A@?0A@EA@HMAC_SHA@yaSSL@@8 0000000140102670     yassl:crypto_wrapper.obj
 0002:00019698       ??_R4HMAC_RMD@yaSSL@@6B@   0000000140102698     yassl:crypto_wrapper.obj
 0002:000196b8       ??_R3HMAC_RMD@yaSSL@@8     00000001401026b8     yassl:crypto_wrapper.obj
 0002:000196d0       ??_R2HMAC_RMD@yaSSL@@8     00000001401026d0     yassl:crypto_wrapper.obj
 0002:000196f0       ??_R1A@?0A@EA@HMAC_RMD@yaSSL@@8 00000001401026f0     yassl:crypto_wrapper.obj
 0002:00019718       ??_R4DES@yaSSL@@6B@        0000000140102718     yassl:crypto_wrapper.obj
 0002:00019738       ??_R3DES@yaSSL@@8          0000000140102738     yassl:crypto_wrapper.obj
 0002:00019750       ??_R2DES@yaSSL@@8          0000000140102750     yassl:crypto_wrapper.obj
 0002:00019770       ??_R1A@?0A@EA@DES@yaSSL@@8 0000000140102770     yassl:crypto_wrapper.obj
 0002:00019798       ??_R4DES_EDE@yaSSL@@6B@    0000000140102798     yassl:crypto_wrapper.obj
 0002:000197b8       ??_R3DES_EDE@yaSSL@@8      00000001401027b8     yassl:crypto_wrapper.obj
 0002:000197d0       ??_R2DES_EDE@yaSSL@@8      00000001401027d0     yassl:crypto_wrapper.obj
 0002:000197f0       ??_R1A@?0A@EA@DES_EDE@yaSSL@@8 00000001401027f0     yassl:crypto_wrapper.obj
 0002:00019818       ??_R4DSS@yaSSL@@6B@        0000000140102818     yassl:crypto_wrapper.obj
 0002:00019838       ??_R3DSS@yaSSL@@8          0000000140102838     yassl:crypto_wrapper.obj
 0002:00019850       ??_R2DSS@yaSSL@@8          0000000140102850     yassl:crypto_wrapper.obj
 0002:00019870       ??_R1A@?0A@EA@DSS@yaSSL@@8 0000000140102870     yassl:crypto_wrapper.obj
 0002:00019898       ??_R4RSA@yaSSL@@6B@        0000000140102898     yassl:crypto_wrapper.obj
 0002:000198b8       ??_R3RSA@yaSSL@@8          00000001401028b8     yassl:crypto_wrapper.obj
 0002:000198d0       ??_R2RSA@yaSSL@@8          00000001401028d0     yassl:crypto_wrapper.obj
 0002:000198f0       ??_R1A@?0A@EA@RSA@yaSSL@@8 00000001401028f0     yassl:crypto_wrapper.obj
 0002:00019918       ??_R4HandShakeHeader@yaSSL@@6B@ 0000000140102918     yassl:yassl_imp.obj
 0002:00019938       ??_R3HandShakeHeader@yaSSL@@8 0000000140102938     yassl:yassl_imp.obj
 0002:00019950       ??_R2HandShakeHeader@yaSSL@@8 0000000140102950     yassl:yassl_imp.obj
 0002:00019970       ??_R1A@?0A@EA@HandShakeHeader@yaSSL@@8 0000000140102970     yassl:yassl_imp.obj
 0002:00019998       ??_R4ServerKeyBase@yaSSL@@6B@ 0000000140102998     yassl:yassl_imp.obj
 0002:000199b8       ??_R3ServerKeyBase@yaSSL@@8 00000001401029b8     yassl:yassl_imp.obj
 0002:000199d0       ??_R2ServerKeyBase@yaSSL@@8 00000001401029d0     yassl:yassl_imp.obj
 0002:000199e8       ??_R1A@?0A@EA@ServerKeyBase@yaSSL@@8 00000001401029e8     yassl:yassl_imp.obj
 0002:00019a10       ??_R4ClientKeyBase@yaSSL@@6B@ 0000000140102a10     yassl:yassl_imp.obj
 0002:00019a30       ??_R3ClientKeyBase@yaSSL@@8 0000000140102a30     yassl:yassl_imp.obj
 0002:00019a48       ??_R2ClientKeyBase@yaSSL@@8 0000000140102a48     yassl:yassl_imp.obj
 0002:00019a60       ??_R1A@?0A@EA@ClientKeyBase@yaSSL@@8 0000000140102a60     yassl:yassl_imp.obj
 0002:00019a88       ??_R4ClientDiffieHellmanPublic@yaSSL@@6B@ 0000000140102a88     yassl:yassl_imp.obj
 0002:00019aa8       ??_R3ClientDiffieHellmanPublic@yaSSL@@8 0000000140102aa8     yassl:yassl_imp.obj
 0002:00019ac0       ??_R2ClientDiffieHellmanPublic@yaSSL@@8 0000000140102ac0     yassl:yassl_imp.obj
 0002:00019ae0       ??_R1A@?0A@EA@ClientDiffieHellmanPublic@yaSSL@@8 0000000140102ae0     yassl:yassl_imp.obj
 0002:00019b08       ??_R4ChangeCipherSpec@yaSSL@@6B@ 0000000140102b08     yassl:yassl_imp.obj
 0002:00019b28       ??_R3ChangeCipherSpec@yaSSL@@8 0000000140102b28     yassl:yassl_imp.obj
 0002:00019b40       ??_R2ChangeCipherSpec@yaSSL@@8 0000000140102b40     yassl:yassl_imp.obj
 0002:00019b60       ??_R1A@?0A@EA@ChangeCipherSpec@yaSSL@@8 0000000140102b60     yassl:yassl_imp.obj
 0002:00019b88       ??_R4Alert@yaSSL@@6B@      0000000140102b88     yassl:yassl_imp.obj
 0002:00019ba8       ??_R3Alert@yaSSL@@8        0000000140102ba8     yassl:yassl_imp.obj
 0002:00019bc0       ??_R2Alert@yaSSL@@8        0000000140102bc0     yassl:yassl_imp.obj
 0002:00019be0       ??_R1A@?0A@EA@Alert@yaSSL@@8 0000000140102be0     yassl:yassl_imp.obj
 0002:00019c08       ??_R4Data@yaSSL@@6B@       0000000140102c08     yassl:yassl_imp.obj
 0002:00019c28       ??_R3Data@yaSSL@@8         0000000140102c28     yassl:yassl_imp.obj
 0002:00019c40       ??_R2Data@yaSSL@@8         0000000140102c40     yassl:yassl_imp.obj
 0002:00019c60       ??_R1A@?0A@EA@Data@yaSSL@@8 0000000140102c60     yassl:yassl_imp.obj
 0002:00019c88       ??_R4Certificate@yaSSL@@6B@ 0000000140102c88     yassl:yassl_imp.obj
 0002:00019ca8       ??_R3Certificate@yaSSL@@8  0000000140102ca8     yassl:yassl_imp.obj
 0002:00019cc0       ??_R2Certificate@yaSSL@@8  0000000140102cc0     yassl:yassl_imp.obj
 0002:00019ce0       ??_R1A@?0A@EA@Certificate@yaSSL@@8 0000000140102ce0     yassl:yassl_imp.obj
 0002:00019d08       ??_R4ServerHello@yaSSL@@6B@ 0000000140102d08     yassl:yassl_imp.obj
 0002:00019d28       ??_R3ServerHello@yaSSL@@8  0000000140102d28     yassl:yassl_imp.obj
 0002:00019d40       ??_R2ServerHello@yaSSL@@8  0000000140102d40     yassl:yassl_imp.obj
 0002:00019d60       ??_R1A@?0A@EA@ServerHello@yaSSL@@8 0000000140102d60     yassl:yassl_imp.obj
 0002:00019d88       ??_R4ServerHelloDone@yaSSL@@6B@ 0000000140102d88     yassl:yassl_imp.obj
 0002:00019da8       ??_R3ServerHelloDone@yaSSL@@8 0000000140102da8     yassl:yassl_imp.obj
 0002:00019dc0       ??_R2ServerHelloDone@yaSSL@@8 0000000140102dc0     yassl:yassl_imp.obj
 0002:00019de0       ??_R1A@?0A@EA@ServerHelloDone@yaSSL@@8 0000000140102de0     yassl:yassl_imp.obj
 0002:00019e08       ??_R4ClientHello@yaSSL@@6B@ 0000000140102e08     yassl:yassl_imp.obj
 0002:00019e28       ??_R3ClientHello@yaSSL@@8  0000000140102e28     yassl:yassl_imp.obj
 0002:00019e40       ??_R2ClientHello@yaSSL@@8  0000000140102e40     yassl:yassl_imp.obj
 0002:00019e60       ??_R1A@?0A@EA@ClientHello@yaSSL@@8 0000000140102e60     yassl:yassl_imp.obj
 0002:00019e88       ??_R4ServerKeyExchange@yaSSL@@6B@ 0000000140102e88     yassl:yassl_imp.obj
 0002:00019ea8       ??_R3ServerKeyExchange@yaSSL@@8 0000000140102ea8     yassl:yassl_imp.obj
 0002:00019ec0       ??_R2ServerKeyExchange@yaSSL@@8 0000000140102ec0     yassl:yassl_imp.obj
 0002:00019ee0       ??_R1A@?0A@EA@ServerKeyExchange@yaSSL@@8 0000000140102ee0     yassl:yassl_imp.obj
 0002:00019f08       ??_R4CertificateVerify@yaSSL@@6B@ 0000000140102f08     yassl:yassl_imp.obj
 0002:00019f28       ??_R3CertificateVerify@yaSSL@@8 0000000140102f28     yassl:yassl_imp.obj
 0002:00019f40       ??_R2CertificateVerify@yaSSL@@8 0000000140102f40     yassl:yassl_imp.obj
 0002:00019f60       ??_R1A@?0A@EA@CertificateVerify@yaSSL@@8 0000000140102f60     yassl:yassl_imp.obj
 0002:00019f88       ??_R4ClientKeyExchange@yaSSL@@6B@ 0000000140102f88     yassl:yassl_imp.obj
 0002:00019fa8       ??_R3ClientKeyExchange@yaSSL@@8 0000000140102fa8     yassl:yassl_imp.obj
 0002:00019fc0       ??_R2ClientKeyExchange@yaSSL@@8 0000000140102fc0     yassl:yassl_imp.obj
 0002:00019fe0       ??_R1A@?0A@EA@ClientKeyExchange@yaSSL@@8 0000000140102fe0     yassl:yassl_imp.obj
 0002:0001a008       ??_R4Finished@yaSSL@@6B@   0000000140103008     yassl:yassl_imp.obj
 0002:0001a028       ??_R3Finished@yaSSL@@8     0000000140103028     yassl:yassl_imp.obj
 0002:0001a040       ??_R2Finished@yaSSL@@8     0000000140103040     yassl:yassl_imp.obj
 0002:0001a060       ??_R1A@?0A@EA@Finished@yaSSL@@8 0000000140103060     yassl:yassl_imp.obj
 0002:0001a088       ??_R4HelloRequest@yaSSL@@6B@ 0000000140103088     yassl:yassl_imp.obj
 0002:0001a0a8       ??_R3HelloRequest@yaSSL@@8 00000001401030a8     yassl:yassl_imp.obj
 0002:0001a0c0       ??_R2HelloRequest@yaSSL@@8 00000001401030c0     yassl:yassl_imp.obj
 0002:0001a0e0       ??_R1A@?0A@EA@HelloRequest@yaSSL@@8 00000001401030e0     yassl:yassl_imp.obj
 0002:0001a108       ??_R4RSA_Server@yaSSL@@6B@ 0000000140103108     yassl:yassl_imp.obj
 0002:0001a128       ??_R3RSA_Server@yaSSL@@8   0000000140103128     yassl:yassl_imp.obj
 0002:0001a140       ??_R2RSA_Server@yaSSL@@8   0000000140103140     yassl:yassl_imp.obj
 0002:0001a160       ??_R1A@?0A@EA@RSA_Server@yaSSL@@8 0000000140103160     yassl:yassl_imp.obj
 0002:0001a188       ??_R4Fortezza_Server@yaSSL@@6B@ 0000000140103188     yassl:yassl_imp.obj
 0002:0001a1a8       ??_R3Fortezza_Server@yaSSL@@8 00000001401031a8     yassl:yassl_imp.obj
 0002:0001a1c0       ??_R2Fortezza_Server@yaSSL@@8 00000001401031c0     yassl:yassl_imp.obj
 0002:0001a1e0       ??_R1A@?0A@EA@Fortezza_Server@yaSSL@@8 00000001401031e0     yassl:yassl_imp.obj
 0002:0001a208       ??_R4FortezzaKeys@yaSSL@@6B@ 0000000140103208     yassl:yassl_imp.obj
 0002:0001a228       ??_R3FortezzaKeys@yaSSL@@8 0000000140103228     yassl:yassl_imp.obj
 0002:0001a240       ??_R2FortezzaKeys@yaSSL@@8 0000000140103240     yassl:yassl_imp.obj
 0002:0001a260       ??_R1A@?0A@EA@FortezzaKeys@yaSSL@@8 0000000140103260     yassl:yassl_imp.obj
 0002:0001a288       ??_R4EncryptedPreMasterSecret@yaSSL@@6B@ 0000000140103288     yassl:yassl_imp.obj
 0002:0001a2a8       ??_R3EncryptedPreMasterSecret@yaSSL@@8 00000001401032a8     yassl:yassl_imp.obj
 0002:0001a2c0       ??_R2EncryptedPreMasterSecret@yaSSL@@8 00000001401032c0     yassl:yassl_imp.obj
 0002:0001a2e0       ??_R1A@?0A@EA@EncryptedPreMasterSecret@yaSSL@@8 00000001401032e0     yassl:yassl_imp.obj
 0002:0001a308       ??_R4DH_Server@yaSSL@@6B@  0000000140103308     yassl:yassl_imp.obj
 0002:0001a328       ??_R3DH_Server@yaSSL@@8    0000000140103328     yassl:yassl_imp.obj
 0002:0001a340       ??_R2DH_Server@yaSSL@@8    0000000140103340     yassl:yassl_imp.obj
 0002:0001a360       ??_R1A@?0A@EA@DH_Server@yaSSL@@8 0000000140103360     yassl:yassl_imp.obj
 0002:0001a388       ??_R4CertificateRequest@yaSSL@@6B@ 0000000140103388     yassl:yassl_imp.obj
 0002:0001a3a8       ??_R3CertificateRequest@yaSSL@@8 00000001401033a8     yassl:yassl_imp.obj
 0002:0001a3c0       ??_R2CertificateRequest@yaSSL@@8 00000001401033c0     yassl:yassl_imp.obj
 0002:0001a3e0       ??_R1A@?0A@EA@CertificateRequest@yaSSL@@8 00000001401033e0     yassl:yassl_imp.obj
 0002:0001a408       ??_R4type_info@@6B@        0000000140103408     LIBCMT:typinfo.obj
 0002:0001a430       ??_R3type_info@@8          0000000140103430     LIBCMT:typinfo.obj
 0002:0001a448       ??_R2type_info@@8          0000000140103448     LIBCMT:typinfo.obj
 0002:0001a458       ??_R1A@?0A@EA@type_info@@8 0000000140103458     LIBCMT:typinfo.obj
 0002:0001a480       ??_R4bad_alloc@std@@6B@    0000000140103480     LIBCMT:new.obj
 0002:0001a4a8       ??_R3bad_alloc@std@@8      00000001401034a8     LIBCMT:new.obj
 0002:0001a4c0       ??_R2bad_alloc@std@@8      00000001401034c0     LIBCMT:new.obj
 0002:0001a4d8       ??_R1A@?0A@EA@bad_alloc@std@@8 00000001401034d8     LIBCMT:new.obj
 0002:0001a500       ??_R1A@?0A@EA@exception@std@@8 0000000140103500     LIBCMT:new.obj
 0002:0001a528       ??_R3exception@std@@8      0000000140103528     LIBCMT:new.obj
 0002:0001a540       ??_R2exception@std@@8      0000000140103540     LIBCMT:new.obj
 0002:0001a550       ??_R4exception@std@@6B@    0000000140103550     LIBCMT:stdexcpt.obj
 0002:0001a578       ??_R4bad_cast@std@@6B@     0000000140103578     LIBCMT:stdexcpt.obj
 0002:0001a5a0       ??_R3bad_cast@std@@8       00000001401035a0     LIBCMT:stdexcpt.obj
 0002:0001a5b8       ??_R2bad_cast@std@@8       00000001401035b8     LIBCMT:stdexcpt.obj
 0002:0001a5d0       ??_R1A@?0A@EA@bad_cast@std@@8 00000001401035d0     LIBCMT:stdexcpt.obj
 0002:0001a5f8       ??_R4bad_typeid@std@@6B@   00000001401035f8     LIBCMT:stdexcpt.obj
 0002:0001a620       ??_R3bad_typeid@std@@8     0000000140103620     LIBCMT:stdexcpt.obj
 0002:0001a638       ??_R2bad_typeid@std@@8     0000000140103638     LIBCMT:stdexcpt.obj
 0002:0001a650       ??_R1A@?0A@EA@bad_typeid@std@@8 0000000140103650     LIBCMT:stdexcpt.obj
 0002:0001a678       ??_R4__non_rtti_object@std@@6B@ 0000000140103678     LIBCMT:stdexcpt.obj
 0002:0001a6a0       ??_R3__non_rtti_object@std@@8 00000001401036a0     LIBCMT:stdexcpt.obj
 0002:0001a6b8       ??_R2__non_rtti_object@std@@8 00000001401036b8     LIBCMT:stdexcpt.obj
 0002:0001a6d8       ??_R1A@?0A@EA@__non_rtti_object@std@@8 00000001401036d8     LIBCMT:stdexcpt.obj
 0002:0001a700       ??_R4DNameNode@@6B@        0000000140103700     LIBCMT:undname.obj
 0002:0001a728       ??_R3DNameNode@@8          0000000140103728     LIBCMT:undname.obj
 0002:0001a740       ??_R2DNameNode@@8          0000000140103740     LIBCMT:undname.obj
 0002:0001a750       ??_R1A@?0A@EA@DNameNode@@8 0000000140103750     LIBCMT:undname.obj
 0002:0001a778       ??_R4charNode@@6B@         0000000140103778     LIBCMT:undname.obj
 0002:0001a7a0       ??_R3charNode@@8           00000001401037a0     LIBCMT:undname.obj
 0002:0001a7b8       ??_R2charNode@@8           00000001401037b8     LIBCMT:undname.obj
 0002:0001a7d0       ??_R1A@?0A@EA@charNode@@8  00000001401037d0     LIBCMT:undname.obj
 0002:0001a7f8       ??_R4pDNameNode@@6B@       00000001401037f8     LIBCMT:undname.obj
 0002:0001a820       ??_R3pDNameNode@@8         0000000140103820     LIBCMT:undname.obj
 0002:0001a838       ??_R2pDNameNode@@8         0000000140103838     LIBCMT:undname.obj
 0002:0001a850       ??_R1A@?0A@EA@pDNameNode@@8 0000000140103850     LIBCMT:undname.obj
 0002:0001a878       ??_R4DNameStatusNode@@6B@  0000000140103878     LIBCMT:undname.obj
 0002:0001a8a0       ??_R3DNameStatusNode@@8    00000001401038a0     LIBCMT:undname.obj
 0002:0001a8b8       ??_R2DNameStatusNode@@8    00000001401038b8     LIBCMT:undname.obj
 0002:0001a8d0       ??_R1A@?0A@EA@DNameStatusNode@@8 00000001401038d0     LIBCMT:undname.obj
 0002:0001a8f8       ??_R4pcharNode@@6B@        00000001401038f8     LIBCMT:undname.obj
 0002:0001a920       ??_R3pcharNode@@8          0000000140103920     LIBCMT:undname.obj
 0002:0001a938       ??_R2pcharNode@@8          0000000140103938     LIBCMT:undname.obj
 0002:0001a950       ??_R1A@?0A@EA@pcharNode@@8 0000000140103950     LIBCMT:undname.obj
 0002:0001a978       ??_R4HASH64withTransform@TaoCrypt@@6B@ 0000000140103978     taocrypt:hash.obj
 0002:0001a998       ??_R3HASH64withTransform@TaoCrypt@@8 0000000140103998     taocrypt:hash.obj
 0002:0001a9b0       ??_R2HASH64withTransform@TaoCrypt@@8 00000001401039b0     taocrypt:hash.obj
 0002:0001a9d0       ??_R1A@?0A@EA@HASH64withTransform@TaoCrypt@@8 00000001401039d0     taocrypt:hash.obj
 0002:0001a9f8       ??_R4HASHwithTransform@TaoCrypt@@6B@ 00000001401039f8     taocrypt:hash.obj
 0002:0001aa18       ??_R4MultiplicativeGroupT@AbstractRing@TaoCrypt@@6B@ 0000000140103a18     taocrypt:integer.obj
 0002:0001aa38       ??_R3MultiplicativeGroupT@AbstractRing@TaoCrypt@@8 0000000140103a38     taocrypt:integer.obj
 0002:0001aa50       ??_R2MultiplicativeGroupT@AbstractRing@TaoCrypt@@8 0000000140103a50     taocrypt:integer.obj
 0002:0001aa70       ??_R1A@?0A@EA@MultiplicativeGroupT@AbstractRing@TaoCrypt@@8 0000000140103a70     taocrypt:integer.obj
 0002:0001aa98       ??_R1A@?0A@EA@AbstractGroup@TaoCrypt@@8 0000000140103a98     taocrypt:integer.obj
 0002:0001aac0       ??_R3AbstractGroup@TaoCrypt@@8 0000000140103ac0     taocrypt:integer.obj
 0002:0001aad8       ??_R2AbstractGroup@TaoCrypt@@8 0000000140103ad8     taocrypt:integer.obj
 0002:0001aaf0       ??_R4ModularArithmetic@TaoCrypt@@6B@ 0000000140103af0     taocrypt:integer.obj
 0002:0001ab10       ??_R3ModularArithmetic@TaoCrypt@@8 0000000140103b10     taocrypt:integer.obj
 0002:0001ab28       ??_R2ModularArithmetic@TaoCrypt@@8 0000000140103b28     taocrypt:integer.obj
 0002:0001ab50       ??_R1A@?0A@EA@ModularArithmetic@TaoCrypt@@8 0000000140103b50     taocrypt:integer.obj
 0002:0001ab78       ??_R1A@?0A@EA@AbstractRing@TaoCrypt@@8 0000000140103b78     taocrypt:integer.obj
 0002:0001aba0       ??_R3AbstractRing@TaoCrypt@@8 0000000140103ba0     taocrypt:integer.obj
 0002:0001abb8       ??_R2AbstractRing@TaoCrypt@@8 0000000140103bb8     taocrypt:integer.obj
 0002:0001abd8       ??_R4MontgomeryRepresentation@TaoCrypt@@6B@ 0000000140103bd8     taocrypt:integer.obj
 0002:0001abf8       ??_R3MontgomeryRepresentation@TaoCrypt@@8 0000000140103bf8     taocrypt:integer.obj
 0002:0001ac10       ??_R2MontgomeryRepresentation@TaoCrypt@@8 0000000140103c10     taocrypt:integer.obj
 0002:0001ac40       ??_R1A@?0A@EA@MontgomeryRepresentation@TaoCrypt@@8 0000000140103c40     taocrypt:integer.obj
 0002:0001ac68       ??_R4EuclideanDomainOf@TaoCrypt@@6B@ 0000000140103c68     taocrypt:integer.obj
 0002:0001ac88       ??_R3EuclideanDomainOf@TaoCrypt@@8 0000000140103c88     taocrypt:integer.obj
 0002:0001aca0       ??_R2EuclideanDomainOf@TaoCrypt@@8 0000000140103ca0     taocrypt:integer.obj
 0002:0001acd0       ??_R1A@?0A@EA@EuclideanDomainOf@TaoCrypt@@8 0000000140103cd0     taocrypt:integer.obj
 0002:0001acf8       ??_R1A@?0A@EA@AbstractEuclideanDomain@TaoCrypt@@8 0000000140103cf8     taocrypt:integer.obj
 0002:0001ad20       ??_R3AbstractEuclideanDomain@TaoCrypt@@8 0000000140103d20     taocrypt:integer.obj
 0002:0001ad38       ??_R2AbstractEuclideanDomain@TaoCrypt@@8 0000000140103d38     taocrypt:integer.obj
 0002:0001ad60       ??_R4SHA256@TaoCrypt@@6B@  0000000140103d60     taocrypt:sha.obj
 0002:0001ad80       ??_R3SHA256@TaoCrypt@@8    0000000140103d80     taocrypt:sha.obj
 0002:0001ad98       ??_R2SHA256@TaoCrypt@@8    0000000140103d98     taocrypt:sha.obj
 0002:0001adc0       ??_R1A@?0A@EA@SHA256@TaoCrypt@@8 0000000140103dc0     taocrypt:sha.obj
 0002:0001ade8       ??_R4SHA224@TaoCrypt@@6B@  0000000140103de8     taocrypt:sha.obj
 0002:0001ae08       ??_R3SHA224@TaoCrypt@@8    0000000140103e08     taocrypt:sha.obj
 0002:0001ae20       ??_R2SHA224@TaoCrypt@@8    0000000140103e20     taocrypt:sha.obj
 0002:0001ae48       ??_R1A@?0A@EA@SHA224@TaoCrypt@@8 0000000140103e48     taocrypt:sha.obj
 0002:0001ae70       ??_R4SHA512@TaoCrypt@@6B@  0000000140103e70     taocrypt:sha.obj
 0002:0001ae90       ??_R3SHA512@TaoCrypt@@8    0000000140103e90     taocrypt:sha.obj
 0002:0001aea8       ??_R2SHA512@TaoCrypt@@8    0000000140103ea8     taocrypt:sha.obj
 0002:0001aed0       ??_R1A@?0A@EA@SHA512@TaoCrypt@@8 0000000140103ed0     taocrypt:sha.obj
 0002:0001aef8       ??_R4SHA384@TaoCrypt@@6B@  0000000140103ef8     taocrypt:sha.obj
 0002:0001af18       ??_R3SHA384@TaoCrypt@@8    0000000140103f18     taocrypt:sha.obj
 0002:0001af30       ??_R2SHA384@TaoCrypt@@8    0000000140103f30     taocrypt:sha.obj
 0002:0001af58       ??_R1A@?0A@EA@SHA384@TaoCrypt@@8 0000000140103f58     taocrypt:sha.obj
 0002:0001af80       ??_R4BER_Decoder@TaoCrypt@@6B@ 0000000140103f80     taocrypt:dsa.obj
 0002:0001afa0       ??_R3BER_Decoder@TaoCrypt@@8 0000000140103fa0     taocrypt:dsa.obj
 0002:0001afb8       ??_R2BER_Decoder@TaoCrypt@@8 0000000140103fb8     taocrypt:dsa.obj
 0002:0001afd0       ??_R1A@?0A@EA@BER_Decoder@TaoCrypt@@8 0000000140103fd0     taocrypt:dsa.obj
 0002:0001aff8       ??_R4DSA_Private_Decoder@TaoCrypt@@6B@ 0000000140103ff8     taocrypt:dsa.obj
 0002:0001b018       ??_R3DSA_Private_Decoder@TaoCrypt@@8 0000000140104018     taocrypt:dsa.obj
 0002:0001b030       ??_R2DSA_Private_Decoder@TaoCrypt@@8 0000000140104030     taocrypt:dsa.obj
 0002:0001b050       ??_R1A@?0A@EA@DSA_Private_Decoder@TaoCrypt@@8 0000000140104050     taocrypt:dsa.obj
 0002:0001b078       ??_R4DSA_Public_Decoder@TaoCrypt@@6B@ 0000000140104078     taocrypt:dsa.obj
 0002:0001b098       ??_R3DSA_Public_Decoder@TaoCrypt@@8 0000000140104098     taocrypt:dsa.obj
 0002:0001b0b0       ??_R2DSA_Public_Decoder@TaoCrypt@@8 00000001401040b0     taocrypt:dsa.obj
 0002:0001b0d0       ??_R1A@?0A@EA@DSA_Public_Decoder@TaoCrypt@@8 00000001401040d0     taocrypt:dsa.obj
 0002:0001b0f8       ??_R4DH_Decoder@TaoCrypt@@6B@ 00000001401040f8     taocrypt:dh.obj
 0002:0001b118       ??_R3DH_Decoder@TaoCrypt@@8 0000000140104118     taocrypt:dh.obj
 0002:0001b130       ??_R2DH_Decoder@TaoCrypt@@8 0000000140104130     taocrypt:dh.obj
 0002:0001b150       ??_R1A@?0A@EA@DH_Decoder@TaoCrypt@@8 0000000140104150     taocrypt:dh.obj
 0002:0001b178       ??_R4RSA_Private_Decoder@TaoCrypt@@6B@ 0000000140104178     taocrypt:rsa.obj
 0002:0001b198       ??_R3RSA_Private_Decoder@TaoCrypt@@8 0000000140104198     taocrypt:rsa.obj
 0002:0001b1b0       ??_R2RSA_Private_Decoder@TaoCrypt@@8 00000001401041b0     taocrypt:rsa.obj
 0002:0001b1d0       ??_R1A@?0A@EA@RSA_Private_Decoder@TaoCrypt@@8 00000001401041d0     taocrypt:rsa.obj
 0002:0001b1f8       ??_R4RSA_Public_Decoder@TaoCrypt@@6B@ 00000001401041f8     taocrypt:rsa.obj
 0002:0001b218       ??_R3RSA_Public_Decoder@TaoCrypt@@8 0000000140104218     taocrypt:rsa.obj
 0002:0001b230       ??_R2RSA_Public_Decoder@TaoCrypt@@8 0000000140104230     taocrypt:rsa.obj
 0002:0001b250       ??_R1A@?0A@EA@RSA_Public_Decoder@TaoCrypt@@8 0000000140104250     taocrypt:rsa.obj
 0002:0001b278       ??_R4DER_Encoder@TaoCrypt@@6B@ 0000000140104278     taocrypt:asn.obj
 0002:0001b298       ??_R3DER_Encoder@TaoCrypt@@8 0000000140104298     taocrypt:asn.obj
 0002:0001b2b0       ??_R2DER_Encoder@TaoCrypt@@8 00000001401042b0     taocrypt:asn.obj
 0002:0001b2c8       ??_R1A@?0A@EA@DER_Encoder@TaoCrypt@@8 00000001401042c8     taocrypt:asn.obj
 0002:0001b2f0       ??_R4CertDecoder@TaoCrypt@@6B@ 00000001401042f0     taocrypt:asn.obj
 0002:0001b310       ??_R3CertDecoder@TaoCrypt@@8 0000000140104310     taocrypt:asn.obj
 0002:0001b328       ??_R2CertDecoder@TaoCrypt@@8 0000000140104328     taocrypt:asn.obj
 0002:0001b348       ??_R1A@?0A@EA@CertDecoder@TaoCrypt@@8 0000000140104348     taocrypt:asn.obj
 0002:0001b370       ??_R4Signature_Encoder@TaoCrypt@@6B@ 0000000140104370     taocrypt:asn.obj
 0002:0001b390       ??_R3Signature_Encoder@TaoCrypt@@8 0000000140104390     taocrypt:asn.obj
 0002:0001b3a8       ??_R2Signature_Encoder@TaoCrypt@@8 00000001401043a8     taocrypt:asn.obj
 0002:0001b3c8       ??_R1A@?0A@EA@Signature_Encoder@TaoCrypt@@8 00000001401043c8     taocrypt:asn.obj
 0002:0001b3f0       ??_R4MD2@TaoCrypt@@6B@     00000001401043f0     taocrypt:md2.obj
 0002:0001b410       ??_R3MD2@TaoCrypt@@8       0000000140104410     taocrypt:md2.obj
 0002:0001b428       ??_R2MD2@TaoCrypt@@8       0000000140104428     taocrypt:md2.obj
 0002:0001b448       ??_R1A@?0A@EA@MD2@TaoCrypt@@8 0000000140104448     taocrypt:md2.obj
 0002:0001be08       __rtc_iaa                  0000000140104e08     LIBCMT:initsect.obj
 0002:0001bf18       __rtc_izz                  0000000140104f18     LIBCMT:initsect.obj
 0002:0001c028       __rtc_taa                  0000000140105028     LIBCMT:initsect.obj
 0002:0001c138       __rtc_tzz                  0000000140105138     LIBCMT:initsect.obj
 0002:0002cdf8       _TI2?AVbad_alloc@std@@     0000000140115df8     LIBCMT:new.obj
 0002:0002ce18       _CTA2?AVbad_alloc@std@@    0000000140115e18     LIBCMT:new.obj
 0002:0002ce30       _CT??_R0?AVbad_alloc@std@@@8??0bad_alloc@std@@QEAA@AEBV01@@Z24 0000000140115e30     LIBCMT:new.obj
 0002:0002ce58       _CT??_R0?AVexception@std@@@8??0exception@std@@QEAA@AEBV01@@Z24 0000000140115e58     LIBCMT:new.obj
 0003:00000000       ??_R0?AVCommand@@@8        0000000140116000     command.obj
 0003:00000028       ??_R0?AVShow_instance_status@@@8 0000000140116028     commands.obj
 0003:00000060       ??_R0?AVShow_instance_options@@@8 0000000140116060     commands.obj
 0003:00000098       ??_R0?AVStart_instance@@@8 0000000140116098     commands.obj
 0003:000000c8       ??_R0?AVShow_instance_log@@@8 00000001401160c8     commands.obj
 0003:000000f8       ??_R0?AVShow_instance_log_files@@@8 00000001401160f8     commands.obj
 0003:00000130       ??_R0?AVSet_option@@@8     0000000140116130     commands.obj
 0003:00000158       ??_R0?AVStop_instance@@@8  0000000140116158     commands.obj
 0003:000001c0       ?config_file@Options@@2PEBDEB 00000001401161c0     options.obj
 0003:000001c8       ?log_file_name@Options@@2PEBDEB 00000001401161c8     options.obj
 0003:000001d0       ?pid_file_name@Options@@2PEBDEB 00000001401161d0     options.obj
 0003:000001d8       ?password_file_name@Options@@2PEBDEB 00000001401161d8     options.obj
 0003:000001e0       ?default_mysqld_path@Options@@2PEBDEB 00000001401161e0     options.obj
 0003:000001e8       ?monitoring_interval@Options@@2IA 00000001401161e8     options.obj
 0003:000001ec       ?port_number@Options@@2IA  00000001401161ec     options.obj
 0003:00000a00       ??_R0?AVShow_instances@@@8 0000000140116a00     parse.obj
 0003:00000a30       ??_R0?AVFlush_instances@@@8 0000000140116a30     parse.obj
 0003:00000a60       ??_R0?AVSyntax_error@@@8   0000000140116a60     parse.obj
 0003:00000a90       ??_R0?AVUnset_option@@@8   0000000140116a90     parse.obj
 0003:00000abc       ?net_buffer_length@@3KA    0000000140116abc     priv.obj
 0003:00000ac0       ?max_allowed_packet@@3KA   0000000140116ac0     priv.obj
 0003:00000ac4       ?net_read_timeout@@3KA     0000000140116ac4     priv.obj
 0003:00000ac8       ?net_write_timeout@@3KA    0000000140116ac8     priv.obj
 0003:00000acc       ?net_retry_count@@3KA      0000000140116acc     priv.obj
 0003:00000ad0       ?mysqld_net_retry_count@@3KA 0000000140116ad0     priv.obj
 0003:00000ae0       ??_R0?AVIMService@@@8      0000000140116ae0     IMService.obj
 0003:00000b08       ??_R0?AVWindowsService@@@8 0000000140116b08     IMService.obj
 0003:00000b40       sqlstate_map               0000000140116b40     sql_state.obj
 0003:000021e0       unknown_sqlstate           00000001401181e0     client.obj
 0003:000021e8       not_error_sqlstate         00000001401181e8     client.obj
 0003:000021f0       cant_connect_sqlstate      00000001401181f0     client.obj
 0003:000021f8       default_client_charset_info 00000001401181f8     client.obj
 0003:00002338       sql_protocol_names_lib     0000000140118338     client.obj
 0003:00002360       sql_protocol_typelib       0000000140118360     client.obj
 0003:00002410       client_errors              0000000140118410     errmsg.obj
 0003:00002634       my_thread_end_wait_time    0000000140118634     mysys:my_thr_init.obj
 0003:00002638       my_pthread_create_detached 0000000140118638     mysys:my_pthread.obj
 0003:00002640       default_charset_info       0000000140118640     mysys:charset.obj
 0003:00002660       my_umask                   0000000140118660     mysys:my_static.obj
 0003:00002664       my_umask_dir               0000000140118664     mysys:my_static.obj
 0003:00002668       my_file_limit              0000000140118668     mysys:my_static.obj
 0003:0000266c       my_default_record_cache_size 000000014011866c     mysys:my_static.obj
 0003:00002670       my_file_info               0000000140118670     mysys:my_static.obj
 0003:00002678       soundex_map                0000000140118678     mysys:my_static.obj
 0003:00002680       my_once_extra              0000000140118680     mysys:my_static.obj
 0003:00002684       my_time_to_wait_for_lock   0000000140118684     mysys:my_static.obj
 0003:00002688       sf_min_adress              0000000140118688     mysys:my_static.obj
 0003:00002690       raid_type_string           0000000140118690     mysys:my_static.obj
 0003:000026a0       my_abort_hook              00000001401186a0     mysys:my_static.obj
 0003:000026a8       error_handler_hook         00000001401186a8     mysys:my_static.obj
 0003:000026b0       fatal_error_handler_hook   00000001401186b0     mysys:my_static.obj
 0003:000026b8       my_getopt_error_reporter   00000001401186b8     mysys:my_getopt.obj
 0003:000026f0       disabled_my_option         00000001401186f0     mysys:my_getopt.obj
 0003:000026f8       my_getopt_print_errors     00000001401186f8     mysys:my_getopt.obj
 0003:000027f0       globerrs                   00000001401187f0     mysys:errors.obj
 0003:000028d8       _dig_vec_upper             00000001401188d8     strings:int2str.obj
 0003:00002900       _dig_vec_lower             0000000140118900     strings:int2str.obj
 0003:00002d40       cs_to_uni                  0000000140118d40     strings:ctype-latin1.obj
 0003:00002f40       pl00                       0000000140118f40     strings:ctype-latin1.obj
 0003:00003040       pl01                       0000000140119040     strings:ctype-latin1.obj
 0003:00003140       pl02                       0000000140119140     strings:ctype-latin1.obj
 0003:00003240       pl20                       0000000140119240     strings:ctype-latin1.obj
 0003:00003340       pl21                       0000000140119340     strings:ctype-latin1.obj
 0003:00003440       uni_to_cs                  0000000140119440     strings:ctype-latin1.obj
 0003:00003d10       my_charset_latin1          0000000140119d10     strings:ctype-latin1.obj
 0003:00003ec0       combo1map                  0000000140119ec0     strings:ctype-latin1.obj
 0003:00003fc0       combo2map                  0000000140119fc0     strings:ctype-latin1.obj
 0003:00004130       my_charset_latin1_german2_ci 000000014011a130     strings:ctype-latin1.obj
 0003:000041e0       my_charset_latin1_bin      000000014011a1e0     strings:ctype-latin1.obj
 0003:00004330       my_charset_8bit_handler    000000014011a330     strings:ctype-simple.obj
 0003:00004400       my_collation_8bit_simple_ci_handler 000000014011a400     strings:ctype-simple.obj
 0003:00004670       my_collation_8bit_bin_handler 000000014011a670     strings:ctype-bin.obj
 0003:00004800       my_charset_bin             000000014011a800     strings:ctype-bin.obj
 0003:00004aa0       page000data                000000014011aaa0     strings:ctype-uca.obj
 0003:000052a0       page001data                000000014011b2a0     strings:ctype-uca.obj
 0003:000058a0       page002data                000000014011b8a0     strings:ctype-uca.obj
 0003:00005ea0       page003data                000000014011bea0     strings:ctype-uca.obj
 0003:000066a0       page004data                000000014011c6a0     strings:ctype-uca.obj
 0003:00006ca0       page005data                000000014011cca0     strings:ctype-uca.obj
 0003:000072a0       page006data                000000014011d2a0     strings:ctype-uca.obj
 0003:000078a0       page007data                000000014011d8a0     strings:ctype-uca.obj
 0003:00007ea0       page009data                000000014011dea0     strings:ctype-uca.obj
 0003:000084a0       page00Adata                000000014011e4a0     strings:ctype-uca.obj
 0003:00008aa0       page00Bdata                000000014011eaa0     strings:ctype-uca.obj
 0003:000090a0       page00Cdata                000000014011f0a0     strings:ctype-uca.obj
 0003:000096a0       page00Ddata                000000014011f6a0     strings:ctype-uca.obj
 0003:00009ca0       page00Edata                000000014011fca0     strings:ctype-uca.obj
 0003:0000a2a0       page00Fdata                00000001401202a0     strings:ctype-uca.obj
 0003:0000a8a0       page010data                00000001401208a0     strings:ctype-uca.obj
 0003:0000aea0       page011data                0000000140120ea0     strings:ctype-uca.obj
 0003:0000b4a0       page012data                00000001401214a0     strings:ctype-uca.obj
 0003:0000baa0       page013data                0000000140121aa0     strings:ctype-uca.obj
 0003:0000c0a0       page014data                00000001401220a0     strings:ctype-uca.obj
 0003:0000c6a0       page015data                00000001401226a0     strings:ctype-uca.obj
 0003:0000caa0       page016data                0000000140122aa0     strings:ctype-uca.obj
 0003:0000d0a0       page017data                00000001401230a0     strings:ctype-uca.obj
 0003:0000d6a0       page018data                00000001401236a0     strings:ctype-uca.obj
 0003:0000dca0       page019data                0000000140123ca0     strings:ctype-uca.obj
 0003:0000e2a0       page01Ddata                00000001401242a0     strings:ctype-uca.obj
 0003:0000e8a0       page01Edata                00000001401248a0     strings:ctype-uca.obj
 0003:0000eea0       page01Fdata                0000000140124ea0     strings:ctype-uca.obj
 0003:0000f4a0       page020data                00000001401254a0     strings:ctype-uca.obj
 0003:0000fea0       page021data                0000000140125ea0     strings:ctype-uca.obj
 0003:000108a0       page022data                00000001401268a0     strings:ctype-uca.obj
 0003:000110a0       page023data                00000001401270a0     strings:ctype-uca.obj
 0003:000116a0       page024data                00000001401276a0     strings:ctype-uca.obj
 0003:000120a0       page025data                00000001401280a0     strings:ctype-uca.obj
 0003:000124a0       page026data                00000001401284a0     strings:ctype-uca.obj
 0003:00012aa0       page027data                0000000140128aa0     strings:ctype-uca.obj
 0003:000130a0       page028data                00000001401290a0     strings:ctype-uca.obj
 0003:000134a0       page029data                00000001401294a0     strings:ctype-uca.obj
 0003:000138a0       page02Adata                00000001401298a0     strings:ctype-uca.obj
 0003:000142a0       page02Bdata                000000014012a2a0     strings:ctype-uca.obj
 0003:000148a0       page02Edata                000000014012a8a0     strings:ctype-uca.obj
 0003:00014ea0       page02Fdata                000000014012aea0     strings:ctype-uca.obj
 0003:000154a0       page030data                000000014012b4a0     strings:ctype-uca.obj
 0003:00015aa0       page031data                000000014012baa0     strings:ctype-uca.obj
 0003:000160a0       page032data                000000014012c0a0     strings:ctype-uca.obj
 0003:000170a0       page033data                000000014012d0a0     strings:ctype-uca.obj
 0003:000182a0       page04Ddata                000000014012e2a0     strings:ctype-uca.obj
 0003:000188a0       page0A0data                000000014012e8a0     strings:ctype-uca.obj
 0003:00018ca0       page0A1data                000000014012eca0     strings:ctype-uca.obj
 0003:000190a0       page0A2data                000000014012f0a0     strings:ctype-uca.obj
 0003:000194a0       page0A3data                000000014012f4a0     strings:ctype-uca.obj
 0003:000198a0       page0A4data                000000014012f8a0     strings:ctype-uca.obj
 0003:00019ea0       page0F9data                000000014012fea0     strings:ctype-uca.obj
 0003:0001a4a0       page0FAdata                00000001401304a0     strings:ctype-uca.obj
 0003:0001aaa0       page0FBdata                0000000140130aa0     strings:ctype-uca.obj
 0003:0001b2a0       page0FCdata                00000001401312a0     strings:ctype-uca.obj
 0003:0001b8a0       page0FDdata                00000001401318a0     strings:ctype-uca.obj
 0003:0001caa0       page0FEdata                0000000140132aa0     strings:ctype-uca.obj
 0003:0001d0a0       page0FFdata                00000001401330a0     strings:ctype-uca.obj
 0003:0001d6a0       uca_length                 00000001401336a0     strings:ctype-uca.obj
 0003:0001d7a0       uca_weight                 00000001401337a0     strings:ctype-uca.obj
 0003:0001dfc0       my_collation_ucs2_uca_handler 0000000140133fc0     strings:ctype-uca.obj
 0003:0001e020       my_charset_ucs2_unicode_ci 0000000140134020     strings:ctype-uca.obj
 0003:0001e0d0       my_charset_ucs2_icelandic_uca_ci 00000001401340d0     strings:ctype-uca.obj
 0003:0001e180       my_charset_ucs2_latvian_uca_ci 0000000140134180     strings:ctype-uca.obj
 0003:0001e230       my_charset_ucs2_romanian_uca_ci 0000000140134230     strings:ctype-uca.obj
 0003:0001e2e0       my_charset_ucs2_slovenian_uca_ci 00000001401342e0     strings:ctype-uca.obj
 0003:0001e390       my_charset_ucs2_polish_uca_ci 0000000140134390     strings:ctype-uca.obj
 0003:0001e440       my_charset_ucs2_estonian_uca_ci 0000000140134440     strings:ctype-uca.obj
 0003:0001e4f0       my_charset_ucs2_spanish_uca_ci 00000001401344f0     strings:ctype-uca.obj
 0003:0001e5a0       my_charset_ucs2_swedish_uca_ci 00000001401345a0     strings:ctype-uca.obj
 0003:0001e650       my_charset_ucs2_turkish_uca_ci 0000000140134650     strings:ctype-uca.obj
 0003:0001e700       my_charset_ucs2_czech_uca_ci 0000000140134700     strings:ctype-uca.obj
 0003:0001e7b0       my_charset_ucs2_danish_uca_ci 00000001401347b0     strings:ctype-uca.obj
 0003:0001e860       my_charset_ucs2_lithuanian_uca_ci 0000000140134860     strings:ctype-uca.obj
 0003:0001e910       my_charset_ucs2_slovak_uca_ci 0000000140134910     strings:ctype-uca.obj
 0003:0001e9c0       my_charset_ucs2_spanish2_uca_ci 00000001401349c0     strings:ctype-uca.obj
 0003:0001ea70       my_charset_ucs2_roman_uca_ci 0000000140134a70     strings:ctype-uca.obj
 0003:0001eb20       my_charset_ucs2_persian_uca_ci 0000000140134b20     strings:ctype-uca.obj
 0003:0001ebd0       my_charset_ucs2_esperanto_uca_ci 0000000140134bd0     strings:ctype-uca.obj
 0003:0001ec80       my_charset_ucs2_hungarian_uca_ci 0000000140134c80     strings:ctype-uca.obj
 0003:0001ed30       my_collation_any_uca_handler 0000000140134d30     strings:ctype-uca.obj
 0003:0001eea0       my_charset_utf8_unicode_ci 0000000140134ea0     strings:ctype-uca.obj
 0003:0001ef50       my_charset_utf8_icelandic_uca_ci 0000000140134f50     strings:ctype-uca.obj
 0003:0001f000       my_charset_utf8_latvian_uca_ci 0000000140135000     strings:ctype-uca.obj
 0003:0001f0b0       my_charset_utf8_romanian_uca_ci 00000001401350b0     strings:ctype-uca.obj
 0003:0001f160       my_charset_utf8_slovenian_uca_ci 0000000140135160     strings:ctype-uca.obj
 0003:0001f210       my_charset_utf8_polish_uca_ci 0000000140135210     strings:ctype-uca.obj
 0003:0001f2c0       my_charset_utf8_estonian_uca_ci 00000001401352c0     strings:ctype-uca.obj
 0003:0001f370       my_charset_utf8_spanish_uca_ci 0000000140135370     strings:ctype-uca.obj
 0003:0001f420       my_charset_utf8_swedish_uca_ci 0000000140135420     strings:ctype-uca.obj
 0003:0001f4d0       my_charset_utf8_turkish_uca_ci 00000001401354d0     strings:ctype-uca.obj
 0003:0001f580       my_charset_utf8_czech_uca_ci 0000000140135580     strings:ctype-uca.obj
 0003:0001f630       my_charset_utf8_danish_uca_ci 0000000140135630     strings:ctype-uca.obj
 0003:0001f6e0       my_charset_utf8_lithuanian_uca_ci 00000001401356e0     strings:ctype-uca.obj
 0003:0001f790       my_charset_utf8_slovak_uca_ci 0000000140135790     strings:ctype-uca.obj
 0003:0001f840       my_charset_utf8_spanish2_uca_ci 0000000140135840     strings:ctype-uca.obj
 0003:0001f8f0       my_charset_utf8_roman_uca_ci 00000001401358f0     strings:ctype-uca.obj
 0003:0001f9a0       my_charset_utf8_persian_uca_ci 00000001401359a0     strings:ctype-uca.obj
 0003:0001fa50       my_charset_utf8_esperanto_uca_ci 0000000140135a50     strings:ctype-uca.obj
 0003:0001fb00       my_charset_utf8_hungarian_uca_ci 0000000140135b00     strings:ctype-uca.obj
 0003:00032fb0       my_charset_cp932_japanese_ci 0000000140148fb0     strings:ctype-cp932.obj
 0003:00033060       my_charset_cp932_bin       0000000140149060     strings:ctype-cp932.obj
 0003:00033110       ctype_latin1_german1_ci    0000000140149110     strings:ctype-extra.obj
 0003:00033220       to_lower_latin1_german1_ci 0000000140149220     strings:ctype-extra.obj
 0003:00033320       to_upper_latin1_german1_ci 0000000140149320     strings:ctype-extra.obj
 0003:00033420       sort_order_latin1_german1_ci 0000000140149420     strings:ctype-extra.obj
 0003:00033520       to_uni_latin1_german1_ci   0000000140149520     strings:ctype-extra.obj
 0003:00033720       ctype_latin2_general_ci    0000000140149720     strings:ctype-extra.obj
 0003:00033830       to_lower_latin2_general_ci 0000000140149830     strings:ctype-extra.obj
 0003:00033930       to_upper_latin2_general_ci 0000000140149930     strings:ctype-extra.obj
 0003:00033a30       sort_order_latin2_general_ci 0000000140149a30     strings:ctype-extra.obj
 0003:00033b30       to_uni_latin2_general_ci   0000000140149b30     strings:ctype-extra.obj
 0003:00033d30       ctype_latin1_danish_ci     0000000140149d30     strings:ctype-extra.obj
 0003:00033e40       to_lower_latin1_danish_ci  0000000140149e40     strings:ctype-extra.obj
 0003:00033f40       to_upper_latin1_danish_ci  0000000140149f40     strings:ctype-extra.obj
 0003:00034040       sort_order_latin1_danish_ci 000000014014a040     strings:ctype-extra.obj
 0003:00034140       to_uni_latin1_danish_ci    000000014014a140     strings:ctype-extra.obj
 0003:00034340       ctype_latin2_hungarian_ci  000000014014a340     strings:ctype-extra.obj
 0003:00034450       to_lower_latin2_hungarian_ci 000000014014a450     strings:ctype-extra.obj
 0003:00034550       to_upper_latin2_hungarian_ci 000000014014a550     strings:ctype-extra.obj
 0003:00034650       sort_order_latin2_hungarian_ci 000000014014a650     strings:ctype-extra.obj
 0003:00034750       to_uni_latin2_hungarian_ci 000000014014a750     strings:ctype-extra.obj
 0003:00034950       ctype_cp1250_general_ci    000000014014a950     strings:ctype-extra.obj
 0003:00034a60       to_lower_cp1250_general_ci 000000014014aa60     strings:ctype-extra.obj
 0003:00034b60       to_upper_cp1250_general_ci 000000014014ab60     strings:ctype-extra.obj
 0003:00034c60       sort_order_cp1250_general_ci 000000014014ac60     strings:ctype-extra.obj
 0003:00034d60       to_uni_cp1250_general_ci   000000014014ad60     strings:ctype-extra.obj
 0003:00034f60       ctype_latin2_croatian_ci   000000014014af60     strings:ctype-extra.obj
 0003:00035070       to_lower_latin2_croatian_ci 000000014014b070     strings:ctype-extra.obj
 0003:00035170       to_upper_latin2_croatian_ci 000000014014b170     strings:ctype-extra.obj
 0003:00035270       sort_order_latin2_croatian_ci 000000014014b270     strings:ctype-extra.obj
 0003:00035370       to_uni_latin2_croatian_ci  000000014014b370     strings:ctype-extra.obj
 0003:00035570       ctype_cp1250_croatian_ci   000000014014b570     strings:ctype-extra.obj
 0003:00035680       to_lower_cp1250_croatian_ci 000000014014b680     strings:ctype-extra.obj
 0003:00035780       to_upper_cp1250_croatian_ci 000000014014b780     strings:ctype-extra.obj
 0003:00035880       sort_order_cp1250_croatian_ci 000000014014b880     strings:ctype-extra.obj
 0003:00035980       to_uni_cp1250_croatian_ci  000000014014b980     strings:ctype-extra.obj
 0003:00035b80       ctype_latin1_general_ci    000000014014bb80     strings:ctype-extra.obj
 0003:00035c90       to_lower_latin1_general_ci 000000014014bc90     strings:ctype-extra.obj
 0003:00035d90       to_upper_latin1_general_ci 000000014014bd90     strings:ctype-extra.obj
 0003:00035e90       sort_order_latin1_general_ci 000000014014be90     strings:ctype-extra.obj
 0003:00035f90       to_uni_latin1_general_ci   000000014014bf90     strings:ctype-extra.obj
 0003:00036190       ctype_latin1_general_cs    000000014014c190     strings:ctype-extra.obj
 0003:000362a0       to_lower_latin1_general_cs 000000014014c2a0     strings:ctype-extra.obj
 0003:000363a0       to_upper_latin1_general_cs 000000014014c3a0     strings:ctype-extra.obj
 0003:000364a0       sort_order_latin1_general_cs 000000014014c4a0     strings:ctype-extra.obj
 0003:000365a0       to_uni_latin1_general_cs   000000014014c5a0     strings:ctype-extra.obj
 0003:000367a0       ctype_cp1250_bin           000000014014c7a0     strings:ctype-extra.obj
 0003:000368b0       to_lower_cp1250_bin        000000014014c8b0     strings:ctype-extra.obj
 0003:000369b0       to_upper_cp1250_bin        000000014014c9b0     strings:ctype-extra.obj
 0003:00036ab0       to_uni_cp1250_bin          000000014014cab0     strings:ctype-extra.obj
 0003:00036cb0       ctype_latin2_bin           000000014014ccb0     strings:ctype-extra.obj
 0003:00036dc0       to_lower_latin2_bin        000000014014cdc0     strings:ctype-extra.obj
 0003:00036ec0       to_upper_latin2_bin        000000014014cec0     strings:ctype-extra.obj
 0003:00036fc0       to_uni_latin2_bin          000000014014cfc0     strings:ctype-extra.obj
 0003:000371c0       ctype_latin1_spanish_ci    000000014014d1c0     strings:ctype-extra.obj
 0003:000372d0       to_lower_latin1_spanish_ci 000000014014d2d0     strings:ctype-extra.obj
 0003:000373d0       to_upper_latin1_spanish_ci 000000014014d3d0     strings:ctype-extra.obj
 0003:000374d0       sort_order_latin1_spanish_ci 000000014014d4d0     strings:ctype-extra.obj
 0003:000375d0       to_uni_latin1_spanish_ci   000000014014d5d0     strings:ctype-extra.obj
 0003:000377d0       compiled_charsets          000000014014d7d0     strings:ctype-extra.obj
 0003:0003c2c0       my_unicase_default         00000001401522c0     strings:ctype-utf8.obj
 0003:0003d0c0       my_unicase_turkish         00000001401530c0     strings:ctype-utf8.obj
 0003:0003dc30       my_charset_utf8_handler    0000000140153c30     strings:ctype-utf8.obj
 0003:0003dd00       my_charset_utf8_general_ci 0000000140153d00     strings:ctype-utf8.obj
 0003:0003ddb0       my_charset_utf8_bin        0000000140153db0     strings:ctype-utf8.obj
 0003:00058660       my_charset_ujis_japanese_ci 000000014016e660     strings:ctype-ujis.obj
 0003:00058710       my_charset_ujis_bin        000000014016e710     strings:ctype-ujis.obj
 0003:00058bc0       my_charset_ucs2_handler    000000014016ebc0     strings:ctype-ucs2.obj
 0003:00058c90       my_charset_ucs2_general_ci 000000014016ec90     strings:ctype-ucs2.obj
 0003:00058d40       my_charset_ucs2_bin        000000014016ed40     strings:ctype-ucs2.obj
 0003:0005b430       my_charset_tis620_thai_ci  0000000140171430     strings:ctype-tis620.obj
 0003:0005b4e0       my_charset_tis620_bin      00000001401714e0     strings:ctype-tis620.obj
 0003:0006b6e0       my_charset_sjis_japanese_ci 00000001401816e0     strings:ctype-sjis.obj
 0003:0006b790       my_charset_sjis_bin        0000000140181790     strings:ctype-sjis.obj
 0003:000930b0       my_charset_gbk_chinese_ci  00000001401a90b0     strings:ctype-gbk.obj
 0003:00093160       my_charset_gbk_bin         00000001401a9160     strings:ctype-gbk.obj
 0003:000a8760       my_charset_gb2312_chinese_ci 00000001401be760     strings:ctype-gb2312.obj
 0003:000a8810       my_charset_gb2312_bin      00000001401be810     strings:ctype-gb2312.obj
 0003:000c9560       my_charset_euckr_korean_ci 00000001401df560     strings:ctype-euc_kr.obj
 0003:000c9610       my_charset_euckr_bin       00000001401df610     strings:ctype-euc_kr.obj
 0003:000e43c0       my_charset_eucjpms_japanese_ci 00000001401fa3c0     strings:ctype-eucjpms.obj
 0003:000e4470       my_charset_eucjpms_bin     00000001401fa470     strings:ctype-eucjpms.obj
 0003:000e4de0       my_charset_latin2_czech_ci 00000001401fade0     strings:ctype-czech.obj
 0003:000e5bf0       my_charset_cp1250_czech_ci 00000001401fbbf0     strings:ctype-win1250ch.obj
 0003:000fc5a0       my_charset_big5_chinese_ci 00000001402125a0     strings:ctype-big5.obj
 0003:000fc650       my_charset_big5_bin        0000000140212650     strings:ctype-big5.obj
 0003:000fe530       my_collation_mb_bin_handler 0000000140214530     strings:ctype-mb.obj
 0003:000fe588       my_str_malloc              0000000140214588     strings:str_alloc.obj
 0003:000fe590       my_str_free                0000000140214590     strings:str_alloc.obj
 0003:000fea30       ??_R0?AUMessage@yaSSL@@@8  0000000140214a30     yassl:ssl.obj
 0003:000fea58       ??_R0?AVvirtual_base@yaSSL@@@8 0000000140214a58     yassl:ssl.obj
 0003:000fea88       ??_R0?AVHandShakeBase@yaSSL@@@8 0000000140214a88     yassl:ssl.obj
 0003:000feab8       ??_R0?AVHASH@TaoCrypt@@@8  0000000140214ab8     yassl:ssl.obj
 0003:000feae0       ??_R0?AVvirtual_base@TaoCrypt@@@8 0000000140214ae0     yassl:ssl.obj
 0003:000feb10       ??_R0?AVMD5@TaoCrypt@@@8   0000000140214b10     yassl:ssl.obj
 0003:000feb38       ??_R0?AVHASHwithTransform@TaoCrypt@@@8 0000000140214b38     yassl:ssl.obj
 0003:000feb70       ??_R0?AVMD4@TaoCrypt@@@8   0000000140214b70     yassl:ssl.obj
 0003:000ff3f0       ??_R0?AUDigest@yaSSL@@@8   00000001402153f0     yassl:crypto_wrapper.obj
 0003:000ff418       ??_R0?AUBulkCipher@yaSSL@@@8 0000000140215418     yassl:crypto_wrapper.obj
 0003:000ff440       ??_R0?AUAuth@yaSSL@@@8     0000000140215440     yassl:crypto_wrapper.obj
 0003:000ff468       ??_R0?AVSHA@TaoCrypt@@@8   0000000140215468     yassl:crypto_wrapper.obj
 0003:000ff490       ??_R0?AVRIPEMD160@TaoCrypt@@@8 0000000140215490     yassl:crypto_wrapper.obj
 0003:000ff4c0       ??_R0?AVMode_BASE@TaoCrypt@@@8 00000001402154c0     yassl:crypto_wrapper.obj
 0003:000ff4f0       ??_R0?AVDES@TaoCrypt@@@8   00000001402154f0     yassl:crypto_wrapper.obj
 0003:000ff518       ??_R0?AVBasicDES@TaoCrypt@@@8 0000000140215518     yassl:crypto_wrapper.obj
 0003:000ff540       ??_R0?AVDES_EDE3@TaoCrypt@@@8 0000000140215540     yassl:crypto_wrapper.obj
 0003:000ff568       ??_R0?AVAES@TaoCrypt@@@8   0000000140215568     yassl:crypto_wrapper.obj
 0003:000ff590       ??_R0?AVMD5@yaSSL@@@8      0000000140215590     yassl:crypto_wrapper.obj
 0003:000ff5b0       ??_R0?AVSHA@yaSSL@@@8      00000001402155b0     yassl:crypto_wrapper.obj
 0003:000ff5d0       ??_R0?AVRMD@yaSSL@@@8      00000001402155d0     yassl:crypto_wrapper.obj
 0003:000ff5f0       ??_R0?AVRC4@yaSSL@@@8      00000001402155f0     yassl:crypto_wrapper.obj
 0003:000ff610       ??_R0?AVAES@yaSSL@@@8      0000000140215610     yassl:crypto_wrapper.obj
 0003:000ff630       ??_R0?AVHMAC_MD5@yaSSL@@@8 0000000140215630     yassl:crypto_wrapper.obj
 0003:000ff658       ??_R0?AVHMAC_SHA@yaSSL@@@8 0000000140215658     yassl:crypto_wrapper.obj
 0003:000ff680       ??_R0?AVHMAC_RMD@yaSSL@@@8 0000000140215680     yassl:crypto_wrapper.obj
 0003:000ff6a8       ??_R0?AVDES@yaSSL@@@8      00000001402156a8     yassl:crypto_wrapper.obj
 0003:000ff6c8       ??_R0?AVDES_EDE@yaSSL@@@8  00000001402156c8     yassl:crypto_wrapper.obj
 0003:000ff6f0       ??_R0?AVDSS@yaSSL@@@8      00000001402156f0     yassl:crypto_wrapper.obj
 0003:000ff710       ??_R0?AVRSA@yaSSL@@@8      0000000140215710     yassl:crypto_wrapper.obj
 0003:000ffb40       ??_R0?AVHandShakeHeader@yaSSL@@@8 0000000140215b40     yassl:yassl_imp.obj
 0003:000ffb70       ??_R0?AUServerKeyBase@yaSSL@@@8 0000000140215b70     yassl:yassl_imp.obj
 0003:000ffba0       ??_R0?AUClientKeyBase@yaSSL@@@8 0000000140215ba0     yassl:yassl_imp.obj
 0003:000ffbd0       ??_R0?AVClientDiffieHellmanPublic@yaSSL@@@8 0000000140215bd0     yassl:yassl_imp.obj
 0003:000ffc08       ??_R0?AVChangeCipherSpec@yaSSL@@@8 0000000140215c08     yassl:yassl_imp.obj
 0003:000ffc38       ??_R0?AVAlert@yaSSL@@@8    0000000140215c38     yassl:yassl_imp.obj
 0003:000ffc60       ??_R0?AVData@yaSSL@@@8     0000000140215c60     yassl:yassl_imp.obj
 0003:000ffc88       ??_R0?AVCertificate@yaSSL@@@8 0000000140215c88     yassl:yassl_imp.obj
 0003:000ffcb0       ??_R0?AVServerHello@yaSSL@@@8 0000000140215cb0     yassl:yassl_imp.obj
 0003:000ffcd8       ??_R0?AUServerHelloDone@yaSSL@@@8 0000000140215cd8     yassl:yassl_imp.obj
 0003:000ffd08       ??_R0?AVClientHello@yaSSL@@@8 0000000140215d08     yassl:yassl_imp.obj
 0003:000ffd30       ??_R0?AVServerKeyExchange@yaSSL@@@8 0000000140215d30     yassl:yassl_imp.obj
 0003:000ffd60       ??_R0?AVCertificateVerify@yaSSL@@@8 0000000140215d60     yassl:yassl_imp.obj
 0003:000ffd90       ??_R0?AVClientKeyExchange@yaSSL@@@8 0000000140215d90     yassl:yassl_imp.obj
 0003:000ffdc0       ??_R0?AVFinished@yaSSL@@@8 0000000140215dc0     yassl:yassl_imp.obj
 0003:000ffde8       ??_R0?AUHelloRequest@yaSSL@@@8 0000000140215de8     yassl:yassl_imp.obj
 0003:000ffe18       ??_R0?AURSA_Server@yaSSL@@@8 0000000140215e18     yassl:yassl_imp.obj
 0003:000ffe40       ??_R0?AUFortezza_Server@yaSSL@@@8 0000000140215e40     yassl:yassl_imp.obj
 0003:000ffe70       ??_R0?AUFortezzaKeys@yaSSL@@@8 0000000140215e70     yassl:yassl_imp.obj
 0003:000ffea0       ??_R0?AVEncryptedPreMasterSecret@yaSSL@@@8 0000000140215ea0     yassl:yassl_imp.obj
 0003:000ffed8       ??_R0?AVDH_Server@yaSSL@@@8 0000000140215ed8     yassl:yassl_imp.obj
 0003:000fff00       ??_R0?AVCertificateRequest@yaSSL@@@8 0000000140215f00     yassl:yassl_imp.obj
 0003:00100bb0       _fltused                   0000000140216bb0     LIBCMT:fpinit.obj
 0003:00100bb4       _ldused                    0000000140216bb4     LIBCMT:fpinit.obj
 0003:00100bc0       ??_R0?AVtype_info@@@8      0000000140216bc0     LIBCMT:typinfo.obj
 0003:00100be0       __security_cookie          0000000140216be0     LIBCMT:gs_cookie.obj
 0003:00100be8       __security_cookie_complement 0000000140216be8     LIBCMT:gs_cookie.obj
 0003:00100bf8       ??_R0?AVbad_alloc@std@@@8  0000000140216bf8     LIBCMT:new.obj
 0003:00100c20       ??_R0?AVexception@std@@@8  0000000140216c20     LIBCMT:new.obj
 0003:00100dc0       _iob                       0000000140216dc0     LIBCMT:_file.obj
 0003:00101180       _aexit_rtn                 0000000140217180     LIBCMT:crt0dat.obj
 0003:00101194       __app_type                 0000000140217194     LIBCMT:crt0.obj
 0003:001011c0       _cfltcvt_tab               00000001402171c0     LIBCMT:cmiscdat.obj
 0003:00101218       __abort_behavior           0000000140217218     LIBCMT:abort.obj
 0003:00101390       __flsindex                 0000000140217390     LIBCMT:tidtable.obj
 0003:00101394       __getvalueindex            0000000140217394     LIBCMT:tidtable.obj
 0003:001013a0       ??_R0?AVbad_cast@std@@@8   00000001402173a0     LIBCMT:stdexcpt.obj
 0003:001013c8       ??_R0?AVbad_typeid@std@@@8 00000001402173c8     LIBCMT:stdexcpt.obj
 0003:001013f0       ??_R0?AV__non_rtti_object@std@@@8 00000001402173f0     LIBCMT:stdexcpt.obj
 0003:00101420       __nullstring               0000000140217420     LIBCMT:output.obj
 0003:00101428       __wnullstring              0000000140217428     LIBCMT:output.obj
 0003:00101430       __badioinfo                0000000140217430     LIBCMT:ioinit.obj
 0003:00101490       _sys_errlist               0000000140217490     LIBCMT:syserr.obj
 0003:001015f0       _sys_nerr                  00000001402175f0     LIBCMT:syserr.obj
 0003:00101840       _XcptActTab                0000000140217840     LIBCMT:winxfltr.obj
 0003:001018e0       _First_FPE_Indx            00000001402178e0     LIBCMT:winxfltr.obj
 0003:001018e4       _Num_FPE                   00000001402178e4     LIBCMT:winxfltr.obj
 0003:001018e8       _XcptActTabSize            00000001402178e8     LIBCMT:winxfltr.obj
 0003:001018ec       _XcptActTabCount           00000001402178ec     LIBCMT:winxfltr.obj
 0003:001018f0       __initialmbcinfo           00000001402178f0     LIBCMT:mbctype.obj
 0003:00101b10       _mbctype                   0000000140217b10     LIBCMT:mbctype.obj
 0003:00101c20       _mbcasemap                 0000000140217c20     LIBCMT:mbctype.obj
 0003:00101d20       __ptmbcinfo                0000000140217d20     LIBCMT:mbctype.obj
 0003:00101e28       __globallocalestatus       0000000140217e28     LIBCMT:glstatus.obj
 0003:00101e30       __clocalestr               0000000140217e30     LIBCMT:nlsdata2.obj
 0003:00101e40       __initiallocinfo           0000000140217e40     LIBCMT:nlsdata2.obj
 0003:00101fa0       __ptlocinfo                0000000140217fa0     LIBCMT:nlsdata2.obj
 0003:00101fa8       __lc_clike                 0000000140217fa8     LIBCMT:nlsdata2.obj
 0003:00101fb0       __initiallocalestructinfo  0000000140217fb0     LIBCMT:nlsdata2.obj
 0003:00101fc0       _coninpfh                  0000000140217fc0     LIBCMT:initcon.obj
 0003:00101fc8       _confh                     0000000140217fc8     LIBCMT:initcon.obj
 0003:00101fd0       _amblksiz                  0000000140217fd0     LIBCMT:heapinit.obj
 0003:00101fe0       _timezone                  0000000140217fe0     LIBCMT:timeset.obj
 0003:00101fe4       _daylight                  0000000140217fe4     LIBCMT:timeset.obj
 0003:00101fe8       _dstbias                   0000000140217fe8     LIBCMT:timeset.obj
 0003:00102070       _tzname                    0000000140218070     LIBCMT:timeset.obj
 0003:00102080       _lpdays                    0000000140218080     LIBCMT:days.obj
 0003:001020b8       _days                      00000001402180b8     LIBCMT:days.obj
 0003:001020f0       _lookuptrailbytes          00000001402180f0     LIBCMT:read.obj
 0003:001021f0       ??_R0?AVDNameNode@@@8      00000001402181f0     LIBCMT:undname.obj
 0003:00102210       ??_R0?AVcharNode@@@8       0000000140218210     LIBCMT:undname.obj
 0003:00102230       ??_R0?AVpDNameNode@@@8     0000000140218230     LIBCMT:undname.obj
 0003:00102258       ??_R0?AVDNameStatusNode@@@8 0000000140218258     LIBCMT:undname.obj
 0003:00102280       ??_R0?AVpcharNode@@@8      0000000140218280     LIBCMT:undname.obj
 0003:00102470       _matherr_flag              0000000140218470     LIBCMT:matherr.obj
 0003:00102478       _pctype                    0000000140218478     LIBCMT:ctype.obj
 0003:00102480       _pwctype                   0000000140218480     LIBCMT:ctype.obj
 0003:00102490       __lc_time_c                0000000140218490     LIBCMT:strftime.obj
 0003:001025f8       __lc_time_curr             00000001402185f8     LIBCMT:strftime.obj
 0003:00102600       __lconv_static_decimal     0000000140218600     LIBCMT:lconv.obj
 0003:00102610       __lconv_c                  0000000140218610     LIBCMT:lconv.obj
 0003:00102668       __lconv                    0000000140218668     LIBCMT:lconv.obj
 0003:00102670       __mb_cur_max               0000000140218670     LIBCMT:nlsdata1.obj
 0003:00102674       __decimal_point            0000000140218674     LIBCMT:nlsdata1.obj
 0003:00102678       __decimal_point_length     0000000140218678     LIBCMT:nlsdata1.obj
 0003:001026b8       _d_inf                     00000001402186b8     LIBCMT:util.obj
 0003:001026c0       _d_ind                     00000001402186c0     LIBCMT:util.obj
 0003:001026c8       _d_max                     00000001402186c8     LIBCMT:util.obj
 0003:001026d0       _d_min                     00000001402186d0     LIBCMT:util.obj
 0003:001026d8       _d_mzero                   00000001402186d8     LIBCMT:util.obj
 0003:001026e0       _pow10pos                  00000001402186e0     LIBCMT:constpow.obj
 0003:00102840       _pow10neg                  0000000140218840     LIBCMT:constpow.obj
 0003:001029a0       ??_R0?AVHASH64withTransform@TaoCrypt@@@8 00000001402189a0     taocrypt:hash.obj
 0003:001029e0       ??_R0?AVMultiplicativeGroupT@AbstractRing@TaoCrypt@@@8 00000001402189e0     taocrypt:integer.obj
 0003:00102a28       ??_R0?AVAbstractGroup@TaoCrypt@@@8 0000000140218a28     taocrypt:integer.obj
 0003:00102a58       ??_R0?AVModularArithmetic@TaoCrypt@@@8 0000000140218a58     taocrypt:integer.obj
 0003:00102a90       ??_R0?AVAbstractRing@TaoCrypt@@@8 0000000140218a90     taocrypt:integer.obj
 0003:00102ac0       ??_R0?AVMontgomeryRepresentation@TaoCrypt@@@8 0000000140218ac0     taocrypt:integer.obj
 0003:00102af8       ??_R0?AVEuclideanDomainOf@TaoCrypt@@@8 0000000140218af8     taocrypt:integer.obj
 0003:00102b30       ??_R0?AVAbstractEuclideanDomain@TaoCrypt@@@8 0000000140218b30     taocrypt:integer.obj
 0003:00102b68       ??_R0?AVSHA256@TaoCrypt@@@8 0000000140218b68     taocrypt:sha.obj
 0003:00102b90       ??_R0?AVSHA224@TaoCrypt@@@8 0000000140218b90     taocrypt:sha.obj
 0003:00102bb8       ??_R0?AVSHA512@TaoCrypt@@@8 0000000140218bb8     taocrypt:sha.obj
 0003:00102be0       ??_R0?AVSHA384@TaoCrypt@@@8 0000000140218be0     taocrypt:sha.obj
 0003:00102c08       ?Te0@AES@TaoCrypt@@0PEBIEB 0000000140218c08     taocrypt:aes.obj
 0003:00102c10       ?Te1@AES@TaoCrypt@@0PEBIEB 0000000140218c10     taocrypt:aes.obj
 0003:00102c18       ?Te2@AES@TaoCrypt@@0PEBIEB 0000000140218c18     taocrypt:aes.obj
 0003:00102c20       ?Te3@AES@TaoCrypt@@0PEBIEB 0000000140218c20     taocrypt:aes.obj
 0003:00102c28       ?Te4@AES@TaoCrypt@@0PEBIEB 0000000140218c28     taocrypt:aes.obj
 0003:00102c30       ?Td0@AES@TaoCrypt@@0PEBIEB 0000000140218c30     taocrypt:aes.obj
 0003:00102c38       ?Td1@AES@TaoCrypt@@0PEBIEB 0000000140218c38     taocrypt:aes.obj
 0003:00102c40       ?Td2@AES@TaoCrypt@@0PEBIEB 0000000140218c40     taocrypt:aes.obj
 0003:00102c48       ?Td3@AES@TaoCrypt@@0PEBIEB 0000000140218c48     taocrypt:aes.obj
 0003:00102c50       ?Td4@AES@TaoCrypt@@0PEBIEB 0000000140218c50     taocrypt:aes.obj
 0003:00102c60       ??_R0?AVBER_Decoder@TaoCrypt@@@8 0000000140218c60     taocrypt:dsa.obj
 0003:00102c90       ??_R0?AVDSA_Private_Decoder@TaoCrypt@@@8 0000000140218c90     taocrypt:dsa.obj
 0003:00102cc8       ??_R0?AVDSA_Public_Decoder@TaoCrypt@@@8 0000000140218cc8     taocrypt:dsa.obj
 0003:00102d08       ??_R0?AVDH_Decoder@TaoCrypt@@@8 0000000140218d08     taocrypt:dh.obj
 0003:00102d40       ??_R0?AVRSA_Private_Decoder@TaoCrypt@@@8 0000000140218d40     taocrypt:rsa.obj
 0003:00102d78       ??_R0?AVRSA_Public_Decoder@TaoCrypt@@@8 0000000140218d78     taocrypt:rsa.obj
 0003:00102db8       ??_R0?AVDER_Encoder@TaoCrypt@@@8 0000000140218db8     taocrypt:asn.obj
 0003:00102de8       ??_R0?AVCertDecoder@TaoCrypt@@@8 0000000140218de8     taocrypt:asn.obj
 0003:00102e18       ??_R0?AVSignature_Encoder@TaoCrypt@@@8 0000000140218e18     taocrypt:asn.obj
 0003:00102e58       ??_R0?AVMD2@TaoCrypt@@@8   0000000140218e58     taocrypt:md2.obj
 0003:001364a0       ?have_signal@@3_NA         000000014024c4a0     manager.obj
 0003:001364b0       ?remove_service@Options@@2DA 000000014024c4b0     options.obj
 0003:001364b1       ?install_as_service@Options@@2DA 000000014024c4b1     options.obj
 0003:001364b2       ?stand_alone@Options@@2DA  000000014024c4b2     options.obj
 0003:001364c0       ?default_log_file_name@@3PADA 000000014024c4c0     options.obj
 0003:001366c0       ?default_password_file_name@@3PADA 000000014024c6c0     options.obj
 0003:001368c0       ?windows_config_file@@3PADA 000000014024c8c0     options.obj
 0003:00136ac0       ?bind_address@Options@@2PEBDEB 000000014024cac0     options.obj
 0003:00136ac8       ?saved_argv@Options@@2PEAPEADEA 000000014024cac8     options.obj
 0003:00136ad0       ?is_forced_default_file@Options@@2_NA 000000014024cad0     options.obj
 0003:00136c0c       ?manager_pid@@3HA          000000014024cc0c     priv.obj
 0003:00136c10       ?open_files_limit@@3KA     000000014024cc10     priv.obj
 0003:00136c14       ?linuxthreads@@3_NA        000000014024cc14     priv.obj
 0003:00136c18       ?test_flags@@3IA           000000014024cc18     priv.obj
 0003:00136c1c       ?bytes_sent@@3KA           000000014024cc1c     priv.obj
 0003:00136c20       ?bytes_received@@3KA       000000014024cc20     priv.obj
 0003:00136c38       mysql_port                 000000014024cc38     client.obj
 0003:00136c40       mysql_unix_port            000000014024cc40     client.obj
 0003:00136c4c       THR_thread_count           000000014024cc4c     mysys:my_thr_init.obj
 0003:00136c80       thd_lib_detected           000000014024cc80     mysys:my_pthread.obj
 0003:00136c88       charsets_dir               000000014024cc88     mysys:charset.obj
 0003:00136ca0       my_defaults_file           000000014024cca0     mysys:default.obj
 0003:00136ca8       my_defaults_group_suffix   000000014024cca8     mysys:default.obj
 0003:00136cb0       my_defaults_extra_file     000000014024ccb0     mysys:default.obj
 0003:00136cc0       timed_mutexes              000000014024ccc0     mysys:my_static.obj
 0003:00136cc1       my_disable_locking         000000014024ccc1     mysys:my_static.obj
 0003:00136cc2       my_disable_async_io        000000014024ccc2     mysys:my_static.obj
 0003:00136cc3       my_disable_flush_key_blocks 000000014024ccc3     mysys:my_static.obj
 0003:00136cc4       my_stream_opened           000000014024ccc4     mysys:my_static.obj
 0003:00136cc8       home_dir                   000000014024ccc8     mysys:my_static.obj
 0003:00136cd0       my_progname                000000014024ccd0     mysys:my_static.obj
 0003:00136cd8       my_file_opened             000000014024ccd8     mysys:my_static.obj
 0003:00136cdc       my_tmp_file_created        000000014024ccdc     mysys:my_static.obj
 0003:00136ce0       curr_dir                   000000014024cce0     mysys:my_static.obj
 0003:00136ee0       home_dir_buff              000000014024cee0     mysys:my_static.obj
 0003:001370e0       my_file_info_default       000000014024d0e0     mysys:my_static.obj
 0003:00137ee0       my_dont_interrupt          000000014024dee0     mysys:my_static.obj
 0003:00137ee4       _my_signals                000000014024dee4     mysys:my_static.obj
 0003:00137ee8       my_once_root_block         000000014024dee8     mysys:my_static.obj
 0003:00137ef0       _my_sig_remember           000000014024def0     mysys:my_static.obj
 0003:00137f90       sf_malloc_prehunc          000000014024df90     mysys:my_static.obj
 0003:00137f94       sf_malloc_endhunc          000000014024df94     mysys:my_static.obj
 0003:00137f98       sf_malloc_quick            000000014024df98     mysys:my_static.obj
 0003:00137f9c       sf_malloc_count            000000014024df9c     mysys:my_static.obj
 0003:00137fa0       sf_malloc_cur_memory       000000014024dfa0     mysys:my_static.obj
 0003:00137fa8       sf_malloc_max_memory       000000014024dfa8     mysys:my_static.obj
 0003:00137fb0       sf_max_adress              000000014024dfb0     mysys:my_static.obj
 0003:00137fb8       sf_malloc_root             000000014024dfb8     mysys:my_static.obj
 0003:00137fc0       my_have_got_alarm          000000014024dfc0     mysys:my_static.obj
 0003:00137fc4       my_disable_symlinks        000000014024dfc4     mysys:my_static.obj
 0003:00137fc5       mysys_uses_curses          000000014024dfc5     mysys:my_static.obj
 0003:00137fc8       have_tcpip                 000000014024dfc8     mysys:my_init.obj
 0003:00137fc9       my_init_done               000000014024dfc9     mysys:my_init.obj
 0003:00137fcc       mysys_usage_id             000000014024dfcc     mysys:my_init.obj
 0003:00137fd8       thr_alarm_inited           000000014024dfd8     mysys:thr_alarm.obj
 0003:00137fd9       alarm_thread_running       000000014024dfd9     mysys:thr_alarm.obj
 0003:00137fda       my_use_symdir              000000014024dfda     mysys:mf_pack.obj
 0003:00138014       __fastflag                 000000014024e014     LIBCMT:fpinit.obj
 0003:00138040       _cflush                    000000014024e040     LIBCMT:_file.obj
 0003:00138048       _umaskval                  000000014024e048     LIBCMT:crt0dat.obj
 0003:0013804c       _osplatform                000000014024e04c     LIBCMT:crt0dat.obj
 0003:00138050       _osver                     000000014024e050     LIBCMT:crt0dat.obj
 0003:00138054       _winver                    000000014024e054     LIBCMT:crt0dat.obj
 0003:00138058       _winmajor                  000000014024e058     LIBCMT:crt0dat.obj
 0003:0013805c       _winminor                  000000014024e05c     LIBCMT:crt0dat.obj
 0003:00138060       __argc                     000000014024e060     LIBCMT:crt0dat.obj
 0003:00138064       _exitflag                  000000014024e064     LIBCMT:crt0dat.obj
 0003:00138068       __argv                     000000014024e068     LIBCMT:crt0dat.obj
 0003:00138070       __wargv                    000000014024e070     LIBCMT:crt0dat.obj
 0003:00138078       _environ                   000000014024e078     LIBCMT:crt0dat.obj
 0003:00138080       __initenv                  000000014024e080     LIBCMT:crt0dat.obj
 0003:00138088       _wenviron                  000000014024e088     LIBCMT:crt0dat.obj
 0003:00138090       __winitenv                 000000014024e090     LIBCMT:crt0dat.obj
 0003:00138098       _pgmptr                    000000014024e098     LIBCMT:crt0dat.obj
 0003:001380a0       _wpgmptr                   000000014024e0a0     LIBCMT:crt0dat.obj
 0003:001380a8       _C_Termination_Done        000000014024e0a8     LIBCMT:crt0dat.obj
 0003:001380ac       _C_Exit_Done               000000014024e0ac     LIBCMT:crt0dat.obj
 0003:001380d8       __idtabsiz                 000000014024e0d8     LIBCMT:popen.obj
 0003:001380e0       __idpairs                  000000014024e0e0     LIBCMT:popen.obj
 0003:001380e8       _aenvptr                   000000014024e0e8     LIBCMT:crt0.obj
 0003:001380f0       _wenvptr                   000000014024e0f0     LIBCMT:crt0.obj
 0003:001380f8       __error_mode               000000014024e0f8     LIBCMT:crt0.obj
 0003:001380fc       _tls_index                 000000014024e0fc     LIBCMT:tlssup.obj
 0003:001381c0       __pInvalidArgHandler       000000014024e1c0     LIBCMT:invarg.obj
 0003:00138500       __pPurecall                000000014024e500     LIBCMT:inithelp.obj
 0003:00138a80       ?_pnhHeap@@3P6AH_K@ZEA     000000014024ea80     LIBCMT:handler.obj
 0003:00138a88       _stdbuf                    000000014024ea88     LIBCMT:_sftbuf.obj
 0003:00138a98       _maxwait                   000000014024ea98     LIBCMT:crtheap.obj
 0003:00138cd0       ?__pInconsistency@@3P6AXXZEA 000000014024ecd0     LIBCMT:hooks.obj
 0003:00138cf0       __mbulinfo                 000000014024ecf0     LIBCMT:mbctype.obj
 0003:00138cfc       __mbcodepage               000000014024ecfc     LIBCMT:mbctype.obj
 0003:00138d00       __ismbcodepage             000000014024ed00     LIBCMT:mbctype.obj
 0003:00138d04       __mblcid                   000000014024ed04     LIBCMT:mbctype.obj
 0003:00138d08       __locale_changed           000000014024ed08     LIBCMT:setlocal.obj
 0003:00138d10       __lc_handle                000000014024ed10     LIBCMT:nlsdata2.obj
 0003:00138d28       __lc_codepage              000000014024ed28     LIBCMT:nlsdata2.obj
 0003:00138d2c       __lc_collate_cp            000000014024ed2c     LIBCMT:nlsdata2.obj
 0003:00138e40       _crtheap                   000000014024ee40     LIBCMT:heapinit.obj
 0003:00138e48       _newmode                   000000014024ee48     LIBCMT:_newmode.obj
 0003:00138e4c       _outputformat              000000014024ee4c     LIBCMT:outputformat.obj
 0003:00138e50       ?pArgList@UnDecorator@@0PEAVReplicator@@EA 000000014024ee50     LIBCMT:undname.obj
 0003:00138e80       ?pZNameList@UnDecorator@@0PEAVReplicator@@EA 000000014024ee80     LIBCMT:undname.obj
 0003:00138e88       ?pTemplateArgList@UnDecorator@@0PEAVReplicator@@EA 000000014024ee88     LIBCMT:undname.obj
 0003:00138e90       ?gName@UnDecorator@@0PEBDEB 000000014024ee90     LIBCMT:undname.obj
 0003:00138e98       ?name@UnDecorator@@0PEBDEB 000000014024ee98     LIBCMT:undname.obj
 0003:00138ea0       ?outputString@UnDecorator@@0PEADEA 000000014024eea0     LIBCMT:undname.obj
 0003:00138ea8       ?maxStringLength@UnDecorator@@0HA 000000014024eea8     LIBCMT:undname.obj
 0003:00138eac       ?disableFlags@UnDecorator@@0KA 000000014024eeac     LIBCMT:undname.obj
 0003:00138eb0       ?m_pGetParameter@UnDecorator@@0P6APEADJ@ZEA 000000014024eeb0     LIBCMT:undname.obj
 0003:00138eb8       ?fExplicitTemplateParams@UnDecorator@@0_NA 000000014024eeb8     LIBCMT:undname.obj
 0003:00138eb9       ?fGetTemplateArgumentList@UnDecorator@@0_NA 000000014024eeb9     LIBCMT:undname.obj
 0003:00138ef4       _commode                   000000014024eef4     LIBCMT:ncommode.obj
 0003:00138f00       __lconv_static_null        000000014024ef00     LIBCMT:lconv.obj
 0003:00138f04       _fmode                     000000014024ef04     LIBCMT:txtmode.obj
 0003:00138f40       mysql_server_last_error    000000014024ef40     <common>
 0003:001391b0       mysql_server_last_errno    000000014024f1b0     <common>
 0003:001391b4       thr_client_alarm           000000014024f1b4     <common>
 0003:001391c0       errbuff                    000000014024f1c0     <common>
 0003:00139430       my_signals                 000000014024f430     <common>
 0003:00139440       all_charsets               000000014024f440     <common>
 0003:00139e00       THR_LOCK_threads           000000014024fe00     <common>
 0003:00139ea0       LOCK_gethostbyname_r       000000014024fea0     <common>
 0003:00139ee0       THR_LOCK_myisam_mmap       000000014024fee0     <common>
 0003:00139f20       THR_COND_threads           000000014024ff20     <common>
 0003:00139f80       THR_LOCK_malloc            000000014024ff80     <common>
 0003:00139fc0       THR_LOCK_isam              000000014024ffc0     <common>
 0003:0013a000       THR_LOCK_myisam            0000000140250000     <common>
 0003:0013a040       THR_LOCK_heap              0000000140250040     <common>
 0003:0013a080       THR_LOCK_open              0000000140250080     <common>
 0003:0013a0c0       THR_LOCK_charset           00000001402500c0     <common>
 0003:0013a100       THR_LOCK_lock              0000000140250100     <common>
 0003:0013a140       LOCK_localtime_r           0000000140250140     <common>
 0003:0013a180       THR_LOCK_net               0000000140250180     <common>
 0003:0013a1a8       _debugger_hook_dummy       00000001402501a8     <common>
 0003:0013a1b4       __setlc_active             00000001402501b4     <common>
 0003:0013a1c4       __unguarded_readlc_active  00000001402501c4     <common>
 0003:0013a1c8       _nhandle                   00000001402501c8     <common>
 0003:0013a240       __pioinfo                  0000000140250240     <common>
 0003:0013a440       _pDestructExceptionObject  0000000140250440     <common>
 0003:0013a458       _acmdln                    0000000140250458     <common>
 0003:0013a46c       __env_initialized          000000014025046c     <common>
 0003:0013a480       __onexitend                0000000140250480     <common>
 0003:0013a488       __onexitbegin              0000000140250488     <common>
 0003:0013a490       __mbctype_initialized      0000000140250490     <common>
 0003:0013a498       __dyn_tls_init_callback    0000000140250498     <common>
 0003:0013a4a0       __piob                     00000001402504a0     <common>
 0003:0013a800       _bufin                     0000000140250800     <common>
 0003:0013b800       _nstream                   0000000140251800     <common>
 0005:00000000       __IMPORT_DESCRIPTOR_KERNEL32 000000014025f000     kernel32:KERNEL32.dll
 0005:00000014       __IMPORT_DESCRIPTOR_ADVAPI32 000000014025f014     advapi32:ADVAPI32.dll
 0005:00000028       __IMPORT_DESCRIPTOR_WSOCK32 000000014025f028     wsock32:WSOCK32.dll
 0005:0000003c       __IMPORT_DESCRIPTOR_USER32 000000014025f03c     user32:USER32.dll
 0005:00000050       __NULL_IMPORT_DESCRIPTOR   000000014025f050     kernel32:KERNEL32.dll
 0005:00000848       __imp_CryptGenRandom       000000014025f848     advapi32:ADVAPI32.dll
 0005:00000850       __imp_RegEnumValueA        000000014025f850     advapi32:ADVAPI32.dll
 0005:00000858       __imp_RegOpenKeyExA        000000014025f858     advapi32:ADVAPI32.dll
 0005:00000860       __imp_CryptAcquireContextA 000000014025f860     advapi32:ADVAPI32.dll
 0005:00000868       __imp_CryptReleaseContext  000000014025f868     advapi32:ADVAPI32.dll
 0005:00000870       __imp_StartServiceCtrlDispatcherA 000000014025f870     advapi32:ADVAPI32.dll
 0005:00000878       __imp_RegisterServiceCtrlHandlerA 000000014025f878     advapi32:ADVAPI32.dll
 0005:00000880       __imp_DeleteService        000000014025f880     advapi32:ADVAPI32.dll
 0005:00000888       __imp_CreateServiceA       000000014025f888     advapi32:ADVAPI32.dll
 0005:00000890       __imp_SetServiceStatus     000000014025f890     advapi32:ADVAPI32.dll
 0005:00000898       __imp_OpenSCManagerA       000000014025f898     advapi32:ADVAPI32.dll
 0005:000008a0       __imp_OpenServiceA         000000014025f8a0     advapi32:ADVAPI32.dll
 0005:000008a8       __imp_CloseServiceHandle   000000014025f8a8     advapi32:ADVAPI32.dll
 0005:000008b0       __imp_RegCloseKey          000000014025f8b0     advapi32:ADVAPI32.dll
 0005:000008b8       \177ADVAPI32_NULL_THUNK_DATA 000000014025f8b8     advapi32:ADVAPI32.dll
 0005:00000920       __imp_GetModuleHandleA     000000014025f920     kernel32:KERNEL32.dll
 0005:00000928       __imp_TerminateProcess     000000014025f928     kernel32:KERNEL32.dll
 0005:00000930       __imp_OpenProcess          000000014025f930     kernel32:KERNEL32.dll
 0005:00000938       __imp_Sleep                000000014025f938     kernel32:KERNEL32.dll
 0005:00000940       __imp_GetCurrentThreadId   000000014025f940     kernel32:KERNEL32.dll
 0005:00000948       __imp_GetCurrentProcess    000000014025f948     kernel32:KERNEL32.dll
 0005:00000950       __imp_SetNamedPipeHandleState 000000014025f950     kernel32:KERNEL32.dll
 0005:00000958       __imp_WaitNamedPipeA       000000014025f958     kernel32:KERNEL32.dll
 0005:00000960       __imp_CreateFileA          000000014025f960     kernel32:KERNEL32.dll
 0005:00000968       __imp_DuplicateHandle      000000014025f968     kernel32:KERNEL32.dll
 0005:00000970       __imp_GetProcAddress       000000014025f970     kernel32:KERNEL32.dll
 0005:00000978       __imp_CreateRemoteThread   000000014025f978     kernel32:KERNEL32.dll
 0005:00000980       __imp_GetLastError         000000014025f980     kernel32:KERNEL32.dll
 0005:00000988       __imp_SetLastError         000000014025f988     kernel32:KERNEL32.dll
 0005:00000990       __imp_CreateProcessA       000000014025f990     kernel32:KERNEL32.dll
 0005:00000998       __imp_WaitForSingleObject  000000014025f998     kernel32:KERNEL32.dll
 0005:000009a0       __imp_GetExitCodeProcess   000000014025f9a0     kernel32:KERNEL32.dll
 0005:000009a8       __imp_CloseHandle          000000014025f9a8     kernel32:KERNEL32.dll
 0005:000009b0       __imp_GetSystemTimeAsFileTime 000000014025f9b0     kernel32:KERNEL32.dll
 0005:000009b8       __imp_EnterCriticalSection 000000014025f9b8     kernel32:KERNEL32.dll
 0005:000009c0       __imp_SetEnvironmentVariableW 000000014025f9c0     kernel32:KERNEL32.dll
 0005:000009c8       __imp_LeaveCriticalSection 000000014025f9c8     kernel32:KERNEL32.dll
 0005:000009d0       __imp_DeleteCriticalSection 000000014025f9d0     kernel32:KERNEL32.dll
 0005:000009d8       __imp_GetModuleFileNameA   000000014025f9d8     kernel32:KERNEL32.dll
 0005:000009e0       __imp_WriteConsoleW        000000014025f9e0     kernel32:KERNEL32.dll
 0005:000009e8       __imp_GetConsoleOutputCP   000000014025f9e8     kernel32:KERNEL32.dll
 0005:000009f0       __imp_WriteConsoleA        000000014025f9f0     kernel32:KERNEL32.dll
 0005:000009f8       __imp_IsValidLocale        000000014025f9f8     kernel32:KERNEL32.dll
 0005:00000a00       __imp_EnumSystemLocalesA   000000014025fa00     kernel32:KERNEL32.dll
 0005:00000a08       __imp_GetUserDefaultLCID   000000014025fa08     kernel32:KERNEL32.dll
 0005:00000a10       __imp_GetTimeFormatA       000000014025fa10     kernel32:KERNEL32.dll
 0005:00000a18       __imp_GetDateFormatA       000000014025fa18     kernel32:KERNEL32.dll
 0005:00000a20       __imp_GetStringTypeW       000000014025fa20     kernel32:KERNEL32.dll
 0005:00000a28       __imp_GetStringTypeA       000000014025fa28     kernel32:KERNEL32.dll
 0005:00000a30       __imp_SetEnvironmentVariableA 000000014025fa30     kernel32:KERNEL32.dll
 0005:00000a38       __imp_CompareStringW       000000014025fa38     kernel32:KERNEL32.dll
 0005:00000a40       __imp_CompareStringA       000000014025fa40     kernel32:KERNEL32.dll
 0005:00000a48       __imp_LCMapStringW         000000014025fa48     kernel32:KERNEL32.dll
 0005:00000a50       __imp_LCMapStringA         000000014025fa50     kernel32:KERNEL32.dll
 0005:00000a58       __imp_GetLocaleInfoW       000000014025fa58     kernel32:KERNEL32.dll
 0005:00000a60       __imp_MultiByteToWideChar  000000014025fa60     kernel32:KERNEL32.dll
 0005:00000a68       __imp_FlushFileBuffers     000000014025fa68     kernel32:KERNEL32.dll
 0005:00000a70       __imp_GetConsoleCP         000000014025fa70     kernel32:KERNEL32.dll
 0005:00000a78       __imp_HeapSize             000000014025fa78     kernel32:KERNEL32.dll
 0005:00000a80       __imp_CreateEventA         000000014025fa80     kernel32:KERNEL32.dll
 0005:00000a88       __imp_SetEvent             000000014025fa88     kernel32:KERNEL32.dll
 0005:00000a90       __imp_ResetEvent           000000014025fa90     kernel32:KERNEL32.dll
 0005:00000a98       __imp_WaitForMultipleObjects 000000014025fa98     kernel32:KERNEL32.dll
 0005:00000aa0       __imp_TryEnterCriticalSection 000000014025faa0     kernel32:KERNEL32.dll
 0005:00000aa8       __imp_SetThreadPriority    000000014025faa8     kernel32:KERNEL32.dll
 0005:00000ab0       __imp_GetLocaleInfoA       000000014025fab0     kernel32:KERNEL32.dll
 0005:00000ab8       __imp_GetSystemDirectoryA  000000014025fab8     kernel32:KERNEL32.dll
 0005:00000ac0       __imp_GetWindowsDirectoryA 000000014025fac0     kernel32:KERNEL32.dll
 0005:00000ac8       __imp_DeleteFileA          000000014025fac8     kernel32:KERNEL32.dll
 0005:00000ad0       __imp_MoveFileA            000000014025fad0     kernel32:KERNEL32.dll
 0005:00000ad8       __imp_GetTickCount         000000014025fad8     kernel32:KERNEL32.dll
 0005:00000ae0       __imp_GetFileAttributesExA 000000014025fae0     kernel32:KERNEL32.dll
 0005:00000ae8       __imp_SetEndOfFile         000000014025fae8     kernel32:KERNEL32.dll
 0005:00000af0       __imp_SetFilePointer       000000014025faf0     kernel32:KERNEL32.dll
 0005:00000af8       __imp_GetFileAttributesA   000000014025faf8     kernel32:KERNEL32.dll
 0005:00000b00       __imp_GetFullPathNameA     000000014025fb00     kernel32:KERNEL32.dll
 0005:00000b08       __imp_ReadFile             000000014025fb08     kernel32:KERNEL32.dll
 0005:00000b10       __imp_WriteFile            000000014025fb10     kernel32:KERNEL32.dll
 0005:00000b18       __imp_UnmapViewOfFile      000000014025fb18     kernel32:KERNEL32.dll
 0005:00000b20       __imp_FindClose            000000014025fb20     kernel32:KERNEL32.dll
 0005:00000b28       __imp_FindNextFileA        000000014025fb28     kernel32:KERNEL32.dll
 0005:00000b30       __imp_FindFirstFileA       000000014025fb30     kernel32:KERNEL32.dll
 0005:00000b38       __imp_QueryPerformanceCounter 000000014025fb38     kernel32:KERNEL32.dll
 0005:00000b40       __imp_QueryPerformanceFrequency 000000014025fb40     kernel32:KERNEL32.dll
 0005:00000b48       __imp_FileTimeToSystemTime 000000014025fb48     kernel32:KERNEL32.dll
 0005:00000b50       __imp_FileTimeToLocalFileTime 000000014025fb50     kernel32:KERNEL32.dll
 0005:00000b58       __imp_GetDriveTypeA        000000014025fb58     kernel32:KERNEL32.dll
 0005:00000b60       __imp_ExitProcess          000000014025fb60     kernel32:KERNEL32.dll
 0005:00000b68       __imp_SetConsoleCtrlHandler 000000014025fb68     kernel32:KERNEL32.dll
 0005:00000b70       __imp_ReadConsoleInputA    000000014025fb70     kernel32:KERNEL32.dll
 0005:00000b78       __imp_SetConsoleMode       000000014025fb78     kernel32:KERNEL32.dll
 0005:00000b80       __imp_GetConsoleMode       000000014025fb80     kernel32:KERNEL32.dll
 0005:00000b88       __imp_PeekConsoleInputA    000000014025fb88     kernel32:KERNEL32.dll
 0005:00000b90       __imp_GetNumberOfConsoleInputEvents 000000014025fb90     kernel32:KERNEL32.dll
 0005:00000b98       __imp_GetCommandLineA      000000014025fb98     kernel32:KERNEL32.dll
 0005:00000ba0       __imp_HeapFree             000000014025fba0     kernel32:KERNEL32.dll
 0005:00000ba8       __imp_GetVersionExA        000000014025fba8     kernel32:KERNEL32.dll
 0005:00000bb0       __imp_HeapAlloc            000000014025fbb0     kernel32:KERNEL32.dll
 0005:00000bb8       __imp_GetProcessHeap       000000014025fbb8     kernel32:KERNEL32.dll
 0005:00000bc0       __imp_HeapReAlloc          000000014025fbc0     kernel32:KERNEL32.dll
 0005:00000bc8       __imp_GetFileInformationByHandle 000000014025fbc8     kernel32:KERNEL32.dll
 0005:00000bd0       __imp_PeekNamedPipe        000000014025fbd0     kernel32:KERNEL32.dll
 0005:00000bd8       __imp_GetFileType          000000014025fbd8     kernel32:KERNEL32.dll
 0005:00000be0       __imp_SetStdHandle         000000014025fbe0     kernel32:KERNEL32.dll
 0005:00000be8       __imp_ExitThread           000000014025fbe8     kernel32:KERNEL32.dll
 0005:00000bf0       __imp_ResumeThread         000000014025fbf0     kernel32:KERNEL32.dll
 0005:00000bf8       __imp_CreateThread         000000014025fbf8     kernel32:KERNEL32.dll
 0005:00000c00       __imp_WideCharToMultiByte  000000014025fc00     kernel32:KERNEL32.dll
 0005:00000c08       __imp_GetTimeZoneInformation 000000014025fc08     kernel32:KERNEL32.dll
 0005:00000c10       __imp_UnhandledExceptionFilter 000000014025fc10     kernel32:KERNEL32.dll
 0005:00000c18       __imp_SetUnhandledExceptionFilter 000000014025fc18     kernel32:KERNEL32.dll
 0005:00000c20       __imp_IsDebuggerPresent    000000014025fc20     kernel32:KERNEL32.dll
 0005:00000c28       __imp_RtlCaptureContext    000000014025fc28     kernel32:KERNEL32.dll
 0005:00000c30       __imp_GetStdHandle         000000014025fc30     kernel32:KERNEL32.dll
 0005:00000c38       __imp_FlsGetValue          000000014025fc38     kernel32:KERNEL32.dll
 0005:00000c40       __imp_TlsAlloc             000000014025fc40     kernel32:KERNEL32.dll
 0005:00000c48       __imp_FlsSetValue          000000014025fc48     kernel32:KERNEL32.dll
 0005:00000c50       __imp_TlsFree              000000014025fc50     kernel32:KERNEL32.dll
 0005:00000c58       __imp_FlsFree              000000014025fc58     kernel32:KERNEL32.dll
 0005:00000c60       __imp_TlsSetValue          000000014025fc60     kernel32:KERNEL32.dll
 0005:00000c68       __imp_GetCurrentThread     000000014025fc68     kernel32:KERNEL32.dll
 0005:00000c70       __imp_FlsAlloc             000000014025fc70     kernel32:KERNEL32.dll
 0005:00000c78       __imp_GetCurrentDirectoryA 000000014025fc78     kernel32:KERNEL32.dll
 0005:00000c80       __imp_SetCurrentDirectoryA 000000014025fc80     kernel32:KERNEL32.dll
 0005:00000c88       __imp_RtlVirtualUnwind     000000014025fc88     kernel32:KERNEL32.dll
 0005:00000c90       __imp_RtlLookupFunctionEntry 000000014025fc90     kernel32:KERNEL32.dll
 0005:00000c98       __imp_RaiseException       000000014025fc98     kernel32:KERNEL32.dll
 0005:00000ca0       __imp_RtlPcToFileHeader    000000014025fca0     kernel32:KERNEL32.dll
 0005:00000ca8       __imp_RtlUnwindEx          000000014025fca8     kernel32:KERNEL32.dll
 0005:00000cb0       __imp_SetHandleCount       000000014025fcb0     kernel32:KERNEL32.dll
 0005:00000cb8       __imp_GetStartupInfoA      000000014025fcb8     kernel32:KERNEL32.dll
 0005:00000cc0       __imp_FatalAppExitA        000000014025fcc0     kernel32:KERNEL32.dll
 0005:00000cc8       __imp_FreeLibrary          000000014025fcc8     kernel32:KERNEL32.dll
 0005:00000cd0       __imp_LoadLibraryA         000000014025fcd0     kernel32:KERNEL32.dll
 0005:00000cd8       __imp_CreatePipe           000000014025fcd8     kernel32:KERNEL32.dll
 0005:00000ce0       __imp_GetCPInfo            000000014025fce0     kernel32:KERNEL32.dll
 0005:00000ce8       __imp_GetACP               000000014025fce8     kernel32:KERNEL32.dll
 0005:00000cf0       __imp_GetOEMCP             000000014025fcf0     kernel32:KERNEL32.dll
 0005:00000cf8       __imp_IsValidCodePage      000000014025fcf8     kernel32:KERNEL32.dll
 0005:00000d00       __imp_FreeEnvironmentStringsA 000000014025fd00     kernel32:KERNEL32.dll
 0005:00000d08       __imp_GetEnvironmentStrings 000000014025fd08     kernel32:KERNEL32.dll
 0005:00000d10       __imp_FreeEnvironmentStringsW 000000014025fd10     kernel32:KERNEL32.dll
 0005:00000d18       __imp_GetEnvironmentStringsW 000000014025fd18     kernel32:KERNEL32.dll
 0005:00000d20       __imp_HeapSetInformation   000000014025fd20     kernel32:KERNEL32.dll
 0005:00000d28       __imp_HeapCreate           000000014025fd28     kernel32:KERNEL32.dll
 0005:00000d30       __imp_HeapDestroy          000000014025fd30     kernel32:KERNEL32.dll
 0005:00000d38       __imp_GetCurrentProcessId  000000014025fd38     kernel32:KERNEL32.dll
 0005:00000d40       __imp_InitializeCriticalSection 000000014025fd40     kernel32:KERNEL32.dll
 0005:00000d48       \177KERNEL32_NULL_THUNK_DATA 000000014025fd48     kernel32:KERNEL32.dll
 0005:00000e70       __imp_PeekMessageA         000000014025fe70     user32:USER32.dll
 0005:00000e78       __imp_KillTimer            000000014025fe78     user32:USER32.dll
 0005:00000e80       __imp_SetTimer             000000014025fe80     user32:USER32.dll
 0005:00000e88       \177USER32_NULL_THUNK_DATA 000000014025fe88     user32:USER32.dll
 0005:00000ee0       __imp_recv                 000000014025fee0     wsock32:WSOCK32.dll
 0005:00000ee8       __imp_gethostbyname        000000014025fee8     wsock32:WSOCK32.dll
 0005:00000ef0       __imp_inet_ntoa            000000014025fef0     wsock32:WSOCK32.dll
 0005:00000ef8       __imp_WSAStartup           000000014025fef8     wsock32:WSOCK32.dll
 0005:00000f00       __imp_WSACleanup           000000014025ff00     wsock32:WSOCK32.dll
 0005:00000f08       __imp_WSAGetLastError      000000014025ff08     wsock32:WSOCK32.dll
 0005:00000f10       __imp_connect              000000014025ff10     wsock32:WSOCK32.dll
 0005:00000f18       __imp_send                 000000014025ff18     wsock32:WSOCK32.dll
 0005:00000f20       __imp___WSAFDIsSet         000000014025ff20     wsock32:WSOCK32.dll
 0005:00000f28       __imp_accept               000000014025ff28     wsock32:WSOCK32.dll
 0005:00000f30       __imp_shutdown             000000014025ff30     wsock32:WSOCK32.dll
 0005:00000f38       __imp_socket               000000014025ff38     wsock32:WSOCK32.dll
 0005:00000f40       __imp_inet_addr            000000014025ff40     wsock32:WSOCK32.dll
 0005:00000f48       __imp_htonl                000000014025ff48     wsock32:WSOCK32.dll
 0005:00000f50       __imp_htons                000000014025ff50     wsock32:WSOCK32.dll
 0005:00000f58       __imp_ntohs                000000014025ff58     wsock32:WSOCK32.dll
 0005:00000f60       __imp_getpeername          000000014025ff60     wsock32:WSOCK32.dll
 0005:00000f68       __imp_WSASetLastError      000000014025ff68     wsock32:WSOCK32.dll
 0005:00000f70       __imp_select               000000014025ff70     wsock32:WSOCK32.dll
 0005:00000f78       __imp_setsockopt           000000014025ff78     wsock32:WSOCK32.dll
 0005:00000f80       __imp_bind                 000000014025ff80     wsock32:WSOCK32.dll
 0005:00000f88       __imp_listen               000000014025ff88     wsock32:WSOCK32.dll
 0005:00000f90       __imp_closesocket          000000014025ff90     wsock32:WSOCK32.dll
 0005:00000f98       __imp_ioctlsocket          000000014025ff98     wsock32:WSOCK32.dll
 0005:00000fa0       __imp_gethostname          000000014025ffa0     wsock32:WSOCK32.dll
 0005:00000fa8       \177WSOCK32_NULL_THUNK_DATA 000000014025ffa8     wsock32:WSOCK32.dll
 0006:00000000       _tls_start                 0000000140261000     LIBCMT:tlssup.obj
 0006:00000110       THR_KEY_mysys              0000000140261110     mysys:my_thr_init.obj
 0006:000002f6       _tls_end                   00000001402612f6     LIBCMT:tlssup.obj

 entry point at        0001:0005b840

